 MFCO42D

 Timestamp is 35887129 (Wed Jun 17 18:45:13 1998)

 Preferred load address is 5f500000

 Start         Length     Name                   Class
 0001:00000000 0004cc3aH .text                   CODE
 0001:0004cc40 0000004cH .text$AFX_CORE1         CODE
 0001:0004cc90 000055fbH .text$AFX_CORE4         CODE
 0001:00052290 0000278aH .text$AFX_INIT          CODE
 0001:00054a20 00010a91H .text$AFX_OLE1          CODE
 0001:000654c0 000092b5H .text$AFX_OLE2          CODE
 0001:0006e780 00007912H .text$AFX_OLE3          CODE
 0001:000760a0 0000d60bH .text$AFX_OLE4          CODE
 0001:000836b0 00003f01H .text$AFX_OLE5          CODE
 0001:000875c0 00000285H .text$AFX_TERM          CODE
 0001:00087850 00001103H .text$AFX_VDEL          CODE
 0001:00088960 0000463cH .text$x                 CODE
 0002:00000000 00001178H .idata$5                DATA
 0002:00001180 0000dc3cH .rdata                  DATA
 0002:0000edc0 00003dccH .rdata$r                DATA
 0002:00012b90 00009c08H .xdata$x                DATA
 0002:0001c798 000000e0H .didat$2                DATA
 0002:0001c878 00000020H .didat$3                DATA
 0002:0001c898 0000026cH .didat$4                DATA
 0002:0001cb04 0000074aH .didat$6                DATA
 0002:0001d250 0000026cH .didat$7                DATA
 0002:0001d4bc 00000064H .idata$2                DATA
 0002:0001d520 00000014H .idata$3                DATA
 0002:0001d534 00001178H .idata$4                DATA
 0002:0001e6ac 00000b30H .idata$6                DATA
 0002:0001f1e0 000032a8H .edata                  DATA
 0003:00000000 00000004H .CRT$XCA                DATA
 0003:00000004 0000000cH .CRT$XCL                DATA
 0003:00000010 00000028H .CRT$XCU                DATA
 0003:00000038 00000004H .CRT$XCZ                DATA
 0003:0000003c 00000004H .CRT$XIA                DATA
 0003:00000040 00000004H .CRT$XIZ                DATA
 0003:00000050 00002950H .data                   DATA
 0003:000029a0 0000026cH .didat$5                DATA
 0003:00002c10 0000147cH .bss                    DATA
 0004:00000000 00000448H .rsrc$01                DATA
 0004:00000450 000021d0H .rsrc$02                DATA

  Address         Publics by Value              Rva+Base     Lib:Object

 0001:00000000       __tcsncmp                  5f501000 f i oleinit.obj
 0001:00000020       __tcsinc                   5f501020 f i olecli1.obj
 0001:00000040       ?AtlA2WHelper@@YGPAGPAGPBDH@Z 5f501040 f i olecli1.obj
 0001:00000060       ?AtlA2WHelper@@YGPAGPAGPBDHI@Z 5f501060 f i olecli1.obj
 0001:000000f0       ?AtlW2AHelper@@YGPADPADPBGH@Z 5f5010f0 f i olecli1.obj
 0001:00000110       ?AtlW2AHelper@@YGPADPADPBGHI@Z 5f501110 f i olecli1.obj
 0001:000001a0       ??9@YAHABU_GUID@@0@Z       5f5011a0 f i oledisp1.obj
 0001:000001c0       __tcschr                   5f5011c0 f i oledlgs1.obj
 0001:000001e0       ??1CNoTrackObject@@UAE@XZ  5f5011e0 f i oledata.obj
 0001:00000200       ??_ECNoTrackObject@@UAEPAXI@Z 5f501200 f i oledata.obj
 0001:00000200       ??_GCNoTrackObject@@UAEPAXI@Z 5f501200 f i oledata.obj
 0001:00000230       ?AfxCheckError@@YGXJ@Z     5f501230 f   olevar.obj
 0001:00000256       ?_AfxCompareSafeArrays@@YGHPAUtagSAFEARRAY@@0@Z 5f501256 f   olevar.obj
 0001:000006a4       ?_AfxCreateOneDimArray@@YGXAAUtagVARIANT@@K@Z 5f5016a4 f   olevar.obj
 0001:000007d6       ?_AfxCopyBinaryData@@YGXPAUtagSAFEARRAY@@PBXK@Z 5f5017d6 f   olevar.obj
 0001:00000818       ??0COleVariant@@QAE@ABUtagVARIANT@@@Z 5f501818 f   olevar.obj
 0001:00000845       ??0COleVariant@@QAE@PBUtagVARIANT@@@Z 5f501845 f   olevar.obj
 0001:00000872       ??0COleVariant@@QAE@ABV0@@Z 5f501872 f   olevar.obj
 0001:0000089f       ??0COleVariant@@QAE@PBDG@Z 5f50189f f   olevar.obj
 0001:000009c1       ?SetString@COleVariant@@QAEXPBDG@Z 5f5019c1 f   olevar.obj
 0001:00000ae8       ??0COleVariant@@QAE@FG@Z   5f501ae8 f   olevar.obj
 0001:00000b79       ??0COleVariant@@QAE@JG@Z   5f501b79 f   olevar.obj
 0001:00000c36       ?_ClearCompat@COleVariant@@QAEXXZ 5f501c36 f   olevar.obj
 0001:00000c49       ?ChangeType@COleVariant@@QAEXGPAUtagVARIANT@@@Z 5f501c49 f   olevar.obj
 0001:00000c9a       ?Attach@COleVariant@@QAEXAAUtagVARIANT@@@Z 5f501c9a f   olevar.obj
 0001:00000cc9       ?Detach@COleVariant@@QAE?AUtagVARIANT@@XZ 5f501cc9 f   olevar.obj
 0001:00000d17       ??8COleVariant@@QBEHABUtagVARIANT@@@Z 5f501d17 f   olevar.obj
 0001:00000fd4       ??4COleVariant@@QAEABV0@ABUtagVARIANT@@@Z 5f501fd4 f   olevar.obj
 0001:00000ff8       ??4COleVariant@@QAEABV0@PBUtagVARIANT@@@Z 5f501ff8 f   olevar.obj
 0001:0000101c       ??4COleVariant@@QAEABV0@ABV0@@Z 5f50201c f   olevar.obj
 0001:00001040       ??4COleVariant@@QAEABV0@QBD@Z 5f502040 f   olevar.obj
 0001:000010fc       ??4COleVariant@@QAEABV0@ABVCString@@@Z 5f5020fc f   olevar.obj
 0001:000011ab       ??4COleVariant@@QAEABV0@E@Z 5f5021ab f   olevar.obj
 0001:000011e1       ??4COleVariant@@QAEABV0@F@Z 5f5021e1 f   olevar.obj
 0001:00001251       ??4COleVariant@@QAEABV0@J@Z 5f502251 f   olevar.obj
 0001:000012d3       ??4COleVariant@@QAEABV0@ABVCOleCurrency@@@Z 5f5022d3 f   olevar.obj
 0001:00001311       ??4COleVariant@@QAEABV0@M@Z 5f502311 f   olevar.obj
 0001:00001347       ??4COleVariant@@QAEABV0@N@Z 5f502347 f   olevar.obj
 0001:00001383       ??4COleVariant@@QAEABV0@ABVCOleDateTime@@@Z 5f502383 f   olevar.obj
 0001:000013c1       ??4COleVariant@@QAEABV0@ABVCByteArray@@@Z 5f5023c1 f   olevar.obj
 0001:00001404       ??4COleVariant@@QAEABV0@ABVCLongBinary@@@Z 5f502404 f   olevar.obj
 0001:0000145a       ?AfxVariantInit@@YGXPAUtagVARIANT@@@Z 5f50245a f   olevar.obj
 0001:00001471       ??6@YGAAVCDumpContext@@AAV0@VCOleVariant@@@Z 5f502471 f   olevar.obj
 0001:0000186c       ??6@YGAAVCArchive@@AAV0@VCOleVariant@@@Z 5f50286c f   olevar.obj
 0001:00001cd2       ??5@YGAAVCArchive@@AAV0@AAVCOleVariant@@@Z 5f502cd2 f   olevar.obj
 0001:000020c9       ?ConstructElements@@YGXPAVCOleVariant@@H@Z 5f5030c9 f   olevar.obj
 0001:0000218c       ?DestructElements@@YGXPAVCOleVariant@@H@Z 5f50318c f   olevar.obj
 0001:000021f6       ?CopyElements@@YGXPAVCOleVariant@@PBV1@H@Z 5f5031f6 f   olevar.obj
 0001:000022a1       ?SerializeElements@@YGXAAVCArchive@@PAVCOleVariant@@H@Z 5f5032a1 f   olevar.obj
 0001:0000235b       ?DumpElements@@YGXAAVCDumpContext@@PBVCOleVariant@@H@Z 5f50335b f   olevar.obj
 0001:000023a1       ?HashKey@@YGIABUtagVARIANT@@@Z 5f5033a1 f   olevar.obj
 0001:000024cc       ??0COleCurrency@@QAE@JJ@Z  5f5034cc f   olevar.obj
 0001:000024f6       ??4COleCurrency@@QAEABV0@TtagCY@@@Z 5f5034f6 f   olevar.obj
 0001:0000251e       ??4COleCurrency@@QAEABV0@ABV0@@Z 5f50351e f   olevar.obj
 0001:0000254a       ??4COleCurrency@@QAEABV0@ABUtagVARIANT@@@Z 5f50354a f   olevar.obj
 0001:00002662       ??MCOleCurrency@@QBEHABV0@@Z 5f503662 f   olevar.obj
 0001:000026fb       ??OCOleCurrency@@QBEHABV0@@Z 5f5036fb f   olevar.obj
 0001:00002794       ??NCOleCurrency@@QBEHABV0@@Z 5f503794 f   olevar.obj
 0001:0000282c       ??PCOleCurrency@@QBEHABV0@@Z 5f50382c f   olevar.obj
 0001:000028c4       ??HCOleCurrency@@QBE?AV0@ABV0@@Z 5f5038c4 f   olevar.obj
 0001:000029b8       ??GCOleCurrency@@QBE?AV0@ABV0@@Z 5f5039b8 f   olevar.obj
 0001:00002aac       ??GCOleCurrency@@QBE?AV0@XZ 5f503aac f   olevar.obj
 0001:00002b3b       ??DCOleCurrency@@QBE?AV0@J@Z 5f503b3b f   olevar.obj
 0001:00002e8e       ??KCOleCurrency@@QBE?AV0@J@Z 5f503e8e f   olevar.obj
 0001:000031f6       ?SetCurrency@COleCurrency@@QAEXJJ@Z 5f5041f6 f   olevar.obj
 0001:000032a6       ?ParseCurrency@COleCurrency@@QAEHPBDKK@Z 5f5042a6 f   olevar.obj
 0001:0000344c       ?Format@COleCurrency@@QBE?AVCString@@KK@Z 5f50444c f   olevar.obj
 0001:000035f9       ??6@YGAAVCDumpContext@@AAV0@VCOleCurrency@@@Z 5f5045f9 f   olevar.obj
 0001:00003695       ??6@YGAAVCArchive@@AAV0@VCOleCurrency@@@Z 5f504695 f   olevar.obj
 0001:000036c0       ??5@YGAAVCArchive@@AAV0@AAVCOleCurrency@@@Z 5f5046c0 f   olevar.obj
 0001:000036f1       ?_AfxOleDateFromTm@@YGHGGGGGGAAN@Z 5f5046f1 f   olevar.obj
 0001:0000390c       ?_AfxTmFromOleDate@@YGHNAAUtm@@@Z 5f50490c f   olevar.obj
 0001:00003bf9       ?_AfxTmConvertToStandardFormat@@YGXAAUtm@@@Z 5f504bf9 f   olevar.obj
 0001:00003c3f       ?_AfxDoubleFromDate@@YGNN@Z 5f504c3f f   olevar.obj
 0001:00003c7d       ?_AfxDateFromDouble@@YGNN@Z 5f504c7d f   olevar.obj
 0001:00003cb8       ?GetTickCount@COleDateTime@@SG?AV1@XZ 5f504cb8 f   olevar.obj
 0001:00003ce4       ?GetAsSystemTime@COleDateTime@@QBEHAAU_SYSTEMTIME@@@Z 5f504ce4 f   olevar.obj
 0001:00003d7e       ?GetYear@COleDateTime@@QBEHXZ 5f504d7e f   olevar.obj
 0001:00003db6       ?GetMonth@COleDateTime@@QBEHXZ 5f504db6 f   olevar.obj
 0001:00003dee       ?GetDay@COleDateTime@@QBEHXZ 5f504dee f   olevar.obj
 0001:00003e26       ?GetHour@COleDateTime@@QBEHXZ 5f504e26 f   olevar.obj
 0001:00003e5e       ?GetMinute@COleDateTime@@QBEHXZ 5f504e5e f   olevar.obj
 0001:00003e96       ?GetSecond@COleDateTime@@QBEHXZ 5f504e96 f   olevar.obj
 0001:00003ece       ?GetDayOfWeek@COleDateTime@@QBEHXZ 5f504ece f   olevar.obj
 0001:00003f06       ?GetDayOfYear@COleDateTime@@QBEHXZ 5f504f06 f   olevar.obj
 0001:00003f3e       ??4COleDateTime@@QAEABV0@ABUtagVARIANT@@@Z 5f504f3e f   olevar.obj
 0001:00004053       ??4COleDateTime@@QAEABV0@N@Z 5f505053 f   olevar.obj
 0001:0000407b       ??4COleDateTime@@QAEABV0@ABJ@Z 5f50507b f   olevar.obj
 0001:00004122       ??4COleDateTime@@QAEABV0@ABU_SYSTEMTIME@@@Z 5f505122 f   olevar.obj
 0001:00004175       ??4COleDateTime@@QAEABV0@ABU_FILETIME@@@Z 5f505175 f   olevar.obj
 0001:00004216       ??MCOleDateTime@@QBEHABV0@@Z 5f505216 f   olevar.obj
 0001:000042b5       ??OCOleDateTime@@QBEHABV0@@Z 5f5052b5 f   olevar.obj
 0001:00004354       ??NCOleDateTime@@QBEHABV0@@Z 5f505354 f   olevar.obj
 0001:000043f3       ??PCOleDateTime@@QBEHABV0@@Z 5f5053f3 f   olevar.obj
 0001:00004492       ??HCOleDateTime@@QBE?AV0@ABVCOleDateTimeSpan@@@Z 5f505492 f   olevar.obj
 0001:00004557       ??GCOleDateTime@@QBE?AV0@ABVCOleDateTimeSpan@@@Z 5f505557 f   olevar.obj
 0001:0000461c       ??GCOleDateTime@@QBE?AVCOleDateTimeSpan@@ABV0@@Z 5f50561c f   olevar.obj
 0001:000046d2       ?SetDateTime@COleDateTime@@QAEHHHHHHH@Z 5f5056d2 f   olevar.obj
 0001:00004717       ?ParseDateTime@COleDateTime@@QAEHPBDKK@Z 5f505717 f   olevar.obj
 0001:000048b7       ?Format@COleDateTime@@QBE?AVCString@@KK@Z 5f5058b7 f   olevar.obj
 0001:00004a64       ?Format@COleDateTime@@QBE?AVCString@@PBD@Z 5f505a64 f   olevar.obj
 0001:00004bbe       ?Format@COleDateTime@@QBE?AVCString@@I@Z 5f505bbe f   olevar.obj
 0001:00004c5e       ?CheckRange@COleDateTime@@IAEXXZ 5f505c5e f   olevar.obj
 0001:00004c97       ??6@YGAAVCDumpContext@@AAV0@VCOleDateTime@@@Z 5f505c97 f   olevar.obj
 0001:00004d33       ??6@YGAAVCArchive@@AAV0@VCOleDateTime@@@Z 5f505d33 f   olevar.obj
 0001:00004d56       ??5@YGAAVCArchive@@AAV0@AAVCOleDateTime@@@Z 5f505d56 f   olevar.obj
 0001:00004d78       ?GetHours@COleDateTimeSpan@@QBEJXZ 5f505d78 f   olevar.obj
 0001:00004df1       ?GetMinutes@COleDateTimeSpan@@QBEJXZ 5f505df1 f   olevar.obj
 0001:00004e71       ?GetSeconds@COleDateTimeSpan@@QBEJXZ 5f505e71 f   olevar.obj
 0001:00004ef7       ??4COleDateTimeSpan@@QAEABV0@N@Z 5f505ef7 f   olevar.obj
 0001:00004f1f       ??4COleDateTimeSpan@@QAEABV0@ABV0@@Z 5f505f1f f   olevar.obj
 0001:00004f4b       ??HCOleDateTimeSpan@@QBE?AV0@ABV0@@Z 5f505f4b f   olevar.obj
 0001:00004ff0       ??GCOleDateTimeSpan@@QBE?AV0@ABV0@@Z 5f505ff0 f   olevar.obj
 0001:00005095       ?SetDateTimeSpan@COleDateTimeSpan@@QAEXJHHH@Z 5f506095 f   olevar.obj
 0001:000050d5       ?Format@COleDateTimeSpan@@QBE?AVCString@@PBD@Z 5f5060d5 f   olevar.obj
 0001:00005362       ?Format@COleDateTimeSpan@@QBE?AVCString@@I@Z 5f506362 f   olevar.obj
 0001:00005402       ?CheckRange@COleDateTimeSpan@@QAEXXZ 5f506402 f   olevar.obj
 0001:0000543b       ??6@YGAAVCDumpContext@@AAV0@VCOleDateTimeSpan@@@Z 5f50643b f   olevar.obj
 0001:000054db       ??6@YGAAVCArchive@@AAV0@VCOleDateTimeSpan@@@Z 5f5064db f   olevar.obj
 0001:000054fe       ??5@YGAAVCArchive@@AAV0@AAVCOleDateTimeSpan@@@Z 5f5064fe f   olevar.obj
 0001:00005520       ??0COleSafeArray@@QAE@ABUtagSAFEARRAY@@G@Z 5f506520 f   olevar.obj
 0001:0000557e       ??0COleSafeArray@@QAE@PBUtagSAFEARRAY@@G@Z 5f50657e f   olevar.obj
 0001:000055dc       ??0COleSafeArray@@QAE@ABV0@@Z 5f5065dc f   olevar.obj
 0001:0000561d       ??0COleSafeArray@@QAE@ABUtagVARIANT@@@Z 5f50661d f   olevar.obj
 0001:0000565e       ??0COleSafeArray@@QAE@PBUtagVARIANT@@@Z 5f50665e f   olevar.obj
 0001:0000569f       ?Attach@COleSafeArray@@QAEXAAUtagVARIANT@@@Z 5f50669f f   olevar.obj
 0001:00005700       ?Detach@COleSafeArray@@QAE?AUtagVARIANT@@XZ 5f506700 f   olevar.obj
 0001:0000574e       ??4COleSafeArray@@QAEAAV0@ABV0@@Z 5f50674e f   olevar.obj
 0001:000057a4       ??4COleSafeArray@@QAEAAV0@ABUtagVARIANT@@@Z 5f5067a4 f   olevar.obj
 0001:000057fa       ??4COleSafeArray@@QAEAAV0@PBUtagVARIANT@@@Z 5f5067fa f   olevar.obj
 0001:00005850       ??4COleSafeArray@@QAEAAV0@ABVCOleVariant@@@Z 5f506850 f   olevar.obj
 0001:000058a6       ??8COleSafeArray@@QBEHABUtagSAFEARRAY@@@Z 5f5068a6 f   olevar.obj
 0001:000058c3       ??8COleSafeArray@@QBEHPBUtagSAFEARRAY@@@Z 5f5068c3 f   olevar.obj
 0001:000058e0       ??8COleSafeArray@@QBEHABV0@@Z 5f5068e0 f   olevar.obj
 0001:00005918       ??8COleSafeArray@@QBEHABUtagVARIANT@@@Z 5f506918 f   olevar.obj
 0001:00005950       ??8COleSafeArray@@QBEHPBUtagVARIANT@@@Z 5f506950 f   olevar.obj
 0001:00005988       ??8COleSafeArray@@QBEHABVCOleVariant@@@Z 5f506988 f   olevar.obj
 0001:000059c0       ?_AfxDumpSafeArrayElement@@YAXAAVCDumpContext@@AAVCOleSafeArray@@PAJ@Z 5f5069c0 f   olevar.obj
 0001:00005c7b       ??6@YGAAVCDumpContext@@AAV0@AAVCOleSafeArray@@@Z 5f506c7b f   olevar.obj
 0001:00005eed       ?CreateOneDim@COleSafeArray@@QAEXGKPBXJ@Z 5f506eed f   olevar.obj
 0001:00005f78       ?GetOneDimSize@COleSafeArray@@QAEKXZ 5f506f78 f   olevar.obj
 0001:00005fd7       ?ResizeOneDim@COleSafeArray@@QAEXK@Z 5f506fd7 f   olevar.obj
 0001:0000602c       ?Create@COleSafeArray@@QAEXGKPAK@Z 5f50702c f   olevar.obj
 0001:00006157       ?Create@COleSafeArray@@QAEXGKPAUtagSAFEARRAYBOUND@@@Z 5f507157 f   olevar.obj
 0001:000062d5       ?AccessData@COleSafeArray@@QAEXPAPAX@Z 5f5072d5 f   olevar.obj
 0001:000062f9       ?UnaccessData@COleSafeArray@@QAEXXZ 5f5072f9 f   olevar.obj
 0001:00006317       ?AllocData@COleSafeArray@@QAEXXZ 5f507317 f   olevar.obj
 0001:00006335       ?AllocDescriptor@COleSafeArray@@QAEXK@Z 5f507335 f   olevar.obj
 0001:00006359       ?Copy@COleSafeArray@@QAEXPAPAUtagSAFEARRAY@@@Z 5f507359 f   olevar.obj
 0001:0000637d       ?GetLBound@COleSafeArray@@QAEXKPAJ@Z 5f50737d f   olevar.obj
 0001:000063a5       ?GetUBound@COleSafeArray@@QAEXKPAJ@Z 5f5073a5 f   olevar.obj
 0001:000063cd       ?GetElement@COleSafeArray@@QAEXPAJPAX@Z 5f5073cd f   olevar.obj
 0001:000063f5       ?PtrOfIndex@COleSafeArray@@QAEXPAJPAPAX@Z 5f5073f5 f   olevar.obj
 0001:0000641d       ?PutElement@COleSafeArray@@QAEXPAJPAX@Z 5f50741d f   olevar.obj
 0001:00006445       ?Redim@COleSafeArray@@QAEXPAUtagSAFEARRAYBOUND@@@Z 5f507445 f   olevar.obj
 0001:00006469       ?Lock@COleSafeArray@@QAEXXZ 5f507469 f   olevar.obj
 0001:00006487       ?Unlock@COleSafeArray@@QAEXXZ 5f507487 f   olevar.obj
 0001:000064a5       ?Destroy@COleSafeArray@@QAEXXZ 5f5074a5 f   olevar.obj
 0001:000064c3       ?DestroyData@COleSafeArray@@QAEXXZ 5f5074c3 f   olevar.obj
 0001:000064e1       ?DestroyDescriptor@COleSafeArray@@QAEXXZ 5f5074e1 f   olevar.obj
 0001:000064ff       ?AfxSafeArrayInit@@YGXPAVCOleSafeArray@@@Z 5f5074ff f   olevar.obj
 0001:00006516       ?DDX_Text@@YGXPAVCDataExchange@@HAAVCOleDateTime@@@Z 5f507516 f   olevar.obj
 0001:0000661e       ?DDX_Text@@YGXPAVCDataExchange@@HAAVCOleCurrency@@@Z 5f50761e f   olevar.obj
 0001:00006730       ??_GCOleVariant@@QAEPAXI@Z 5f507730 f i olevar.obj
 0001:00006760       ?HashKey@@YGIK@Z           5f507760 f i olevar.obj
 0001:00006770       ??2@YAPAXIPAX@Z            5f507770 f i olevar.obj
 0001:00006780       ??3@YAXPAX0@Z              5f507780 f i olevar.obj
 0001:00006790       ??0COleVariant@@QAE@PBU_ITEMIDLIST@@@Z 5f507790 f   olevar1.obj
 0001:00006840       ??0AFX_CLASSINIT@@QAE@PAUCRuntimeClass@@@Z 5f507840 f i oledoc1.obj
 0001:00006860       ??_9@$BBAI@AE              5f507860 f i oleipfrm.obj
 0001:00006870       ??0CPushRoutingFrame@@QAE@PAVCFrameWnd@@@Z 5f507870 f i oleipfrm.obj
 0001:000068b0       ??1CPushRoutingFrame@@QAE@XZ 5f5078b0 f i oleipfrm.obj
 0001:000068d0       ?ocslen@@YAIPBG@Z          5f5078d0 f i olemisc.obj
 0001:000068e0       ?ocscpy@@YAPAGPAGPBG@Z     5f5078e0 f i olemisc.obj
 0001:00006910       ?AtlDevModeA2W@@YAPAU_devicemodeW@@PAU1@PAU_devicemodeA@@@Z 5f507910 f i olemisc.obj
 0001:00006a20       ?AtlDevModeW2A@@YGPAU_devicemodeA@@PAU1@PAU_devicemodeW@@@Z 5f507a20 f i olemisc.obj
 0001:00006b30       ?_GetBaseInterfaceMap@CEnumOleVerb@@KGPBUAFX_INTERFACEMAP@@XZ 5f507b30 f   oleverb.obj
 0001:00006b3a       ?GetInterfaceMap@CEnumOleVerb@@MBEPBUAFX_INTERFACEMAP@@XZ 5f507b3a f   oleverb.obj
 0001:00006b4a       ??1CEnumOleVerb@@UAE@XZ    5f507b4a f   oleverb.obj
 0001:00006bad       ?OnNext@CEnumOleVerb@@MAEHPAX@Z 5f507bad f   oleverb.obj
 0001:00006c04       ?EnumOleVerbs@CCmdTarget@@QAEHPAPAUIEnumOLEVERB@@@Z 5f507c04 f   oleverb.obj
 0001:00006e68       ?DoOleVerb@CCmdTarget@@QAEHJPAUtagMSG@@PAUHWND__@@PBUtagRECT@@@Z 5f507e68 f   oleverb.obj
 0001:00006ff0       ??_GCEnumOleVerb@@UAEPAXI@Z 5f507ff0 f i oleverb.obj
 0001:00006ff0       ??_ECEnumOleVerb@@UAEPAXI@Z 5f507ff0 f i oleverb.obj
 0001:00007020       ??0CEnumOleVerb@@QAE@PBXI@Z 5f508020 f i oleverb.obj
 0001:00007050       ?T2CA@@YAPBDPBD@Z          5f508050 f i viewrich.obj
 0001:00007050       ?T2A@@YAPADPAD@Z           5f508050 f i viewrich.obj
 0001:00007060       ?EnableTypeLib@CCmdTarget@@QAEXXZ 5f508060 f   oletyplb.obj
 0001:000070ba       ?GetTypeInfoOfGuid@CCmdTarget@@QAEJKABU_GUID@@PAPAUITypeInfo@@@Z 5f5080ba f   oletyplb.obj
 0001:000072ab       ?AfxGetTypeLibCache@@YGPAVCTypeLibCache@@PBU_GUID@@@Z 5f5082ab f   oletyplb.obj
 0001:000074ae       ?Lock@CTypeLibCache@@QAEXXZ 5f5084ae f   oletyplb.obj
 0001:00007502       ?Lookup@CTypeLibCache@@QAEHKPAPAUITypeLib@@@Z 5f508502 f   oletyplb.obj
 0001:0000757b       ?Cache@CTypeLibCache@@QAEXKPAUITypeLib@@@Z 5f50857b f   oletyplb.obj
 0001:00007633       ?LookupTypeInfo@CTypeLibCache@@QAEHKABU_GUID@@PAPAUITypeInfo@@@Z 5f508633 f   oletyplb.obj
 0001:000076fb       ?CacheTypeInfo@CTypeLibCache@@QAEXKABU_GUID@@PAUITypeInfo@@@Z 5f5086fb f   oletyplb.obj
 0001:00007780       ??0CTypeLibCacheMap@@QAE@XZ 5f508780 f i oletyplb.obj
 0001:000077b0       ??_ECTypeLibCacheMap@@UAEPAXI@Z 5f5087b0 f i oletyplb.obj
 0001:000077b0       ??_GCTypeLibCacheMap@@UAEPAXI@Z 5f5087b0 f i oletyplb.obj
 0001:000077e0       ??1CTypeLibCacheMap@@UAE@XZ 5f5087e0 f i oletyplb.obj
 0001:00007800       ??0CTypeLibCache@@QAE@XZ   5f508800 f i oletyplb.obj
 0001:00007840       ?IsEqualGUID@@YAHABU_GUID@@0@Z 5f508840 f i oletyplb.obj
 0001:00007840       ??8@YAHABU_GUID@@0@Z       5f508840 f i oletyplb.obj
 0001:00007860       ?Create@CDateTimeCtrl@@QAEHKABUtagRECT@@PAVCWnd@@I@Z 5f508860 f   winctrl5.obj
 0001:000078c4       ?GetRange@CDateTimeCtrl@@QBEKPAVCTime@@0@Z 5f5088c4 f   winctrl5.obj
 0001:0000797d       ?GetRange@CDateTimeCtrl@@QBEKPAVCOleDateTime@@0@Z 5f50897d f   winctrl5.obj
 0001:00007a4a       ?SetRange@CDateTimeCtrl@@QAEHPBVCTime@@0@Z 5f508a4a f   winctrl5.obj
 0001:00007ae5       ?SetRange@CDateTimeCtrl@@QAEHPBVCOleDateTime@@0@Z 5f508ae5 f   winctrl5.obj
 0001:00007bee       ?SetTime@CDateTimeCtrl@@QAEHPAU_SYSTEMTIME@@@Z 5f508bee f   winctrl5.obj
 0001:00007c54       ?SetTime@CDateTimeCtrl@@QAEHABVCOleDateTime@@@Z 5f508c54 f   winctrl5.obj
 0001:00007d0c       ?SetTime@CDateTimeCtrl@@QAEHPBVCTime@@@Z 5f508d0c f   winctrl5.obj
 0001:00007d97       ?GetTime@CDateTimeCtrl@@QBEHAAVCOleDateTime@@@Z 5f508d97 f   winctrl5.obj
 0001:00007e3e       ?GetTime@CDateTimeCtrl@@QBEKAAVCTime@@@Z 5f508e3e f   winctrl5.obj
 0001:00007e88       ??1CDateTimeCtrl@@UAE@XZ   5f508e88 f   winctrl5.obj
 0001:00007ed9       ?Create@CMonthCalCtrl@@QAEHKABUtagRECT@@PAVCWnd@@I@Z 5f508ed9 f   winctrl5.obj
 0001:00007f40       ?Create@CMonthCalCtrl@@QAEHKABUtagPOINT@@PAVCWnd@@I@Z 5f508f40 f   winctrl5.obj
 0001:00007fd7       ?SizeMinReq@CMonthCalCtrl@@QAEHH@Z 5f508fd7 f   winctrl5.obj
 0001:0000804d       ?SetToday@CMonthCalCtrl@@QAEXABVCOleDateTime@@@Z 5f50904d f   winctrl5.obj
 0001:0000811d       ?SetToday@CMonthCalCtrl@@QAEXPBVCTime@@@Z 5f50911d f   winctrl5.obj
 0001:000081cc       ?SetCurSel@CMonthCalCtrl@@QAEHABVCOleDateTime@@@Z 5f5091cc f   winctrl5.obj
 0001:0000824d       ?SetCurSel@CMonthCalCtrl@@QAEHABVCTime@@@Z 5f50924d f   winctrl5.obj
 0001:000082c2       ?GetCurSel@CMonthCalCtrl@@QBEHAAVCOleDateTime@@@Z 5f5092c2 f   winctrl5.obj
 0001:00008364       ?GetToday@CMonthCalCtrl@@QBEHAAVCOleDateTime@@@Z 5f509364 f   winctrl5.obj
 0001:00008406       ?GetCurSel@CMonthCalCtrl@@QBEHAAVCTime@@@Z 5f509406 f   winctrl5.obj
 0001:000084aa       ?GetToday@CMonthCalCtrl@@QBEHAAVCTime@@@Z 5f5094aa f   winctrl5.obj
 0001:0000854e       ??1CMonthCalCtrl@@UAE@XZ   5f50954e f   winctrl5.obj
 0001:0000859f       ?GetFirstDayOfWeek@CMonthCalCtrl@@QBEHPAH@Z 5f50959f f   winctrl5.obj
 0001:0000861d       ?SetFirstDayOfWeek@CMonthCalCtrl@@QAEHHPAH@Z 5f50961d f   winctrl5.obj
 0001:0000869b       ?SetDayState@CMonthCalCtrl@@QAEHHPAK@Z 5f50969b f   winctrl5.obj
 0001:00008723       ?SetRange@CMonthCalCtrl@@QAEHPBVCOleDateTime@@0@Z 5f509723 f   winctrl5.obj
 0001:00008835       ?SetRange@CMonthCalCtrl@@QAEHQAU_SYSTEMTIME@@0@Z 5f509835 f   winctrl5.obj
 0001:000088d8       ?GetRange@CMonthCalCtrl@@QBEKPAVCOleDateTime@@0@Z 5f5098d8 f   winctrl5.obj
 0001:00008990       ?GetRange@CMonthCalCtrl@@QBEKPAU_SYSTEMTIME@@0@Z 5f509990 f   winctrl5.obj
 0001:00008a42       ?SetRange@CMonthCalCtrl@@QAEHPBVCTime@@0@Z 5f509a42 f   winctrl5.obj
 0001:00008ae0       ?GetRange@CMonthCalCtrl@@QBEKPAVCTime@@0@Z 5f509ae0 f   winctrl5.obj
 0001:00008b9c       ?GetMonthRange@CMonthCalCtrl@@QBEHAAVCOleDateTime@@0K@Z 5f509b9c f   winctrl5.obj
 0001:00008c5c       ?GetMonthRange@CMonthCalCtrl@@QBEHPAU_SYSTEMTIME@@0K@Z 5f509c5c f   winctrl5.obj
 0001:00008d42       ?GetMonthRange@CMonthCalCtrl@@QBEHAAVCTime@@0K@Z 5f509d42 f   winctrl5.obj
 0001:00008e06       ?GetSelRange@CMonthCalCtrl@@QBEHPAU_SYSTEMTIME@@0@Z 5f509e06 f   winctrl5.obj
 0001:00008f11       ?SetSelRange@CMonthCalCtrl@@QAEHQAU_SYSTEMTIME@@0@Z 5f509f11 f   winctrl5.obj
 0001:00009010       ?SetSelRange@CMonthCalCtrl@@QAEHABVCOleDateTime@@0@Z 5f50a010 f   winctrl5.obj
 0001:000090d6       ?GetSelRange@CMonthCalCtrl@@QBEHAAVCOleDateTime@@0@Z 5f50a0d6 f   winctrl5.obj
 0001:0000919d       ?SetSelRange@CMonthCalCtrl@@QAEHABVCTime@@0@Z 5f50a19d f   winctrl5.obj
 0001:0000924b       ?GetSelRange@CMonthCalCtrl@@QBEHAAVCTime@@0@Z 5f50a24b f   winctrl5.obj
 0001:00009316       ?DDX_DateTimeCtrl@@YGXPAVCDataExchange@@HAAVCOleDateTime@@@Z 5f50a316 f   winctrl5.obj
 0001:0000935f       ?DDX_DateTimeCtrl@@YGXPAVCDataExchange@@HAAVCTime@@@Z 5f50a35f f   winctrl5.obj
 0001:000093a8       ?DDX_MonthCalCtrl@@YGXPAVCDataExchange@@HAAVCOleDateTime@@@Z 5f50a3a8 f   winctrl5.obj
 0001:000093f1       ?DDX_MonthCalCtrl@@YGXPAVCDataExchange@@HAAVCTime@@@Z 5f50a3f1 f   winctrl5.obj
 0001:0000943a       ?DDV_MinMaxDateTime@@YGXPAVCDataExchange@@AAVCTime@@PBV2@2@Z 5f50a43a f   winctrl5.obj
 0001:00009512       ?DDV_MinMaxDateTime@@YGXPAVCDataExchange@@AAVCOleDateTime@@PBV2@2@Z 5f50a512 f   winctrl5.obj
 0001:000095d2       ?DDV_MinMaxMonth@@YGXPAVCDataExchange@@AAVCTime@@PBV2@2@Z 5f50a5d2 f   winctrl5.obj
 0001:000096aa       ?DDV_MinMaxMonth@@YGXPAVCDataExchange@@AAVCOleDateTime@@PBV2@2@Z 5f50a6aa f   winctrl5.obj
 0001:0000976a       ??0CDateTimeCtrl@@QAE@XZ   5f50a76a f   winctrl5.obj
 0001:00009789       ?GetMonthCalFont@CDateTimeCtrl@@QBEPAVCFont@@XZ 5f50a789 f   winctrl5.obj
 0001:000097de       ?GetMonthCalCtrl@CDateTimeCtrl@@QBEPAVCMonthCalCtrl@@XZ 5f50a7de f   winctrl5.obj
 0001:00009833       ?SetMonthCalFont@CDateTimeCtrl@@QAEXPAUHFONT__@@H@Z 5f50a833 f   winctrl5.obj
 0001:0000988d       ?SetMonthCalColor@CDateTimeCtrl@@QAEKHK@Z 5f50a88d f   winctrl5.obj
 0001:000098e2       ?GetTime@CDateTimeCtrl@@QBEKPAU_SYSTEMTIME@@@Z 5f50a8e2 f   winctrl5.obj
 0001:00009952       ?GetMonthCalColor@CDateTimeCtrl@@QBEKH@Z 5f50a952 f   winctrl5.obj
 0001:000099a5       ?SetFormat@CDateTimeCtrl@@QAEHPBD@Z 5f50a9a5 f   winctrl5.obj
 0001:000099f8       ??0CMonthCalCtrl@@QAE@XZ   5f50a9f8 f   winctrl5.obj
 0001:00009a17       ?HitTest@CMonthCalCtrl@@QAEKPAUMCHITTESTINFO@@@Z 5f50aa17 f   winctrl5.obj
 0001:00009a6a       ?GetMinReqRect@CMonthCalCtrl@@QBEHPAUtagRECT@@@Z 5f50aa6a f   winctrl5.obj
 0001:00009ab5       ?SetMonthDelta@CMonthCalCtrl@@QAEHH@Z 5f50aab5 f   winctrl5.obj
 0001:00009b00       ?GetMonthDelta@CMonthCalCtrl@@QBEHXZ 5f50ab00 f   winctrl5.obj
 0001:00009b47       ?GetColor@CMonthCalCtrl@@QBEKH@Z 5f50ab47 f   winctrl5.obj
 0001:00009b92       ?SetColor@CMonthCalCtrl@@QAEKHK@Z 5f50ab92 f   winctrl5.obj
 0001:00009bdf       ?SetMaxSelCount@CMonthCalCtrl@@QAEHH@Z 5f50abdf f   winctrl5.obj
 0001:00009c2a       ?GetMaxSelCount@CMonthCalCtrl@@QBEHXZ 5f50ac2a f   winctrl5.obj
 0001:00009c71       ?SetToday@CMonthCalCtrl@@QAEXQAU_SYSTEMTIME@@@Z 5f50ac71 f   winctrl5.obj
 0001:00009cbc       ?GetToday@CMonthCalCtrl@@QBEHPAU_SYSTEMTIME@@@Z 5f50acbc f   winctrl5.obj
 0001:00009d07       ?SetCurSel@CMonthCalCtrl@@QAEHQAU_SYSTEMTIME@@@Z 5f50ad07 f   winctrl5.obj
 0001:00009d52       ?GetCurSel@CMonthCalCtrl@@QBEHPAU_SYSTEMTIME@@@Z 5f50ad52 f   winctrl5.obj
 0001:00009da0       ??_GCDateTimeCtrl@@UAEPAXI@Z 5f50ada0 f i winctrl5.obj
 0001:00009da0       ??_ECDateTimeCtrl@@UAEPAXI@Z 5f50ada0 f i winctrl5.obj
 0001:00009dd0       ??_ECMonthCalCtrl@@UAEPAXI@Z 5f50add0 f i winctrl5.obj
 0001:00009dd0       ??_GCMonthCalCtrl@@UAEPAXI@Z 5f50add0 f i winctrl5.obj
 0001:00009e00       ?_GetBaseMessageMap@CHtmlView@@KGPBUAFX_MSGMAP@@XZ 5f50ae00 f   viewhtml.obj
 0001:00009e0a       ?GetMessageMap@CHtmlView@@MBEPBUAFX_MSGMAP@@XZ 5f50ae0a f   viewhtml.obj
 0001:00009e1a       ?_GetBaseEventSinkMap@CHtmlView@@KGPBUAFX_EVENTSINKMAP@@XZ 5f50ae1a f   viewhtml.obj
 0001:00009e24       ?GetEventSinkMap@CHtmlView@@MBEPBUAFX_EVENTSINKMAP@@XZ 5f50ae24 f   viewhtml.obj
 0001:00009e34       ??0CHtmlView@@IAE@XZ       5f50ae34 f   viewhtml.obj
 0001:00009e9d       ??1CHtmlView@@UAE@XZ       5f50ae9d f   viewhtml.obj
 0001:00009f1c       ?OnDraw@CHtmlView@@UAEXPAVCDC@@@Z 5f50af1c f   viewhtml.obj
 0001:00009f4f       ?OnFilePrint@CHtmlView@@QAEXXZ 5f50af4f f   viewhtml.obj
 0001:00009fc6       ?AssertValid@CHtmlView@@UBEXXZ 5f50afc6 f   viewhtml.obj
 0001:00009fd9       ?Dump@CHtmlView@@UBEXAAVCDumpContext@@@Z 5f50afd9 f   viewhtml.obj
 0001:00009ff2       ?OnDestroy@CHtmlView@@IAEXXZ 5f50aff2 f   viewhtml.obj
 0001:0000a034       ?OnSize@CHtmlView@@IAEXIHH@Z 5f50b034 f   viewhtml.obj
 0001:0000a0d5       ?OnPaint@CHtmlView@@IAEXXZ 5f50b0d5 f   viewhtml.obj
 0001:0000a0e8       ?Create@CHtmlView@@UAEHPBD0KABUtagRECT@@PAVCWnd@@IPAUCCreateContext@@@Z 5f50b0e8 f   viewhtml.obj
 0001:0000a1f0       ?GetType@CHtmlView@@QBE?AVCString@@XZ 5f50b1f0 f   viewhtml.obj
 0001:0000a2a4       ?GetLeft@CHtmlView@@QBEJXZ 5f50b2a4 f   viewhtml.obj
 0001:0000a2fc       ?GetTop@CHtmlView@@QBEJXZ  5f50b2fc f   viewhtml.obj
 0001:0000a354       ?GetToolBar@CHtmlView@@QBEHXZ 5f50b354 f   viewhtml.obj
 0001:0000a3af       ?GetHeight@CHtmlView@@QBEJXZ 5f50b3af f   viewhtml.obj
 0001:0000a407       ?GetVisible@CHtmlView@@QBEHXZ 5f50b407 f   viewhtml.obj
 0001:0000a463       ?GetLocationName@CHtmlView@@QBE?AVCString@@XZ 5f50b463 f   viewhtml.obj
 0001:0000a517       ?GetLocationURL@CHtmlView@@QBE?AVCString@@XZ 5f50b517 f   viewhtml.obj
 0001:0000a5cb       ?GetBusy@CHtmlView@@QBEHXZ 5f50b5cb f   viewhtml.obj
 0001:0000a624       ?GetReadyState@CHtmlView@@QBE?AW4tagREADYSTATE@@XZ 5f50b624 f   viewhtml.obj
 0001:0000a67f       ?GetOffline@CHtmlView@@QBEHXZ 5f50b67f f   viewhtml.obj
 0001:0000a6db       ?GetSilent@CHtmlView@@QBEHXZ 5f50b6db f   viewhtml.obj
 0001:0000a737       ?GetApplication@CHtmlView@@QBEPAUIDispatch@@XZ 5f50b737 f   viewhtml.obj
 0001:0000a78f       ?GetParentBrowser@CHtmlView@@QBEPAUIDispatch@@XZ 5f50b78f f   viewhtml.obj
 0001:0000a7e7       ?GetContainer@CHtmlView@@QBEPAUIDispatch@@XZ 5f50b7e7 f   viewhtml.obj
 0001:0000a83f       ?GetHtmlDocument@CHtmlView@@QBEPAUIDispatch@@XZ 5f50b83f f   viewhtml.obj
 0001:0000a897       ?GetTopLevelContainer@CHtmlView@@QBEHXZ 5f50b897 f   viewhtml.obj
 0001:0000a8f0       ?GetMenuBar@CHtmlView@@QBEHXZ 5f50b8f0 f   viewhtml.obj
 0001:0000a94c       ?GetFullScreen@CHtmlView@@QBEHXZ 5f50b94c f   viewhtml.obj
 0001:0000a9a8       ?GetStatusBar@CHtmlView@@QBEHXZ 5f50b9a8 f   viewhtml.obj
 0001:0000aa04       ?QueryStatusWB@CHtmlView@@QBE?AW4OLECMDF@@W4OLECMDID@@@Z 5f50ba04 f   viewhtml.obj
 0001:0000aa65       ?ExecWB@CHtmlView@@QAEXW4OLECMDID@@W4OLECMDEXECOPT@@PAUtagVARIANT@@2@Z 5f50ba65 f   viewhtml.obj
 0001:0000aac9       ?GetRegisterAsBrowser@CHtmlView@@QBEHXZ 5f50bac9 f   viewhtml.obj
 0001:0000ab25       ?GetRegisterAsDropTarget@CHtmlView@@QBEHXZ 5f50bb25 f   viewhtml.obj
 0001:0000ab81       ?GetTheaterMode@CHtmlView@@QBEHXZ 5f50bb81 f   viewhtml.obj
 0001:0000abdd       ?GetAddressBar@CHtmlView@@QBEHXZ 5f50bbdd f   viewhtml.obj
 0001:0000ac39       ?LoadFromResource@CHtmlView@@QAEHPBD@Z 5f50bc39 f   viewhtml.obj
 0001:0000ad49       ?LoadFromResource@CHtmlView@@QAEHI@Z 5f50bd49 f   viewhtml.obj
 0001:0000ae59       ?Navigate@CHtmlView@@QAEXPBDK00PAXK@Z 5f50be59 f   viewhtml.obj
 0001:0000afae       ?Navigate2@CHtmlView@@QAEXPAU_ITEMIDLIST@@KPBD@Z 5f50bfae f   viewhtml.obj
 0001:0000b0d8       ?Navigate2@CHtmlView@@QAEXPBDK00PAXK@Z 5f50c0d8 f   viewhtml.obj
 0001:0000b23d       ?Navigate2@CHtmlView@@QAEXPBDKAAVCByteArray@@00@Z 5f50c23d f   viewhtml.obj
 0001:0000b39f       ?PutProperty@CHtmlView@@QAEXPBDABUtagVARIANT@@@Z 5f50c39f f   viewhtml.obj
 0001:0000b46d       ?GetProperty@CHtmlView@@QAEHPBDAAVCString@@@Z 5f50c46d f   viewhtml.obj
 0001:0000b57f       ?GetProperty@CHtmlView@@QAE?AVCOleVariant@@PBD@Z 5f50c57f f   viewhtml.obj
 0001:0000b60f       ?GetFullName@CHtmlView@@QBE?AVCString@@XZ 5f50c60f f   viewhtml.obj
 0001:0000b6c6       ?NavigateComplete2@CHtmlView@@MAEXPAUIDispatch@@PAUtagVARIANT@@@Z 5f50c6c6 f   viewhtml.obj
 0001:0000b7c6       ?BeforeNavigate2@CHtmlView@@MAEXPAUIDispatch@@PAUtagVARIANT@@1111PAH@Z 5f50c7c6 f   viewhtml.obj
 0001:0000ba59       ?DocumentComplete@CHtmlView@@MAEXPAUIDispatch@@PAUtagVARIANT@@@Z 5f50ca59 f   viewhtml.obj
 0001:0000baf0       ?OnProgressChange@CHtmlView@@UAEXJJ@Z 5f50caf0 f   viewhtml.obj
 0001:0000bafd       ?OnCommandStateChange@CHtmlView@@UAEXJH@Z 5f50cafd f   viewhtml.obj
 0001:0000bb0a       ?OnDownloadBegin@CHtmlView@@UAEXXZ 5f50cb0a f   viewhtml.obj
 0001:0000bb15       ?OnDownloadComplete@CHtmlView@@UAEXXZ 5f50cb15 f   viewhtml.obj
 0001:0000bb20       ?OnTitleChange@CHtmlView@@UAEXPBD@Z 5f50cb20 f   viewhtml.obj
 0001:0000bb2d       ?OnPropertyChange@CHtmlView@@UAEXPBD@Z 5f50cb2d f   viewhtml.obj
 0001:0000bb3a       ?OnNewWindow2@CHtmlView@@UAEXPAPAUIDispatch@@PAH@Z 5f50cb3a f   viewhtml.obj
 0001:0000bb4e       ?OnDocumentComplete@CHtmlView@@UAEXPBD@Z 5f50cb4e f   viewhtml.obj
 0001:0000bb5b       ?OnQuit@CHtmlView@@UAEXXZ  5f50cb5b f   viewhtml.obj
 0001:0000bb66       ?OnVisible@CHtmlView@@UAEXH@Z 5f50cb66 f   viewhtml.obj
 0001:0000bb73       ?OnToolBar@CHtmlView@@UAEXH@Z 5f50cb73 f   viewhtml.obj
 0001:0000bb80       ?OnMenuBar@CHtmlView@@UAEXH@Z 5f50cb80 f   viewhtml.obj
 0001:0000bb8d       ?OnStatusBar@CHtmlView@@UAEXH@Z 5f50cb8d f   viewhtml.obj
 0001:0000bb9a       ?OnFullScreen@CHtmlView@@UAEXH@Z 5f50cb9a f   viewhtml.obj
 0001:0000bba7       ?OnTheaterMode@CHtmlView@@UAEXH@Z 5f50cba7 f   viewhtml.obj
 0001:0000bbb4       ?OnNavigateComplete2@CHtmlView@@UAEXPBD@Z 5f50cbb4 f   viewhtml.obj
 0001:0000bbc1       ?OnBeforeNavigate2@CHtmlView@@UAEXPBDK0AAVCByteArray@@0PAH@Z 5f50cbc1 f   viewhtml.obj
 0001:0000bbd5       ?OnStatusTextChange@CHtmlView@@UAEXPBD@Z 5f50cbd5 f   viewhtml.obj
 0001:0000bc01       ?SetRegisterAsBrowser@CHtmlView@@QAEXH@Z 5f50cc01 f   viewhtml.obj
 0001:0000bc5a       ?SetRegisterAsDropTarget@CHtmlView@@QAEXH@Z 5f50cc5a f   viewhtml.obj
 0001:0000bcb3       ?SetTheaterMode@CHtmlView@@QAEXH@Z 5f50ccb3 f   viewhtml.obj
 0001:0000bd0c       ?SetVisible@CHtmlView@@QAEXH@Z 5f50cd0c f   viewhtml.obj
 0001:0000bd65       ?SetMenuBar@CHtmlView@@QAEXH@Z 5f50cd65 f   viewhtml.obj
 0001:0000bdbe       ?SetToolBar@CHtmlView@@QAEXH@Z 5f50cdbe f   viewhtml.obj
 0001:0000be13       ?SetOffline@CHtmlView@@QAEXH@Z 5f50ce13 f   viewhtml.obj
 0001:0000be6c       ?SetSilent@CHtmlView@@QAEXH@Z 5f50ce6c f   viewhtml.obj
 0001:0000bec5       ?GoBack@CHtmlView@@QAEXXZ  5f50cec5 f   viewhtml.obj
 0001:0000bf11       ?GoForward@CHtmlView@@QAEXXZ 5f50cf11 f   viewhtml.obj
 0001:0000bf5d       ?GoHome@CHtmlView@@QAEXXZ  5f50cf5d f   viewhtml.obj
 0001:0000bfa9       ?GoSearch@CHtmlView@@QAEXXZ 5f50cfa9 f   viewhtml.obj
 0001:0000bff5       ?Refresh@CHtmlView@@QAEXXZ 5f50cff5 f   viewhtml.obj
 0001:0000c041       ?Refresh2@CHtmlView@@QAEXH@Z 5f50d041 f   viewhtml.obj
 0001:0000c0e6       ?Stop@CHtmlView@@QAEXXZ    5f50d0e6 f   viewhtml.obj
 0001:0000c132       ?SetFullScreen@CHtmlView@@QAEXH@Z 5f50d132 f   viewhtml.obj
 0001:0000c18b       ?SetAddressBar@CHtmlView@@QAEXH@Z 5f50d18b f   viewhtml.obj
 0001:0000c1e4       ?SetHeight@CHtmlView@@QAEXJ@Z 5f50d1e4 f   viewhtml.obj
 0001:0000c236       ?PutProperty@CHtmlView@@QAEXPBDJ@Z 5f50d236 f   viewhtml.obj
 0001:0000c2ed       ?PutProperty@CHtmlView@@QAEXPBDF@Z 5f50d2ed f   viewhtml.obj
 0001:0000c3a5       ?PutProperty@CHtmlView@@QAEXPBD0@Z 5f50d3a5 f   viewhtml.obj
 0001:0000c45c       ?PutProperty@CHtmlView@@QAEXPBDN@Z 5f50d45c f   viewhtml.obj
 0001:0000c515       ?SetTop@CHtmlView@@QAEXJ@Z 5f50d515 f   viewhtml.obj
 0001:0000c567       ?SetLeft@CHtmlView@@QAEXJ@Z 5f50d567 f   viewhtml.obj
 0001:0000c5b9       ?SetStatusBar@CHtmlView@@QAEXH@Z 5f50d5b9 f   viewhtml.obj
 0001:0000c620       ??_GCHtmlView@@UAEPAXI@Z   5f50d620 f i viewhtml.obj
 0001:0000c620       ??_ECHtmlView@@UAEPAXI@Z   5f50d620 f i viewhtml.obj
 0001:0000c650       ??1CFormView@@UAE@XZ       5f50d650 f i viewhtml.obj
 0001:0000c670       ??_9@$BBDM@AE              5f50d670 f i viewhtml.obj
 0001:0000c680       ??_9@$BBFM@AE              5f50d680 f i viewhtml.obj
 0001:0000c690       ??_9@$BBBM@AE              5f50d690 f i viewhtml.obj
 0001:0000c6a0       ??_9@$BBEA@AE              5f50d6a0 f i viewhtml.obj
 0001:0000c6b0       ??_9@$BBGA@AE              5f50d6b0 f i viewhtml.obj
 0001:0000c6c0       ??_9@$BBCA@AE              5f50d6c0 f i viewhtml.obj
 0001:0000c6d0       ??_9@$BBEE@AE              5f50d6d0 f i viewhtml.obj
 0001:0000c6e0       ??_9@$BBCE@AE              5f50d6e0 f i viewhtml.obj
 0001:0000c6f0       ??_9@$BBEI@AE              5f50d6f0 f i viewhtml.obj
 0001:0000c700       ??_9@$BBCI@AE              5f50d700 f i viewhtml.obj
 0001:0000c710       ??_9@$BBEM@AE              5f50d710 f i viewhtml.obj
 0001:0000c720       ??_9@$BBCM@AE              5f50d720 f i viewhtml.obj
 0001:0000c730       ??_9@$BBFA@AE              5f50d730 f i viewhtml.obj
 0001:0000c740       ??_9@$BBDA@AE              5f50d740 f i viewhtml.obj
 0001:0000c750       ??_9@$BBFE@AE              5f50d750 f i viewhtml.obj
 0001:0000c760       ??_9@$BBDE@AE              5f50d760 f i viewhtml.obj
 0001:0000c770       ??_9@$BBFI@AE              5f50d770 f i viewhtml.obj
 0001:0000c780       ??_9@$BBBI@AE              5f50d780 f i viewhtml.obj
 0001:0000c7c5       ?AfxEnableControlContainer@@YAXPAVCOccManager@@@Z 5f50d7c5 f   occmgr.obj
 0001:0000c7f9       ?_AfxFindFirstDlgItem@@YGPAUDLGITEMTEMPLATE@@PBUDLGTEMPLATE@@@Z 5f50d7f9 f   occmgr.obj
 0001:0000c912       ?_AfxFindNextDlgItem@@YGPAUDLGITEMTEMPLATE@@PAU1@H@Z 5f50d912 f   occmgr.obj
 0001:0000c9bf       ?OnEvent@COccManager@@UAEHPAVCCmdTarget@@IPAUAFX_EVENT@@PAUAFX_CMDHANDLERINFO@@@Z 5f50d9bf f   occmgr.obj
 0001:0000c9e0       ?CreateContainer@COccManager@@UAEPAVCOleControlContainer@@PAVCWnd@@@Z 5f50d9e0 f   occmgr.obj
 0001:0000ca57       ?CreateSite@COccManager@@UAEPAVCOleControlSite@@PAVCOleControlContainer@@@Z 5f50da57 f   occmgr.obj
 0001:0000cad1       ?PreCreateDialog@COccManager@@UAEPBUDLGTEMPLATE@@PAU_AFX_OCC_DIALOG_INFO@@PBU2@@Z 5f50dad1 f   occmgr.obj
 0001:0000cb96       ?PostCreateDialog@COccManager@@UAEXPAU_AFX_OCC_DIALOG_INFO@@@Z 5f50db96 f   occmgr.obj
 0001:0000cbd0       ?SplitDialogTemplate@COccManager@@UAEPAUDLGTEMPLATE@@PBU2@PAPAUDLGITEMTEMPLATE@@@Z 5f50dbd0 f   occmgr.obj
 0001:0000ce36       ?CreateDlgControls@COccManager@@UAEHPAVCWnd@@PBDPAU_AFX_OCC_DIALOG_INFO@@@Z 5f50de36 f   occmgr.obj
 0001:0000cf90       ?CreateDlgControls@COccManager@@UAEHPAVCWnd@@PAXPAU_AFX_OCC_DIALOG_INFO@@@Z 5f50df90 f   occmgr.obj
 0001:0000d34c       ?BindControls@COccManager@@IAEXPAVCWnd@@@Z 5f50e34c f   occmgr.obj
 0001:0000d592       ?CreateDlgControl@COccManager@@IAEPAUHWND__@@PAVCWnd@@PAU2@HPAUDLGITEMTEMPLATE@@GPAEK@Z 5f50e592 f   occmgr.obj
 0001:0000dc0c       ?PrepareOleCtrl@CDataExchange@@QAEPAVCWnd@@H@Z 5f50ec0c f   occmgr.obj
 0001:0000dce0       ??1?$CProcessLocal@VCOccManager@@@@QAE@XZ 5f50ece0 f i occmgr.obj
 0001:0000dd00       ?UnlockResource@@YGHPAX@Z  5f50ed00 f i occmgr.obj
 0001:0000dd10       ?GetData@?$CProcessLocal@VCOccManager@@@@QAEPAVCOccManager@@XZ 5f50ed10 f i occmgr.obj
 0001:0000dd60       ?CreateObject@?$CProcessLocal@VCOccManager@@@@SGPAVCNoTrackObject@@XZ 5f50ed60 f i occmgr.obj
 0001:0000ddd0       ??0COccManager@@QAE@XZ     5f50edd0 f i occmgr.obj
 0001:0000ddf0       ?OnEvent@CCmdTarget@@QAEHIPAUAFX_EVENT@@PAUAFX_CMDHANDLERINFO@@@Z 5f50edf0 f   occevent.obj
 0001:0000e262       ?GetEventSinkEntry@CCmdTarget@@IAGPBUAFX_EVENTSINKMAP_ENTRY@@IPAUAFX_EVENT@@@Z 5f50f262 f   occevent.obj
 0001:0000e320       ?CreateControl@CWnd@@QAEHPBD0KABUtagRECT@@PAV1@IPAVCFile@@HPAG@Z 5f50f320 f   occcont.obj
 0001:0000e398       ?CreateControl@CWnd@@QAEHABU_GUID@@PBDKABUtagRECT@@PAV1@IPAVCFile@@HPAG@Z 5f50f398 f   occcont.obj
 0001:0000e41d       ?CreateControl@CWnd@@QAEHABU_GUID@@PBDKPBUtagPOINT@@PBUtagSIZE@@PAV1@IPAVCFile@@HPAG@Z 5f50f41d f   occcont.obj
 0001:0000e4ca       ?InitControlContainer@CWnd@@IAEHXZ 5f50f4ca f   occcont.obj
 0001:0000e5ea       ?_GetBaseInterfaceMap@COleControlContainer@@KGPBUAFX_INTERFACEMAP@@XZ 5f50f5ea f   occcont.obj
 0001:0000e5f4       ?GetInterfaceMap@COleControlContainer@@MBEPBUAFX_INTERFACEMAP@@XZ 5f50f5f4 f   occcont.obj
 0001:0000e604       ?_GetBaseDispatchMap@COleControlContainer@@KGPBUAFX_DISPMAP@@XZ 5f50f604 f   occcont.obj
 0001:0000e60e       ?GetDispatchMap@COleControlContainer@@MBEPBUAFX_DISPMAP@@XZ 5f50f60e f   occcont.obj
 0001:0000e61e       ??0COleControlContainer@@QAE@PAVCWnd@@@Z 5f50f61e f   occcont.obj
 0001:0000e6c4       ??1COleControlContainer@@UAE@XZ 5f50f6c4 f   occcont.obj
 0001:0000e81f       ?CreateControl@COleControlContainer@@QAEHPAVCWnd@@ABU_GUID@@PBDKABUtagRECT@@IPAVCFile@@HPAGPAPAVCOleControlSite@@@Z 5f50f81f f   occcont.obj
 0001:0000e8a8       ?CreateControl@COleControlContainer@@QAEHPAVCWnd@@ABU_GUID@@PBDKPBUtagPOINT@@PBUtagSIZE@@IPAVCFile@@HPAGPAPAVCOleControlSite@@@Z 5f50f8a8 f   occcont.obj
 0001:0000ea22       ?FindItem@COleControlContainer@@UBEPAVCOleControlSite@@I@Z 5f50fa22 f   occcont.obj
 0001:0000ea72       ?GetAmbientProp@COleControlContainer@@UAEHPAVCOleControlSite@@JPAUtagVARIANT@@@Z 5f50fa72 f   occcont.obj
 0001:0000ed67       ?CreateOleFont@COleControlContainer@@QAEXPAVCFont@@@Z 5f50fd67 f   occcont.obj
 0001:0000efb5       ?FreezeAllEvents@COleControlContainer@@QAEXH@Z 5f50ffb5 f   occcont.obj
 0001:0000effd       ?ScrollChildren@COleControlContainer@@UAEXHH@Z 5f50fffd f   occcont.obj
 0001:0000f0c9       ?OnUIActivate@COleControlContainer@@UAEXPAVCOleControlSite@@@Z 5f5100c9 f   occcont.obj
 0001:0000f129       ?OnUIDeactivate@COleControlContainer@@UAEXPAVCOleControlSite@@@Z 5f510129 f   occcont.obj
 0001:0000f14b       ?CheckDlgButton@COleControlContainer@@UAEXHI@Z 5f51014b f   occcont.obj
 0001:0000f1af       ?CheckRadioButton@COleControlContainer@@UAEXHHH@Z 5f5101af f   occcont.obj
 0001:0000f23e       ?GetDlgItem@COleControlContainer@@UBEPAVCWnd@@H@Z 5f51023e f   occcont.obj
 0001:0000f269       ?GetDlgItem@COleControlContainer@@UBEXHPAPAUHWND__@@@Z 5f510269 f   occcont.obj
 0001:0000f2c0       ?GetDlgItemInt@COleControlContainer@@UBEIHPAHH@Z 5f5102c0 f   occcont.obj
 0001:0000f3bd       ?GetDlgItemTextA@COleControlContainer@@UBEHHPADH@Z 5f5103bd f   occcont.obj
 0001:0000f3f8       ?SendDlgItemMessageA@COleControlContainer@@UAEJHIIJ@Z 5f5103f8 f   occcont.obj
 0001:0000f437       ?SetDlgItemInt@COleControlContainer@@UAEXHIH@Z 5f510437 f   occcont.obj
 0001:0000f48a       ?SetDlgItemTextA@COleControlContainer@@UAEXHPBD@Z 5f51048a f   occcont.obj
 0001:0000f4bf       ?IsDlgButtonChecked@COleControlContainer@@UBEIH@Z 5f5104bf f   occcont.obj
 0001:0000f5ac       ?QueryInterface@XOleIPFrame@COleControlContainer@@UAGJABU_GUID@@PAPAX@Z 5f5105ac f   occcont.obj
 0001:0000f5cf       ?AddRef@XOleIPFrame@COleControlContainer@@UAGKXZ 5f5105cf f   occcont.obj
 0001:0000f5ea       ?Release@XOleIPFrame@COleControlContainer@@UAGKXZ 5f5105ea f   occcont.obj
 0001:0000f605       ?GetWindow@XOleIPFrame@COleControlContainer@@UAGJPAPAUHWND__@@@Z 5f510605 f   occcont.obj
 0001:0000f628       ?ContextSensitiveHelp@XOleIPFrame@COleControlContainer@@UAGJH@Z 5f510628 f   occcont.obj
 0001:0000f634       ?GetBorder@XOleIPFrame@COleControlContainer@@UAGJPAUtagRECT@@@Z 5f510634 f   occcont.obj
 0001:0000f640       ?RequestBorderSpace@XOleIPFrame@COleControlContainer@@UAGJPBUtagRECT@@@Z 5f510640 f   occcont.obj
 0001:0000f64c       ?SetBorderSpace@XOleIPFrame@COleControlContainer@@UAGJPBUtagRECT@@@Z 5f51064c f   occcont.obj
 0001:0000f658       ?SetActiveObject@XOleIPFrame@COleControlContainer@@UAGJPAUIOleInPlaceActiveObject@@PBG@Z 5f510658 f   occcont.obj
 0001:0000f6b4       ?InsertMenus@XOleIPFrame@COleControlContainer@@UAGJPAUHMENU__@@PAUtagOleMenuGroupWidths@@@Z 5f5106b4 f   occcont.obj
 0001:0000f6c0       ?SetMenu@XOleIPFrame@COleControlContainer@@UAGJPAUHMENU__@@PAXPAUHWND__@@@Z 5f5106c0 f   occcont.obj
 0001:0000f6cc       ?RemoveMenus@XOleIPFrame@COleControlContainer@@UAGJPAUHMENU__@@@Z 5f5106cc f   occcont.obj
 0001:0000f6d8       ?SetStatusText@XOleIPFrame@COleControlContainer@@UAGJPBG@Z 5f5106d8 f   occcont.obj
 0001:0000f6e4       ?EnableModeless@XOleIPFrame@COleControlContainer@@UAGJH@Z 5f5106e4 f   occcont.obj
 0001:0000f6ed       ?TranslateAcceleratorA@XOleIPFrame@COleControlContainer@@UAGJPAUtagMSG@@G@Z 5f5106ed f   occcont.obj
 0001:0000f6f9       ?_GetBaseInterfaceMap@CEnumUnknown@@KGPBUAFX_INTERFACEMAP@@XZ 5f5106f9 f   occcont.obj
 0001:0000f703       ?GetInterfaceMap@CEnumUnknown@@MBEPBUAFX_INTERFACEMAP@@XZ 5f510703 f   occcont.obj
 0001:0000f713       ??1CEnumUnknown@@UAE@XZ    5f510713 f   occcont.obj
 0001:0000f7d3       ?OnNext@CEnumUnknown@@MAEHPAX@Z 5f5107d3 f   occcont.obj
 0001:0000f831       ?QueryInterface@XOleContainer@COleControlContainer@@UAGJABU_GUID@@PAPAX@Z 5f510831 f   occcont.obj
 0001:0000f854       ?Release@XOleContainer@COleControlContainer@@UAGKXZ 5f510854 f   occcont.obj
 0001:0000f86f       ?AddRef@XOleContainer@COleControlContainer@@UAGKXZ 5f51086f f   occcont.obj
 0001:0000f88a       ?ParseDisplayName@XOleContainer@COleControlContainer@@UAGJPAUIBindCtx@@PAGPAKPAPAUIMoniker@@@Z 5f51088a f   occcont.obj
 0001:0000f896       ?EnumObjects@XOleContainer@COleControlContainer@@UAGJKPAPAUIEnumUnknown@@@Z 5f510896 f   occcont.obj
 0001:0000fb70       ?LockContainer@XOleContainer@COleControlContainer@@UAGJH@Z 5f510b70 f   occcont.obj
 0001:0000fb80       ??_ECOleControlContainer@@UAEPAXI@Z 5f510b80 f i occcont.obj
 0001:0000fb80       ??_GCOleControlContainer@@UAEPAXI@Z 5f510b80 f i occcont.obj
 0001:0000fbb0       ??0XOleIPFrame@COleControlContainer@@QAE@XZ 5f510bb0 f i occcont.obj
 0001:0000fbd0       ??0XOleContainer@COleControlContainer@@QAE@XZ 5f510bd0 f i occcont.obj
 0001:0000fbf0       ??_ECEnumUnknown@@UAEPAXI@Z 5f510bf0 f i occcont.obj
 0001:0000fbf0       ??_GCEnumUnknown@@UAEPAXI@Z 5f510bf0 f i occcont.obj
 0001:0000fc20       ??0CEnumUnknown@@QAE@PBXI@Z 5f510c20 f i occcont.obj
 0001:0000fc50       ?_GetBaseInterfaceMap@COleControlSite@@KGPBUAFX_INTERFACEMAP@@XZ 5f510c50 f   occsite.obj
 0001:0000fc5a       ?GetInterfaceMap@COleControlSite@@MBEPBUAFX_INTERFACEMAP@@XZ 5f510c5a f   occsite.obj
 0001:0000fc6a       ??0COleControlSite@@QAE@PAVCOleControlContainer@@@Z 5f510c6a f   occsite.obj
 0001:0000fe45       ??1COleControlSite@@UAE@XZ 5f510e45 f   occsite.obj
 0001:00010040       ?SetExtent@COleControlSite@@IAEHXZ 5f511040 f   occsite.obj
 0001:00010128       ?CreateControl@COleControlSite@@QAEJPAVCWnd@@ABU_GUID@@PBDKABUtagRECT@@IPAVCFile@@HPAG@Z 5f511128 f   occsite.obj
 0001:000101ad       ?CreateControl@COleControlSite@@QAEJPAVCWnd@@ABU_GUID@@PBDKPBUtagPOINT@@PBUtagSIZE@@IPAVCFile@@HPAG@Z 5f5111ad f   occsite.obj
 0001:00010653       ?DestroyControl@COleControlSite@@UAEHXZ 5f511653 f   occsite.obj
 0001:000106de       ?_AfxCoCreateInstanceLic@@YGJABU_GUID@@PAUIUnknown@@K0PAPAXPAG@Z 5f5116de f   occsite.obj
 0001:000107e1       ?QuickActivate@COleControlSite@@UAEHXZ 5f5117e1 f   occsite.obj
 0001:00010a84       ?CreateOrLoad@COleControlSite@@IAEJABU_GUID@@PAVCFile@@HPAG@Z 5f511a84 f   occsite.obj
 0001:0001123a       ?GetID@COleControlSite@@QAEIXZ 5f51223a f   occsite.obj
 0001:0001124b       ?DoVerb@COleControlSite@@UAEJJPAUtagMSG@@@Z 5f51224b f   occsite.obj
 0001:00011297       ?IsDefaultButton@COleControlSite@@QAEHXZ 5f512297 f   occsite.obj
 0001:000112d4       ?GetDefBtnCode@COleControlSite@@QAEKXZ 5f5122d4 f   occsite.obj
 0001:00011305       ?SetDefaultButton@COleControlSite@@QAEXH@Z 5f512305 f   occsite.obj
 0001:000113b6       ?ConnectSink@COleControlSite@@IAEKABU_GUID@@PAUIUnknown@@@Z 5f5123b6 f   occsite.obj
 0001:000114b6       ?DisconnectSink@COleControlSite@@IAEXABU_GUID@@K@Z 5f5124b6 f   occsite.obj
 0001:00011588       ?GetEventIID@COleControlSite@@QAEHPAU_GUID@@@Z 5f512588 f   occsite.obj
 0001:0001190c       ?GetControlInfo@COleControlSite@@QAEXXZ 5f51290c f   occsite.obj
 0001:000119a0       ?IsMatchingMnemonic@COleControlSite@@QAEHPAUtagMSG@@@Z 5f5129a0 f   occsite.obj
 0001:00011ae1       ?SendMnemonic@COleControlSite@@QAEXPAUtagMSG@@@Z 5f512ae1 f   occsite.obj
 0001:00011b75       ?FreezeEvents@COleControlSite@@QAEXH@Z 5f512b75 f   occsite.obj
 0001:00011beb       ?AttachWindow@COleControlSite@@IAEXXZ 5f512beb f   occsite.obj
 0001:00011cdc       ?DetachWindow@COleControlSite@@IAEXXZ 5f512cdc f   occsite.obj
 0001:00011d88       ?OnEvent@COleControlSite@@IAEHPAUAFX_EVENT@@@Z 5f512d88 f   occsite.obj
 0001:00011def       ?InvokeHelperV@COleControlSite@@UAEXJGGPAXPBEPAD@Z 5f512def f   occsite.obj
 0001:00011ea7       ?SetPropertyV@COleControlSite@@UAEXJGPAD@Z 5f512ea7 f   occsite.obj
 0001:00011f5f       ?InvokeHelper@COleControlSite@@UAAXJGGPAXPBEZZ 5f512f5f f   occsite.obj
 0001:00011f99       ?GetProperty@COleControlSite@@UBEXJGPAX@Z 5f512f99 f   occsite.obj
 0001:00011fc6       ?SetProperty@COleControlSite@@UAAXJGZZ 5f512fc6 f   occsite.obj
 0001:00011ff3       ?SafeSetProperty@COleControlSite@@UAAHJGZZ 5f512ff3 f   occsite.obj
 0001:000120ad       ?GetStyle@COleControlSite@@UBEKXZ 5f5130ad f   occsite.obj
 0001:000121f9       ?GetExStyle@COleControlSite@@UBEKXZ 5f5131f9 f   occsite.obj
 0001:000122bd       ?ModifyStyle@COleControlSite@@UAEHKKI@Z 5f5132bd f   occsite.obj
 0001:000123a9       ?ModifyStyleEx@COleControlSite@@UAEHKKI@Z 5f5133a9 f   occsite.obj
 0001:0001241d       ?SetWindowTextA@COleControlSite@@UAEXPBD@Z 5f51341d f   occsite.obj
 0001:00012493       ?GetWindowTextA@COleControlSite@@UBEXAAVCString@@@Z 5f513493 f   occsite.obj
 0001:000125c1       ?GetWindowTextA@COleControlSite@@UBEHPADH@Z 5f5135c1 f   occsite.obj
 0001:0001266c       ?GetWindowTextLengthA@COleControlSite@@UBEHXZ 5f51366c f   occsite.obj
 0001:000126d6       ?GetDlgCtrlID@COleControlSite@@UBEHXZ 5f5136d6 f   occsite.obj
 0001:000126e7       ?SetDlgCtrlID@COleControlSite@@UAEHH@Z 5f5136e7 f   occsite.obj
 0001:0001270b       ?MoveWindow@COleControlSite@@UAEXHHHHH@Z 5f51370b f   occsite.obj
 0001:0001282e       ?SetWindowPos@COleControlSite@@UAEHPBVCWnd@@HHHHI@Z 5f51382e f   occsite.obj
 0001:00012945       ?ShowWindow@COleControlSite@@UAEHH@Z 5f513945 f   occsite.obj
 0001:000129c3       ?IsWindowEnabled@COleControlSite@@UBEHXZ 5f5139c3 f   occsite.obj
 0001:00012a64       ?EnableWindow@COleControlSite@@UAEHH@Z 5f513a64 f   occsite.obj
 0001:00012b2d       ?SetFocus@COleControlSite@@UAEPAVCWnd@@XZ 5f513b2d f   occsite.obj
 0001:00012b79       ?EnableDSC@COleControlSite@@UAEXXZ 5f513b79 f   occsite.obj
 0001:00012c14       ?BindDefaultProperty@COleControlSite@@UAEXJGPBDPAVCWnd@@@Z 5f513c14 f   occsite.obj
 0001:00012d64       ?BindProperty@COleControlSite@@UAEXJPAVCWnd@@@Z 5f513d64 f   occsite.obj
 0001:00012fa1       ?AddRef@XOleClientSite@COleControlSite@@UAGKXZ 5f513fa1 f   occsite.obj
 0001:00012fbe       ?Release@XOleClientSite@COleControlSite@@UAGKXZ 5f513fbe f   occsite.obj
 0001:00012fdb       ?QueryInterface@XOleClientSite@COleControlSite@@UAGJABU_GUID@@PAPAX@Z 5f513fdb f   occsite.obj
 0001:00013000       ?SaveObject@XOleClientSite@COleControlSite@@UAGJXZ 5f514000 f   occsite.obj
 0001:0001300c       ?GetMoniker@XOleClientSite@COleControlSite@@UAGJKKPAPAUIMoniker@@@Z 5f51400c f   occsite.obj
 0001:00013018       ?GetContainer@XOleClientSite@COleControlSite@@UAGJPAPAUIOleContainer@@@Z 5f514018 f   occsite.obj
 0001:00013041       ?ShowObject@XOleClientSite@COleControlSite@@UAGJXZ 5f514041 f   occsite.obj
 0001:000130ae       ?OnShowWindow@XOleClientSite@COleControlSite@@UAGJH@Z 5f5140ae f   occsite.obj
 0001:000130b7       ?RequestNewObjectLayout@XOleClientSite@COleControlSite@@UAGJXZ 5f5140b7 f   occsite.obj
 0001:000130c3       ?AddRef@XOleIPSite@COleControlSite@@UAGKXZ 5f5140c3 f   occsite.obj
 0001:000130e0       ?Release@XOleIPSite@COleControlSite@@UAGKXZ 5f5140e0 f   occsite.obj
 0001:000130fd       ?QueryInterface@XOleIPSite@COleControlSite@@UAGJABU_GUID@@PAPAX@Z 5f5140fd f   occsite.obj
 0001:00013122       ?GetWindow@XOleIPSite@COleControlSite@@UAGJPAPAUHWND__@@@Z 5f514122 f   occsite.obj
 0001:0001315d       ?ContextSensitiveHelp@XOleIPSite@COleControlSite@@UAGJH@Z 5f51415d f   occsite.obj
 0001:00013169       ?CanInPlaceActivate@XOleIPSite@COleControlSite@@UAGJXZ 5f514169 f   occsite.obj
 0001:00013172       ?OnInPlaceActivate@XOleIPSite@COleControlSite@@UAGJXZ 5f514172 f   occsite.obj
 0001:0001317b       ?OnUIActivate@XOleIPSite@COleControlSite@@UAGJXZ 5f51417b f   occsite.obj
 0001:000131a7       ?GetWindowContext@XOleIPSite@COleControlSite@@UAGJPAPAUIOleInPlaceFrame@@PAPAUIOleInPlaceUIWindow@@PAUtagRECT@@2PAUtagOIFI@@@Z 5f5141a7 f   occsite.obj
 0001:000133be       ?Scroll@XOleIPSite@COleControlSite@@UAGJUtagSIZE@@@Z 5f5143be f   occsite.obj
 0001:000133ca       ?OnUIDeactivate@XOleIPSite@COleControlSite@@UAGJH@Z 5f5143ca f   occsite.obj
 0001:000133f6       ?OnInPlaceDeactivate@XOleIPSite@COleControlSite@@UAGJXZ 5f5143f6 f   occsite.obj
 0001:00013463       ?DiscardUndoState@XOleIPSite@COleControlSite@@UAGJXZ 5f514463 f   occsite.obj
 0001:0001346c       ?DeactivateAndUndo@XOleIPSite@COleControlSite@@UAGJXZ 5f51446c f   occsite.obj
 0001:00013495       ?OnPosRectChange@XOleIPSite@COleControlSite@@UAGJPBUtagRECT@@@Z 5f514495 f   occsite.obj
 0001:0001351b       ?AddRef@XOleControlSite@COleControlSite@@UAGKXZ 5f51451b f   occsite.obj
 0001:00013538       ?Release@XOleControlSite@COleControlSite@@UAGKXZ 5f514538 f   occsite.obj
 0001:00013555       ?QueryInterface@XOleControlSite@COleControlSite@@UAGJABU_GUID@@PAPAX@Z 5f514555 f   occsite.obj
 0001:0001357a       ?OnControlInfoChanged@XOleControlSite@COleControlSite@@UAGJXZ 5f51457a f   occsite.obj
 0001:00013599       ?LockInPlaceActive@XOleControlSite@COleControlSite@@UAGJH@Z 5f514599 f   occsite.obj
 0001:000135a5       ?GetExtendedControl@XOleControlSite@COleControlSite@@UAGJPAPAUIDispatch@@@Z 5f5145a5 f   occsite.obj
 0001:000135b1       ?TransformCoords@XOleControlSite@COleControlSite@@UAGJPAU_POINTL@@PAUtagPOINTF@@K@Z 5f5145b1 f   occsite.obj
 0001:00013715       ?TranslateAcceleratorA@XOleControlSite@COleControlSite@@UAGJPAUtagMSG@@K@Z 5f514715 f   occsite.obj
 0001:00013721       ?OnFocus@XOleControlSite@COleControlSite@@UAGJH@Z 5f514721 f   occsite.obj
 0001:0001372a       ?ShowPropertyFrame@XOleControlSite@COleControlSite@@UAGJXZ 5f51472a f   occsite.obj
 0001:00013736       ?AddRef@XAmbientProps@COleControlSite@@UAGKXZ 5f514736 f   occsite.obj
 0001:00013753       ?Release@XAmbientProps@COleControlSite@@UAGKXZ 5f514753 f   occsite.obj
 0001:00013770       ?QueryInterface@XAmbientProps@COleControlSite@@UAGJABU_GUID@@PAPAX@Z 5f514770 f   occsite.obj
 0001:00013795       ?GetTypeInfoCount@XAmbientProps@COleControlSite@@UAGJPAI@Z 5f514795 f   occsite.obj
 0001:000137a1       ?GetTypeInfo@XAmbientProps@COleControlSite@@UAGJIKPAPAUITypeInfo@@@Z 5f5147a1 f   occsite.obj
 0001:000137ad       ?GetIDsOfNames@XAmbientProps@COleControlSite@@UAGJABU_GUID@@PAPAGIKPAJ@Z 5f5147ad f   occsite.obj
 0001:000137b9       ?Invoke@XAmbientProps@COleControlSite@@UAGJJABU_GUID@@KGPAUtagDISPPARAMS@@PAUtagVARIANT@@PAUtagEXCEPINFO@@PAI@Z 5f5147b9 f   occsite.obj
 0001:000138e9       ?QueryInterface@XPropertyNotifySink@COleControlSite@@UAGJABU_GUID@@PAPAX@Z 5f5148e9 f   occsite.obj
 0001:00013945       ?AddRef@XPropertyNotifySink@COleControlSite@@UAGKXZ 5f514945 f   occsite.obj
 0001:00013951       ?Release@XPropertyNotifySink@COleControlSite@@UAGKXZ 5f514951 f   occsite.obj
 0001:0001395a       ?OnChanged@XPropertyNotifySink@COleControlSite@@UAGJJ@Z 5f51495a f   occsite.obj
 0001:00013b73       ?OnRequestEdit@XPropertyNotifySink@COleControlSite@@UAGJJ@Z 5f514b73 f   occsite.obj
 0001:00013c4b       ?AddRef@XEventSink@COleControlSite@@UAGKXZ 5f514c4b f   occsite.obj
 0001:00013c57       ?Release@XEventSink@COleControlSite@@UAGKXZ 5f514c57 f   occsite.obj
 0001:00013c60       ?QueryInterface@XEventSink@COleControlSite@@UAGJABU_GUID@@PAPAX@Z 5f514c60 f   occsite.obj
 0001:00013cd3       ?GetTypeInfoCount@XEventSink@COleControlSite@@UAGJPAI@Z 5f514cd3 f   occsite.obj
 0001:00013cdf       ?GetTypeInfo@XEventSink@COleControlSite@@UAGJIKPAPAUITypeInfo@@@Z 5f514cdf f   occsite.obj
 0001:00013ceb       ?GetIDsOfNames@XEventSink@COleControlSite@@UAGJABU_GUID@@PAPAGIKPAJ@Z 5f514ceb f   occsite.obj
 0001:00013cf7       ?Invoke@XEventSink@COleControlSite@@UAGJJABU_GUID@@KGPAUtagDISPPARAMS@@PAUtagVARIANT@@PAUtagEXCEPINFO@@PAI@Z 5f514cf7 f   occsite.obj
 0001:00013e08       ??0CDataSourceControl@@QAE@PAVCOleControlSite@@@Z 5f514e08 f   occsite.obj
 0001:00013f16       ??1CDataSourceControl@@QAE@XZ 5f514f16 f   occsite.obj
 0001:000142da       ?Initialize@CDataSourceControl@@QAEJXZ 5f5152da f   occsite.obj
 0001:000144f8       ?GetCursor@CDataSourceControl@@UAEPAUIUnknown@@XZ 5f5154f8 f   occsite.obj
 0001:000145fb       ?GetMetaData@CDataSourceControl@@QAEJXZ 5f5155fb f   occsite.obj
 0001:00014cb6       ?CopyColumnID@CDataSourceControl@@QAEHPAUtagDBCOLUMNID@@PBU2@@Z 5f515cb6 f   occsite.obj
 0001:00014d81       ?BindProp@CDataSourceControl@@UAEXPAVCOleControlSite@@H@Z 5f515d81 f   occsite.obj
 0001:00014fdb       ?BindProp@CDataSourceControl@@UAEXPAVCDataBoundProperty@@H@Z 5f515fdb f   occsite.obj
 0001:0001506c       ?BindColumns@CDataSourceControl@@UAEXXZ 5f51606c f   occsite.obj
 0001:0001536d       ?GetBoundClientRow@CDataSourceControl@@QAEJXZ 5f51636d f   occsite.obj
 0001:00015415       ?ToVariant@CDataSourceControl@@QAE?AVCOleVariant@@H@Z 5f516415 f   occsite.obj
 0001:00015d93       ?UpdateControls@CDataSourceControl@@UAEJXZ 5f516d93 f   occsite.obj
 0001:00015fe1       ?UpdateCursor@CDataSourceControl@@UAEJXZ 5f516fe1 f   occsite.obj
 0001:00016bca       ??0CDataBoundProperty@@QAE@PAV0@JG@Z 5f517bca f   occsite.obj
 0001:00016c14       ?SetClientSite@CDataBoundProperty@@QAEXPAVCOleControlSite@@@Z 5f517c14 f   occsite.obj
 0001:00016c29       ?SetDSCSite@CDataBoundProperty@@QAEXPAVCOleControlSite@@@Z 5f517c29 f   occsite.obj
 0001:00016c54       ?GetNext@CDataBoundProperty@@QAEPAV1@XZ 5f517c54 f   occsite.obj
 0001:00016c65       ?RemoveSource@CDataBoundProperty@@QAEXXZ 5f517c65 f   occsite.obj
 0001:00016c82       ?Notify@CDataBoundProperty@@QAEXXZ 5f517c82 f   occsite.obj
 0001:00016d56       ?GetCursor@CDataBoundProperty@@QAEPAUIUnknown@@XZ 5f517d56 f   occsite.obj
 0001:00016df0       ?GetCursor@COleControlSite@@IAEJJPAPAUIUnknown@@PAPAX@Z 5f517df0 f   occsite.obj
 0001:00016e4b       ?AddRef@XBoundObjectSite@COleControlSite@@UAGKXZ 5f517e4b f   occsite.obj
 0001:00016eb4       ?Release@XBoundObjectSite@COleControlSite@@UAGKXZ 5f517eb4 f   occsite.obj
 0001:00016f1d       ?QueryInterface@XBoundObjectSite@COleControlSite@@UAGJABU_GUID@@PAPAX@Z 5f517f1d f   occsite.obj
 0001:00016f8e       ?GetCursor@XBoundObjectSite@COleControlSite@@UAGJJPAPAUICursor@@PAPAX@Z 5f517f8e f   occsite.obj
 0001:00017003       ?AddRef@XNotifyDBEvents@COleControlSite@@UAGKXZ 5f518003 f   occsite.obj
 0001:0001700f       ?Release@XNotifyDBEvents@COleControlSite@@UAGKXZ 5f51800f f   occsite.obj
 0001:00017018       ?QueryInterface@XNotifyDBEvents@COleControlSite@@UAGJABU_GUID@@PAPAX@Z 5f518018 f   occsite.obj
 0001:00017074       ?OKToDo@XNotifyDBEvents@COleControlSite@@UAGJKKQAUtagDBNOTIFYREASON@@@Z 5f518074 f   occsite.obj
 0001:000171e3       ?Cancelled@XNotifyDBEvents@COleControlSite@@UAGJKKQAUtagDBNOTIFYREASON@@@Z 5f5181e3 f   occsite.obj
 0001:00017281       ?SyncBefore@XNotifyDBEvents@COleControlSite@@UAGJKKQAUtagDBNOTIFYREASON@@@Z 5f518281 f   occsite.obj
 0001:0001739c       ?AboutToDo@XNotifyDBEvents@COleControlSite@@UAGJKKQAUtagDBNOTIFYREASON@@@Z 5f51839c f   occsite.obj
 0001:0001743a       ?FailedToDo@XNotifyDBEvents@COleControlSite@@UAGJKKQAUtagDBNOTIFYREASON@@@Z 5f51843a f   occsite.obj
 0001:000174d8       ?SyncAfter@XNotifyDBEvents@COleControlSite@@UAGJKKQAUtagDBNOTIFYREASON@@@Z 5f5184d8 f   occsite.obj
 0001:00017641       ?DidEvent@XNotifyDBEvents@COleControlSite@@UAGJKKQAUtagDBNOTIFYREASON@@@Z 5f518641 f   occsite.obj
 0001:0001774a       ?FireEvent@XNotifyDBEvents@COleControlSite@@QAEJKKQAUtagDBNOTIFYREASON@@W4DSCSTATE@@@Z 5f51874a f   occsite.obj
 0001:00017885       ?AddRef@XRowsetNotify@COleControlSite@@UAGKXZ 5f518885 f   occsite.obj
 0001:00017891       ?Release@XRowsetNotify@COleControlSite@@UAGKXZ 5f518891 f   occsite.obj
 0001:0001789a       ?QueryInterface@XRowsetNotify@COleControlSite@@UAGJABU_GUID@@PAPAX@Z 5f51889a f   occsite.obj
 0001:000178f6       ?OnFieldChange@XRowsetNotify@COleControlSite@@UAGJPAUIRowset@@KKQAKKKH@Z 5f5188f6 f   occsite.obj
 0001:00017a74       ?OnRowChange@XRowsetNotify@COleControlSite@@UAGJPAUIRowset@@KQBKKKH@Z 5f518a74 f   occsite.obj
 0001:00017cd3       ?OnRowsetChange@XRowsetNotify@COleControlSite@@UAGJPAUIRowset@@KKH@Z 5f518cd3 f   occsite.obj
 0001:00017e80       ??_GCOleControlSite@@UAEPAXI@Z 5f518e80 f i occsite.obj
 0001:00017e80       ??_ECOleControlSite@@UAEPAXI@Z 5f518e80 f i occsite.obj
 0001:00017eb0       ??0XOleClientSite@COleControlSite@@QAE@XZ 5f518eb0 f i occsite.obj
 0001:00017ed0       ??0XOleIPSite@COleControlSite@@QAE@XZ 5f518ed0 f i occsite.obj
 0001:00017ef0       ??0XOleControlSite@COleControlSite@@QAE@XZ 5f518ef0 f i occsite.obj
 0001:00017f10       ??0XAmbientProps@COleControlSite@@QAE@XZ 5f518f10 f i occsite.obj
 0001:00017f30       ??0XPropertyNotifySink@COleControlSite@@QAE@XZ 5f518f30 f i occsite.obj
 0001:00017f50       ??0XEventSink@COleControlSite@@QAE@XZ 5f518f50 f i occsite.obj
 0001:00017f70       ??0XBoundObjectSite@COleControlSite@@QAE@XZ 5f518f70 f i occsite.obj
 0001:00017f90       ??0XNotifyDBEvents@COleControlSite@@QAE@XZ 5f518f90 f i occsite.obj
 0001:00017fb0       ??0XRowsetNotify@COleControlSite@@QAE@XZ 5f518fb0 f i occsite.obj
 0001:00017fd0       ??0IBoundObjectSite@@QAE@XZ 5f518fd0 f i occsite.obj
 0001:00017ff0       ??0INotifyDBEvents@@QAE@XZ 5f518ff0 f i occsite.obj
 0001:00018010       ??0IRowsetNotify@@QAE@XZ   5f519010 f i occsite.obj
 0001:00018030       ??_GCDataSourceControl@@QAEPAXI@Z 5f519030 f i occsite.obj
 0001:00018060       ??_GCDataBoundProperty@@QAEPAXI@Z 5f519060 f i occsite.obj
 0001:00018090       ??1CDataBoundProperty@@QAE@XZ 5f519090 f i occsite.obj
 0001:000180a0       ??0AFX_EVENT@@QAE@HJPAUtagDISPPARAMS@@PAUtagEXCEPINFO@@PAI@Z 5f5190a0 f i occsite.obj
 0001:00018100       ?ReleaseAccessors@CAccessorBase@ATL@@QAEJPAUIUnknown@@@Z 5f519100 f i occsite.obj
 0001:00018260       ?Close@CDynamicAccessor@ATL@@QAEXXZ 5f519260 f i occsite.obj
 0001:000182e0       ?Close@CAccessorBase@ATL@@QAEXXZ 5f5192e0 f i occsite.obj
 0001:00018360       ??_GCDynamicAccessor@ATL@@QAEPAXI@Z 5f519360 f i occsite.obj
 0001:00018390       ??1CDynamicAccessor@ATL@@QAE@XZ 5f519390 f i occsite.obj
 0001:000183b0       ??_GCRowset@ATL@@QAEPAXI@Z 5f5193b0 f i occsite.obj
 0001:000183e0       ??1CRowset@ATL@@QAE@XZ     5f5193e0 f i occsite.obj
 0001:00018440       ?Close@CRowset@ATL@@QAEXXZ 5f519440 f i occsite.obj
 0001:00018480       ?ReleaseRows@CRowset@ATL@@QAEJXZ 5f519480 f i occsite.obj
 0001:00018510       ??0CRowset@ATL@@QAE@PAUIRowset@@@Z 5f519510 f i occsite.obj
 0001:00018590       ??0CRowset@ATL@@QAE@XZ     5f519590 f i occsite.obj
 0001:00018600       ?MoveFirst@CRowset@ATL@@QAEJXZ 5f519600 f i occsite.obj
 0001:000186b0       ?MoveNext@CRowset@ATL@@QAEJXZ 5f5196b0 f i occsite.obj
 0001:000186d0       ?MoveNext@CRowset@ATL@@QAEJJ_N@Z 5f5196d0 f i occsite.obj
 0001:000187e0       ?AtlTrace2@ATL@@YAXKIPBDZZ 5f5197e0 f i occsite.obj
 0001:00018890       ?GetData@CRowset@ATL@@QAEJXZ 5f519890 f i occsite.obj
 0001:00018940       ?GetNumAccessors@CAccessorBase@ATL@@QBEKXZ 5f519940 f i occsite.obj
 0001:00018960       ?IsAutoAccessor@CAccessorBase@ATL@@QBE_NK@Z 5f519960 f i occsite.obj
 0001:000189f0       ?GetData@CRowset@ATL@@QAEJH@Z 5f5199f0 f i occsite.obj
 0001:00018ae0       ?GetHAccessor@CAccessorBase@ATL@@QBEKK@Z 5f519ae0 f i occsite.obj
 0001:00018b40       ?GetBuffer@CAccessorBase@ATL@@QBEPAEXZ 5f519b40 f i occsite.obj
 0001:00018b60       ?SetupOptionalRowsetInterfaces@CRowset@ATL@@QAEXXZ 5f519b60 f i occsite.obj
 0001:00018ba0       ?SetAccessor@CRowset@ATL@@QAEXPAVCAccessorBase@2@@Z 5f519ba0 f i occsite.obj
 0001:00018bc0       ??0CDynamicAccessor@ATL@@QAE@XZ 5f519bc0 f i occsite.obj
 0001:00018c00       ?GetColumnCount@CDynamicAccessor@ATL@@QBEKXZ 5f519c00 f i occsite.obj
 0001:00018c20       ?BindColumns@CDynamicAccessor@ATL@@QAEJPAUIUnknown@@@Z 5f519c20 f i occsite.obj
 0001:00019170       ?AllocateAccessorMemory@CAccessorBase@ATL@@QAEJH@Z 5f51a170 f i occsite.obj
 0001:00019240       ?BindEntries@CAccessorBase@ATL@@SAJPAUtagDBBINDING@@HPAKKPAUIAccessor@@@Z 5f51a240 f i occsite.obj
 0001:00019420       ?Bind@CAccessorBase@ATL@@SAXPAUtagDBBINDING@@KGKEEKKKKPAUtagDBOBJECT@@@Z 5f51a420 f i occsite.obj
 0001:00019550       ?AddOffset@CDynamicAccessor@ATL@@SAKKK@Z 5f51a550 f i occsite.obj
 0001:00019580       ?GetColumnName@CDynamicAccessor@ATL@@QBEPAGK@Z 5f51a580 f i occsite.obj
 0001:000195c0       ?TranslateColumnNo@CDynamicAccessor@ATL@@QBE_NAAK@Z 5f51a5c0 f i occsite.obj
 0001:00019690       ?GetColumnType@CDynamicAccessor@ATL@@QBE_NKPAG@Z 5f51a690 f i occsite.obj
 0001:000196d0       ?GetValue@CDynamicAccessor@ATL@@QBEPAXK@Z 5f51a6d0 f i occsite.obj
 0001:00019710       ?GetStatus@CDynamicAccessor@ATL@@QBE_NKPAK@Z 5f51a710 f i occsite.obj
 0001:000197b0       ?_GetDataPtr@CDynamicAccessor@ATL@@QBEPAXK@Z 5f51a7b0 f i occsite.obj
 0001:000197e0       ?SetData@CRowset@ATL@@QBEJXZ 5f51a7e0 f i occsite.obj
 0001:00019880       ?SetData@CRowset@ATL@@QBEJH@Z 5f51a880 f i occsite.obj
 0001:00019930       ??0CManualAccessor@ATL@@QAE@XZ 5f51a930 f i occsite.obj
 0001:00019970       ??1CManualAccessor@ATL@@QAE@XZ 5f51a970 f i occsite.obj
 0001:000199b0       ?CreateAccessor@CManualAccessor@ATL@@QAEJHPAXK@Z 5f51a9b0 f i occsite.obj
 0001:00019a80       ?AddBindEntry@CManualAccessor@ATL@@QAEXKGKPAX00@Z 5f51aa80 f i occsite.obj
 0001:00019b60       ?BindColumns@CManualAccessor@ATL@@QAEJPAUIUnknown@@@Z 5f51ab60 f i occsite.obj
 0001:00019c90       ??0AFX_EVENT@@QAE@H@Z      5f51ac90 f i occsite.obj
 0001:00019cf0       ??1?$CComPtr@UIRowsetChange@@@ATL@@QAE@XZ 5f51acf0 f i occsite.obj
 0001:00019cf0       ??1?$CComPtr@UIRowset@@@ATL@@QAE@XZ 5f51acf0 f i occsite.obj
 0001:00019cf0       ??1?$CComPtr@UIColumnsInfo@@@ATL@@QAE@XZ 5f51acf0 f i occsite.obj
 0001:00019cf0       ??1?$CComPtr@UIAccessor@@@ATL@@QAE@XZ 5f51acf0 f i occsite.obj
 0001:00019d20       ??B?$CComPtr@UIAccessor@@@ATL@@QBEPAUIAccessor@@XZ 5f51ad20 f i occsite.obj
 0001:00019d20       ?GetHead@CSimpleList@@QBEPAXXZ 5f51ad20 f i occsite.obj
 0001:00019d20       ??B?$CComPtr@UIRowset@@@ATL@@QBEPAUIRowset@@XZ 5f51ad20 f i occsite.obj
 0001:00019d20       ??B?$CComPtr@UIRowsetChange@@@ATL@@QBEPAUIRowsetChange@@XZ 5f51ad20 f i occsite.obj
 0001:00019d30       ??0?$CComPtr@UIRowsetChange@@@ATL@@QAE@XZ 5f51ad30 f i occsite.obj
 0001:00019d30       ??0?$CComPtr@UIAccessor@@@ATL@@QAE@XZ 5f51ad30 f i occsite.obj
 0001:00019d30       ??0?$CComPtr@UIColumnsInfo@@@ATL@@QAE@XZ 5f51ad30 f i occsite.obj
 0001:00019d30       ??0?$CComPtr@UIRowset@@@ATL@@QAE@XZ 5f51ad30 f i occsite.obj
 0001:00019d50       ??4?$CComPtr@UIRowset@@@ATL@@QAEPAUIRowset@@PAU2@@Z 5f51ad50 f i occsite.obj
 0001:00019d70       ?AtlComPtrAssign@ATL@@YGPAUIUnknown@@PAPAU2@PAU2@@Z 5f51ad70 f i occsite.obj
 0001:00019db0       ?Release@?$CComPtr@UIRowset@@@ATL@@QAEXXZ 5f51adb0 f i occsite.obj
 0001:00019db0       ?Release@?$CComPtr@UIRowsetChange@@@ATL@@QAEXXZ 5f51adb0 f i occsite.obj
 0001:00019de0       ??I?$CComPtr@UIAccessor@@@ATL@@QAEPAPAUIAccessor@@XZ 5f51ade0 f i occsite.obj
 0001:00019de0       ??I?$CComPtr@UIRowsetChange@@@ATL@@QAEPAPAUIRowsetChange@@XZ 5f51ade0 f i occsite.obj
 0001:00019de0       ??I?$CComPtr@UIColumnsInfo@@@ATL@@QAEPAPAUIColumnsInfo@@XZ 5f51ade0 f i occsite.obj
 0001:00019e30       ??C?$CComPtr@UIRowset@@@ATL@@QBEPAV?$_NoAddRefReleaseOnCComPtr@UIRowset@@@1@XZ 5f51ae30 f i occsite.obj
 0001:00019e30       ??C?$CComPtr@UIRowsetChange@@@ATL@@QBEPAV?$_NoAddRefReleaseOnCComPtr@UIRowsetChange@@@1@XZ 5f51ae30 f i occsite.obj
 0001:00019e30       ??C?$CComPtr@UIAccessor@@@ATL@@QBEPAV?$_NoAddRefReleaseOnCComPtr@UIAccessor@@@1@XZ 5f51ae30 f i occsite.obj
 0001:00019e30       ??C?$CComPtr@UIColumnsInfo@@@ATL@@QBEPAV?$_NoAddRefReleaseOnCComPtr@UIColumnsInfo@@@1@XZ 5f51ae30 f i occsite.obj
 0001:00019e80       ?QueryInterface@IUnknown@@QAGJPAPAUIRowsetChange@@@Z 5f51ae80 f i occsite.obj
 0001:00019ea0       ?QueryInterface@IUnknown@@QAGJPAPAUIColumnsInfo@@@Z 5f51aea0 f i occsite.obj
 0001:00019ec0       ?QueryInterface@IUnknown@@QAGJPAPAUIAccessor@@@Z 5f51aec0 f i occsite.obj
 0001:00019ee0       ?GetValue@CDynamicAccessor@ATL@@QBE_NKPAUtagDB_NUMERIC@@@Z 5f51aee0 f i occsite.obj
 0001:00019f20       ?GetValue@CDynamicAccessor@ATL@@QBE_NKPAUtagDBTIME@@@Z 5f51af20 f i occsite.obj
 0001:00019f20       ?GetValue@CDynamicAccessor@ATL@@QBE_NKPAUtagDBDATE@@@Z 5f51af20 f i occsite.obj
 0001:00019f60       ?GetValue@CDynamicAccessor@ATL@@QBE_NKPAUtagDBTIMESTAMP@@@Z 5f51af60 f i occsite.obj
 0001:00019fa0       ?SetValue@CDynamicAccessor@ATL@@QAE_NKABF@Z 5f51afa0 f i occsite.obj
 0001:00019fa0       ?SetValue@CDynamicAccessor@ATL@@QAE_NKABG@Z 5f51afa0 f i occsite.obj
 0001:00019fe0       ?SetValue@CDynamicAccessor@ATL@@QAE_NKABJ@Z 5f51afe0 f i occsite.obj
 0001:00019fe0       ?SetValue@CDynamicAccessor@ATL@@QAE_NKABK@Z 5f51afe0 f i occsite.obj
 0001:00019fe0       ?SetValue@CDynamicAccessor@ATL@@QAE_NKABM@Z 5f51afe0 f i occsite.obj
 0001:0001a020       ?SetValue@CDynamicAccessor@ATL@@QAE_NKABN@Z 5f51b020 f i occsite.obj
 0001:0001a060       ?SetValue@CDynamicAccessor@ATL@@QAE_NKABUtagDBTIMESTAMP@@@Z 5f51b060 f i occsite.obj
 0001:0001a060       ?SetValue@CDynamicAccessor@ATL@@QAE_NKABUtagDEC@@@Z 5f51b060 f i occsite.obj
 0001:0001a0a0       ?SetValue@CDynamicAccessor@ATL@@QAE_NKABC@Z 5f51b0a0 f i occsite.obj
 0001:0001a0a0       ?SetValue@CDynamicAccessor@ATL@@QAE_NKABE@Z 5f51b0a0 f i occsite.obj
 0001:0001a0e0       ?_GetValue@CDynamicAccessor@ATL@@QBEXKPAUtagDB_NUMERIC@@@Z 5f51b0e0 f i occsite.obj
 0001:0001a1a0       ?_GetValue@CDynamicAccessor@ATL@@QBEXKPAUtagDBDATE@@@Z 5f51b1a0 f i occsite.obj
 0001:0001a1a0       ?_GetValue@CDynamicAccessor@ATL@@QBEXKPAUtagDBTIME@@@Z 5f51b1a0 f i occsite.obj
 0001:0001a240       ?_GetValue@CDynamicAccessor@ATL@@QBEXKPAUtagDBTIMESTAMP@@@Z 5f51b240 f i occsite.obj
 0001:0001a2f0       ?_SetValue@CDynamicAccessor@ATL@@QAEXKABG@Z 5f51b2f0 f i occsite.obj
 0001:0001a2f0       ?_SetValue@CDynamicAccessor@ATL@@QAEXKABF@Z 5f51b2f0 f i occsite.obj
 0001:0001a360       ?_SetValue@CDynamicAccessor@ATL@@QAEXKABJ@Z 5f51b360 f i occsite.obj
 0001:0001a360       ?_SetValue@CDynamicAccessor@ATL@@QAEXKABM@Z 5f51b360 f i occsite.obj
 0001:0001a360       ?_SetValue@CDynamicAccessor@ATL@@QAEXKABK@Z 5f51b360 f i occsite.obj
 0001:0001a3d0       ?_SetValue@CDynamicAccessor@ATL@@QAEXKABN@Z 5f51b3d0 f i occsite.obj
 0001:0001a440       ?_SetValue@CDynamicAccessor@ATL@@QAEXKABE@Z 5f51b440 f i occsite.obj
 0001:0001a440       ?_SetValue@CDynamicAccessor@ATL@@QAEXKABC@Z 5f51b440 f i occsite.obj
 0001:0001a4b0       ?_SetValue@CDynamicAccessor@ATL@@QAEXKABUtagDBTIMESTAMP@@@Z 5f51b4b0 f i occsite.obj
 0001:0001a4b0       ?_SetValue@CDynamicAccessor@ATL@@QAEXKABUtagDEC@@@Z 5f51b4b0 f i occsite.obj
 0001:0001a550       ??0COleControlLock@@QAE@ABU_GUID@@@Z 5f51b550 f   occlock.obj
 0001:0001a635       ??1COleControlLock@@UAE@XZ 5f51b635 f   occlock.obj
 0001:0001a682       ?AfxOleLockControl@@YGHABU_GUID@@@Z 5f51b682 f   occlock.obj
 0001:0001a7d0       ?AfxOleLockControl@@YGHPBD@Z 5f51b7d0 f   occlock.obj
 0001:0001a7ff       ?AfxOleUnlockControl@@YGHPBD@Z 5f51b7ff f   occlock.obj
 0001:0001a82e       ?AfxOleUnlockControl@@YGHABU_GUID@@@Z 5f51b82e f   occlock.obj
 0001:0001a8dc       ?AfxOleUnlockAllControls@@YGXXZ 5f51b8dc f   occlock.obj
 0001:0001a990       ??_GCOleControlLock@@UAEPAXI@Z 5f51b990 f i occlock.obj
 0001:0001a990       ??_ECOleControlLock@@UAEPAXI@Z 5f51b990 f i occlock.obj
 0001:0001a9c0       ?IsEmpty@CSimpleList@@QBEHXZ 5f51b9c0 f i occlock.obj
 0001:0001a9e0       ?AddHead@?$CTypedSimpleList@PAVCOleControlLock@@@@QAEXPAVCOleControlLock@@@Z 5f51b9e0 f i occlock.obj
 0001:0001aa00       ?Remove@?$CTypedSimpleList@PAVCOleControlLock@@@@QAEHPAVCOleControlLock@@@Z 5f51ba00 f i occlock.obj
 0001:0001aa20       ??B?$CTypedSimpleList@PAVCOleControlLock@@@@QAEPAVCOleControlLock@@XZ 5f51ba20 f i occlock.obj
 0001:0001aa40       ?DDX_OCText@@YGXPAVCDataExchange@@HJAAVCString@@@Z 5f51ba40 f   occddx.obj
 0001:0001aa90       ?DDX_OCTextRO@@YGXPAVCDataExchange@@HJAAVCString@@@Z 5f51ba90 f   occddx.obj
 0001:0001aae5       ?DDX_OCBool@@YGXPAVCDataExchange@@HJAAH@Z 5f51bae5 f   occddx.obj
 0001:0001ab32       ?DDX_OCBoolRO@@YGXPAVCDataExchange@@HJAAH@Z 5f51bb32 f   occddx.obj
 0001:0001ab53       ?DDX_OCInt@@YGXPAVCDataExchange@@HJAAH@Z 5f51bb53 f   occddx.obj
 0001:0001aba0       ?DDX_OCIntRO@@YGXPAVCDataExchange@@HJAAH@Z 5f51bba0 f   occddx.obj
 0001:0001abc1       ?DDX_OCInt@@YGXPAVCDataExchange@@HJAAJ@Z 5f51bbc1 f   occddx.obj
 0001:0001ac0e       ?DDX_OCIntRO@@YGXPAVCDataExchange@@HJAAJ@Z 5f51bc0e f   occddx.obj
 0001:0001ac2f       ?DDX_OCShort@@YGXPAVCDataExchange@@HJAAF@Z 5f51bc2f f   occddx.obj
 0001:0001ac7d       ?DDX_OCShortRO@@YGXPAVCDataExchange@@HJAAF@Z 5f51bc7d f   occddx.obj
 0001:0001ac9e       ?DDX_OCColor@@YGXPAVCDataExchange@@HJAAK@Z 5f51bc9e f   occddx.obj
 0001:0001aceb       ?DDX_OCColorRO@@YGXPAVCDataExchange@@HJAAK@Z 5f51bceb f   occddx.obj
 0001:0001ad10       ?DDX_OCFloat@@YGXPAVCDataExchange@@HJAAM@Z 5f51bd10 f   occddxf.obj
 0001:0001ad62       ?DDX_OCFloatRO@@YGXPAVCDataExchange@@HJAAM@Z 5f51bd62 f   occddxf.obj
 0001:0001ad95       ?DDX_OCFloat@@YGXPAVCDataExchange@@HJAAN@Z 5f51bd95 f   occddxf.obj
 0001:0001ade6       ?DDX_OCFloatRO@@YGXPAVCDataExchange@@HJAAN@Z 5f51bde6 f   occddxf.obj
 0001:0001ae20       ?_AfxGetDlgCode@@YGKPAVCWnd@@PAUtagMSG@@@Z 5f51be20 f   occdlg.obj
 0001:0001ae6e       ?_AfxDlgSetFocus@@YGXPAVCWnd@@@Z 5f51be6e f   occdlg.obj
 0001:0001aea0       ?_AfxGetChildControl@@YGPAVCWnd@@PAV1@0@Z 5f51bea0 f   occdlg.obj
 0001:0001af5d       ?_AfxNextControl@@YGPAVCWnd@@PAV1@0I@Z 5f51bf5d f   occdlg.obj
 0001:0001b077       ?IsMatchingMnemonic@COccManager@@SAHPAVCWnd@@PAUtagMSG@@@Z 5f51c077 f   occdlg.obj
 0001:0001b0ae       ?_AfxFindNextMnem@@YGPAVCWnd@@PAV1@0PAUtagMSG@@@Z 5f51c0ae f   occdlg.obj
 0001:0001b17a       ?IsLabelControl@COccManager@@SAHPAVCWnd@@@Z 5f51c17a f   occdlg.obj
 0001:0001b1bc       ?_AfxGetNextMnem@@YGPAVCWnd@@PAV1@0PAUtagMSG@@@Z 5f51c1bc f   occdlg.obj
 0001:0001b263       ?UIActivateControl@COccManager@@KAXPAVCWnd@@@Z 5f51c263 f   occdlg.obj
 0001:0001b2e8       ?UIDeactivateIfNecessary@COccManager@@KAXPAVCWnd@@0@Z 5f51c2e8 f   occdlg.obj
 0001:0001b3b1       ?_AfxFindDlgItem@@YGPAVCWnd@@PAV1@K@Z 5f51c3b1 f   occdlg.obj
 0001:0001b42d       ?SetDefaultButton@COccManager@@SAXPAVCWnd@@H@Z 5f51c42d f   occdlg.obj
 0001:0001b48c       ?GetDefBtnCode@COccManager@@SAKPAVCWnd@@@Z 5f51c48c f   occdlg.obj
 0001:0001b4bf       ?_AfxRemoveDefaultButton@@YGXPAVCWnd@@0@Z 5f51c4bf f   occdlg.obj
 0001:0001b545       ?_AfxOriginalDefButton@@YGHPAVCWnd@@@Z 5f51c545 f   occdlg.obj
 0001:0001b594       ?_AfxCheckDefPushButton@@YGXPAVCWnd@@00@Z 5f51c594 f   occdlg.obj
 0001:0001b6ea       ?IsDialogMessageA@COccManager@@UAEHPAVCWnd@@PAUtagMSG@@@Z 5f51c6ea f   occdlg.obj
 0001:0001bc40       ?OnSaveViewState@CDocObjectServer@@MAEXAAVCArchive@@@Z 5f51cc40 f   oledocvw.obj
 0001:0001bc4d       ?OnApplyViewState@CDocObjectServer@@MAEXAAVCArchive@@@Z 5f51cc4d f   oledocvw.obj
 0001:0001bc5a       ?OnActivateView@CDocObjectServer@@MAEJXZ 5f51cc5a f   oledocvw.obj
 0001:0001c4ac       ?AddRef@XOleDocumentView@CDocObjectServer@@UAGKXZ 5f51d4ac f   oledocvw.obj
 0001:0001c516       ?Release@XOleDocumentView@CDocObjectServer@@UAGKXZ 5f51d516 f   oledocvw.obj
 0001:0001c580       ?QueryInterface@XOleDocumentView@CDocObjectServer@@UAGJABU_GUID@@PAPAX@Z 5f51d580 f   oledocvw.obj
 0001:0001c5f2       ?SetInPlaceSite@XOleDocumentView@CDocObjectServer@@UAGJPAUIOleInPlaceSite@@@Z 5f51d5f2 f   oledocvw.obj
 0001:0001c6d1       ?GetInPlaceSite@XOleDocumentView@CDocObjectServer@@UAGJPAPAUIOleInPlaceSite@@@Z 5f51d6d1 f   oledocvw.obj
 0001:0001c793       ?GetDocument@XOleDocumentView@CDocObjectServer@@UAGJPAPAUIUnknown@@@Z 5f51d793 f   oledocvw.obj
 0001:0001c86b       ?OnSetItemRects@CDocObjectServer@@IAEXPAUtagRECT@@0@Z 5f51d86b f   oledocvw.obj
 0001:0001c894       ?SetRect@XOleDocumentView@CDocObjectServer@@UAGJPAUtagRECT@@@Z 5f51d894 f   oledocvw.obj
 0001:0001c999       ?GetRect@XOleDocumentView@CDocObjectServer@@UAGJPAUtagRECT@@@Z 5f51d999 f   oledocvw.obj
 0001:0001ca44       ?SetRectComplex@XOleDocumentView@CDocObjectServer@@UAGJPAUtagRECT@@000@Z 5f51da44 f   oledocvw.obj
 0001:0001caba       ?Show@XOleDocumentView@CDocObjectServer@@UAGJH@Z 5f51daba f   oledocvw.obj
 0001:0001cb6a       ?UIActivate@XOleDocumentView@CDocObjectServer@@UAGJH@Z 5f51db6a f   oledocvw.obj
 0001:0001cc1b       ?Open@XOleDocumentView@CDocObjectServer@@UAGJXZ 5f51dc1b f   oledocvw.obj
 0001:0001ccb5       ?CloseView@XOleDocumentView@CDocObjectServer@@UAGJK@Z 5f51dcb5 f   oledocvw.obj
 0001:0001cd49       ?SaveViewState@XOleDocumentView@CDocObjectServer@@UAGJPAUIStream@@@Z 5f51dd49 f   oledocvw.obj
 0001:0001cf08       ?ApplyViewState@XOleDocumentView@CDocObjectServer@@UAGJPAUIStream@@@Z 5f51df08 f   oledocvw.obj
 0001:0001d0c7       ?Clone@XOleDocumentView@CDocObjectServer@@UAGJPAUIOleInPlaceSite@@PAPAUIOleDocumentView@@@Z 5f51e0c7 f   oledocvw.obj
 0001:0001d140       ?_GetBaseClass@CDocObjectServer@@KGPAUCRuntimeClass@@XZ 5f51e140 f   oledocob.obj
 0001:0001d14a       ?GetRuntimeClass@CDocObjectServer@@UBEPAUCRuntimeClass@@XZ 5f51e14a f   oledocob.obj
 0001:0001d15a       ?_GetBaseMessageMap@CDocObjectServer@@KGPBUAFX_MSGMAP@@XZ 5f51e15a f   oledocob.obj
 0001:0001d164       ?GetMessageMap@CDocObjectServer@@MBEPBUAFX_MSGMAP@@XZ 5f51e164 f   oledocob.obj
 0001:0001d174       ?_GetBaseInterfaceMap@CDocObjectServer@@KGPBUAFX_INTERFACEMAP@@XZ 5f51e174 f   oledocob.obj
 0001:0001d17e       ?GetInterfaceMap@CDocObjectServer@@MBEPBUAFX_INTERFACEMAP@@XZ 5f51e17e f   oledocob.obj
 0001:0001d18e       ??0CDocObjectServer@@QAE@PAVCOleServerDoc@@PAUIOleDocumentSite@@@Z 5f51e18e f   oledocob.obj
 0001:0001d276       ??1CDocObjectServer@@UAE@XZ 5f51e276 f   oledocob.obj
 0001:0001d2c7       ?ReleaseDocSite@CDocObjectServer@@QAEXXZ 5f51e2c7 f   oledocob.obj
 0001:0001d2f7       ?SetDocSite@CDocObjectServer@@QAEXPAUIOleDocumentSite@@@Z 5f51e2f7 f   oledocob.obj
 0001:0001d315       ?OnCloseDocument@CDocObjectServer@@UAEXXZ 5f51e315 f   oledocob.obj
 0001:0001d33c       ?ActivateDocObject@CDocObjectServer@@QAEXXZ 5f51e33c f   oledocob.obj
 0001:0001d3b0       ?OnExecOleCmd@CDocObjectServer@@IAGJPBU_GUID@@KKPAUtagVARIANT@@1@Z 5f51e3b0 f   oledocob.obj
 0001:0001d415       ?GetControllingFrame@CDocObjectServer@@QBEPAVCOleDocIPFrameWnd@@XZ 5f51e415 f   oledocob.obj
 0001:0001d49b       ?DoPreparePrinting@CDocObjectServer@@IAEHPAVCView@@PAUCPrintInfo@@@Z 5f51e49b f   oledocob.obj
 0001:0001d4ba       ?DoPrepareDC@CDocObjectServer@@IAEXPAVCView@@PAVCDC@@PAUCPrintInfo@@@Z 5f51e4ba f   oledocob.obj
 0001:0001d4dd       ?DoPrint@CDocObjectServer@@IAEXPAVCView@@PAVCDC@@PAUCPrintInfo@@@Z 5f51e4dd f   oledocob.obj
 0001:0001d500       ?DoBeginPrinting@CDocObjectServer@@IAEXPAVCView@@PAVCDC@@PAUCPrintInfo@@@Z 5f51e500 f   oledocob.obj
 0001:0001d523       ?DoEndPrinting@CDocObjectServer@@IAEXPAVCView@@PAVCDC@@PAUCPrintInfo@@@Z 5f51e523 f   oledocob.obj
 0001:0001d546       ?AddRef@XPrint@CDocObjectServer@@UAGKXZ 5f51e546 f   oledocob.obj
 0001:0001d5b0       ?Release@XPrint@CDocObjectServer@@UAGKXZ 5f51e5b0 f   oledocob.obj
 0001:0001d61a       ?QueryInterface@XPrint@CDocObjectServer@@UAGJABU_GUID@@PAPAX@Z 5f51e61a f   oledocob.obj
 0001:0001d689       ?SetInitialPageNum@XPrint@CDocObjectServer@@UAGJJ@Z 5f51e689 f   oledocob.obj
 0001:0001d708       ?GetPageInfo@XPrint@CDocObjectServer@@UAGJPAJ0@Z 5f51e708 f   oledocob.obj
 0001:0001d8a6       ?Print@XPrint@CDocObjectServer@@UAGJKPAPAUtagDVTARGETDEVICE@@PAPAUtagPAGESET@@PAUtagSTGMEDIUM@@PAUIContinueCallback@@JPAJ4@Z 5f51e8a6 f   oledocob.obj
 0001:0001e4a1       ?AddRef@XOleDocument@CDocObjectServer@@UAGKXZ 5f51f4a1 f   oledocob.obj
 0001:0001e50b       ?Release@XOleDocument@CDocObjectServer@@UAGKXZ 5f51f50b f   oledocob.obj
 0001:0001e575       ?QueryInterface@XOleDocument@CDocObjectServer@@UAGJABU_GUID@@PAPAX@Z 5f51f575 f   oledocob.obj
 0001:0001e5e4       ?CreateView@XOleDocument@CDocObjectServer@@UAGJPAUIOleInPlaceSite@@PAUIStream@@KPAPAUIOleDocumentView@@@Z 5f51f5e4 f   oledocob.obj
 0001:0001e719       ?GetDocMiscStatus@XOleDocument@CDocObjectServer@@UAGJPAK@Z 5f51f719 f   oledocob.obj
 0001:0001e7be       ?EnumViews@XOleDocument@CDocObjectServer@@UAGJPAPAUIEnumOleDocumentViews@@PAPAUIOleDocumentView@@@Z 5f51f7be f   oledocob.obj
 0001:0001e899       ?AddRef@XOleObject@CDocObjectServer@@UAGKXZ 5f51f899 f   oledocob.obj
 0001:0001e903       ?Release@XOleObject@CDocObjectServer@@UAGKXZ 5f51f903 f   oledocob.obj
 0001:0001e96d       ?QueryInterface@XOleObject@CDocObjectServer@@UAGJABU_GUID@@PAPAX@Z 5f51f96d f   oledocob.obj
 0001:0001e9df       ?SetClientSite@XOleObject@CDocObjectServer@@UAGJPAUIOleClientSite@@@Z 5f51f9df f   oledocob.obj
 0001:0001eac5       ?GetClientSite@XOleObject@CDocObjectServer@@UAGJPAPAUIOleClientSite@@@Z 5f51fac5 f   oledocob.obj
 0001:0001eb56       ?SetHostNames@XOleObject@CDocObjectServer@@UAGJPBG0@Z 5f51fb56 f   oledocob.obj
 0001:0001ebec       ?Close@XOleObject@CDocObjectServer@@UAGJK@Z 5f51fbec f   oledocob.obj
 0001:0001ec7d       ?SetMoniker@XOleObject@CDocObjectServer@@UAGJKPAUIMoniker@@@Z 5f51fc7d f   oledocob.obj
 0001:0001ed13       ?GetMoniker@XOleObject@CDocObjectServer@@UAGJKKPAPAUIMoniker@@@Z 5f51fd13 f   oledocob.obj
 0001:0001edad       ?InitFromData@XOleObject@CDocObjectServer@@UAGJPAUIDataObject@@HK@Z 5f51fdad f   oledocob.obj
 0001:0001ee47       ?GetClipboardData@XOleObject@CDocObjectServer@@UAGJKPAPAUIDataObject@@@Z 5f51fe47 f   oledocob.obj
 0001:0001eedd       ?DoVerb@XOleObject@CDocObjectServer@@UAGJJPAUtagMSG@@PAUIOleClientSite@@JPAUHWND__@@PBUtagRECT@@@Z 5f51fedd f   oledocob.obj
 0001:0001ef83       ?EnumVerbs@XOleObject@CDocObjectServer@@UAGJPAPAUIEnumOLEVERB@@@Z 5f51ff83 f   oledocob.obj
 0001:0001f014       ?Update@XOleObject@CDocObjectServer@@UAGJXZ 5f520014 f   oledocob.obj
 0001:0001f0a2       ?IsUpToDate@XOleObject@CDocObjectServer@@UAGJXZ 5f5200a2 f   oledocob.obj
 0001:0001f130       ?GetUserClassID@XOleObject@CDocObjectServer@@UAGJPAU_GUID@@@Z 5f520130 f   oledocob.obj
 0001:0001f1c1       ?GetUserType@XOleObject@CDocObjectServer@@UAGJKPAPAG@Z 5f5201c1 f   oledocob.obj
 0001:0001f257       ?SetExtent@XOleObject@CDocObjectServer@@UAGJKPAUtagSIZE@@@Z 5f520257 f   oledocob.obj
 0001:0001f317       ?GetExtent@XOleObject@CDocObjectServer@@UAGJKPAUtagSIZE@@@Z 5f520317 f   oledocob.obj
 0001:0001f3ad       ?Advise@XOleObject@CDocObjectServer@@UAGJPAUIAdviseSink@@PAK@Z 5f5203ad f   oledocob.obj
 0001:0001f443       ?Unadvise@XOleObject@CDocObjectServer@@UAGJK@Z 5f520443 f   oledocob.obj
 0001:0001f4d4       ?EnumAdvise@XOleObject@CDocObjectServer@@UAGJPAPAUIEnumSTATDATA@@@Z 5f5204d4 f   oledocob.obj
 0001:0001f565       ?GetMiscStatus@XOleObject@CDocObjectServer@@UAGJKPAK@Z 5f520565 f   oledocob.obj
 0001:0001f5fb       ?SetColorScheme@XOleObject@CDocObjectServer@@UAGJPAUtagLOGPALETTE@@@Z 5f5205fb f   oledocob.obj
 0001:0001f68c       ?AssertValid@CDocObjectServer@@MBEXXZ 5f52068c f   oledocob.obj
 0001:0001f6c8       ?Dump@CDocObjectServer@@MBEXAAVCDumpContext@@@Z 5f5206c8 f   oledocob.obj
 0001:0001f72f       ?_GetBaseClass@CDocObjectServerItem@@KGPAUCRuntimeClass@@XZ 5f52072f f   oledocob.obj
 0001:0001f739       ?GetRuntimeClass@CDocObjectServerItem@@UBEPAUCRuntimeClass@@XZ 5f520739 f   oledocob.obj
 0001:0001f749       ??0CDocObjectServerItem@@IAE@PAVCOleServerDoc@@H@Z 5f520749 f   oledocob.obj
 0001:0001f772       ??1CDocObjectServerItem@@UAE@XZ 5f520772 f   oledocob.obj
 0001:0001f78e       ?OnDoVerb@CDocObjectServerItem@@MAEXJ@Z 5f52078e f   oledocob.obj
 0001:0001f7ef       ?OnHide@CDocObjectServerItem@@MAEXXZ 5f5207ef f   oledocob.obj
 0001:0001f83a       ?OnOpen@CDocObjectServerItem@@MAEXXZ 5f52083a f   oledocob.obj
 0001:0001f883       ?OnShow@CDocObjectServerItem@@MAEXXZ 5f520883 f   oledocob.obj
 0001:0001f8cc       ?AssertValid@CDocObjectServerItem@@UBEXXZ 5f5208cc f   oledocob.obj
 0001:0001f8df       ?Dump@CDocObjectServerItem@@UBEXAAVCDumpContext@@@Z 5f5208df f   oledocob.obj
 0001:0001f900       ??_GCDocObjectServer@@UAEPAXI@Z 5f520900 f i oledocob.obj
 0001:0001f900       ??_ECDocObjectServer@@UAEPAXI@Z 5f520900 f i oledocob.obj
 0001:0001f930       ??0XOleObject@CDocObjectServer@@QAE@XZ 5f520930 f i oledocob.obj
 0001:0001f950       ??0XOleDocument@CDocObjectServer@@QAE@XZ 5f520950 f i oledocob.obj
 0001:0001f970       ??0XOleDocumentView@CDocObjectServer@@QAE@XZ 5f520970 f i oledocob.obj
 0001:0001f990       ??0XOleCommandTarget@CDocObjectServer@@QAE@XZ 5f520990 f i oledocob.obj
 0001:0001f9b0       ??0XPrint@CDocObjectServer@@QAE@XZ 5f5209b0 f i oledocob.obj
 0001:0001f9d0       ??_GCDocObjectServerItem@@UAEPAXI@Z 5f5209d0 f i oledocob.obj
 0001:0001f9d0       ??_ECDocObjectServerItem@@UAEPAXI@Z 5f5209d0 f i oledocob.obj
 0001:0001fa00       ?GetDocument@CDocObjectServerItem@@QBEPAVCOleServerDoc@@XZ 5f520a00 f i oledocob.obj
 0001:0001fa20       ??0COleCmdUI@@QAE@PAU_tagOLECMD@@KPBU_GUID@@@Z 5f520a20 f   oledoctg.obj
 0001:0001fa67       ?Enable@COleCmdUI@@UAEXH@Z 5f520a67 f   oledoctg.obj
 0001:0001fafe       ?SetCheck@COleCmdUI@@UAEXH@Z 5f520afe f   oledoctg.obj
 0001:0001fbb7       ?SetText@COleCmdUI@@UAEXPBD@Z 5f520bb7 f   oledoctg.obj
 0001:0001fbd3       ?DoUpdate@COleCmdUI@@UAEHPAVCCmdTarget@@H@Z 5f520bd3 f   oledoctg.obj
 0001:0001fd5a       ?AddRef@XOleCommandTarget@CDocObjectServer@@UAGKXZ 5f520d5a f   oledoctg.obj
 0001:0001fdc4       ?Release@XOleCommandTarget@CDocObjectServer@@UAGKXZ 5f520dc4 f   oledoctg.obj
 0001:0001fe2e       ?QueryInterface@XOleCommandTarget@CDocObjectServer@@UAGJABU_GUID@@PAPAX@Z 5f520e2e f   oledoctg.obj
 0001:0001fea0       ?_AfxQueryStatusOleCommandHelper@@YGJPAVCCmdTarget@@PBU_GUID@@KQAU_tagOLECMD@@PAU_tagOLECMDTEXT@@@Z 5f520ea0 f   oledoctg.obj
 0001:000200a5       ?QueryStatus@XOleCommandTarget@CDocObjectServer@@UAGJPBU_GUID@@KQAU_tagOLECMD@@PAU_tagOLECMDTEXT@@@Z 5f5210a5 f   oledoctg.obj
 0001:0002013b       ?_AfxExecOleCommandHelper@@YGJPAVCCmdTarget@@PBU_GUID@@KKPAUtagVARIANT@@2@Z 5f52113b f   oledoctg.obj
 0001:0002023f       ?Exec@XOleCommandTarget@CDocObjectServer@@UAGJPBU_GUID@@KKPAUtagVARIANT@@1@Z 5f52123f f   oledoctg.obj
 0001:00020310       ??1COleCmdUI@@QAE@XZ       5f521310 f i oledoctg.obj
 0001:00020330       ?CreateObject@COleDocIPFrameWnd@@SGPAVCObject@@XZ 5f521330 f   oledocip.obj
 0001:0002039e       ?_GetBaseClass@COleDocIPFrameWnd@@KGPAUCRuntimeClass@@XZ 5f52139e f   oledocip.obj
 0001:000203a8       ?GetRuntimeClass@COleDocIPFrameWnd@@UBEPAUCRuntimeClass@@XZ 5f5213a8 f   oledocip.obj
 0001:000203b8       ?_GetBaseMessageMap@COleDocIPFrameWnd@@KGPBUAFX_MSGMAP@@XZ 5f5213b8 f   oledocip.obj
 0001:000203c2       ?GetMessageMap@COleDocIPFrameWnd@@MBEPBUAFX_MSGMAP@@XZ 5f5213c2 f   oledocip.obj
 0001:000203d2       ??0COleDocIPFrameWnd@@QAE@XZ 5f5213d2 f   oledocip.obj
 0001:000203fe       ??1COleDocIPFrameWnd@@UAE@XZ 5f5213fe f   oledocip.obj
 0001:0002041a       ?OnRequestPositionChange@COleDocIPFrameWnd@@MAEXPBUtagRECT@@@Z 5f52141a f   oledocip.obj
 0001:00020492       ?RecalcLayout@COleDocIPFrameWnd@@MAEXH@Z 5f521492 f   oledocip.obj
 0001:000206ec       ?BuildSharedMenu@COleDocIPFrameWnd@@MAEHXZ 5f5216ec f   oledocip.obj
 0001:000208f4       ?DestroySharedMenu@COleDocIPFrameWnd@@MAEXXZ 5f5218f4 f   oledocip.obj
 0001:00020a74       ?AssertValid@COleDocIPFrameWnd@@UBEXXZ 5f521a74 f   oledocip.obj
 0001:00020a87       ?Dump@COleDocIPFrameWnd@@UBEXAAVCDumpContext@@@Z 5f521a87 f   oledocip.obj
 0001:00020aa0       ??_GCOleDocIPFrameWnd@@UAEPAXI@Z 5f521aa0 f i oledocip.obj
 0001:00020ad0       ?_GetBaseClass@COleDocObjectItem@@KGPAUCRuntimeClass@@XZ 5f521ad0 f   oledoccl.obj
 0001:00020ada       ?GetRuntimeClass@COleDocObjectItem@@UBEPAUCRuntimeClass@@XZ 5f521ada f   oledoccl.obj
 0001:00020aea       ?_GetBaseInterfaceMap@COleDocObjectItem@@KGPBUAFX_INTERFACEMAP@@XZ 5f521aea f   oledoccl.obj
 0001:00020af4       ?GetInterfaceMap@COleDocObjectItem@@MBEPBUAFX_INTERFACEMAP@@XZ 5f521af4 f   oledoccl.obj
 0001:00020b04       ??0COleDocObjectItem@@QAE@PAVCOleDocument@@@Z 5f521b04 f   oledoccl.obj
 0001:00020b92       ??1COleDocObjectItem@@UAE@XZ 5f521b92 f   oledoccl.obj
 0001:00020c26       ?AddRef@XOleDocumentSite@COleDocObjectItem@@UAGKXZ 5f521c26 f   oledoccl.obj
 0001:00020c8f       ?Release@XOleDocumentSite@COleDocObjectItem@@UAGKXZ 5f521c8f f   oledoccl.obj
 0001:00020cf8       ?QueryInterface@XOleDocumentSite@COleDocObjectItem@@UAGJABU_GUID@@PAPAX@Z 5f521cf8 f   oledoccl.obj
 0001:00020d69       ?ActivateMe@XOleDocumentSite@COleDocObjectItem@@UAGJPAUIOleDocumentView@@@Z 5f521d69 f   oledoccl.obj
 0001:0002103e       ?ActivateAndShow@COleDocObjectItem@@IAEXXZ 5f52203e f   oledoccl.obj
 0001:00021098       ?OnGetItemPosition@COleDocObjectItem@@MAEXAAVCRect@@@Z 5f522098 f   oledoccl.obj
 0001:0002110e       ?GetActiveView@COleDocObjectItem@@QBEPAUIOleDocumentView@@XZ 5f52210e f   oledoccl.obj
 0001:0002111f       ?Release@COleDocObjectItem@@UAEXW4tagOLECLOSE@@@Z 5f52211f f   oledoccl.obj
 0001:000211a6       ?ExecCommand@COleDocObjectItem@@QAEJKKPBU_GUID@@@Z 5f5221a6 f   oledoccl.obj
 0001:00021217       ?SupportsIPrint@COleDocObjectItem@@IAEHXZ 5f522217 f   oledoccl.obj
 0001:000212bb       ?GetPageCount@COleDocObjectItem@@QAEHPAJ0@Z 5f5222bb f   oledoccl.obj
 0001:00021328       ?GetHelpMenu@COleDocObjectItem@@MAEPAVCMenu@@AAI@Z 5f522328 f   oledoccl.obj
 0001:0002136d       ?OnInsertMenus@COleDocObjectItem@@UAEXPAVCMenu@@PAUtagOleMenuGroupWidths@@@Z 5f52236d f   oledoccl.obj
 0001:000215d3       ?OnRemoveMenus@COleDocObjectItem@@UAEXPAVCMenu@@@Z 5f5225d3 f   oledoccl.obj
 0001:0002165d       ?OnPreparePrinting@COleDocObjectItem@@SAHPAVCView@@PAUCPrintInfo@@H@Z 5f52265d f   oledoccl.obj
 0001:000217d1       ?OnPrint@COleDocObjectItem@@SAXPAVCView@@PAUCPrintInfo@@H@Z 5f5227d1 f   oledoccl.obj
 0001:00021a60       ??_GCOleDocObjectItem@@UAEPAXI@Z 5f522a60 f i oledoccl.obj
 0001:00021a60       ??_ECOleDocObjectItem@@UAEPAXI@Z 5f522a60 f i oledoccl.obj
 0001:00021a90       ??0XOleDocumentSite@COleDocObjectItem@@QAE@XZ 5f522a90 f i oledoccl.obj
 0001:00021ab0       ??0?$CIP@UIUnknown@@$1?IID_IUnknown@@3U_GUID@@B@@QAE@PAUIUnknown@@H@Z 5f522ab0 f i oleasmon.obj
 0001:00021ad0       ??B?$CIP@UIUnknown@@$1?IID_IUnknown@@3U_GUID@@B@@QAEPAUIUnknown@@XZ 5f522ad0 f i oleasmon.obj
 0001:00021af0       ?AddRef@XOleCache@COleControl@@UAGKXZ 5f522af0 f   ctlcache.obj
 0001:00021b0d       ?Release@XOleCache@COleControl@@UAGKXZ 5f522b0d f   ctlcache.obj
 0001:00021b2a       ?QueryInterface@XOleCache@COleControl@@UAGJABU_GUID@@PAPAX@Z 5f522b2a f   ctlcache.obj
 0001:00021b4f       ?Cache@XOleCache@COleControl@@UAGJPAUtagFORMATETC@@KPAK@Z 5f522b4f f   ctlcache.obj
 0001:00021baa       ?Uncache@XOleCache@COleControl@@UAGJK@Z 5f522baa f   ctlcache.obj
 0001:00021bfd       ?EnumCache@XOleCache@COleControl@@UAGJPAPAUIEnumSTATDATA@@@Z 5f522bfd f   ctlcache.obj
 0001:00021c50       ?InitCache@XOleCache@COleControl@@UAGJPAUIDataObject@@@Z 5f522c50 f   ctlcache.obj
 0001:00021ca3       ?SetData@XOleCache@COleControl@@UAGJPAUtagFORMATETC@@PAUtagSTGMEDIUM@@H@Z 5f522ca3 f   ctlcache.obj
 0001:00021d00       ?_AfxGetParkingWindow@@YGPAUHWND__@@XZ 5f522d00 f   ctlcore.obj
 0001:00021ec1       ?_AfxReleaseParkingWindow@@YGXXZ 5f522ec1 f   ctlcore.obj
 0001:0002202d       ?_GetBaseInterfaceMap@COleControl@@KGPBUAFX_INTERFACEMAP@@XZ 5f52302d f   ctlcore.obj
 0001:00022037       ?GetInterfaceMap@COleControl@@MBEPBUAFX_INTERFACEMAP@@XZ 5f523037 f   ctlcore.obj
 0001:00022047       ?_GetBaseMessageMap@COleControl@@KGPBUAFX_MSGMAP@@XZ 5f523047 f   ctlcore.obj
 0001:00022051       ?GetMessageMap@COleControl@@MBEPBUAFX_MSGMAP@@XZ 5f523051 f   ctlcore.obj
 0001:00022061       ??0COleControl@@QAE@XZ     5f523061 f   ctlcore.obj
 0001:0002258f       ??1COleControl@@UAE@XZ     5f52358f f   ctlcore.obj
 0001:00022729       ?ReleaseCaches@COleControl@@IAEXXZ 5f523729 f   ctlcore.obj
 0001:00022aab       ?OnFinalRelease@COleControl@@MAEXXZ 5f523aab f   ctlcore.obj
 0001:00022b00       ?GetInterfaceHook@COleControl@@MAEPAUIUnknown@@PBX@Z 5f523b00 f   ctlcore.obj
 0001:00022ba9       ?SetInitialSize@COleControl@@QAEXHH@Z 5f523ba9 f   ctlcore.obj
 0001:00022beb       ?GetDispatchIID@COleControl@@MAEHPAU_GUID@@@Z 5f523beb f   ctlcore.obj
 0001:00022c2e       ?InitializeIIDs@COleControl@@QAEXPBU_GUID@@0@Z 5f523c2e f   ctlcore.obj
 0001:00022d93       ?AssertValid@COleControl@@UBEXXZ 5f523d93 f   ctlcore.obj
 0001:00022da6       ?_AfxDumpGuid@@YGXAAVCDumpContext@@PBU_GUID@@@Z 5f523da6 f   ctlcore.obj
 0001:00022e4c       ?_AfxDumpHex@@YGXAAVCDumpContext@@K@Z 5f523e4c f   ctlcore.obj
 0001:00022e7a       ?Dump@COleControl@@UBEXAAVCDumpContext@@@Z 5f523e7a f   ctlcore.obj
 0001:00023149       ?_AfxFillPSOnStack@@YGXXZ  5f524149 f   ctlcore.obj
 0001:000231b9       ?DoSuperclassPaint@COleControl@@QAEXPAVCDC@@ABVCRect@@@Z 5f5241b9 f   ctlcore.obj
 0001:00023302       ?IsSubclassedControl@COleControl@@UAEHXZ 5f524302 f   ctlcore.obj
 0001:00023349       ?CreateControlWindow@COleControl@@MAEHPAUHWND__@@ABVCRect@@PBUtagRECT@@@Z 5f524349 f   ctlcore.obj
 0001:000236eb       ?ReparentControlWindow@COleControl@@UAEXPAUHWND__@@0@Z 5f5246eb f   ctlcore.obj
 0001:00023706       ?GetControlSize@COleControl@@QAEXPAH0@Z 5f524706 f   ctlcore.obj
 0001:000237b4       ?SetControlSize@COleControl@@QAEHHH@Z 5f5247b4 f   ctlcore.obj
 0001:00023803       ?SetRectInContainer@COleControl@@QAEHPBUtagRECT@@@Z 5f524803 f   ctlcore.obj
 0001:0002388f       ?OnResetState@COleControl@@UAEXXZ 5f52488f f   ctlcore.obj
 0001:000238c2       ?_AfxDrawBorders@@YGXPAVCDC@@AAVCRect@@HH@Z 5f5248c2 f   ctlcore.obj
 0001:00023923       ?DrawContent@COleControl@@IAEXPAVCDC@@AAVCRect@@@Z 5f524923 f   ctlcore.obj
 0001:00023a39       ?DrawMetafile@COleControl@@IAEXPAVCDC@@AAVCRect@@@Z 5f524a39 f   ctlcore.obj
 0001:00023b00       ?OnDraw@COleControl@@UAEXPAVCDC@@ABVCRect@@1@Z 5f524b00 f   ctlcore.obj
 0001:00023b0d       ?OnDrawMetafile@COleControl@@UAEXPAVCDC@@ABVCRect@@@Z 5f524b0d f   ctlcore.obj
 0001:00023b34       ?GetMetafileData@COleControl@@IAEHPAUtagFORMATETC@@PAUtagSTGMEDIUM@@@Z 5f524b34 f   ctlcore.obj
 0001:00023e13       ?OnCreateAggregates@COleControl@@MAEHXZ 5f524e13 f   ctlcore.obj
 0001:00023e23       ?QueryDefHandler@COleControl@@IAEPAXABU_GUID@@@Z 5f524e23 f   ctlcore.obj
 0001:00023edd       ?InvalidateControl@COleControl@@QAEXPBUtagRECT@@H@Z 5f524edd f   ctlcore.obj
 0001:00024001       ?GetOuterWindow@COleControl@@IBEPAVCWnd@@XZ 5f525001 f   ctlcore.obj
 0001:00024031       ?OnReflectorDestroyed@COleControl@@MAEXXZ 5f525031 f   ctlcore.obj
 0001:00024049       ?SaveState@COleControl@@IAEJPAUIStream@@@Z 5f525049 f   ctlcore.obj
 0001:00024138       ?LoadState@COleControl@@IAEJPAUIStream@@@Z 5f525138 f   ctlcore.obj
 0001:0002429f       ?SendAdvise@COleControl@@IAEXI@Z 5f52529f f   ctlcore.obj
 0001:00024471       ?OnHide@COleControl@@MAEJXZ 5f525471 f   ctlcore.obj
 0001:00024558       ?OnOpen@COleControl@@MAEJHPAUtagMSG@@@Z 5f525558 f   ctlcore.obj
 0001:000246d1       ?CreateFrameWindow@COleControl@@MAEPAVCControlFrameWnd@@XZ 5f5256d1 f   ctlcore.obj
 0001:0002479f       ?OnFrameClose@COleControl@@MAEXXZ 5f52579f f   ctlcore.obj
 0001:0002482d       ?ResizeOpenControl@COleControl@@IAEXHH@Z 5f52582d f   ctlcore.obj
 0001:00024889       ?ResizeFrameWindow@COleControl@@MAEXHH@Z 5f525889 f   ctlcore.obj
 0001:0002492e       ?GetRectInContainer@COleControl@@QAEHPAUtagRECT@@@Z 5f52592e f   ctlcore.obj
 0001:0002496e       ?GetPropPageIDs@COleControl@@MAEPAU_GUID@@AAK@Z 5f52596e f   ctlcore.obj
 0001:00024986       ?OnEdit@COleControl@@UAEHPAUtagMSG@@PAUHWND__@@PBUtagRECT@@@Z 5f525986 f   ctlcore.obj
 0001:000249c6       ?_AfxGetTopLevelWindow@@YGPAUHWND__@@PAU1@@Z 5f5259c6 f   ctlcore.obj
 0001:000249ec       ?OnProperties@COleControl@@UAEHPAUtagMSG@@PAUHWND__@@PBUtagRECT@@@Z 5f5259ec f   ctlcore.obj
 0001:00024b8b       ?GetControlFlags@COleControl@@UAEKXZ 5f525b8b f   ctlcore.obj
 0001:00024b9b       ?OnPaint@COleControl@@IAEXPAVCDC@@@Z 5f525b9b f   ctlcore.obj
 0001:00024da5       ?OnEraseBkgnd@COleControl@@IAEHPAVCDC@@@Z 5f525da5 f   ctlcore.obj
 0001:00024dd7       ?Serialize@COleControl@@MAEXAAVCArchive@@@Z 5f525dd7 f   ctlcore.obj
 0001:00024e26       ?DoPropExchange@COleControl@@UAEXPAVCPropExchange@@@Z 5f525e26 f   ctlcore.obj
 0001:00024e82       ?ControlInfoChanged@COleControl@@QAEXXZ 5f525e82 f   ctlcore.obj
 0001:00024eb1       ?LockInPlaceActive@COleControl@@QAEHH@Z 5f525eb1 f   ctlcore.obj
 0001:00024ef3       ?GetExtendedControl@COleControl@@QAEPAUIDispatch@@XZ 5f525ef3 f   ctlcore.obj
 0001:00024f32       ?TransformCoords@COleControl@@QAEXPAU_POINTL@@PAUtagPOINTF@@K@Z 5f525f32 f   ctlcore.obj
 0001:00024fb5       ?AddRef@XOleControl@COleControl@@UAGKXZ 5f525fb5 f   ctlcore.obj
 0001:00024fd2       ?Release@XOleControl@COleControl@@UAGKXZ 5f525fd2 f   ctlcore.obj
 0001:00024fef       ?QueryInterface@XOleControl@COleControl@@UAGJABU_GUID@@PAPAX@Z 5f525fef f   ctlcore.obj
 0001:00025014       ?GetControlInfo@XOleControl@COleControl@@UAGJPAUtagCONTROLINFO@@@Z 5f526014 f   ctlcore.obj
 0001:0002508b       ?OnMnemonic@XOleControl@COleControl@@UAGJPAUtagMSG@@@Z 5f52608b f   ctlcore.obj
 0001:00025102       ?OnAmbientPropertyChange@XOleControl@COleControl@@UAGJJ@Z 5f526102 f   ctlcore.obj
 0001:000251bb       ?FreezeEvents@XOleControl@COleControl@@UAGJH@Z 5f5261bb f   ctlcore.obj
 0001:000252a1       ?OnGetControlInfo@COleControl@@UAEXPAUtagCONTROLINFO@@@Z 5f5262a1 f   ctlcore.obj
 0001:000252cb       ?OnMnemonic@COleControl@@UAEXPAUtagMSG@@@Z 5f5262cb f   ctlcore.obj
 0001:000252d8       ?OnAmbientPropertyChange@COleControl@@UAEXJ@Z 5f5262d8 f   ctlcore.obj
 0001:000252e5       ?OnFreezeEvents@COleControl@@UAEXH@Z 5f5262e5 f   ctlcore.obj
 0001:000252f2       ?OnSetClientSite@COleControl@@UAEXXZ 5f5262f2 f   ctlcore.obj
 0001:0002533c       ?GetClientSite@COleControl@@QAEPAUIOleClientSite@@XZ 5f52633c f   ctlcore.obj
 0001:00025350       ?TranslateColor@COleControl@@QAEKKPAUHPALETTE__@@@Z 5f526350 f   ctlcore.obj
 0001:0002537b       ?Refresh@COleControl@@QAEXXZ 5f52637b f   ctlcore.obj
 0001:000253a3       ?DoClick@COleControl@@QAEXXZ 5f5263a3 f   ctlcore.obj
 0001:000253be       ?OnNcCreate@COleControl@@IAEHPAUtagCREATESTRUCTA@@@Z 5f5263be f   ctlcore.obj
 0001:000253f5       ?RecreateControlWindow@COleControl@@QAEXXZ 5f5263f5 f   ctlcore.obj
 0001:00025512       ?CreateWindowForSubclassedControl@COleControl@@IAEXXZ 5f526512 f   ctlcore.obj
 0001:0002559b       ?OnMouseActivate@COleControl@@IAEHPAVCWnd@@II@Z 5f52659b f   ctlcore.obj
 0001:000255f7       ?PreModalDialog@COleControl@@QAEXPAUHWND__@@@Z 5f5265f7 f   ctlcore.obj
 0001:0002564c       ?PostModalDialog@COleControl@@QAEXPAUHWND__@@@Z 5f52664c f   ctlcore.obj
 0001:000256a1       ?SetModifiedFlag@COleControl@@QAEXH@Z 5f5266a1 f   ctlcore.obj
 0001:000256d3       ?IsModified@COleControl@@QAEHXZ 5f5266d3 f   ctlcore.obj
 0001:000256ed       ?WillAmbientsBeValidDuringLoad@COleControl@@QAEHXZ 5f5266ed f   ctlcore.obj
 0001:00025707       ?EnableSimpleFrame@COleControl@@QAEXXZ 5f526707 f   ctlcore.obj
 0001:0002572a       ?IgnoreWindowMessage@COleControl@@IAEHIIJPAJ@Z 5f52672a f   ctlcore.obj
 0001:000257c7       ?WindowProc@COleControl@@UAEJIIJ@Z 5f5267c7 f   ctlcore.obj
 0001:00025aa8       ?DefWindowProcA@COleControl@@MAEJIIJ@Z 5f526aa8 f   ctlcore.obj
 0001:00025ad6       ?OnCreate@COleControl@@IAEHPAUtagCREATESTRUCTA@@@Z 5f526ad6 f   ctlcore.obj
 0001:00025b05       ?OnSize@COleControl@@IAEXIHH@Z 5f526b05 f   ctlcore.obj
 0001:00025b38       ?OnMove@COleControl@@IAEXHH@Z 5f526b38 f   ctlcore.obj
 0001:00025b67       ?OnShowWindow@COleControl@@IAEXHI@Z 5f526b67 f   ctlcore.obj
 0001:00025b96       ?OnInitMenuPopup@COleControl@@IAEXPAVCMenu@@IH@Z 5f526b96 f   ctlcore.obj
 0001:00025dca       ?OnMenuSelect@COleControl@@IAEXIIPAUHMENU__@@@Z 5f526dca f   ctlcore.obj
 0001:00025f1b       ?GetMessageString@COleControl@@UBEXIAAVCString@@@Z 5f526f1b f   ctlcore.obj
 0001:00025f8a       ?OnSetMessageString@COleControl@@IAEJIJ@Z 5f526f8a f   ctlcore.obj
 0001:000260f5       ?OnEnterIdle@COleControl@@IAEXIPAVCWnd@@@Z 5f5270f5 f   ctlcore.obj
 0001:0002616b       ?AddRef@XSpecifyPropertyPages@COleControl@@UAGKXZ 5f52716b f   ctlcore.obj
 0001:00026188       ?Release@XSpecifyPropertyPages@COleControl@@UAGKXZ 5f527188 f   ctlcore.obj
 0001:000261a5       ?QueryInterface@XSpecifyPropertyPages@COleControl@@UAGJABU_GUID@@PAPAX@Z 5f5271a5 f   ctlcore.obj
 0001:000261ca       ?GetPages@XSpecifyPropertyPages@COleControl@@UAGJPAUtagCAUUID@@@Z 5f5271ca f   ctlcore.obj
 0001:0002632c       ?OnDestroy@COleControl@@IAEXXZ 5f52732c f   ctlcore.obj
 0001:0002638b       ?OnKillFocus@COleControl@@IAEXPAVCWnd@@@Z 5f52738b f   ctlcore.obj
 0001:000263ca       ?OnSetFocus@COleControl@@IAEXPAVCWnd@@@Z 5f5273ca f   ctlcore.obj
 0001:00026409       ?OnOcmCtlColorBtn@COleControl@@IAEJIJ@Z 5f527409 f   ctlcore.obj
 0001:00026430       ?OnOcmCtlColorDlg@COleControl@@IAEJIJ@Z 5f527430 f   ctlcore.obj
 0001:00026457       ?OnOcmCtlColorEdit@COleControl@@IAEJIJ@Z 5f527457 f   ctlcore.obj
 0001:0002647e       ?OnOcmCtlColorListBox@COleControl@@IAEJIJ@Z 5f52747e f   ctlcore.obj
 0001:000264a5       ?OnOcmCtlColorMsgBox@COleControl@@IAEJIJ@Z 5f5274a5 f   ctlcore.obj
 0001:000264cc       ?OnOcmCtlColorScrollBar@COleControl@@IAEJIJ@Z 5f5274cc f   ctlcore.obj
 0001:000264f3       ?OnOcmCtlColorStatic@COleControl@@IAEJIJ@Z 5f5274f3 f   ctlcore.obj
 0001:0002651a       ?ThrowError@COleControl@@QAEXJII@Z 5f52751a f   ctlcore.obj
 0001:0002656a       ?ThrowError@COleControl@@QAEXJPBDI@Z 5f52756a f   ctlcore.obj
 0001:00026607       ?IsInvokeAllowed@COleControl@@MAEHJ@Z 5f527607 f   ctlcore.obj
 0001:00026630       ??_ECOleControl@@UAEPAXI@Z 5f527630 f i ctlcore.obj
 0001:00026630       ??_GCOleControl@@UAEPAXI@Z 5f527630 f i ctlcore.obj
 0001:00026660       ??0XPersistStorage@COleControl@@QAE@XZ 5f527660 f i ctlcore.obj
 0001:00026680       ??0XPersistStreamInit@COleControl@@QAE@XZ 5f527680 f i ctlcore.obj
 0001:000266a0       ??0XPersistMemory@COleControl@@QAE@XZ 5f5276a0 f i ctlcore.obj
 0001:000266c0       ??0XPersistPropertyBag@COleControl@@QAE@XZ 5f5276c0 f i ctlcore.obj
 0001:000266e0       ??0XOleObject@COleControl@@QAE@XZ 5f5276e0 f i ctlcore.obj
 0001:00026700       ??0XViewObject@COleControl@@QAE@XZ 5f527700 f i ctlcore.obj
 0001:00026720       ??0XDataObject@COleControl@@QAE@XZ 5f527720 f i ctlcore.obj
 0001:00026740       ??0XOleInPlaceObject@COleControl@@QAE@XZ 5f527740 f i ctlcore.obj
 0001:00026760       ??0XOleInPlaceActiveObject@COleControl@@QAE@XZ 5f527760 f i ctlcore.obj
 0001:00026780       ??0XOleCache@COleControl@@QAE@XZ 5f527780 f i ctlcore.obj
 0001:000267a0       ??0XOleControl@COleControl@@QAE@XZ 5f5277a0 f i ctlcore.obj
 0001:000267c0       ??0XProvideClassInfo@COleControl@@QAE@XZ 5f5277c0 f i ctlcore.obj
 0001:000267e0       ??0XSpecifyPropertyPages@COleControl@@QAE@XZ 5f5277e0 f i ctlcore.obj
 0001:00026800       ??0XPerPropertyBrowsing@COleControl@@QAE@XZ 5f527800 f i ctlcore.obj
 0001:00026820       ??0XFontNotification@COleControl@@QAE@XZ 5f527820 f i ctlcore.obj
 0001:00026840       ??0XQuickActivate@COleControl@@QAE@XZ 5f527840 f i ctlcore.obj
 0001:00026860       ??0XPointerInactive@COleControl@@QAE@XZ 5f527860 f i ctlcore.obj
 0001:00026880       ??0IPersistMemory@@QAE@XZ  5f527880 f i ctlcore.obj
 0001:00026880       ??0IPersistPropertyBag@@QAE@XZ 5f527880 f i ctlcore.obj
 0001:00026880       ??0IPersistStreamInit@@QAE@XZ 5f527880 f i ctlcore.obj
 0001:00026880       ??0IPersistStream@@QAE@XZ  5f527880 f i ctlcore.obj
 0001:000268a0       ??0IViewObjectEx@@QAE@XZ   5f5278a0 f i ctlcore.obj
 0001:000268c0       ??0IOleInPlaceObjectWindowless@@QAE@XZ 5f5278c0 f i ctlcore.obj
 0001:000268e0       ??0IConnectionPoint@@QAE@XZ 5f5278e0 f i ctlcore.obj
 0001:000268e0       ??0IOleControlSite@@QAE@XZ 5f5278e0 f i ctlcore.obj
 0001:000268e0       ??0IPointerInactive@@QAE@XZ 5f5278e0 f i ctlcore.obj
 0001:000268e0       ??0IOleDocumentSite@@QAE@XZ 5f5278e0 f i ctlcore.obj
 0001:000268e0       ??0IPerPropertyBrowsing@@QAE@XZ 5f5278e0 f i ctlcore.obj
 0001:000268e0       ??0IOleCache@@QAE@XZ       5f5278e0 f i ctlcore.obj
 0001:000268e0       ??0IOleControl@@QAE@XZ     5f5278e0 f i ctlcore.obj
 0001:000268e0       ??0IProvideClassInfo@@QAE@XZ 5f5278e0 f i ctlcore.obj
 0001:000268e0       ??0IViewObject@@QAE@XZ     5f5278e0 f i ctlcore.obj
 0001:000268e0       ??0IConnectionPointContainer@@QAE@XZ 5f5278e0 f i ctlcore.obj
 0001:000268e0       ??0IQuickActivate@@QAE@XZ  5f5278e0 f i ctlcore.obj
 0001:000268e0       ??0IOleDocument@@QAE@XZ    5f5278e0 f i ctlcore.obj
 0001:000268e0       ??0IPrint@@QAE@XZ          5f5278e0 f i ctlcore.obj
 0001:000268e0       ??0IPropertyPage@@QAE@XZ   5f5278e0 f i ctlcore.obj
 0001:000268e0       ??0ISpecifyPropertyPages@@QAE@XZ 5f5278e0 f i ctlcore.obj
 0001:000268e0       ??0IOleDocumentView@@QAE@XZ 5f5278e0 f i ctlcore.obj
 0001:000268e0       ??0IPropertyNotifySink@@QAE@XZ 5f5278e0 f i ctlcore.obj
 0001:00026900       ??0IProvideClassInfo2@@QAE@XZ 5f527900 f i ctlcore.obj
 0001:00026900       ??0IPropertyPage2@@QAE@XZ  5f527900 f i ctlcore.obj
 0001:00026900       ??0IViewObject2@@QAE@XZ    5f527900 f i ctlcore.obj
 0001:00026920       ??0XEventConnPt@COleControl@@QAE@XZ 5f527920 f i ctlcore.obj
 0001:00026950       ??0XPropConnPt@COleControl@@QAE@XZ 5f527950 f i ctlcore.obj
 0001:00026980       ?GetIID@XPropConnPt@COleControl@@UAEABU_GUID@@XZ 5f527980 f i ctlcore.obj
 0001:00026990       ??_GXEventConnPt@COleControl@@UAEPAXI@Z 5f527990 f i ctlcore.obj
 0001:00026990       ??_EXPropConnPt@COleControl@@UAEPAXI@Z 5f527990 f i ctlcore.obj
 0001:00026990       ??_GXPropConnPt@COleControl@@UAEPAXI@Z 5f527990 f i ctlcore.obj
 0001:00026990       ??_EXEventConnPt@COleControl@@UAEPAXI@Z 5f527990 f i ctlcore.obj
 0001:000269c0       ??1XEventConnPt@COleControl@@UAE@XZ 5f5279c0 f i ctlcore.obj
 0001:000269c0       ??1XPropConnPt@COleControl@@UAE@XZ 5f5279c0 f i ctlcore.obj
 0001:000269e0       ?_AfxIsEqualGUID@@YAHABU_GUID@@0@Z 5f5279e0 f i ctlcore.obj
 0001:00026a40       ??0CReflectorWnd@@QAE@XZ   5f527a40 f i ctlcore.obj
 0001:00026a70       ??_ECControlFrameWnd@@UAEPAXI@Z 5f527a70 f i ctlcore.obj
 0001:00026a70       ??_GCReflectorWnd@@UAEPAXI@Z 5f527a70 f i ctlcore.obj
 0001:00026a70       ??_GCControlFrameWnd@@UAEPAXI@Z 5f527a70 f i ctlcore.obj
 0001:00026a70       ??_ECReflectorWnd@@UAEPAXI@Z 5f527a70 f i ctlcore.obj
 0001:00026aa0       ??0CParkingWnd@@QAE@XZ     5f527aa0 f i ctlcore.obj
 0001:00026b40       ??_ECParkingWnd@@UAEPAXI@Z 5f527b40 f i ctlcore.obj
 0001:00026b40       ??_GCParkingWnd@@UAEPAXI@Z 5f527b40 f i ctlcore.obj
 0001:00026b70       ??1CParkingWnd@@UAE@XZ     5f527b70 f i ctlcore.obj
 0001:00026bc0       ?_GetBaseConnectionMap@COleControl@@KGPBUAFX_CONNECTIONMAP@@XZ 5f527bc0 f   ctlconn.obj
 0001:00026bca       ?GetConnectionMap@COleControl@@MBEPBUAFX_CONNECTIONMAP@@XZ 5f527bca f   ctlconn.obj
 0001:00026bda       ?GetConnectionHook@COleControl@@MAEPAUIConnectionPoint@@ABU_GUID@@@Z 5f527bda f   ctlconn.obj
 0001:00026c13       ?GetExtraConnectionPoints@COleControl@@MAEHPAVCPtrArray@@@Z 5f527c13 f   ctlconn.obj
 0001:00026c36       ?AddRef@XProvideClassInfo@COleControl@@UAGKXZ 5f527c36 f   ctlconn.obj
 0001:00026c53       ?Release@XProvideClassInfo@COleControl@@UAGKXZ 5f527c53 f   ctlconn.obj
 0001:00026c70       ?QueryInterface@XProvideClassInfo@COleControl@@UAGJABU_GUID@@PAPAX@Z 5f527c70 f   ctlconn.obj
 0001:00026c95       ?GetClassInfoA@XProvideClassInfo@COleControl@@UAGJPAPAUITypeInfo@@@Z 5f527c95 f   ctlconn.obj
 0001:00026d1f       ?GetGUID@XProvideClassInfo@COleControl@@UAGJKPAU_GUID@@@Z 5f527d1f f   ctlconn.obj
 0001:00026d88       ?OnAdvise@XEventConnPt@COleControl@@UAEXH@Z 5f527d88 f   ctlconn.obj
 0001:00026df8       ?GetIID@XEventConnPt@COleControl@@UAEABU_GUID@@XZ 5f527df8 f   ctlconn.obj
 0001:00026e26       ?QuerySinkInterface@XEventConnPt@COleControl@@UAEPAUIUnknown@@PAU3@@Z 5f527e26 f   ctlconn.obj
 0001:00026e78       ?OnEventAdvise@COleControl@@UAEXH@Z 5f527e78 f   ctlconn.obj
 0001:00026e85       ?AfxConnectionAdvise@@YGHPAUIUnknown@@ABU_GUID@@0HPAK@Z 5f527e85 f   ctlconn.obj
 0001:00027019       ?AfxConnectionUnadvise@@YGHPAUIUnknown@@ABU_GUID@@0HK@Z 5f528019 f   ctlconn.obj
 0001:00027190       ?_AfxRegisterClipFormat@@YGGABU_GUID@@@Z 5f528190 f   ctldata.obj
 0001:0002721a       ?_AfxGetClipboardFormatConvertVBX@@YGGXZ 5f52821a f   ctldata.obj
 0001:0002726b       ?_AfxGetClipboardFormatPersistPropset@@YGGXZ 5f52826b f   ctldata.obj
 0001:000272bc       ?_AfxOleMatchPropsetClipFormat@@YGHGPAU_GUID@@@Z 5f5282bc f   ctldata.obj
 0001:0002734f       ?AddRef@XDataObject@COleControl@@UAGKXZ 5f52834f f   ctldata.obj
 0001:0002736c       ?Release@XDataObject@COleControl@@UAGKXZ 5f52836c f   ctldata.obj
 0001:00027389       ?QueryInterface@XDataObject@COleControl@@UAGJABU_GUID@@PAPAX@Z 5f528389 f   ctldata.obj
 0001:000273ae       ?GetData@XDataObject@COleControl@@UAGJPAUtagFORMATETC@@PAUtagSTGMEDIUM@@@Z 5f5283ae f   ctldata.obj
 0001:000273f5       ?GetDataHere@XDataObject@COleControl@@UAGJPAUtagFORMATETC@@PAUtagSTGMEDIUM@@@Z 5f5283f5 f   ctldata.obj
 0001:0002743c       ?QueryGetData@XDataObject@COleControl@@UAGJPAUtagFORMATETC@@@Z 5f52843c f   ctldata.obj
 0001:0002747f       ?GetCanonicalFormatEtc@XDataObject@COleControl@@UAGJPAUtagFORMATETC@@0@Z 5f52847f f   ctldata.obj
 0001:000274c6       ?SetData@XDataObject@COleControl@@UAGJPAUtagFORMATETC@@PAUtagSTGMEDIUM@@H@Z 5f5284c6 f   ctldata.obj
 0001:00027511       ?EnumFormatEtc@XDataObject@COleControl@@UAGJKPAPAUIEnumFORMATETC@@@Z 5f528511 f   ctldata.obj
 0001:00027558       ?DAdvise@XDataObject@COleControl@@UAGJPAUtagFORMATETC@@KPAUIAdviseSink@@PAK@Z 5f528558 f   ctldata.obj
 0001:000275f4       ?DUnadvise@XDataObject@COleControl@@UAGJK@Z 5f5285f4 f   ctldata.obj
 0001:00027664       ?EnumDAdvise@XDataObject@COleControl@@UAGJPAPAUIEnumSTATDATA@@@Z 5f528664 f   ctldata.obj
 0001:000276dd       ??0CControlDataSource@COleControl@@QAE@PAV1@@Z 5f5286dd f   ctldata.obj
 0001:00027711       ?OnRenderGlobalData@CControlDataSource@COleControl@@MAEHPAUtagFORMATETC@@PAPAX@Z 5f528711 f   ctldata.obj
 0001:0002774d       ?OnRenderFileData@CControlDataSource@COleControl@@MAEHPAUtagFORMATETC@@PAVCFile@@@Z 5f52874d f   ctldata.obj
 0001:00027789       ?OnRenderData@CControlDataSource@COleControl@@MAEHPAUtagFORMATETC@@PAUtagSTGMEDIUM@@@Z 5f528789 f   ctldata.obj
 0001:000277e0       ?OnSetData@CControlDataSource@COleControl@@MAEHPAUtagFORMATETC@@PAUtagSTGMEDIUM@@H@Z 5f5287e0 f   ctldata.obj
 0001:00027820       ?OnRenderGlobalData@COleControl@@UAEHPAUtagFORMATETC@@PAPAX@Z 5f528820 f   ctldata.obj
 0001:0002789e       ?OnRenderFileData@COleControl@@UAEHPAUtagFORMATETC@@PAVCFile@@@Z 5f52889e f   ctldata.obj
 0001:00027904       ?OnRenderData@COleControl@@UAEHPAUtagFORMATETC@@PAUtagSTGMEDIUM@@@Z 5f528904 f   ctldata.obj
 0001:000279da       ?OnSetData@COleControl@@UAEHPAUtagFORMATETC@@PAUtagSTGMEDIUM@@H@Z 5f5289da f   ctldata.obj
 0001:00027aa3       ?GetDataSource@COleControl@@IAEPAVCControlDataSource@1@XZ 5f528aa3 f   ctldata.obj
 0001:00027bf0       ?SetInitialDataFormats@COleControl@@MAEXXZ 5f528bf0 f   ctldata.obj
 0001:00027ca0       ??_ECControlDataSource@COleControl@@UAEPAXI@Z 5f528ca0 f i ctldata.obj
 0001:00027ca0       ??_GCControlDataSource@COleControl@@UAEPAXI@Z 5f528ca0 f i ctldata.obj
 0001:00027cd0       ??1CControlDataSource@COleControl@@UAE@XZ 5f528cd0 f i ctldata.obj
 0001:00027cf0       ?InitStockEventMask@COleControl@@IAEXXZ 5f528cf0 f   ctlevent.obj
 0001:00027deb       ?GetEventMap@COleControl@@MBEPBUAFX_EVENTMAP@@XZ 5f528deb f   ctlevent.obj
 0001:00027dfb       ?GetEventMapEntry@COleControl@@IBEPBUAFX_EVENTMAP_ENTRY@@PBDPAJ@Z 5f528dfb f   ctlevent.obj
 0001:00027eff       ?FireEventV@COleControl@@IAEXJPAEPAD@Z 5f528eff f   ctlevent.obj
 0001:00028021       ?FireEvent@COleControl@@QAAXJPAEZZ 5f529021 f   ctlevent.obj
 0001:0002804a       ?_AfxShiftState@@YGFXZ     5f52904a f   ctlevent.obj
 0001:000280a2       ?OnSysKeyDown@COleControl@@IAEXIII@Z 5f5290a2 f   ctlevent.obj
 0001:00028119       ?OnSysKeyUp@COleControl@@IAEXIII@Z 5f529119 f   ctlevent.obj
 0001:00028190       ?OnKeyDown@COleControl@@IAEXIII@Z 5f529190 f   ctlevent.obj
 0001:00028207       ?OnKeyUp@COleControl@@IAEXIII@Z 5f529207 f   ctlevent.obj
 0001:0002827e       ?KeyUp@COleControl@@IAEXPAG@Z 5f52927e f   ctlevent.obj
 0001:000282dc       ?KeyDown@COleControl@@IAEXPAG@Z 5f5292dc f   ctlevent.obj
 0001:0002833a       ?_AfxPostTrailByte@@YGXPAVCWnd@@E@Z 5f52933a f   ctlevent.obj
 0001:000283f4       ?OnGetDlgCode@COleControl@@IAEIXZ 5f5293f4 f   ctlevent.obj
 0001:00028440       ?OnChar@COleControl@@IAEXIII@Z 5f529440 f   ctlevent.obj
 0001:00028722       ?OnKeyPressEvent@COleControl@@UAEXG@Z 5f529722 f   ctlevent.obj
 0001:0002872f       ?OnKeyDownEvent@COleControl@@UAEXGG@Z 5f52972f f   ctlevent.obj
 0001:0002873c       ?OnKeyUpEvent@COleControl@@UAEXGG@Z 5f52973c f   ctlevent.obj
 0001:00028749       ?ButtonDown@COleControl@@IAEXGIVCPoint@@@Z 5f529749 f   ctlevent.obj
 0001:00028837       ?ButtonUp@COleControl@@IAEXGIVCPoint@@@Z 5f529837 f   ctlevent.obj
 0001:00028994       ?ButtonDblClk@COleControl@@IAEXGIVCPoint@@@Z 5f529994 f   ctlevent.obj
 0001:00028a47       ?OnMouseMove@COleControl@@IAEXIVCPoint@@@Z 5f529a47 f   ctlevent.obj
 0001:00028aa9       ?OnLButtonDown@COleControl@@IAEXIVCPoint@@@Z 5f529aa9 f   ctlevent.obj
 0001:00028acc       ?OnLButtonUp@COleControl@@IAEXIVCPoint@@@Z 5f529acc f   ctlevent.obj
 0001:00028aef       ?OnLButtonDblClk@COleControl@@IAEXIVCPoint@@@Z 5f529aef f   ctlevent.obj
 0001:00028b12       ?OnMButtonDown@COleControl@@IAEXIVCPoint@@@Z 5f529b12 f   ctlevent.obj
 0001:00028b35       ?OnMButtonUp@COleControl@@IAEXIVCPoint@@@Z 5f529b35 f   ctlevent.obj
 0001:00028b58       ?OnMButtonDblClk@COleControl@@IAEXIVCPoint@@@Z 5f529b58 f   ctlevent.obj
 0001:00028b7b       ?OnRButtonDown@COleControl@@IAEXIVCPoint@@@Z 5f529b7b f   ctlevent.obj
 0001:00028b9e       ?OnRButtonUp@COleControl@@IAEXIVCPoint@@@Z 5f529b9e f   ctlevent.obj
 0001:00028bc1       ?OnRButtonDblClk@COleControl@@IAEXIVCPoint@@@Z 5f529bc1 f   ctlevent.obj
 0001:00028be4       ?OnButtonDown@COleControl@@IAEXGIVCPoint@@@Z 5f529be4 f   ctlevent.obj
 0001:00028c40       ?OnButtonUp@COleControl@@IAEXGIVCPoint@@@Z 5f529c40 f   ctlevent.obj
 0001:00028d12       ?OnButtonDblClk@COleControl@@IAEXGIVCPoint@@@Z 5f529d12 f   ctlevent.obj
 0001:00028d58       ?OnCancelMode@COleControl@@IAEXXZ 5f529d58 f   ctlevent.obj
 0001:00028dc6       ?OnClick@COleControl@@UAEXG@Z 5f529dc6 f   ctlevent.obj
 0001:00028dea       ?FireError@COleControl@@QAEXJPBDI@Z 5f529dea f   ctlevent.obj
 0001:00028f71       ?DisplayError@COleControl@@UAEXJPBD00I@Z 5f529f71 f   ctlevent.obj
 0001:00028f90       ?_GetBaseMessageMap@CControlFrameWnd@@KGPBUAFX_MSGMAP@@XZ 5f529f90 f   ctlframe.obj
 0001:00028f9a       ?GetMessageMap@CControlFrameWnd@@MBEPBUAFX_MSGMAP@@XZ 5f529f9a f   ctlframe.obj
 0001:00028faa       ??0CControlFrameWnd@@QAE@PAVCOleControl@@@Z 5f529faa f   ctlframe.obj
 0001:00028fd4       ?PreCreateWindow@CControlFrameWnd@@UAEHAAUtagCREATESTRUCTA@@@Z 5f529fd4 f   ctlframe.obj
 0001:00029021       ?Create@CControlFrameWnd@@UAEHPBD@Z 5f52a021 f   ctlframe.obj
 0001:0002907c       ?OnClose@CControlFrameWnd@@IAEXXZ 5f52a07c f   ctlframe.obj
 0001:000290a6       ?PostNcDestroy@CControlFrameWnd@@MAEXXZ 5f52a0a6 f   ctlframe.obj
 0001:000290de       ?OnActivate@CControlFrameWnd@@IAEXIPAVCWnd@@H@Z 5f52a0de f   ctlframe.obj
 0001:00029110       ??1CReflectorWnd@@UAE@XZ   5f52a110 f i ctlframe.obj
 0001:00029110       ??1CControlFrameWnd@@UAE@XZ 5f52a110 f i ctlframe.obj
 0001:00029130       ??0CFontHolder@@QAE@PAUIPropertyNotifySink@@@Z 5f52a130 f   ctlfont.obj
 0001:00029190       ?SetFontNotifySink@CFontHolder@@QAEXPAUIPropertyNotifySink@@@Z 5f52a190 f   ctlfont.obj
 0001:000291da       ??1CFontHolder@@QAE@XZ     5f52a1da f   ctlfont.obj
 0001:000291ed       ?ReleaseFont@CFontHolder@@QAEXXZ 5f52a1ed f   ctlfont.obj
 0001:00029250       ?InitializeFont@CFontHolder@@QAEXPBUtagFONTDESC@@PAUIDispatch@@@Z 5f52a250 f   ctlfont.obj
 0001:0002939c       ?_AfxIsSameFont@@YGHAAVCFontHolder@@PBUtagFONTDESC@@PAUIFontDisp@@@Z 5f52a39c f   ctlfont.obj
 0001:000295fb       ?GetFontHandle@CFontHolder@@QAEPAUHFONT__@@XZ 5f52a5fb f   ctlfont.obj
 0001:0002961c       ?GetFontHandle@CFontHolder@@QAEPAUHFONT__@@JJ@Z 5f52a61c f   ctlfont.obj
 0001:00029697       ?Select@CFontHolder@@QAEPAVCFont@@PAVCDC@@JJ@Z 5f52a697 f   ctlfont.obj
 0001:00029748       ?QueryTextMetrics@CFontHolder@@QAEXPAUtagTEXTMETRICA@@@Z 5f52a748 f   ctlfont.obj
 0001:000297b8       ?GetFontDispatch@CFontHolder@@QAEPAUIFontDisp@@XZ 5f52a7b8 f   ctlfont.obj
 0001:0002982a       ?SetFont@CFontHolder@@QAEXPAUIFont@@@Z 5f52a82a f   ctlfont.obj
 0001:000298af       ?GetDisplayString@CFontHolder@@QAEHAAVCString@@@Z 5f52a8af f   ctlfont.obj
 0001:000298d0       ??0_AFXCTL_UIACTIVE_INFO@@QAE@PAUHMENU__@@PAUIOleInPlaceFrame@@@Z 5f52a8d0 f   ctlinplc.obj
 0001:000299f7       ??1_AFXCTL_UIACTIVE_INFO@@QAE@XZ 5f52a9f7 f   ctlinplc.obj
 0001:00029a4f       ?_GetClippingCoordinates@@YGXPBUtagRECT@@0PAU1@PAUtagPOINT@@@Z 5f52aa4f f   ctlinplc.obj
 0001:00029b03       ?OnActivateInPlace@COleControl@@MAEJHPAUtagMSG@@@Z 5f52ab03 f   ctlinplc.obj
 0001:0002a27b       ?ForwardActivationMsg@COleControl@@IAEXPAUtagMSG@@@Z 5f52b27b f   ctlinplc.obj
 0001:0002a3a1       ?OnGetInPlaceMenu@COleControl@@UAEPAUHMENU__@@XZ 5f52b3a1 f   ctlinplc.obj
 0001:0002a3ae       ?BuildSharedMenu@COleControl@@MAEHXZ 5f52b3ae f   ctlinplc.obj
 0001:0002a533       ?DestroySharedMenu@COleControl@@MAEXXZ 5f52b533 f   ctlinplc.obj
 0001:0002a66e       ?AddFrameLevelUI@COleControl@@MAEXXZ 5f52b66e f   ctlinplc.obj
 0001:0002a6fa       ?RemoveFrameLevelUI@COleControl@@MAEXXZ 5f52b6fa f   ctlinplc.obj
 0001:0002a7c8       ?OnShowToolBars@COleControl@@UAEXXZ 5f52b7c8 f   ctlinplc.obj
 0001:0002a7ed       ?OnHideToolBars@COleControl@@UAEXXZ 5f52b7ed f   ctlinplc.obj
 0001:0002a7f8       ?AddRef@XOleInPlaceObject@COleControl@@UAGKXZ 5f52b7f8 f   ctlinplc.obj
 0001:0002a815       ?Release@XOleInPlaceObject@COleControl@@UAGKXZ 5f52b815 f   ctlinplc.obj
 0001:0002a832       ?QueryInterface@XOleInPlaceObject@COleControl@@UAGJABU_GUID@@PAPAX@Z 5f52b832 f   ctlinplc.obj
 0001:0002a857       ?GetWindow@XOleInPlaceObject@COleControl@@UAGJPAPAUHWND__@@@Z 5f52b857 f   ctlinplc.obj
 0001:0002a8b3       ?ContextSensitiveHelp@XOleInPlaceObject@COleControl@@UAGJH@Z 5f52b8b3 f   ctlinplc.obj
 0001:0002a8bf       ?InPlaceDeactivate@XOleInPlaceObject@COleControl@@UAGJXZ 5f52b8bf f   ctlinplc.obj
 0001:0002aa1c       ?UIDeactivate@XOleInPlaceObject@COleControl@@UAGJXZ 5f52ba1c f   ctlinplc.obj
 0001:0002ab5e       ?SetObjectRects@XOleInPlaceObject@COleControl@@UAGJPBUtagRECT@@0@Z 5f52bb5e f   ctlinplc.obj
 0001:0002abe3       ?OnSetObjectRects@COleControl@@UAEHPBUtagRECT@@0@Z 5f52bbe3 f   ctlinplc.obj
 0001:0002ad80       ?ReactivateAndUndo@XOleInPlaceObject@COleControl@@UAGJXZ 5f52bd80 f   ctlinplc.obj
 0001:0002ad8c       ?AddRef@XOleInPlaceActiveObject@COleControl@@UAGKXZ 5f52bd8c f   ctlinplc.obj
 0001:0002ada9       ?Release@XOleInPlaceActiveObject@COleControl@@UAGKXZ 5f52bda9 f   ctlinplc.obj
 0001:0002adc6       ?QueryInterface@XOleInPlaceActiveObject@COleControl@@UAGJABU_GUID@@PAPAX@Z 5f52bdc6 f   ctlinplc.obj
 0001:0002adeb       ?GetWindow@XOleInPlaceActiveObject@COleControl@@UAGJPAPAUHWND__@@@Z 5f52bdeb f   ctlinplc.obj
 0001:0002ae1a       ?ContextSensitiveHelp@XOleInPlaceActiveObject@COleControl@@UAGJH@Z 5f52be1a f   ctlinplc.obj
 0001:0002ae26       ?TranslateAcceleratorA@XOleInPlaceActiveObject@COleControl@@UAGJPAUtagMSG@@@Z 5f52be26 f   ctlinplc.obj
 0001:0002aef6       ?OnFrameWindowActivate@XOleInPlaceActiveObject@COleControl@@UAGJH@Z 5f52bef6 f   ctlinplc.obj
 0001:0002aeff       ?OnDocWindowActivate@XOleInPlaceActiveObject@COleControl@@UAGJH@Z 5f52beff f   ctlinplc.obj
 0001:0002af9b       ?ResizeBorder@XOleInPlaceActiveObject@COleControl@@UAGJPBUtagRECT@@PAUIOleInPlaceUIWindow@@H@Z 5f52bf9b f   ctlinplc.obj
 0001:0002afa4       ?EnableModeless@XOleInPlaceActiveObject@COleControl@@UAGJH@Z 5f52bfa4 f   ctlinplc.obj
 0001:0002afb0       ??_G_AFXCTL_UIACTIVE_INFO@@QAEPAXI@Z 5f52bfb0 f i ctlinplc.obj
 0001:0002afe0       ?AfxVerifyLicFile@@YGHPAUHINSTANCE__@@PBDPBGI@Z 5f52bfe0 f   ctllic.obj
 0001:0002b1d0       __tcsrchr                  5f52c1d0 f i ctllic.obj
 0001:0002b1f0       ??0CConnectionPoint@@QAE@XZ 5f52c1f0 f   oleconn.obj
 0001:0002b25b       ??1CConnectionPoint@@UAE@XZ 5f52c25b f   oleconn.obj
 0001:0002b32e       ?GetStartPosition@CConnectionPoint@@QBEPAU__POSITION@@XZ 5f52c32e f   oleconn.obj
 0001:0002b397       ?GetNextConnection@CConnectionPoint@@QBEPAUIUnknown@@AAPAU__POSITION@@@Z 5f52c397 f   oleconn.obj
 0001:0002b4ba       ?GetConnections@CConnectionPoint@@QAEPBVCPtrArray@@XZ 5f52c4ba f   oleconn.obj
 0001:0002b512       ?OnAdvise@CConnectionPoint@@UAEXH@Z 5f52c512 f   oleconn.obj
 0001:0002b52f       ?GetMaxConnections@CConnectionPoint@@UAEHXZ 5f52c52f f   oleconn.obj
 0001:0002b54d       ?GetContainer@CConnectionPoint@@UAEPAUIConnectionPointContainer@@XZ 5f52c54d f   oleconn.obj
 0001:0002b5b0       ?CreateConnectionArray@CConnectionPoint@@QAEXXZ 5f52c5b0 f   oleconn.obj
 0001:0002b6bb       ?GetConnectionCount@CConnectionPoint@@QAEHXZ 5f52c6bb f   oleconn.obj
 0001:0002b6ee       ?QuerySinkInterface@CConnectionPoint@@UAEPAUIUnknown@@PAU2@@Z 5f52c6ee f   oleconn.obj
 0001:0002b722       ?Release@XConnPt@CConnectionPoint@@UAGKXZ 5f52c722 f   oleconn.obj
 0001:0002b73d       ?AddRef@XConnPt@CConnectionPoint@@UAGKXZ 5f52c73d f   oleconn.obj
 0001:0002b758       ?QueryInterface@XConnPt@CConnectionPoint@@UAGJABU_GUID@@PAPAX@Z 5f52c758 f   oleconn.obj
 0001:0002b7e3       ?GetConnectionInterface@XConnPt@CConnectionPoint@@UAGJPAU_GUID@@@Z 5f52c7e3 f   oleconn.obj
 0001:0002b84d       ?GetConnectionPointContainer@XConnPt@CConnectionPoint@@UAGJPAPAUIConnectionPointContainer@@@Z 5f52c84d f   oleconn.obj
 0001:0002b8b2       ?Advise@XConnPt@CConnectionPoint@@UAGJPAUIUnknown@@PAK@Z 5f52c8b2 f   oleconn.obj
 0001:0002b9da       ?Unadvise@XConnPt@CConnectionPoint@@UAGJK@Z 5f52c9da f   oleconn.obj
 0001:0002bac4       ?_GetBaseInterfaceMap@CEnumConnections@@KGPBUAFX_INTERFACEMAP@@XZ 5f52cac4 f   oleconn.obj
 0001:0002bace       ?GetInterfaceMap@CEnumConnections@@MBEPBUAFX_INTERFACEMAP@@XZ 5f52cace f   oleconn.obj
 0001:0002bade       ??0CEnumConnections@@QAE@PBXI@Z 5f52cade f   oleconn.obj
 0001:0002bb15       ??1CEnumConnections@@UAE@XZ 5f52cb15 f   oleconn.obj
 0001:0002bbc8       ?OnNext@CEnumConnections@@MAEHPAX@Z 5f52cbc8 f   oleconn.obj
 0001:0002bbfe       ?OnClone@CEnumConnections@@MAEPAVCEnumArray@@XZ 5f52cbfe f   oleconn.obj
 0001:0002bd08       ?AddConnection@CEnumConnections@@QAEXPAUtagCONNECTDATA@@@Z 5f52cd08 f   oleconn.obj
 0001:0002be31       ?EnumConnections@XConnPt@CConnectionPoint@@UAGJPAPAUIEnumConnections@@@Z 5f52ce31 f   oleconn.obj
 0001:0002c01b       ?_GetBaseInterfaceMap@CEnumConnPoints@@KGPBUAFX_INTERFACEMAP@@XZ 5f52d01b f   oleconn.obj
 0001:0002c025       ?GetInterfaceMap@CEnumConnPoints@@MBEPBUAFX_INTERFACEMAP@@XZ 5f52d025 f   oleconn.obj
 0001:0002c035       ??0CEnumConnPoints@@QAE@PBXI@Z 5f52d035 f   oleconn.obj
 0001:0002c06c       ??1CEnumConnPoints@@UAE@XZ 5f52d06c f   oleconn.obj
 0001:0002c11f       ?OnNext@CEnumConnPoints@@MAEHPAX@Z 5f52d11f f   oleconn.obj
 0001:0002c155       ?AddConnPoint@CEnumConnPoints@@QAEXPAUIConnectionPoint@@@Z 5f52d155 f   oleconn.obj
 0001:0002c271       ?AddRef@COleConnPtContainer@@UAGKXZ 5f52d271 f   oleconn.obj
 0001:0002c28c       ?Release@COleConnPtContainer@@UAGKXZ 5f52d28c f   oleconn.obj
 0001:0002c2a7       ?QueryInterface@COleConnPtContainer@@UAGJABU_GUID@@PAPAX@Z 5f52d2a7 f   oleconn.obj
 0001:0002c2ca       ?EnumConnectionPoints@COleConnPtContainer@@UAGJPAPAUIEnumConnectionPoints@@@Z 5f52d2ca f   oleconn.obj
 0001:0002c4d3       ?FindConnectionPoint@COleConnPtContainer@@UAGJABU_GUID@@PAPAUIConnectionPoint@@@Z 5f52d4d3 f   oleconn.obj
 0001:0002c5b9       ?EnableConnections@CCmdTarget@@QAEXXZ 5f52d5b9 f   oleconn.obj
 0001:0002c650       ??_ECConnectionPoint@@UAEPAXI@Z 5f52d650 f i oleconn.obj
 0001:0002c650       ??_GCConnectionPoint@@UAEPAXI@Z 5f52d650 f i oleconn.obj
 0001:0002c680       ??0XConnPt@CConnectionPoint@@QAE@XZ 5f52d680 f i oleconn.obj
 0001:0002c6a0       ??_GCEnumConnections@@UAEPAXI@Z 5f52d6a0 f i oleconn.obj
 0001:0002c6a0       ??_ECEnumConnections@@UAEPAXI@Z 5f52d6a0 f i oleconn.obj
 0001:0002c6d0       ??_ECEnumConnPoints@@UAEPAXI@Z 5f52d6d0 f i oleconn.obj
 0001:0002c6d0       ??_GCEnumConnPoints@@UAEPAXI@Z 5f52d6d0 f i oleconn.obj
 0001:0002c700       ??0COleConnPtContainer@@QAE@XZ 5f52d700 f i oleconn.obj
 0001:0002c720       ??4COleConnPtContainer@@QAEAAV0@ABV0@@Z 5f52d720 f i oleconn.obj
 0001:0002c740       ??4IConnectionPointContainer@@QAEAAU0@ABU0@@Z 5f52d740 f i oleconn.obj
 0001:0002c760       ?AddRef@XOleObject@COleControl@@UAGKXZ 5f52d760 f   ctlobj.obj
 0001:0002c77d       ?Release@XOleObject@COleControl@@UAGKXZ 5f52d77d f   ctlobj.obj
 0001:0002c79a       ?QueryInterface@XOleObject@COleControl@@UAGJABU_GUID@@PAPAX@Z 5f52d79a f   ctlobj.obj
 0001:0002c7bf       ?SetClientSite@XOleObject@COleControl@@UAGJPAUIOleClientSite@@@Z 5f52d7bf f   ctlobj.obj
 0001:0002cab2       ?GetClientSite@XOleObject@COleControl@@UAGJPAPAUIOleClientSite@@@Z 5f52dab2 f   ctlobj.obj
 0001:0002cb34       ?SetHostNames@XOleObject@COleControl@@UAGJPBG0@Z 5f52db34 f   ctlobj.obj
 0001:0002cb3d       ?Close@XOleObject@COleControl@@UAGJK@Z 5f52db3d f   ctlobj.obj
 0001:0002cbb4       ?OnClose@COleControl@@UAEXK@Z 5f52dbb4 f   ctlobj.obj
 0001:0002cc1d       ?SetMoniker@XOleObject@COleControl@@UAGJKPAUIMoniker@@@Z 5f52dc1d f   ctlobj.obj
 0001:0002cc29       ?GetMoniker@XOleObject@COleControl@@UAGJKKPAPAUIMoniker@@@Z 5f52dc29 f   ctlobj.obj
 0001:0002cc35       ?InitFromData@XOleObject@COleControl@@UAGJPAUIDataObject@@HK@Z 5f52dc35 f   ctlobj.obj
 0001:0002cc41       ?GetClipboardData@XOleObject@COleControl@@UAGJKPAPAUIDataObject@@@Z 5f52dc41 f   ctlobj.obj
 0001:0002cc4d       ?DoVerb@XOleObject@COleControl@@UAGJJPAUtagMSG@@PAUIOleClientSite@@JPAUHWND__@@PBUtagRECT@@@Z 5f52dc4d f   ctlobj.obj
 0001:0002cf73       ?OnDoVerb@COleControl@@UAEHJPAUtagMSG@@PAUHWND__@@PBUtagRECT@@@Z 5f52df73 f   ctlobj.obj
 0001:0002cf98       ?EnumVerbs@XOleObject@COleControl@@UAGJPAPAUIEnumOLEVERB@@@Z 5f52df98 f   ctlobj.obj
 0001:0002d019       ?OnEnumVerbs@COleControl@@UAEHPAPAUIEnumOLEVERB@@@Z 5f52e019 f   ctlobj.obj
 0001:0002d032       ?Update@XOleObject@COleControl@@UAGJXZ 5f52e032 f   ctlobj.obj
 0001:0002d03b       ?IsUpToDate@XOleObject@COleControl@@UAGJXZ 5f52e03b f   ctlobj.obj
 0001:0002d044       ?GetUserClassID@XOleObject@COleControl@@UAGJPAU_GUID@@@Z 5f52e044 f   ctlobj.obj
 0001:0002d06b       ?GetUserType@XOleObject@COleControl@@UAGJKPAPAG@Z 5f52e06b f   ctlobj.obj
 0001:0002d139       ?GetUserType@COleControl@@IAEXPAD@Z 5f52e139 f   ctlobj.obj
 0001:0002d204       ?SetExtent@XOleObject@COleControl@@UAGJKPAUtagSIZE@@@Z 5f52e204 f   ctlobj.obj
 0001:0002d24a       ?OnSetExtent@COleControl@@UAEHPAUtagSIZE@@@Z 5f52e24a f   ctlobj.obj
 0001:0002d3b6       ?GetExtent@XOleObject@COleControl@@UAGJKPAUtagSIZE@@@Z 5f52e3b6 f   ctlobj.obj
 0001:0002d3fb       ?Advise@XOleObject@COleControl@@UAGJPAUIAdviseSink@@PAK@Z 5f52e3fb f   ctlobj.obj
 0001:0002d45c       ?Unadvise@XOleObject@COleControl@@UAGJK@Z 5f52e45c f   ctlobj.obj
 0001:0002d4a0       ?EnumAdvise@XOleObject@COleControl@@UAGJPAPAUIEnumSTATDATA@@@Z 5f52e4a0 f   ctlobj.obj
 0001:0002d4e4       ?GetMiscStatus@XOleObject@COleControl@@UAGJKPAK@Z 5f52e4e4 f   ctlobj.obj
 0001:0002d556       ?SetColorScheme@XOleObject@COleControl@@UAGJPAUtagLOGPALETTE@@@Z 5f52e556 f   ctlobj.obj
 0001:0002d570       ??0CPictureHolder@@QAE@XZ  5f52e570 f   ctlpict.obj
 0001:0002d587       ??1CPictureHolder@@QAE@XZ  5f52e587 f   ctlpict.obj
 0001:0002d5b9       ?CreateEmpty@CPictureHolder@@QAEHXZ 5f52e5b9 f   ctlpict.obj
 0001:0002d619       ?CreateFromBitmap@CPictureHolder@@QAEHI@Z 5f52e619 f   ctlpict.obj
 0001:0002d68c       ?CreateFromBitmap@CPictureHolder@@QAEHPAVCBitmap@@PAVCPalette@@H@Z 5f52e68c f   ctlpict.obj
 0001:0002d6e7       ?CreateFromBitmap@CPictureHolder@@QAEHPAUHBITMAP__@@PAUHPALETTE__@@H@Z 5f52e6e7 f   ctlpict.obj
 0001:0002d757       ?CreateFromMetafile@CPictureHolder@@QAEHPAUHMETAFILE__@@HHH@Z 5f52e757 f   ctlpict.obj
 0001:0002d7cd       ?CreateFromIcon@CPictureHolder@@QAEHI@Z 5f52e7cd f   ctlpict.obj
 0001:0002d7fd       ?CreateFromIcon@CPictureHolder@@QAEHPAUHICON__@@H@Z 5f52e7fd f   ctlpict.obj
 0001:0002d867       ?GetPictureDispatch@CPictureHolder@@QAEPAUIPictureDisp@@XZ 5f52e867 f   ctlpict.obj
 0001:0002d8c5       ?SetPictureDispatch@CPictureHolder@@QAEXPAUIPictureDisp@@@Z 5f52e8c5 f   ctlpict.obj
 0001:0002d94a       ?Render@CPictureHolder@@QAEXPAVCDC@@ABVCRect@@1@Z 5f52e94a f   ctlpict.obj
 0001:0002d9db       ?GetType@CPictureHolder@@QAEFXZ 5f52e9db f   ctlpict.obj
 0001:0002da0e       ?GetDisplayString@CPictureHolder@@QAEHAAVCString@@@Z 5f52ea0e f   ctlpict.obj
 0001:0002db40       ?_AfxGetArchiveStream@@YGPAUIStream@@AAVCArchive@@AAVCArchiveStream@@@Z 5f52eb40 f   ctlpropx.obj
 0001:0002dbf8       ?_AfxInitBlob@@YGHPAPAXPAX@Z 5f52ebf8 f   ctlpropx.obj
 0001:0002dcc5       ?_AfxCopyBlob@@YGHPAPAXPAX@Z 5f52ecc5 f   ctlpropx.obj
 0001:0002dd08       ?_AfxCopyPropValue@@YGHGPAXPBX@Z 5f52ed08 f   ctlpropx.obj
 0001:0002de73       ?ExchangeExtent@COleControl@@QAEHPAVCPropExchange@@@Z 5f52ee73 f   ctlpropx.obj
 0001:0002df19       ?SerializeVersion@COleControl@@QAEKAAVCArchive@@KH@Z 5f52ef19 f   ctlpropx.obj
 0001:0002df7a       ?ResetVersion@COleControl@@QAEXK@Z 5f52ef7a f   ctlpropx.obj
 0001:0002df90       ?SerializeExtent@COleControl@@QAEXAAVCArchive@@@Z 5f52ef90 f   ctlpropx.obj
 0001:0002e021       ?ExchangeVersion@CPropExchange@@UAEHAAKKH@Z 5f52f021 f   ctlpropx.obj
 0001:0002e0a2       ??0CArchivePropExchange@@QAE@AAVCArchive@@@Z 5f52f0a2 f   ctlpropx.obj
 0001:0002e114       ?ExchangeProp@CArchivePropExchange@@UAEHPBDGPAXPBX@Z 5f52f114 f   ctlpropx.obj
 0001:0002e403       ?ExchangeBlobProp@CArchivePropExchange@@UAEHPBDPAPAXPAX@Z 5f52f403 f   ctlpropx.obj
 0001:0002e5dc       ?_AfxPeekAtClassIDInStream@@YGHPAUIStream@@PAU_GUID@@@Z 5f52f5dc f   ctlpropx.obj
 0001:0002e637       ?_AfxIsSameUnknownObject@@YGHABU_GUID@@PAUIUnknown@@1@Z 5f52f637 f   ctlpropx.obj
 0001:0002e740       ?ExchangePersistentProp@CArchivePropExchange@@UAEHPBDPAPAUIUnknown@@ABU_GUID@@PAU2@@Z 5f52f740 f   ctlpropx.obj
 0001:0002ebe7       ?ExchangeFontProp@CArchivePropExchange@@UAEHPBDAAVCFontHolder@@PBUtagFONTDESC@@PAUIFontDisp@@@Z 5f52fbe7 f   ctlpropx.obj
 0001:0002ee43       ??0CResetPropExchange@@QAE@XZ 5f52fe43 f   ctlpropx.obj
 0001:0002ee6c       ?ExchangeProp@CResetPropExchange@@UAEHPBDGPAXPBX@Z 5f52fe6c f   ctlpropx.obj
 0001:0002ef16       ?ExchangeBlobProp@CResetPropExchange@@UAEHPBDPAPAXPAX@Z 5f52ff16 f   ctlpropx.obj
 0001:0002efc2       ?ExchangePersistentProp@CResetPropExchange@@UAEHPBDPAPAUIUnknown@@ABU_GUID@@PAU2@@Z 5f52ffc2 f   ctlpropx.obj
 0001:0002f0b6       ?ExchangeFontProp@CResetPropExchange@@UAEHPBDAAVCFontHolder@@PBUtagFONTDESC@@PAUIFontDisp@@@Z 5f5300b6 f   ctlpropx.obj
 0001:0002f19a       ??0CAsyncPropExchange@@QAE@K@Z 5f53019a f   ctlpropx.obj
 0001:0002f1d8       ?ExchangeVersion@CAsyncPropExchange@@UAEHAAKKH@Z 5f5301d8 f   ctlpropx.obj
 0001:0002f226       ?ExchangeProp@CAsyncPropExchange@@UAEHPBDGPAXPBX@Z 5f530226 f   ctlpropx.obj
 0001:0002f25e       ?ExchangeBlobProp@CAsyncPropExchange@@UAEHPBDPAPAXPAX@Z 5f53025e f   ctlpropx.obj
 0001:0002f296       ?ExchangeFontProp@CAsyncPropExchange@@UAEHPBDAAVCFontHolder@@PBUtagFONTDESC@@PAUIFontDisp@@@Z 5f530296 f   ctlpropx.obj
 0001:0002f2ce       ?ExchangePersistentProp@CAsyncPropExchange@@UAEHPBDPAPAUIUnknown@@ABU_GUID@@PAU2@@Z 5f5302ce f   ctlpropx.obj
 0001:0002f306       ?PX_Short@@YAHPAVCPropExchange@@PBDAAF@Z 5f530306 f   ctlpropx.obj
 0001:0002f3c6       ?PX_Short@@YAHPAVCPropExchange@@PBDAAFF@Z 5f5303c6 f   ctlpropx.obj
 0001:0002f488       ?PX_UShort@@YAHPAVCPropExchange@@PBDAAG@Z 5f530488 f   ctlpropx.obj
 0001:0002f548       ?PX_UShort@@YAHPAVCPropExchange@@PBDAAGG@Z 5f530548 f   ctlpropx.obj
 0001:0002f60a       ?PX_Long@@YAHPAVCPropExchange@@PBDAAJ@Z 5f53060a f   ctlpropx.obj
 0001:0002f6ca       ?PX_Long@@YAHPAVCPropExchange@@PBDAAJJ@Z 5f5306ca f   ctlpropx.obj
 0001:0002f78c       ?PX_ULong@@YAHPAVCPropExchange@@PBDAAK@Z 5f53078c f   ctlpropx.obj
 0001:0002f84c       ?PX_ULong@@YAHPAVCPropExchange@@PBDAAKK@Z 5f53084c f   ctlpropx.obj
 0001:0002f90e       ?PX_Color@@YAHPAVCPropExchange@@PBDAAK@Z 5f53090e f   ctlpropx.obj
 0001:0002f9ce       ?PX_Color@@YAHPAVCPropExchange@@PBDAAKK@Z 5f5309ce f   ctlpropx.obj
 0001:0002fa90       ?PX_Bool@@YAHPAVCPropExchange@@PBDAAH@Z 5f530a90 f   ctlpropx.obj
 0001:0002fb50       ?PX_Bool@@YAHPAVCPropExchange@@PBDAAHH@Z 5f530b50 f   ctlpropx.obj
 0001:0002fc12       ?PX_String@@YAHPAVCPropExchange@@PBDAAVCString@@@Z 5f530c12 f   ctlpropx.obj
 0001:0002fcd2       ?PX_String@@YAHPAVCPropExchange@@PBDAAVCString@@ABV2@@Z 5f530cd2 f   ctlpropx.obj
 0001:0002fd94       ?PX_String@@YAHPAVCPropExchange@@PBDAAVCString@@1@Z 5f530d94 f   ctlpropx.obj
 0001:0002fe56       ?PX_Currency@@YAHPAVCPropExchange@@PBDAATtagCY@@@Z 5f530e56 f   ctlpropx.obj
 0001:0002ff16       ?PX_Currency@@YAHPAVCPropExchange@@PBDAATtagCY@@T2@@Z 5f530f16 f   ctlpropx.obj
 0001:0002ffd8       ?PX_Float@@YAHPAVCPropExchange@@PBDAAM@Z 5f530fd8 f   ctlpropx.obj
 0001:00030098       ?PX_Float@@YAHPAVCPropExchange@@PBDAAMM@Z 5f531098 f   ctlpropx.obj
 0001:0003015a       ?PX_Double@@YAHPAVCPropExchange@@PBDAAN@Z 5f53115a f   ctlpropx.obj
 0001:0003021a       ?PX_Double@@YAHPAVCPropExchange@@PBDAANN@Z 5f53121a f   ctlpropx.obj
 0001:000302dc       ?PX_Blob@@YAHPAVCPropExchange@@PBDAAPAXPAX@Z 5f5312dc f   ctlpropx.obj
 0001:0003039c       ?PX_Font@@YAHPAVCPropExchange@@PBDAAVCFontHolder@@PBUtagFONTDESC@@PAUIFontDisp@@@Z 5f53139c f   ctlpropx.obj
 0001:000304c2       ?PX_IUnknown@@YAHPAVCPropExchange@@PBDAAPAUIUnknown@@ABU_GUID@@PAU2@@Z 5f5314c2 f   ctlpropx.obj
 0001:000305ec       ?PX_Picture@@YAHPAVCPropExchange@@PBDAAVCPictureHolder@@@Z 5f5315ec f   ctlpropx.obj
 0001:000306b9       ?PX_Picture@@YAHPAVCPropExchange@@PBDAAVCPictureHolder@@2@Z 5f5316b9 f   ctlpropx.obj
 0001:0003078a       ?PX_VBXFontConvert@@YAHPAVCPropExchange@@AAVCFontHolder@@@Z 5f53178a f   ctlpropx.obj
 0001:000309f8       ?_Afx_PX_DataPath@@YGHPAVCPropExchange@@PBDAAVCDataPathProperty@@GPBX@Z 5f5319f8 f   ctlpropx.obj
 0001:00030c1c       ?PX_DataPath@@YAHPAVCPropExchange@@PBDAAVCDataPathProperty@@1@Z 5f531c1c f   ctlpropx.obj
 0001:00030c38       ?PX_DataPath@@YAHPAVCPropExchange@@PBDAAVCDataPathProperty@@ABVCString@@@Z 5f531c38 f   ctlpropx.obj
 0001:00030c60       ?_GetBaseInterfaceMap@COlePropertyPage@@KGPBUAFX_INTERFACEMAP@@XZ 5f531c60 f   ctlppg.obj
 0001:00030c6a       ?GetInterfaceMap@COlePropertyPage@@MBEPBUAFX_INTERFACEMAP@@XZ 5f531c6a f   ctlppg.obj
 0001:00030c7a       ?_GetBaseMessageMap@COlePropertyPage@@KGPBUAFX_MSGMAP@@XZ 5f531c7a f   ctlppg.obj
 0001:00030c84       ?GetMessageMap@COlePropertyPage@@MBEPBUAFX_MSGMAP@@XZ 5f531c84 f   ctlppg.obj
 0001:00030c94       ??0AFX_DDPDATA@@QAE@PAXHH0IPBD@Z 5f531c94 f   ctlppg.obj
 0001:00030ceb       ?_AfxCleanupDDPs@@YGXAAVCPtrArray@@@Z 5f531ceb f   ctlppg.obj
 0001:00030d8a       ?_ValidatePageDialog@@YAXAAVCDialogTemplate@@AAVCString@@PAVCOlePropertyPage@@@Z 5f531d8a f   ctlppg.obj
 0001:0003102a       ??0COlePropertyPage@@QAE@II@Z 5f53202a f   ctlppg.obj
 0001:000311aa       ?OnSetPageSite@COlePropertyPage@@UAEXXZ 5f5321aa f   ctlppg.obj
 0001:000313a2       ?OnInitDialog@COlePropertyPage@@UAEHXZ 5f5323a2 f   ctlppg.obj
 0001:000313b7       ?PreTranslateMessage@COlePropertyPage@@MAEHPAUtagMSG@@@Z 5f5323b7 f   ctlppg.obj
 0001:000314e6       ?CleanupObjectArray@COlePropertyPage@@IAEXXZ 5f5324e6 f   ctlppg.obj
 0001:00031622       ??1COlePropertyPage@@UAE@XZ 5f532622 f   ctlppg.obj
 0001:00031761       ?OnFinalRelease@COlePropertyPage@@MAEXXZ 5f532761 f   ctlppg.obj
 0001:000317ad       ?WindowProc@COlePropertyPage@@MAEJIIJ@Z 5f5327ad f   ctlppg.obj
 0001:0003187d       ?OnCtlColor@COlePropertyPage@@IAEPAUHBRUSH__@@PAVCDC@@PAVCWnd@@I@Z 5f53287d f   ctlppg.obj
 0001:000318ef       ?OnHelp@COlePropertyPage@@UAEHPBD@Z 5f5328ef f   ctlppg.obj
 0001:000318fe       ?OnEditProperty@COlePropertyPage@@UAEHJ@Z 5f5328fe f   ctlppg.obj
 0001:0003190d       ?OnObjectsChanged@COlePropertyPage@@UAEXXZ 5f53290d f   ctlppg.obj
 0001:00031918       ?GetObjectArray@COlePropertyPage@@QAEPAPAUIDispatch@@PAK@Z 5f532918 f   ctlppg.obj
 0001:00031979       ?SetModifiedFlag@COlePropertyPage@@QAEXH@Z 5f532979 f   ctlppg.obj
 0001:000319ff       ?IsModified@COlePropertyPage@@QAEHXZ 5f5329ff f   ctlppg.obj
 0001:00031a10       ?SetPageName@COlePropertyPage@@QAEXPBD@Z 5f532a10 f   ctlppg.obj
 0001:00031a5e       ?SetDialogResource@COlePropertyPage@@QAEXPAX@Z 5f532a5e f   ctlppg.obj
 0001:00031b13       ?SetHelpInfo@COlePropertyPage@@QAEXPBD0K@Z 5f532b13 f   ctlppg.obj
 0001:00031bb4       ?GetPageSite@COlePropertyPage@@QAEPAUIPropertyPageSite@@XZ 5f532bb4 f   ctlppg.obj
 0001:00031bc8       ?MessageBoxA@COlePropertyPage@@QAEHPBD0I@Z 5f532bc8 f   ctlppg.obj
 0001:00031c0d       ?AddRef@XPropertyPage@COlePropertyPage@@UAGKXZ 5f532c0d f   ctlppg.obj
 0001:00031c2a       ?Release@XPropertyPage@COlePropertyPage@@UAGKXZ 5f532c2a f   ctlppg.obj
 0001:00031c47       ?QueryInterface@XPropertyPage@COlePropertyPage@@UAGJABU_GUID@@PAPAX@Z 5f532c47 f   ctlppg.obj
 0001:00031c6c       ?SetPageSite@XPropertyPage@COlePropertyPage@@UAGJPAUIPropertyPageSite@@@Z 5f532c6c f   ctlppg.obj
 0001:00031d8a       ?Activate@XPropertyPage@COlePropertyPage@@UAGJPAUHWND__@@PBUtagRECT@@H@Z 5f532d8a f   ctlppg.obj
 0001:00031fdf       ?EnumChildProc@COlePropertyPage@@KGHPAUHWND__@@J@Z 5f532fdf f   ctlppg.obj
 0001:00032043       ?EnumControls@COlePropertyPage@@KGHPAUHWND__@@J@Z 5f533043 f   ctlppg.obj
 0001:00032106       ?Deactivate@XPropertyPage@COlePropertyPage@@UAGJXZ 5f533106 f   ctlppg.obj
 0001:00032176       ?GetPageInfo@XPropertyPage@COlePropertyPage@@UAGJPAUtagPROPPAGEINFO@@@Z 5f533176 f   ctlppg.obj
 0001:00032239       ?SetObjects@XPropertyPage@COlePropertyPage@@UAGJKPAPAUIUnknown@@@Z 5f533239 f   ctlppg.obj
 0001:00032479       ?Show@XPropertyPage@COlePropertyPage@@UAGJI@Z 5f533479 f   ctlppg.obj
 0001:000324aa       ?Move@XPropertyPage@COlePropertyPage@@UAGJPBUtagRECT@@@Z 5f5334aa f   ctlppg.obj
 0001:00032506       ?IsPageDirty@XPropertyPage@COlePropertyPage@@UAGJXZ 5f533506 f   ctlppg.obj
 0001:00032527       ?Apply@XPropertyPage@COlePropertyPage@@UAGJXZ 5f533527 f   ctlppg.obj
 0001:00032681       ?Help@XPropertyPage@COlePropertyPage@@UAGJPBG@Z 5f533681 f   ctlppg.obj
 0001:000327c8       ?_AfxAtEndOfTabList@@YGHPAVCDialog@@I@Z 5f5337c8 f   ctlppg.obj
 0001:00032861       ?TranslateAcceleratorA@XPropertyPage@COlePropertyPage@@UAGJPAUtagMSG@@@Z 5f533861 f   ctlppg.obj
 0001:00032ac6       ?EditProperty@XPropertyPage@COlePropertyPage@@UAGJJ@Z 5f533ac6 f   ctlppg.obj
 0001:00032b5a       ?AddRef@XPropNotifySink@COlePropertyPage@@UAGKXZ 5f533b5a f   ctlppg.obj
 0001:00032b66       ?Release@XPropNotifySink@COlePropertyPage@@UAGKXZ 5f533b66 f   ctlppg.obj
 0001:00032b6f       ?QueryInterface@XPropNotifySink@COlePropertyPage@@UAGJABU_GUID@@PAPAX@Z 5f533b6f f   ctlppg.obj
 0001:00032bba       ?OnRequestEdit@XPropNotifySink@COlePropertyPage@@UAGJJ@Z 5f533bba f   ctlppg.obj
 0001:00032bc3       ?OnChanged@XPropNotifySink@COlePropertyPage@@UAGJJ@Z 5f533bc3 f   ctlppg.obj
 0001:00032c63       ?_AfxIsRadioButton@@YGHPAUHWND__@@@Z 5f533c63 f   ctlppg.obj
 0001:00032ca0       ?OnCommand@COlePropertyPage@@MAEHIJ@Z 5f533ca0 f   ctlppg.obj
 0001:00032fb3       ?IgnoreApply@COlePropertyPage@@QAEXI@Z 5f533fb3 f   ctlppg.obj
 0001:00032fd2       ?GetControlStatus@COlePropertyPage@@QAEHI@Z 5f533fd2 f   ctlppg.obj
 0001:0003302e       ?SetControlStatus@COlePropertyPage@@QAEHIH@Z 5f53402e f   ctlppg.obj
 0001:0003308f       ?SetPropText@COlePropertyPage@@QAEHPBDAAE@Z 5f53408f f   ctlppg.obj
 0001:00033200       ?GetPropText@COlePropertyPage@@QAEHPBDPAE@Z 5f534200 f   ctlppg.obj
 0001:00033396       ?SetPropText@COlePropertyPage@@QAEHPBDAAF@Z 5f534396 f   ctlppg.obj
 0001:00033506       ?GetPropText@COlePropertyPage@@QAEHPBDPAF@Z 5f534506 f   ctlppg.obj
 0001:0003369a       ?SetPropText@COlePropertyPage@@QAEHPBDAAH@Z 5f53469a f   ctlppg.obj
 0001:00033809       ?GetPropText@COlePropertyPage@@QAEHPBDPAH@Z 5f534809 f   ctlppg.obj
 0001:00033994       ?SetPropText@COlePropertyPage@@QAEHPBDAAI@Z 5f534994 f   ctlppg.obj
 0001:00033b03       ?GetPropText@COlePropertyPage@@QAEHPBDPAI@Z 5f534b03 f   ctlppg.obj
 0001:00033c8e       ?SetPropText@COlePropertyPage@@QAEHPBDAAJ@Z 5f534c8e f   ctlppg.obj
 0001:00033dfd       ?GetPropText@COlePropertyPage@@QAEHPBDPAJ@Z 5f534dfd f   ctlppg.obj
 0001:00033f88       ?SetPropText@COlePropertyPage@@QAEHPBDAAK@Z 5f534f88 f   ctlppg.obj
 0001:000340f7       ?GetPropText@COlePropertyPage@@QAEHPBDPAK@Z 5f5350f7 f   ctlppg.obj
 0001:00034282       ?SetPropText@COlePropertyPage@@QAEHPBDAAM@Z 5f535282 f   ctlppg.obj
 0001:000343f6       ?GetPropText@COlePropertyPage@@QAEHPBDPAM@Z 5f5353f6 f   ctlppg.obj
 0001:00034587       ?SetPropText@COlePropertyPage@@QAEHPBDAAN@Z 5f535587 f   ctlppg.obj
 0001:000346fa       ?GetPropText@COlePropertyPage@@QAEHPBDPAN@Z 5f5356fa f   ctlppg.obj
 0001:00034899       ?SetPropText@COlePropertyPage@@QAEHPBDAAVCString@@@Z 5f535899 f   ctlppg.obj
 0001:00034a0b       ?GetPropText@COlePropertyPage@@QAEHPBDPAVCString@@@Z 5f535a0b f   ctlppg.obj
 0001:00034c09       ?SetPropCheck@COlePropertyPage@@QAEHPBDH@Z 5f535c09 f   ctlppg.obj
 0001:00034d8c       ?GetPropCheck@COlePropertyPage@@QAEHPBDPAH@Z 5f535d8c f   ctlppg.obj
 0001:00034f33       ?SetPropRadio@COlePropertyPage@@QAEHPBDH@Z 5f535f33 f   ctlppg.obj
 0001:000350a9       ?GetPropRadio@COlePropertyPage@@QAEHPBDPAH@Z 5f5360a9 f   ctlppg.obj
 0001:00035235       ?SetPropIndex@COlePropertyPage@@QAEHPBDH@Z 5f536235 f   ctlppg.obj
 0001:00035252       ?GetPropIndex@COlePropertyPage@@QAEHPBDPAH@Z 5f536252 f   ctlppg.obj
 0001:0003526f       ?DDP_EndText@@YGXPAVCDataExchange@@HPAEPBD@Z 5f53626f f   ctlppg.obj
 0001:000352a8       ?DDP_Text@@YGXPAVCDataExchange@@HAAEPBD@Z 5f5362a8 f   ctlppg.obj
 0001:000353cd       ?DDP_EndText@@YGXPAVCDataExchange@@HPAFPBD@Z 5f5363cd f   ctlppg.obj
 0001:00035406       ?DDP_Text@@YGXPAVCDataExchange@@HAAFPBD@Z 5f536406 f   ctlppg.obj
 0001:0003552b       ?DDP_EndText@@YGXPAVCDataExchange@@HPAHPBD@Z 5f53652b f   ctlppg.obj
 0001:00035564       ?DDP_Text@@YGXPAVCDataExchange@@HAAHPBD@Z 5f536564 f   ctlppg.obj
 0001:00035689       ?DDP_EndText@@YGXPAVCDataExchange@@HPAIPBD@Z 5f536689 f   ctlppg.obj
 0001:000356c2       ?DDP_Text@@YGXPAVCDataExchange@@HAAIPBD@Z 5f5366c2 f   ctlppg.obj
 0001:000357e7       ?DDP_EndText@@YGXPAVCDataExchange@@HPAJPBD@Z 5f5367e7 f   ctlppg.obj
 0001:00035820       ?DDP_Text@@YGXPAVCDataExchange@@HAAJPBD@Z 5f536820 f   ctlppg.obj
 0001:00035945       ?DDP_EndText@@YGXPAVCDataExchange@@HPAKPBD@Z 5f536945 f   ctlppg.obj
 0001:0003597e       ?DDP_Text@@YGXPAVCDataExchange@@HAAKPBD@Z 5f53697e f   ctlppg.obj
 0001:00035aa3       ?DDP_EndText@@YGXPAVCDataExchange@@HPAMPBD@Z 5f536aa3 f   ctlppg.obj
 0001:00035adc       ?DDP_Text@@YGXPAVCDataExchange@@HAAMPBD@Z 5f536adc f   ctlppg.obj
 0001:00035c01       ?DDP_EndText@@YGXPAVCDataExchange@@HPANPBD@Z 5f536c01 f   ctlppg.obj
 0001:00035c3a       ?DDP_Text@@YGXPAVCDataExchange@@HAANPBD@Z 5f536c3a f   ctlppg.obj
 0001:00035d5f       ?DDP_EndText@@YGXPAVCDataExchange@@HPAVCString@@PBD@Z 5f536d5f f   ctlppg.obj
 0001:00035d98       ?DDP_Text@@YGXPAVCDataExchange@@HAAVCString@@PBD@Z 5f536d98 f   ctlppg.obj
 0001:00035ebd       ?DDP_EndCheck@@YGXPAVCDataExchange@@HPAHPBD@Z 5f536ebd f   ctlppg.obj
 0001:00035ef8       ?DDP_Check@@YGXPAVCDataExchange@@HAAHPBD@Z 5f536ef8 f   ctlppg.obj
 0001:0003601d       ?DDP_EndRadio@@YGXPAVCDataExchange@@HPAHPBD@Z 5f53701d f   ctlppg.obj
 0001:00036058       ?DDP_Radio@@YGXPAVCDataExchange@@HAAHPBD@Z 5f537058 f   ctlppg.obj
 0001:0003617d       ?DDP_PostProcessing@@YGXPAVCDataExchange@@@Z 5f53717d f   ctlppg.obj
 0001:000364e0       ??_EAFX_DDPDATA@@UAEPAXI@Z 5f5374e0 f i ctlppg.obj
 0001:000364e0       ??_GAFX_DDPDATA@@UAEPAXI@Z 5f5374e0 f i ctlppg.obj
 0001:00036510       ??1AFX_DDPDATA@@UAE@XZ     5f537510 f i ctlppg.obj
 0001:00036530       ??_GCOlePropertyPage@@UAEPAXI@Z 5f537530 f i ctlppg.obj
 0001:00036530       ??_ECOlePropertyPage@@UAEPAXI@Z 5f537530 f i ctlppg.obj
 0001:00036560       ??0XPropertyPage@COlePropertyPage@@QAE@XZ 5f537560 f i ctlppg.obj
 0001:00036580       ??0XPropNotifySink@COlePropertyPage@@QAE@XZ 5f537580 f i ctlppg.obj
 0001:000365a0       ?InitStockPropMask@COleControl@@IAEXXZ 5f5375a0 f   ctlprop.obj
 0001:00036682       ?_AfxToggleBorderStyle@@YGXPAVCWnd@@@Z 5f537682 f   ctlprop.obj
 0001:000366c8       ?_AfxToggleAppearance@@YGXPAVCWnd@@@Z 5f5376c8 f   ctlprop.obj
 0001:0003670e       ?ExchangeStockProps@COleControl@@QAEXPAVCPropExchange@@@Z 5f53770e f   ctlprop.obj
 0001:00036b13       ?SerializeStockProps@COleControl@@QAEXAAVCArchive@@@Z 5f537b13 f   ctlprop.obj
 0001:000370df       ?ResetStockProps@COleControl@@QAEXXZ 5f5380df f   ctlprop.obj
 0001:0003725a       ?GetAppearance@COleControl@@QAEFXZ 5f53825a f   ctlprop.obj
 0001:0003726f       ?SetAppearance@COleControl@@QAEXF@Z 5f53826f f   ctlprop.obj
 0001:00037366       ?OnAppearanceChanged@COleControl@@UAEXXZ 5f538366 f   ctlprop.obj
 0001:0003737d       ?GetBackColor@COleControl@@QAEKXZ 5f53837d f   ctlprop.obj
 0001:00037391       ?SetBackColor@COleControl@@QAEXK@Z 5f538391 f   ctlprop.obj
 0001:00037428       ?OnBackColorChanged@COleControl@@UAEXXZ 5f538428 f   ctlprop.obj
 0001:0003743f       ?GetBorderStyle@COleControl@@QAEFXZ 5f53843f f   ctlprop.obj
 0001:00037454       ?SetBorderStyle@COleControl@@QAEXF@Z 5f538454 f   ctlprop.obj
 0001:0003754b       ?OnBorderStyleChanged@COleControl@@UAEXXZ 5f53854b f   ctlprop.obj
 0001:00037562       ?InternalGetText@COleControl@@QAEABVCString@@XZ 5f538562 f   ctlprop.obj
 0001:0003761a       ?GetText@COleControl@@QAEPAGXZ 5f53861a f   ctlprop.obj
 0001:00037634       ?SetText@COleControl@@QAEXPBD@Z 5f538634 f   ctlprop.obj
 0001:00037680       ?OnSetText@COleControl@@IAEJIJ@Z 5f538680 f   ctlprop.obj
 0001:0003786a       ?OnTextChanged@COleControl@@UAEXXZ 5f53886a f   ctlprop.obj
 0001:00037881       ?GetEnabled@COleControl@@QAEHXZ 5f538881 f   ctlprop.obj
 0001:00037895       ?SetEnabled@COleControl@@QAEXH@Z 5f538895 f   ctlprop.obj
 0001:00037959       ?OnEnabledChanged@COleControl@@UAEXXZ 5f538959 f   ctlprop.obj
 0001:00037970       ?InternalGetFont@COleControl@@QAEAAVCFontHolder@@XZ 5f538970 f   ctlprop.obj
 0001:00037983       ?GetFont@COleControl@@QAEPAUIFontDisp@@XZ 5f538983 f   ctlprop.obj
 0001:0003799c       ?SetFont@COleControl@@QAEXPAUIFontDisp@@@Z 5f53899c f   ctlprop.obj
 0001:00037a24       ?OnFontChanged@COleControl@@UAEXXZ 5f538a24 f   ctlprop.obj
 0001:00037b41       ?GetForeColor@COleControl@@QAEKXZ 5f538b41 f   ctlprop.obj
 0001:00037b55       ?SetForeColor@COleControl@@QAEXK@Z 5f538b55 f   ctlprop.obj
 0001:00037bec       ?OnForeColorChanged@COleControl@@UAEXXZ 5f538bec f   ctlprop.obj
 0001:00037c03       ?GetHwnd@COleControl@@QAEIXZ 5f538c03 f   ctlprop.obj
 0001:00037c4b       ?GetReadyState@COleControl@@QAEJXZ 5f538c4b f   ctlprop.obj
 0001:00037c5f       ?AddRef@XFontNotification@COleControl@@UAGKXZ 5f538c5f f   ctlprop.obj
 0001:00037c6b       ?Release@XFontNotification@COleControl@@UAGKXZ 5f538c6b f   ctlprop.obj
 0001:00037c74       ?QueryInterface@XFontNotification@COleControl@@UAGJABU_GUID@@PAPAX@Z 5f538c74 f   ctlprop.obj
 0001:00037cdc       ?OnChanged@XFontNotification@COleControl@@UAGJJ@Z 5f538cdc f   ctlprop.obj
 0001:00037d71       ?OnRequestEdit@XFontNotification@COleControl@@UAGJJ@Z 5f538d71 f   ctlprop.obj
 0001:00037d7a       ?SelectStockFont@COleControl@@QAEPAVCFont@@PAVCDC@@@Z 5f538d7a f   ctlprop.obj
 0001:00037d9c       ?SelectFontObject@COleControl@@QAEPAVCFont@@PAVCDC@@AAVCFontHolder@@@Z 5f538d9c f   ctlprop.obj
 0001:00037dcb       ?GetStockTextMetrics@COleControl@@QAEXPAUtagTEXTMETRICA@@@Z 5f538dcb f   ctlprop.obj
 0001:00037dea       ?GetFontTextMetrics@COleControl@@QAEXPAUtagTEXTMETRICA@@AAVCFontHolder@@@Z 5f538dea f   ctlprop.obj
 0001:00037e03       ?_GetI4Property@@YGHPAUIDispatch@@JPAK@Z 5f538e03 f   ctlprop.obj
 0001:00037eed       ?GetAmbientDispatchDriver@COleControl@@IAEPAVCOleDispatchDriver@@XZ 5f538eed f   ctlprop.obj
 0001:00037f77       ?GetAmbientProperty@COleControl@@QAEHJGPAX@Z 5f538f77 f   ctlprop.obj
 0001:000381d3       ?AmbientAppearance@COleControl@@QAEFXZ 5f5391d3 f   ctlprop.obj
 0001:00038202       ?AmbientBackColor@COleControl@@QAEKXZ 5f539202 f   ctlprop.obj
 0001:00038234       ?AmbientDisplayName@COleControl@@QAE?AVCString@@XZ 5f539234 f   ctlprop.obj
 0001:000382af       ?AmbientFont@COleControl@@QAEPAUIFontDisp@@XZ 5f5392af f   ctlprop.obj
 0001:000382dd       ?AmbientForeColor@COleControl@@QAEKXZ 5f5392dd f   ctlprop.obj
 0001:0003830f       ?AmbientLocaleID@COleControl@@QAEKXZ 5f53930f f   ctlprop.obj
 0001:0003833d       ?AmbientScaleUnits@COleControl@@QAE?AVCString@@XZ 5f53933d f   ctlprop.obj
 0001:000383b8       ?AmbientTextAlign@COleControl@@QAEFXZ 5f5393b8 f   ctlprop.obj
 0001:000383e6       ?AmbientUserMode@COleControl@@QAEHXZ 5f5393e6 f   ctlprop.obj
 0001:00038414       ?AmbientUIDead@COleControl@@QAEHXZ 5f539414 f   ctlprop.obj
 0001:00038442       ?AmbientShowGrabHandles@COleControl@@QAEHXZ 5f539442 f   ctlprop.obj
 0001:00038470       ?AmbientShowHatching@COleControl@@QAEHXZ 5f539470 f   ctlprop.obj
 0001:0003849e       ?BoundPropertyChanged@COleControl@@QAEXJ@Z 5f53949e f   ctlprop.obj
 0001:00038511       ?BoundPropertyRequestEdit@COleControl@@QAEHJ@Z 5f539511 f   ctlprop.obj
 0001:00038591       ?SetNotPermitted@COleControl@@QAEXXZ 5f539591 f   ctlprop.obj
 0001:000385b0       ?SetNotSupported@COleControl@@QAEXXZ 5f5395b0 f   ctlprop.obj
 0001:000385cf       ?GetNotSupported@COleControl@@QAEXXZ 5f5395cf f   ctlprop.obj
 0001:000385ee       ?AddRef@XPerPropertyBrowsing@COleControl@@UAGKXZ 5f5395ee f   ctlprop.obj
 0001:0003860b       ?Release@XPerPropertyBrowsing@COleControl@@UAGKXZ 5f53960b f   ctlprop.obj
 0001:00038628       ?QueryInterface@XPerPropertyBrowsing@COleControl@@UAGJABU_GUID@@PAPAX@Z 5f539628 f   ctlprop.obj
 0001:0003864d       ?GetDisplayString@XPerPropertyBrowsing@COleControl@@UAGJJPAPAG@Z 5f53964d f   ctlprop.obj
 0001:00038747       ?OnGetDisplayString@COleControl@@UAEHJAAVCString@@@Z 5f539747 f   ctlprop.obj
 0001:00038826       ?MapPropertyToPage@XPerPropertyBrowsing@COleControl@@UAGJJPAU_GUID@@@Z 5f539826 f   ctlprop.obj
 0001:00038960       ?OnMapPropertyToPage@COleControl@@UAEHJPAU_GUID@@PAH@Z 5f539960 f   ctlprop.obj
 0001:000389fc       ?GetPredefinedStrings@XPerPropertyBrowsing@COleControl@@UAGJJPAUtagCALPOLESTR@@PAUtagCADWORD@@@Z 5f5399fc f   ctlprop.obj
 0001:00038d4d       ?OnGetPredefinedStrings@COleControl@@UAEHJPAVCStringArray@@PAVCDWordArray@@@Z 5f539d4d f   ctlprop.obj
 0001:00038e64       ?GetPredefinedValue@XPerPropertyBrowsing@COleControl@@UAGJJKPAUtagVARIANT@@@Z 5f539e64 f   ctlprop.obj
 0001:00038f24       ?OnGetPredefinedValue@COleControl@@UAEHJKPAUtagVARIANT@@@Z 5f539f24 f   ctlprop.obj
 0001:00038f74       ?Load@COleControl@@QAEXPBDAAVCDataPathProperty@@@Z 5f539f74 f   ctlprop.obj
 0001:00038f9e       ?Open@CDataPathProperty@@UAEHPAVCFileException@@@Z 5f539f9e f   ctlprop.obj
 0001:00038fe9       ?Open@CDataPathProperty@@UAEHPBDPAVCFileException@@@Z 5f539fe9 f   ctlprop.obj
 0001:00039014       ?Open@CDataPathProperty@@UAEHPAVCOleControl@@PAVCFileException@@@Z 5f53a014 f   ctlprop.obj
 0001:0003903f       ?Open@CDataPathProperty@@UAEHPBDPAVCOleControl@@PAVCFileException@@@Z 5f53a03f f   ctlprop.obj
 0001:00039076       ?ResetData@CDataPathProperty@@UAEXXZ 5f53a076 f   ctlprop.obj
 0001:00039081       ?AssertValid@CDataPathProperty@@UBEXXZ 5f53a081 f   ctlprop.obj
 0001:00039094       ?Dump@CDataPathProperty@@UBEXAAVCDumpContext@@@Z 5f53a094 f   ctlprop.obj
 0001:000390ef       ?OnDataAvailable@CCachedDataPathProperty@@UAEXKK@Z 5f53a0ef f   ctlprop.obj
 0001:000391c7       ?Close@CCachedDataPathProperty@@UAEXXZ 5f53a1c7 f   ctlprop.obj
 0001:000391eb       ?ResetData@CCachedDataPathProperty@@UAEXXZ 5f53a1eb f   ctlprop.obj
 0001:00039207       ?AssertValid@CCachedDataPathProperty@@UBEXXZ 5f53a207 f   ctlprop.obj
 0001:00039229       ?Dump@CCachedDataPathProperty@@UBEXAAVCDumpContext@@@Z 5f53a229 f   ctlprop.obj
 0001:00039260       ?_AfxCopyString@@YGPAGPBD@Z 5f53a260 f i ctlprop.obj
 0001:000392c0       ?_AfxTransferFileContent@@YAKPAVCFile@@0@Z 5f53a2c0 f i ctlprop.obj
 0001:00039320       ?_AfxCreateMemoryStream@@YGPAUIStream@@XZ 5f53a320 f   ctlpset.obj
 0001:000393ca       ?GetPropsetData@COleControl@@IAEHPAUtagFORMATETC@@PAUtagSTGMEDIUM@@ABU_GUID@@@Z 5f53a3ca f   ctlpset.obj
 0001:000399e0       ?SetPropsetData@COleControl@@IAEHPAUtagFORMATETC@@PAUtagSTGMEDIUM@@ABU_GUID@@@Z 5f53a9e0 f   ctlpset.obj
 0001:00039dca       ??0CPropsetPropExchange@@QAE@AAVCPropertySection@@PAUIStorage@@H@Z 5f53adca f   ctlpset.obj
 0001:00039e78       ?_AfxGetSizeOfVarType@@YGIG@Z 5f53ae78 f   ctlpset.obj
 0001:00039ef3       ?_AfxCoerceNumber@@YGHPAXG0G@Z 5f53aef3 f   ctlpset.obj
 0001:00039fb3       ?_AfxIsSamePropValue@@YGHGPBX0@Z 5f53afb3 f   ctlpset.obj
 0001:0003a09c       ?ExchangeProp@CPropsetPropExchange@@UAEHPBDGPAXPBX@Z 5f53b09c f   ctlpset.obj
 0001:0003a4fc       ?ExchangeBlobProp@CPropsetPropExchange@@UAEHPBDPAPAXPAX@Z 5f53b4fc f   ctlpset.obj
 0001:0003a6e1       ?_AfxSaveStreamDataAsBlobProp@@YGHPAUIStream@@AAVCPropertySection@@KK@Z 5f53b6e1 f   ctlpset.obj
 0001:0003a7ee       ?_AfxInitStreamDataFromBlobProp@@YGHPAUIStream@@PAVCProperty@@@Z 5f53b7ee f   ctlpset.obj
 0001:0003a868       ?_AfxCreateFontFromStream@@YGPAUIFont@@PAUIStream@@@Z 5f53b868 f   ctlpset.obj
 0001:0003aa07       ?_AfxLoadObjectFromStreamedPropset@@YGHPAUIUnknown@@PAUIStream@@@Z 5f53ba07 f   ctlpset.obj
 0001:0003ab3e       ?_AfxGetClassIDFromStreamedPropset@@YGHPAU_GUID@@PAUIStream@@@Z 5f53bb3e f   ctlpset.obj
 0001:0003abd9       ?_AfxCreateObjectFromStreamedPropset@@YGPAUIUnknown@@PAUIStream@@ABU_GUID@@@Z 5f53bbd9 f   ctlpset.obj
 0001:0003acf5       ?_AfxLoadStreamFromPropset@@YGPAUIStream@@AAVCPropertySection@@PBDAAK@Z 5f53bcf5 f   ctlpset.obj
 0001:0003adc2       ?_AfxSaveObjectInPropset@@YGHPAUIUnknown@@AAVCPropertySection@@K@Z 5f53bdc2 f   ctlpset.obj
 0001:0003afa9       ?ExchangePersistentProp@CPropsetPropExchange@@UAEHPBDPAPAUIUnknown@@ABU_GUID@@PAU2@@Z 5f53bfa9 f   ctlpset.obj
 0001:0003b23d       ?ExchangeFontProp@CPropsetPropExchange@@UAEHPBDAAVCFontHolder@@PBUtagFONTDESC@@PAUIFontDisp@@@Z 5f53c23d f   ctlpset.obj
 0001:0003b440       ?AddRef@XPersistStorage@COleControl@@UAGKXZ 5f53c440 f   ctlpstg.obj
 0001:0003b45d       ?Release@XPersistStorage@COleControl@@UAGKXZ 5f53c45d f   ctlpstg.obj
 0001:0003b47a       ?QueryInterface@XPersistStorage@COleControl@@UAGJABU_GUID@@PAPAX@Z 5f53c47a f   ctlpstg.obj
 0001:0003b49f       ?GetClassID@XPersistStorage@COleControl@@UAGJPAU_GUID@@@Z 5f53c49f f   ctlpstg.obj
 0001:0003b4c6       ?IsDirty@XPersistStorage@COleControl@@UAGJXZ 5f53c4c6 f   ctlpstg.obj
 0001:0003b54b       ?InitNew@XPersistStorage@COleControl@@UAGJPAUIStorage@@@Z 5f53c54b f   ctlpstg.obj
 0001:0003b63c       ?Load@XPersistStorage@COleControl@@UAGJPAUIStorage@@@Z 5f53c63c f   ctlpstg.obj
 0001:0003b7f5       ?Save@XPersistStorage@COleControl@@UAGJPAUIStorage@@H@Z 5f53c7f5 f   ctlpstg.obj
 0001:0003b97f       ?SaveCompleted@XPersistStorage@COleControl@@UAGJPAUIStorage@@@Z 5f53c97f f   ctlpstg.obj
 0001:0003b9ed       ?HandsOffStorage@XPersistStorage@COleControl@@UAGJXZ 5f53c9ed f   ctlpstg.obj
 0001:0003ba40       ?AddRef@XPersistStreamInit@COleControl@@UAGKXZ 5f53ca40 f   ctlpstm.obj
 0001:0003ba5d       ?Release@XPersistStreamInit@COleControl@@UAGKXZ 5f53ca5d f   ctlpstm.obj
 0001:0003ba7a       ?QueryInterface@XPersistStreamInit@COleControl@@UAGJABU_GUID@@PAPAX@Z 5f53ca7a f   ctlpstm.obj
 0001:0003ba9f       ?GetClassID@XPersistStreamInit@COleControl@@UAGJPAU_GUID@@@Z 5f53ca9f f   ctlpstm.obj
 0001:0003bac6       ?IsDirty@XPersistStreamInit@COleControl@@UAGJXZ 5f53cac6 f   ctlpstm.obj
 0001:0003baef       ?Load@XPersistStreamInit@COleControl@@UAGJPAUIStream@@@Z 5f53caef f   ctlpstm.obj
 0001:0003bb5c       ?Save@XPersistStreamInit@COleControl@@UAGJPAUIStream@@H@Z 5f53cb5c f   ctlpstm.obj
 0001:0003bbea       ?GetSizeMax@XPersistStreamInit@COleControl@@UAGJPAT_ULARGE_INTEGER@@@Z 5f53cbea f   ctlpstm.obj
 0001:0003bbf6       ?InitNew@XPersistStreamInit@COleControl@@UAGJXZ 5f53cbf6 f   ctlpstm.obj
 0001:0003bca9       ?AddRef@XPersistMemory@COleControl@@UAGKXZ 5f53cca9 f   ctlpstm.obj
 0001:0003bcc6       ?Release@XPersistMemory@COleControl@@UAGKXZ 5f53ccc6 f   ctlpstm.obj
 0001:0003bce3       ?QueryInterface@XPersistMemory@COleControl@@UAGJABU_GUID@@PAPAX@Z 5f53cce3 f   ctlpstm.obj
 0001:0003bd08       ?GetClassID@XPersistMemory@COleControl@@UAGJPAU_GUID@@@Z 5f53cd08 f   ctlpstm.obj
 0001:0003bd2f       ?IsDirty@XPersistMemory@COleControl@@UAGJXZ 5f53cd2f f   ctlpstm.obj
 0001:0003bd58       ?Load@XPersistMemory@COleControl@@UAGJPAXK@Z 5f53cd58 f   ctlpstm.obj
 0001:0003bf17       ?Save@XPersistMemory@COleControl@@UAGJPAXHK@Z 5f53cf17 f   ctlpstm.obj
 0001:0003bf23       ?GetSizeMax@XPersistMemory@COleControl@@UAGJPAK@Z 5f53cf23 f   ctlpstm.obj
 0001:0003bf2f       ?InitNew@XPersistMemory@COleControl@@UAGJXZ 5f53cf2f f   ctlpstm.obj
 0001:0003bff0       ?Create@CReflectorWnd@@QAEHABVCRect@@PAUHWND__@@@Z 5f53cff0 f   ctlrefl.obj
 0001:0003c069       ?PostNcDestroy@CReflectorWnd@@MAEXXZ 5f53d069 f   ctlrefl.obj
 0001:0003c0be       ?WindowProc@CReflectorWnd@@MAEJIIJ@Z 5f53d0be f   ctlrefl.obj
 0001:0003c2dc       ?SetControl@CReflectorWnd@@QAEXPAVCOleControl@@@Z 5f53d2dc f   ctlrefl.obj
 0001:0003c2f2       ?WindowProc@CParkingWnd@@UAEJIIJ@Z 5f53d2f2 f   ctlrefl.obj
 0001:0003c4e0       ?_AfxRecursiveRegDeleteKey@@YGJPAUHKEY__@@PAD@Z 5f53d4e0 f   ctlreg.obj
 0001:0003c540       ?_AfxUnregisterInterfaces@@YAXPAUITypeLib@@@Z 5f53d540 f   ctlreg.obj
 0001:0003c690       ?AfxOleRegisterTypeLib@@YGHPAUHINSTANCE__@@ABU_GUID@@PBD2@Z 5f53d690 f   ctlreg.obj
 0001:0003c9f3       ?AfxOleUnregisterTypeLib@@YGHABU_GUID@@GGK@Z 5f53d9f3 f   ctlreg.obj
 0001:0003ce5d       ?AfxOleRegisterControlClass@@YGHPAUHINSTANCE__@@ABU_GUID@@PBDIIHK1GG@Z 5f53de5d f   ctlreg.obj
 0001:0003d3d5       ?AfxOleUnregisterClass@@YGHABU_GUID@@PBD@Z 5f53e3d5 f   ctlreg.obj
 0001:0003d6c3       ?AfxOleRegisterPropertyPageClass@@YGHPAUHINSTANCE__@@ABU_GUID@@I@Z 5f53e6c3 f   ctlreg.obj
 0001:0003d6dd       ?AfxOleRegisterPropertyPageClass@@YGHPAUHINSTANCE__@@ABU_GUID@@IH@Z 5f53e6dd f   ctlreg.obj
 0001:0003d9d0       ?_AfxRegDeleteKeySucceeded@@YAHJ@Z 5f53e9d0 f i ctlreg.obj
 0001:0003da00       ?_AfxOffsetTrackerRect@@YGXAAVCRect@@PAVCWnd@@@Z 5f53ea00 f   ctltrack.obj
 0001:0003daa4       ?CreateTracker@COleControl@@IAEXHH@Z 5f53eaa4 f   ctltrack.obj
 0001:0003dac3       ?CreateTracker@COleControl@@IAEXHHPBUtagRECT@@@Z 5f53eac3 f   ctltrack.obj
 0001:0003dd34       ?DestroyTracker@COleControl@@IAEXXZ 5f53ed34 f   ctltrack.obj
 0001:0003de21       ?OnNcPaint@COleControl@@IAEXXZ 5f53ee21 f   ctltrack.obj
 0001:0003dfe7       ?OnNcCalcSize@COleControl@@IAEXHPAUtagNCCALCSIZE_PARAMS@@@Z 5f53efe7 f   ctltrack.obj
 0001:0003e079       ?OnNcHitTest@COleControl@@IAEIVCPoint@@@Z 5f53f079 f   ctltrack.obj
 0001:0003e1c2       ?OnNcLButtonDown@COleControl@@IAEXIVCPoint@@@Z 5f53f1c2 f   ctltrack.obj
 0001:0003e44d       ?OnSetCursor@COleControl@@IAEHPAVCWnd@@II@Z 5f53f44d f   ctltrack.obj
 0001:0003e4e0       ??0CControlRectTracker@@QAE@PBUtagRECT@@I@Z 5f53f4e0 f i ctltrack.obj
 0001:0003e550       ??_ECControlRectTracker@@UAEPAXI@Z 5f53f550 f i ctltrack.obj
 0001:0003e550       ??_GCControlRectTracker@@UAEPAXI@Z 5f53f550 f i ctltrack.obj
 0001:0003e580       ??1CControlRectTracker@@UAE@XZ 5f53f580 f i ctltrack.obj
 0001:0003e5a0       ?OnGetColorSet@COleControl@@UAEHPAUtagDVTARGETDEVICE@@PAUHDC__@@PAPAUtagLOGPALETTE@@@Z 5f53f5a0 f   ctlview.obj
 0001:0003e5af       ?OnGetViewExtent@COleControl@@UAEHKJPAUtagDVTARGETDEVICE@@PAUtagSIZE@@@Z 5f53f5af f   ctlview.obj
 0001:0003e5f6       ?OnGetViewRect@COleControl@@UAEHKPAU_RECTL@@@Z 5f53f5f6 f   ctlview.obj
 0001:0003e64b       ?OnGetViewStatus@COleControl@@UAEKXZ 5f53f64b f   ctlview.obj
 0001:0003e65b       ?OnQueryHitPoint@COleControl@@UAEHKPBUtagRECT@@UtagPOINT@@JPAK@Z 5f53f65b f   ctlview.obj
 0001:0003e680       ?OnQueryHitRect@COleControl@@UAEHKPBUtagRECT@@0JPAK@Z 5f53f680 f   ctlview.obj
 0001:0003e6a5       ?OnGetNaturalExtent@COleControl@@UAEHKJPAUtagDVTARGETDEVICE@@PAUHDC__@@PAUtagExtentInfo@@PAUtagSIZE@@@Z 5f53f6a5 f   ctlview.obj
 0001:0003e6b4       ?AddRef@XViewObject@COleControl@@UAGKXZ 5f53f6b4 f   ctlview.obj
 0001:0003e6d1       ?Release@XViewObject@COleControl@@UAGKXZ 5f53f6d1 f   ctlview.obj
 0001:0003e6ee       ?QueryInterface@XViewObject@COleControl@@UAGJABU_GUID@@PAPAX@Z 5f53f6ee f   ctlview.obj
 0001:0003e713       ?Draw@XViewObject@COleControl@@UAGJKJPAXPAUtagDVTARGETDEVICE@@PAUHDC__@@2PBU_RECTL@@3P6GHK@ZK@Z 5f53f713 f   ctlview.obj
 0001:0003e98c       ?GetColorSet@XViewObject@COleControl@@UAGJKJPAXPAUtagDVTARGETDEVICE@@PAUHDC__@@PAPAUtagLOGPALETTE@@@Z 5f53f98c f   ctlview.obj
 0001:0003ea28       ?Freeze@XViewObject@COleControl@@UAGJKJPAXPAK@Z 5f53fa28 f   ctlview.obj
 0001:0003ea34       ?Unfreeze@XViewObject@COleControl@@UAGJK@Z 5f53fa34 f   ctlview.obj
 0001:0003ea40       ?SetAdvise@XViewObject@COleControl@@UAGJKKPAUIAdviseSink@@@Z 5f53fa40 f   ctlview.obj
 0001:0003eb96       ?GetAdvise@XViewObject@COleControl@@UAGJPAK0PAPAUIAdviseSink@@@Z 5f53fb96 f   ctlview.obj
 0001:0003ec43       ?GetExtent@XViewObject@COleControl@@UAGJKJPAUtagDVTARGETDEVICE@@PAUtagSIZE@@@Z 5f53fc43 f   ctlview.obj
 0001:0003ec84       ?GetRect@XViewObject@COleControl@@UAGJKPAU_RECTL@@@Z 5f53fc84 f   ctlview.obj
 0001:0003ecbd       ?GetViewStatus@XViewObject@COleControl@@UAGJPAK@Z 5f53fcbd f   ctlview.obj
 0001:0003ece7       ?QueryHitPoint@XViewObject@COleControl@@UAGJKPBUtagRECT@@UtagPOINT@@JPAK@Z 5f53fce7 f   ctlview.obj
 0001:0003ed30       ?QueryHitRect@XViewObject@COleControl@@UAGJKPBUtagRECT@@0JPAK@Z 5f53fd30 f   ctlview.obj
 0001:0003ed75       ?GetNaturalExtent@XViewObject@COleControl@@UAGJKJPAUtagDVTARGETDEVICE@@PAUHDC__@@PAUtagExtentInfo@@PAUtagSIZE@@@Z 5f53fd75 f   ctlview.obj
 0001:0003edc0       ??0_AFXCTL_ADVISE_INFO@@QAE@XZ 5f53fdc0 f i ctlview.obj
 0001:0003edc0       ??0CAccessorBase@ATL@@QAE@XZ 5f53fdc0 f i ctlview.obj
 0001:0003edf0       ?_AfxCountPrefixedStringA@@YGPAXPBD@Z 5f53fdf0 f   olepset.obj
 0001:0003ee41       ?_AfxCountPrefixedStringW@@YGPAXPBG@Z 5f53fe41 f   olepset.obj
 0001:0003ee99       ??0CProperty@@QAE@XZ       5f53fe99 f   olepset.obj
 0001:0003eec4       ??0CProperty@@QAE@KQAXK@Z  5f53fec4 f   olepset.obj
 0001:0003ef03       ??1CProperty@@QAE@XZ       5f53ff03 f   olepset.obj
 0001:0003ef16       ?Set@CProperty@@QAEHKQAXK@Z 5f53ff16 f   olepset.obj
 0001:0003ef40       ?Set@CProperty@@QAEHQAXK@Z 5f53ff40 f   olepset.obj
 0001:0003ef62       ?Set@CProperty@@QAEHQAX@Z  5f53ff62 f   olepset.obj
 0001:0003f266       ?Get@CProperty@@QAEPAXXZ   5f540266 f   olepset.obj
 0001:0003f27b       ?Get@CProperty@@QAEPAXPAK@Z 5f54027b f   olepset.obj
 0001:0003f39f       ?GetType@CProperty@@QAEKXZ 5f54039f f   olepset.obj
 0001:0003f3b0       ?SetType@CProperty@@QAEXK@Z 5f5403b0 f   olepset.obj
 0001:0003f3c6       ?GetID@CProperty@@QAEKXZ   5f5403c6 f   olepset.obj
 0001:0003f3d6       ?SetID@CProperty@@QAEXK@Z  5f5403d6 f   olepset.obj
 0001:0003f3eb       ?GetRawValue@CProperty@@QAEPAXXZ 5f5403eb f   olepset.obj
 0001:0003f3fc       ?WriteToStream@CProperty@@QAEHPAUIStream@@@Z 5f5403fc f   olepset.obj
 0001:0003f622       ?ReadFromStream@CProperty@@QAEHPAUIStream@@@Z 5f540622 f   olepset.obj
 0001:0003f92c       ?AllocValue@CProperty@@AAEPAXK@Z 5f54092c f   olepset.obj
 0001:0003f952       ?FreeValue@CProperty@@AAEXXZ 5f540952 f   olepset.obj
 0001:0003f980       ??0CPropertySection@@QAE@XZ 5f540980 f   olepset.obj
 0001:0003fa1e       ??0CPropertySection@@QAE@U_GUID@@@Z 5f540a1e f   olepset.obj
 0001:0003fab2       ??1CPropertySection@@QAE@XZ 5f540ab2 f   olepset.obj
 0001:0003fb1b       ?GetFormatID@CPropertySection@@QAE?AU_GUID@@XZ 5f540b1b f   olepset.obj
 0001:0003fb47       ?SetFormatID@CPropertySection@@QAEXU_GUID@@@Z 5f540b47 f   olepset.obj
 0001:0003fb6e       ?Set@CPropertySection@@QAEHKPAXK@Z 5f540b6e f   olepset.obj
 0001:0003fc3e       ?Set@CPropertySection@@QAEHKPAX@Z 5f540c3e f   olepset.obj
 0001:0003fc8b       ?Get@CPropertySection@@QAEPAXK@Z 5f540c8b f   olepset.obj
 0001:0003fca6       ?Get@CPropertySection@@QAEPAXKPAK@Z 5f540ca6 f   olepset.obj
 0001:0003fcda       ?Remove@CPropertySection@@QAEXK@Z 5f540cda f   olepset.obj
 0001:0003fd6b       ?RemoveAll@CPropertySection@@QAEXXZ 5f540d6b f   olepset.obj
 0001:0003fdd9       ?GetProperty@CPropertySection@@QAEPAVCProperty@@K@Z 5f540dd9 f   olepset.obj
 0001:0003fe23       ?AddProperty@CPropertySection@@QAEXPAVCProperty@@@Z 5f540e23 f   olepset.obj
 0001:0003fe4e       ?GetSize@CPropertySection@@QAEKXZ 5f540e4e f   olepset.obj
 0001:0003fe5f       ?GetCount@CPropertySection@@QAEKXZ 5f540e5f f   olepset.obj
 0001:0003fe75       ?GetList@CPropertySection@@QAEPAVCPtrList@@XZ 5f540e75 f   olepset.obj
 0001:0003fe86       ?WriteToStream@CPropertySection@@QAEHPAUIStream@@@Z 5f540e86 f   olepset.obj
 0001:00040131       ?ReadFromStream@CPropertySection@@QAEHPAUIStream@@T_LARGE_INTEGER@@@Z 5f541131 f   olepset.obj
 0001:00040307       ?GetID@CPropertySection@@QAEHPBDPAK@Z 5f541307 f   olepset.obj
 0001:000403a8       ?SetName@CPropertySection@@QAEHKPBD@Z 5f5413a8 f   olepset.obj
 0001:000404ec       ?ReadNameDictFromStream@CPropertySection@@QAEHPAUIStream@@@Z 5f5414ec f   olepset.obj
 0001:00040642       ?_AfxWriteNameDictEntry@@YGHPAUIStream@@KAAVCString@@@Z 5f541642 f   olepset.obj
 0001:00040712       ?WriteNameDictToStream@CPropertySection@@QAEHPAUIStream@@@Z 5f541712 f   olepset.obj
 0001:0004083c       ?SetSectionName@CPropertySection@@QAEHPBD@Z 5f54183c f   olepset.obj
 0001:0004085d       ?GetSectionName@CPropertySection@@QAEPBDXZ 5f54185d f   olepset.obj
 0001:00040873       ??0CPropertySet@@QAE@XZ    5f541873 f   olepset.obj
 0001:000408e8       ??0CPropertySet@@QAE@U_GUID@@@Z 5f5418e8 f   olepset.obj
 0001:00040953       ??1CPropertySet@@QAE@XZ    5f541953 f   olepset.obj
 0001:0004099e       ?Set@CPropertySet@@QAEHU_GUID@@KPAXK@Z 5f54199e f   olepset.obj
 0001:00040a8b       ?Set@CPropertySet@@QAEHU_GUID@@KPAX@Z 5f541a8b f   olepset.obj
 0001:00040adb       ?Get@CPropertySet@@QAEPAXU_GUID@@KPAK@Z 5f541adb f   olepset.obj
 0001:00040b2b       ?Get@CPropertySet@@QAEPAXU_GUID@@K@Z 5f541b2b f   olepset.obj
 0001:00040b62       ?Remove@CPropertySet@@QAEXU_GUID@@K@Z 5f541b62 f   olepset.obj
 0001:00040baa       ?Remove@CPropertySet@@QAEXU_GUID@@@Z 5f541baa f   olepset.obj
 0001:00040c4b       ?RemoveAll@CPropertySet@@QAEXXZ 5f541c4b f   olepset.obj
 0001:00040cb9       ?GetSection@CPropertySet@@QAEPAVCPropertySection@@U_GUID@@@Z 5f541cb9 f   olepset.obj
 0001:00040d0d       ?AddSection@CPropertySet@@QAEPAVCPropertySection@@U_GUID@@@Z 5f541d0d f   olepset.obj
 0001:00040de9       ?AddSection@CPropertySet@@QAEXPAVCPropertySection@@@Z 5f541de9 f   olepset.obj
 0001:00040e14       ?GetProperty@CPropertySet@@QAEPAVCProperty@@U_GUID@@K@Z 5f541e14 f   olepset.obj
 0001:00040e60       ?AddProperty@CPropertySet@@QAEXU_GUID@@PAVCProperty@@@Z 5f541e60 f   olepset.obj
 0001:00040ea8       ?GetByteOrder@CPropertySet@@QAEGXZ 5f541ea8 f   olepset.obj
 0001:00040eb9       ?GetFormatVersion@CPropertySet@@QAEGXZ 5f541eb9 f   olepset.obj
 0001:00040ecb       ?SetFormatVersion@CPropertySet@@QAEXG@Z 5f541ecb f   olepset.obj
 0001:00040ee3       ?GetOSVersion@CPropertySet@@QAEKXZ 5f541ee3 f   olepset.obj
 0001:00040ef4       ?SetOSVersion@CPropertySet@@QAEXK@Z 5f541ef4 f   olepset.obj
 0001:00040f0a       ?GetClassID@CPropertySet@@QAE?AU_GUID@@XZ 5f541f0a f   olepset.obj
 0001:00040f39       ?SetClassID@CPropertySet@@QAEXU_GUID@@@Z 5f541f39 f   olepset.obj
 0001:00040f63       ?GetCount@CPropertySet@@QAEKXZ 5f541f63 f   olepset.obj
 0001:00040f79       ?GetList@CPropertySet@@QAEPAVCPtrList@@XZ 5f541f79 f   olepset.obj
 0001:00040f8a       ?WriteToStream@CPropertySet@@QAEHPAUIStream@@@Z 5f541f8a f   olepset.obj
 0001:00041142       ?ReadFromStream@CPropertySet@@QAEHPAUIStream@@@Z 5f542142 f   olepset.obj
 0001:00041320       ??_GCProperty@@QAEPAXI@Z   5f542320 f i olepset.obj
 0001:00041350       ??_GCPropertySection@@QAEPAXI@Z 5f542350 f i olepset.obj
 0001:00041380       ??0CBlobProperty@@QAE@PAX@Z 5f542380 f   ctlpbag.obj
 0001:000413b4       ?GetBlob@CBlobProperty@@QAEPAXXZ 5f5423b4 f   ctlpbag.obj
 0001:000413c5       ?AddRef@CBlobProperty@@UAGKXZ 5f5423c5 f   ctlpbag.obj
 0001:000413d9       ?Release@CBlobProperty@@UAGKXZ 5f5423d9 f   ctlpbag.obj
 0001:00041410       ?QueryInterface@CBlobProperty@@UAGJABU_GUID@@PAPAX@Z 5f542410 f   ctlpbag.obj
 0001:0004147c       ?GetClassID@CBlobProperty@@UAGJPAU_GUID@@@Z 5f54247c f   ctlpbag.obj
 0001:000414ab       ?IsDirty@CBlobProperty@@UAGJXZ 5f5424ab f   ctlpbag.obj
 0001:000414b4       ?Load@CBlobProperty@@UAGJPAUIStream@@@Z 5f5424b4 f   ctlpbag.obj
 0001:0004159c       ?Save@CBlobProperty@@UAGJPAUIStream@@H@Z 5f54259c f   ctlpbag.obj
 0001:00041614       ?GetSizeMax@CBlobProperty@@UAGJPAT_ULARGE_INTEGER@@@Z 5f542614 f   ctlpbag.obj
 0001:00041661       ??0CPropbagPropExchange@@QAE@PAUIPropertyBag@@PAUIErrorLog@@HH@Z 5f542661 f   ctlpbag.obj
 0001:000416ca       ??1CPropbagPropExchange@@QAE@XZ 5f5426ca f   ctlpbag.obj
 0001:00041734       ?ExchangeProp@CPropbagPropExchange@@UAEHPBDGPAXPBX@Z 5f542734 f   ctlpbag.obj
 0001:00041c1b       ?ExchangeBlobProp@CPropbagPropExchange@@UAEHPBDPAPAXPAX@Z 5f542c1b f   ctlpbag.obj
 0001:00041f14       ?ExchangeFontProp@CPropbagPropExchange@@UAEHPBDAAVCFontHolder@@PBUtagFONTDESC@@PAUIFontDisp@@@Z 5f542f14 f   ctlpbag.obj
 0001:00042210       ?ExchangePersistentProp@CPropbagPropExchange@@UAEHPBDPAPAUIUnknown@@ABU_GUID@@PAU2@@Z 5f543210 f   ctlpbag.obj
 0001:000424e2       ?AddRef@XPersistPropertyBag@COleControl@@UAGKXZ 5f5434e2 f   ctlpbag.obj
 0001:000424ff       ?Release@XPersistPropertyBag@COleControl@@UAGKXZ 5f5434ff f   ctlpbag.obj
 0001:0004251c       ?QueryInterface@XPersistPropertyBag@COleControl@@UAGJABU_GUID@@PAPAX@Z 5f54351c f   ctlpbag.obj
 0001:00042541       ?GetClassID@XPersistPropertyBag@COleControl@@UAGJPAU_GUID@@@Z 5f543541 f   ctlpbag.obj
 0001:00042568       ?InitNew@XPersistPropertyBag@COleControl@@UAGJXZ 5f543568 f   ctlpbag.obj
 0001:0004261b       ?Load@XPersistPropertyBag@COleControl@@UAGJPAUIPropertyBag@@PAUIErrorLog@@@Z 5f54361b f   ctlpbag.obj
 0001:00042773       ?Save@XPersistPropertyBag@COleControl@@UAGJPAUIPropertyBag@@HH@Z 5f543773 f   ctlpbag.obj
 0001:000428c5       ??0_AFXCTL_AMBIENT_CACHE@@QAE@XZ 5f5438c5 f   ctlquick.obj
 0001:000428e4       ?Cache@_AFXCTL_AMBIENT_CACHE@@QAEXPAUtagQACONTAINER@@@Z 5f5438e4 f   ctlquick.obj
 0001:0004296c       ?AddRef@XQuickActivate@COleControl@@UAGKXZ 5f54396c f   ctlquick.obj
 0001:00042989       ?Release@XQuickActivate@COleControl@@UAGKXZ 5f543989 f   ctlquick.obj
 0001:000429a6       ?QueryInterface@XQuickActivate@COleControl@@UAGJABU_GUID@@PAPAX@Z 5f5439a6 f   ctlquick.obj
 0001:000429cb       ?QuickActivate@XQuickActivate@COleControl@@UAGJPAUtagQACONTAINER@@PAUtagQACONTROL@@@Z 5f5439cb f   ctlquick.obj
 0001:00042b59       ?SetContentExtent@XQuickActivate@COleControl@@UAGJPAUtagSIZE@@@Z 5f543b59 f   ctlquick.obj
 0001:00042b8a       ?GetContentExtent@XQuickActivate@COleControl@@UAGJPAUtagSIZE@@@Z 5f543b8a f   ctlquick.obj
 0001:00042bc0       ??1?$CThreadLocal@V_AFXCTL_AMBIENT_CACHE@@@@QAE@XZ 5f543bc0 f i ctlquick.obj
 0001:00042be0       ??_G_AFXCTL_AMBIENT_CACHE@@UAEPAXI@Z 5f543be0 f i ctlquick.obj
 0001:00042be0       ??_ECOccManager@@UAEPAXI@Z 5f543be0 f i ctlquick.obj
 0001:00042be0       ??_GCOccManager@@UAEPAXI@Z 5f543be0 f i ctlquick.obj
 0001:00042be0       ??_E_AFXCTL_AMBIENT_CACHE@@UAEPAXI@Z 5f543be0 f i ctlquick.obj
 0001:00042c10       ??1_AFXCTL_AMBIENT_CACHE@@UAE@XZ 5f543c10 f i ctlquick.obj
 0001:00042c10       ??1COccManager@@UAE@XZ     5f543c10 f i ctlquick.obj
 0001:00042c30       ?_GetBaseClass@CWindowlessDC@@KGPAUCRuntimeClass@@XZ 5f543c30 f   ctlnownd.obj
 0001:00042c3a       ?GetRuntimeClass@CWindowlessDC@@UBEPAUCRuntimeClass@@XZ 5f543c3a f   ctlnownd.obj
 0001:00042c4a       ??0CWindowlessDC@@QAE@PAUHDC__@@AAVCPoint@@@Z 5f543c4a f   ctlnownd.obj
 0001:00042d15       ?Detach@CWindowlessDC@@QAEPAUHDC__@@XZ 5f543d15 f   ctlnownd.obj
 0001:00042d65       ?GetClientOffset@COleControl@@UBEXPAJ0@Z 5f543d65 f   ctlnownd.obj
 0001:00042dde       ?ParentToClient@COleControl@@UBEIPBUtagRECT@@PAUtagPOINT@@H@Z 5f543dde f   ctlnownd.obj
 0001:00042ea3       ?ClientToParent@COleControl@@UBEXPBUtagRECT@@PAUtagPOINT@@@Z 5f543ea3 f   ctlnownd.obj
 0001:00042ef3       ?GetActivationPolicy@COleControl@@UAEKXZ 5f543ef3 f   ctlnownd.obj
 0001:00042f00       ?OnInactiveSetCursor@COleControl@@UAEHPBUtagRECT@@JJKH@Z 5f543f00 f   ctlnownd.obj
 0001:00042f9c       ?OnInactiveMouseMove@COleControl@@UAEXPBUtagRECT@@JJK@Z 5f543f9c f   ctlnownd.obj
 0001:00043003       ?AddRef@XPointerInactive@COleControl@@UAGKXZ 5f544003 f   ctlnownd.obj
 0001:00043020       ?Release@XPointerInactive@COleControl@@UAGKXZ 5f544020 f   ctlnownd.obj
 0001:0004303d       ?QueryInterface@XPointerInactive@COleControl@@UAGJABU_GUID@@PAPAX@Z 5f54403d f   ctlnownd.obj
 0001:00043062       ?GetActivationPolicy@XPointerInactive@COleControl@@UAGJPAK@Z 5f544062 f   ctlnownd.obj
 0001:0004308c       ?OnInactiveSetCursor@XPointerInactive@COleControl@@UAGJPBUtagRECT@@JJKH@Z 5f54408c f   ctlnownd.obj
 0001:000430c8       ?OnInactiveMouseMove@XPointerInactive@COleControl@@UAGJPBUtagRECT@@JJK@Z 5f5440c8 f   ctlnownd.obj
 0001:000430fd       ?OnWindowlessMessage@COleControl@@UAEHIIJPAJ@Z 5f5440fd f   ctlnownd.obj
 0001:0004319e       ?GetWindowlessDropTarget@COleControl@@UAEPAUIDropTarget@@XZ 5f54419e f   ctlnownd.obj
 0001:000431ab       ?OnWindowMessage@XOleInPlaceObject@COleControl@@UAGJIIJPAJ@Z 5f5441ab f   ctlnownd.obj
 0001:000431e3       ?GetDropTarget@XOleInPlaceObject@COleControl@@UAGJPAPAUIDropTarget@@@Z 5f5441e3 f   ctlnownd.obj
 0001:0004321e       ?SetCapture@COleControl@@QAEPAVCWnd@@XZ 5f54421e f   ctlnownd.obj
 0001:000432d2       ?ReleaseCapture@COleControl@@QAEHXZ 5f5442d2 f   ctlnownd.obj
 0001:00043379       ?GetCapture@COleControl@@QAEPAVCWnd@@XZ 5f544379 f   ctlnownd.obj
 0001:00043421       ?SetFocus@COleControl@@QAEPAVCWnd@@XZ 5f544421 f   ctlnownd.obj
 0001:000434d5       ?GetFocus@COleControl@@QAEPAVCWnd@@XZ 5f5444d5 f   ctlnownd.obj
 0001:0004357d       ?GetDC@COleControl@@QAEPAVCDC@@PBUtagRECT@@K@Z 5f54457d f   ctlnownd.obj
 0001:000437c9       ?ReleaseDC@COleControl@@QAEHPAVCDC@@@Z 5f5447c9 f   ctlnownd.obj
 0001:000438e9       ?InvalidateRgn@COleControl@@QAEXPAVCRgn@@H@Z 5f5448e9 f   ctlnownd.obj
 0001:00043a41       ?ScrollWindow@COleControl@@QAEXHHPBUtagRECT@@0@Z 5f544a41 f   ctlnownd.obj
 0001:00043bc1       ?ClipCaretRect@COleControl@@QAEHPAUtagRECT@@@Z 5f544bc1 f   ctlnownd.obj
 0001:00043c97       ?GetClientRect@COleControl@@UBEXPAUtagRECT@@@Z 5f544c97 f   ctlnownd.obj
 0001:00043e00       ??_ECWindowlessDC@@UAEPAXI@Z 5f544e00 f i ctlnownd.obj
 0001:00043e00       ??_GCWindowlessDC@@UAEPAXI@Z 5f544e00 f i ctlnownd.obj
 0001:00043e30       ??1CWindowlessDC@@UAE@XZ   5f544e30 f i ctlnownd.obj
 0001:00043e50       ??0CColorButton@@QAE@XZ    5f544e50 f   ppgcolor.obj
 0001:00043e79       ?SetFaceColor@CColorButton@@QAEXK@Z 5f544e79 f   ppgcolor.obj
 0001:00043e8f       ?colGetFaceColor@CColorButton@@QAEKXZ 5f544e8f f   ppgcolor.obj
 0001:00043ea0       ?SetState@CColorButton@@QAEXH@Z 5f544ea0 f   ppgcolor.obj
 0001:00043eb6       ?DrawItem@CColorButton@@MAEXPAUtagDRAWITEMSTRUCT@@@Z 5f544eb6 f   ppgcolor.obj
 0001:00044151       ?_GetBaseMessageMap@CColorPropPage@@KGPBUAFX_MSGMAP@@XZ 5f545151 f   ppgcolor.obj
 0001:0004415b       ?GetMessageMap@CColorPropPage@@MBEPBUAFX_MSGMAP@@XZ 5f54515b f   ppgcolor.obj
 0001:0004416b       ??0CColorPropPage@@QAE@XZ  5f54516b f   ppgcolor.obj
 0001:0004420f       ?OnInitDialog@CColorPropPage@@MAEHXZ 5f54520f f   ppgcolor.obj
 0001:000442dd       ?FillSysColors@CColorPropPage@@IAEXXZ 5f5452dd f   ppgcolor.obj
 0001:00044398       ?DoDataExchange@CColorPropPage@@MAEXPAVCDataExchange@@@Z 5f545398 f   ppgcolor.obj
 0001:000445be       ?SetColorProp@CColorPropPage@@IAEHPAVCDataExchange@@KPBD@Z 5f5455be f   ppgcolor.obj
 0001:000447ca       ?GetColorProp@CColorPropPage@@IAEHPAVCDataExchange@@PAKPBD@Z 5f5457ca f   ppgcolor.obj
 0001:000449a5       ?OnSelect@CColorPropPage@@AAEXXZ 5f5459a5 f   ppgcolor.obj
 0001:000449c7       ?SetButton@CColorPropPage@@AAEXPAVCColorButton@@@Z 5f5459c7 f   ppgcolor.obj
 0001:00044a3c       ?OnSelchangeColorprop@CColorPropPage@@AAEXXZ 5f545a3c f   ppgcolor.obj
 0001:00044a58       ?_AfxDraw3DFrame@@YAXPAVCDC@@VCRect@@KK@Z 5f545a58 f   ppgcolor.obj
 0001:00044c1b       ?_AfxDraw3DButtonFrame@@YAXPAVCDC@@VCRect@@H@Z 5f545c1b f   ppgcolor.obj
 0001:00044e25       ?_AfxInitPalette@@YAPAUHPALETTE__@@XZ 5f545e25 f   ppgcolor.obj
 0001:00045058       ?OnSelchangeSystemcolors@CColorPropPage@@AAEXXZ 5f546058 f   ppgcolor.obj
 0001:0004509c       ?OnEditProperty@CColorPropPage@@MAEHJ@Z 5f54609c f   ppgcolor.obj
 0001:000450be       ?OnObjectsChanged@CColorPropPage@@MAEXXZ 5f5460be f   ppgcolor.obj
 0001:000451ce       ?GetClassID@CColorPropPage@@UAEJPAU_GUID@@@Z 5f5461ce f   ppgcolor.obj
 0001:00045203       ?UpdateRegistry@CColorPropPageFactory@CColorPropPage@@UAEHH@Z 5f546203 f   ppgcolor.obj
 0001:00045240       ??_ECColorButton@@UAEPAXI@Z 5f546240 f i ppgcolor.obj
 0001:00045240       ??_GCColorButton@@UAEPAXI@Z 5f546240 f i ppgcolor.obj
 0001:00045270       ??1CColorButton@@UAE@XZ    5f546270 f i ppgcolor.obj
 0001:00045290       ??_GCColorPropPage@@UAEPAXI@Z 5f546290 f i ppgcolor.obj
 0001:00045290       ??_ECColorPropPage@@UAEPAXI@Z 5f546290 f i ppgcolor.obj
 0001:000452c0       ??1CStockPropPage@@UAE@XZ  5f5462c0 f i ppgcolor.obj
 0001:00045310       ??1CColorPropPage@@UAE@XZ  5f546310 f i ppgcolor.obj
 0001:00045390       ??0CColorPropPageFactory@CColorPropPage@@QAE@ABU_GUID@@PAUCRuntimeClass@@HPBD@Z 5f546390 f i ppgcolor.obj
 0001:000453d0       ?_GetBaseMessageMap@CFontPropPage@@KGPBUAFX_MSGMAP@@XZ 5f5463d0 f   ppgfont.obj
 0001:000453da       ?GetMessageMap@CFontPropPage@@MBEPBUAFX_MSGMAP@@XZ 5f5463da f   ppgfont.obj
 0001:000453ea       ??0CFontPropPage@@QAE@XZ   5f5463ea f   ppgfont.obj
 0001:000454ba       ?_AfxStringFromCy@@YAHAAVCString@@AATtagCY@@@Z 5f5464ba f   ppgfont.obj
 0001:0004553d       ?_AfxCyFromString@@YAHAATtagCY@@PBD@Z 5f54653d f   ppgfont.obj
 0001:0004562b       ?_AfxDrawMaskedBitmap@@YAXPAVCDC@@PAVCBitmap@@1HHHH@Z 5f54662b f   ppgfont.obj
 0001:00045761       ?_AfxInitMaskFromBitmap@@YAXPAVCBitmap@@0@Z 5f546761 f   ppgfont.obj
 0001:00045873       ?DoDataExchange@CFontPropPage@@MAEXPAVCDataExchange@@@Z 5f546873 f   ppgfont.obj
 0001:00045b84       ?SetFontProps@CFontPropPage@@IAEHPAVCDataExchange@@UtagFONTOBJECT@@PBD@Z 5f546b84 f   ppgfont.obj
 0001:00045ed9       ?GetFontProps@CFontPropPage@@IAEHPAVCDataExchange@@PAUtagFONTOBJECT@@PBDPAUtagMERGEOBJECT@@@Z 5f546ed9 f   ppgfont.obj
 0001:00046294       ?OnInitDialog@CFontPropPage@@MAEHXZ 5f547294 f   ppgfont.obj
 0001:000462c7       ?FillFacenameList@CFontPropPage@@IAEXXZ 5f5472c7 f   ppgfont.obj
 0001:000463b6       ?EnumFontFamiliesCallBack@CFontPropPage@@KGHPAUtagENUMLOGFONTA@@PAUtagNEWTEXTMETRICA@@HJ@Z 5f5473b6 f   ppgfont.obj
 0001:00046407       ?FillSizeList@CFontPropPage@@IAEXXZ 5f547407 f   ppgfont.obj
 0001:00046815       ?EnumFontFamiliesCallBack2@CFontPropPage@@KGHPAUtagENUMLOGFONTA@@PAUtagNEWTEXTMETRICA@@HJ@Z 5f547815 f   ppgfont.obj
 0001:0004698e       ??0CFontComboBox@@QAE@XZ   5f54798e f   ppgfont.obj
 0001:00046a1e       ??1CFontComboBox@@UAE@XZ   5f547a1e f   ppgfont.obj
 0001:00046a81       ?AddFont@CFontComboBox@@QAEHPAUtagLOGFONTA@@K@Z 5f547a81 f   ppgfont.obj
 0001:00046bc6       ?GetFontItem@CFontComboBox@@QAEPAUFONTITEM_PPG@@H@Z 5f547bc6 f   ppgfont.obj
 0001:00046c94       ?GetLogFont@CFontComboBox@@QAEPAUtagLOGFONTA@@H@Z 5f547c94 f   ppgfont.obj
 0001:00046cb0       ?GetFontType@CFontComboBox@@QAEKH@Z 5f547cb0 f   ppgfont.obj
 0001:00046ccb       ?GetCurrentName@CFontComboBox@@QAE?AVCString@@XZ 5f547ccb f   ppgfont.obj
 0001:00046d3f       ?DrawItem@CFontComboBox@@UAEXPAUtagDRAWITEMSTRUCT@@@Z 5f547d3f f   ppgfont.obj
 0001:00046ef9       ?DeleteItem@CFontComboBox@@UAEXPAUtagDELETEITEMSTRUCT@@@Z 5f547ef9 f   ppgfont.obj
 0001:00046f7f       ?AddSize@CSizeComboBox@@QAEHHJ@Z 5f547f7f f   ppgfont.obj
 0001:00047121       ?GetPointSize@CSizeComboBox@@QAEXAATtagCY@@@Z 5f548121 f   ppgfont.obj
 0001:00047161       ?GetHeight@CSizeComboBox@@QAEJH@Z 5f548161 f   ppgfont.obj
 0001:00047210       ?UpdateLogFont@CSizeComboBox@@QAEXPAUtagLOGFONTA@@H@Z 5f548210 f   ppgfont.obj
 0001:0004725e       ?OnEditupdateFontnames@CFontPropPage@@IAEXXZ 5f54825e f   ppgfont.obj
 0001:00047308       ?OnEditupdateFontsizes@CFontPropPage@@IAEXXZ 5f548308 f   ppgfont.obj
 0001:00047380       ?OnSelchangeFontnames@CFontPropPage@@IAEXXZ 5f548380 f   ppgfont.obj
 0001:00047393       ?UpdateSampleFont@CFontPropPage@@IAEXXZ 5f548393 f   ppgfont.obj
 0001:000474b7       ?OnPaint@CFontPropPage@@MAEXXZ 5f5484b7 f   ppgfont.obj
 0001:0004771d       ?OnSelchangeFontsizes@CFontPropPage@@IAEXXZ 5f54871d f   ppgfont.obj
 0001:00047764       ?OnSelchangeFontstyles@CFontPropPage@@IAEXXZ 5f548764 f   ppgfont.obj
 0001:000477b7       ?OnEditchangeFontstyles@CFontPropPage@@IAEXXZ 5f5487b7 f   ppgfont.obj
 0001:0004788e       ?SelectFontFromList@CFontPropPage@@IAEXVCString@@PAUtagMERGEOBJECT@@@Z 5f54888e f   ppgfont.obj
 0001:00047a58       ?OnStrikeout@CFontPropPage@@IAEXXZ 5f548a58 f   ppgfont.obj
 0001:00047aa6       ?OnUnderline@CFontPropPage@@IAEXXZ 5f548aa6 f   ppgfont.obj
 0001:00047af4       ?OnSelchangeFontprop@CFontPropPage@@IAEXXZ 5f548af4 f   ppgfont.obj
 0001:00047b10       ?OnEditProperty@CFontPropPage@@MAEHJ@Z 5f548b10 f   ppgfont.obj
 0001:00047b32       ?OnObjectsChanged@CFontPropPage@@MAEXXZ 5f548b32 f   ppgfont.obj
 0001:00047c6f       ?GetClassID@CFontPropPage@@UAEJPAU_GUID@@@Z 5f548c6f f   ppgfont.obj
 0001:00047ca4       ?UpdateRegistry@CFontPropPageFactory@CFontPropPage@@UAEHH@Z 5f548ca4 f   ppgfont.obj
 0001:00047ce0       ??_GCFontPropPage@@UAEPAXI@Z 5f548ce0 f i ppgfont.obj
 0001:00047ce0       ??_ECFontPropPage@@UAEPAXI@Z 5f548ce0 f i ppgfont.obj
 0001:00047d10       ??0CSizeComboBox@@QAE@XZ   5f548d10 f i ppgfont.obj
 0001:00047d30       ??1CSizeComboBox@@UAE@XZ   5f548d30 f i ppgfont.obj
 0001:00047d50       ??1CFontPropPage@@UAE@XZ   5f548d50 f i ppgfont.obj
 0001:00047e10       ??_GCSizeComboBox@@UAEPAXI@Z 5f548e10 f i ppgfont.obj
 0001:00047e10       ??_ECSizeComboBox@@UAEPAXI@Z 5f548e10 f i ppgfont.obj
 0001:00047e40       ??0tagFONTOBJECT@@QAE@XZ   5f548e40 f i ppgfont.obj
 0001:00047e60       ??1tagFONTOBJECT@@QAE@XZ   5f548e60 f i ppgfont.obj
 0001:00047e80       ??0tagFONTOBJECT@@QAE@ABU0@@Z 5f548e80 f i ppgfont.obj
 0001:00047ef0       ??_GCFontComboBox@@UAEPAXI@Z 5f548ef0 f i ppgfont.obj
 0001:00047ef0       ??_ECFontComboBox@@UAEPAXI@Z 5f548ef0 f i ppgfont.obj
 0001:00047f20       ??_9@$BOM@AE               5f548f20 f i ppgfont.obj
 0001:00047f30       ??0CFontPropPageFactory@CFontPropPage@@QAE@ABU_GUID@@PAUCRuntimeClass@@HPBD@Z 5f548f30 f i ppgfont.obj
 0001:00047f70       ??_ECColorPropPageFactory@CColorPropPage@@UAEPAXI@Z 5f548f70 f i ppgfont.obj
 0001:00047f70       ??_GCFontPropPageFactory@CFontPropPage@@UAEPAXI@Z 5f548f70 f i ppgfont.obj
 0001:00047f70       ??_ECFontPropPageFactory@CFontPropPage@@UAEPAXI@Z 5f548f70 f i ppgfont.obj
 0001:00047f70       ??_ECPicturePropPageFactory@CPicturePropPage@@UAEPAXI@Z 5f548f70 f i ppgfont.obj
 0001:00047f70       ??_GCPicturePropPageFactory@CPicturePropPage@@UAEPAXI@Z 5f548f70 f i ppgfont.obj
 0001:00047f70       ??_GCColorPropPageFactory@CColorPropPage@@UAEPAXI@Z 5f548f70 f i ppgfont.obj
 0001:00047fa0       ?_GetBaseMessageMap@CPicturePropPage@@KGPBUAFX_MSGMAP@@XZ 5f548fa0 f   ppgpict.obj
 0001:00047faa       ?GetMessageMap@CPicturePropPage@@MBEPBUAFX_MSGMAP@@XZ 5f548faa f   ppgpict.obj
 0001:00047fba       ??0CPicturePropPage@@QAE@XZ 5f548fba f   ppgpict.obj
 0001:0004803d       ??1CPicturePropPage@@UAE@XZ 5f54903d f   ppgpict.obj
 0001:000480db       ?OnInitDialog@CPicturePropPage@@MAEHXZ 5f5490db f   ppgpict.obj
 0001:0004813a       ?DoDataExchange@CPicturePropPage@@MAEXPAVCDataExchange@@@Z 5f54913a f   ppgpict.obj
 0001:00048209       ?SetPictureProp@CPicturePropPage@@IAEHPAVCDataExchange@@PAUIPictureDisp@@PBD@Z 5f549209 f   ppgpict.obj
 0001:00048426       ?GetPictureProp@CPicturePropPage@@IAEHPAVCDataExchange@@PAPAUIPictureDisp@@PBD@Z 5f549426 f   ppgpict.obj
 0001:0004865e       ?OnPaint@CPicturePropPage@@IAEXXZ 5f54965e f   ppgpict.obj
 0001:000488d3       ?_AfxCreateStreamOnFile@@YAJPBDPAPAUIStream@@PAJ@Z 5f5498d3 f   ppgpict.obj
 0001:00048ae6       ?OnBrowse@CPicturePropPage@@IAEXXZ 5f549ae6 f   ppgpict.obj
 0001:00048e9a       ?OnClear@CPicturePropPage@@IAEXXZ 5f549e9a f   ppgpict.obj
 0001:00048ef8       ?ChangePicture@CPicturePropPage@@IAEXPAUIPicture@@@Z 5f549ef8 f   ppgpict.obj
 0001:00048fe1       ?OnSelchangePictProp@CPicturePropPage@@IAEXXZ 5f549fe1 f   ppgpict.obj
 0001:00049099       ?OnEditProperty@CPicturePropPage@@MAEHJ@Z 5f54a099 f   ppgpict.obj
 0001:000490bb       ?OnObjectsChanged@CPicturePropPage@@MAEXXZ 5f54a0bb f   ppgpict.obj
 0001:00049178       ?GetClassID@CPicturePropPage@@UAEJPAU_GUID@@@Z 5f54a178 f   ppgpict.obj
 0001:000491ad       ?UpdateRegistry@CPicturePropPageFactory@CPicturePropPage@@UAEHH@Z 5f54a1ad f   ppgpict.obj
 0001:000491f0       ??_ECPicturePropPage@@UAEPAXI@Z 5f54a1f0 f i ppgpict.obj
 0001:000491f0       ??_GCPicturePropPage@@UAEPAXI@Z 5f54a1f0 f i ppgpict.obj
 0001:00049220       ??0CFileStatus@@QAE@XZ     5f54a220 f i ppgpict.obj
 0001:00049250       ??1CFileDialog@@UAE@XZ     5f54a250 f i ppgpict.obj
 0001:000492a0       ??0CPicturePropPageFactory@CPicturePropPage@@QAE@ABU_GUID@@PAUCRuntimeClass@@HPBD@Z 5f54a2a0 f i ppgpict.obj
 0001:000492e0       ??1CFontPropPageFactory@CFontPropPage@@UAE@XZ 5f54a2e0 f i ppgpict.obj
 0001:000492e0       ??1CPicturePropPageFactory@CPicturePropPage@@UAE@XZ 5f54a2e0 f i ppgpict.obj
 0001:000492e0       ??1CColorPropPageFactory@CColorPropPage@@UAE@XZ 5f54a2e0 f i ppgpict.obj
 0001:00049300       ?_GetBaseMessageMap@CStockPropPage@@KGPBUAFX_MSGMAP@@XZ 5f54a300 f   ppgstock.obj
 0001:0004930a       ?GetMessageMap@CStockPropPage@@MBEPBUAFX_MSGMAP@@XZ 5f54a30a f   ppgstock.obj
 0001:0004931a       ?_AfxSizeComboToContent@@YAXPAVCComboBox@@@Z 5f54a31a f   ppgstock.obj
 0001:000493a8       ??0CStockPropPage@@QAE@II@Z 5f54a3a8 f   ppgstock.obj
 0001:00049419       ?FillPropnameList@CStockPropPage@@IAEXABU_GUID@@HAAVCComboBox@@@Z 5f54a419 f   ppgstock.obj
 0001:0004974e       ?OnSelchangePropname@CStockPropPage@@IAEXAAVCComboBox@@@Z 5f54a74e f   ppgstock.obj
 0001:000497d1       ?OnEditProperty@CStockPropPage@@IAEHJAAVCComboBox@@@Z 5f54a7d1 f   ppgstock.obj
 0001:00049839       ?AfxOleTypeMatchGuid@@YGHPAUITypeInfo@@PAUtagTYPEDESC@@ABU_GUID@@K@Z 5f54a839 f   ppgstock.obj
 0001:00049a00       ??_GCStockPropPage@@UAEPAXI@Z 5f54aa00 f i ppgstock.obj
 0001:00049a00       ??_ECStockPropPage@@UAEPAXI@Z 5f54aa00 f i ppgstock.obj
 0001:00049a30       ?IsOptimizedDraw@COleControl@@QAEHXZ 5f54aa30 f   ctlinl.obj
 0001:00049a4a       ?IsConvertingVBX@COleControl@@QAEHXZ 5f54aa4a f   ctlinl.obj
 0001:00049a64       ?FireKeyDown@COleControl@@QAEXPAGF@Z 5f54aa64 f   ctlinl.obj
 0001:00049a90       ?FireKeyUp@COleControl@@QAEXPAGF@Z 5f54aa90 f   ctlinl.obj
 0001:00049abc       ?FireKeyPress@COleControl@@QAEXPAG@Z 5f54aabc f   ctlinl.obj
 0001:00049ae3       ?FireMouseDown@COleControl@@QAEXFFJJ@Z 5f54aae3 f   ctlinl.obj
 0001:00049b18       ?FireMouseUp@COleControl@@QAEXFFJJ@Z 5f54ab18 f   ctlinl.obj
 0001:00049b4d       ?FireMouseMove@COleControl@@QAEXFFJJ@Z 5f54ab4d f   ctlinl.obj
 0001:00049b82       ?FireClick@COleControl@@QAEXXZ 5f54ab82 f   ctlinl.obj
 0001:00049ba0       ?FireDblClick@COleControl@@QAEXXZ 5f54aba0 f   ctlinl.obj
 0001:00049bbe       ?FireReadyStateChange@COleControl@@QAEXXZ 5f54abbe f   ctlinl.obj
 0001:00049be9       ?InternalSetReadyState@COleControl@@QAEXJ@Z 5f54abe9 f   ctlinl.obj
 0001:00049c41       ?ExchangeVersion@COleControl@@QAEHPAVCPropExchange@@KH@Z 5f54ac41 f   ctlinl.obj
 0001:00049c67       ?GetStockEventMask@COleControl@@IBEKXZ 5f54ac67 f   ctlinl.obj
 0001:00049c85       ?GetStockPropMask@COleControl@@IBEKXZ 5f54ac85 f   ctlinl.obj
 0001:00049ca0       ?RequestAsynchronousExchange@COleControl@@QAEXK@Z 5f54aca0 f   ctlinl.obj
 0001:00049cc6       ??0CPropExchange@@IAE@XZ   5f54acc6 f   ctlinl.obj
 0001:00049cf1       ?IsLoading@CPropExchange@@QAEHXZ 5f54acf1 f   ctlinl.obj
 0001:00049d02       ?GetVersion@CPropExchange@@QAEKXZ 5f54ad02 f   ctlinl.obj
 0001:00049d13       ?IsAsynchronous@CPropExchange@@QAEHXZ 5f54ad13 f   ctlinl.obj
 0001:00049d24       ??0CDataPathProperty@@QAE@PAVCOleControl@@@Z 5f54ad24 f   ctlinl.obj
 0001:00049d86       ??0CDataPathProperty@@QAE@PBDPAVCOleControl@@@Z 5f54ad86 f   ctlinl.obj
 0001:00049dec       ?SetPath@CDataPathProperty@@QAEXPBD@Z 5f54adec f   ctlinl.obj
 0001:00049e18       ?GetPath@CDataPathProperty@@QBE?AVCString@@XZ 5f54ae18 f   ctlinl.obj
 0001:00049e59       ?GetControl@CDataPathProperty@@QAEPAVCOleControl@@XZ 5f54ae59 f   ctlinl.obj
 0001:00049e7a       ?SetControl@CDataPathProperty@@QAEXPAVCOleControl@@@Z 5f54ae7a f   ctlinl.obj
 0001:00049ea0       ??0CCachedDataPathProperty@@QAE@PAVCOleControl@@@Z 5f54aea0 f   ctlinl.obj
 0001:00049f02       ??0CCachedDataPathProperty@@QAE@PBDPAVCOleControl@@@Z 5f54af02 f   ctlinl.obj
 0001:00049f68       ?DDP_LBString@@YGXPAVCDataExchange@@HAAVCString@@PBD@Z 5f54af68 f   ctlinl.obj
 0001:00049f84       ?DDP_LBStringExact@@YGXPAVCDataExchange@@HAAVCString@@PBD@Z 5f54af84 f   ctlinl.obj
 0001:00049fa0       ?DDP_LBIndex@@YGXPAVCDataExchange@@HAAHPBD@Z 5f54afa0 f   ctlinl.obj
 0001:00049fbc       ?DDP_CBString@@YGXPAVCDataExchange@@HAAVCString@@PBD@Z 5f54afbc f   ctlinl.obj
 0001:00049fd8       ?DDP_CBStringExact@@YGXPAVCDataExchange@@HAAVCString@@PBD@Z 5f54afd8 f   ctlinl.obj
 0001:00049ff4       ?DDP_CBIndex@@YGXPAVCDataExchange@@HAAHPBD@Z 5f54aff4 f   ctlinl.obj
 0001:0004a010       ??_GCDataPathProperty@@UAEPAXI@Z 5f54b010 f i ctlinl.obj
 0001:0004a040       ??_GCCachedDataPathProperty@@UAEPAXI@Z 5f54b040 f i ctlinl.obj
 0001:0004a06c       ?AfxAssertFailedLine@@YGHPBDH@Z 5f54b06c f   MFC42D:MFC42D.DLL
 0001:0004a072       ?AfxSetModuleState@@YGPAVAFX_MODULE_STATE@@PAV1@@Z 5f54b072 f   MFC42D:MFC42D.DLL
 0001:0004a078       ?AfxGetThreadState@@YGPAV_AFX_THREAD_STATE@@XZ 5f54b078 f   MFC42D:MFC42D.DLL
 0001:0004a07e       ?AfxGetModuleState@@YGPAVAFX_MODULE_STATE@@XZ 5f54b07e f   MFC42D:MFC42D.DLL
 0001:0004a084       ?AfxTermThread@@YGXPAUHINSTANCE__@@@Z 5f54b084 f   MFC42D:MFC42D.DLL
 0001:0004a08a       ?AfxTermExtensionModule@@YGXAAUAFX_EXTENSION_MODULE@@H@Z 5f54b08a f   MFC42D:MFC42D.DLL
 0001:0004a090       ??0CDynLinkLibrary@@QAE@AAUAFX_EXTENSION_MODULE@@H@Z 5f54b090 f   MFC42D:MFC42D.DLL
 0001:0004a096       ??2CObject@@SGPAXI@Z       5f54b096 f   MFC42D:MFC42D.DLL
 0001:0004a09c       ?AfxWinInit@@YGHPAUHINSTANCE__@@0PADH@Z 5f54b09c f   MFC42D:MFC42D.DLL
 0001:0004a0a2       ?AfxCoreInitModule@@YGXXZ  5f54b0a2 f   MFC42D:MFC42D.DLL
 0001:0004a0a8       ?AfxInitExtensionModule@@YGHAAUAFX_EXTENSION_MODULE@@PAUHINSTANCE__@@@Z 5f54b0a8 f   MFC42D:MFC42D.DLL
 0001:0004a0ae       ??3CObject@@SGXPAX@Z       5f54b0ae f   MFC42D:MFC42D.DLL
 0001:0004a0b4       ?AfxGetAppModuleState@@YGPAVAFX_MODULE_STATE@@XZ 5f54b0b4 f   MFC42D:MFC42D.DLL
 0001:0004a0ba       ??1AFX_MAINTAIN_STATE2@@QAE@XZ 5f54b0ba f   MFC42D:MFC42D.DLL
 0001:0004a0c0       ??0AFX_MAINTAIN_STATE2@@QAE@PAVAFX_MODULE_STATE@@@Z 5f54b0c0 f   MFC42D:MFC42D.DLL
 0001:0004a0c6       ??0CWinApp@@QAE@PBD@Z      5f54b0c6 f   MFC42D:MFC42D.DLL
 0001:0004a0cc       ??1CWinApp@@UAE@XZ         5f54b0cc f   MFC42D:MFC42D.DLL
 0001:0004a0d2       ?AfxWndProc@@YGJPAUHWND__@@IIJ@Z 5f54b0d2 f   MFC42D:MFC42D.DLL
 0001:0004a0d8       ??0AFX_MODULE_STATE@@QAE@HP6GJPAUHWND__@@IIJ@ZKH@Z 5f54b0d8 f   MFC42D:MFC42D.DLL
 0001:0004a0de       ??1AFX_MODULE_STATE@@UAE@XZ 5f54b0de f   MFC42D:MFC42D.DLL
 0001:0004a0e4       ??3@YAXPAX@Z               5f54b0e4 f   MFC42D:MFC42D.DLL
 0001:0004a0ea       ??2@YAPAXI@Z               5f54b0ea f   MFC42D:MFC42D.DLL
 0001:0004a0f0       ??1CCmdTarget@@UAE@XZ      5f54b0f0 f   MFC42D:MFC42D.DLL
 0001:0004a0f6       ??1CMemFile@@UAE@XZ        5f54b0f6 f   MFC42D:MFC42D.DLL
 0001:0004a0fc       ??1CString@@QAE@XZ         5f54b0fc f   MFC42D:MFC42D.DLL
 0001:0004a102       ??1CDC@@UAE@XZ             5f54b102 f   MFC42D:MFC42D.DLL
 0001:0004a108       ??1CDWordArray@@UAE@XZ     5f54b108 f   MFC42D:MFC42D.DLL
 0001:0004a10e       ??1CView@@UAE@XZ           5f54b10e f   MFC42D:MFC42D.DLL
 0001:0004a114       ??3CObject@@SGXPAXPBDH@Z   5f54b114 f   MFC42D:MFC42D.DLL
 0001:0004a11a       ?AfxOleGetMessageFilter@@YGPAVCOleMessageFilter@@XZ 5f54b11a f   MFC42D:MFC42D.DLL
 0001:0004a120       ??2CObject@@SGPAXIPBDH@Z   5f54b120 f   MFC42D:MFC42D.DLL
 0001:0004a126       ?AfxGetThread@@YGPAVCWinThread@@XZ 5f54b126 f   MFC42D:MFC42D.DLL
 0001:0004a12c       ?AfxTrace@@YAXPBDZZ        5f54b12c f   MFC42D:MFC42D.DLL
 0001:0004a132       ?AfxOleSetUserCtrl@@YGXH@Z 5f54b132 f   MFC42D:MFC42D.DLL
 0001:0004a138       ?GetConnectionHook@CCmdTarget@@MAEPAUIConnectionPoint@@ABU_GUID@@@Z 5f54b138 f   MFC42D:MFC42D.DLL
 0001:0004a13e       ?GetExtraConnectionPoints@CCmdTarget@@MAEHPAVCPtrArray@@@Z 5f54b13e f   MFC42D:MFC42D.DLL
 0001:0004a144       ?GetInterfaceHook@CCmdTarget@@UAEPAUIUnknown@@PBX@Z 5f54b144 f   MFC42D:MFC42D.DLL
 0001:0004a14a       ?OnCreateAggregates@CCmdTarget@@UAEHXZ 5f54b14a f   MFC42D:MFC42D.DLL
 0001:0004a150       ?GetEventSinkMap@CCmdTarget@@MBEPBUAFX_EVENTSINKMAP@@XZ 5f54b150 f   MFC42D:MFC42D.DLL
 0001:0004a156       ?GetConnectionMap@CCmdTarget@@MBEPBUAFX_CONNECTIONMAP@@XZ 5f54b156 f   MFC42D:MFC42D.DLL
 0001:0004a15c       ?GetDispatchMap@CCmdTarget@@MBEPBUAFX_DISPMAP@@XZ 5f54b15c f   MFC42D:MFC42D.DLL
 0001:0004a162       ?GetCommandMap@CCmdTarget@@MBEPBUAFX_OLECMDMAP@@XZ 5f54b162 f   MFC42D:MFC42D.DLL
 0001:0004a168       ?GetMessageMap@CCmdTarget@@MBEPBUAFX_MSGMAP@@XZ 5f54b168 f   MFC42D:MFC42D.DLL
 0001:0004a16e       ?GetTypeLib@CCmdTarget@@UAEJKPAPAUITypeLib@@@Z 5f54b16e f   MFC42D:MFC42D.DLL
 0001:0004a174       ?GetTypeLibCache@CCmdTarget@@UAEPAVCTypeLibCache@@XZ 5f54b174 f   MFC42D:MFC42D.DLL
 0001:0004a17a       ?GetTypeInfoCount@CCmdTarget@@UAEIXZ 5f54b17a f   MFC42D:MFC42D.DLL
 0001:0004a180       ?GetDispatchIID@CCmdTarget@@UAEHPAU_GUID@@@Z 5f54b180 f   MFC42D:MFC42D.DLL
 0001:0004a186       ?IsInvokeAllowed@CCmdTarget@@UAEHJ@Z 5f54b186 f   MFC42D:MFC42D.DLL
 0001:0004a18c       ?OnFinalRelease@CCmdTarget@@UAEXXZ 5f54b18c f   MFC42D:MFC42D.DLL
 0001:0004a192       ?OnCmdMsg@CCmdTarget@@UAEHIHPAXPAUAFX_CMDHANDLERINFO@@@Z 5f54b192 f   MFC42D:MFC42D.DLL
 0001:0004a198       ?AfxOleLockApp@@YGXXZ      5f54b198 f   MFC42D:MFC42D.DLL
 0001:0004a19e       ?AfxAssertValidObject@@YGXPBVCObject@@PBDH@Z 5f54b19e f   MFC42D:MFC42D.DLL
 0001:0004a1a4       ?AfxOleUnlockApp@@YGXXZ    5f54b1a4 f   MFC42D:MFC42D.DLL
 0001:0004a1aa       ?AfxGetApp@@YGPAVCWinApp@@XZ 5f54b1aa f   MFC42D:MFC42D.DLL
 0001:0004a1b0       ?Delete@CException@@QAEXXZ 5f54b1b0 f   MFC42D:MFC42D.DLL
 0001:0004a1b6       ?IsKindOf@CObject@@QBEHPBUCRuntimeClass@@@Z 5f54b1b6 f   MFC42D:MFC42D.DLL
 0001:0004a1bc       ?AfxGetAppName@@YGPBDXZ    5f54b1bc f   MFC42D:MFC42D.DLL
 0001:0004a1c2       ??BCString@@QBEPBDXZ       5f54b1c2 f   MFC42D:MFC42D.DLL
 0001:0004a1c8       ?GetTitle@CDocument@@QBEABVCString@@XZ 5f54b1c8 f   MFC42D:MFC42D.DLL
 0001:0004a1ce       ?AfxIsValidAddress@@YGHPBXIH@Z 5f54b1ce f   MFC42D:MFC42D.DLL
 0001:0004a1d4       ?AfxThrowArchiveException@@YGXHPBD@Z 5f54b1d4 f   MFC42D:MFC42D.DLL
 0001:0004a1da       ?Read@CArchive@@QAEIPAXI@Z 5f54b1da f   MFC42D:MFC42D.DLL
 0001:0004a1e0       ?AfxThrowMemoryException@@YGXXZ 5f54b1e0 f   MFC42D:MFC42D.DLL
 0001:0004a1e6       ??5CArchive@@QAEAAV0@AAK@Z 5f54b1e6 f   MFC42D:MFC42D.DLL
 0001:0004a1ec       ?Write@CArchive@@QAEXPBXI@Z 5f54b1ec f   MFC42D:MFC42D.DLL
 0001:0004a1f2       ??6CArchive@@QAEAAV0@K@Z   5f54b1f2 f   MFC42D:MFC42D.DLL
 0001:0004a1f8       ??5CArchive@@QAEAAV0@AAG@Z 5f54b1f8 f   MFC42D:MFC42D.DLL
 0001:0004a1fe       ??6CArchive@@QAEAAV0@G@Z   5f54b1fe f   MFC42D:MFC42D.DLL
 0001:0004a204       ?IsStoring@CArchive@@QBEHXZ 5f54b204 f   MFC42D:MFC42D.DLL
 0001:0004a20a       ?GetClientRect@CWnd@@QBEXPAUtagRECT@@@Z 5f54b20a f   MFC42D:MFC42D.DLL
 0001:0004a210       ?IsEmpty@CString@@QBEHXZ   5f54b210 f   MFC42D:MFC42D.DLL
 0001:0004a216       ?GetPathName@CDocument@@QBEABVCString@@XZ 5f54b216 f   MFC42D:MFC42D.DLL
 0001:0004a21c       ?GetParentFrame@CWnd@@QBEPAVCFrameWnd@@XZ 5f54b21c f   MFC42D:MFC42D.DLL
 0001:0004a222       ?AfxGetFileTitle@@YGIPBDPADI@Z 5f54b222 f   MFC42D:MFC42D.DLL
 0001:0004a228       ?IsPrinting@CDC@@QBEHXZ    5f54b228 f   MFC42D:MFC42D.DLL
 0001:0004a22e       ?GetWindowExt@CDC@@QBE?AVCSize@@XZ 5f54b22e f   MFC42D:MFC42D.DLL
 0001:0004a234       ?GetWindowOrg@CDC@@QBE?AVCPoint@@XZ 5f54b234 f   MFC42D:MFC42D.DLL
 0001:0004a23a       ?DPtoHIMETRIC@CDC@@QBEXPAUtagSIZE@@@Z 5f54b23a f   MFC42D:MFC42D.DLL
 0001:0004a240       ?AfxIsValidString@@YGHPBDH@Z 5f54b240 f   MFC42D:MFC42D.DLL
 0001:0004a246       ??6CDumpContext@@QAEAAV0@E@Z 5f54b246 f   MFC42D:MFC42D.DLL
 0001:0004a24c       ??6CDumpContext@@QAEAAV0@J@Z 5f54b24c f   MFC42D:MFC42D.DLL
 0001:0004a252       ??6CDumpContext@@QAEAAV0@H@Z 5f54b252 f   MFC42D:MFC42D.DLL
 0001:0004a258       ??6CDumpContext@@QAEAAV0@K@Z 5f54b258 f   MFC42D:MFC42D.DLL
 0001:0004a25e       ??6CDumpContext@@QAEAAV0@PBX@Z 5f54b25e f   MFC42D:MFC42D.DLL
 0001:0004a264       ??6CDumpContext@@QAEAAV0@PBD@Z 5f54b264 f   MFC42D:MFC42D.DLL
 0001:0004a26a       ?Dump@CCmdTarget@@UBEXAAVCDumpContext@@@Z 5f54b26a f   MFC42D:MFC42D.DLL
 0001:0004a270       ?AssertValid@CCmdTarget@@UBEXXZ 5f54b270 f   MFC42D:MFC42D.DLL
 0001:0004a276       ?Serialize@CObject@@UAEXAAVCArchive@@@Z 5f54b276 f   MFC42D:MFC42D.DLL
 0001:0004a27c       ?GetRuntimeClass@CCmdTarget@@UBEPAUCRuntimeClass@@XZ 5f54b27c f   MFC42D:MFC42D.DLL
 0001:0004a282       ??0CString@@QAE@XZ         5f54b282 f   MFC42D:MFC42D.DLL
 0001:0004a288       ??0CCmdTarget@@QAE@XZ      5f54b288 f   MFC42D:MFC42D.DLL
 0001:0004a28e       ?DelayUpdateFrameTitle@CFrameWnd@@QAEXXZ 5f54b28e f   MFC42D:MFC42D.DLL
 0001:0004a294       ?SendMessageA@CWnd@@QAEJIIJ@Z 5f54b294 f   MFC42D:MFC42D.DLL
 0001:0004a29a       ?GetSafeHmenu@CMenu@@QBEPAUHMENU__@@XZ 5f54b29a f   MFC42D:MFC42D.DLL
 0001:0004a2a0       ?AfxDynamicDownCast@@YAPAVCObject@@PAUCRuntimeClass@@PAV1@@Z 5f54b2a0 f   MFC42D:MFC42D.DLL
 0001:0004a2a6       ?IsWindowEnabled@CWnd@@QBEHXZ 5f54b2a6 f   MFC42D:MFC42D.DLL
 0001:0004a2ac       ?GetSafeHwnd@CWnd@@QBEPAUHWND__@@XZ 5f54b2ac f   MFC42D:MFC42D.DLL
 0001:0004a2b2       ?AfxIsDescendant@@YGHPAUHWND__@@0@Z 5f54b2b2 f   MFC42D:MFC42D.DLL
 0001:0004a2b8       ?AfxStaticDownCast@@YAPAVCObject@@PAUCRuntimeClass@@PAV1@@Z 5f54b2b8 f   MFC42D:MFC42D.DLL
 0001:0004a2be       ?GetParent@CWnd@@QBEPAV1@XZ 5f54b2be f   MFC42D:MFC42D.DLL
 0001:0004a2c4       ?GetFocus@CWnd@@SGPAV1@XZ  5f54b2c4 f   MFC42D:MFC42D.DLL
 0001:0004a2ca       ?GetDocument@CView@@QBEPAVCDocument@@XZ 5f54b2ca f   MFC42D:MFC42D.DLL
 0001:0004a2d0       ?ModifyStyle@CWnd@@QAEHKKI@Z 5f54b2d0 f   MFC42D:MFC42D.DLL
 0001:0004a2d6       ?GetStyle@CWnd@@QBEKXZ     5f54b2d6 f   MFC42D:MFC42D.DLL
 0001:0004a2dc       ?ShowControlBar@CFrameWnd@@QAEXPAVCControlBar@@HH@Z 5f54b2dc f   MFC42D:MFC42D.DLL
 0001:0004a2e2       ?GetBarStyle@CControlBar@@QAEKXZ 5f54b2e2 f   MFC42D:MFC42D.DLL
 0001:0004a2e8       ?GetNext@CPtrList@@QAEAAPAXAAPAU__POSITION@@@Z 5f54b2e8 f   MFC42D:MFC42D.DLL
 0001:0004a2ee       ?GetHeadPosition@CPtrList@@QBEPAU__POSITION@@XZ 5f54b2ee f   MFC42D:MFC42D.DLL
 0001:0004a2f4       ?GetDocTemplate@CDocument@@QBEPAVCDocTemplate@@XZ 5f54b2f4 f   MFC42D:MFC42D.DLL
 0001:0004a2fa       ?GetTopLevelFrame@CWnd@@QBEPAVCFrameWnd@@XZ 5f54b2fa f   MFC42D:MFC42D.DLL
 0001:0004a300       ?GetParentSplitter@CView@@SGPAVCSplitterWnd@@PBVCWnd@@H@Z 5f54b300 f   MFC42D:MFC42D.DLL
 0001:0004a306       ?SetFocus@CWnd@@QAEPAV1@XZ 5f54b306 f   MFC42D:MFC42D.DLL
 0001:0004a30c       ?GetTopLevelParent@CWnd@@QBEPAV1@XZ 5f54b30c f   MFC42D:MFC42D.DLL
 0001:0004a312       ?AfxGetMainWnd@@YGPAVCWnd@@XZ 5f54b312 f   MFC42D:MFC42D.DLL
 0001:0004a318       ?DelayRecalcLayout@CFrameWnd@@QAEXH@Z 5f54b318 f   MFC42D:MFC42D.DLL
 0001:0004a31e       ?IsRectEmpty@CRect@@QBEHXZ 5f54b31e f   MFC42D:MFC42D.DLL
 0001:0004a324       ?IntersectRect@CRect@@QAEHPBUtagRECT@@0@Z 5f54b324 f   MFC42D:MFC42D.DLL
 0001:0004a32a       ??BCRect@@QAEPAUtagRECT@@XZ 5f54b32a f   MFC42D:MFC42D.DLL
 0001:0004a330       ??BCRect@@QBEPBUtagRECT@@XZ 5f54b330 f   MFC42D:MFC42D.DLL
 0001:0004a336       ??0CRect@@QAE@XZ           5f54b336 f   MFC42D:MFC42D.DLL
 0001:0004a33c       ?FromHandle@CWnd@@SGPAV1@PAUHWND__@@@Z 5f54b33c f   MFC42D:MFC42D.DLL
 0001:0004a342       ?PostMessageA@CWnd@@QAEHIIJ@Z 5f54b342 f   MFC42D:MFC42D.DLL
 0001:0004a348       ?CanEnterHelpMode@CFrameWnd@@QAEHXZ 5f54b348 f   MFC42D:MFC42D.DLL
 0001:0004a34e       ??4CString@@QAEABV0@PBG@Z  5f54b34e f   MFC42D:MFC42D.DLL
 0001:0004a354       ?Empty@CString@@QAEXXZ     5f54b354 f   MFC42D:MFC42D.DLL
 0001:0004a35a       ?FromHandle@CMenu@@SGPAV1@PAUHMENU__@@@Z 5f54b35a f   MFC42D:MFC42D.DLL
 0001:0004a360       ??0CSize@@QAE@UtagSIZE@@@Z 5f54b360 f   MFC42D:MFC42D.DLL
 0001:0004a366       ?CopyRect@CRect@@QAEXPBUtagRECT@@@Z 5f54b366 f   MFC42D:MFC42D.DLL
 0001:0004a36c       ?GetData@CProcessLocalObject@@QAEPAVCNoTrackObject@@P6GPAV2@XZ@Z 5f54b36c f   MFC42D:MFC42D.DLL
 0001:0004a372       ??3CNoTrackObject@@SGXPAX@Z 5f54b372 f   MFC42D:MFC42D.DLL
 0001:0004a378       ??2CNoTrackObject@@SGPAXI@Z 5f54b378 f   MFC42D:MFC42D.DLL
 0001:0004a37e       ?SetRectEmpty@CRect@@QAEXXZ 5f54b37e f   MFC42D:MFC42D.DLL
 0001:0004a384       ?SetRect@CRect@@QAEXHHHH@Z 5f54b384 f   MFC42D:MFC42D.DLL
 0001:0004a38a       ??0CSize@@QAE@HH@Z         5f54b38a f   MFC42D:MFC42D.DLL
 0001:0004a390       ?AfxIsValidString@@YGHPBGH@Z 5f54b390 f   MFC42D:MFC42D.DLL
 0001:0004a396       ?GetBufferSetLength@CString@@QAEPADH@Z 5f54b396 f   MFC42D:MFC42D.DLL
 0001:0004a39c       ?AfxA2WHelper@@YGPAGPAGPBDH@Z 5f54b39c f   MFC42D:MFC42D.DLL
 0001:0004a3a2       ?AfxW2AHelper@@YGPADPADPBGH@Z 5f54b3a2 f   MFC42D:MFC42D.DLL
 0001:0004a3a8       ?SetHandle@CSharedFile@@QAEXPAXH@Z 5f54b3a8 f   MFC42D:MFC42D.DLL
 0001:0004a3ae       ??0CSharedFile@@QAE@II@Z   5f54b3ae f   MFC42D:MFC42D.DLL
 0001:0004a3b4       ??0CFile@@QAE@XZ           5f54b3b4 f   MFC42D:MFC42D.DLL
 0001:0004a3ba       ??2@YAPAXIPBDH@Z           5f54b3ba f   MFC42D:MFC42D.DLL
 0001:0004a3c0       ??1CSharedFile@@UAE@XZ     5f54b3c0 f   MFC42D:MFC42D.DLL
 0001:0004a3c6       ?Detach@CSharedFile@@QAEPAXXZ 5f54b3c6 f   MFC42D:MFC42D.DLL
 0001:0004a3cc       ??6CDumpContext@@QAEAAV0@G@Z 5f54b3cc f   MFC42D:MFC42D.DLL
 0001:0004a3d2       ??6CDumpContext@@QAEAAV0@I@Z 5f54b3d2 f   MFC42D:MFC42D.DLL
 0001:0004a3d8       ?GetData@CString@@IBEPAUCStringData@@XZ 5f54b3d8 f   MFC42D:MFC42D.DLL
 0001:0004a3de       ?ReportError@CException@@UAEHII@Z 5f54b3de f   MFC42D:MFC42D.DLL
 0001:0004a3e4       ?Dump@CObject@@UBEXAAVCDumpContext@@@Z 5f54b3e4 f   MFC42D:MFC42D.DLL
 0001:0004a3ea       ?AssertValid@CObject@@UBEXXZ 5f54b3ea f   MFC42D:MFC42D.DLL
 0001:0004a3f0       ??1CException@@UAE@XZ      5f54b3f0 f   MFC42D:MFC42D.DLL
 0001:0004a3f6       ??3CException@@SGXPAX@Z    5f54b3f6 f   MFC42D:MFC42D.DLL
 0001:0004a3fc       ?AfxLoadString@@YGHIPADI@Z 5f54b3fc f   MFC42D:MFC42D.DLL
 0001:0004a402       ??4CString@@QAEABV0@PBD@Z  5f54b402 f   MFC42D:MFC42D.DLL
 0001:0004a408       ??0CException@@QAE@XZ      5f54b408 f   MFC42D:MFC42D.DLL
 0001:0004a40e       ??3CException@@SGXPAXPBDH@Z 5f54b40e f   MFC42D:MFC42D.DLL
 0001:0004a414       ?PreInitDialog@CDialog@@MAEXXZ 5f54b414 f   MFC42D:MFC42D.DLL
 0001:0004a41a       ?OnCancel@CCommonDialog@@MAEXXZ 5f54b41a f   MFC42D:MFC42D.DLL
 0001:0004a420       ?OnOK@CCommonDialog@@MAEXXZ 5f54b420 f   MFC42D:MFC42D.DLL
 0001:0004a426       ?OnSetFont@CDialog@@UAEXPAVCFont@@@Z 5f54b426 f   MFC42D:MFC42D.DLL
 0001:0004a42c       ?OnInitDialog@CDialog@@UAEHXZ 5f54b42c f   MFC42D:MFC42D.DLL
 0001:0004a432       ?SetOccDialogInfo@CDialog@@MAEHPAU_AFX_OCC_DIALOG_INFO@@@Z 5f54b432 f   MFC42D:MFC42D.DLL
 0001:0004a438       ?IsFrameWnd@CWnd@@UBEHXZ   5f54b438 f   MFC42D:MFC42D.DLL
 0001:0004a43e       ?CheckAutoCenter@CDialog@@UAEHXZ 5f54b43e f   MFC42D:MFC42D.DLL
 0001:0004a444       ?OnChildNotify@CWnd@@MAEHIIJPAJ@Z 5f54b444 f   MFC42D:MFC42D.DLL
 0001:0004a44a       ?PostNcDestroy@CWnd@@MAEXXZ 5f54b44a f   MFC42D:MFC42D.DLL
 0001:0004a450       ?DefWindowProcA@CWnd@@MAEJIIJ@Z 5f54b450 f   MFC42D:MFC42D.DLL
 0001:0004a456       ?OnWndMsg@CWnd@@MAEHIIJPAJ@Z 5f54b456 f   MFC42D:MFC42D.DLL
 0001:0004a45c       ?WindowProc@CWnd@@MAEJIIJ@Z 5f54b45c f   MFC42D:MFC42D.DLL
 0001:0004a462       ?OnAmbientProperty@CWnd@@UAEHPAVCOleControlSite@@JPAUtagVARIANT@@@Z 5f54b462 f   MFC42D:MFC42D.DLL
 0001:0004a468       ?PreTranslateMessage@CDialog@@UAEHPAUtagMSG@@@Z 5f54b468 f   MFC42D:MFC42D.DLL
 0001:0004a46e       ?EndModalState@CWnd@@UAEXXZ 5f54b46e f   MFC42D:MFC42D.DLL
 0001:0004a474       ?BeginModalState@CWnd@@UAEXXZ 5f54b474 f   MFC42D:MFC42D.DLL
 0001:0004a47a       ?DoDataExchange@CWnd@@MAEXPAVCDataExchange@@@Z 5f54b47a f   MFC42D:MFC42D.DLL
 0001:0004a480       ?GetSuperWndProcAddr@CWnd@@MAEPAP6GJPAUHWND__@@IIJ@ZXZ 5f54b480 f   MFC42D:MFC42D.DLL
 0001:0004a486       ?OnNotify@CWnd@@MAEHIJPAJ@Z 5f54b486 f   MFC42D:MFC42D.DLL
 0001:0004a48c       ?OnCommand@CWnd@@MAEHIJ@Z  5f54b48c f   MFC42D:MFC42D.DLL
 0001:0004a492       ?EndModalLoop@CWnd@@UAEXH@Z 5f54b492 f   MFC42D:MFC42D.DLL
 0001:0004a498       ?ContinueModal@CWnd@@UAEHXZ 5f54b498 f   MFC42D:MFC42D.DLL
 0001:0004a49e       ?WinHelpA@CWnd@@UAEXKI@Z   5f54b49e f   MFC42D:MFC42D.DLL
 0001:0004a4a4       ?GetScrollBarCtrl@CWnd@@UBEPAVCScrollBar@@H@Z 5f54b4a4 f   MFC42D:MFC42D.DLL
 0001:0004a4aa       ?OnToolHitTest@CWnd@@UBEHVCPoint@@PAUtagTOOLINFOA@@@Z 5f54b4aa f   MFC42D:MFC42D.DLL
 0001:0004a4b0       ?CalcWindowRect@CWnd@@UAEXPAUtagRECT@@I@Z 5f54b4b0 f   MFC42D:MFC42D.DLL
 0001:0004a4b6       ?PreCreateWindow@CWnd@@UAEHAAUtagCREATESTRUCTA@@@Z 5f54b4b6 f   MFC42D:MFC42D.DLL
 0001:0004a4bc       ?DestroyWindow@CWnd@@UAEHXZ 5f54b4bc f   MFC42D:MFC42D.DLL
 0001:0004a4c2       ?Create@CWnd@@UAEHPBD0KABUtagRECT@@PAV1@IPAUCCreateContext@@@Z 5f54b4c2 f   MFC42D:MFC42D.DLL
 0001:0004a4c8       ?PreSubclassWindow@CWnd@@UAEXXZ 5f54b4c8 f   MFC42D:MFC42D.DLL
 0001:0004a4ce       ?GetInterfaceMap@CCmdTarget@@MBEPBUAFX_INTERFACEMAP@@XZ 5f54b4ce f   MFC42D:MFC42D.DLL
 0001:0004a4d4       ?GetMessageMap@CCommonDialog@@MBEPBUAFX_MSGMAP@@XZ 5f54b4d4 f   MFC42D:MFC42D.DLL
 0001:0004a4da       ?OnFinalRelease@CWnd@@UAEXXZ 5f54b4da f   MFC42D:MFC42D.DLL
 0001:0004a4e0       ?OnCmdMsg@CDialog@@UAEHIHPAXPAUAFX_CMDHANDLERINFO@@@Z 5f54b4e0 f   MFC42D:MFC42D.DLL
 0001:0004a4e6       ?AssertValid@CDialog@@UBEXXZ 5f54b4e6 f   MFC42D:MFC42D.DLL
 0001:0004a4ec       ?AfxHelpEnabled@@YGHXZ     5f54b4ec f   MFC42D:MFC42D.DLL
 0001:0004a4f2       ??1CDialog@@UAE@XZ         5f54b4f2 f   MFC42D:MFC42D.DLL
 0001:0004a4f8       ?AfxMessageBox@@YGHIII@Z   5f54b4f8 f   MFC42D:MFC42D.DLL
 0001:0004a4fe       ?Format@CString@@QAAXPBDZZ 5f54b4fe f   MFC42D:MFC42D.DLL
 0001:0004a504       ?AfxStringFromCLSID@@YG?AVCString@@ABU_GUID@@@Z 5f54b504 f   MFC42D:MFC42D.DLL
 0001:0004a50a       ?PostModal@CDialog@@IAEXXZ 5f54b50a f   MFC42D:MFC42D.DLL
 0001:0004a510       ?PreModal@CDialog@@IAEPAUHWND__@@XZ 5f54b510 f   MFC42D:MFC42D.DLL
 0001:0004a516       ??1CWaitCursor@@QAE@XZ     5f54b516 f   MFC42D:MFC42D.DLL
 0001:0004a51c       ??0CWaitCursor@@QAE@XZ     5f54b51c f   MFC42D:MFC42D.DLL
 0001:0004a522       ?LoadStringA@CString@@QAEHI@Z 5f54b522 f   MFC42D:MFC42D.DLL
 0001:0004a528       ??6@YGAAVCDumpContext@@AAV0@ABVCString@@@Z 5f54b528 f   MFC42D:MFC42D.DLL
 0001:0004a52e       ?AfxThrowResourceException@@YGXXZ 5f54b52e f   MFC42D:MFC42D.DLL
 0001:0004a534       ??0CString@@QAE@PBD@Z      5f54b534 f   MFC42D:MFC42D.DLL
 0001:0004a53a       ??0CString@@QAE@PBDH@Z     5f54b53a f   MFC42D:MFC42D.DLL
 0001:0004a540       ?AfxDlgProc@@YGHPAUHWND__@@IIJ@Z 5f54b540 f   MFC42D:MFC42D.DLL
 0001:0004a546       ?DoModal@CDialog@@UAEHXZ   5f54b546 f   MFC42D:MFC42D.DLL
 0001:0004a54c       ??0CCommonDialog@@QAE@PAVCWnd@@@Z 5f54b54c f   MFC42D:MFC42D.DLL
 0001:0004a552       ?Dump@CDialog@@UBEXAAVCDumpContext@@@Z 5f54b552 f   MFC42D:MFC42D.DLL
 0001:0004a558       ?Detach@CWnd@@QAEPAUHWND__@@XZ 5f54b558 f   MFC42D:MFC42D.DLL
 0001:0004a55e       ?AfxUnhookWindowCreate@@YGHXZ 5f54b55e f   MFC42D:MFC42D.DLL
 0001:0004a564       ?AfxHookWindowCreate@@YGXPAVCWnd@@@Z 5f54b564 f   MFC42D:MFC42D.DLL
 0001:0004a56a       ?GetSafeOwner_@CWnd@@SGPAUHWND__@@PAU2@PAPAU2@@Z 5f54b56a f   MFC42D:MFC42D.DLL
 0001:0004a570       ?CenterWindow@CWnd@@QAEXPAV1@@Z 5f54b570 f   MFC42D:MFC42D.DLL
 0001:0004a576       ??4CString@@QAEABV0@ABV0@@Z 5f54b576 f   MFC42D:MFC42D.DLL
 0001:0004a57c       ??0CString@@QAE@ABV0@@Z    5f54b57c f   MFC42D:MFC42D.DLL
 0001:0004a582       ??1CProcessLocalObject@@QAE@XZ 5f54b582 f   MFC42D:MFC42D.DLL
 0001:0004a588       ?GetData@CByteArray@@QBEPBEXZ 5f54b588 f   MFC42D:MFC42D.DLL
 0001:0004a58e       ?GetSize@CByteArray@@QBEHXZ 5f54b58e f   MFC42D:MFC42D.DLL
 0001:0004a594       ??6CDumpContext@@QAEAAV0@N@Z 5f54b594 f   MFC42D:MFC42D.DLL
 0001:0004a59a       ??6CDumpContext@@QAEAAV0@M@Z 5f54b59a f   MFC42D:MFC42D.DLL
 0001:0004a5a0       ??6CDumpContext@@QAEAAV0@PBG@Z 5f54b5a0 f   MFC42D:MFC42D.DLL
 0001:0004a5a6       ??0CArchiveStream@@QAE@PAVCArchive@@@Z 5f54b5a6 f   MFC42D:MFC42D.DLL
 0001:0004a5ac       ??6CArchive@@QAEAAV0@N@Z   5f54b5ac f   MFC42D:MFC42D.DLL
 0001:0004a5b2       ??6CArchive@@QAEAAV0@M@Z   5f54b5b2 f   MFC42D:MFC42D.DLL
 0001:0004a5b8       ??6CArchive@@QAEAAV0@J@Z   5f54b5b8 f   MFC42D:MFC42D.DLL
 0001:0004a5be       ??6CArchive@@QAEAAV0@E@Z   5f54b5be f   MFC42D:MFC42D.DLL
 0001:0004a5c4       ??5CArchive@@QAEAAV0@AAN@Z 5f54b5c4 f   MFC42D:MFC42D.DLL
 0001:0004a5ca       ??5CArchive@@QAEAAV0@AAM@Z 5f54b5ca f   MFC42D:MFC42D.DLL
 0001:0004a5d0       ??5CArchive@@QAEAAV0@AAJ@Z 5f54b5d0 f   MFC42D:MFC42D.DLL
 0001:0004a5d6       ??5CArchive@@QAEAAV0@AAE@Z 5f54b5d6 f   MFC42D:MFC42D.DLL
 0001:0004a5dc       ?HashKey@@YGIPBG@Z         5f54b5dc f   MFC42D:MFC42D.DLL
 0001:0004a5e2       ?ReleaseBuffer@CString@@QAEXH@Z 5f54b5e2 f   MFC42D:MFC42D.DLL
 0001:0004a5e8       ?GetLength@CString@@QBEHXZ 5f54b5e8 f   MFC42D:MFC42D.DLL
 0001:0004a5ee       ??YCString@@QAEABV0@PBD@Z  5f54b5ee f   MFC42D:MFC42D.DLL
 0001:0004a5f4       ?GetBuffer@CString@@QAEPADH@Z 5f54b5f4 f   MFC42D:MFC42D.DLL
 0001:0004a5fa       ?GetDepth@CDumpContext@@QBEHXZ 5f54b5fa f   MFC42D:MFC42D.DLL
 0001:0004a600       ?AfxSetWindowText@@YGXPAUHWND__@@PBD@Z 5f54b600 f   MFC42D:MFC42D.DLL
 0001:0004a606       ?Fail@CDataExchange@@QAEXXZ 5f54b606 f   MFC42D:MFC42D.DLL
 0001:0004a60c       ?PrepareEditCtrl@CDataExchange@@QAEPAUHWND__@@H@Z 5f54b60c f   MFC42D:MFC42D.DLL
 0001:0004a612       ?GetDefaultAccelerator@CDocument@@UAEPAUHACCEL__@@XZ 5f54b612 f   MFC42D:MFC42D.DLL
 0001:0004a618       ?GetDefaultMenu@CDocument@@UAEPAUHMENU__@@XZ 5f54b618 f   MFC42D:MFC42D.DLL
 0001:0004a61e       ?UpdateFrameCounts@CDocument@@UAEXXZ 5f54b61e f   MFC42D:MFC42D.DLL
 0001:0004a624       ?DoFileSave@CDocument@@UAEHXZ 5f54b624 f   MFC42D:MFC42D.DLL
 0001:0004a62a       ?DoSave@CDocument@@UAEHPBDH@Z 5f54b62a f   MFC42D:MFC42D.DLL
 0001:0004a630       ?CanCloseFrame@CDocument@@UAEHPAVCFrameWnd@@@Z 5f54b630 f   MFC42D:MFC42D.DLL
 0001:0004a636       ?ReleaseFile@CDocument@@UAEXPAVCFile@@H@Z 5f54b636 f   MFC42D:MFC42D.DLL
 0001:0004a63c       ?GetFile@CDocument@@UAEPAVCFile@@PBDIPAVCFileException@@@Z 5f54b63c f   MFC42D:MFC42D.DLL
 0001:0004a642       ?ReportSaveLoadException@CDocument@@UAEXPBDPAVCException@@HI@Z 5f54b642 f   MFC42D:MFC42D.DLL
 0001:0004a648       ?OnChangedViewList@CDocument@@UAEXXZ 5f54b648 f   MFC42D:MFC42D.DLL
 0001:0004a64e       ?GetNextView@CDocument@@UBEPAVCView@@AAPAU__POSITION@@@Z 5f54b64e f   MFC42D:MFC42D.DLL
 0001:0004a654       ?GetFirstViewPosition@CDocument@@UBEPAU__POSITION@@XZ 5f54b654 f   MFC42D:MFC42D.DLL
 0001:0004a65a       ?SetModifiedFlag@CDocument@@UAEXH@Z 5f54b65a f   MFC42D:MFC42D.DLL
 0001:0004a660       ?IsModified@CDocument@@UAEHXZ 5f54b660 f   MFC42D:MFC42D.DLL
 0001:0004a666       ?SetTitle@CDocument@@UAEXPBD@Z 5f54b666 f   MFC42D:MFC42D.DLL
 0001:0004a66c       ?GetMessageMap@CDocument@@MBEPBUAFX_MSGMAP@@XZ 5f54b66c f   MFC42D:MFC42D.DLL
 0001:0004a672       ?OnFinalRelease@CDocument@@UAEXXZ 5f54b672 f   MFC42D:MFC42D.DLL
 0001:0004a678       ??1CObList@@UAE@XZ         5f54b678 f   MFC42D:MFC42D.DLL
 0001:0004a67e       ??1CDocument@@UAE@XZ       5f54b67e f   MFC42D:MFC42D.DLL
 0001:0004a684       ?IsEmpty@CObList@@QBEHXZ   5f54b684 f   MFC42D:MFC42D.DLL
 0001:0004a68a       ?IsEmpty@CPtrList@@QBEHXZ  5f54b68a f   MFC42D:MFC42D.DLL
 0001:0004a690       ??0CObList@@QAE@H@Z        5f54b690 f   MFC42D:MFC42D.DLL
 0001:0004a696       ??0CDocument@@QAE@XZ       5f54b696 f   MFC42D:MFC42D.DLL
 0001:0004a69c       ?GetCount@CObList@@QBEHXZ  5f54b69c f   MFC42D:MFC42D.DLL
 0001:0004a6a2       ?AddTail@CObList@@QAEPAU__POSITION@@PAVCObject@@@Z 5f54b6a2 f   MFC42D:MFC42D.DLL
 0001:0004a6a8       ?RemoveAt@CObList@@QAEXPAU__POSITION@@@Z 5f54b6a8 f   MFC42D:MFC42D.DLL
 0001:0004a6ae       ?Find@CObList@@QBEPAU__POSITION@@PAVCObject@@PAU2@@Z 5f54b6ae f   MFC42D:MFC42D.DLL
 0001:0004a6b4       ?GetHeadPosition@CObList@@QBEPAU__POSITION@@XZ 5f54b6b4 f   MFC42D:MFC42D.DLL
 0001:0004a6ba       ?GetNext@CObList@@QBEPAVCObject@@AAPAU__POSITION@@@Z 5f54b6ba f   MFC42D:MFC42D.DLL
 0001:0004a6c0       ?SetPathName@CDocument@@UAEXPBDH@Z 5f54b6c0 f   MFC42D:MFC42D.DLL
 0001:0004a6c6       ??6@YGAAVCArchive@@AAV0@PBVCObject@@@Z 5f54b6c6 f   MFC42D:MFC42D.DLL
 0001:0004a6cc       ?SaveModified@CDocument@@UAEHXZ 5f54b6cc f   MFC42D:MFC42D.DLL
 0001:0004a6d2       ?AfxMessageBox@@YGHPBDII@Z 5f54b6d2 f   MFC42D:MFC42D.DLL
 0001:0004a6d8       ?AfxFormatString1@@YGXAAVCString@@IPBD@Z 5f54b6d8 f   MFC42D:MFC42D.DLL
 0001:0004a6de       ?OnNewDocument@CDocument@@UAEHXZ 5f54b6de f   MFC42D:MFC42D.DLL
 0001:0004a6e4       ?OnOpenDocument@CDocument@@UAEHPBD@Z 5f54b6e4 f   MFC42D:MFC42D.DLL
 0001:0004a6ea       ?AfxComparePath@@YGHPBD0@Z 5f54b6ea f   MFC42D:MFC42D.DLL
 0001:0004a6f0       ?OnSaveDocument@CDocument@@UAEHPBD@Z 5f54b6f0 f   MFC42D:MFC42D.DLL
 0001:0004a6f6       ?OnCloseDocument@CDocument@@UAEXXZ 5f54b6f6 f   MFC42D:MFC42D.DLL
 0001:0004a6fc       ??1CFileException@@UAE@XZ  5f54b6fc f   MFC42D:MFC42D.DLL
 0001:0004a702       ??1CArchive@@QAE@XZ        5f54b702 f   MFC42D:MFC42D.DLL
 0001:0004a708       ?Close@CArchive@@QAEXXZ    5f54b708 f   MFC42D:MFC42D.DLL
 0001:0004a70e       ??0CArchive@@QAE@PAVCFile@@IHPAX@Z 5f54b70e f   MFC42D:MFC42D.DLL
 0001:0004a714       ?AfxThrowFileException@@YGXHJPBD@Z 5f54b714 f   MFC42D:MFC42D.DLL
 0001:0004a71a       ??0CFileException@@QAE@HJPBD@Z 5f54b71a f   MFC42D:MFC42D.DLL
 0001:0004a720       ?AssertValid@CDocument@@UBEXXZ 5f54b720 f   MFC42D:MFC42D.DLL
 0001:0004a726       ?Dump@CDocument@@UBEXAAVCDumpContext@@@Z 5f54b726 f   MFC42D:MFC42D.DLL
 0001:0004a72c       ?AfxClassInit@@YGXPAUCRuntimeClass@@@Z 5f54b72c f   MFC42D:MFC42D.DLL
 0001:0004a732       ?ReadObject@CArchive@@QAEPAVCObject@@PBUCRuntimeClass@@@Z 5f54b732 f   MFC42D:MFC42D.DLL
 0001:0004a738       ?AfxUnlockGlobals@@YGXH@Z  5f54b738 f   MFC42D:MFC42D.DLL
 0001:0004a73e       ?AfxLockGlobals@@YGXH@Z    5f54b73e f   MFC42D:MFC42D.DLL
 0001:0004a744       ?PtInRect@CRect@@QBEHUtagPOINT@@@Z 5f54b744 f   MFC42D:MFC42D.DLL
 0001:0004a74a       ?GetCapture@CWnd@@SGPAV1@XZ 5f54b74a f   MFC42D:MFC42D.DLL
 0001:0004a750       ?SetCapture@CWnd@@QAEPAV1@XZ 5f54b750 f   MFC42D:MFC42D.DLL
 0001:0004a756       ?InflateRect@CRect@@QAEXHH@Z 5f54b756 f   MFC42D:MFC42D.DLL
 0001:0004a75c       ?IsRectNull@CRect@@QBEHXZ  5f54b75c f   MFC42D:MFC42D.DLL
 0001:0004a762       ??0CPoint@@QAE@XZ          5f54b762 f   MFC42D:MFC42D.DLL
 0001:0004a768       ?ScreenToClient@CWnd@@QBEXPAUtagPOINT@@@Z 5f54b768 f   MFC42D:MFC42D.DLL
 0001:0004a76e       ??0CPoint@@QAE@HH@Z        5f54b76e f   MFC42D:MFC42D.DLL
 0001:0004a774       ?IsDerivedFrom@CRuntimeClass@@QBEHPBU1@@Z 5f54b774 f   MFC42D:MFC42D.DLL
 0001:0004a77a       ?CreateObject@CRuntimeClass@@QAEPAVCObject@@XZ 5f54b77a f   MFC42D:MFC42D.DLL
 0001:0004a780       ?AddHead@CSimpleList@@QAEXPAX@Z 5f54b780 f   MFC42D:MFC42D.DLL
 0001:0004a786       ?Remove@CSimpleList@@QAEHPAX@Z 5f54b786 f   MFC42D:MFC42D.DLL
 0001:0004a78c       ?ExitHelpMode@CFrameWnd@@UAEXXZ 5f54b78c f   MFC42D:MFC42D.DLL
 0001:0004a792       ?DelayUpdateFrameMenu@CFrameWnd@@UAEXPAUHMENU__@@@Z 5f54b792 f   MFC42D:MFC42D.DLL
 0001:0004a798       ?GetDefaultAccelerator@CFrameWnd@@UAEPAUHACCEL__@@XZ 5f54b798 f   MFC42D:MFC42D.DLL
 0001:0004a79e       ?OnUpdateFrameMenu@CFrameWnd@@UAEXPAUHMENU__@@@Z 5f54b79e f   MFC42D:MFC42D.DLL
 0001:0004a7a4       ?OnUpdateFrameTitle@CFrameWnd@@UAEXH@Z 5f54b7a4 f   MFC42D:MFC42D.DLL
 0001:0004a7aa       ?OnCreateClient@CFrameWnd@@MAEHPAUtagCREATESTRUCTA@@PAUCCreateContext@@@Z 5f54b7aa f   MFC42D:MFC42D.DLL
 0001:0004a7b0       ?NegotiateBorderSpace@CFrameWnd@@UAEHIPAUtagRECT@@@Z 5f54b7b0 f   MFC42D:MFC42D.DLL
 0001:0004a7b6       ?GetMessageBar@CFrameWnd@@UAEPAVCWnd@@XZ 5f54b7b6 f   MFC42D:MFC42D.DLL
 0001:0004a7bc       ?OnSetPreviewMode@CFrameWnd@@UAEXHPAUCPrintPreviewState@@@Z 5f54b7bc f   MFC42D:MFC42D.DLL
 0001:0004a7c2       ?ActivateFrame@CFrameWnd@@UAEXH@Z 5f54b7c2 f   MFC42D:MFC42D.DLL
 0001:0004a7c8       ?GetMessageString@CFrameWnd@@UBEXIAAVCString@@@Z 5f54b7c8 f   MFC42D:MFC42D.DLL
 0001:0004a7ce       ?GetActiveFrame@CFrameWnd@@UAEPAV1@XZ 5f54b7ce f   MFC42D:MFC42D.DLL
 0001:0004a7d4       ?GetActiveDocument@CFrameWnd@@UAEPAVCDocument@@XZ 5f54b7d4 f   MFC42D:MFC42D.DLL
 0001:0004a7da       ?LoadFrame@CFrameWnd@@UAEHIKPAVCWnd@@PAUCCreateContext@@@Z 5f54b7da f   MFC42D:MFC42D.DLL
 0001:0004a7e0       ?SetOccDialogInfo@CWnd@@MAEHPAU_AFX_OCC_DIALOG_INFO@@@Z 5f54b7e0 f   MFC42D:MFC42D.DLL
 0001:0004a7e6       ?IsFrameWnd@CFrameWnd@@UBEHXZ 5f54b7e6 f   MFC42D:MFC42D.DLL
 0001:0004a7ec       ?CheckAutoCenter@CWnd@@UAEHXZ 5f54b7ec f   MFC42D:MFC42D.DLL
 0001:0004a7f2       ?PreTranslateMessage@CFrameWnd@@UAEHPAUtagMSG@@@Z 5f54b7f2 f   MFC42D:MFC42D.DLL
 0001:0004a7f8       ?EndModalState@CFrameWnd@@UAEXXZ 5f54b7f8 f   MFC42D:MFC42D.DLL
 0001:0004a7fe       ?BeginModalState@CFrameWnd@@UAEXXZ 5f54b7fe f   MFC42D:MFC42D.DLL
 0001:0004a804       ?OnCommand@CFrameWnd@@MAEHIJ@Z 5f54b804 f   MFC42D:MFC42D.DLL
 0001:0004a80a       ?PreCreateWindow@CFrameWnd@@MAEHAAUtagCREATESTRUCTA@@@Z 5f54b80a f   MFC42D:MFC42D.DLL
 0001:0004a810       ?GetMessageMap@CFrameWnd@@MBEPBUAFX_MSGMAP@@XZ 5f54b810 f   MFC42D:MFC42D.DLL
 0001:0004a816       ?Dump@CFrameWnd@@UBEXAAVCDumpContext@@@Z 5f54b816 f   MFC42D:MFC42D.DLL
 0001:0004a81c       ?GetRuntimeClass@CFrameWnd@@UBEPAUCRuntimeClass@@XZ 5f54b81c f   MFC42D:MFC42D.DLL
 0001:0004a822       ??1CFrameWnd@@UAE@XZ       5f54b822 f   MFC42D:MFC42D.DLL
 0001:0004a828       ?RemoveFrameWnd@CFrameWnd@@IAEXXZ 5f54b828 f   MFC42D:MFC42D.DLL
 0001:0004a82e       ??0CFrameWnd@@QAE@XZ       5f54b82e f   MFC42D:MFC42D.DLL
 0001:0004a834       ?AddFrameWnd@CFrameWnd@@IAEXXZ 5f54b834 f   MFC42D:MFC42D.DLL
 0001:0004a83a       ?AfxCallWndProc@@YGJPAVCWnd@@PAUHWND__@@IIJ@Z 5f54b83a f   MFC42D:MFC42D.DLL
 0001:0004a840       ?PostNcDestroy@CFrameWnd@@MAEXXZ 5f54b840 f   MFC42D:MFC42D.DLL
 0001:0004a846       ?OnCmdMsg@CFrameWnd@@UAEHIHPAXPAUAFX_CMDHANDLERINFO@@@Z 5f54b846 f   MFC42D:MFC42D.DLL
 0001:0004a84c       ?ModifyStyleEx@CWnd@@QAEHKKI@Z 5f54b84c f   MFC42D:MFC42D.DLL
 0001:0004a852       ?OnCreate@CFrameWnd@@IAEHPAUtagCREATESTRUCTA@@@Z 5f54b852 f   MFC42D:MFC42D.DLL
 0001:0004a858       ?OnDestroy@CFrameWnd@@IAEXXZ 5f54b858 f   MFC42D:MFC42D.DLL
 0001:0004a85e       ?DestroyDockBars@CFrameWnd@@QAEXXZ 5f54b85e f   MFC42D:MFC42D.DLL
 0001:0004a864       ?DisconnectViews@CDocument@@QAEXXZ 5f54b864 f   MFC42D:MFC42D.DLL
 0001:0004a86a       ?OnWindowPosChanging@CWnd@@IAEXPAUtagWINDOWPOS@@@Z 5f54b86a f   MFC42D:MFC42D.DLL
 0001:0004a870       ?LoadAccelTable@CFrameWnd@@QAEHPBD@Z 5f54b870 f   MFC42D:MFC42D.DLL
 0001:0004a876       ??0CRect@@QAE@HHHH@Z       5f54b876 f   MFC42D:MFC42D.DLL
 0001:0004a87c       ?GetDlgItem@CWnd@@QBEPAV1@H@Z 5f54b87c f   MFC42D:MFC42D.DLL
 0001:0004a882       ?ScreenToClient@CWnd@@QBEXPAUtagRECT@@@Z 5f54b882 f   MFC42D:MFC42D.DLL
 0001:0004a888       ?ClientToScreen@CWnd@@QBEXPAUtagRECT@@@Z 5f54b888 f   MFC42D:MFC42D.DLL
 0001:0004a88e       ?AfxRepositionWindow@@YGXPAUAFX_SIZEPARENTPARAMS@@PAUHWND__@@PBUtagRECT@@@Z 5f54b88e f   MFC42D:MFC42D.DLL
 0001:0004a894       ?RepositionBars@CWnd@@QAEXIIIIPAUtagRECT@@PBU2@H@Z 5f54b894 f   MFC42D:MFC42D.DLL
 0001:0004a89a       ?ContinueRouting@CCmdUI@@QAEXXZ 5f54b89a f   MFC42D:MFC42D.DLL
 0001:0004a8a0       ?OnUpdateControlBarMenu@CFrameWnd@@QAEXPAVCCmdUI@@@Z 5f54b8a0 f   MFC42D:MFC42D.DLL
 0001:0004a8a6       ?GetControlBar@CFrameWnd@@QAEPAVCControlBar@@I@Z 5f54b8a6 f   MFC42D:MFC42D.DLL
 0001:0004a8ac       ?OnBarCheck@CFrameWnd@@QAEHI@Z 5f54b8ac f   MFC42D:MFC42D.DLL
 0001:0004a8b2       ?OnContextHelp@CFrameWnd@@QAEXXZ 5f54b8b2 f   MFC42D:MFC42D.DLL
 0001:0004a8b8       ?AssertValid@CFrameWnd@@UBEXXZ 5f54b8b8 f   MFC42D:MFC42D.DLL
 0001:0004a8be       ??6@YGAAVCDumpContext@@AAV0@ABUtagRECT@@@Z 5f54b8be f   MFC42D:MFC42D.DLL
 0001:0004a8c4       ??9@YG_NABVCString@@PBD@Z  5f54b8c4 f   MFC42D:MFC42D.DLL
 0001:0004a8ca       ?SendInitialUpdate@CDocument@@QAEXXZ 5f54b8ca f   MFC42D:MFC42D.DLL
 0001:0004a8d0       ?AfxOleGetUserCtrl@@YGHXZ  5f54b8d0 f   MFC42D:MFC42D.DLL
 0001:0004a8d6       ??6CDumpContext@@QAEAAV0@PBVCObject@@@Z 5f54b8d6 f   MFC42D:MFC42D.DLL
 0001:0004a8dc       ??YCString@@QAEABV0@D@Z    5f54b8dc f   MFC42D:MFC42D.DLL
 0001:0004a8e2       ?GetBufferPtr@CFile@@UAEIIIPAPAX0@Z 5f54b8e2 f   MFC42D:MFC42D.DLL
 0001:0004a8e8       ?Open@CFile@@UAEHPBDIPAVCFileException@@@Z 5f54b8e8 f   MFC42D:MFC42D.DLL
 0001:0004a8ee       ?SetFilePath@CFile@@UAEXPBD@Z 5f54b8ee f   MFC42D:MFC42D.DLL
 0001:0004a8f4       ?GetFilePath@CFile@@UBE?AVCString@@XZ 5f54b8f4 f   MFC42D:MFC42D.DLL
 0001:0004a8fa       ?GetFileTitle@CFile@@UBE?AVCString@@XZ 5f54b8fa f   MFC42D:MFC42D.DLL
 0001:0004a900       ?GetFileName@CFile@@UBE?AVCString@@XZ 5f54b900 f   MFC42D:MFC42D.DLL
 0001:0004a906       ??1CFile@@UAE@XZ           5f54b906 f   MFC42D:MFC42D.DLL
 0001:0004a90c       ?AfxFullPath@@YGHPADPBD@Z  5f54b90c f   MFC42D:MFC42D.DLL
 0001:0004a912       ?OsErrorToException@CFileException@@SGHJ@Z 5f54b912 f   MFC42D:MFC42D.DLL
 0001:0004a918       ??4CTime@@QAEABV0@ABV0@@Z  5f54b918 f   MFC42D:MFC42D.DLL
 0001:0004a91e       ??0CTime@@QAE@ABU_FILETIME@@H@Z 5f54b91e f   MFC42D:MFC42D.DLL
 0001:0004a924       ?AssertValid@CFile@@UBEXXZ 5f54b924 f   MFC42D:MFC42D.DLL
 0001:0004a92a       ?Dump@CFile@@UBEXAAVCDumpContext@@@Z 5f54b92a f   MFC42D:MFC42D.DLL
 0001:0004a930       ??9CSize@@QBEHUtagSIZE@@@Z 5f54b930 f   MFC42D:MFC42D.DLL
 0001:0004a936       ?HIMETRICtoDP@CDC@@QBEXPAUtagSIZE@@@Z 5f54b936 f   MFC42D:MFC42D.DLL
 0001:0004a93c       ?Size@CRect@@QBE?AVCSize@@XZ 5f54b93c f   MFC42D:MFC42D.DLL
 0001:0004a942       ??0CSize@@QAE@XZ           5f54b942 f   MFC42D:MFC42D.DLL
 0001:0004a948       ?IsWindowVisible@CWnd@@QBEHXZ 5f54b948 f   MFC42D:MFC42D.DLL
 0001:0004a94e       ?AfxFormatString2@@YGXAAVCString@@IPBD1@Z 5f54b94e f   MFC42D:MFC42D.DLL
 0001:0004a954       ?HideApplication@CWinApp@@QAEXXZ 5f54b954 f   MFC42D:MFC42D.DLL
 0001:0004a95a       ?SetActiveWindow@CWnd@@QAEPAV1@XZ 5f54b95a f   MFC42D:MFC42D.DLL
 0001:0004a960       ?ShowWindow@CWnd@@QAEHH@Z  5f54b960 f   MFC42D:MFC42D.DLL
 0001:0004a966       ?SetForegroundWindow@CWnd@@QAEHXZ 5f54b966 f   MFC42D:MFC42D.DLL
 0001:0004a96c       ?GetLastActivePopup@CWnd@@QBEPAV1@XZ 5f54b96c f   MFC42D:MFC42D.DLL
 0001:0004a972       ?UpdateWindow@CWnd@@QAEXXZ 5f54b972 f   MFC42D:MFC42D.DLL
 0001:0004a978       ?ShowOwnedWindows@CFrameWnd@@QAEXH@Z 5f54b978 f   MFC42D:MFC42D.DLL
 0001:0004a97e       ?Attach@CWnd@@QAEHPAUHWND__@@@Z 5f54b97e f   MFC42D:MFC42D.DLL
 0001:0004a984       ?CreateOleFrame@CDocTemplate@@QAEPAVCFrameWnd@@PAVCWnd@@PAVCDocument@@H@Z 5f54b984 f   MFC42D:MFC42D.DLL
 0001:0004a98a       ?GetExStyle@CWnd@@QBEKXZ   5f54b98a f   MFC42D:MFC42D.DLL
 0001:0004a990       ?GetDescendantWindow@CWnd@@QBEPAV1@HH@Z 5f54b990 f   MFC42D:MFC42D.DLL
 0001:0004a996       ?SetActiveView@CFrameWnd@@QAEXPAVCView@@H@Z 5f54b996 f   MFC42D:MFC42D.DLL
 0001:0004a99c       ?SetParent@CWnd@@QAEPAV1@PAV1@@Z 5f54b99c f   MFC42D:MFC42D.DLL
 0001:0004a9a2       ?GetActiveView@CFrameWnd@@QBEPAVCView@@XZ 5f54b9a2 f   MFC42D:MFC42D.DLL
 0001:0004a9a8       ?IsFloating@CControlBar@@QBEHXZ 5f54b9a8 f   MFC42D:MFC42D.DLL
 0001:0004a9ae       ?EnableWindow@CWnd@@QAEHH@Z 5f54b9ae f   MFC42D:MFC42D.DLL
 0001:0004a9b4       ?InModalState@CFrameWnd@@QBEHXZ 5f54b9b4 f   MFC42D:MFC42D.DLL
 0001:0004a9ba       ?Close@CMetaFileDC@@QAEPAUHMETAFILE__@@XZ 5f54b9ba f   MFC42D:MFC42D.DLL
 0001:0004a9c0       ?SetAttribDC@CMetaFileDC@@UAEXPAUHDC__@@@Z 5f54b9c0 f   MFC42D:MFC42D.DLL
 0001:0004a9c6       ??1CMetaFileDC@@UAE@XZ     5f54b9c6 f   MFC42D:MFC42D.DLL
 0001:0004a9cc       ?Create@CMetaFileDC@@QAEHPBD@Z 5f54b9cc f   MFC42D:MFC42D.DLL
 0001:0004a9d2       ??0CMetaFileDC@@QAE@XZ     5f54b9d2 f   MFC42D:MFC42D.DLL
 0001:0004a9d8       ?Left@CString@@QBE?AV1@H@Z 5f54b9d8 f   MFC42D:MFC42D.DLL
 0001:0004a9de       ?Mid@CString@@QBE?AV1@H@Z  5f54b9de f   MFC42D:MFC42D.DLL
 0001:0004a9e4       ?Find@CString@@QBEHD@Z     5f54b9e4 f   MFC42D:MFC42D.DLL
 0001:0004a9ea       ?AfxGetModuleShortFileName@@YGXPAUHINSTANCE__@@AAVCString@@@Z 5f54b9ea f   MFC42D:MFC42D.DLL
 0001:0004a9f0       ?AfxGetInstanceHandle@@YGPAUHINSTANCE__@@XZ 5f54b9f0 f   MFC42D:MFC42D.DLL
 0001:0004a9f6       ?_AfxDeleteRegKey@@YGHPBD@Z 5f54b9f6 f   MFC42D:MFC42D.DLL
 0001:0004a9fc       ?AfxFormatStrings@@YGXAAVCString@@PBDPBQBDH@Z 5f54b9fc f   MFC42D:MFC42D.DLL
 0001:0004aa02       ?GetNextDocTemplate@CWinApp@@QBEPAVCDocTemplate@@AAPAU__POSITION@@@Z 5f54ba02 f   MFC42D:MFC42D.DLL
 0001:0004aa08       ?GetFirstDocTemplatePosition@CWinApp@@QBEPAU__POSITION@@XZ 5f54ba08 f   MFC42D:MFC42D.DLL
 0001:0004aa0e       ?OnCmdMsg@CDocument@@UAEHIHPAXPAUAFX_CMDHANDLERINFO@@@Z 5f54ba0e f   MFC42D:MFC42D.DLL
 0001:0004aa14       ?GetRoutingView_@CCmdTarget@@KGPAVCView@@XZ 5f54ba14 f   MFC42D:MFC42D.DLL
 0001:0004aa1a       ?InsertMenuA@CMenu@@QAEHIIIPBD@Z 5f54ba1a f   MFC42D:MFC42D.DLL
 0001:0004aa20       ?DeleteMenu@CMenu@@QAEHII@Z 5f54ba20 f   MFC42D:MFC42D.DLL
 0001:0004aa26       ?GetMenuStringA@CMenu@@QBEHIPADHI@Z 5f54ba26 f   MFC42D:MFC42D.DLL
 0001:0004aa2c       ?AfxFindMessageEntry@@YGPBUAFX_MSGMAP_ENTRY@@PBU1@III@Z 5f54ba2c f   MFC42D:MFC42D.DLL
 0001:0004aa32       ?OnSize@CWnd@@IAEXIHH@Z    5f54ba32 f   MFC42D:MFC42D.DLL
 0001:0004aa38       ?OnEndPrintPreview@CView@@MAEXPAVCDC@@PAUCPrintInfo@@UtagPOINT@@PAVCPreviewView@@@Z 5f54ba38 f   MFC42D:MFC42D.DLL
 0001:0004aa3e       ?OnPreparePrinting@CView@@MAEHPAUCPrintInfo@@@Z 5f54ba3e f   MFC42D:MFC42D.DLL
 0001:0004aa44       ?OnDraw@CCtrlView@@MAEXPAVCDC@@@Z 5f54ba44 f   MFC42D:MFC42D.DLL
 0001:0004aa4a       ?OnUpdate@CView@@MAEXPAV1@JPAVCObject@@@Z 5f54ba4a f   MFC42D:MFC42D.DLL
 0001:0004aa50       ?OnActivateFrame@CView@@MAEXIPAVCFrameWnd@@@Z 5f54ba50 f   MFC42D:MFC42D.DLL
 0001:0004aa56       ?OnActivateView@CView@@MAEXHPAV1@0@Z 5f54ba56 f   MFC42D:MFC42D.DLL
 0001:0004aa5c       ?OnDragScroll@CView@@UAEKKVCPoint@@@Z 5f54ba5c f   MFC42D:MFC42D.DLL
 0001:0004aa62       ?OnDropEx@CView@@UAEKPAVCOleDataObject@@KKVCPoint@@@Z 5f54ba62 f   MFC42D:MFC42D.DLL
 0001:0004aa68       ?OnDrop@CView@@UAEHPAVCOleDataObject@@KVCPoint@@@Z 5f54ba68 f   MFC42D:MFC42D.DLL
 0001:0004aa6e       ?OnDragLeave@CView@@UAEXXZ 5f54ba6e f   MFC42D:MFC42D.DLL
 0001:0004aa74       ?OnDragOver@CView@@UAEKPAVCOleDataObject@@KVCPoint@@@Z 5f54ba74 f   MFC42D:MFC42D.DLL
 0001:0004aa7a       ?OnDragEnter@CView@@UAEKPAVCOleDataObject@@KVCPoint@@@Z 5f54ba7a f   MFC42D:MFC42D.DLL
 0001:0004aa80       ?OnScrollBy@CView@@UAEHVCSize@@H@Z 5f54ba80 f   MFC42D:MFC42D.DLL
 0001:0004aa86       ?OnScroll@CView@@UAEHIIH@Z 5f54ba86 f   MFC42D:MFC42D.DLL
 0001:0004aa8c       ?PostNcDestroy@CView@@MAEXXZ 5f54ba8c f   MFC42D:MFC42D.DLL
 0001:0004aa92       ?PreTranslateMessage@CWnd@@UAEHPAUtagMSG@@@Z 5f54ba92 f   MFC42D:MFC42D.DLL
 0001:0004aa98       ?GetScrollBarCtrl@CView@@UBEPAVCScrollBar@@H@Z 5f54ba98 f   MFC42D:MFC42D.DLL
 0001:0004aa9e       ?CalcWindowRect@CView@@UAEXPAUtagRECT@@I@Z 5f54ba9e f   MFC42D:MFC42D.DLL
 0001:0004aaa4       ?OnCmdMsg@CView@@UAEHIHPAXPAUAFX_CMDHANDLERINFO@@@Z 5f54baa4 f   MFC42D:MFC42D.DLL
 0001:0004aaaa       ??0CDWordArray@@QAE@XZ     5f54baaa f   MFC42D:MFC42D.DLL
 0001:0004aab0       ??0CDC@@QAE@XZ             5f54bab0 f   MFC42D:MFC42D.DLL
 0001:0004aab6       ??0CCtrlView@@QAE@PBDK@Z   5f54bab6 f   MFC42D:MFC42D.DLL
 0001:0004aabc       ?PreCreateWindow@CCtrlView@@MAEHAAUtagCREATESTRUCTA@@@Z 5f54babc f   MFC42D:MFC42D.DLL
 0001:0004aac2       ?AfxInitRichEdit@@YGHXZ    5f54bac2 f   MFC42D:MFC42D.DLL
 0001:0004aac8       ?SetOptions@CRichEditCtrl@@QAEXGK@Z 5f54bac8 f   MFC42D:MFC42D.DLL
 0001:0004aace       ?DragAcceptFiles@CWnd@@QAEXH@Z 5f54bace f   MFC42D:MFC42D.DLL
 0001:0004aad4       ?GetIRichEditOle@CRichEditCtrl@@QBEPAUIRichEditOle@@XZ 5f54bad4 f   MFC42D:MFC42D.DLL
 0001:0004aada       ?SetOLECallback@CRichEditCtrl@@QAEHPAUIRichEditOleCallback@@@Z 5f54bada f   MFC42D:MFC42D.DLL
 0001:0004aae0       ?SetEventMask@CRichEditCtrl@@QAEKK@Z 5f54bae0 f   MFC42D:MFC42D.DLL
 0001:0004aae6       ?LimitText@CRichEditCtrl@@QAEXJ@Z 5f54bae6 f   MFC42D:MFC42D.DLL
 0001:0004aaec       ?OnCreate@CView@@IAEHPAUtagCREATESTRUCTA@@@Z 5f54baec f   MFC42D:MFC42D.DLL
 0001:0004aaf2       ?OnInitialUpdate@CView@@UAEXXZ 5f54baf2 f   MFC42D:MFC42D.DLL
 0001:0004aaf8       ?EmptyUndoBuffer@CRichEditCtrl@@QAEXXZ 5f54baf8 f   MFC42D:MFC42D.DLL
 0001:0004aafe       ?SetWindowTextA@CWnd@@QAEXPBD@Z 5f54bafe f   MFC42D:MFC42D.DLL
 0001:0004ab04       ?SetTargetDevice@CRichEditCtrl@@QAEHAAVCDC@@J@Z 5f54bb04 f   MFC42D:MFC42D.DLL
 0001:0004ab0a       ?CreateDCA@CDC@@QAEHPBD00PBX@Z 5f54bb0a f   MFC42D:MFC42D.DLL
 0001:0004ab10       ?CreatePrinterDC@CWinApp@@QAEHAAVCDC@@@Z 5f54bb10 f   MFC42D:MFC42D.DLL
 0001:0004ab16       ?SetTargetDevice@CRichEditCtrl@@QAEHPAUHDC__@@J@Z 5f54bb16 f   MFC42D:MFC42D.DLL
 0001:0004ab1c       ?Invalidate@CWnd@@QAEXH@Z  5f54bb1c f   MFC42D:MFC42D.DLL
 0001:0004ab22       ?StreamIn@CRichEditCtrl@@QAEJHAAU_editstream@@@Z 5f54bb22 f   MFC42D:MFC42D.DLL
 0001:0004ab28       ?StreamOut@CRichEditCtrl@@QAEJHAAU_editstream@@@Z 5f54bb28 f   MFC42D:MFC42D.DLL
 0001:0004ab2e       ?ReadHuge@CFile@@QAEKPAXK@Z 5f54bb2e f   MFC42D:MFC42D.DLL
 0001:0004ab34       ?WriteHuge@CFile@@QAEXPBXK@Z 5f54bb34 f   MFC42D:MFC42D.DLL
 0001:0004ab3a       ?GetFile@CArchive@@QBEPAVCFile@@XZ 5f54bb3a f   MFC42D:MFC42D.DLL
 0001:0004ab40       ?Flush@CArchive@@QAEXXZ    5f54bb40 f   MFC42D:MFC42D.DLL
 0001:0004ab46       ?FormatRange@CRichEditCtrl@@QAEJPAU_formatrange@@H@Z 5f54bb46 f   MFC42D:MFC42D.DLL
 0001:0004ab4c       ?Add@CDWordArray@@QAEHK@Z  5f54bb4c f   MFC42D:MFC42D.DLL
 0001:0004ab52       ?GetSize@CDWordArray@@QBEHXZ 5f54bb52 f   MFC42D:MFC42D.DLL
 0001:0004ab58       ?DPtoLP@CDC@@QBEXPAUtagRECT@@@Z 5f54bb58 f   MFC42D:MFC42D.DLL
 0001:0004ab5e       ?GetDeviceCaps@CDC@@QBEHH@Z 5f54bb5e f   MFC42D:MFC42D.DLL
 0001:0004ab64       ?IntersectClipRect@CDC@@QAEHHHHH@Z 5f54bb64 f   MFC42D:MFC42D.DLL
 0001:0004ab6a       ?SetMaxPage@CPrintInfo@@QAEXI@Z 5f54bb6a f   MFC42D:MFC42D.DLL
 0001:0004ab70       ??ACDWordArray@@QAEAAKH@Z  5f54bb70 f   MFC42D:MFC42D.DLL
 0001:0004ab76       ?RemoveAll@CDWordArray@@QAEXXZ 5f54bb76 f   MFC42D:MFC42D.DLL
 0001:0004ab7c       ?GetSel@CRichEditCtrl@@QBEXAAJ0@Z 5f54bb7c f   MFC42D:MFC42D.DLL
 0001:0004ab82       ?CanUndo@CRichEditCtrl@@QBEHXZ 5f54bb82 f   MFC42D:MFC42D.DLL
 0001:0004ab88       ?Cut@CRichEditCtrl@@QAEXXZ 5f54bb88 f   MFC42D:MFC42D.DLL
 0001:0004ab8e       ?Copy@CRichEditCtrl@@QAEXXZ 5f54bb8e f   MFC42D:MFC42D.DLL
 0001:0004ab94       ?Paste@CRichEditCtrl@@QAEXXZ 5f54bb94 f   MFC42D:MFC42D.DLL
 0001:0004ab9a       ?Clear@CRichEditCtrl@@QAEXXZ 5f54bb9a f   MFC42D:MFC42D.DLL
 0001:0004aba0       ?Undo@CRichEditCtrl@@QAEHXZ 5f54bba0 f   MFC42D:MFC42D.DLL
 0001:0004aba6       ?SetSel@CRichEditCtrl@@QAEXJJ@Z 5f54bba6 f   MFC42D:MFC42D.DLL
 0001:0004abac       ?OnDestroy@CView@@IAEXXZ   5f54bbac f   MFC42D:MFC42D.DLL
 0001:0004abb2       ?GetCharFormat@CFontDialog@@QBEXAAU_charformat@@@Z 5f54bbb2 f   MFC42D:MFC42D.DLL
 0001:0004abb8       ?DoModal@CFontDialog@@UAEHXZ 5f54bbb8 f   MFC42D:MFC42D.DLL
 0001:0004abbe       ??0CFontDialog@@QAE@ABU_charformat@@KPAVCDC@@PAVCWnd@@@Z 5f54bbbe f   MFC42D:MFC42D.DLL
 0001:0004abc4       ?PasteSpecial@CRichEditCtrl@@QAEXIKPAUHMETAFILE__@@@Z 5f54bbc4 f   MFC42D:MFC42D.DLL
 0001:0004abca       ?OnKeyDown@CWnd@@IAEXIII@Z 5f54bbca f   MFC42D:MFC42D.DLL
 0001:0004abd0       ?CenterPoint@CRect@@QBE?AVCPoint@@XZ 5f54bbd0 f   MFC42D:MFC42D.DLL
 0001:0004abd6       ?SetSel@CRichEditCtrl@@QAEXAAU_charrange@@@Z 5f54bbd6 f   MFC42D:MFC42D.DLL
 0001:0004abdc       ?GetSel@CRichEditCtrl@@QBEXAAU_charrange@@@Z 5f54bbdc f   MFC42D:MFC42D.DLL
 0001:0004abe2       ?CanPaste@CRichEditCtrl@@QBEHI@Z 5f54bbe2 f   MFC42D:MFC42D.DLL
 0001:0004abe8       ?GetSelectionCharFormat@CRichEditCtrl@@QBEKAAU_charformat@@@Z 5f54bbe8 f   MFC42D:MFC42D.DLL
 0001:0004abee       ?GetParaFormat@CRichEditCtrl@@QBEKAAU_paraformat@@@Z 5f54bbee f   MFC42D:MFC42D.DLL
 0001:0004abf4       ?SetSelectionCharFormat@CRichEditCtrl@@QAEHAAU_charformat@@@Z 5f54bbf4 f   MFC42D:MFC42D.DLL
 0001:0004abfa       ?SetParaFormat@CRichEditCtrl@@QAEHAAU_paraformat@@@Z 5f54bbfa f   MFC42D:MFC42D.DLL
 0001:0004ac00       ?MoveWindow@CWnd@@QAEXPBUtagRECT@@H@Z 5f54bc00 f   MFC42D:MFC42D.DLL
 0001:0004ac06       ?OffsetRect@CRect@@QAEXHH@Z 5f54bc06 f   MFC42D:MFC42D.DLL
 0001:0004ac0c       ?Height@CRect@@QBEHXZ      5f54bc0c f   MFC42D:MFC42D.DLL
 0001:0004ac12       ?GetWindowRect@CWnd@@QBEXPAUtagRECT@@@Z 5f54bc12 f   MFC42D:MFC42D.DLL
 0001:0004ac18       ?ClientToScreen@CWnd@@QBEXPAUtagPOINT@@@Z 5f54bc18 f   MFC42D:MFC42D.DLL
 0001:0004ac1e       ?GetCharPos@CRichEditCtrl@@QBE?AVCPoint@@J@Z 5f54bc1e f   MFC42D:MFC42D.DLL
 0001:0004ac24       ?Create@CFindReplaceDialog@@QAEHHPBD0KPAVCWnd@@@Z 5f54bc24 f   MFC42D:MFC42D.DLL
 0001:0004ac2a       ??0CFindReplaceDialog@@QAE@XZ 5f54bc2a f   MFC42D:MFC42D.DLL
 0001:0004ac30       ?FindOneOf@CString@@QBEHPBD@Z 5f54bc30 f   MFC42D:MFC42D.DLL
 0001:0004ac36       ?GetSelText@CRichEditCtrl@@QBE?AVCString@@XZ 5f54bc36 f   MFC42D:MFC42D.DLL
 0001:0004ac3c       ?ReplaceSel@CRichEditCtrl@@QAEXPBDH@Z 5f54bc3c f   MFC42D:MFC42D.DLL
 0001:0004ac42       ?HideSelection@CRichEditCtrl@@QAEXHH@Z 5f54bc42 f   MFC42D:MFC42D.DLL
 0001:0004ac48       ?ReplaceAll@CFindReplaceDialog@@QBEHXZ 5f54bc48 f   MFC42D:MFC42D.DLL
 0001:0004ac4e       ?GetReplaceString@CFindReplaceDialog@@QBE?AVCString@@XZ 5f54bc4e f   MFC42D:MFC42D.DLL
 0001:0004ac54       ?ReplaceCurrent@CFindReplaceDialog@@QBEHXZ 5f54bc54 f   MFC42D:MFC42D.DLL
 0001:0004ac5a       ?GetFindString@CFindReplaceDialog@@QBE?AVCString@@XZ 5f54bc5a f   MFC42D:MFC42D.DLL
 0001:0004ac60       ?SearchDown@CFindReplaceDialog@@QBEHXZ 5f54bc60 f   MFC42D:MFC42D.DLL
 0001:0004ac66       ?MatchCase@CFindReplaceDialog@@QBEHXZ 5f54bc66 f   MFC42D:MFC42D.DLL
 0001:0004ac6c       ?MatchWholeWord@CFindReplaceDialog@@QBEHXZ 5f54bc6c f   MFC42D:MFC42D.DLL
 0001:0004ac72       ?FindNext@CFindReplaceDialog@@QBEHXZ 5f54bc72 f   MFC42D:MFC42D.DLL
 0001:0004ac78       ?IsTerminating@CFindReplaceDialog@@QBEHXZ 5f54bc78 f   MFC42D:MFC42D.DLL
 0001:0004ac7e       ?GetNotifier@CFindReplaceDialog@@SGPAV1@J@Z 5f54bc7e f   MFC42D:MFC42D.DLL
 0001:0004ac84       ?FindTextA@CRichEditCtrl@@QBEJKPAU_findtextexa@@@Z 5f54bc84 f   MFC42D:MFC42D.DLL
 0001:0004ac8a       ?AssertValid@CCtrlView@@UBEXXZ 5f54bc8a f   MFC42D:MFC42D.DLL
 0001:0004ac90       ?Dump@CCtrlView@@UBEXAAVCDumpContext@@@Z 5f54bc90 f   MFC42D:MFC42D.DLL
 0001:0004ac96       ?GetModify@CRichEditCtrl@@QBEHXZ 5f54bc96 f   MFC42D:MFC42D.DLL
 0001:0004ac9c       ?SetModify@CRichEditCtrl@@QAEXH@Z 5f54bc9c f   MFC42D:MFC42D.DLL
 0001:0004aca2       ??0CRect@@QAE@UtagPOINT@@UtagSIZE@@@Z 5f54bca2 f   MFC42D:MFC42D.DLL
 0001:0004aca8       ?GetTextLength@CRichEditCtrl@@QBEJXZ 5f54bca8 f   MFC42D:MFC42D.DLL
 0001:0004acae       ??0_AFX_EDIT_STATE@@QAE@XZ 5f54bcae f   MFC42D:MFC42D.DLL
 0001:0004acb4       ??1_AFX_RICHEDIT_STATE@@UAE@XZ 5f54bcb4 f   MFC42D:MFC42D.DLL
 0001:0004acba       ?AfxOleCanExitApp@@YGHXZ   5f54bcba f   MFC42D:MFC42D.DLL
 0001:0004acc0       ??3@YAXPAXPBDH@Z           5f54bcc0 f   MFC42D:MFC42D.DLL
 0001:0004acc6       ?Lookup@CMapPtrToPtr@@QBEHPAXAAPAX@Z 5f54bcc6 f   MFC42D:MFC42D.DLL
 0001:0004accc       ?SetAt@CMapPtrToPtr@@QAEXPAX0@Z 5f54bccc f   MFC42D:MFC42D.DLL
 0001:0004acd2       ?RemoveAll@CTypeLibCacheMap@@UAEXPAX@Z 5f54bcd2 f   MFC42D:MFC42D.DLL
 0001:0004acd8       ?Dump@CMapPtrToPtr@@UBEXAAVCDumpContext@@@Z 5f54bcd8 f   MFC42D:MFC42D.DLL
 0001:0004acde       ?AssertValid@CMapPtrToPtr@@UBEXXZ 5f54bcde f   MFC42D:MFC42D.DLL
 0001:0004ace4       ?GetRuntimeClass@CMapPtrToPtr@@UBEPAUCRuntimeClass@@XZ 5f54bce4 f   MFC42D:MFC42D.DLL
 0001:0004acea       ??0CMapPtrToPtr@@QAE@H@Z   5f54bcea f   MFC42D:MFC42D.DLL
 0001:0004acf0       ??1CMapPtrToPtr@@UAE@XZ    5f54bcf0 f   MFC42D:MFC42D.DLL
 0001:0004acf6       ?AfxEndDeferRegisterClass@@YGHJ@Z 5f54bcf6 f   MFC42D:MFC42D.DLL
 0001:0004acfc       ??0CTime@@QAE@ABU_SYSTEMTIME@@H@Z 5f54bcfc f   MFC42D:MFC42D.DLL
 0001:0004ad02       ?GetAsSystemTime@CTime@@QBEHAAU_SYSTEMTIME@@@Z 5f54bd02 f   MFC42D:MFC42D.DLL
 0001:0004ad08       ?GetMessageMap@CWnd@@MBEPBUAFX_MSGMAP@@XZ 5f54bd08 f   MFC42D:MFC42D.DLL
 0001:0004ad0e       ?Dump@CWnd@@UBEXAAVCDumpContext@@@Z 5f54bd0e f   MFC42D:MFC42D.DLL
 0001:0004ad14       ?AssertValid@CWnd@@UBEXXZ  5f54bd14 f   MFC42D:MFC42D.DLL
 0001:0004ad1a       ??1CWnd@@UAE@XZ            5f54bd1a f   MFC42D:MFC42D.DLL
 0001:0004ad20       ?SetWindowPos@CWnd@@QAEHPBV1@HHHHI@Z 5f54bd20 f   MFC42D:MFC42D.DLL
 0001:0004ad26       ?Width@CRect@@QBEHXZ       5f54bd26 f   MFC42D:MFC42D.DLL
 0001:0004ad2c       ?PrepareCtrl@CDataExchange@@QAEPAUHWND__@@H@Z 5f54bd2c f   MFC42D:MFC42D.DLL
 0001:0004ad32       ??MCTime@@QBEHV0@@Z        5f54bd32 f   MFC42D:MFC42D.DLL
 0001:0004ad38       ??OCTime@@QBEHV0@@Z        5f54bd38 f   MFC42D:MFC42D.DLL
 0001:0004ad3e       ??NCTime@@QBEHV0@@Z        5f54bd3e f   MFC42D:MFC42D.DLL
 0001:0004ad44       ??0CTime@@QAE@ABV0@@Z      5f54bd44 f   MFC42D:MFC42D.DLL
 0001:0004ad4a       ??0CWnd@@QAE@XZ            5f54bd4a f   MFC42D:MFC42D.DLL
 0001:0004ad50       ?FromHandle@CFont@@SGPAV1@PAUHFONT__@@@Z 5f54bd50 f   MFC42D:MFC42D.DLL
 0001:0004ad56       ?OnEndPrinting@CView@@MAEXPAVCDC@@PAUCPrintInfo@@@Z 5f54bd56 f   MFC42D:MFC42D.DLL
 0001:0004ad5c       ?OnPrint@CView@@MAEXPAVCDC@@PAUCPrintInfo@@@Z 5f54bd5c f   MFC42D:MFC42D.DLL
 0001:0004ad62       ?OnBeginPrinting@CView@@MAEXPAVCDC@@PAUCPrintInfo@@@Z 5f54bd62 f   MFC42D:MFC42D.DLL
 0001:0004ad68       ?OnActivateFrame@CFormView@@MAEXIPAVCFrameWnd@@@Z 5f54bd68 f   MFC42D:MFC42D.DLL
 0001:0004ad6e       ?OnActivateView@CFormView@@MAEXHPAVCView@@0@Z 5f54bd6e f   MFC42D:MFC42D.DLL
 0001:0004ad74       ?OnInitialUpdate@CFormView@@UAEXXZ 5f54bd74 f   MFC42D:MFC42D.DLL
 0001:0004ad7a       ?OnPrepareDC@CScrollView@@UAEXPAVCDC@@PAUCPrintInfo@@@Z 5f54bd7a f   MFC42D:MFC42D.DLL
 0001:0004ad80       ?OnScrollBy@CScrollView@@UAEHVCSize@@H@Z 5f54bd80 f   MFC42D:MFC42D.DLL
 0001:0004ad86       ?OnScroll@CScrollView@@UAEHIIH@Z 5f54bd86 f   MFC42D:MFC42D.DLL
 0001:0004ad8c       ?IsSelected@CView@@UBEHPBVCObject@@@Z 5f54bd8c f   MFC42D:MFC42D.DLL
 0001:0004ad92       ?SetOccDialogInfo@CFormView@@MAEHPAU_AFX_OCC_DIALOG_INFO@@@Z 5f54bd92 f   MFC42D:MFC42D.DLL
 0001:0004ad98       ?PreTranslateMessage@CFormView@@MAEHPAUtagMSG@@@Z 5f54bd98 f   MFC42D:MFC42D.DLL
 0001:0004ad9e       ?CalcWindowRect@CScrollView@@UAEXPAUtagRECT@@I@Z 5f54bd9e f   MFC42D:MFC42D.DLL
 0001:0004ada4       ?PreCreateWindow@CView@@MAEHAAUtagCREATESTRUCTA@@@Z 5f54bda4 f   MFC42D:MFC42D.DLL
 0001:0004adaa       ??0CFormView@@IAE@PBD@Z    5f54bdaa f   MFC42D:MFC42D.DLL
 0001:0004adb0       ??1CScrollView@@UAE@XZ     5f54bdb0 f   MFC42D:MFC42D.DLL
 0001:0004adb6       ?AssertValid@CFormView@@UBEXXZ 5f54bdb6 f   MFC42D:MFC42D.DLL
 0001:0004adbc       ?Dump@CFormView@@UBEXAAVCDumpContext@@@Z 5f54bdbc f   MFC42D:MFC42D.DLL
 0001:0004adc2       ?OnSize@CScrollView@@QAEXIHH@Z 5f54bdc2 f   MFC42D:MFC42D.DLL
 0001:0004adc8       ?Default@CWnd@@IAEJXZ      5f54bdc8 f   MFC42D:MFC42D.DLL
 0001:0004adce       ?GetControlUnknown@CWnd@@QAEPAUIUnknown@@XZ 5f54bdce f   MFC42D:MFC42D.DLL
 0001:0004add4       ??0CString@@QAE@PBG@Z      5f54bdd4 f   MFC42D:MFC42D.DLL
 0001:0004adda       ?AfxGetResourceHandle@@YGPAUHINSTANCE__@@XZ 5f54bdda f   MFC42D:MFC42D.DLL
 0001:0004ade0       ?InvokeHelper@CWnd@@QAAXJGGPAXPBEZZ 5f54bde0 f   MFC42D:MFC42D.DLL
 0001:0004ade6       ??1CByteArray@@UAE@XZ      5f54bde6 f   MFC42D:MFC42D.DLL
 0001:0004adec       ?GetData@CByteArray@@QAEPAEXZ 5f54bdec f   MFC42D:MFC42D.DLL
 0001:0004adf2       ?SetSize@CByteArray@@QAEXHH@Z 5f54bdf2 f   MFC42D:MFC42D.DLL
 0001:0004adf8       ??0CByteArray@@QAE@XZ      5f54bdf8 f   MFC42D:MFC42D.DLL
 0001:0004adfe       ?SetMessageText@CFrameWnd@@QAEXPBD@Z 5f54bdfe f   MFC42D:MFC42D.DLL
 0001:0004ae04       ?AfxFindResourceHandle@@YGPAUHINSTANCE__@@PBD0@Z 5f54be04 f   MFC42D:MFC42D.DLL
 0001:0004ae0a       ?GetNextAssoc@CMapPtrToPtr@@QBEXAAPAU__POSITION@@AAPAX1@Z 5f54be0a f   MFC42D:MFC42D.DLL
 0001:0004ae10       ?GetStartPosition@CMapPtrToPtr@@QBEPAU__POSITION@@XZ 5f54be10 f   MFC42D:MFC42D.DLL
 0001:0004ae16       ??0CMemFile@@QAE@PAEII@Z   5f54be16 f   MFC42D:MFC42D.DLL
 0001:0004ae1c       ?AfxThrowNotSupportedException@@YGXXZ 5f54be1c f   MFC42D:MFC42D.DLL
 0001:0004ae22       ?TopLeft@CRect@@QAEAAVCPoint@@XZ 5f54be22 f   MFC42D:MFC42D.DLL
 0001:0004ae28       ??0CRect@@QAE@ABUtagRECT@@@Z 5f54be28 f   MFC42D:MFC42D.DLL
 0001:0004ae2e       ?RemoveAll@CMapPtrToPtr@@QAEXXZ 5f54be2e f   MFC42D:MFC42D.DLL
 0001:0004ae34       ?RemoveKey@CMapPtrToPtr@@QAEHPAX@Z 5f54be34 f   MFC42D:MFC42D.DLL
 0001:0004ae3a       ?GetFont@CWnd@@QBEPAVCFont@@XZ 5f54be3a f   MFC42D:MFC42D.DLL
 0001:0004ae40       ??1CWindowDC@@UAE@XZ       5f54be40 f   MFC42D:MFC42D.DLL
 0001:0004ae46       ?GetTextColor@CDC@@QBEKXZ  5f54be46 f   MFC42D:MFC42D.DLL
 0001:0004ae4c       ?GetBkColor@CDC@@QBEKXZ    5f54be4c f   MFC42D:MFC42D.DLL
 0001:0004ae52       ??0CWindowDC@@QAE@PAVCWnd@@@Z 5f54be52 f   MFC42D:MFC42D.DLL
 0001:0004ae58       ?AfxGetCtl3dState@@YGPAV_AFX_CTL3D_STATE@@XZ 5f54be58 f   MFC42D:MFC42D.DLL
 0001:0004ae5e       ?GetLogFont@CFont@@QAEHPAUtagLOGFONTA@@@Z 5f54be5e f   MFC42D:MFC42D.DLL
 0001:0004ae64       ??1CFont@@UAE@XZ           5f54be64 f   MFC42D:MFC42D.DLL
 0001:0004ae6a       ?CreateStockObject@CGdiObject@@QAEHH@Z 5f54be6a f   MFC42D:MFC42D.DLL
 0001:0004ae70       ??0CFont@@QAE@XZ           5f54be70 f   MFC42D:MFC42D.DLL
 0001:0004ae76       ?GetWindowTextA@CWnd@@QBEHPADH@Z 5f54be76 f   MFC42D:MFC42D.DLL
 0001:0004ae7c       ?GetProperty@CWnd@@QBEXJGPAX@Z 5f54be7c f   MFC42D:MFC42D.DLL
 0001:0004ae82       ?GetCount@CMapPtrToPtr@@QBEHXZ 5f54be82 f   MFC42D:MFC42D.DLL
 0001:0004ae88       ??1CClientDC@@UAE@XZ       5f54be88 f   MFC42D:MFC42D.DLL
 0001:0004ae8e       ??0CClientDC@@QAE@PAVCWnd@@@Z 5f54be8e f   MFC42D:MFC42D.DLL
 0001:0004ae94       ?UnsubclassWindow@CWnd@@QAEPAUHWND__@@XZ 5f54be94 f   MFC42D:MFC42D.DLL
 0001:0004ae9a       ?ModifyStyle@CWnd@@SGHPAUHWND__@@KKI@Z 5f54be9a f   MFC42D:MFC42D.DLL
 0001:0004aea0       ?ModifyStyleEx@CWnd@@SGHPAUHWND__@@KKI@Z 5f54bea0 f   MFC42D:MFC42D.DLL
 0001:0004aea6       ??0CRect@@QAE@PBUtagRECT@@@Z 5f54bea6 f   MFC42D:MFC42D.DLL
 0001:0004aeac       ??1CPtrList@@UAE@XZ        5f54beac f   MFC42D:MFC42D.DLL
 0001:0004aeb2       ??0CPtrList@@QAE@H@Z       5f54beb2 f   MFC42D:MFC42D.DLL
 0001:0004aeb8       ?RemoveAll@CPtrList@@QAEXXZ 5f54beb8 f   MFC42D:MFC42D.DLL
 0001:0004aebe       ?GetHead@CPtrList@@QAEAAPAXXZ 5f54bebe f   MFC42D:MFC42D.DLL
 0001:0004aec4       ?MoveWindow@CWnd@@QAEXHHHHH@Z 5f54bec4 f   MFC42D:MFC42D.DLL
 0001:0004aeca       ?GetDesktopWindow@CWnd@@SGPAV1@XZ 5f54beca f   MFC42D:MFC42D.DLL
 0001:0004aed0       ?RemoveAt@CPtrList@@QAEXPAU__POSITION@@@Z 5f54bed0 f   MFC42D:MFC42D.DLL
 0001:0004aed6       ??8@YG_NABVCString@@PBD@Z  5f54bed6 f   MFC42D:MFC42D.DLL
 0001:0004aedc       ?AddTail@CPtrList@@QAEPAU__POSITION@@PAX@Z 5f54bedc f   MFC42D:MFC42D.DLL
 0001:0004aee2       ??8@YG_NABVCString@@0@Z    5f54bee2 f   MFC42D:MFC42D.DLL
 0001:0004aee8       ?Find@CPtrList@@QBEPAU__POSITION@@PAXPAU2@@Z 5f54bee8 f   MFC42D:MFC42D.DLL
 0001:0004aeee       ?GetCount@CPtrList@@QBEHXZ 5f54beee f   MFC42D:MFC42D.DLL
 0001:0004aef4       ?SetProperty@CWnd@@QAAXJGZZ 5f54bef4 f   MFC42D:MFC42D.DLL
 0001:0004aefa       ?GetNextWindow@CWnd@@QBEPAV1@I@Z 5f54befa f   MFC42D:MFC42D.DLL
 0001:0004af00       ?GetTopWindow@CWnd@@QBEPAV1@XZ 5f54bf00 f   MFC42D:MFC42D.DLL
 0001:0004af06       ?GetNextDlgGroupItem@CWnd@@QBEPAV1@PAV1@H@Z 5f54bf06 f   MFC42D:MFC42D.DLL
 0001:0004af0c       ?GetNextDlgTabItem@CWnd@@QBEPAV1@PAV1@H@Z 5f54bf0c f   MFC42D:MFC42D.DLL
 0001:0004af12       ?IsChild@CWnd@@QBEHPBV1@@Z 5f54bf12 f   MFC42D:MFC42D.DLL
 0001:0004af18       ?GetDlgCtrlID@CWnd@@QBEHXZ 5f54bf18 f   MFC42D:MFC42D.DLL
 0001:0004af1e       ?GetFromPage@CPrintInfo@@QBEIXZ 5f54bf1e f   MFC42D:MFC42D.DLL
 0001:0004af24       ?GetToPage@CPrintInfo@@QBEIXZ 5f54bf24 f   MFC42D:MFC42D.DLL
 0001:0004af2a       ?GetMinPage@CPrintInfo@@QBEIXZ 5f54bf2a f   MFC42D:MFC42D.DLL
 0001:0004af30       ??1CPrintInfo@@QAE@XZ      5f54bf30 f   MFC42D:MFC42D.DLL
 0001:0004af36       ??0CPrintInfo@@QAE@XZ      5f54bf36 f   MFC42D:MFC42D.DLL
 0001:0004af3c       ?AbortDoc@CDC@@QAEHXZ      5f54bf3c f   MFC42D:MFC42D.DLL
 0001:0004af42       ?EndDoc@CDC@@QAEHXZ        5f54bf42 f   MFC42D:MFC42D.DLL
 0001:0004af48       ?EndPage@CDC@@QAEHXZ       5f54bf48 f   MFC42D:MFC42D.DLL
 0001:0004af4e       ?StartPage@CDC@@QAEHXZ     5f54bf4e f   MFC42D:MFC42D.DLL
 0001:0004af54       ?GetMaxPage@CPrintInfo@@QBEIXZ 5f54bf54 f   MFC42D:MFC42D.DLL
 0001:0004af5a       ?Detach@CDC@@QAEPAUHDC__@@XZ 5f54bf5a f   MFC42D:MFC42D.DLL
 0001:0004af60       ?StartDocA@CDC@@QAEHPAU_DOCINFOA@@@Z 5f54bf60 f   MFC42D:MFC42D.DLL
 0001:0004af66       ?SetAbortProc@CDC@@QAEHP6GHPAUHDC__@@H@Z@Z 5f54bf66 f   MFC42D:MFC42D.DLL
 0001:0004af6c       ?_AfxAbortProc@@YGHPAUHDC__@@H@Z 5f54bf6c f   MFC42D:MFC42D.DLL
 0001:0004af72       ?Attach@CDC@@QAEHPAUHDC__@@@Z 5f54bf72 f   MFC42D:MFC42D.DLL
 0001:0004af78       ?GetWindowTextA@CWnd@@QBEXAAVCString@@@Z 5f54bf78 f   MFC42D:MFC42D.DLL
 0001:0004af7e       ?SetRadio@CCmdUI@@UAEXH@Z  5f54bf7e f   MFC42D:MFC42D.DLL
 0001:0004af84       ??0CCmdUI@@QAE@XZ          5f54bf84 f   MFC42D:MFC42D.DLL
 0001:0004af8a       ?Right@CString@@QBE?AV1@H@Z 5f54bf8a f   MFC42D:MFC42D.DLL
 0001:0004af90       ?RemoveMenu@CMenu@@QAEHII@Z 5f54bf90 f   MFC42D:MFC42D.DLL
 0001:0004af96       ?GetMenuItemCount@CMenu@@QBEIXZ 5f54bf96 f   MFC42D:MFC42D.DLL
 0001:0004af9c       ?CreateMenu@CMenu@@QAEHXZ  5f54bf9c f   MFC42D:MFC42D.DLL
 0001:0004afa2       ??0CMenu@@QAE@XZ           5f54bfa2 f   MFC42D:MFC42D.DLL
 0001:0004afa8       ?Remove@CString@@QAEHD@Z   5f54bfa8 f   MFC42D:MFC42D.DLL
 0001:0004afae       ?GetMenuStringA@CMenu@@QBEHIAAVCString@@I@Z 5f54bfae f   MFC42D:MFC42D.DLL
 0001:0004afb4       ?GetSubMenu@CMenu@@QBEPAV1@H@Z 5f54bfb4 f   MFC42D:MFC42D.DLL
 0001:0004afba       ?SetStatusText@CControlBar@@UAEHH@Z 5f54bfba f   MFC42D:MFC42D.DLL
 0001:0004afc0       ?DoPaint@CControlBar@@UAEXPAVCDC@@@Z 5f54bfc0 f   MFC42D:MFC42D.DLL
 0001:0004afc6       ?OnBarStyleChange@CControlBar@@UAEXKK@Z 5f54bfc6 f   MFC42D:MFC42D.DLL
 0001:0004afcc       ?IsDockBar@CControlBar@@UBEHXZ 5f54bfcc f   MFC42D:MFC42D.DLL
 0001:0004afd2       ?RecalcDelayShow@CControlBar@@UAEKPAUAFX_SIZEPARENTPARAMS@@@Z 5f54bfd2 f   MFC42D:MFC42D.DLL
 0001:0004afd8       ?IsVisible@CControlBar@@UBEHXZ 5f54bfd8 f   MFC42D:MFC42D.DLL
 0001:0004afde       ?DelayShow@CControlBar@@UAEXH@Z 5f54bfde f   MFC42D:MFC42D.DLL
 0001:0004afe4       ?CalcDynamicLayout@CControlBar@@UAE?AVCSize@@HK@Z 5f54bfe4 f   MFC42D:MFC42D.DLL
 0001:0004afea       ?CalcFixedLayout@CControlBar@@UAE?AVCSize@@HH@Z 5f54bfea f   MFC42D:MFC42D.DLL
 0001:0004aff0       ?PostNcDestroy@CControlBar@@UAEXXZ 5f54bff0 f   MFC42D:MFC42D.DLL
 0001:0004aff6       ?WindowProc@CControlBar@@UAEJIIJ@Z 5f54bff6 f   MFC42D:MFC42D.DLL
 0001:0004affc       ?PreTranslateMessage@CControlBar@@UAEHPAUtagMSG@@@Z 5f54bffc f   MFC42D:MFC42D.DLL
 0001:0004b002       ?PreCreateWindow@CControlBar@@UAEHAAUtagCREATESTRUCTA@@@Z 5f54c002 f   MFC42D:MFC42D.DLL
 0001:0004b008       ?DestroyWindow@CControlBar@@UAEHXZ 5f54c008 f   MFC42D:MFC42D.DLL
 0001:0004b00e       ?Dump@CControlBar@@UBEXAAVCDumpContext@@@Z 5f54c00e f   MFC42D:MFC42D.DLL
 0001:0004b014       ?AssertValid@CControlBar@@UBEXXZ 5f54c014 f   MFC42D:MFC42D.DLL
 0001:0004b01a       ??1CControlBar@@UAE@XZ     5f54c01a f   MFC42D:MFC42D.DLL
 0001:0004b020       ??0CRectTracker@@QAE@XZ    5f54c020 f   MFC42D:MFC42D.DLL
 0001:0004b026       ??0CControlBar@@IAE@XZ     5f54c026 f   MFC42D:MFC42D.DLL
 0001:0004b02c       ??1CRectTracker@@UAE@XZ    5f54c02c f   MFC42D:MFC42D.DLL
 0001:0004b032       ??1CPaintDC@@UAE@XZ        5f54c032 f   MFC42D:MFC42D.DLL
 0001:0004b038       ?Draw@CRectTracker@@QBEXPAVCDC@@@Z 5f54c038 f   MFC42D:MFC42D.DLL
 0001:0004b03e       ?SetBrushOrg@CDC@@QAE?AVCPoint@@HH@Z 5f54c03e f   MFC42D:MFC42D.DLL
 0001:0004b044       ??0CPaintDC@@QAE@PAVCWnd@@@Z 5f54c044 f   MFC42D:MFC42D.DLL
 0001:0004b04a       ?SetCursor@CRectTracker@@QBEHPAVCWnd@@I@Z 5f54c04a f   MFC42D:MFC42D.DLL
 0001:0004b050       ?OnSetCursor@CWnd@@IAEHPAV1@II@Z 5f54c050 f   MFC42D:MFC42D.DLL
 0001:0004b056       ?HitTest@CRectTracker@@QBEHVCPoint@@@Z 5f54c056 f   MFC42D:MFC42D.DLL
 0001:0004b05c       ?GetOwner@CWnd@@QBEPAV1@XZ 5f54c05c f   MFC42D:MFC42D.DLL
 0001:0004b062       ?Track@CRectTracker@@QAEHPAVCWnd@@VCPoint@@H0@Z 5f54c062 f   MFC42D:MFC42D.DLL
 0001:0004b068       ?SetWindowOrg@CDC@@QAE?AVCPoint@@HH@Z 5f54c068 f   MFC42D:MFC42D.DLL
 0001:0004b06e       ?SetViewportExt@CDC@@QAE?AVCSize@@UtagSIZE@@@Z 5f54c06e f   MFC42D:MFC42D.DLL
 0001:0004b074       ?CreateEx@CWnd@@QAEHKPBD0KHHHHPAUHWND__@@PAUHMENU__@@PAX@Z 5f54c074 f   MFC42D:MFC42D.DLL
 0001:0004b07a       ?LPtoDP@CDC@@QBEXPAUtagRECT@@@Z 5f54c07a f   MFC42D:MFC42D.DLL
 0001:0004b080       ?SetWindowExt@CDC@@UAE?AVCSize@@HH@Z 5f54c080 f   MFC42D:MFC42D.DLL
 0001:0004b086       ?SetMapMode@CDC@@UAEHH@Z   5f54c086 f   MFC42D:MFC42D.DLL
 0001:0004b08c       ?InvalidateRect@CWnd@@QAEXPBUtagRECT@@H@Z 5f54c08c f   MFC42D:MFC42D.DLL
 0001:0004b092       ?OffsetRect@CRect@@QAEXUtagPOINT@@@Z 5f54c092 f   MFC42D:MFC42D.DLL
 0001:0004b098       ?AfxUnlockTempMaps@@YGHH@Z 5f54c098 f   MFC42D:MFC42D.DLL
 0001:0004b09e       ?AfxLockTempMaps@@YGXXZ    5f54c09e f   MFC42D:MFC42D.DLL
 0001:0004b0a4       ?ValidateRect@CWnd@@QAEXPBUtagRECT@@@Z 5f54c0a4 f   MFC42D:MFC42D.DLL
 0001:0004b0aa       ?OnEraseBkgnd@CWnd@@IAEHPAVCDC@@@Z 5f54c0aa f   MFC42D:MFC42D.DLL
 0001:0004b0b0       ?IsLoading@CArchive@@QBEHXZ 5f54c0b0 f   MFC42D:MFC42D.DLL
 0001:0004b0b6       ?OnNcCreate@CWnd@@IAEHPAUtagCREATESTRUCTA@@@Z 5f54c0b6 f   MFC42D:MFC42D.DLL
 0001:0004b0bc       ?OnMouseActivate@CWnd@@IAEHPAV1@II@Z 5f54c0bc f   MFC42D:MFC42D.DLL
 0001:0004b0c2       ?ReflectChildNotify@CWnd@@IAEHIIJPAJ@Z 5f54c0c2 f   MFC42D:MFC42D.DLL
 0001:0004b0c8       ?OnCreate@CWnd@@IAEHPAUtagCREATESTRUCTA@@@Z 5f54c0c8 f   MFC42D:MFC42D.DLL
 0001:0004b0ce       ?OnMove@CWnd@@IAEXHH@Z     5f54c0ce f   MFC42D:MFC42D.DLL
 0001:0004b0d4       ?OnShowWindow@CWnd@@IAEXHI@Z 5f54c0d4 f   MFC42D:MFC42D.DLL
 0001:0004b0da       ?DoUpdate@CCmdUI@@QAEHPAVCCmdTarget@@H@Z 5f54c0da f   MFC42D:MFC42D.DLL
 0001:0004b0e0       ?GetMenuItemID@CMenu@@QBEIH@Z 5f54c0e0 f   MFC42D:MFC42D.DLL
 0001:0004b0e6       ?AfxCancelModes@@YGXPAUHWND__@@@Z 5f54c0e6 f   MFC42D:MFC42D.DLL
 0001:0004b0ec       ?OnDestroy@CWnd@@IAEXXZ    5f54c0ec f   MFC42D:MFC42D.DLL
 0001:0004b0f2       ?OnKillFocus@CWnd@@IAEXPAV1@@Z 5f54c0f2 f   MFC42D:MFC42D.DLL
 0001:0004b0f8       ?OnSetFocus@CWnd@@IAEXPAV1@@Z 5f54c0f8 f   MFC42D:MFC42D.DLL
 0001:0004b0fe       ?GetData@CThreadLocalObject@@QAEPAVCNoTrackObject@@P6GPAV2@XZ@Z 5f54c0fe f   MFC42D:MFC42D.DLL
 0001:0004b104       ?GetRuntimeClass@CWnd@@UBEPAUCRuntimeClass@@XZ 5f54c104 f   MFC42D:MFC42D.DLL
 0001:0004b10a       ?Add@CPtrArray@@QAEHPAX@Z  5f54c10a f   MFC42D:MFC42D.DLL
 0001:0004b110       ?OnGetDlgCode@CWnd@@IAEIXZ 5f54c110 f   MFC42D:MFC42D.DLL
 0001:0004b116       ?OnCancelMode@CWnd@@IAEXXZ 5f54c116 f   MFC42D:MFC42D.DLL
 0001:0004b11c       ?MessageBoxA@CWnd@@QAEHPBD0I@Z 5f54c11c f   MFC42D:MFC42D.DLL
 0001:0004b122       ?ExitInstance@CWinApp@@UAEHXZ 5f54c122 f   MFC42D:MFC42D.DLL
 0001:0004b128       ?OnActivate@CWnd@@IAEXIPAV1@H@Z 5f54c128 f   MFC42D:MFC42D.DLL
 0001:0004b12e       ??4CRect@@QAEXABUtagRECT@@@Z 5f54c12e f   MFC42D:MFC42D.DLL
 0001:0004b134       ?Read@CFile@@UAEIPAXI@Z    5f54c134 f   MFC42D:MFC42D.DLL
 0001:0004b13a       ?_wcstombsz@@YAHPADPBGI@Z  5f54c13a f   MFC42D:MFC42D.DLL
 0001:0004b140       ??0CFile@@QAE@PBDI@Z       5f54c140 f   MFC42D:MFC42D.DLL
 0001:0004b146       ?GetSize@CPtrArray@@QBEHXZ 5f54c146 f   MFC42D:MFC42D.DLL
 0001:0004b14c       ?GetAt@CPtrArray@@QBEPAXH@Z 5f54c14c f   MFC42D:MFC42D.DLL
 0001:0004b152       ??0CPtrArray@@QAE@XZ       5f54c152 f   MFC42D:MFC42D.DLL
 0001:0004b158       ?RemoveAt@CPtrArray@@QAEXHH@Z 5f54c158 f   MFC42D:MFC42D.DLL
 0001:0004b15e       ??1CPtrArray@@UAE@XZ       5f54c15e f   MFC42D:MFC42D.DLL
 0001:0004b164       ??1CBitmap@@UAE@XZ         5f54c164 f   MFC42D:MFC42D.DLL
 0001:0004b16a       ?Detach@CGdiObject@@QAEPAXXZ 5f54c16a f   MFC42D:MFC42D.DLL
 0001:0004b170       ?LoadBitmapA@CBitmap@@QAEHI@Z 5f54c170 f   MFC42D:MFC42D.DLL
 0001:0004b176       ??0CBitmap@@QAE@XZ         5f54c176 f   MFC42D:MFC42D.DLL
 0001:0004b17c       ?GetSafeHandle@CGdiObject@@QBEPAXXZ 5f54c17c f   MFC42D:MFC42D.DLL
 0001:0004b182       ?LoadIconA@CWinApp@@QBEPAUHICON__@@I@Z 5f54c182 f   MFC42D:MFC42D.DLL
 0001:0004b188       ??6@YGAAVCArchive@@AAV0@ABVCString@@@Z 5f54c188 f   MFC42D:MFC42D.DLL
 0001:0004b18e       ??5@YGAAVCArchive@@AAV0@AAVCString@@@Z 5f54c18e f   MFC42D:MFC42D.DLL
 0001:0004b194       ?OnQuery3dControls@CWnd@@IAEJIJ@Z 5f54c194 f   MFC42D:MFC42D.DLL
 0001:0004b19a       ?GetRuntimeClass@CObject@@UBEPAUCRuntimeClass@@XZ 5f54c19a f   MFC42D:MFC42D.DLL
 0001:0004b1a0       ??0CObject@@IAE@XZ         5f54c1a0 f   MFC42D:MFC42D.DLL
 0001:0004b1a6       ??1CObject@@UAE@XZ         5f54c1a6 f   MFC42D:MFC42D.DLL
 0001:0004b1ac       ?RemoveAll@CPtrArray@@QAEXXZ 5f54c1ac f   MFC42D:MFC42D.DLL
 0001:0004b1b2       ??ACPtrArray@@QAEAAPAXH@Z  5f54c1b2 f   MFC42D:MFC42D.DLL
 0001:0004b1b8       ?GetFont@CDialogTemplate@@QBEHAAVCString@@AAG@Z 5f54c1b8 f   MFC42D:MFC42D.DLL
 0001:0004b1be       ?GetSizeInDialogUnits@CDialogTemplate@@QBEXPAUtagSIZE@@@Z 5f54c1be f   MFC42D:MFC42D.DLL
 0001:0004b1c4       ?AddHead@CPtrList@@QAEPAU__POSITION@@PAX@Z 5f54c1c4 f   MFC42D:MFC42D.DLL
 0001:0004b1ca       ?AfxEnableMemoryTracking@@YGHH@Z 5f54c1ca f   MFC42D:MFC42D.DLL
 0001:0004b1d0       ?OnCancel@CDialog@@MAEXXZ  5f54c1d0 f   MFC42D:MFC42D.DLL
 0001:0004b1d6       ?OnOK@CDialog@@MAEXXZ      5f54c1d6 f   MFC42D:MFC42D.DLL
 0001:0004b1dc       ??0CDialog@@QAE@XZ         5f54c1dc f   MFC42D:MFC42D.DLL
 0001:0004b1e2       ??1CDialogTemplate@@QAE@XZ 5f54c1e2 f   MFC42D:MFC42D.DLL
 0001:0004b1e8       ?Detach@CDialogTemplate@@QAEPAXXZ 5f54c1e8 f   MFC42D:MFC42D.DLL
 0001:0004b1ee       ?GetSizeInPixels@CDialogTemplate@@QBEXPAUtagSIZE@@@Z 5f54c1ee f   MFC42D:MFC42D.DLL
 0001:0004b1f4       ?SetFont@CDialogTemplate@@QAEHPBDG@Z 5f54c1f4 f   MFC42D:MFC42D.DLL
 0001:0004b1fa       ?AfxGetPropSheetFont@@YGHAAVCString@@AAGH@Z 5f54c1fa f   MFC42D:MFC42D.DLL
 0001:0004b200       ?HasFont@CDialogTemplate@@QBEHXZ 5f54c200 f   MFC42D:MFC42D.DLL
 0001:0004b206       ?Load@CDialogTemplate@@QAEHPBD@Z 5f54c206 f   MFC42D:MFC42D.DLL
 0001:0004b20c       ??0CDialogTemplate@@QAE@PBUDLGTEMPLATE@@@Z 5f54c20c f   MFC42D:MFC42D.DLL
 0001:0004b212       ?GetCurrentMessage@CWnd@@KGPBUtagMSG@@XZ 5f54c212 f   MFC42D:MFC42D.DLL
 0001:0004b218       ?SendChildNotifyLastMsg@CWnd@@QAEHPAJ@Z 5f54c218 f   MFC42D:MFC42D.DLL
 0001:0004b21e       ??0CDialogTemplate@@QAE@PAX@Z 5f54c21e f   MFC42D:MFC42D.DLL
 0001:0004b224       ?UpdateData@CWnd@@QAEHH@Z  5f54c224 f   MFC42D:MFC42D.DLL
 0001:0004b22a       ?Create@CDialog@@QAEHIPAVCWnd@@@Z 5f54c22a f   MFC42D:MFC42D.DLL
 0001:0004b230       ?CreateIndirect@CDialog@@QAEHPAXPAVCWnd@@@Z 5f54c230 f   MFC42D:MFC42D.DLL
 0001:0004b236       ?GetWindow@CWnd@@QBEPAV1@I@Z 5f54c236 f   MFC42D:MFC42D.DLL
 0001:0004b23c       ?GotoDlgCtrl@CDialog@@QAEXPAVCWnd@@@Z 5f54c23c f   MFC42D:MFC42D.DLL
 0001:0004b242       ?GetDefID@CDialog@@QBEKXZ  5f54c242 f   MFC42D:MFC42D.DLL
 0001:0004b248       ?GetAt@CDWordArray@@QBEKH@Z 5f54c248 f   MFC42D:MFC42D.DLL
 0001:0004b24e       ??9@YG_NABVCString@@0@Z    5f54c24e f   MFC42D:MFC42D.DLL
 0001:0004b254       ??6CArchive@@QAEAAV0@H@Z   5f54c254 f   MFC42D:MFC42D.DLL
 0001:0004b25a       ??6CArchive@@QAEAAV0@F@Z   5f54c25a f   MFC42D:MFC42D.DLL
 0001:0004b260       ??5CArchive@@QAEAAV0@AAH@Z 5f54c260 f   MFC42D:MFC42D.DLL
 0001:0004b266       ??5CArchive@@QAEAAV0@AAF@Z 5f54c266 f   MFC42D:MFC42D.DLL
 0001:0004b26c       ?GetAt@CStringArray@@QBE?AVCString@@H@Z 5f54c26c f   MFC42D:MFC42D.DLL
 0001:0004b272       ??1CStringArray@@UAE@XZ    5f54c272 f   MFC42D:MFC42D.DLL
 0001:0004b278       ?GetSize@CStringArray@@QBEHXZ 5f54c278 f   MFC42D:MFC42D.DLL
 0001:0004b27e       ??0CStringArray@@QAE@XZ    5f54c27e f   MFC42D:MFC42D.DLL
 0001:0004b284       ?RemoveAll@CStringArray@@QAEXXZ 5f54c284 f   MFC42D:MFC42D.DLL
 0001:0004b28a       ?Add@CStringArray@@QAEHABVCString@@@Z 5f54c28a f   MFC42D:MFC42D.DLL
 0001:0004b290       ?SeekToEnd@CFile@@QAEKXZ   5f54c290 f   MFC42D:MFC42D.DLL
 0001:0004b296       ?Compare@CString@@QBEHPBD@Z 5f54c296 f   MFC42D:MFC42D.DLL
 0001:0004b29c       ?AfxDelRegTreeHelper@@YGJPAUHKEY__@@ABVCString@@@Z 5f54c29c f   MFC42D:MFC42D.DLL
 0001:0004b2a2       ?ReverseFind@CString@@QBEHD@Z 5f54c2a2 f   MFC42D:MFC42D.DLL
 0001:0004b2a8       ??1CBrush@@UAE@XZ          5f54c2a8 f   MFC42D:MFC42D.DLL
 0001:0004b2ae       ?FillRect@CDC@@QAEXPBUtagRECT@@PAVCBrush@@@Z 5f54c2ae f   MFC42D:MFC42D.DLL
 0001:0004b2b4       ??0CBrush@@QAE@K@Z         5f54c2b4 f   MFC42D:MFC42D.DLL
 0001:0004b2ba       ??9CRect@@QBEHABUtagRECT@@@Z 5f54c2ba f   MFC42D:MFC42D.DLL
 0001:0004b2c0       ?GetHandleSize@CRectTracker@@MBEHPBUtagRECT@@@Z 5f54c2c0 f   MFC42D:MFC42D.DLL
 0001:0004b2c6       ?GetHandleMask@CRectTracker@@UBEIXZ 5f54c2c6 f   MFC42D:MFC42D.DLL
 0001:0004b2cc       ?OnChangedRect@CRectTracker@@UAEXABVCRect@@@Z 5f54c2cc f   MFC42D:MFC42D.DLL
 0001:0004b2d2       ?AdjustRect@CRectTracker@@UAEXHPAUtagRECT@@@Z 5f54c2d2 f   MFC42D:MFC42D.DLL
 0001:0004b2d8       ?DrawTrackerRect@CRectTracker@@UAEXPBUtagRECT@@PAVCWnd@@PAVCDC@@1@Z 5f54c2d8 f   MFC42D:MFC42D.DLL
 0001:0004b2de       ??0CRectTracker@@QAE@PBUtagRECT@@I@Z 5f54c2de f   MFC42D:MFC42D.DLL
 0001:0004b2e4       ?FromHandle@CDC@@SGPAV1@PAUHDC__@@@Z 5f54c2e4 f   MFC42D:MFC42D.DLL
 0001:0004b2ea       ??1CMapStringToPtr@@UAE@XZ 5f54c2ea f   MFC42D:MFC42D.DLL
 0001:0004b2f0       ??0CMapStringToPtr@@QAE@H@Z 5f54c2f0 f   MFC42D:MFC42D.DLL
 0001:0004b2f6       ?Lookup@CMapStringToPtr@@QBEHPBDAAPAX@Z 5f54c2f6 f   MFC42D:MFC42D.DLL
 0001:0004b2fc       ?MakeLower@CString@@QAEXXZ 5f54c2fc f   MFC42D:MFC42D.DLL
 0001:0004b302       ?SetAt@CMapStringToPtr@@QAEXPBDPAX@Z 5f54c302 f   MFC42D:MFC42D.DLL
 0001:0004b308       ?GetNextAssoc@CMapStringToPtr@@QBEXAAPAU__POSITION@@AAVCString@@AAPAX@Z 5f54c308 f   MFC42D:MFC42D.DLL
 0001:0004b30e       ?GetStartPosition@CMapStringToPtr@@QBEPAU__POSITION@@XZ 5f54c30e f   MFC42D:MFC42D.DLL
 0001:0004b314       ?GetCount@CMapStringToPtr@@QBEHXZ 5f54c314 f   MFC42D:MFC42D.DLL
 0001:0004b31a       ??1CThreadLocalObject@@QAE@XZ 5f54c31a f   MFC42D:MFC42D.DLL
 0001:0004b320       ?Escape@CDC@@UAEHHHPBDPAX@Z 5f54c320 f   MFC42D:MFC42D.DLL
 0001:0004b326       ?GrayStringA@CDC@@UAEHPAVCBrush@@P6GHPAUHDC__@@JH@ZJHHHHH@Z 5f54c326 f   MFC42D:MFC42D.DLL
 0001:0004b32c       ?DrawTextA@CDC@@UAEHPBDHPAUtagRECT@@I@Z 5f54c32c f   MFC42D:MFC42D.DLL
 0001:0004b332       ?TabbedTextOutA@CDC@@UAE?AVCSize@@HHPBDHHPAHH@Z 5f54c332 f   MFC42D:MFC42D.DLL
 0001:0004b338       ?ExtTextOutA@CDC@@UAEHHHIPBUtagRECT@@PBDIPAH@Z 5f54c338 f   MFC42D:MFC42D.DLL
 0001:0004b33e       ?TextOutA@CDC@@UAEHHHPBDH@Z 5f54c33e f   MFC42D:MFC42D.DLL
 0001:0004b344       ?RectVisible@CDC@@UBEHPBUtagRECT@@@Z 5f54c344 f   MFC42D:MFC42D.DLL
 0001:0004b34a       ?PtVisible@CDC@@UBEHHH@Z   5f54c34a f   MFC42D:MFC42D.DLL
 0001:0004b350       ?GetClipBox@CDC@@UBEHPAUtagRECT@@@Z 5f54c350 f   MFC42D:MFC42D.DLL
 0001:0004b356       ?ScaleWindowExt@CDC@@UAE?AVCSize@@HHHH@Z 5f54c356 f   MFC42D:MFC42D.DLL
 0001:0004b35c       ?ScaleViewportExt@CDC@@UAE?AVCSize@@HHHH@Z 5f54c35c f   MFC42D:MFC42D.DLL
 0001:0004b362       ?SetViewportExt@CDC@@UAE?AVCSize@@HH@Z 5f54c362 f   MFC42D:MFC42D.DLL
 0001:0004b368       ?OffsetViewportOrg@CDC@@UAE?AVCPoint@@HH@Z 5f54c368 f   MFC42D:MFC42D.DLL
 0001:0004b36e       ?SetViewportOrg@CDC@@UAE?AVCPoint@@HH@Z 5f54c36e f   MFC42D:MFC42D.DLL
 0001:0004b374       ?SetTextColor@CDC@@UAEKK@Z 5f54c374 f   MFC42D:MFC42D.DLL
 0001:0004b37a       ?SetBkColor@CDC@@UAEKK@Z   5f54c37a f   MFC42D:MFC42D.DLL
 0001:0004b380       ?SelectObject@CDC@@UAEPAVCFont@@PAV2@@Z 5f54c380 f   MFC42D:MFC42D.DLL
 0001:0004b386       ?SelectStockObject@CDC@@UAEPAVCGdiObject@@H@Z 5f54c386 f   MFC42D:MFC42D.DLL
 0001:0004b38c       ?RestoreDC@CDC@@UAEHH@Z    5f54c38c f   MFC42D:MFC42D.DLL
 0001:0004b392       ?SaveDC@CDC@@UAEHXZ        5f54c392 f   MFC42D:MFC42D.DLL
 0001:0004b398       ?ReleaseOutputDC@CDC@@UAEXXZ 5f54c398 f   MFC42D:MFC42D.DLL
 0001:0004b39e       ?ReleaseAttribDC@CDC@@UAEXXZ 5f54c39e f   MFC42D:MFC42D.DLL
 0001:0004b3a4       ?SetOutputDC@CDC@@UAEXPAUHDC__@@@Z 5f54c3a4 f   MFC42D:MFC42D.DLL
 0001:0004b3aa       ?SetAttribDC@CDC@@UAEXPAUHDC__@@@Z 5f54c3aa f   MFC42D:MFC42D.DLL
 0001:0004b3b0       ?Dump@CDC@@UBEXAAVCDumpContext@@@Z 5f54c3b0 f   MFC42D:MFC42D.DLL
 0001:0004b3b6       ?AssertValid@CDC@@UBEXXZ   5f54c3b6 f   MFC42D:MFC42D.DLL
 0001:0004b3bc       ?SetViewportOrg@CDC@@QAE?AVCPoint@@UtagPOINT@@@Z 5f54c3bc f   MFC42D:MFC42D.DLL
 0001:0004b3c2       ??HCPoint@@QBE?AV0@UtagPOINT@@@Z 5f54c3c2 f   MFC42D:MFC42D.DLL
 0001:0004b3c8       ?GetViewportOrg@CDC@@QBE?AVCPoint@@XZ 5f54c3c8 f   MFC42D:MFC42D.DLL
 0001:0004b3ce       ?GetDC@CWnd@@QAEPAVCDC@@XZ 5f54c3ce f   MFC42D:MFC42D.DLL
 0001:0004b3d4       ?ReleaseDC@CWnd@@QAEHPAVCDC@@@Z 5f54c3d4 f   MFC42D:MFC42D.DLL
 0001:0004b3da       ?InvalidateRgn@CWnd@@QAEXPAVCRgn@@H@Z 5f54c3da f   MFC42D:MFC42D.DLL
 0001:0004b3e0       ??1CRgn@@UAE@XZ            5f54c3e0 f   MFC42D:MFC42D.DLL
 0001:0004b3e6       ??BCRgn@@QBEPAUHRGN__@@XZ  5f54c3e6 f   MFC42D:MFC42D.DLL
 0001:0004b3ec       ?OffsetRgn@CRgn@@QAEHUtagPOINT@@@Z 5f54c3ec f   MFC42D:MFC42D.DLL
 0001:0004b3f2       ?CopyRgn@CRgn@@QAEHPAV1@@Z 5f54c3f2 f   MFC42D:MFC42D.DLL
 0001:0004b3f8       ??0CRgn@@QAE@XZ            5f54c3f8 f   MFC42D:MFC42D.DLL
 0001:0004b3fe       ?ScrollWindow@CWnd@@QAEXHHPBUtagRECT@@0@Z 5f54c3fe f   MFC42D:MFC42D.DLL
 0001:0004b404       ?OnChildNotify@CButton@@MAEHIIJPAJ@Z 5f54c404 f   MFC42D:MFC42D.DLL
 0001:0004b40a       ?GetRuntimeClass@CButton@@UBEPAUCRuntimeClass@@XZ 5f54c40a f   MFC42D:MFC42D.DLL
 0001:0004b410       ??0CButton@@QAE@XZ         5f54c410 f   MFC42D:MFC42D.DLL
 0001:0004b416       ??1CButton@@UAE@XZ         5f54c416 f   MFC42D:MFC42D.DLL
 0001:0004b41c       ?GetNearestColor@CDC@@QBEKK@Z 5f54c41c f   MFC42D:MFC42D.DLL
 0001:0004b422       ?GetState@CButton@@QBEIXZ  5f54c422 f   MFC42D:MFC42D.DLL
 0001:0004b428       ?RealizePalette@CDC@@QAEIXZ 5f54c428 f   MFC42D:MFC42D.DLL
 0001:0004b42e       ?SelectPalette@CDC@@QAEPAVCPalette@@PAV2@H@Z 5f54c42e f   MFC42D:MFC42D.DLL
 0001:0004b434       ?FromHandle@CPalette@@SGPAV1@PAUHPALETTE__@@@Z 5f54c434 f   MFC42D:MFC42D.DLL
 0001:0004b43a       ??1CComboBox@@UAE@XZ       5f54c43a f   MFC42D:MFC42D.DLL
 0001:0004b440       ??0CComboBox@@QAE@XZ       5f54c440 f   MFC42D:MFC42D.DLL
 0001:0004b446       ?SubclassDlgItem@CWnd@@QAEHIPAV1@@Z 5f54c446 f   MFC42D:MFC42D.DLL
 0001:0004b44c       ?SetCurSel@CComboBox@@QAEHH@Z 5f54c44c f   MFC42D:MFC42D.DLL
 0001:0004b452       ?SetItemData@CComboBox@@QAEHHK@Z 5f54c452 f   MFC42D:MFC42D.DLL
 0001:0004b458       ?AddString@CComboBox@@QAEHPBD@Z 5f54c458 f   MFC42D:MFC42D.DLL
 0001:0004b45e       ?GetCount@CComboBox@@QBEHXZ 5f54c45e f   MFC42D:MFC42D.DLL
 0001:0004b464       ?GetItemData@CComboBox@@QBEKH@Z 5f54c464 f   MFC42D:MFC42D.DLL
 0001:0004b46a       ?GetCurSel@CComboBox@@QBEHXZ 5f54c46a f   MFC42D:MFC42D.DLL
 0001:0004b470       ?DDX_Control@@YGXPAVCDataExchange@@HAAVCWnd@@@Z 5f54c470 f   MFC42D:MFC42D.DLL
 0001:0004b476       ?LineTo@CDC@@QAEHHH@Z      5f54c476 f   MFC42D:MFC42D.DLL
 0001:0004b47c       ?MoveTo@CDC@@QAE?AVCPoint@@HH@Z 5f54c47c f   MFC42D:MFC42D.DLL
 0001:0004b482       ?SelectObject@CDC@@QAEPAVCPen@@PAV2@@Z 5f54c482 f   MFC42D:MFC42D.DLL
 0001:0004b488       ??0CPen@@QAE@HHK@Z         5f54c488 f   MFC42D:MFC42D.DLL
 0001:0004b48e       ?FrameRect@CDC@@QAEXPBUtagRECT@@PAVCBrush@@@Z 5f54c48e f   MFC42D:MFC42D.DLL
 0001:0004b494       ??1CStatic@@UAE@XZ         5f54c494 f   MFC42D:MFC42D.DLL
 0001:0004b49a       ??0CStatic@@QAE@XZ         5f54c49a f   MFC42D:MFC42D.DLL
 0001:0004b4a0       ?DeleteItem@CComboBox@@UAEXPAUtagDELETEITEMSTRUCT@@@Z 5f54c4a0 f   MFC42D:MFC42D.DLL
 0001:0004b4a6       ?CompareItem@CComboBox@@UAEHPAUtagCOMPAREITEMSTRUCT@@@Z 5f54c4a6 f   MFC42D:MFC42D.DLL
 0001:0004b4ac       ?MeasureItem@CComboBox@@UAEXPAUtagMEASUREITEMSTRUCT@@@Z 5f54c4ac f   MFC42D:MFC42D.DLL
 0001:0004b4b2       ?DrawItem@CComboBox@@UAEXPAUtagDRAWITEMSTRUCT@@@Z 5f54c4b2 f   MFC42D:MFC42D.DLL
 0001:0004b4b8       ?OnChildNotify@CComboBox@@MAEHIIJPAJ@Z 5f54c4b8 f   MFC42D:MFC42D.DLL
 0001:0004b4be       ?GetRuntimeClass@CComboBox@@UBEPAUCRuntimeClass@@XZ 5f54c4be f   MFC42D:MFC42D.DLL
 0001:0004b4c4       ?BitBlt@CDC@@QAEHHHHHPAV1@HHK@Z 5f54c4c4 f   MFC42D:MFC42D.DLL
 0001:0004b4ca       ?SelectObject@CDC@@QAEPAVCBitmap@@PAV2@@Z 5f54c4ca f   MFC42D:MFC42D.DLL
 0001:0004b4d0       ?CreateCompatibleDC@CDC@@QAEHPAV1@@Z 5f54c4d0 f   MFC42D:MFC42D.DLL
 0001:0004b4d6       ?GetPixel@CDC@@QBEKHH@Z    5f54c4d6 f   MFC42D:MFC42D.DLL
 0001:0004b4dc       ?CreateBitmap@CBitmap@@QAEHHHIIPBX@Z 5f54c4dc f   MFC42D:MFC42D.DLL
 0001:0004b4e2       ?GetObjectA@CGdiObject@@QBEHHPAX@Z 5f54c4e2 f   MFC42D:MFC42D.DLL
 0001:0004b4e8       ?GetSafeHdc@CDC@@QBEPAUHDC__@@XZ 5f54c4e8 f   MFC42D:MFC42D.DLL
 0001:0004b4ee       ?ResetContent@CComboBox@@QAEXXZ 5f54c4ee f   MFC42D:MFC42D.DLL
 0001:0004b4f4       ?SelectString@CComboBox@@QAEHHPBD@Z 5f54c4f4 f   MFC42D:MFC42D.DLL
 0001:0004b4fa       ?FindString@CComboBox@@QBEHHPBD@Z 5f54c4fa f   MFC42D:MFC42D.DLL
 0001:0004b500       ?GetLBText@CComboBox@@QBEXHAAVCString@@@Z 5f54c500 f   MFC42D:MFC42D.DLL
 0001:0004b506       ?DrawFocusRect@CDC@@QAEXPBUtagRECT@@@Z 5f54c506 f   MFC42D:MFC42D.DLL
 0001:0004b50c       ?GetTextMetricsA@CDC@@QBEHPAUtagTEXTMETRICA@@@Z 5f54c50c f   MFC42D:MFC42D.DLL
 0001:0004b512       ?InsertString@CComboBox@@QAEHHPBD@Z 5f54c512 f   MFC42D:MFC42D.DLL
 0001:0004b518       ?SetEditSel@CComboBox@@QAEHHH@Z 5f54c518 f   MFC42D:MFC42D.DLL
 0001:0004b51e       ?FindStringExact@CComboBox@@QBEHHPBD@Z 5f54c51e f   MFC42D:MFC42D.DLL
 0001:0004b524       ?CreateFontIndirectA@CFont@@QAEHPBUtagLOGFONTA@@@Z 5f54c524 f   MFC42D:MFC42D.DLL
 0001:0004b52a       ?DeleteObject@CGdiObject@@QAEHXZ 5f54c52a f   MFC42D:MFC42D.DLL
 0001:0004b530       ?GetTextExtent@CDC@@QBE?AVCSize@@PBDH@Z 5f54c530 f   MFC42D:MFC42D.DLL
 0001:0004b536       ?SetBkMode@CDC@@QAEHH@Z    5f54c536 f   MFC42D:MFC42D.DLL
 0001:0004b53c       ?SetCheck@CButton@@QAEXH@Z 5f54c53c f   MFC42D:MFC42D.DLL
 0001:0004b542       ?GetCheck@CButton@@QBEHXZ  5f54c542 f   MFC42D:MFC42D.DLL
 0001:0004b548       ?GetStatus@CFile@@SGHPBDAAUCFileStatus@@@Z 5f54c548 f   MFC42D:MFC42D.DLL
 0001:0004b54e       ??0CTime@@QAE@XZ           5f54c54e f   MFC42D:MFC42D.DLL
 0001:0004b554       ?GetPathName@CFileDialog@@QBE?AVCString@@XZ 5f54c554 f   MFC42D:MFC42D.DLL
 0001:0004b55a       ?DoModal@CFileDialog@@UAEHXZ 5f54c55a f   MFC42D:MFC42D.DLL
 0001:0004b560       ??0CFileDialog@@QAE@HPBD0K0PAVCWnd@@@Z 5f54c560 f   MFC42D:MFC42D.DLL
 0001:0004b566       ??0CMemFile@@QAE@I@Z       5f54c566 f   MFC42D:MFC42D.DLL
 0001:0004b56c       ___CxxFrameHandler         5f54c56c f   msvcrtd:MSVCRTD.dll
 0001:0004b580       __onexit                   5f54c580 f   msvcrtd:atonexit.obj
 0001:0004b5c0       _atexit                    5f54c5c0 f   msvcrtd:atonexit.obj
 0001:0004b5e0       ??_L@YGXPAXIHP6EX0@Z1@Z    5f54c5e0 f   msvcrtd:ehvecctr.obj
 0001:0004b680       ??_M@YGXPAXIHP6EX0@Z@Z     5f54c680 f   msvcrtd:ehvecdtr.obj
 0001:0004b730       ?__ArrayUnwind@@YGXPAXIHP6EX0@Z@Z 5f54c730 f   msvcrtd:ehvecdtr.obj
 0001:0004b7dc       _memmove                   5f54c7dc f   msvcrtd:MSVCRTD.dll
 0001:0004b7e2       __mbsnbcmp                 5f54c7e2 f   msvcrtd:MSVCRTD.dll
 0001:0004b7f0       ??0type_info@@AAE@ABV0@@Z  5f54c7f0 f   msvcrtd:ti_inst.obj
 0001:0004b810       ??_Etype_info@@UAEPAXI@Z   5f54c810 f i msvcrtd:ti_inst.obj
 0001:0004b810       ??_Gtype_info@@UAEPAXI@Z   5f54c810 f i msvcrtd:ti_inst.obj
 0001:0004b840       ??4type_info@@AAEAAV0@ABV0@@Z 5f54c840 f   msvcrtd:ti_inst.obj
 0001:0004b850       __chkstk                   5f54c850 f   msvcrtd:chkstk.obj
 0001:0004b850       __alloca_probe             5f54c850 f   msvcrtd:chkstk.obj
 0001:0004b880       _atol                      5f54c880 f   msvcrtd:MSVCRTD.dll
 0001:0004b886       __mbsinc                   5f54c886 f   msvcrtd:MSVCRTD.dll
 0001:0004b88c       _memcmp                    5f54c88c f   msvcrtd:MSVCRTD.dll
 0001:0004b892       __CrtDbgReport             5f54c892 f   msvcrtd:MSVCRTD.dll
 0001:0004b898       __CxxThrowException@8      5f54c898 f   msvcrtd:MSVCRTD.dll
 0001:0004b89e       _memcpy                    5f54c89e f   msvcrtd:MSVCRTD.dll
 0001:0004b8a4       _wcslen                    5f54c8a4 f   msvcrtd:MSVCRTD.dll
 0001:0004b8aa       _memset                    5f54c8aa f   msvcrtd:MSVCRTD.dll
 0001:0004b8b0       __purecall                 5f54c8b0 f   msvcrtd:MSVCRTD.dll
 0001:0004b8b6       _free                      5f54c8b6 f   msvcrtd:MSVCRTD.dll
 0001:0004b8bc       __strdup                   5f54c8bc f   msvcrtd:MSVCRTD.dll
 0001:0004b8c2       _realloc                   5f54c8c2 f   msvcrtd:MSVCRTD.dll
 0001:0004b8c8       __mbschr                   5f54c8c8 f   msvcrtd:MSVCRTD.dll
 0001:0004b8ce       __ftol                     5f54c8ce f   msvcrtd:MSVCRTD.dll
 0001:0004b8d4       _labs                      5f54c8d4 f   msvcrtd:MSVCRTD.dll
 0001:0004b8da       _floor                     5f54c8da f   msvcrtd:MSVCRTD.dll
 0001:0004b8e0       _fabs                      5f54c8e0 f   msvcrtd:MSVCRTD.dll
 0001:0004b8e6       _ceil                      5f54c8e6 f   msvcrtd:MSVCRTD.dll
 0001:0004b8ec       _time                      5f54c8ec f   msvcrtd:MSVCRTD.dll
 0001:0004b8f2       _localtime                 5f54c8f2 f   msvcrtd:MSVCRTD.dll
 0001:0004b8f8       _strftime                  5f54c8f8 f   msvcrtd:MSVCRTD.dll
 0001:0004b8fe       _modf                      5f54c8fe f   msvcrtd:MSVCRTD.dll
 0001:0004b904       __itoa                     5f54c904 f   msvcrtd:MSVCRTD.dll
 0001:0004b90a       _swprintf                  5f54c90a f   msvcrtd:MSVCRTD.dll
 0001:0004b910       _malloc                    5f54c910 f   msvcrtd:MSVCRTD.dll
 0001:0004b916       _strtoul                   5f54c916 f   msvcrtd:MSVCRTD.dll
 0001:0004b91c       _strtol                    5f54c91c f   msvcrtd:MSVCRTD.dll
 0001:0004b922       __ismbcdigit               5f54c922 f   msvcrtd:MSVCRTD.dll
 0001:0004b928       __ismbcspace               5f54c928 f   msvcrtd:MSVCRTD.dll
 0001:0004b92e       __ultoa                    5f54c92e f   msvcrtd:MSVCRTD.dll
 0001:0004b934       __ltoa                     5f54c934 f   msvcrtd:MSVCRTD.dll
 0001:0004b93a       __vsnprintf                5f54c93a f   msvcrtd:MSVCRTD.dll
 0001:0004b940       _wcscpy                    5f54c940 f   msvcrtd:MSVCRTD.dll
 0001:0004b946       _wcsncpy                   5f54c946 f   msvcrtd:MSVCRTD.dll
 0001:0004b94c       __mbsrchr                  5f54c94c f   msvcrtd:MSVCRTD.dll
 0001:0004b960       __CRT_INIT@12              5f54c960 f   msvcrtd:crtdll.obj
 0001:0004ba70       __DllMainCRTStartup@12     5f54ca70 f   msvcrtd:crtdll.obj
 0001:0004bb64       ___dllonexit               5f54cb64 f   msvcrtd:MSVCRTD.dll
 0001:0004bb6a       __except_handler3          5f54cb6a f   msvcrtd:MSVCRTD.dll
 0001:0004bb70       ?terminate@@YAXXZ          5f54cb70 f   msvcrtd:MSVCRTD.dll
 0001:0004bb76       ??1type_info@@UAE@XZ       5f54cb76 f   msvcrtd:MSVCRTD.dll
 0001:0004bb7c       __free_dbg                 5f54cb7c f   msvcrtd:MSVCRTD.dll
 0001:0004bb82       __initterm                 5f54cb82 f   msvcrtd:MSVCRTD.dll
 0001:0004bb88       __malloc_dbg               5f54cb88 f   msvcrtd:MSVCRTD.dll
 0001:0004bb8e       _FreeLibrary@4             5f54cb8e f   kernel32:KERNEL32.dll
 0001:0004bb94       _GetModuleHandleA@4        5f54cb94 f   kernel32:KERNEL32.dll
 0001:0004bb9a       _LocalFree@4               5f54cb9a f   kernel32:KERNEL32.dll
 0001:0004bba0       _LocalAlloc@8              5f54cba0 f   kernel32:KERNEL32.dll
 0001:0004bba6       _LoadLibraryA@4            5f54cba6 f   kernel32:KERNEL32.dll
 0001:0004bbac       _GetTickCount@0            5f54cbac f   kernel32:KERNEL32.dll
 0001:0004bbb2       _lstrlenA@4                5f54cbb2 f   kernel32:KERNEL32.dll
 0001:0004bbb8       _lstrlenW@4                5f54cbb8 f   kernel32:KERNEL32.dll
 0001:0004bbbe       _MultiByteToWideChar@24    5f54cbbe f   kernel32:KERNEL32.dll
 0001:0004bbc4       _WideCharToMultiByte@32    5f54cbc4 f   kernel32:KERNEL32.dll
 0001:0004bbca       _GlobalFree@4              5f54cbca f   kernel32:KERNEL32.dll
 0001:0004bbd0       _GlobalUnlock@4            5f54cbd0 f   kernel32:KERNEL32.dll
 0001:0004bbd6       _GlobalLock@4              5f54cbd6 f   kernel32:KERNEL32.dll
 0001:0004bbdc       _GlobalAlloc@8             5f54cbdc f   kernel32:KERNEL32.dll
 0001:0004bbe2       _InterlockedDecrement@4    5f54cbe2 f   kernel32:KERNEL32.dll
 0001:0004bbe8       _InterlockedIncrement@4    5f54cbe8 f   kernel32:KERNEL32.dll
 0001:0004bbee       _lstrcmpiA@8               5f54cbee f   kernel32:KERNEL32.dll
 0001:0004bbf4       _lstrcpynA@12              5f54cbf4 f   kernel32:KERNEL32.dll
 0001:0004bbfa       _FileTimeToSystemTime@8    5f54cbfa f   kernel32:KERNEL32.dll
 0001:0004bc00       _GetLastError@0            5f54cc00 f   kernel32:KERNEL32.dll
 0001:0004bc06       _FileTimeToLocalFileTime@8 5f54cc06 f   kernel32:KERNEL32.dll
 0001:0004bc0c       _GetProfileIntA@12         5f54cc0c f   kernel32:KERNEL32.dll
 0001:0004bc12       _GetCurrentThreadId@0      5f54cc12 f   kernel32:KERNEL32.dll
 0001:0004bc18       _lstrcmpA@8                5f54cc18 f   kernel32:KERNEL32.dll
 0001:0004bc1e       _FormatMessageA@28         5f54cc1e f   kernel32:KERNEL32.dll
 0001:0004bc24       _GlobalSize@4              5f54cc24 f   kernel32:KERNEL32.dll
 0001:0004bc2a       _CopyFileA@12              5f54cc2a f   kernel32:KERNEL32.dll
 0001:0004bc30       _MulDiv@12                 5f54cc30 f   kernel32:KERNEL32.dll
 0001:0004bc36       _lstrcatA@8                5f54cc36 f   kernel32:KERNEL32.dll
 0001:0004bc3c       _GetModuleFileNameA@12     5f54cc3c f   kernel32:KERNEL32.dll
 0001:0004bc42       _FreeResource@4            5f54cc42 f   kernel32:KERNEL32.dll
 0001:0004bc48       _LockResource@4            5f54cc48 f   kernel32:KERNEL32.dll
 0001:0004bc4e       _LoadResource@8            5f54cc4e f   kernel32:KERNEL32.dll
 0001:0004bc54       _FindResourceA@12          5f54cc54 f   kernel32:KERNEL32.dll
 0001:0004bc5a       _GetThreadLocale@0         5f54cc5a f   kernel32:KERNEL32.dll
 0001:0004bc60       _OutputDebugStringA@4      5f54cc60 f   kernel32:KERNEL32.dll
 0001:0004bc66       _lstrcpyW@8                5f54cc66 f   kernel32:KERNEL32.dll
 0001:0004bc6c       _GetUserDefaultLCID@0      5f54cc6c f   kernel32:KERNEL32.dll
 0001:0004bc72       _IsDBCSLeadByte@4          5f54cc72 f   kernel32:KERNEL32.dll
 0001:0004bc78       _lstrcpyA@8                5f54cc78 f   kernel32:KERNEL32.dll
 0001:0004bc7e       _GetVersion@0              5f54cc7e f   kernel32:KERNEL32.dll
 0001:0004bc84       _CopyMetaFileA@8           5f54cc84 f   gdi32:GDI32.dll
 0001:0004bc8a       _CreateDCA@16              5f54cc8a f   gdi32:GDI32.dll
 0001:0004bc90       _GetDeviceCaps@8           5f54cc90 f   gdi32:GDI32.dll
 0001:0004bc96       _DeleteMetaFile@4          5f54cc96 f   gdi32:GDI32.dll
 0001:0004bc9c       _DeleteDC@4                5f54cc9c f   gdi32:GDI32.dll
 0001:0004bca2       _ScaleWindowExtEx@24       5f54cca2 f   gdi32:GDI32.dll
 0001:0004bca8       _DPtoLP@12                 5f54cca8 f   gdi32:GDI32.dll
 0001:0004bcae       _LPtoDP@12                 5f54ccae f   gdi32:GDI32.dll
 0001:0004bcb4       _SetMapMode@8              5f54ccb4 f   gdi32:GDI32.dll
 0001:0004bcba       _SelectObject@8            5f54ccba f   gdi32:GDI32.dll
 0001:0004bcc0       _GetPaletteEntries@16      5f54ccc0 f   gdi32:GDI32.dll
 0001:0004bcc6       _CreatePalette@4           5f54ccc6 f   gdi32:GDI32.dll
 0001:0004bccc       _EnumFontFamiliesA@16      5f54cccc f   gdi32:GDI32.dll
 0001:0004bcd2       _RegisterClipboardFormatA@4 5f54ccd2 f   user32:USER32.dll
 0001:0004bcd8       _wsprintfA                 5f54ccd8 f   user32:USER32.dll
 0001:0004bcde       _CopyAcceleratorTableA@12  5f54ccde f   user32:USER32.dll
 0001:0004bce4       _GetActiveWindow@0         5f54cce4 f   user32:USER32.dll
 0001:0004bcea       _IsWindow@4                5f54ccea f   user32:USER32.dll
 0001:0004bcf0       _CopyRect@8                5f54ccf0 f   user32:USER32.dll
 0001:0004bcf6       _IsClipboardFormatAvailable@4 5f54ccf6 f   user32:USER32.dll
 0001:0004bcfc       _SendMessageA@16           5f54ccfc f   user32:USER32.dll
 0001:0004bd02       _EnableWindow@8            5f54cd02 f   user32:USER32.dll
 0001:0004bd08       _GetWindowTextA@12         5f54cd08 f   user32:USER32.dll
 0001:0004bd0e       _GetWindowTextLengthA@4    5f54cd0e f   user32:USER32.dll
 0001:0004bd14       _InSendMessage@0           5f54cd14 f   user32:USER32.dll
 0001:0004bd1a       _ReleaseCapture@0          5f54cd1a f   user32:USER32.dll
 0001:0004bd20       _PeekMessageA@20           5f54cd20 f   user32:USER32.dll
 0001:0004bd26       _GetKeyState@4             5f54cd26 f   user32:USER32.dll
 0001:0004bd2c       _GetCursorPos@4            5f54cd2c f   user32:USER32.dll
 0001:0004bd32       _DispatchMessageA@4        5f54cd32 f   user32:USER32.dll
 0001:0004bd38       _PostThreadMessageA@16     5f54cd38 f   user32:USER32.dll
 0001:0004bd3e       _DestroyMenu@4             5f54cd3e f   user32:USER32.dll
 0001:0004bd44       _CreateMenu@0              5f54cd44 f   user32:USER32.dll
 0001:0004bd4a       _IsMenu@4                  5f54cd4a f   user32:USER32.dll
 0001:0004bd50       _GetMenuItemID@8           5f54cd50 f   user32:USER32.dll
 0001:0004bd56       _InsertMenuA@20            5f54cd56 f   user32:USER32.dll
 0001:0004bd5c       _AppendMenuA@16            5f54cd5c f   user32:USER32.dll
 0001:0004bd62       _GetMenuStringA@20         5f54cd62 f   user32:USER32.dll
 0001:0004bd68       _GetMenuState@12           5f54cd68 f   user32:USER32.dll
 0001:0004bd6e       _GetSubMenu@8              5f54cd6e f   user32:USER32.dll
 0001:0004bd74       _GetMenuItemCount@4        5f54cd74 f   user32:USER32.dll
 0001:0004bd7a       _RemoveMenu@12             5f54cd7a f   user32:USER32.dll
 0001:0004bd80       _ReleaseDC@8               5f54cd80 f   user32:USER32.dll
 0001:0004bd86       _WindowFromDC@4            5f54cd86 f   user32:USER32.dll
 0001:0004bd8c       _GetDC@4                   5f54cd8c f   user32:USER32.dll
 0001:0004bd92       _IsRectEmpty@4             5f54cd92 f   user32:USER32.dll
 0001:0004bd98       _SetScrollRange@20         5f54cd98 f   user32:USER32.dll
 0001:0004bd9e       _SetFocus@4                5f54cd9e f   user32:USER32.dll
 0001:0004bda4       _GetParent@4               5f54cda4 f   user32:USER32.dll
 0001:0004bdaa       _GetFocus@0                5f54cdaa f   user32:USER32.dll
 0001:0004bdb0       _DestroyIcon@4             5f54cdb0 f   user32:USER32.dll
 0001:0004bdb6       _RegisterWindowMessageA@4  5f54cdb6 f   user32:USER32.dll
 0001:0004bdbc       _CountClipboardFormats@0   5f54cdbc f   user32:USER32.dll
 0001:0004bdc2       _GetSystemMetrics@4        5f54cdc2 f   user32:USER32.dll
 0001:0004bdc8       _MessageBeep@4             5f54cdc8 f   user32:USER32.dll
 0001:0004bdce       _GetWindowLongA@8          5f54cdce f   user32:USER32.dll
 0001:0004bdd4       _AdjustWindowRectEx@16     5f54cdd4 f   user32:USER32.dll
 0001:0004bdda       _SetWindowContextHelpId@8  5f54cdda f   user32:USER32.dll
 0001:0004bde0       _GetWindow@8               5f54cde0 f   user32:USER32.dll
 0001:0004bde6       _SetWindowPos@28           5f54cde6 f   user32:USER32.dll
 0001:0004bdec       _MapDialogRect@8           5f54cdec f   user32:USER32.dll
 0001:0004bdf2       _GetDlgItem@8              5f54cdf2 f   user32:USER32.dll
 0001:0004bdf8       _CharNextA@4               5f54cdf8 f   user32:USER32.dll
 0001:0004bdfe       _IsWindowVisible@4         5f54cdfe f   user32:USER32.dll
 0001:0004be04       _IsDialogMessageA@8        5f54ce04 f   user32:USER32.dll
 0001:0004be0a       _GetDlgCtrlID@4            5f54ce0a f   user32:USER32.dll
 0001:0004be10       _ClipCursor@4              5f54ce10 f   user32:USER32.dll
 0001:0004be16       _InflateRect@12            5f54ce16 f   user32:USER32.dll
 0001:0004be1c       _DestroyWindow@4           5f54ce1c f   user32:USER32.dll
 0001:0004be22       _SetWindowLongA@12         5f54ce22 f   user32:USER32.dll
 0001:0004be28       _DefWindowProcA@16         5f54ce28 f   user32:USER32.dll
 0001:0004be2e       _CallWindowProcA@20        5f54ce2e f   user32:USER32.dll
 0001:0004be34       _SetParent@8               5f54ce34 f   user32:USER32.dll
 0001:0004be3a       _DrawEdge@16               5f54ce3a f   user32:USER32.dll
 0001:0004be40       _ShowWindow@8              5f54ce40 f   user32:USER32.dll
 0001:0004be46       _GetWindowRect@8           5f54ce46 f   user32:USER32.dll
 0001:0004be4c       _GetMenu@4                 5f54ce4c f   user32:USER32.dll
 0001:0004be52       _GetDesktopWindow@0        5f54ce52 f   user32:USER32.dll
 0001:0004be58       _PostMessageA@16           5f54ce58 f   user32:USER32.dll
 0001:0004be5e       _GetClassNameA@12          5f54ce5e f   user32:USER32.dll
 0001:0004be64       _IsChild@8                 5f54ce64 f   user32:USER32.dll
 0001:0004be6a       _IntersectRect@12          5f54ce6a f   user32:USER32.dll
 0001:0004be70       _ScreenToClient@8          5f54ce70 f   user32:USER32.dll
 0001:0004be76       _MessageBoxA@16            5f54ce76 f   user32:USER32.dll
 0001:0004be7c       _EnumChildWindows@12       5f54ce7c f   user32:USER32.dll
 0001:0004be82       _LockWindowUpdate@4        5f54ce82 f   user32:USER32.dll
 0001:0004be88       _GetSysColor@4             5f54ce88 f   user32:USER32.dll
 0001:0004be8e       _SetCursor@4               5f54ce8e f   user32:USER32.dll
 0001:0004be94       _LoadCursorA@8             5f54ce94 f   user32:USER32.dll
 0001:0004be9a       _PtInRect@12               5f54ce9a f   user32:USER32.dll
 0001:0004bea0       _SetRectEmpty@4            5f54cea0 f   user32:USER32.dll
 0001:0004bea6       _OffsetRect@12             5f54cea6 f   user32:USER32.dll
 0001:0004beac       _GetDialogBaseUnits@0      5f54ceac f   user32:USER32.dll
 0001:0004beb2       __imp_load__OleCreateFontIndirect@12 5f54ceb2     olepro32:OLEPRO32.DLL
 0001:0004bebe       __tailMerge_OLEPRO32       5f54cebe     olepro32:OLEPRO32.DLL
 0001:0004becc       _OleCreateFontIndirect@12  5f54cecc     olepro32:OLEPRO32.DLL
 0001:0004bed2       __imp_load__OleCreatePropertyFrame@44 5f54ced2     olepro32:OLEPRO32.DLL
 0001:0004bede       _OleCreatePropertyFrame@44 5f54cede     olepro32:OLEPRO32.DLL
 0001:0004bee4       __imp_load__OleTranslateColor@12 5f54cee4     olepro32:OLEPRO32.DLL
 0001:0004bef0       _OleTranslateColor@12      5f54cef0     olepro32:OLEPRO32.DLL
 0001:0004bef6       __imp_load__OleCreatePictureIndirect@16 5f54cef6     olepro32:OLEPRO32.DLL
 0001:0004bf02       _OleCreatePictureIndirect@16 5f54cf02     olepro32:OLEPRO32.DLL
 0001:0004bf08       __imp_load__OleLoadPicture@20 5f54cf08     olepro32:OLEPRO32.DLL
 0001:0004bf14       _OleLoadPicture@20         5f54cf14     olepro32:OLEPRO32.DLL
 0001:0004bf1a       __imp_load__RegCloseKey@4  5f54cf1a     advapi32:ADVAPI32.dll
 0001:0004bf26       __tailMerge_ADVAPI32       5f54cf26     advapi32:ADVAPI32.dll
 0001:0004bf34       _RegCloseKey@4             5f54cf34     advapi32:ADVAPI32.dll
 0001:0004bf3a       __imp_load__RegQueryValueExA@24 5f54cf3a     advapi32:ADVAPI32.dll
 0001:0004bf46       _RegQueryValueExA@24       5f54cf46     advapi32:ADVAPI32.dll
 0001:0004bf4c       __imp_load__RegOpenKeyExA@20 5f54cf4c     advapi32:ADVAPI32.dll
 0001:0004bf58       _RegOpenKeyExA@20          5f54cf58     advapi32:ADVAPI32.dll
 0001:0004bf5e       __imp_load__RegEnumKeyA@16 5f54cf5e     advapi32:ADVAPI32.dll
 0001:0004bf6a       _RegEnumKeyA@16            5f54cf6a     advapi32:ADVAPI32.dll
 0001:0004bf70       __imp_load__RegSetValueA@20 5f54cf70     advapi32:ADVAPI32.dll
 0001:0004bf7c       _RegSetValueA@20           5f54cf7c     advapi32:ADVAPI32.dll
 0001:0004bf82       __imp_load__RegOpenKeyA@12 5f54cf82     advapi32:ADVAPI32.dll
 0001:0004bf8e       _RegOpenKeyA@12            5f54cf8e     advapi32:ADVAPI32.dll
 0001:0004bf94       __imp_load__RegQueryValueA@16 5f54cf94     advapi32:ADVAPI32.dll
 0001:0004bfa0       _RegQueryValueA@16         5f54cfa0     advapi32:ADVAPI32.dll
 0001:0004bfa6       __imp_load__RegSetValueExA@24 5f54cfa6     advapi32:ADVAPI32.dll
 0001:0004bfb2       _RegSetValueExA@24         5f54cfb2     advapi32:ADVAPI32.dll
 0001:0004bfb8       __imp_load__RegCreateKeyA@12 5f54cfb8     advapi32:ADVAPI32.dll
 0001:0004bfc4       _RegCreateKeyA@12          5f54cfc4     advapi32:ADVAPI32.dll
 0001:0004bfca       __imp_load__RegDeleteKeyA@8 5f54cfca     advapi32:ADVAPI32.dll
 0001:0004bfd6       _RegDeleteKeyA@8           5f54cfd6     advapi32:ADVAPI32.dll
 0001:0004bfdc       __imp_load__OleInitialize@4 5f54cfdc     ole32:ole32.dll
 0001:0004bfe8       __tailMerge_ole32          5f54cfe8     ole32:ole32.dll
 0001:0004bff6       _OleInitialize@4           5f54cff6     ole32:ole32.dll
 0001:0004bffc       __imp_load__OleUninitialize@0 5f54cffc     ole32:ole32.dll
 0001:0004c008       _OleUninitialize@0         5f54d008     ole32:ole32.dll
 0001:0004c00e       __imp_load__CoFreeUnusedLibraries@0 5f54d00e     ole32:ole32.dll
 0001:0004c01a       _CoFreeUnusedLibraries@0   5f54d01a     ole32:ole32.dll
 0001:0004c020       __imp_load__OleLockRunning@12 5f54d020     ole32:ole32.dll
 0001:0004c02c       _OleLockRunning@12         5f54d02c     ole32:ole32.dll
 0001:0004c032       __imp_load__CoTaskMemFree@4 5f54d032     ole32:ole32.dll
 0001:0004c03e       _CoTaskMemFree@4           5f54d03e     ole32:ole32.dll
 0001:0004c044       __imp_load__StringFromCLSID@8 5f54d044     ole32:ole32.dll
 0001:0004c050       _StringFromCLSID@8         5f54d050     ole32:ole32.dll
 0001:0004c056       __imp_load__OleSetContainedObject@8 5f54d056     ole32:ole32.dll
 0001:0004c062       _OleSetContainedObject@8   5f54d062     ole32:ole32.dll
 0001:0004c068       __imp_load__OleCreateFromData@28 5f54d068     ole32:ole32.dll
 0001:0004c074       _OleCreateFromData@28      5f54d074     ole32:ole32.dll
 0001:0004c07a       __imp_load__OleCreateLinkFromData@28 5f54d07a     ole32:ole32.dll
 0001:0004c086       _OleCreateLinkFromData@28  5f54d086     ole32:ole32.dll
 0001:0004c08c       __imp_load__OleCreateStaticFromData@28 5f54d08c     ole32:ole32.dll
 0001:0004c098       _OleCreateStaticFromData@28 5f54d098     ole32:ole32.dll
 0001:0004c09e       __imp_load__OleCreateFromFile@32 5f54d09e     ole32:ole32.dll
 0001:0004c0aa       _OleCreateFromFile@32      5f54d0aa     ole32:ole32.dll
 0001:0004c0b0       __imp_load__OleCreateLinkToFile@28 5f54d0b0     ole32:ole32.dll
 0001:0004c0bc       _OleCreateLinkToFile@28    5f54d0bc     ole32:ole32.dll
 0001:0004c0c2       __imp_load__OleCreate@28   5f54d0c2     ole32:ole32.dll
 0001:0004c0ce       _OleCreate@28              5f54d0ce     ole32:ole32.dll
 0001:0004c0d4       __imp_load__OleLoad@16     5f54d0d4     ole32:ole32.dll
 0001:0004c0e0       _OleLoad@16                5f54d0e0     ole32:ole32.dll
 0001:0004c0e6       __imp_load__OleSave@12     5f54d0e6     ole32:ole32.dll
 0001:0004c0f2       _OleSave@12                5f54d0f2     ole32:ole32.dll
 0001:0004c0f8       __imp_load__StgCreateDocfileOnILockBytes@16 5f54d0f8     ole32:ole32.dll
 0001:0004c104       _StgCreateDocfileOnILockBytes@16 5f54d104     ole32:ole32.dll
 0001:0004c10a       __imp_load__CreateILockBytesOnHGlobal@12 5f54d10a     ole32:ole32.dll
 0001:0004c116       _CreateILockBytesOnHGlobal@12 5f54d116     ole32:ole32.dll
 0001:0004c11c       __imp_load__StgOpenStorageOnILockBytes@24 5f54d11c     ole32:ole32.dll
 0001:0004c128       _StgOpenStorageOnILockBytes@24 5f54d128     ole32:ole32.dll
 0001:0004c12e       __imp_load__StgIsStorageILockBytes@4 5f54d12e     ole32:ole32.dll
 0001:0004c13a       _StgIsStorageILockBytes@4  5f54d13a     ole32:ole32.dll
 0001:0004c140       __imp_load__GetHGlobalFromILockBytes@8 5f54d140     ole32:ole32.dll
 0001:0004c14c       _GetHGlobalFromILockBytes@8 5f54d14c     ole32:ole32.dll
 0001:0004c152       __imp_load__ReleaseStgMedium@4 5f54d152     ole32:ole32.dll
 0001:0004c15e       _ReleaseStgMedium@4        5f54d15e     ole32:ole32.dll
 0001:0004c164       __imp_load__OleGetIconOfClass@12 5f54d164     ole32:ole32.dll
 0001:0004c170       _OleGetIconOfClass@12      5f54d170     ole32:ole32.dll
 0001:0004c176       __imp_load__WriteClassStm@8 5f54d176     ole32:ole32.dll
 0001:0004c182       _WriteClassStm@8           5f54d182     ole32:ole32.dll
 0001:0004c188       __imp_load__OleSaveToStream@8 5f54d188     ole32:ole32.dll
 0001:0004c194       _OleSaveToStream@8         5f54d194     ole32:ole32.dll
 0001:0004c19a       __imp_load__CreateStreamOnHGlobal@12 5f54d19a     ole32:ole32.dll
 0001:0004c1a6       _CreateStreamOnHGlobal@12  5f54d1a6     ole32:ole32.dll
 0001:0004c1ac       __imp_load__CreateGenericComposite@12 5f54d1ac     ole32:ole32.dll
 0001:0004c1b8       _CreateGenericComposite@12 5f54d1b8     ole32:ole32.dll
 0001:0004c1be       __imp_load__CreateItemMoniker@12 5f54d1be     ole32:ole32.dll
 0001:0004c1ca       _CreateItemMoniker@12      5f54d1ca     ole32:ole32.dll
 0001:0004c1d0       __imp_load__OleIsRunning@4 5f54d1d0     ole32:ole32.dll
 0001:0004c1dc       _OleIsRunning@4            5f54d1dc     ole32:ole32.dll
 0001:0004c1e2       __imp_load__OleSetMenuDescriptor@20 5f54d1e2     ole32:ole32.dll
 0001:0004c1ee       _OleSetMenuDescriptor@20   5f54d1ee     ole32:ole32.dll
 0001:0004c1f4       __imp_load__OleQueryCreateFromData@4 5f54d1f4     ole32:ole32.dll
 0001:0004c200       _OleQueryCreateFromData@4  5f54d200     ole32:ole32.dll
 0001:0004c206       __imp_load__OleQueryLinkFromData@4 5f54d206     ole32:ole32.dll
 0001:0004c212       _OleQueryLinkFromData@4    5f54d212     ole32:ole32.dll
 0001:0004c218       __imp_load__OleRun@4       5f54d218     ole32:ole32.dll
 0001:0004c224       _OleRun@4                  5f54d224     ole32:ole32.dll
 0001:0004c22a       __imp_load__CoTaskMemAlloc@4 5f54d22a     ole32:ole32.dll
 0001:0004c236       _CoTaskMemAlloc@4          5f54d236     ole32:ole32.dll
 0001:0004c23c       __imp_load__OleGetClipboard@4 5f54d23c     ole32:ole32.dll
 0001:0004c248       _OleGetClipboard@4         5f54d248     ole32:ole32.dll
 0001:0004c24e       __imp_load__OleIsCurrentClipboard@4 5f54d24e     ole32:ole32.dll
 0001:0004c25a       _OleIsCurrentClipboard@4   5f54d25a     ole32:ole32.dll
 0001:0004c260       __imp_load__OleSetClipboard@4 5f54d260     ole32:ole32.dll
 0001:0004c26c       _OleSetClipboard@4         5f54d26c     ole32:ole32.dll
 0001:0004c272       __imp_load__OleFlushClipboard@0 5f54d272     ole32:ole32.dll
 0001:0004c27e       _OleFlushClipboard@0       5f54d27e     ole32:ole32.dll
 0001:0004c284       __imp_load__CLSIDFromProgID@8 5f54d284     ole32:ole32.dll
 0001:0004c290       _CLSIDFromProgID@8         5f54d290     ole32:ole32.dll
 0001:0004c296       __imp_load__CLSIDFromString@8 5f54d296     ole32:ole32.dll
 0001:0004c2a2       _CLSIDFromString@8         5f54d2a2     ole32:ole32.dll
 0001:0004c2a8       __imp_load__CoCreateInstance@20 5f54d2a8     ole32:ole32.dll
 0001:0004c2b4       _CoCreateInstance@20       5f54d2b4     ole32:ole32.dll
 0001:0004c2ba       __imp_load__CreateBindCtx@8 5f54d2ba     ole32:ole32.dll
 0001:0004c2c6       _CreateBindCtx@8           5f54d2c6     ole32:ole32.dll
 0001:0004c2cc       __imp_load__CreateFileMoniker@8 5f54d2cc     ole32:ole32.dll
 0001:0004c2d8       _CreateFileMoniker@8       5f54d2d8     ole32:ole32.dll
 0001:0004c2de       __imp_load__GetClassFile@8 5f54d2de     ole32:ole32.dll
 0001:0004c2ea       _GetClassFile@8            5f54d2ea     ole32:ole32.dll
 0001:0004c2f0       __imp_load__OleRegGetUserType@12 5f54d2f0     ole32:ole32.dll
 0001:0004c2fc       _OleRegGetUserType@12      5f54d2fc     ole32:ole32.dll
 0001:0004c302       __imp_load__ReadFmtUserTypeStg@12 5f54d302     ole32:ole32.dll
 0001:0004c30e       _ReadFmtUserTypeStg@12     5f54d30e     ole32:ole32.dll
 0001:0004c314       __imp_load__ReadClassStg@8 5f54d314     ole32:ole32.dll
 0001:0004c320       _ReadClassStg@8            5f54d320     ole32:ole32.dll
 0001:0004c326       __imp_load__CoGetMalloc@8  5f54d326     ole32:ole32.dll
 0001:0004c332       _CoGetMalloc@8             5f54d332     ole32:ole32.dll
 0001:0004c338       __imp_load__StgCreateDocfile@16 5f54d338     ole32:ole32.dll
 0001:0004c344       _StgCreateDocfile@16       5f54d344     ole32:ole32.dll
 0001:0004c34a       __imp_load__StgOpenStorage@24 5f54d34a     ole32:ole32.dll
 0001:0004c356       _StgOpenStorage@24         5f54d356     ole32:ole32.dll
 0001:0004c35c       __imp_load__StgIsStorageFile@4 5f54d35c     ole32:ole32.dll
 0001:0004c368       _StgIsStorageFile@4        5f54d368     ole32:ole32.dll
 0001:0004c36e       __imp_load__DoDragDrop@16  5f54d36e     ole32:ole32.dll
 0001:0004c37a       _DoDragDrop@16             5f54d37a     ole32:ole32.dll
 0001:0004c380       __imp_load__RegisterDragDrop@8 5f54d380     ole32:ole32.dll
 0001:0004c38c       _RegisterDragDrop@8        5f54d38c     ole32:ole32.dll
 0001:0004c392       __imp_load__CoLockObjectExternal@12 5f54d392     ole32:ole32.dll
 0001:0004c39e       _CoLockObjectExternal@12   5f54d39e     ole32:ole32.dll
 0001:0004c3a4       __imp_load__RevokeDragDrop@4 5f54d3a4     ole32:ole32.dll
 0001:0004c3b0       _RevokeDragDrop@4          5f54d3b0     ole32:ole32.dll
 0001:0004c3b6       __imp_load__CoRegisterMessageFilter@8 5f54d3b6     ole32:ole32.dll
 0001:0004c3c2       _CoRegisterMessageFilter@8 5f54d3c2     ole32:ole32.dll
 0001:0004c3c8       __imp_load__CoRegisterClassObject@20 5f54d3c8     ole32:ole32.dll
 0001:0004c3d4       _CoRegisterClassObject@20  5f54d3d4     ole32:ole32.dll
 0001:0004c3da       __imp_load__CoRevokeClassObject@4 5f54d3da     ole32:ole32.dll
 0001:0004c3e6       _CoRevokeClassObject@4     5f54d3e6     ole32:ole32.dll
 0001:0004c3ec       __imp_load__OleTranslateAccelerator@12 5f54d3ec     ole32:ole32.dll
 0001:0004c3f8       _OleTranslateAccelerator@12 5f54d3f8     ole32:ole32.dll
 0001:0004c3fe       __imp_load__IsAccelerator@16 5f54d3fe     ole32:ole32.dll
 0001:0004c40a       _IsAccelerator@16          5f54d40a     ole32:ole32.dll
 0001:0004c410       __imp_load__OleCreateMenuDescriptor@8 5f54d410     ole32:ole32.dll
 0001:0004c41c       _OleCreateMenuDescriptor@8 5f54d41c     ole32:ole32.dll
 0001:0004c422       __imp_load__OleDestroyMenuDescriptor@4 5f54d422     ole32:ole32.dll
 0001:0004c42e       _OleDestroyMenuDescriptor@4 5f54d42e     ole32:ole32.dll
 0001:0004c434       __imp_load__GetRunningObjectTable@8 5f54d434     ole32:ole32.dll
 0001:0004c440       _GetRunningObjectTable@8   5f54d440     ole32:ole32.dll
 0001:0004c446       __imp_load__WriteClassStg@8 5f54d446     ole32:ole32.dll
 0001:0004c452       _WriteClassStg@8           5f54d452     ole32:ole32.dll
 0001:0004c458       __imp_load__OleDuplicateData@12 5f54d458     ole32:ole32.dll
 0001:0004c464       _OleDuplicateData@12       5f54d464     ole32:ole32.dll
 0001:0004c46a       __imp_load__SetConvertStg@8 5f54d46a     ole32:ole32.dll
 0001:0004c476       _SetConvertStg@8           5f54d476     ole32:ole32.dll
 0001:0004c47c       __imp_load__WriteFmtUserTypeStg@12 5f54d47c     ole32:ole32.dll
 0001:0004c488       _WriteFmtUserTypeStg@12    5f54d488     ole32:ole32.dll
 0001:0004c48e       __imp_load__CoTreatAsClass@8 5f54d48e     ole32:ole32.dll
 0001:0004c49a       _CoTreatAsClass@8          5f54d49a     ole32:ole32.dll
 0001:0004c4a0       __imp_load__CoDisconnectObject@8 5f54d4a0     ole32:ole32.dll
 0001:0004c4ac       _CoDisconnectObject@8      5f54d4ac     ole32:ole32.dll
 0001:0004c4b2       __imp_load__OleRegEnumVerbs@8 5f54d4b2     ole32:ole32.dll
 0001:0004c4be       _OleRegEnumVerbs@8         5f54d4be     ole32:ole32.dll
 0001:0004c4c4       __imp_load__OleRegGetMiscStatus@12 5f54d4c4     ole32:ole32.dll
 0001:0004c4d0       _OleRegGetMiscStatus@12    5f54d4d0     ole32:ole32.dll
 0001:0004c4d6       __imp_load__CreateOleAdviseHolder@4 5f54d4d6     ole32:ole32.dll
 0001:0004c4e2       _CreateOleAdviseHolder@4   5f54d4e2     ole32:ole32.dll
 0001:0004c4e8       __imp_load__CreateDataAdviseHolder@4 5f54d4e8     ole32:ole32.dll
 0001:0004c4f4       _CreateDataAdviseHolder@4  5f54d4f4     ole32:ole32.dll
 0001:0004c4fa       __imp_load__CoGetClassObject@20 5f54d4fa     ole32:ole32.dll
 0001:0004c506       _CoGetClassObject@20       5f54d506     ole32:ole32.dll
 0001:0004c50c       __imp_load__StringFromGUID2@12 5f54d50c     ole32:ole32.dll
 0001:0004c518       _StringFromGUID2@12        5f54d518     ole32:ole32.dll
 0001:0004c51e       __imp_load__CreateDataCache@16 5f54d51e     ole32:ole32.dll
 0001:0004c52a       _CreateDataCache@16        5f54d52a     ole32:ole32.dll
 0001:0004c530       __imp_load__ReadClassStm@8 5f54d530     ole32:ole32.dll
 0001:0004c53c       _ReadClassStm@8            5f54d53c     ole32:ole32.dll
 0001:0004c542       __imp_load__OleLoadFromStream@12 5f54d542     ole32:ole32.dll
 0001:0004c54e       _OleLoadFromStream@12      5f54d54e     ole32:ole32.dll
 0001:0004c554       __imp_load__SysStringLen@4 5f54d554     oleaut32:OLEAUT32.dll
 0001:0004c560       __tailMerge_OLEAUT32       5f54d560     oleaut32:OLEAUT32.dll
 0001:0004c56e       _SysStringLen@4            5f54d56e     oleaut32:OLEAUT32.dll
 0001:0004c574       __imp_load__SysAllocStringByteLen@8 5f54d574     oleaut32:OLEAUT32.dll
 0001:0004c580       _SysAllocStringByteLen@8   5f54d580     oleaut32:OLEAUT32.dll
 0001:0004c586       __imp_load__VariantCopy@8  5f54d586     oleaut32:OLEAUT32.dll
 0001:0004c592       _VariantCopy@8             5f54d592     oleaut32:OLEAUT32.dll
 0001:0004c598       __imp_load__VariantClear@4 5f54d598     oleaut32:OLEAUT32.dll
 0001:0004c5a4       _VariantClear@4            5f54d5a4     oleaut32:OLEAUT32.dll
 0001:0004c5aa       __imp_load__VariantChangeType@16 5f54d5aa     oleaut32:OLEAUT32.dll
 0001:0004c5b6       _VariantChangeType@16      5f54d5b6     oleaut32:OLEAUT32.dll
 0001:0004c5bc       __imp_load__SysAllocStringLen@8 5f54d5bc     oleaut32:OLEAUT32.dll
 0001:0004c5c8       _SysAllocStringLen@8       5f54d5c8     oleaut32:OLEAUT32.dll
 0001:0004c5ce       __imp_load__SysReAllocStringLen@12 5f54d5ce     oleaut32:OLEAUT32.dll
 0001:0004c5da       _SysReAllocStringLen@12    5f54d5da     oleaut32:OLEAUT32.dll
 0001:0004c5e0       __imp_load__SysFreeString@4 5f54d5e0     oleaut32:OLEAUT32.dll
 0001:0004c5ec       _SysFreeString@4           5f54d5ec     oleaut32:OLEAUT32.dll
 0001:0004c5f2       __imp_load__SysAllocString@4 5f54d5f2     oleaut32:OLEAUT32.dll
 0001:0004c5fe       _SysAllocString@4          5f54d5fe     oleaut32:OLEAUT32.dll
 0001:0004c604       __imp_load__SafeArrayUnaccessData@4 5f54d604     oleaut32:OLEAUT32.dll
 0001:0004c610       _SafeArrayUnaccessData@4   5f54d610     oleaut32:OLEAUT32.dll
 0001:0004c616       __imp_load__SafeArrayAccessData@8 5f54d616     oleaut32:OLEAUT32.dll
 0001:0004c622       _SafeArrayAccessData@8     5f54d622     oleaut32:OLEAUT32.dll
 0001:0004c628       __imp_load__SafeArrayGetUBound@12 5f54d628     oleaut32:OLEAUT32.dll
 0001:0004c634       _SafeArrayGetUBound@12     5f54d634     oleaut32:OLEAUT32.dll
 0001:0004c63a       __imp_load__SafeArrayGetLBound@12 5f54d63a     oleaut32:OLEAUT32.dll
 0001:0004c646       _SafeArrayGetLBound@12     5f54d646     oleaut32:OLEAUT32.dll
 0001:0004c64c       __imp_load__SafeArrayGetElemsize@4 5f54d64c     oleaut32:OLEAUT32.dll
 0001:0004c658       _SafeArrayGetElemsize@4    5f54d658     oleaut32:OLEAUT32.dll
 0001:0004c65e       __imp_load__SafeArrayGetDim@4 5f54d65e     oleaut32:OLEAUT32.dll
 0001:0004c66a       _SafeArrayGetDim@4         5f54d66a     oleaut32:OLEAUT32.dll
 0001:0004c670       __imp_load__SafeArrayRedim@8 5f54d670     oleaut32:OLEAUT32.dll
 0001:0004c67c       _SafeArrayRedim@8          5f54d67c     oleaut32:OLEAUT32.dll
 0001:0004c682       __imp_load__SafeArrayCreate@12 5f54d682     oleaut32:OLEAUT32.dll
 0001:0004c68e       _SafeArrayCreate@12        5f54d68e     oleaut32:OLEAUT32.dll
 0001:0004c694       __imp_load__SysStringByteLen@4 5f54d694     oleaut32:OLEAUT32.dll
 0001:0004c6a0       _SysStringByteLen@4        5f54d6a0     oleaut32:OLEAUT32.dll
 0001:0004c6a6       __imp_load__VarCyFromStr@16 5f54d6a6     oleaut32:OLEAUT32.dll
 0001:0004c6b2       _VarCyFromStr@16           5f54d6b2     oleaut32:OLEAUT32.dll
 0001:0004c6b8       __imp_load__VarBstrFromCy@20 5f54d6b8     oleaut32:OLEAUT32.dll
 0001:0004c6c4       _VarBstrFromCy@20          5f54d6c4     oleaut32:OLEAUT32.dll
 0001:0004c6ca       __imp_load__VarDateFromStr@16 5f54d6ca     oleaut32:OLEAUT32.dll
 0001:0004c6d6       _VarDateFromStr@16         5f54d6d6     oleaut32:OLEAUT32.dll
 0001:0004c6dc       __imp_load__VarBstrFromDate@20 5f54d6dc     oleaut32:OLEAUT32.dll
 0001:0004c6e8       _VarBstrFromDate@20        5f54d6e8     oleaut32:OLEAUT32.dll
 0001:0004c6ee       __imp_load__SafeArrayCopy@8 5f54d6ee     oleaut32:OLEAUT32.dll
 0001:0004c6fa       _SafeArrayCopy@8           5f54d6fa     oleaut32:OLEAUT32.dll
 0001:0004c700       __imp_load__SafeArrayAllocData@4 5f54d700     oleaut32:OLEAUT32.dll
 0001:0004c70c       _SafeArrayAllocData@4      5f54d70c     oleaut32:OLEAUT32.dll
 0001:0004c712       __imp_load__SafeArrayAllocDescriptor@8 5f54d712     oleaut32:OLEAUT32.dll
 0001:0004c71e       _SafeArrayAllocDescriptor@8 5f54d71e     oleaut32:OLEAUT32.dll
 0001:0004c724       __imp_load__SafeArrayGetElement@12 5f54d724     oleaut32:OLEAUT32.dll
 0001:0004c730       _SafeArrayGetElement@12    5f54d730     oleaut32:OLEAUT32.dll
 0001:0004c736       __imp_load__SafeArrayPtrOfIndex@12 5f54d736     oleaut32:OLEAUT32.dll
 0001:0004c742       _SafeArrayPtrOfIndex@12    5f54d742     oleaut32:OLEAUT32.dll
 0001:0004c748       __imp_load__SafeArrayPutElement@12 5f54d748     oleaut32:OLEAUT32.dll
 0001:0004c754       _SafeArrayPutElement@12    5f54d754     oleaut32:OLEAUT32.dll
 0001:0004c75a       __imp_load__SafeArrayLock@4 5f54d75a     oleaut32:OLEAUT32.dll
 0001:0004c766       _SafeArrayLock@4           5f54d766     oleaut32:OLEAUT32.dll
 0001:0004c76c       __imp_load__SafeArrayUnlock@4 5f54d76c     oleaut32:OLEAUT32.dll
 0001:0004c778       _SafeArrayUnlock@4         5f54d778     oleaut32:OLEAUT32.dll
 0001:0004c77e       __imp_load__SafeArrayDestroy@4 5f54d77e     oleaut32:OLEAUT32.dll
 0001:0004c78a       _SafeArrayDestroy@4        5f54d78a     oleaut32:OLEAUT32.dll
 0001:0004c790       __imp_load__SafeArrayDestroyData@4 5f54d790     oleaut32:OLEAUT32.dll
 0001:0004c79c       _SafeArrayDestroyData@4    5f54d79c     oleaut32:OLEAUT32.dll
 0001:0004c7a2       __imp_load__SafeArrayDestroyDescriptor@4 5f54d7a2     oleaut32:OLEAUT32.dll
 0001:0004c7ae       _SafeArrayDestroyDescriptor@4 5f54d7ae     oleaut32:OLEAUT32.dll
 0001:0004c7b4       __imp_load__SafeArrayCreateVector@12 5f54d7b4     oleaut32:OLEAUT32.dll
 0001:0004c7c0       _SafeArrayCreateVector@12  5f54d7c0     oleaut32:OLEAUT32.dll
 0001:0004c7c6       __imp_load__DosDateTimeToVariantTime@12 5f54d7c6     oleaut32:OLEAUT32.dll
 0001:0004c7d2       _DosDateTimeToVariantTime@12 5f54d7d2     oleaut32:OLEAUT32.dll
 0001:0004c7d8       __imp_load__LoadTypeLib@8  5f54d7d8     oleaut32:OLEAUT32.dll
 0001:0004c7e4       _LoadTypeLib@8             5f54d7e4     oleaut32:OLEAUT32.dll
 0001:0004c7ea       __imp_load__VariantTimeToSystemTime@12 5f54d7ea     oleaut32:OLEAUT32.dll
 0001:0004c7f6       _VariantTimeToSystemTime@12 5f54d7f6     oleaut32:OLEAUT32.dll
 0001:0004c7fc       __imp_load__RegisterTypeLib@12 5f54d7fc     oleaut32:OLEAUT32.dll
 0001:0004c808       _RegisterTypeLib@12        5f54d808     oleaut32:OLEAUT32.dll
 0001:0004c80e       __imp_load__LoadRegTypeLib@20 5f54d80e     oleaut32:OLEAUT32.dll
 0001:0004c81a       _LoadRegTypeLib@20         5f54d81a     oleaut32:OLEAUT32.dll
 0001:0004c820       __imp_load__OleUIInsertObjectA@4 5f54d820     oledlg:oledlg.dll
 0001:0004c82c       __tailMerge_oledlg         5f54d82c     oledlg:oledlg.dll
 0001:0004c83a       _OleUIInsertObjectA@4      5f54d83a     oledlg:oledlg.dll
 0001:0004c840       __imp_load__OleUIConvertA@4 5f54d840     oledlg:oledlg.dll
 0001:0004c84c       _OleUIConvertA@4           5f54d84c     oledlg:oledlg.dll
 0001:0004c852       __imp_load__OleUIChangeIconA@4 5f54d852     oledlg:oledlg.dll
 0001:0004c85e       _OleUIChangeIconA@4        5f54d85e     oledlg:oledlg.dll
 0001:0004c864       __imp_load__OleUIEditLinksA@4 5f54d864     oledlg:oledlg.dll
 0001:0004c870       _OleUIEditLinksA@4         5f54d870     oledlg:oledlg.dll
 0001:0004c876       __imp_load__OleUIUpdateLinksA@16 5f54d876     oledlg:oledlg.dll
 0001:0004c882       _OleUIUpdateLinksA@16      5f54d882     oledlg:oledlg.dll
 0001:0004c888       __imp_load__OleUIPasteSpecialA@4 5f54d888     oledlg:oledlg.dll
 0001:0004c894       _OleUIPasteSpecialA@4      5f54d894     oledlg:oledlg.dll
 0001:0004c89a       __imp_load__OleUIBusyA@4   5f54d89a     oledlg:oledlg.dll
 0001:0004c8a6       _OleUIBusyA@4              5f54d8a6     oledlg:oledlg.dll
 0001:0004c8ac       __imp_load__OleUIObjectPropertiesA@4 5f54d8ac     oledlg:oledlg.dll
 0001:0004c8b8       _OleUIObjectPropertiesA@4  5f54d8b8     oledlg:oledlg.dll
 0001:0004c8be       __imp_load__OleUIChangeSourceA@4 5f54d8be     oledlg:oledlg.dll
 0001:0004c8ca       _OleUIChangeSourceA@4      5f54d8ca     oledlg:oledlg.dll
 0001:0004c8d0       __imp_load__OleUIAddVerbMenuA@36 5f54d8d0     oledlg:oledlg.dll
 0001:0004c8dc       _OleUIAddVerbMenuA@36      5f54d8dc     oledlg:oledlg.dll
 0001:0004c8e2       __imp_load__CreateURLMoniker@12 5f54d8e2     urlmon:urlmon.dll
 0001:0004c8ee       __tailMerge_urlmon         5f54d8ee     urlmon:urlmon.dll
 0001:0004c8fc       _CreateURLMoniker@12       5f54d8fc     urlmon:urlmon.dll
 0001:0004c902       __imp_load__CreateAsyncBindCtx@16 5f54d902     urlmon:urlmon.dll
 0001:0004c90e       _CreateAsyncBindCtx@16     5f54d90e     urlmon:urlmon.dll
 0001:0004c914       __imp_load__RegisterBindStatusCallback@16 5f54d914     urlmon:urlmon.dll
 0001:0004c920       _RegisterBindStatusCallback@16 5f54d920     urlmon:urlmon.dll
 0001:0004c926       __imp_load__IsAsyncMoniker@4 5f54d926     urlmon:urlmon.dll
 0001:0004c932       _IsAsyncMoniker@4          5f54d932     urlmon:urlmon.dll
 0001:0004c938       __imp_load__ExtractIconA@12 5f54d938     shell32:SHELL32.dll
 0001:0004c944       __tailMerge_SHELL32        5f54d944     shell32:SHELL32.dll
 0001:0004c952       _ExtractIconA@12           5f54d952     shell32:SHELL32.dll
 0001:0004c958       __imp_load__DragFinish@4   5f54d958     shell32:SHELL32.dll
 0001:0004c964       _DragFinish@4              5f54d964     shell32:SHELL32.dll
 0001:0004c96a       __imp_load__DragQueryFileA@16 5f54d96a     shell32:SHELL32.dll
 0001:0004c976       _DragQueryFileA@16         5f54d976     shell32:SHELL32.dll
 0001:0004c97c       ___delayLoadHelper@8       5f54d97c f   delayimp:delayhlp.obj
 0001:0004cb75       ___FUnloadDelayLoadedDLL@4 5f54db75 f   delayimp:delayhlp.obj
 0001:0004cc28       _GetProcAddress@8          5f54dc28 f   kernel32:KERNEL32.dll
 0001:0004cc2e       _InterlockedExchange@8     5f54dc2e f   kernel32:KERNEL32.dll
 0001:0004cc34       _RaiseException@16         5f54dc34 f   kernel32:KERNEL32.dll
 0001:0004cc40       ?_GetBaseClass@COleControlModule@@KGPAUCRuntimeClass@@XZ 5f54dc40 f   ctlmodul.obj
 0001:0004cc4a       ?GetRuntimeClass@COleControlModule@@UBEPAUCRuntimeClass@@XZ 5f54dc4a f   ctlmodul.obj
 0001:0004cc5a       ?InitInstance@COleControlModule@@UAEHXZ 5f54dc5a f   ctlmodul.obj
 0001:0004cc74       ?ExitInstance@COleControlModule@@UAEHXZ 5f54dc74 f   ctlmodul.obj
 0001:0004cc90       ??0CReObject@@QAE@XZ       5f54dc90 f   viewrich.obj
 0001:0004ccba       ??0CReObject@@QAE@PAVCRichEditCntrItem@@@Z 5f54dcba f   viewrich.obj
 0001:0004cdf5       ??1CReObject@@QAE@XZ       5f54ddf5 f   viewrich.obj
 0001:0004ce70       ?_GetBaseMessageMap@CRichEditView@@KGPBUAFX_MSGMAP@@XZ 5f54de70 f   viewrich.obj
 0001:0004ce7a       ?GetMessageMap@CRichEditView@@MBEPBUAFX_MSGMAP@@XZ 5f54de7a f   viewrich.obj
 0001:0004ce8a       ??0CRichEditView@@QAE@XZ   5f54de8a f   viewrich.obj
 0001:0004cfc0       ?PreCreateWindow@CRichEditView@@MAEHAAUtagCREATESTRUCTA@@@Z 5f54dfc0 f   viewrich.obj
 0001:0004d01b       ?OnCreate@CRichEditView@@IAEHPAUtagCREATESTRUCTA@@@Z 5f54e01b f   viewrich.obj
 0001:0004d10c       ?OnInitialUpdate@CRichEditView@@MAEXXZ 5f54e10c f   viewrich.obj
 0001:0004d139       ?DeleteContents@CRichEditView@@UAEXXZ 5f54e139 f   viewrich.obj
 0001:0004d1c9       ?WrapChanged@CRichEditView@@MAEXXZ 5f54e1c9 f   viewrich.obj
 0001:0004d29f       ?Serialize@CRichEditView@@UAEXAAVCArchive@@@Z 5f54e29f f   viewrich.obj
 0001:0004d309       ?Stream@CRichEditView@@QAEXAAVCArchive@@H@Z 5f54e309 f   viewrich.obj
 0001:0004d3bf       ?EditStreamCallBack@CRichEditView@@SGKKPAEJPAJ@Z 5f54e3bf f   viewrich.obj
 0001:0004d53a       ?OnBeginPrinting@CRichEditView@@MAEXPAVCDC@@PAUCPrintInfo@@@Z 5f54e53a f   viewrich.obj
 0001:0004d5ee       ?PaginateTo@CRichEditView@@IAEHPAVCDC@@PAUCPrintInfo@@@Z 5f54e5ee f   viewrich.obj
 0001:0004d831       ?OnPrepareDC@CRichEditView@@UAEXPAVCDC@@PAUCPrintInfo@@@Z 5f54e831 f   viewrich.obj
 0001:0004d8de       ?PrintPage@CRichEditView@@QAEJPAVCDC@@JJ@Z 5f54e8de f   viewrich.obj
 0001:0004da27       ?PrintInsideRect@CRichEditView@@QAEJPAVCDC@@AAUtagRECT@@JJH@Z 5f54ea27 f   viewrich.obj
 0001:0004db77       ?OnPrint@CRichEditView@@MAEXPAVCDC@@PAUCPrintInfo@@@Z 5f54eb77 f   viewrich.obj
 0001:0004dd1e       ?OnEndPrinting@CRichEditView@@MAEXPAVCDC@@PAUCPrintInfo@@@Z 5f54ed1e f   viewrich.obj
 0001:0004dd5f       ?_GetBaseInterfaceMap@CRichEditView@@KGPBUAFX_INTERFACEMAP@@XZ 5f54ed5f f   viewrich.obj
 0001:0004dd69       ?GetInterfaceMap@CRichEditView@@MBEPBUAFX_INTERFACEMAP@@XZ 5f54ed69 f   viewrich.obj
 0001:0004dd79       ?AddRef@XRichEditOleCallback@CRichEditView@@UAGKXZ 5f54ed79 f   viewrich.obj
 0001:0004dd96       ?Release@XRichEditOleCallback@CRichEditView@@UAGKXZ 5f54ed96 f   viewrich.obj
 0001:0004ddb3       ?QueryInterface@XRichEditOleCallback@CRichEditView@@UAGJABU_GUID@@PAPAX@Z 5f54edb3 f   viewrich.obj
 0001:0004ddd8       ?GetNewStorage@XRichEditOleCallback@CRichEditView@@UAGJPAPAUIStorage@@@Z 5f54edd8 f   viewrich.obj
 0001:0004de92       ?GetInPlaceContext@XRichEditOleCallback@CRichEditView@@UAGJPAPAUIOleInPlaceFrame@@PAPAUIOleInPlaceUIWindow@@PAUtagOIFI@@@Z 5f54ee92 f   viewrich.obj
 0001:0004df07       ?ShowContainerUI@XRichEditOleCallback@CRichEditView@@UAGJH@Z 5f54ef07 f   viewrich.obj
 0001:0004df74       ?QueryInsertObject@XRichEditOleCallback@CRichEditView@@UAGJPAU_GUID@@PAUIStorage@@J@Z 5f54ef74 f   viewrich.obj
 0001:0004dfe8       ?DeleteObject@XRichEditOleCallback@CRichEditView@@UAGJPAUIOleObject@@@Z 5f54efe8 f   viewrich.obj
 0001:0004e00e       ?QueryAcceptData@XRichEditOleCallback@CRichEditView@@UAGJPAUIDataObject@@PAGKHPAX@Z 5f54f00e f   viewrich.obj
 0001:0004e091       ?ContextSensitiveHelp@XRichEditOleCallback@CRichEditView@@UAGJH@Z 5f54f091 f   viewrich.obj
 0001:0004e09d       ?GetClipboardData@XRichEditOleCallback@CRichEditView@@UAGJPAU_charrange@@KPAPAUIDataObject@@@Z 5f54f09d f   viewrich.obj
 0001:0004e1a1       ?GetDragDropEffect@XRichEditOleCallback@CRichEditView@@UAGJHKPAK@Z 5f54f1a1 f   viewrich.obj
 0001:0004e20a       ?GetContextMenu@XRichEditOleCallback@CRichEditView@@UAGJGPAUIOleObject@@PAU_charrange@@PAPAUHMENU__@@@Z 5f54f20a f   viewrich.obj
 0001:0004e2b6       ?OnCharEffect@CRichEditView@@QAEXKK@Z 5f54f2b6 f   viewrich.obj
 0001:0004e334       ?OnUpdateCharEffect@CRichEditView@@QAEXPAVCCmdUI@@KK@Z 5f54f334 f   viewrich.obj
 0001:0004e388       ?OnParaAlign@CRichEditView@@QAEXG@Z 5f54f388 f   viewrich.obj
 0001:0004e3c9       ?OnUpdateParaAlign@CRichEditView@@QAEXPAVCCmdUI@@G@Z 5f54f3c9 f   viewrich.obj
 0001:0004e43e       ?OnUpdateNeedSel@CRichEditView@@IAEXPAVCCmdUI@@@Z 5f54f43e f   viewrich.obj
 0001:0004e4a0       ?OnUpdateNeedClip@CRichEditView@@IAEXPAVCCmdUI@@@Z 5f54f4a0 f   viewrich.obj
 0001:0004e4d3       ?OnUpdateNeedText@CRichEditView@@IAEXPAVCCmdUI@@@Z 5f54f4d3 f   viewrich.obj
 0001:0004e50c       ?OnUpdateNeedFind@CRichEditView@@IAEXPAVCCmdUI@@@Z 5f54f50c f   viewrich.obj
 0001:0004e575       ?OnUpdateEditUndo@CRichEditView@@IAEXPAVCCmdUI@@@Z 5f54f575 f   viewrich.obj
 0001:0004e5af       ?OnEditCut@CRichEditView@@IAEXXZ 5f54f5af f   viewrich.obj
 0001:0004e5dc       ?OnEditCopy@CRichEditView@@IAEXXZ 5f54f5dc f   viewrich.obj
 0001:0004e609       ?OnEditPaste@CRichEditView@@IAEXXZ 5f54f609 f   viewrich.obj
 0001:0004e640       ?OnEditClear@CRichEditView@@IAEXXZ 5f54f640 f   viewrich.obj
 0001:0004e66d       ?OnEditUndo@CRichEditView@@IAEXXZ 5f54f66d f   viewrich.obj
 0001:0004e6b4       ?OnEditSelectAll@CRichEditView@@IAEXXZ 5f54f6b4 f   viewrich.obj
 0001:0004e6e5       ?OnEditFind@CRichEditView@@IAEXXZ 5f54f6e5 f   viewrich.obj
 0001:0004e70d       ?OnEditReplace@CRichEditView@@IAEXXZ 5f54f70d f   viewrich.obj
 0001:0004e735       ?OnEditRepeat@CRichEditView@@IAEXXZ 5f54f735 f   viewrich.obj
 0001:0004e787       ?OnCancelEditCntr@CRichEditView@@IAEXXZ 5f54f787 f   viewrich.obj
 0001:0004e7a4       ?OnInsertObject@CRichEditView@@IAEXXZ 5f54f7a4 f   viewrich.obj
 0001:0004e9b8       ?OnSelChange@CRichEditView@@IAEXPAUtagNMHDR@@PAJ@Z 5f54f9b8 f   viewrich.obj
 0001:0004ea14       ?OnDestroy@CRichEditView@@IAEXXZ 5f54fa14 f   viewrich.obj
 0001:0004ea42       ?OnEditProperties@CRichEditView@@IAEXXZ 5f54fa42 f   viewrich.obj
 0001:0004eb2e       ?OnUpdateEditProperties@CRichEditView@@IAEXPAVCCmdUI@@@Z 5f54fb2e f   viewrich.obj
 0001:0004eb54       ?OnCharBold@CRichEditView@@IAEXXZ 5f54fb54 f   viewrich.obj
 0001:0004eb6b       ?OnUpdateCharBold@CRichEditView@@IAEXPAVCCmdUI@@@Z 5f54fb6b f   viewrich.obj
 0001:0004eb88       ?OnCharItalic@CRichEditView@@IAEXXZ 5f54fb88 f   viewrich.obj
 0001:0004eb9f       ?OnUpdateCharItalic@CRichEditView@@IAEXPAVCCmdUI@@@Z 5f54fb9f f   viewrich.obj
 0001:0004ebbc       ?OnCharUnderline@CRichEditView@@IAEXXZ 5f54fbbc f   viewrich.obj
 0001:0004ebd3       ?OnUpdateCharUnderline@CRichEditView@@IAEXPAVCCmdUI@@@Z 5f54fbd3 f   viewrich.obj
 0001:0004ebf0       ?OnParaCenter@CRichEditView@@IAEXXZ 5f54fbf0 f   viewrich.obj
 0001:0004ec05       ?OnUpdateParaCenter@CRichEditView@@IAEXPAVCCmdUI@@@Z 5f54fc05 f   viewrich.obj
 0001:0004ec20       ?OnParaLeft@CRichEditView@@IAEXXZ 5f54fc20 f   viewrich.obj
 0001:0004ec35       ?OnUpdateParaLeft@CRichEditView@@IAEXPAVCCmdUI@@@Z 5f54fc35 f   viewrich.obj
 0001:0004ec50       ?OnParaRight@CRichEditView@@IAEXXZ 5f54fc50 f   viewrich.obj
 0001:0004ec65       ?OnUpdateParaRight@CRichEditView@@IAEXPAVCCmdUI@@@Z 5f54fc65 f   viewrich.obj
 0001:0004ec80       ?OnBullet@CRichEditView@@IAEXXZ 5f54fc80 f   viewrich.obj
 0001:0004ed3b       ?OnUpdateBullet@CRichEditView@@IAEXPAVCCmdUI@@@Z 5f54fd3b f   viewrich.obj
 0001:0004ed92       ?OnFormatFont@CRichEditView@@IAEXXZ 5f54fd92 f   viewrich.obj
 0001:0004ee57       ?OnColorPick@CRichEditView@@IAEXK@Z 5f54fe57 f   viewrich.obj
 0001:0004eeb3       ?OnColorDefault@CRichEditView@@IAEXXZ 5f54feb3 f   viewrich.obj
 0001:0004ef01       ?OnEditPasteSpecial@CRichEditView@@IAEXXZ 5f54ff01 f   viewrich.obj
 0001:0004f060       ?OnUpdateEditPasteSpecial@CRichEditView@@IAEXPAVCCmdUI@@@Z 5f550060 f   viewrich.obj
 0001:0004f080       ?OnKeyDown@CRichEditView@@IAEXIII@Z 5f550080 f   viewrich.obj
 0001:0004f113       ?OnDropFiles@CRichEditView@@IAEXPAUHDROP__@@@Z 5f550113 f   viewrich.obj
 0001:0004f261       ?OnDevModeChange@CRichEditView@@IAEXPAD@Z 5f550261 f   viewrich.obj
 0001:0004f2cf       ?IsRichEditFormat@CRichEditView@@SAHG@Z 5f5502cf f   viewrich.obj
 0001:0004f319       ?CanPaste@CRichEditView@@QBEHXZ 5f550319 f   viewrich.obj
 0001:0004f3e3       ?GetCharFormatSelection@CRichEditView@@QAEAAU_charformat@@XZ 5f5503e3 f   viewrich.obj
 0001:0004f428       ?GetParaFormatSelection@CRichEditView@@QAEAAU_paraformat@@XZ 5f550428 f   viewrich.obj
 0001:0004f46d       ?SetCharFormat@CRichEditView@@QAEXU_charformat@@@Z 5f55046d f   viewrich.obj
 0001:0004f4d9       ?SetParaFormat@CRichEditView@@QAEHAAU_paraformat@@@Z 5f5504d9 f   viewrich.obj
 0001:0004f551       ?GetSelectedItem@CRichEditView@@QBEPAVCRichEditCntrItem@@XZ 5f550551 f   viewrich.obj
 0001:0004f64c       ?GetInPlaceActiveItem@CRichEditView@@QBEPAVCRichEditCntrItem@@XZ 5f55064c f   viewrich.obj
 0001:0004f753       ?InsertItem@CRichEditView@@QAEJPAVCRichEditCntrItem@@@Z 5f550753 f   viewrich.obj
 0001:0004f824       ?InsertFileAsObject@CRichEditView@@QAEXPBD@Z 5f550824 f   viewrich.obj
 0001:0004f990       ?DoPaste@CRichEditView@@QAEXAAVCOleDataObject@@GPAX@Z 5f550990 f   viewrich.obj
 0001:0004fcd5       ?OnPrinterChanged@CRichEditView@@MAEXABVCDC@@@Z 5f550cd5 f   viewrich.obj
 0001:0004fdae       ?OnPasteNativeObject@CRichEditView@@MAEHPAUIStorage@@@Z 5f550dae f   viewrich.obj
 0001:0004fdbd       ?GetContextMenu@CRichEditView@@MAEPAUHMENU__@@GPAUIOleObject@@PAU_charrange@@@Z 5f550dbd f   viewrich.obj
 0001:0004fdcc       ?GetClipboardData@CRichEditView@@MAEJPAU_charrange@@KPAUIDataObject@@PAPAU3@@Z 5f550dcc f   viewrich.obj
 0001:0004fdde       ?QueryAcceptData@CRichEditView@@MAEJPAUIDataObject@@PAGKHPAX@Z 5f550dde f   viewrich.obj
 0001:0004ff68       ?GetWindowContext@CRichEditView@@QAEJPAPAUIOleInPlaceFrame@@PAPAUIOleInPlaceUIWindow@@PAUtagOIFI@@@Z 5f550f68 f   viewrich.obj
 0001:0004ffbc       ?ShowContainerUI@CRichEditView@@QAEJH@Z 5f550fbc f   viewrich.obj
 0001:0005001a       ?AdjustDialogPosition@CRichEditView@@QAEXPAVCDialog@@@Z 5f55101a f   viewrich.obj
 0001:0005012a       ?OnEditFindReplace@CRichEditView@@IAEXH@Z 5f55112a f   viewrich.obj
 0001:0005040d       ?OnFindNext@CRichEditView@@MAEXPBDHHH@Z 5f55140d f   viewrich.obj
 0001:000504af       ?OnReplaceSel@CRichEditView@@MAEXPBDHHH0@Z 5f5514af f   viewrich.obj
 0001:000505da       ?OnReplaceAll@CRichEditView@@MAEXPBD0HH@Z 5f5515da f   viewrich.obj
 0001:00050759       ?OnFindReplaceCmd@CRichEditView@@IAEJIJ@Z 5f551759 f   viewrich.obj
 0001:00050a15       ?SameAsSelected@CRichEditView@@IAEHPBDHH@Z 5f551a15 f   viewrich.obj
 0001:00050af2       ?FindTextA@CRichEditView@@QAEHPAV_AFX_RICHEDIT_STATE@@@Z 5f551af2 f   viewrich.obj
 0001:00050b47       ?FindTextA@CRichEditView@@QAEHPBDHH@Z 5f551b47 f   viewrich.obj
 0001:00050bc0       ?FindTextSimple@CRichEditView@@QAEHPAV_AFX_RICHEDIT_STATE@@@Z 5f551bc0 f   viewrich.obj
 0001:00050c15       ?FindTextSimple@CRichEditView@@QAEHPBDHH@Z 5f551c15 f   viewrich.obj
 0001:00050de0       ?FindAndSelect@CRichEditView@@QAEJKAAU_findtextexa@@@Z 5f551de0 f   viewrich.obj
 0001:00050e28       ?TextNotFound@CRichEditView@@QAEXPBD@Z 5f551e28 f   viewrich.obj
 0001:00050e64       ?OnTextNotFound@CRichEditView@@MAEXPBD@Z 5f551e64 f   viewrich.obj
 0001:00050e79       ?AssertValid@CRichEditView@@UBEXXZ 5f551e79 f   viewrich.obj
 0001:00050ed3       ?Dump@CRichEditView@@UBEXAAVCDumpContext@@@Z 5f551ed3 f   viewrich.obj
 0001:00050feb       ?IsSelected@CRichEditView@@MBEHPBVCObject@@@Z 5f551feb f   viewrich.obj
 0001:0005100a       ??0CRichEditDoc@@IAE@XZ    5f55200a f   viewrich.obj
 0001:00051083       ?GetView@CRichEditDoc@@UBEPAVCRichEditView@@XZ 5f552083 f   viewrich.obj
 0001:000510da       ?IsModified@CRichEditDoc@@UAEHXZ 5f5520da f   viewrich.obj
 0001:00051101       ?SetModifiedFlag@CRichEditDoc@@UAEXH@Z 5f552101 f   viewrich.obj
 0001:0005117d       ?GetInPlaceActiveItem@CRichEditDoc@@UAEPAVCOleClientItem@@PAVCWnd@@@Z 5f55217d f   viewrich.obj
 0001:000511cb       ?SetPathName@CRichEditDoc@@UAEXPBDH@Z 5f5521cb f   viewrich.obj
 0001:000511e8       ?SetTitle@CRichEditDoc@@UAEXPBD@Z 5f5521e8 f   viewrich.obj
 0001:000512a7       ?LookupItem@CRichEditDoc@@QBEPAVCRichEditCntrItem@@PAUIOleObject@@@Z 5f5522a7 f   viewrich.obj
 0001:000512fb       ?CreateClientItem@CRichEditDoc@@UBEPAVCRichEditCntrItem@@PAU_reobject@@@Z 5f5522fb f   viewrich.obj
 0001:00051379       ?MarkItemsClear@CRichEditDoc@@IBEXXZ 5f552379 f   viewrich.obj
 0001:000513ce       ?DeleteUnmarkedItems@CRichEditDoc@@IBEXXZ 5f5523ce f   viewrich.obj
 0001:00051445       ?GetStartPosition@CRichEditDoc@@UBEPAU__POSITION@@XZ 5f552445 f   viewrich.obj
 0001:0005146c       ?UpdateObjectCache@CRichEditDoc@@IAEXXZ 5f55246c f   viewrich.obj
 0001:000515f0       ?GetPrimarySelectedItem@CRichEditDoc@@UAEPAVCOleClientItem@@PAVCView@@@Z 5f5525f0 f   viewrich.obj
 0001:00051636       ?DeleteContents@CRichEditDoc@@UAEXXZ 5f552636 f   viewrich.obj
 0001:000516f1       ?Serialize@CRichEditDoc@@UAEXAAVCArchive@@@Z 5f5526f1 f   viewrich.obj
 0001:00051726       ?AssertValid@CRichEditDoc@@UBEXXZ 5f552726 f   viewrich.obj
 0001:00051739       ?Dump@CRichEditDoc@@UBEXAAVCDumpContext@@@Z 5f552739 f   viewrich.obj
 0001:00051752       ?PreCloseFrame@CRichEditDoc@@UAEXPAVCFrameWnd@@@Z 5f552752 f   viewrich.obj
 0001:00051853       ?UpdateModifiedFlag@CRichEditDoc@@UAEXXZ 5f552853 f   viewrich.obj
 0001:0005185e       ?OnGetEmbeddedItem@CRichEditDoc@@MAEPAVCOleServerItem@@XZ 5f55285e f   viewrich.obj
 0001:00051894       ??0CRichEditCntrItem@@QAE@PAU_reobject@@PAVCRichEditDoc@@@Z 5f552894 f   viewrich.obj
 0001:000519f0       ??1CRichEditCntrItem@@UAE@XZ 5f5529f0 f   viewrich.obj
 0001:00051a54       ?OnDeactivateUI@CRichEditCntrItem@@UAEXH@Z 5f552a54 f   viewrich.obj
 0001:00051ac7       ?ShowContainerUI@CRichEditCntrItem@@QAEJH@Z 5f552ac7 f   viewrich.obj
 0001:00051b31       ?OnChangeItemPosition@CRichEditCntrItem@@MAEHABVCRect@@@Z 5f552b31 f   viewrich.obj
 0001:00051b53       ?CanActivate@CRichEditCntrItem@@UAEHXZ 5f552b53 f   viewrich.obj
 0001:00051b97       ?GetWindowContext@CRichEditCntrItem@@QAEJPAPAUIOleInPlaceFrame@@PAPAUIOleInPlaceUIWindow@@PAUtagOIFI@@@Z 5f552b97 f   viewrich.obj
 0001:00051bf3       ?ConvertTo@CRichEditCntrItem@@UAEHABU_GUID@@@Z 5f552bf3 f   viewrich.obj
 0001:00051cd5       ?ActivateAs@CRichEditCntrItem@@UAEHPBDABU_GUID@@1@Z 5f552cd5 f   viewrich.obj
 0001:00051d23       ?SetDrawAspect@CRichEditCntrItem@@UAEXW4tagDVASPECT@@@Z 5f552d23 f   viewrich.obj
 0001:00051d6f       ?SyncToRichEditObject@CRichEditCntrItem@@QAEXAAU_reobject@@@Z 5f552d6f f   viewrich.obj
 0001:00051d8b       ?AssertValid@CRichEditCntrItem@@UBEXXZ 5f552d8b f   viewrich.obj
 0001:00051d9e       ?Dump@CRichEditCntrItem@@UBEXAAVCDumpContext@@@Z 5f552d9e f   viewrich.obj
 0001:00051db7       ?GetClientSite@CRichEditCntrItem@@UAEPAUIOleClientSite@@XZ 5f552db7 f   viewrich.obj
 0001:00051e86       ?GetRichEditCtrl@CRichEditView@@QBEAAVCRichEditCtrl@@XZ 5f552e86 f   viewrich.obj
 0001:00051e94       ?GetPrintWidth@CRichEditView@@QBEHXZ 5f552e94 f   viewrich.obj
 0001:00051eb4       ?GetPrintRect@CRichEditView@@QBE?AVCRect@@XZ 5f552eb4 f   viewrich.obj
 0001:00051f18       ?GetPageRect@CRichEditView@@QBE?AVCRect@@XZ 5f552f18 f   viewrich.obj
 0001:00051f87       ?SetPaperSize@CRichEditView@@QAEXVCSize@@@Z 5f552f87 f   viewrich.obj
 0001:00051fa9       ?GetPaperSize@CRichEditView@@QBE?AVCSize@@XZ 5f552fa9 f   viewrich.obj
 0001:00051fd0       ?SetMargins@CRichEditView@@QAEXABVCRect@@@Z 5f552fd0 f   viewrich.obj
 0001:00051ffc       ?GetMargins@CRichEditView@@QBE?AVCRect@@XZ 5f552ffc f   viewrich.obj
 0001:0005202b       ?GetTextLength@CRichEditView@@QBEJXZ 5f55302b f   viewrich.obj
 0001:00052045       ?GetDocument@CRichEditView@@QBEPAVCRichEditDoc@@XZ 5f553045 f   viewrich.obj
 0001:000520a7       ?GetStreamFormat@CRichEditDoc@@QBEHXZ 5f5530a7 f   viewrich.obj
 0001:000520c4       ?InvalidateObjectCache@CRichEditDoc@@QAEXXZ 5f5530c4 f   viewrich.obj
 0001:000520dc       ?Mark@CRichEditCntrItem@@QAEXH@Z 5f5530dc f   viewrich.obj
 0001:000520f2       ?IsMarked@CRichEditCntrItem@@QAEHXZ 5f5530f2 f   viewrich.obj
 0001:00052127       ?GetDocument@CRichEditCntrItem@@QAEPAVCRichEditDoc@@XZ 5f553127 f   viewrich.obj
 0001:0005213a       ?GetActiveView@CRichEditCntrItem@@QAEPAVCRichEditView@@XZ 5f55313a f   viewrich.obj
 0001:00052150       ??_GCRichEditView@@UAEPAXI@Z 5f553150 f i viewrich.obj
 0001:00052180       ??0XRichEditOleCallback@CRichEditView@@QAE@XZ 5f553180 f i viewrich.obj
 0001:000521a0       ??0IRichEditOleCallback@@QAE@XZ 5f5531a0 f i viewrich.obj
 0001:000521c0       ??0_afxRichEditCookie@@QAE@AAVCArchive@@@Z 5f5531c0 f i viewrich.obj
 0001:000521f0       ??1CFontDialog@@UAE@XZ     5f5531f0 f i viewrich.obj
 0001:00052210       ??_ECRichEditDoc@@UAEPAXI@Z 5f553210 f i viewrich.obj
 0001:00052210       ??_GCRichEditDoc@@UAEPAXI@Z 5f553210 f i viewrich.obj
 0001:00052240       ??1CRichEditDoc@@UAE@XZ    5f553240 f i viewrich.obj
 0001:00052260       ??_GCRichEditCntrItem@@UAEPAXI@Z 5f553260 f i viewrich.obj
 0001:00052290       _RawDllMain@12             5f553290 f   dllole.obj
 0001:00052396       _DllMain@12                5f553396 f   dllole.obj
 0001:0005254f       ?AfxOleInitModule@@YGXXZ   5f55354f f   dllole.obj
 0001:00052617       _DllGetClassObject@12      5f553617 f   dllole.obj
 0001:00052650       _DllCanUnloadNow@0         5f553650 f   dllole.obj
 0001:0005267b       _DllRegisterServer@0       5f55367b f   dllole.obj
 0001:000526c4       _DllUnregisterServer@0     5f5536c4 f   dllole.obj
 0001:0005274e       ?AfxWndProcDllOle@@YGJPAUHWND__@@IIJ@Z 5f55374e f   dllole.obj
 0001:000527b8       ??1_AFX_INIT_OLE_DLL_STATE@@QAE@XZ 5f5537b8 f   dllole.obj
 0001:00052854       ?_AfxGetOleModuleState@@YGPAVAFX_MODULE_STATE@@XZ 5f553854 f   dllole.obj
 0001:00052879       ??0OLE_DATA@@QAE@XZ        5f553879 f   oleinit.obj
 0001:00052952       ?AfxOleInit@@YGHXZ         5f553952 f   oleinit.obj
 0001:00052aaa       ?AfxOleTerm@@YGXH@Z        5f553aaa f   oleinit.obj
 0001:00052b3e       ?AfxOleTermOrFreeLib@@YGXHH@Z 5f553b3e f   oleinit.obj
 0001:00052b9d       ?_AfxParseOption@@YGHPADPBD@Z 5f553b9d f   oleinit.obj
 0001:00052c31       ?RunEmbedded@CWinApp@@QAEHXZ 5f553c31 f   oleinit.obj
 0001:00052c8a       ?RunAutomated@CWinApp@@QAEHXZ 5f553c8a f   oleinit.obj
 0001:00052cf0       ?_GetBaseClass@COleLinkingDoc@@KGPAUCRuntimeClass@@XZ 5f553cf0 f   olecli1.obj
 0001:00052cfa       ?GetRuntimeClass@COleLinkingDoc@@UBEPAUCRuntimeClass@@XZ 5f553cfa f   olecli1.obj
 0001:00052d10       ?AfxBSTR2CString@@YGXPAVCString@@PAG@Z 5f553d10 f   olecnvrt.obj
 0001:00052db3       ?AfxBSTR2ABSTR@@YGPAGPAG@Z 5f553db3 f   olecnvrt.obj
 0001:00052e3b       ?AfxTaskStringA2W@@YGPAGPBD@Z 5f553e3b f   olecnvrt.obj
 0001:00052e5e       ?AfxTaskStringW2A@@YGPADPBG@Z 5f553e5e f   olecnvrt.obj
 0001:00052e81       ?AfxDevModeA2W@@YGPAU_devicemodeW@@PAU1@PAU_devicemodeA@@@Z 5f553e81 f   olecnvrt.obj
 0001:00052f4e       ?AfxDevModeW2A@@YGPAU_devicemodeA@@PAU1@PAU_devicemodeW@@@Z 5f553f4e f   olecnvrt.obj
 0001:0005301b       ?AfxTextMetricA2W@@YGPAUtagTEXTMETRICW@@PAU1@PAUtagTEXTMETRICA@@@Z 5f55401b f   olecnvrt.obj
 0001:000530ef       ?AfxTextMetricW2A@@YGPAUtagTEXTMETRICA@@PAU1@PAUtagTEXTMETRICW@@@Z 5f5540ef f   olecnvrt.obj
 0001:000531d3       ?AfxAllocTaskWideString@@YGPAGPBG@Z 5f5541d3 f   olecnvrt.obj
 0001:00053227       ?AfxAllocTaskWideString@@YGPAGPBD@Z 5f554227 f   olecnvrt.obj
 0001:000532a1       ?AfxAllocTaskAnsiString@@YGPADPBG@Z 5f5542a1 f   olecnvrt.obj
 0001:00053321       ?AfxAllocTaskAnsiString@@YGPADPBD@Z 5f554321 f   olecnvrt.obj
 0001:00053380       ?_GetBaseClass@COleDispatchException@@KGPAUCRuntimeClass@@XZ 5f554380 f   oledisp1.obj
 0001:0005338a       ?GetRuntimeClass@COleDispatchException@@UBEPAUCRuntimeClass@@XZ 5f55438a f   oledisp1.obj
 0001:000533a0       ?_GetBaseClass@COleInsertDialog@@KGPAUCRuntimeClass@@XZ 5f5543a0 f   oledlgs1.obj
 0001:000533aa       ?GetRuntimeClass@COleInsertDialog@@UBEPAUCRuntimeClass@@XZ 5f5543aa f   oledlgs1.obj
 0001:000533ba       ?_GetBaseClass@COleConvertDialog@@KGPAUCRuntimeClass@@XZ 5f5543ba f   oledlgs1.obj
 0001:000533c4       ?GetRuntimeClass@COleConvertDialog@@UBEPAUCRuntimeClass@@XZ 5f5543c4 f   oledlgs1.obj
 0001:000533d4       ?_GetBaseClass@COleChangeIconDialog@@KGPAUCRuntimeClass@@XZ 5f5543d4 f   oledlgs1.obj
 0001:000533de       ?GetRuntimeClass@COleChangeIconDialog@@UBEPAUCRuntimeClass@@XZ 5f5543de f   oledlgs1.obj
 0001:000533ee       ?_GetBaseClass@COleLinksDialog@@KGPAUCRuntimeClass@@XZ 5f5543ee f   oledlgs1.obj
 0001:000533f8       ?GetRuntimeClass@COleLinksDialog@@UBEPAUCRuntimeClass@@XZ 5f5543f8 f   oledlgs1.obj
 0001:00053408       ?_GetBaseClass@COleUpdateDialog@@KGPAUCRuntimeClass@@XZ 5f554408 f   oledlgs1.obj
 0001:00053412       ?GetRuntimeClass@COleUpdateDialog@@UBEPAUCRuntimeClass@@XZ 5f554412 f   oledlgs1.obj
 0001:00053422       ?_GetBaseClass@COlePasteSpecialDialog@@KGPAUCRuntimeClass@@XZ 5f554422 f   oledlgs1.obj
 0001:0005342c       ?GetRuntimeClass@COlePasteSpecialDialog@@UBEPAUCRuntimeClass@@XZ 5f55442c f   oledlgs1.obj
 0001:00053440       ?_GetBaseClass@COleDialog@@KGPAUCRuntimeClass@@XZ 5f554440 f   oledlgs2.obj
 0001:0005344a       ?GetRuntimeClass@COleDialog@@UBEPAUCRuntimeClass@@XZ 5f55444a f   oledlgs2.obj
 0001:0005345a       ?_GetBaseClass@COleBusyDialog@@KGPAUCRuntimeClass@@XZ 5f55445a f   oledlgs2.obj
 0001:00053464       ?GetRuntimeClass@COleBusyDialog@@UBEPAUCRuntimeClass@@XZ 5f554464 f   oledlgs2.obj
 0001:00053480       ?_GetBaseClass@COlePropertiesDialog@@KGPAUCRuntimeClass@@XZ 5f554480 f   oledlgs3.obj
 0001:0005348a       ?GetRuntimeClass@COlePropertiesDialog@@UBEPAUCRuntimeClass@@XZ 5f55448a f   oledlgs3.obj
 0001:0005349a       ?_GetBaseClass@COleChangeSourceDialog@@KGPAUCRuntimeClass@@XZ 5f55449a f   oledlgs3.obj
 0001:000534a4       ?GetRuntimeClass@COleChangeSourceDialog@@UBEPAUCRuntimeClass@@XZ 5f5544a4 f   oledlgs3.obj
 0001:000534c0       ??0_AFX_OLE_STATE@@QAE@XZ  5f5544c0 f   oledata.obj
 0001:000534df       ??1_AFX_OLE_STATE@@UAE@XZ  5f5544df f   oledata.obj
 0001:00053530       ??_E_AFX_OLE_STATE@@UAEPAXI@Z 5f554530 f i oledata.obj
 0001:00053530       ??_G_AFX_OLE_STATE@@UAEPAXI@Z 5f554530 f i oledata.obj
 0001:00053560       ??0CNoTrackObject@@QAE@XZ  5f554560 f i oledata.obj
 0001:00053580       ??1?$CProcessLocal@V_AFX_OLE_STATE@@@@QAE@XZ 5f554580 f i oledata.obj
 0001:000535a0       ?CreateObject@CDocItem@@SGPAVCObject@@XZ 5f5545a0 f   oledoc1.obj
 0001:0005360e       ?_GetBaseClass@CDocItem@@KGPAUCRuntimeClass@@XZ 5f55460e f   oledoc1.obj
 0001:00053618       ?GetRuntimeClass@CDocItem@@UBEPAUCRuntimeClass@@XZ 5f554618 f   oledoc1.obj
 0001:00053646       ??5@YGAAVCArchive@@AAV0@AAPAVCDocItem@@@Z 5f554646 f   oledoc1.obj
 0001:00053662       ?_GetBaseClass@COleDocument@@KGPAUCRuntimeClass@@XZ 5f554662 f   oledoc1.obj
 0001:0005366c       ?GetRuntimeClass@COleDocument@@UBEPAUCRuntimeClass@@XZ 5f55466c f   oledoc1.obj
 0001:0005367c       ?_GetBaseClass@COleClientItem@@KGPAUCRuntimeClass@@XZ 5f55467c f   oledoc1.obj
 0001:00053686       ?GetRuntimeClass@COleClientItem@@UBEPAUCRuntimeClass@@XZ 5f554686 f   oledoc1.obj
 0001:00053696       ?_GetBaseClass@COleServerItem@@KGPAUCRuntimeClass@@XZ 5f554696 f   oledoc1.obj
 0001:000536a0       ?GetRuntimeClass@COleServerItem@@UBEPAUCRuntimeClass@@XZ 5f5546a0 f   oledoc1.obj
 0001:000536b0       ??0COleMessageFilter@@QAE@XZ 5f5546b0 f   olemsgf.obj
 0001:00053767       ?Register@COleMessageFilter@@QAEHXZ 5f554767 f   olemsgf.obj
 0001:000537d0       ??_ECOleMessageFilter@@UAEPAXI@Z 5f5547d0 f i olemsgf.obj
 0001:000537d0       ??_GCOleMessageFilter@@UAEPAXI@Z 5f5547d0 f i olemsgf.obj
 0001:00053800       ??0XMessageFilter@COleMessageFilter@@QAE@XZ 5f554800 f i olemsgf.obj
 0001:00053820       ??0COleObjectFactory@@QAE@ABU_GUID@@PAUCRuntimeClass@@HPBD@Z 5f554820 f   olefact.obj
 0001:000539a5       ?Unregister@COleObjectFactory@@QAEHXZ 5f5549a5 f   olefact.obj
 0001:000539b5       ?Register@COleObjectFactory@@UAEHXZ 5f5549b5 f   olefact.obj
 0001:00053abd       ?UnregisterAll@COleObjectFactory@@SGHXZ 5f554abd f   olefact.obj
 0001:00053b2a       ?RegisterAll@COleObjectFactory@@SGHXZ 5f554b2a f   olefact.obj
 0001:00053c42       ?_GetBaseClass@COleObjectFactory@@KGPAUCRuntimeClass@@XZ 5f554c42 f   olefact.obj
 0001:00053c4c       ?GetRuntimeClass@COleObjectFactory@@UBEPAUCRuntimeClass@@XZ 5f554c4c f   olefact.obj
 0001:00053c60       ??_GCOleObjectFactory@@UAEPAXI@Z 5f554c60 f i olefact.obj
 0001:00053c60       ??_ECOleObjectFactory@@UAEPAXI@Z 5f554c60 f i olefact.obj
 0001:00053c90       ??0XClassFactory@COleObjectFactory@@QAE@XZ 5f554c90 f i olefact.obj
 0001:00053cb0       ??0IClassFactory2@@QAE@XZ  5f554cb0 f i olefact.obj
 0001:00053cd0       ??0IClassFactory@@QAE@XZ   5f554cd0 f i olefact.obj
 0001:00053cd0       ??0IMessageFilter@@QAE@XZ  5f554cd0 f i olefact.obj
 0001:00053cf0       ?AddHead@?$CTypedSimpleList@PAVCOleObjectFactory@@@@QAEXPAVCOleObjectFactory@@@Z 5f554cf0 f i olefact.obj
 0001:00053d10       ?Remove@?$CTypedSimpleList@PAVCOleObjectFactory@@@@QAEHPAVCOleObjectFactory@@@Z 5f554d10 f i olefact.obj
 0001:00053d30       ??B?$CTypedSimpleList@PAVCDynLinkLibrary@@@@QAEPAVCDynLinkLibrary@@XZ 5f554d30 f i olefact.obj
 0001:00053d50       ?CreateObject@COleIPFrameWnd@@SGPAVCObject@@XZ 5f554d50 f   oleipfrm.obj
 0001:00053dc1       ?_GetBaseClass@COleIPFrameWnd@@KGPAUCRuntimeClass@@XZ 5f554dc1 f   oleipfrm.obj
 0001:00053dcb       ?GetRuntimeClass@COleIPFrameWnd@@UBEPAUCRuntimeClass@@XZ 5f554dcb f   oleipfrm.obj
 0001:00053de0       ?_GetBaseClass@COleException@@KGPAUCRuntimeClass@@XZ 5f554de0 f   olemisc.obj
 0001:00053dea       ?GetRuntimeClass@COleException@@UBEPAUCRuntimeClass@@XZ 5f554dea f   olemisc.obj
 0001:00053e00       ?_GetBaseClass@COleStreamFile@@KGPAUCRuntimeClass@@XZ 5f554e00 f   olestrm.obj
 0001:00053e0a       ?GetRuntimeClass@COleStreamFile@@UBEPAUCRuntimeClass@@XZ 5f554e0a f   olestrm.obj
 0001:00053e20       ?_GetBaseClass@COleServerDoc@@KGPAUCRuntimeClass@@XZ 5f554e20 f   olesvr1.obj
 0001:00053e2a       ?GetRuntimeClass@COleServerDoc@@UBEPAUCRuntimeClass@@XZ 5f554e2a f   olesvr1.obj
 0001:00053e40       ?CreateObject@CRichEditCntrItem@@SGPAVCObject@@XZ 5f554e40 f   viewrich.obj
 0001:00053eb5       ?_GetBaseClass@CRichEditCntrItem@@KGPAUCRuntimeClass@@XZ 5f554eb5 f   viewrich.obj
 0001:00053ebf       ?GetRuntimeClass@CRichEditCntrItem@@UBEPAUCRuntimeClass@@XZ 5f554ebf f   viewrich.obj
 0001:00053eed       ??5@YGAAVCArchive@@AAV0@AAPAVCRichEditCntrItem@@@Z 5f554eed f   viewrich.obj
 0001:00053f09       ?_GetBaseClass@CRichEditDoc@@KGPAUCRuntimeClass@@XZ 5f554f09 f   viewrich.obj
 0001:00053f13       ?GetRuntimeClass@CRichEditDoc@@UBEPAUCRuntimeClass@@XZ 5f554f13 f   viewrich.obj
 0001:00053f23       ?CreateObject@CRichEditView@@SGPAVCObject@@XZ 5f554f23 f   viewrich.obj
 0001:00053f94       ?_GetBaseClass@CRichEditView@@KGPAUCRuntimeClass@@XZ 5f554f94 f   viewrich.obj
 0001:00053f9e       ?GetRuntimeClass@CRichEditView@@UBEPAUCRuntimeClass@@XZ 5f554f9e f   viewrich.obj
 0001:00053fb0       ??B?$CProcessLocal@V_AFX_RICHEDIT_STATE@@@@QAEPAV_AFX_RICHEDIT_STATE@@XZ 5f554fb0 f i viewrich.obj
 0001:00053fd0       ?GetData@?$CProcessLocal@V_AFX_RICHEDIT_STATE@@@@QAEPAV_AFX_RICHEDIT_STATE@@XZ 5f554fd0 f i viewrich.obj
 0001:00054020       ?CreateObject@?$CProcessLocal@V_AFX_RICHEDIT_STATE@@@@SGPAVCNoTrackObject@@XZ 5f555020 f i viewrich.obj
 0001:00054090       ??0_AFX_RICHEDIT_STATE@@QAE@XZ 5f555090 f i viewrich.obj
 0001:000540b0       ??_G_AFX_RICHEDIT_STATE@@UAEPAXI@Z 5f5550b0 f i viewrich.obj
 0001:000540b0       ??_E_AFX_RICHEDIT_STATE@@UAEPAXI@Z 5f5550b0 f i viewrich.obj
 0001:000540e0       ?_GetBaseClass@CMonikerFile@@KGPAUCRuntimeClass@@XZ 5f5550e0 f   olemon.obj
 0001:000540ea       ?GetRuntimeClass@CMonikerFile@@UBEPAUCRuntimeClass@@XZ 5f5550ea f   olemon.obj
 0001:00054100       ?Release@?$_CIP@UIMoniker@@$1?IID_IMoniker@@3U_GUID@@B@@QAEXXZ 5f555100 f i olemon.obj
 0001:00054100       ?Release@?$_CIP@UIBinding@@$1?IID_IBinding@@3U_GUID@@B@@QAEXXZ 5f555100 f i olemon.obj
 0001:00054150       ??4?$CIP@UIBindCtx@@$1?IID_IBindCtx@@3U_GUID@@B@@QAEAAV0@PAUIBindCtx@@@Z 5f555150 f i olemon.obj
 0001:00054150       ??4?$CIP@UIMoniker@@$1?IID_IMoniker@@3U_GUID@@B@@QAEAAV0@PAUIMoniker@@@Z 5f555150 f i olemon.obj
 0001:00054150       ??4?$CIP@UIBindHost@@$1?IID_IBindHost@@3U_GUID@@B@@QAEAAV0@PAUIBindHost@@@Z 5f555150 f i olemon.obj
 0001:00054150       ??4?$CIP@UIBinding@@$1?IID_IBinding@@3U_GUID@@B@@QAEAAV0@PAUIBinding@@@Z 5f555150 f i olemon.obj
 0001:00054170       ??I?$_CIP@UIBindStatusCallback@@$1?IID_IBindStatusCallback@@3U_GUID@@B@@QAEPAPAUIBindStatusCallback@@XZ 5f555170 f i olemon.obj
 0001:00054170       ??I?$_CIP@UIStream@@$1?IID_IStream@@3U_GUID@@B@@QAEPAPAUIStream@@XZ 5f555170 f i olemon.obj
 0001:00054170       ??I?$_CIP@UIMoniker@@$1?IID_IMoniker@@3U_GUID@@B@@QAEPAPAUIMoniker@@XZ 5f555170 f i olemon.obj
 0001:00054170       ??I?$_CIP@UIBindCtx@@$1?IID_IBindCtx@@3U_GUID@@B@@QAEPAPAUIBindCtx@@XZ 5f555170 f i olemon.obj
 0001:00054190       ??7?$_CIP@UIMoniker@@$1?IID_IMoniker@@3U_GUID@@B@@QAEHXZ 5f555190 f i olemon.obj
 0001:00054190       ??7?$_CIP@UIBindCtx@@$1?IID_IBindCtx@@3U_GUID@@B@@QAEHXZ 5f555190 f i olemon.obj
 0001:00054190       ??7?$_CIP@UIBindStatusCallback@@$1?IID_IBindStatusCallback@@3U_GUID@@B@@QAEHXZ 5f555190 f i olemon.obj
 0001:000541b0       ??0?$CIP@UIBindHost@@$1?IID_IBindHost@@3U_GUID@@B@@QAE@PAUIBindHost@@H@Z 5f5551b0 f i olemon.obj
 0001:000541b0       ??0?$CIP@UIBindCtx@@$1?IID_IBindCtx@@3U_GUID@@B@@QAE@PAUIBindCtx@@H@Z 5f5551b0 f i olemon.obj
 0001:000541d0       ?Detach@?$_CIP@UIStream@@$1?IID_IStream@@3U_GUID@@B@@QAEXXZ 5f5551d0 f i olemon.obj
 0001:00054210       ?_AddRef@?$_CIP@UIBindHost@@$1?IID_IBindHost@@3U_GUID@@B@@AAEXXZ 5f555210 f i olemon.obj
 0001:00054210       ?_AddRef@?$_CIP@UIBindCtx@@$1?IID_IBindCtx@@3U_GUID@@B@@AAEXXZ 5f555210 f i olemon.obj
 0001:00054210       ?_AddRef@?$_CIP@UIMoniker@@$1?IID_IMoniker@@3U_GUID@@B@@AAEXXZ 5f555210 f i olemon.obj
 0001:00054210       ?_AddRef@?$_CIP@UIBinding@@$1?IID_IBinding@@3U_GUID@@B@@AAEXXZ 5f555210 f i olemon.obj
 0001:00054210       ?_AddRef@?$_CIP@UIBindStatusCallback@@$1?IID_IBindStatusCallback@@3U_GUID@@B@@AAEXXZ 5f555210 f i olemon.obj
 0001:00054210       ?_AddRef@?$_CIP@UIUnknown@@$1?IID_IUnknown@@3U_GUID@@B@@AAEXXZ 5f555210 f i olemon.obj
 0001:00054210       ?_AddRef@?$_CIP@UIServiceProvider@@$1?IID_IServiceProvider@@3U_GUID@@B@@AAEXXZ 5f555210 f i olemon.obj
 0001:00054240       ?_Release@?$_CIP@UIBindHost@@$1?IID_IBindHost@@3U_GUID@@B@@AAEXXZ 5f555240 f i olemon.obj
 0001:00054240       ?_Release@?$_CIP@UIUnknown@@$1?IID_IUnknown@@3U_GUID@@B@@AAEXXZ 5f555240 f i olemon.obj
 0001:00054240       ?_Release@?$_CIP@UIBinding@@$1?IID_IBinding@@3U_GUID@@B@@AAEXXZ 5f555240 f i olemon.obj
 0001:00054240       ?_Release@?$_CIP@UIBindCtx@@$1?IID_IBindCtx@@3U_GUID@@B@@AAEXXZ 5f555240 f i olemon.obj
 0001:00054240       ?_Release@?$_CIP@UIStream@@$1?IID_IStream@@3U_GUID@@B@@AAEXXZ 5f555240 f i olemon.obj
 0001:00054240       ?_Release@?$_CIP@UIServiceProvider@@$1?IID_IServiceProvider@@3U_GUID@@B@@AAEXXZ 5f555240 f i olemon.obj
 0001:00054240       ?_Release@?$_CIP@UIBindStatusCallback@@$1?IID_IBindStatusCallback@@3U_GUID@@B@@AAEXXZ 5f555240 f i olemon.obj
 0001:00054240       ?_Release@?$_CIP@UIMoniker@@$1?IID_IMoniker@@3U_GUID@@B@@AAEXXZ 5f555240 f i olemon.obj
 0001:00054270       ?_GetBaseClass@CDateTimeCtrl@@KGPAUCRuntimeClass@@XZ 5f555270 f   winctrl5.obj
 0001:0005427a       ?GetRuntimeClass@CDateTimeCtrl@@UBEPAUCRuntimeClass@@XZ 5f55527a f   winctrl5.obj
 0001:0005428a       ?_GetBaseClass@CMonthCalCtrl@@KGPAUCRuntimeClass@@XZ 5f55528a f   winctrl5.obj
 0001:00054294       ?GetRuntimeClass@CMonthCalCtrl@@UBEPAUCRuntimeClass@@XZ 5f555294 f   winctrl5.obj
 0001:000542b0       ?CreateObject@CHtmlView@@SGPAVCObject@@XZ 5f5552b0 f   viewhtml.obj
 0001:00054321       ?_GetBaseClass@CHtmlView@@KGPAUCRuntimeClass@@XZ 5f555321 f   viewhtml.obj
 0001:0005432b       ?GetRuntimeClass@CHtmlView@@UBEPAUCRuntimeClass@@XZ 5f55532b f   viewhtml.obj
 0001:00054340       ?_GetBaseClass@CAsyncMonikerFile@@KGPAUCRuntimeClass@@XZ 5f555340 f   oleasmon.obj
 0001:0005434a       ?GetRuntimeClass@CAsyncMonikerFile@@UBEPAUCRuntimeClass@@XZ 5f55534a f   oleasmon.obj
 0001:00054360       ??0?$CIP@UIBindHost@@$1?IID_IBindHost@@3U_GUID@@B@@QAE@XZ 5f555360 f i oleasmon.obj
 0001:00054360       ??0?$CIP@UIMoniker@@$1?IID_IMoniker@@3U_GUID@@B@@QAE@XZ 5f555360 f i oleasmon.obj
 0001:00054360       ??0?$CIP@UIBindCtx@@$1?IID_IBindCtx@@3U_GUID@@B@@QAE@XZ 5f555360 f i oleasmon.obj
 0001:00054360       ??0?$CIP@UIServiceProvider@@$1?IID_IServiceProvider@@3U_GUID@@B@@QAE@XZ 5f555360 f i oleasmon.obj
 0001:00054360       ??0?$CIP@UIBinding@@$1?IID_IBinding@@3U_GUID@@B@@QAE@XZ 5f555360 f i oleasmon.obj
 0001:00054360       ??0?$CIP@UIBindStatusCallback@@$1?IID_IBindStatusCallback@@3U_GUID@@B@@QAE@XZ 5f555360 f i oleasmon.obj
 0001:00054360       ??0?$CIP@UIStream@@$1?IID_IStream@@3U_GUID@@B@@QAE@XZ 5f555360 f i oleasmon.obj
 0001:00054380       ??C?$_CIP@UIBinding@@$1?IID_IBinding@@3U_GUID@@B@@QBEPAUIBinding@@XZ 5f555380 f i oleasmon.obj
 0001:000543c0       ??B?$_CIP@UIBindCtx@@$1?IID_IBindCtx@@3U_GUID@@B@@QBEPAUIBindCtx@@XZ 5f5553c0 f i oleasmon.obj
 0001:000543c0       ??B?$_CIP@UIServiceProvider@@$1?IID_IServiceProvider@@3U_GUID@@B@@QBEPAUIServiceProvider@@XZ 5f5553c0 f i oleasmon.obj
 0001:000543c0       ??B?$_CIP@UIBindHost@@$1?IID_IBindHost@@3U_GUID@@B@@QBEPAUIBindHost@@XZ 5f5553c0 f i oleasmon.obj
 0001:000543c0       ??B?$_CIP@UIBinding@@$1?IID_IBinding@@3U_GUID@@B@@QBEPAUIBinding@@XZ 5f5553c0 f i oleasmon.obj
 0001:000543c0       ?GetInterfacePtr@?$_CIP@UIMoniker@@$1?IID_IMoniker@@3U_GUID@@B@@QBEPAUIMoniker@@XZ 5f5553c0 f i oleasmon.obj
 0001:000543c0       ?GetInterfacePtr@?$_CIP@UIUnknown@@$1?IID_IUnknown@@3U_GUID@@B@@QBEPAUIUnknown@@XZ 5f5553c0 f i oleasmon.obj
 0001:000543c0       ??B?$_CIP@UIServiceProvider@@$1?IID_IServiceProvider@@3U_GUID@@B@@QAEPAUIUnknown@@XZ 5f5553c0 f i oleasmon.obj
 0001:000543c0       ?GetInterfacePtr@?$_CIP@UIBinding@@$1?IID_IBinding@@3U_GUID@@B@@QBEPAUIBinding@@XZ 5f5553c0 f i oleasmon.obj
 0001:000543c0       ?GetInterfacePtr@?$_CIP@UIStream@@$1?IID_IStream@@3U_GUID@@B@@QBEPAUIStream@@XZ 5f5553c0 f i oleasmon.obj
 0001:000543c0       ??B?$_CIP@UIMoniker@@$1?IID_IMoniker@@3U_GUID@@B@@QBEPAUIMoniker@@XZ 5f5553c0 f i oleasmon.obj
 0001:000543c0       ?GetInterfacePtr@?$_CIP@UIBindHost@@$1?IID_IBindHost@@3U_GUID@@B@@QBEPAUIBindHost@@XZ 5f5553c0 f i oleasmon.obj
 0001:000543c0       ??B?$_CIP@UIBindStatusCallback@@$1?IID_IBindStatusCallback@@3U_GUID@@B@@QBEPAUIBindStatusCallback@@XZ 5f5553c0 f i oleasmon.obj
 0001:000543c0       ??B?$_CIP@UIStream@@$1?IID_IStream@@3U_GUID@@B@@QBEPAUIStream@@XZ 5f5553c0 f i oleasmon.obj
 0001:000543c0       ?GetInterfacePtr@?$_CIP@UIServiceProvider@@$1?IID_IServiceProvider@@3U_GUID@@B@@QBEPAUIServiceProvider@@XZ 5f5553c0 f i oleasmon.obj
 0001:000543d0       ?QueryInterface@?$_CIP@UIBindHost@@$1?IID_IBindHost@@3U_GUID@@B@@QAEJPAUIUnknown@@@Z 5f5553d0 f i oleasmon.obj
 0001:00054440       ?QueryInterface@?$_CIP@UIBindStatusCallback@@$1?IID_IBindStatusCallback@@3U_GUID@@B@@QAEJPAUIUnknown@@@Z 5f555440 f i oleasmon.obj
 0001:000544b0       ?QueryInterface@?$_CIP@UIServiceProvider@@$1?IID_IServiceProvider@@3U_GUID@@B@@QAEJPAUIUnknown@@@Z 5f5554b0 f i oleasmon.obj
 0001:00054520       ?GetIID@?$_CIP@UIBindHost@@$1?IID_IBindHost@@3U_GUID@@B@@SAABU_GUID@@XZ 5f555520 f i oleasmon.obj
 0001:00054550       ?Attach@?$_CIP@UIServiceProvider@@$1?IID_IServiceProvider@@3U_GUID@@B@@QAEXPAUIServiceProvider@@@Z 5f555550 f i oleasmon.obj
 0001:00054550       ?Attach@?$_CIP@UIBindStatusCallback@@$1?IID_IBindStatusCallback@@3U_GUID@@B@@QAEXPAUIBindStatusCallback@@@Z 5f555550 f i oleasmon.obj
 0001:00054550       ?Attach@?$_CIP@UIBindHost@@$1?IID_IBindHost@@3U_GUID@@B@@QAEXPAUIBindHost@@@Z 5f555550 f i oleasmon.obj
 0001:00054570       ?GetIID@?$_CIP@UIBindStatusCallback@@$1?IID_IBindStatusCallback@@3U_GUID@@B@@SAABU_GUID@@XZ 5f555570 f i oleasmon.obj
 0001:000545a0       ?GetIID@?$_CIP@UIServiceProvider@@$1?IID_IServiceProvider@@3U_GUID@@B@@SAABU_GUID@@XZ 5f5555a0 f i oleasmon.obj
 0001:000545d0       ??4?$_CIP@UIBindStatusCallback@@$1?IID_IBindStatusCallback@@3U_GUID@@B@@QAEAAV0@PAUIBindStatusCallback@@@Z 5f5555d0 f i oleasmon.obj
 0001:000545d0       ??4?$_CIP@UIMoniker@@$1?IID_IMoniker@@3U_GUID@@B@@QAEAAV0@PAUIMoniker@@@Z 5f5555d0 f i oleasmon.obj
 0001:000545d0       ??4?$_CIP@UIBinding@@$1?IID_IBinding@@3U_GUID@@B@@QAEAAV0@PAUIBinding@@@Z 5f5555d0 f i oleasmon.obj
 0001:000545d0       ??4?$_CIP@UIBindHost@@$1?IID_IBindHost@@3U_GUID@@B@@QAEAAV0@PAUIBindHost@@@Z 5f5555d0 f i oleasmon.obj
 0001:000545d0       ??4?$_CIP@UIServiceProvider@@$1?IID_IServiceProvider@@3U_GUID@@B@@QAEAAV0@PAUIServiceProvider@@@Z 5f5555d0 f i oleasmon.obj
 0001:000545d0       ??4?$_CIP@UIBindCtx@@$1?IID_IBindCtx@@3U_GUID@@B@@QAEAAV0@PAUIBindCtx@@@Z 5f5555d0 f i oleasmon.obj
 0001:00054620       ??0?$_CIP@UIMoniker@@$1?IID_IMoniker@@3U_GUID@@B@@QAE@XZ 5f555620 f i oleasmon.obj
 0001:00054620       ??0?$_CIP@UIBindHost@@$1?IID_IBindHost@@3U_GUID@@B@@QAE@XZ 5f555620 f i oleasmon.obj
 0001:00054620       ??0?$_CIP@UIStream@@$1?IID_IStream@@3U_GUID@@B@@QAE@XZ 5f555620 f i oleasmon.obj
 0001:00054620       ??0?$_CIP@UIBindStatusCallback@@$1?IID_IBindStatusCallback@@3U_GUID@@B@@QAE@XZ 5f555620 f i oleasmon.obj
 0001:00054620       ??0?$_CIP@UIBinding@@$1?IID_IBinding@@3U_GUID@@B@@QAE@XZ 5f555620 f i oleasmon.obj
 0001:00054620       ??0?$_CIP@UIBindCtx@@$1?IID_IBindCtx@@3U_GUID@@B@@QAE@XZ 5f555620 f i oleasmon.obj
 0001:00054620       ??0?$_CIP@UIServiceProvider@@$1?IID_IServiceProvider@@3U_GUID@@B@@QAE@XZ 5f555620 f i oleasmon.obj
 0001:00054640       ??1?$CIP@UIBindHost@@$1?IID_IBindHost@@3U_GUID@@B@@QAE@XZ 5f555640 f i oleasmon.obj
 0001:00054640       ??1?$CIP@UIBindCtx@@$1?IID_IBindCtx@@3U_GUID@@B@@QAE@XZ 5f555640 f i oleasmon.obj
 0001:00054640       ??1?$CIP@UIStream@@$1?IID_IStream@@3U_GUID@@B@@QAE@XZ 5f555640 f i oleasmon.obj
 0001:00054640       ??1?$CIP@UIBindStatusCallback@@$1?IID_IBindStatusCallback@@3U_GUID@@B@@QAE@XZ 5f555640 f i oleasmon.obj
 0001:00054640       ??1?$CIP@UIMoniker@@$1?IID_IMoniker@@3U_GUID@@B@@QAE@XZ 5f555640 f i oleasmon.obj
 0001:00054640       ??1?$CIP@UIBinding@@$1?IID_IBinding@@3U_GUID@@B@@QAE@XZ 5f555640 f i oleasmon.obj
 0001:00054640       ??1?$CIP@UIServiceProvider@@$1?IID_IServiceProvider@@3U_GUID@@B@@QAE@XZ 5f555640 f i oleasmon.obj
 0001:00054660       ??1?$_CIP@UIBindHost@@$1?IID_IBindHost@@3U_GUID@@B@@QAE@XZ 5f555660 f i oleasmon.obj
 0001:00054660       ??1?$_CIP@UIMoniker@@$1?IID_IMoniker@@3U_GUID@@B@@QAE@XZ 5f555660 f i oleasmon.obj
 0001:00054660       ??1?$_CIP@UIBinding@@$1?IID_IBinding@@3U_GUID@@B@@QAE@XZ 5f555660 f i oleasmon.obj
 0001:00054660       ??1?$_CIP@UIBindStatusCallback@@$1?IID_IBindStatusCallback@@3U_GUID@@B@@QAE@XZ 5f555660 f i oleasmon.obj
 0001:00054660       ??1?$_CIP@UIStream@@$1?IID_IStream@@3U_GUID@@B@@QAE@XZ 5f555660 f i oleasmon.obj
 0001:00054660       ??1?$_CIP@UIServiceProvider@@$1?IID_IServiceProvider@@3U_GUID@@B@@QAE@XZ 5f555660 f i oleasmon.obj
 0001:00054660       ??1?$_CIP@UIBindCtx@@$1?IID_IBindCtx@@3U_GUID@@B@@QAE@XZ 5f555660 f i oleasmon.obj
 0001:00054660       ??1?$_CIP@UIUnknown@@$1?IID_IUnknown@@3U_GUID@@B@@QAE@XZ 5f555660 f i oleasmon.obj
 0001:00054680       ??0?$_CIP@UIBindCtx@@$1?IID_IBindCtx@@3U_GUID@@B@@QAE@PAUIBindCtx@@H@Z 5f555680 f i oleasmon.obj
 0001:00054680       ??0?$_CIP@UIUnknown@@$1?IID_IUnknown@@3U_GUID@@B@@QAE@PAUIUnknown@@H@Z 5f555680 f i oleasmon.obj
 0001:00054680       ??0?$_CIP@UIBindHost@@$1?IID_IBindHost@@3U_GUID@@B@@QAE@PAUIBindHost@@H@Z 5f555680 f i oleasmon.obj
 0001:000546d0       ?_GetBaseClass@COleResizeBar@@KGPAUCRuntimeClass@@XZ 5f5556d0 f   olebar.obj
 0001:000546da       ?GetRuntimeClass@COleResizeBar@@UBEPAUCRuntimeClass@@XZ 5f5556da f   olebar.obj
 0001:000546f0       ?_GetBaseClass@COleControl@@KGPAUCRuntimeClass@@XZ 5f5556f0 f   ctlcore.obj
 0001:000546fa       ?GetRuntimeClass@COleControl@@UBEPAUCRuntimeClass@@XZ 5f5556fa f   ctlcore.obj
 0001:00054710       ?GetData@?$CThreadLocal@V_AFXCTL_AMBIENT_CACHE@@@@QAEPAV_AFXCTL_AMBIENT_CACHE@@XZ 5f555710 f i ctlcore.obj
 0001:00054760       ?CreateObject@?$CThreadLocal@V_AFXCTL_AMBIENT_CACHE@@@@SGPAVCNoTrackObject@@XZ 5f555760 f i ctlcore.obj
 0001:000547d0       ?_GetBaseClass@COlePropertyPage@@KGPAUCRuntimeClass@@XZ 5f5557d0 f   ctlppg.obj
 0001:000547da       ?GetRuntimeClass@COlePropertyPage@@UBEPAUCRuntimeClass@@XZ 5f5557da f   ctlppg.obj
 0001:000547f0       ?_GetBaseClass@CDataPathProperty@@KGPAUCRuntimeClass@@XZ 5f5557f0 f   ctlprop.obj
 0001:000547fa       ?GetRuntimeClass@CDataPathProperty@@UBEPAUCRuntimeClass@@XZ 5f5557fa f   ctlprop.obj
 0001:0005480a       ?_GetBaseClass@CCachedDataPathProperty@@KGPAUCRuntimeClass@@XZ 5f55580a f   ctlprop.obj
 0001:00054814       ?GetRuntimeClass@CCachedDataPathProperty@@UBEPAUCRuntimeClass@@XZ 5f555814 f   ctlprop.obj
 0001:00054830       ??B?$CThreadLocal@V_AFXCTL_AMBIENT_CACHE@@@@QAEPAV_AFXCTL_AMBIENT_CACHE@@XZ 5f555830 f i ctlprop.obj
 0001:00054830       ??C?$CThreadLocal@V_AFXCTL_AMBIENT_CACHE@@@@QAEPAV_AFXCTL_AMBIENT_CACHE@@XZ 5f555830 f i ctlprop.obj
 0001:00054850       ?CreateObject@CColorPropPage@@SGPAVCObject@@XZ 5f555850 f   ppgcolor.obj
 0001:000548c1       ?_GetBaseClass@CColorPropPage@@KGPAUCRuntimeClass@@XZ 5f5558c1 f   ppgcolor.obj
 0001:000548cb       ?GetRuntimeClass@CColorPropPage@@UBEPAUCRuntimeClass@@XZ 5f5558cb f   ppgcolor.obj
 0001:000548e0       ?CreateObject@CFontPropPage@@SGPAVCObject@@XZ 5f5558e0 f   ppgfont.obj
 0001:00054951       ?_GetBaseClass@CFontPropPage@@KGPAUCRuntimeClass@@XZ 5f555951 f   ppgfont.obj
 0001:0005495b       ?GetRuntimeClass@CFontPropPage@@UBEPAUCRuntimeClass@@XZ 5f55595b f   ppgfont.obj
 0001:00054970       ?CreateObject@CPicturePropPage@@SGPAVCObject@@XZ 5f555970 f   ppgpict.obj
 0001:000549e1       ?_GetBaseClass@CPicturePropPage@@KGPAUCRuntimeClass@@XZ 5f5559e1 f   ppgpict.obj
 0001:000549eb       ?GetRuntimeClass@CPicturePropPage@@UBEPAUCRuntimeClass@@XZ 5f5559eb f   ppgpict.obj
 0001:00054a00       ?_GetBaseClass@CStockPropPage@@KGPAUCRuntimeClass@@XZ 5f555a00 f   ppgstock.obj
 0001:00054a0a       ?GetRuntimeClass@CStockPropPage@@UBEPAUCRuntimeClass@@XZ 5f555a0a f   ppgstock.obj
 0001:00054a20       ??0COleClientItem@@QAE@PAVCOleDocument@@@Z 5f555a20 f   olecli1.obj
 0001:00054bb3       ??1COleClientItem@@UAE@XZ  5f555bb3 f   olecli1.obj
 0001:00054c44       ?Delete@COleClientItem@@QAEXH@Z 5f555c44 f   olecli1.obj
 0001:00054d68       ?Release@COleClientItem@@UAEXW4tagOLECLOSE@@@Z 5f555d68 f   olecli1.obj
 0001:00054fe3       ?Close@COleClientItem@@QAEXW4tagOLECLOSE@@@Z 5f555fe3 f   olecli1.obj
 0001:000550f2       ?GetNewItemNumber@COleClientItem@@QAEKXZ 5f5560f2 f   olecli1.obj
 0001:00055190       ?GetItemName@COleClientItem@@QBEXPAD@Z 5f556190 f   olecli1.obj
 0001:00055218       ?GetIconFromRegistry@COleClientItem@@QBEPAUHICON__@@XZ 5f556218 f   olecli1.obj
 0001:00055256       ?GetIconFromRegistry@COleClientItem@@SAPAUHICON__@@AAU_GUID@@@Z 5f556256 f   olecli1.obj
 0001:000555f7       ?UpdateItemType@COleClientItem@@QAEXXZ 5f5565f7 f   olecli1.obj
 0001:000556ae       ?FinishCreate@COleClientItem@@MAEHJ@Z 5f5566ae f   olecli1.obj
 0001:00055a9e       ?CreateFromClipboard@COleClientItem@@QAEHW4tagOLERENDER@@GPAUtagFORMATETC@@@Z 5f556a9e f   olecli1.obj
 0001:00055bd9       ?CreateLinkFromClipboard@COleClientItem@@QAEHW4tagOLERENDER@@GPAUtagFORMATETC@@@Z 5f556bd9 f   olecli1.obj
 0001:00055d14       ?CreateStaticFromClipboard@COleClientItem@@QAEHW4tagOLERENDER@@GPAUtagFORMATETC@@@Z 5f556d14 f   olecli1.obj
 0001:00055e4f       ?CreateFromData@COleClientItem@@QAEHPAVCOleDataObject@@W4tagOLERENDER@@GPAUtagFORMATETC@@@Z 5f556e4f f   olecli1.obj
 0001:00055fb7       ?CreateLinkFromData@COleClientItem@@QAEHPAVCOleDataObject@@W4tagOLERENDER@@GPAUtagFORMATETC@@@Z 5f556fb7 f   olecli1.obj
 0001:0005611f       ?CreateStaticFromData@COleClientItem@@QAEHPAVCOleDataObject@@W4tagOLERENDER@@GPAUtagFORMATETC@@@Z 5f55711f f   olecli1.obj
 0001:00056287       ?CreateFromFile@COleClientItem@@QAEHPBDABU_GUID@@W4tagOLERENDER@@GPAUtagFORMATETC@@@Z 5f557287 f   olecli1.obj
 0001:00056450       ?CreateLinkFromFile@COleClientItem@@QAEHPBDW4tagOLERENDER@@GPAUtagFORMATETC@@@Z 5f557450 f   olecli1.obj
 0001:00056615       ?CreateNewItem@COleClientItem@@QAEHABU_GUID@@W4tagOLERENDER@@GPAUtagFORMATETC@@@Z 5f557615 f   olecli1.obj
 0001:00056770       ?CreateCloneFrom@COleClientItem@@QAEHPBV1@@Z 5f557770 f   olecli1.obj
 0001:0005698f       ?IsModified@COleClientItem@@QBEHXZ 5f55798f f   olecli1.obj
 0001:00056aa3       ?GetItemStorageFlat@COleClientItem@@QAEXXZ 5f557aa3 f   olecli1.obj
 0001:00056bf2       ?ReadItemFlat@COleClientItem@@QAEXAAVCArchive@@@Z 5f557bf2 f   olecli1.obj
 0001:00056e7a       ?WriteItemFlat@COleClientItem@@QAEXAAVCArchive@@@Z 5f557e7a f   olecli1.obj
 0001:0005707f       ?GetItemStorageCompound@COleClientItem@@QAEXXZ 5f55807f f   olecli1.obj
 0001:0005725a       ?ReadItemCompound@COleClientItem@@QAEXAAVCArchive@@@Z 5f55825a f   olecli1.obj
 0001:000575ec       ?WriteItemCompound@COleClientItem@@QAEXAAVCArchive@@@Z 5f5585ec f   olecli1.obj
 0001:00057906       ?GetItemStorage@COleClientItem@@UAEXXZ 5f558906 f   olecli1.obj
 0001:00057931       ?ReadItem@COleClientItem@@UAEXAAVCArchive@@@Z 5f558931 f   olecli1.obj
 0001:00057966       ?WriteItem@COleClientItem@@UAEXAAVCArchive@@@Z 5f558966 f   olecli1.obj
 0001:0005799b       ?CommitItem@COleClientItem@@UAEXH@Z 5f55899b f   olecli1.obj
 0001:00057ada       ?Serialize@COleClientItem@@UAEXAAVCArchive@@@Z 5f558ada f   olecli1.obj
 0001:00057da6       ?OnChange@COleClientItem@@UAEXW4OLE_NOTIFICATION@@K@Z 5f558da6 f   olecli1.obj
 0001:00057e6e       ?OnDataChange@COleClientItem@@MAEXPAUtagFORMATETC@@PAUtagSTGMEDIUM@@@Z 5f558e6e f   olecli1.obj
 0001:00057ea4       ?OnGetItemPosition@COleClientItem@@MAEXAAVCRect@@@Z 5f558ea4 f   olecli1.obj
 0001:00057eb1       ?OnGetClipRect@COleClientItem@@MAEXAAVCRect@@@Z 5f558eb1 f   olecli1.obj
 0001:00057f27       ?OnShowItem@COleClientItem@@MAEXXZ 5f558f27 f   olecli1.obj
 0001:00058053       ?GetClassID@COleClientItem@@QBEXPAU_GUID@@@Z 5f559053 f   olecli1.obj
 0001:00058107       ?GetExtent@COleClientItem@@QAEHPAUtagSIZE@@W4tagDVASPECT@@@Z 5f559107 f   olecli1.obj
 0001:000581b6       ?GetCachedExtent@COleClientItem@@QAEHPAUtagSIZE@@W4tagDVASPECT@@@Z 5f5591b6 f   olecli1.obj
 0001:00058291       ?SetIconicMetafile@COleClientItem@@QAEHPAX@Z 5f559291 f   olecli1.obj
 0001:000583da       ?GetIconicMetafile@COleClientItem@@QAEPAXXZ 5f5593da f   olecli1.obj
 0001:0005871e       ?SetDrawAspect@COleClientItem@@UAEXW4tagDVASPECT@@@Z 5f55971e f   olecli1.obj
 0001:00058796       ?GetPrintDeviceInfo@COleClientItem@@IAEHPAPAUIOleCache@@PAPAUtagDVTARGETDEVICE@@PAK@Z 5f559796 f   olecli1.obj
 0001:000588c8       ?AttachDataObject@COleClientItem@@QBEXAAVCOleDataObject@@@Z 5f5598c8 f   olecli1.obj
 0001:00058955       ?Draw@COleClientItem@@QAEHPAVCDC@@PBUtagRECT@@W4tagDVASPECT@@@Z 5f559955 f   olecli1.obj
 0001:00058b37       ?GetEmbeddedItemData@COleClientItem@@IAEXPAUtagSTGMEDIUM@@@Z 5f559b37 f   olecli1.obj
 0001:00058cfd       ?AddCachedData@COleClientItem@@IAEXPAVCOleDataSource@@@Z 5f559cfd f   olecli1.obj
 0001:00058e9b       ?GetLinkSourceData@COleClientItem@@IAEHPAUtagSTGMEDIUM@@@Z 5f559e9b f   olecli1.obj
 0001:000590f6       ?GetObjectDescriptorData@COleClientItem@@IAEXPAUtagPOINT@@PAUtagSIZE@@PAUtagSTGMEDIUM@@@Z 5f55a0f6 f   olecli1.obj
 0001:000592c6       ?SetHostNames@COleClientItem@@QAEXPBD0@Z 5f55a2c6 f   olecli1.obj
 0001:00059441       ?SetExtent@COleClientItem@@QAEXABVCSize@@W4tagDVASPECT@@@Z 5f55a441 f   olecli1.obj
 0001:000594b3       ?_GetBaseInterfaceMap@COleClientItem@@KGPBUAFX_INTERFACEMAP@@XZ 5f55a4b3 f   olecli1.obj
 0001:000594bd       ?GetInterfaceMap@COleClientItem@@MBEPBUAFX_INTERFACEMAP@@XZ 5f55a4bd f   olecli1.obj
 0001:000594cd       ?AddRef@XOleClientSite@COleClientItem@@UAGKXZ 5f55a4cd f   olecli1.obj
 0001:000594e8       ?Release@XOleClientSite@COleClientItem@@UAGKXZ 5f55a4e8 f   olecli1.obj
 0001:00059503       ?QueryInterface@XOleClientSite@COleClientItem@@UAGJABU_GUID@@PAPAX@Z 5f55a503 f   olecli1.obj
 0001:00059526       ?SaveObject@XOleClientSite@COleClientItem@@UAGJXZ 5f55a526 f   olecli1.obj
 0001:00059638       ?GetMoniker@XOleClientSite@COleClientItem@@UAGJKKPAPAUIMoniker@@@Z 5f55a638 f   olecli1.obj
 0001:00059970       ?GetContainer@XOleClientSite@COleClientItem@@UAGJPAPAUIOleContainer@@@Z 5f55a970 f   olecli1.obj
 0001:00059a13       ?ShowObject@XOleClientSite@COleClientItem@@UAGJXZ 5f55aa13 f   olecli1.obj
 0001:00059ae9       ?OnShowWindow@XOleClientSite@COleClientItem@@UAGJH@Z 5f55aae9 f   olecli1.obj
 0001:00059c0c       ?RequestNewObjectLayout@XOleClientSite@COleClientItem@@UAGJXZ 5f55ac0c f   olecli1.obj
 0001:00059c18       ?AddRef@XAdviseSink@COleClientItem@@UAGKXZ 5f55ac18 f   olecli1.obj
 0001:00059c33       ?Release@XAdviseSink@COleClientItem@@UAGKXZ 5f55ac33 f   olecli1.obj
 0001:00059c4e       ?QueryInterface@XAdviseSink@COleClientItem@@UAGJABU_GUID@@PAPAX@Z 5f55ac4e f   olecli1.obj
 0001:00059c71       ?OnDataChange@XAdviseSink@COleClientItem@@UAGXPAUtagFORMATETC@@PAUtagSTGMEDIUM@@@Z 5f55ac71 f   olecli1.obj
 0001:00059cf3       ?OnViewChange@XAdviseSink@COleClientItem@@UAGXKJ@Z 5f55acf3 f   olecli1.obj
 0001:00059d70       ?OnRename@XAdviseSink@COleClientItem@@UAGXPAUIMoniker@@@Z 5f55ad70 f   olecli1.obj
 0001:00059d77       ?OnSave@XAdviseSink@COleClientItem@@UAGXXZ 5f55ad77 f   olecli1.obj
 0001:00059df2       ?OnClose@XAdviseSink@COleClientItem@@UAGXXZ 5f55adf2 f   olecli1.obj
 0001:00059e6d       ?AssertValid@COleClientItem@@UBEXXZ 5f55ae6d f   olecli1.obj
 0001:00059f03       ?Dump@COleClientItem@@UBEXAAVCDumpContext@@@Z 5f55af03 f   olecli1.obj
 0001:0005a0cc       ?GetLastStatus@COleClientItem@@QBEJXZ 5f55b0cc f   olecli1.obj
 0001:0005a0f0       ?GetDocument@COleClientItem@@QBEPAVCOleDocument@@XZ 5f55b0f0 f   olecli1.obj
 0001:0005a114       ?GetType@COleClientItem@@QBE?AW4OLE_OBJTYPE@@XZ 5f55b114 f   olecli1.obj
 0001:0005a138       ?GetDrawAspect@COleClientItem@@QBE?AW4tagDVASPECT@@XZ 5f55b138 f   olecli1.obj
 0001:0005a15c       ?IsRunning@COleClientItem@@QBEHXZ 5f55b15c f   olecli1.obj
 0001:0005a1b0       ?GetItemState@COleClientItem@@QBEIXZ 5f55b1b0 f   olecli1.obj
 0001:0005a1d4       ?IsInPlaceActive@COleClientItem@@QBEHXZ 5f55b1d4 f   olecli1.obj
 0001:0005a219       ?IsOpen@COleClientItem@@QBEHXZ 5f55b219 f   olecli1.obj
 0001:0005a243       ?IsLinkUpToDate@COleClientItem@@QBEHXZ 5f55b243 f   olecli1.obj
 0001:0005a2a1       ?GetActiveView@COleClientItem@@QBEPAVCView@@XZ 5f55b2a1 f   olecli1.obj
 0001:0005a2b2       ?BeginDeferErrors@COleLinkingDoc@@QAEXXZ 5f55b2b2 f   olecli1.obj
 0001:0005a2fe       ??1COleDataObject@@QAE@XZ  5f55b2fe f   olecli1.obj
 0001:0005a320       ??_GCOleClientItem@@UAEPAXI@Z 5f55b320 f i olecli1.obj
 0001:0005a320       ??_ECOleClientItem@@UAEPAXI@Z 5f55b320 f i olecli1.obj
 0001:0005a350       ??0XOleClientSite@COleClientItem@@QAE@XZ 5f55b350 f i olecli1.obj
 0001:0005a370       ??0XAdviseSink@COleClientItem@@QAE@XZ 5f55b370 f i olecli1.obj
 0001:0005a390       ??0XOleIPSite@COleClientItem@@QAE@XZ 5f55b390 f i olecli1.obj
 0001:0005a3b0       ??0IOleInPlaceSite@@QAE@XZ 5f55b3b0 f i olecli1.obj
 0001:0005a3d0       ??0IUnknown@@QAE@XZ        5f55b3d0 f i olecli1.obj
 0001:0005a3e0       ??0IOleWindow@@QAE@XZ      5f55b3e0 f i olecli1.obj
 0001:0005a3e0       ??0IOleClientSite@@QAE@XZ  5f55b3e0 f i olecli1.obj
 0001:0005a3e0       ??0IAdviseSink@@QAE@XZ     5f55b3e0 f i olecli1.obj
 0001:0005a400       ?GetClientSite@COleClientItem@@MAEPAUIOleClientSite@@XZ 5f55b400 f   olecli3.obj
 0001:0005a453       ?Activate@COleClientItem@@QAEXJPAVCView@@PAUtagMSG@@@Z 5f55b453 f   olecli3.obj
 0001:0005a5ec       ?CheckGeneral@COleClientItem@@MAEXJ@Z 5f55b5ec f   olecli3.obj
 0001:0005a64d       ?CopyToClipboard@COleClientItem@@QAEXH@Z 5f55b64d f   olecli3.obj
 0001:0005a744       ?OnGetClipboardData@COleClientItem@@UAEPAVCOleDataSource@@HPAUtagPOINT@@PAUtagSIZE@@@Z 5f55b744 f   olecli3.obj
 0001:0005a876       ?DoDragDrop@COleClientItem@@QAEKPBUtagRECT@@VCPoint@@HK0@Z 5f55b876 f   olecli3.obj
 0001:0005aa91       ?GetClipboardData@COleClientItem@@QAEXPAVCOleDataSource@@HPAUtagPOINT@@PAUtagSIZE@@@Z 5f55ba91 f   olecli3.obj
 0001:0005ab9b       ?CanPaste@COleClientItem@@SGHXZ 5f55bb9b f   olecli3.obj
 0001:0005ac42       ?CanPasteLink@COleClientItem@@SGHXZ 5f55bc42 f   olecli3.obj
 0001:0005ac9f       ?CanCreateFromData@COleClientItem@@SGHPBVCOleDataObject@@@Z 5f55bc9f f   olecli3.obj
 0001:0005acfd       ?CanCreateLinkFromData@COleClientItem@@SGHPBVCOleDataObject@@@Z 5f55bcfd f   olecli3.obj
 0001:0005ad5b       ?ConvertTo@COleClientItem@@UAEHABU_GUID@@@Z 5f55bd5b f   olecli3.obj
 0001:0005aebb       ?Reload@COleClientItem@@QAEHXZ 5f55bebb f   olecli3.obj
 0001:0005af6b       ?ActivateAs@COleClientItem@@UAEHPBDABU_GUID@@1@Z 5f55bf6b f   olecli3.obj
 0001:0005b06f       ?SetPrintDevice@COleClientItem@@QAEHPBUtagDVTARGETDEVICE@@@Z 5f55c06f f   olecli3.obj
 0001:0005b285       ?SetPrintDevice@COleClientItem@@QAEHPBUtagPDA@@@Z 5f55c285 f   olecli3.obj
 0001:0005b300       ?GetUserType@COleClientItem@@QAEXW4tagUSERCLASSTYPE@@AAVCString@@@Z 5f55c300 f   olecli3.obj
 0001:0005b3d3       ?Run@COleClientItem@@QAEXXZ 5f55c3d3 f   olecli3.obj
 0001:0005b47c       ?UpdateLink@COleClientItem@@QAEHXZ 5f55c47c f   olecli3.obj
 0001:0005b528       ?FreezeLink@COleClientItem@@UAEHXZ 5f55c528 f   olecli3.obj
 0001:0005b88f       ?GetLinkUpdateOptions@COleClientItem@@QAE?AW4tagOLEUPDATE@@XZ 5f55c88f f   olecli3.obj
 0001:0005b940       ?SetLinkUpdateOptions@COleClientItem@@QAEXW4tagOLEUPDATE@@@Z 5f55c940 f   olecli3.obj
 0001:0005b9f0       ??0COleDocument@@QAE@XZ    5f55c9f0 f   oledoc1.obj
 0001:0005bb4f       ??1COleDocument@@UAE@XZ    5f55cb4f f   oledoc1.obj
 0001:0005bc91       ?AddItem@COleDocument@@UAEXPAVCDocItem@@@Z 5f55cc91 f   oledoc1.obj
 0001:0005bd14       ?RemoveItem@COleDocument@@UAEXPAVCDocItem@@@Z 5f55cd14 f   oledoc1.obj
 0001:0005be00       ?GetStartPosition@COleDocument@@UBEPAU__POSITION@@XZ 5f55ce00 f   oledoc1.obj
 0001:0005be26       ?GetNextItem@COleDocument@@UBEPAVCDocItem@@AAPAU__POSITION@@@Z 5f55ce26 f   oledoc1.obj
 0001:0005bed6       ?GetNextItemOfKind@COleDocument@@IBEPAVCDocItem@@AAPAU__POSITION@@PAUCRuntimeClass@@@Z 5f55ced6 f   oledoc1.obj
 0001:0005bf2e       ?GetNextClientItem@COleDocument@@QBEPAVCOleClientItem@@AAPAU__POSITION@@@Z 5f55cf2e f   oledoc1.obj
 0001:0005bf54       ?GetNextServerItem@COleDocument@@QBEPAVCOleServerItem@@AAPAU__POSITION@@@Z 5f55cf54 f   oledoc1.obj
 0001:0005bf7a       ?DeleteContents@COleDocument@@UAEXXZ 5f55cf7a f   oledoc1.obj
 0001:0005bfdf       ?SetPathName@COleDocument@@UAEXPBDH@Z 5f55cfdf f   oledoc1.obj
 0001:0005c106       ?Serialize@COleDocument@@UAEXAAVCArchive@@@Z 5f55d106 f   oledoc1.obj
 0001:0005c22e       ?CommitItems@COleDocument@@QAEXH@Z 5f55d22e f   oledoc1.obj
 0001:0005c277       ?HasBlankItems@COleDocument@@QBEHXZ 5f55d277 f   oledoc1.obj
 0001:0005c2f0       ?UpdateModifiedFlag@COleDocument@@UAEXXZ 5f55d2f0 f   oledoc1.obj
 0001:0005c353       ?PreCloseFrame@COleDocument@@UAEXPAVCFrameWnd@@@Z 5f55d353 f   oledoc1.obj
 0001:0005c42c       ?SaveModified@COleDocument@@UAEHXZ 5f55d42c f   oledoc1.obj
 0001:0005c5b3       ?OnShowViews@COleDocument@@UAEXH@Z 5f55d5b3 f   oledoc1.obj
 0001:0005c5c0       ?OnIdle@COleDocument@@UAEXXZ 5f55d5c0 f   oledoc1.obj
 0001:0005c680       ?GetFirstFrame@COleDocument@@QAEPAVCFrameWnd@@XZ 5f55d680 f   oledoc1.obj
 0001:0005c731       ?GetMoniker@COleDocument@@UAEPAUIMoniker@@W4tagOLEGETMONIKER@@@Z 5f55d731 f   oledoc1.obj
 0001:0005c7e9       ?GetContainer@COleDocument@@UAEPAUIOleItemContainer@@XZ 5f55d7e9 f   oledoc1.obj
 0001:0005c7f6       ?OnNewDocument@COleDocument@@UAEHXZ 5f55d7f6 f   oledoc1.obj
 0001:0005c8a7       ?OnOpenDocument@COleDocument@@UAEHPBD@Z 5f55d8a7 f   oledoc1.obj
 0001:0005cc62       ?OnSaveDocument@COleDocument@@UAEHPBD@Z 5f55dc62 f   oledoc1.obj
 0001:0005d04c       ?OnCloseDocument@COleDocument@@UAEXXZ 5f55e04c f   oledoc1.obj
 0001:0005d0d0       ?SaveToStorage@COleDocument@@MAEXPAVCObject@@@Z 5f55e0d0 f   oledoc1.obj
 0001:0005d2d1       ?LoadFromStorage@COleDocument@@MAEXXZ 5f55e2d1 f   oledoc1.obj
 0001:0005d4ba       ?AssertValid@COleDocument@@UBEXXZ 5f55e4ba f   oledoc1.obj
 0001:0005d562       ?Dump@COleDocument@@UBEXAAVCDumpContext@@@Z 5f55e562 f   oledoc1.obj
 0001:0005d67a       ??0CDocItem@@IAE@XZ        5f55e67a f   oledoc1.obj
 0001:0005d6a3       ??1CDocItem@@UAE@XZ        5f55e6a3 f   oledoc1.obj
 0001:0005d715       ?Serialize@CDocItem@@UAEXAAVCArchive@@@Z 5f55e715 f   oledoc1.obj
 0001:0005d7ea       ?IsBlank@CDocItem@@UBEHXZ  5f55e7ea f   oledoc1.obj
 0001:0005d7f7       ?AssertValid@CDocItem@@UBEXXZ 5f55e7f7 f   oledoc1.obj
 0001:0005d824       ?Dump@CDocItem@@UBEXAAVCDumpContext@@@Z 5f55e824 f   oledoc1.obj
 0001:0005d865       ?GetDocument@CDocItem@@QBEPAVCDocument@@XZ 5f55e865 f   oledoc1.obj
 0001:0005d876       ?EnableCompoundFile@COleDocument@@QAEXH@Z 5f55e876 f   oledoc1.obj
 0001:0005d88c       ?SetBusyReply@COleMessageFilter@@QAEXW4tagSERVERCALL@@@Z 5f55e88c f   oledoc1.obj
 0001:0005d8b2       ?SetRetryReply@COleMessageFilter@@QAEXK@Z 5f55e8b2 f   oledoc1.obj
 0001:0005d8d8       ?SetMessagePendingDelay@COleMessageFilter@@QAEXK@Z 5f55e8d8 f   oledoc1.obj
 0001:0005d8fe       ?EnableBusyDialog@COleMessageFilter@@QAEXH@Z 5f55e8fe f   oledoc1.obj
 0001:0005d924       ?EnableNotRespondingDialog@COleMessageFilter@@QAEXH@Z 5f55e924 f   oledoc1.obj
 0001:0005d950       ??_ECOleDocument@@UAEPAXI@Z 5f55e950 f i oledoc1.obj
 0001:0005d950       ??_GCOleDocument@@UAEPAXI@Z 5f55e950 f i oledoc1.obj
 0001:0005d980       ??_GCDocItem@@UAEPAXI@Z    5f55e980 f i oledoc1.obj
 0001:0005d980       ??_ECDocItem@@UAEPAXI@Z    5f55e980 f i oledoc1.obj
 0001:0005d9b0       ?ApplyPrintDevice@COleDocument@@QAEHPBUtagDVTARGETDEVICE@@@Z 5f55e9b0 f   oledoc2.obj
 0001:0005da7e       ?ApplyPrintDevice@COleDocument@@QAEHPBUtagPDA@@@Z 5f55ea7e f   oledoc2.obj
 0001:0005db10       ?AfxGetScodeString@@YGPBDJ@Z 5f55eb10 f   olemisc.obj
 0001:0005db54       ?AfxGetScodeRangeString@@YGPBDJ@Z 5f55eb54 f   olemisc.obj
 0001:0005dbaa       ?AfxGetSeverityString@@YGPBDJ@Z 5f55ebaa f   olemisc.obj
 0001:0005dbc1       ?AfxGetFacilityString@@YGPBDJ@Z 5f55ebc1 f   olemisc.obj
 0001:0005dbf2       ?AfxGetFullScodeString@@YGPBDJ@Z 5f55ebf2 f   olemisc.obj
 0001:0005dc8a       ?AfxThrowOleException@@YGXJ@Z 5f55ec8a f   olemisc.obj
 0001:0005dd31       ?GetErrorMessage@COleException@@UAEHPADIPAI@Z 5f55ed31 f   olemisc.obj
 0001:0005ddd6       ?Process@COleException@@SGJPBVCException@@@Z 5f55edd6 f   olemisc.obj
 0001:0005de3d       ?AfxMergeMenus@@YGPAUHMENU__@@PAU1@0PAJHH@Z 5f55ee3d f   olemisc.obj
 0001:0005e1e9       ?AfxUnmergeMenus@@YGXPAUHMENU__@@00@Z 5f55f1e9 f   olemisc.obj
 0001:0005e381       ?_AfxFillFormatEtc@@YGPAUtagFORMATETC@@PAU1@G0@Z 5f55f381 f   olemisc.obj
 0001:0005e3fc       ?_AfxCopyGlobalMemory@@YGPAXPAX0@Z 5f55f3fc f   olemisc.obj
 0001:0005e4fd       ?_AfxCopyStgMedium@@YGHGPAUtagSTGMEDIUM@@0@Z 5f55f4fd f   olemisc.obj
 0001:0005ec11       ?_AfxOleGetObjectDescriptorData@@YGPAXU_GUID@@KUtagSIZE@@U_POINTL@@KPBG3@Z 5f55fc11 f   olemisc.obj
 0001:0005ed8c       ?_AfxOleGetObjectDescriptorData@@YGPAXPAUIOleObject@@PBGKU_POINTL@@PAUtagSIZE@@@Z 5f55fd8c f   olemisc.obj
 0001:0005f1a4       ?_AfxOleDoConvert@@YGJPAUIStorage@@ABU_GUID@@@Z 5f5601a4 f   olemisc.obj
 0001:0005f30c       ?_AfxOleDoTreatAsClass@@YGJPBDABU_GUID@@1@Z 5f56030c f   olemisc.obj
 0001:0005f3b8       ?_AfxOleCreateTargetDevice@@YGPAUtagDVTARGETDEVICE@@PAUtagDEVNAMES@@PAU_devicemodeA@@@Z 5f5603b8 f   olemisc.obj
 0001:0005f72e       ?_AfxOleCreateTargetDevice@@YGPAUtagDVTARGETDEVICE@@PAUtagPDA@@@Z 5f56072e f   olemisc.obj
 0001:0005f7af       ?_AfxOleGetFirstMoniker@@YGPAUIMoniker@@PAU1@@Z 5f5607af f   olemisc.obj
 0001:0005f887       ?_AfxOleGetLenFilePrefixOfMoniker@@YGKPAUIMoniker@@@Z 5f560887 f   olemisc.obj
 0001:0005f9f2       ?_AfxOleCopyTargetDevice@@YGPAUtagDVTARGETDEVICE@@PAU1@@Z 5f5609f2 f   olemisc.obj
 0001:0005fa38       ?_AfxOleCopyFormatEtc@@YGXPAUtagFORMATETC@@0@Z 5f560a38 f   olemisc.obj
 0001:0005fac7       ?_AfxOleCreateDC@@YGPAUHDC__@@PAUtagDVTARGETDEVICE@@@Z 5f560ac7 f   olemisc.obj
 0001:0005fc93       ?_AfxDeleteMetafilePict@@YGXPAX@Z 5f560c93 f   olemisc.obj
 0001:0005fcc3       ?_AfxXformSizeInPixelsToHimetric@@YGXPAUHDC__@@PAUtagSIZE@@1@Z 5f560cc3 f   olemisc.obj
 0001:0005fd52       ?_AfxXformSizeInHimetricToPixels@@YGXPAUHDC__@@PAUtagSIZE@@1@Z 5f560d52 f   olemisc.obj
 0001:0005fdf0       ??0COleStreamFile@@QAE@PAUIStream@@@Z 5f560df0 f   olestrm.obj
 0001:0005ff65       ??1COleStreamFile@@UAE@XZ  5f560f65 f   olestrm.obj
 0001:0005fffd       ?Detach@COleStreamFile@@QAEPAUIStream@@XZ 5f560ffd f   olestrm.obj
 0001:00060020       ?Attach@COleStreamFile@@QAEXPAUIStream@@@Z 5f561020 f   olestrm.obj
 0001:00060083       ?_AfxReadFromStream@@YGJPAUIStream@@PAXIAAK@Z 5f561083 f   olestrm.obj
 0001:0006010b       ?_AfxFillOleFileException@@YGXPAVCFileException@@J@Z 5f56110b f   olestrm.obj
 0001:00060233       ?_AfxThrowOleFileException@@YGXJ@Z 5f561233 f   olestrm.obj
 0001:000602a6       ?GetStatus@COleStreamFile@@QBEHAAUCFileStatus@@@Z 5f5612a6 f   olestrm.obj
 0001:0006042a       ?GetStorageName@COleStreamFile@@UBE?BVCString@@XZ 5f56142a f   olestrm.obj
 0001:0006046e       ?GetPosition@COleStreamFile@@UBEKXZ 5f56146e f   olestrm.obj
 0001:0006051a       ?OpenStream@COleStreamFile@@QAEHPAUIStorage@@PBDKPAVCFileException@@@Z 5f56151a f   olestrm.obj
 0001:000606b6       ?CreateStream@COleStreamFile@@QAEHPAUIStorage@@PBDKPAVCFileException@@@Z 5f5616b6 f   olestrm.obj
 0001:00060922       ?CreateMemoryStream@COleStreamFile@@QAEHPAVCFileException@@@Z 5f561922 f   olestrm.obj
 0001:000609da       ?Duplicate@COleStreamFile@@UBEPAVCFile@@XZ 5f5619da f   olestrm.obj
 0001:00060b68       ?Seek@COleStreamFile@@UAEJJI@Z 5f561b68 f   olestrm.obj
 0001:00060c44       ?SetLength@COleStreamFile@@UAEXK@Z 5f561c44 f   olestrm.obj
 0001:00060cc8       ?GetLength@COleStreamFile@@UBEKXZ 5f561cc8 f   olestrm.obj
 0001:00060d5e       ?Read@COleStreamFile@@UAEIPAXI@Z 5f561d5e f   olestrm.obj
 0001:00060dd6       ?Write@COleStreamFile@@UAEXPBXI@Z 5f561dd6 f   olestrm.obj
 0001:00060ea8       ?LockRange@COleStreamFile@@UAEXKK@Z 5f561ea8 f   olestrm.obj
 0001:00060f43       ?UnlockRange@COleStreamFile@@UAEXKK@Z 5f561f43 f   olestrm.obj
 0001:00060fde       ?Abort@COleStreamFile@@UAEXXZ 5f561fde f   olestrm.obj
 0001:0006104d       ?Flush@COleStreamFile@@UAEXXZ 5f56204d f   olestrm.obj
 0001:000610bc       ?Close@COleStreamFile@@UAEXXZ 5f5620bc f   olestrm.obj
 0001:00061124       ?GetStream@COleStreamFile@@QBEPAUIStream@@XZ 5f562124 f   olestrm.obj
 0001:00061135       ?AssertValid@COleStreamFile@@UBEXXZ 5f562135 f   olestrm.obj
 0001:00061148       ?Dump@COleStreamFile@@UBEXAAVCDumpContext@@@Z 5f562148 f   olestrm.obj
 0001:000611b0       ??_GCOleStreamFile@@UAEPAXI@Z 5f5621b0 f i olestrm.obj
 0001:000611e0       ?AfxGetIIDString@@YGPBDABU_GUID@@@Z 5f5621e0 f   oleunk.obj
 0001:000612a6       ?_AfxQueryInterface@@YGPAUIUnknown@@PAU1@ABU_GUID@@@Z 5f5622a6 f   oleunk.obj
 0001:000612fb       ?_AfxRelease@@YGKPAPAUIUnknown@@@Z 5f5622fb f   oleunk.obj
 0001:00061356       ?EnableAggregation@CCmdTarget@@QAEXXZ 5f562356 f   oleunk.obj
 0001:00061387       ?ExternalAddRef@CCmdTarget@@QAEKXZ 5f562387 f   oleunk.obj
 0001:000613b7       ?InternalRelease@CCmdTarget@@QAEKXZ 5f5623b7 f   oleunk.obj
 0001:00061468       ?ExternalRelease@CCmdTarget@@QAEKXZ 5f562468 f   oleunk.obj
 0001:00061498       ?GetInterface@CCmdTarget@@QAEPAUIUnknown@@PBX@Z 5f562498 f   oleunk.obj
 0001:00061665       ?QueryAggregates@CCmdTarget@@QAEPAUIUnknown@@PBX@Z 5f562665 f   oleunk.obj
 0001:0006174a       ?InternalQueryInterface@CCmdTarget@@QAEKPBXPAPAX@Z 5f56274a f   oleunk.obj
 0001:0006179e       ?ExternalQueryInterface@CCmdTarget@@QAEKPBXPAPAX@Z 5f56279e f   oleunk.obj
 0001:000617df       ?AddRef@CInnerUnknown@@UAGKXZ 5f5627df f   oleunk.obj
 0001:000617fa       ?Release@CInnerUnknown@@UAGKXZ 5f5627fa f   oleunk.obj
 0001:00061861       ?QueryInterface@CInnerUnknown@@UAGJABU_GUID@@PAPAX@Z 5f562861 f   oleunk.obj
 0001:000618ad       ?ExternalDisconnect@CCmdTarget@@QAEXXZ 5f5628ad f   oleunk.obj
 0001:0006191e       ?GetControllingUnknown@CCmdTarget@@QAEPAUIUnknown@@XZ 5f56291e f   oleunk.obj
 0001:0006194f       ??0COleException@@QAE@XZ   5f56294f f   oleunk.obj
 0001:00061978       ??1COleException@@UAE@XZ   5f562978 f   oleunk.obj
 0001:00061994       ?InternalAddRef@CCmdTarget@@QAEKXZ 5f562994 f   oleunk.obj
 0001:000619d8       ?IsRegistered@COleObjectFactory@@UBEHXZ 5f5629d8 f   oleunk.obj
 0001:000619ff       ?GetClassID@COleObjectFactory@@QBEABU_GUID@@XZ 5f5629ff f   oleunk.obj
 0001:00061a20       ??1COleDispatchDriver@@QAE@XZ 5f562a20 f   oleunk.obj
 0001:00061a33       ??BCOleDispatchDriver@@QAEPAUIDispatch@@XZ 5f562a33 f   oleunk.obj
 0001:00061a43       ??0COleVariant@@QAE@XZ     5f562a43 f   oleunk.obj
 0001:00061a5a       ??1COleVariant@@QAE@XZ     5f562a5a f   oleunk.obj
 0001:00061a90       ?Clear@COleVariant@@QAEXXZ 5f562a90 f   oleunk.obj
 0001:00061ac6       ??0COleVariant@@QAE@PBD@Z  5f562ac6 f   oleunk.obj
 0001:00061aea       ??0COleVariant@@QAE@AAVCString@@@Z 5f562aea f   oleunk.obj
 0001:00061b0e       ??0COleVariant@@QAE@E@Z    5f562b0e f   oleunk.obj
 0001:00061b2f       ??0COleVariant@@QAE@ABVCOleCurrency@@@Z 5f562b2f f   oleunk.obj
 0001:00061b58       ??0COleVariant@@QAE@M@Z    5f562b58 f   oleunk.obj
 0001:00061b79       ??0COleVariant@@QAE@N@Z    5f562b79 f   oleunk.obj
 0001:00061ba0       ??0COleVariant@@QAE@ABVCOleDateTime@@@Z 5f562ba0 f   oleunk.obj
 0001:00061bc9       ??0COleVariant@@QAE@ABVCByteArray@@@Z 5f562bc9 f   oleunk.obj
 0001:00061bed       ??0COleVariant@@QAE@ABVCLongBinary@@@Z 5f562bed f   oleunk.obj
 0001:00061c11       ??8COleVariant@@QBEHPBUtagVARIANT@@@Z 5f562c11 f   oleunk.obj
 0001:00061c2a       ??BCOleVariant@@QAEPAUtagVARIANT@@XZ 5f562c2a f   oleunk.obj
 0001:00061c38       ??BCOleVariant@@QBEPBUtagVARIANT@@XZ 5f562c38 f   oleunk.obj
 0001:00061c46       ??0COleCurrency@@QAE@XZ    5f562c46 f   oleunk.obj
 0001:00061c71       ??0COleCurrency@@QAE@TtagCY@@@Z 5f562c71 f   oleunk.obj
 0001:00061c99       ??0COleCurrency@@QAE@ABV0@@Z 5f562c99 f   oleunk.obj
 0001:00061cc5       ??0COleCurrency@@QAE@ABUtagVARIANT@@@Z 5f562cc5 f   oleunk.obj
 0001:00061ce1       ?GetStatus@COleCurrency@@QBE?AW4CurrencyStatus@1@XZ 5f562ce1 f   oleunk.obj
 0001:00061cf2       ?SetStatus@COleCurrency@@QAEXW4CurrencyStatus@1@@Z 5f562cf2 f   oleunk.obj
 0001:00061d08       ??YCOleCurrency@@QAEABV0@ABV0@@Z 5f562d08 f   oleunk.obj
 0001:00061d33       ??ZCOleCurrency@@QAEABV0@ABV0@@Z 5f562d33 f   oleunk.obj
 0001:00061d5e       ??XCOleCurrency@@QAEABV0@J@Z 5f562d5e f   oleunk.obj
 0001:00061d89       ??_0COleCurrency@@QAEABV0@J@Z 5f562d89 f   oleunk.obj
 0001:00061db4       ??8COleCurrency@@QBEHABV0@@Z 5f562db4 f   oleunk.obj
 0001:00061dfe       ??9COleCurrency@@QBEHABV0@@Z 5f562dfe f   oleunk.obj
 0001:00061e48       ??BCOleCurrency@@QBE?ATtagCY@@XZ 5f562e48 f   oleunk.obj
 0001:00061e68       ??0COleDateTime@@QAE@XZ    5f562e68 f   oleunk.obj
 0001:00061e90       ??0COleDateTime@@QAE@ABV0@@Z 5f562e90 f   oleunk.obj
 0001:00061ebc       ??0COleDateTime@@QAE@ABUtagVARIANT@@@Z 5f562ebc f   oleunk.obj
 0001:00061ed8       ??0COleDateTime@@QAE@N@Z   5f562ed8 f   oleunk.obj
 0001:00061f00       ??0COleDateTime@@QAE@J@Z   5f562f00 f   oleunk.obj
 0001:00061f1c       ??0COleDateTime@@QAE@ABU_SYSTEMTIME@@@Z 5f562f1c f   oleunk.obj
 0001:00061f38       ??0COleDateTime@@QAE@ABU_FILETIME@@@Z 5f562f38 f   oleunk.obj
 0001:00061f54       ??0COleDateTime@@QAE@HHHHHH@Z 5f562f54 f   oleunk.obj
 0001:00061f84       ??0COleDateTime@@QAE@GG@Z  5f562f84 f   oleunk.obj
 0001:00061fb3       ??4COleDateTime@@QAEABV0@ABV0@@Z 5f562fb3 f   oleunk.obj
 0001:00061fdf       ?GetStatus@COleDateTime@@QBE?AW4DateTimeStatus@1@XZ 5f562fdf f   oleunk.obj
 0001:00061ff0       ?SetStatus@COleDateTime@@QAEXW4DateTimeStatus@1@@Z 5f562ff0 f   oleunk.obj
 0001:00062006       ??8COleDateTime@@QBEHABV0@@Z 5f563006 f   oleunk.obj
 0001:00062047       ??9COleDateTime@@QBEHABV0@@Z 5f563047 f   oleunk.obj
 0001:00062088       ??YCOleDateTime@@QAEABV0@VCOleDateTimeSpan@@@Z 5f563088 f   oleunk.obj
 0001:000620b3       ??ZCOleDateTime@@QAEABV0@VCOleDateTimeSpan@@@Z 5f5630b3 f   oleunk.obj
 0001:000620de       ??BCOleDateTime@@QBENXZ    5f5630de f   oleunk.obj
 0001:000620ee       ?SetDate@COleDateTime@@QAEHHHH@Z 5f5630ee f   oleunk.obj
 0001:00062115       ?SetTime@COleDateTime@@QAEHHHH@Z 5f563115 f   oleunk.obj
 0001:0006213f       ??0COleDateTimeSpan@@QAE@XZ 5f56313f f   oleunk.obj
 0001:00062167       ??0COleDateTimeSpan@@QAE@N@Z 5f563167 f   oleunk.obj
 0001:0006218f       ??0COleDateTimeSpan@@QAE@ABV0@@Z 5f56318f f   oleunk.obj
 0001:000621bb       ??0COleDateTimeSpan@@QAE@JHHH@Z 5f5631bb f   oleunk.obj
 0001:000621e3       ?GetStatus@COleDateTimeSpan@@QBE?AW4DateTimeSpanStatus@1@XZ 5f5631e3 f   oleunk.obj
 0001:000621f4       ?SetStatus@COleDateTimeSpan@@QAEXW4DateTimeSpanStatus@1@@Z 5f5631f4 f   oleunk.obj
 0001:0006220a       ?GetTotalDays@COleDateTimeSpan@@QBENXZ 5f56320a f   oleunk.obj
 0001:00062246       ?GetTotalHours@COleDateTimeSpan@@QBENXZ 5f563246 f   oleunk.obj
 0001:0006229b       ?GetTotalMinutes@COleDateTimeSpan@@QBENXZ 5f56329b f   oleunk.obj
 0001:000622f6       ?GetTotalSeconds@COleDateTimeSpan@@QBENXZ 5f5632f6 f   oleunk.obj
 0001:00062357       ?GetDays@COleDateTimeSpan@@QBEJXZ 5f563357 f   oleunk.obj
 0001:00062398       ??8COleDateTimeSpan@@QBEHABV0@@Z 5f563398 f   oleunk.obj
 0001:000623d9       ??9COleDateTimeSpan@@QBEHABV0@@Z 5f5633d9 f   oleunk.obj
 0001:0006241a       ??MCOleDateTimeSpan@@QBEHABV0@@Z 5f56341a f   oleunk.obj
 0001:0006249f       ??OCOleDateTimeSpan@@QBEHABV0@@Z 5f56349f f   oleunk.obj
 0001:00062524       ??NCOleDateTimeSpan@@QBEHABV0@@Z 5f563524 f   oleunk.obj
 0001:000625a9       ??PCOleDateTimeSpan@@QBEHABV0@@Z 5f5635a9 f   oleunk.obj
 0001:0006262e       ??YCOleDateTimeSpan@@QAEABV0@V0@@Z 5f56362e f   oleunk.obj
 0001:00062659       ??ZCOleDateTimeSpan@@QAEABV0@V0@@Z 5f563659 f   oleunk.obj
 0001:00062684       ??GCOleDateTimeSpan@@QBE?AV0@XZ 5f563684 f   oleunk.obj
 0001:000626a9       ??BCOleDateTimeSpan@@QBENXZ 5f5636a9 f   oleunk.obj
 0001:000626b9       ??0COleSafeArray@@QAE@XZ   5f5636b9 f   oleunk.obj
 0001:000626d8       ??1COleSafeArray@@QAE@XZ   5f5636d8 f   oleunk.obj
 0001:000626eb       ?Clear@COleSafeArray@@QAEXXZ 5f5636eb f   oleunk.obj
 0001:00062724       ??BCOleSafeArray@@QAEPAUtagVARIANT@@XZ 5f563724 f   oleunk.obj
 0001:00062732       ??BCOleSafeArray@@QBEPBUtagVARIANT@@XZ 5f563732 f   oleunk.obj
 0001:00062740       ?GetDim@COleSafeArray@@QAEKXZ 5f563740 f   oleunk.obj
 0001:00062758       ?GetElemSize@COleSafeArray@@QAEKXZ 5f563758 f   oleunk.obj
 0001:00062770       ??0CInnerUnknown@@QAE@XZ   5f563770 f i oleunk.obj
 0001:00062790       ??_ECOleException@@UAEPAXI@Z 5f563790 f i oleunk.obj
 0001:00062790       ??_GCOleException@@UAEPAXI@Z 5f563790 f i oleunk.obj
 0001:000627c0       ??1CMonikerFile@@UAE@XZ    5f5637c0 f   olemon.obj
 0001:00062833       ?Flush@CMonikerFile@@UAEXXZ 5f563833 f   olemon.obj
 0001:00062898       ?Open@CMonikerFile@@MAEHPBDPAUIBindHost@@PAUIBindStatusCallback@@PAUIBindCtx@@PAVCFileException@@@Z 5f563898 f   olemon.obj
 0001:000628df       ?Attach@CMonikerFile@@IAEHPBDPAUIBindHost@@PAUIBindStatusCallback@@PAUIBindCtx@@PAVCFileException@@@Z 5f5638df f   olemon.obj
 0001:00062b1d       ?Open@CMonikerFile@@UAEHPBDPAVCFileException@@@Z 5f563b1d f   olemon.obj
 0001:00062bc5       ?Open@CMonikerFile@@UAEHPAUIMoniker@@PAVCFileException@@@Z 5f563bc5 f   olemon.obj
 0001:00062c75       ?Open@CMonikerFile@@MAEHPAUIMoniker@@PAUIBindHost@@PAUIBindStatusCallback@@PAUIBindCtx@@PAVCFileException@@@Z 5f563c75 f   olemon.obj
 0001:00062ca9       ?Attach@CMonikerFile@@IAEHPAUIMoniker@@PAUIBindHost@@PAUIBindStatusCallback@@PAUIBindCtx@@PAVCFileException@@@Z 5f563ca9 f   olemon.obj
 0001:00062e2f       ?Close@CMonikerFile@@UAEXXZ 5f563e2f f   olemon.obj
 0001:00062e5c       ?Detach@CMonikerFile@@QAEHPAVCFileException@@@Z 5f563e5c f   olemon.obj
 0001:00062f6d       ?CreateBindHost@CMonikerFile@@KAPAUIBindHost@@XZ 5f563f6d f   olemon.obj
 0001:00062ff0       ?CreateBindContext@CMonikerFile@@IAEPAUIBindCtx@@PAVCFileException@@@Z 5f563ff0 f   olemon.obj
 0001:00062fff       ?PostBindToStream@CMonikerFile@@MAEHPAVCFileException@@@Z 5f563fff f   olemon.obj
 0001:000630bc       ?AssertValid@CMonikerFile@@UBEXXZ 5f5640bc f   olemon.obj
 0001:000630cf       ?Dump@CMonikerFile@@UBEXAAVCDumpContext@@@Z 5f5640cf f   olemon.obj
 0001:00063115       ??0CMonikerFile@@QAE@XZ    5f564115 f   olemon.obj
 0001:0006316e       ?GetMoniker@CMonikerFile@@QBEPAUIMoniker@@XZ 5f56416e f   olemon.obj
 0001:00063194       ?GetBinding@CAsyncMonikerFile@@QBEPAUIBinding@@XZ 5f564194 f   olemon.obj
 0001:000631ba       ?SetBinding@CAsyncMonikerFile@@IAEXPAUIBinding@@@Z 5f5641ba f   olemon.obj
 0001:000631e6       ?SetFormatEtc@CAsyncMonikerFile@@IAEXPAUtagFORMATETC@@@Z 5f5641e6 f   olemon.obj
 0001:0006320c       ?GetFormatEtc@CAsyncMonikerFile@@QBEPAUtagFORMATETC@@XZ 5f56420c f   olemon.obj
 0001:00063230       ??_GCMonikerFile@@UAEPAXI@Z 5f564230 f i olemon.obj
 0001:00063260       ??0_AfxBindHost@@QAE@XZ    5f564260 f i olemon.obj
 0001:00063290       ?AddRef@_AfxBindHost@@UAGKXZ 5f564290 f i olemon.obj
 0001:000632b0       ?Release@_AfxBindHost@@UAGKXZ 5f5642b0 f i olemon.obj
 0001:00063300       ?QueryInterface@_AfxBindHost@@UAGJABU_GUID@@PAPAX@Z 5f564300 f i olemon.obj
 0001:00063360       ?CreateMoniker@_AfxBindHost@@UAGJPAGPAUIBindCtx@@PAPAUIMoniker@@K@Z 5f564360 f i olemon.obj
 0001:000633d0       ?MonikerBindToStorage@_AfxBindHost@@UAGJPAUIMoniker@@PAUIBindCtx@@PAUIBindStatusCallback@@ABU_GUID@@PAPAX@Z 5f5643d0 f i olemon.obj
 0001:00063590       ?MonikerBindToObject@_AfxBindHost@@EAGJPAUIMoniker@@PAUIBindCtx@@PAUIBindStatusCallback@@ABU_GUID@@PAPAX@Z 5f564590 f i olemon.obj
 0001:000635d0       ??0IBindHost@@QAE@XZ       5f5645d0 f i olemon.obj
 0001:000635f0       ??_G_AfxBindHost@@QAEPAXI@Z 5f5645f0 f i olemon.obj
 0001:00063620       ??1_AfxBindHost@@QAE@XZ    5f564620 f i olemon.obj
 0001:00063660       ?_AfxTrySPForBindHost@@YGPAUIBindHost@@PAUIServiceProvider@@@Z 5f564660 f i oleasmon.obj
 0001:000636c0       ?_AfxTryQIForBindHost@@YGPAUIBindHost@@PAUIUnknown@@@Z 5f5646c0 f i oleasmon.obj
 0001:00063770       ??0CAsyncMonikerFile@@QAE@XZ 5f564770 f   oleasmon.obj
 0001:000637db       ??1CAsyncMonikerFile@@UAE@XZ 5f5647db f   oleasmon.obj
 0001:0006383b       ?EndCallbacks@CAsyncMonikerFile@@IAEXXZ 5f56483b f   oleasmon.obj
 0001:000638a6       ?Read@CAsyncMonikerFile@@UAEIPAXI@Z 5f5648a6 f   oleasmon.obj
 0001:00063930       ?Close@CAsyncMonikerFile@@UAEXXZ 5f564930 f   oleasmon.obj
 0001:0006399d       ?Open@CAsyncMonikerFile@@UAEHPAUIMoniker@@PAUIBindHost@@PAVCFileException@@@Z 5f56499d f   oleasmon.obj
 0001:00063ad5       ?Open@CAsyncMonikerFile@@UAEHPBDPAUIBindHost@@PAVCFileException@@@Z 5f564ad5 f   oleasmon.obj
 0001:00063c0d       ?Open@CAsyncMonikerFile@@UAEHPBDPAVCFileException@@@Z 5f564c0d f   oleasmon.obj
 0001:00063c86       ?Open@CAsyncMonikerFile@@UAEHPAUIMoniker@@PAVCFileException@@@Z 5f564c86 f   oleasmon.obj
 0001:00063cff       ?Open@CAsyncMonikerFile@@UAEHPBDPAUIServiceProvider@@PAVCFileException@@@Z 5f564cff f   oleasmon.obj
 0001:00063dee       ?Open@CAsyncMonikerFile@@UAEHPBDPAUIUnknown@@PAVCFileException@@@Z 5f564dee f   oleasmon.obj
 0001:00063f27       ?Open@CAsyncMonikerFile@@UAEHPAUIMoniker@@PAUIServiceProvider@@PAVCFileException@@@Z 5f564f27 f   oleasmon.obj
 0001:0006401c       ?Open@CAsyncMonikerFile@@UAEHPAUIMoniker@@PAUIUnknown@@PAVCFileException@@@Z 5f56501c f   oleasmon.obj
 0001:00064160       ?PostBindToStream@CAsyncMonikerFile@@MAEHPAVCFileException@@@Z 5f565160 f   oleasmon.obj
 0001:00064192       ?CreateBindStatusCallback@CAsyncMonikerFile@@MAEPAUIUnknown@@PAU2@@Z 5f565192 f   oleasmon.obj
 0001:00064288       ?GetBindInfo@CAsyncMonikerFile@@MBEKXZ 5f565288 f   oleasmon.obj
 0001:00064298       ?GetPriority@CAsyncMonikerFile@@MBEJXZ 5f565298 f   oleasmon.obj
 0001:000642a5       ?OnDataAvailable@CAsyncMonikerFile@@MAEXKK@Z 5f5652a5 f   oleasmon.obj
 0001:000642b2       ?OnLowResource@CAsyncMonikerFile@@MAEXXZ 5f5652b2 f   oleasmon.obj
 0001:000642bd       ?OnStartBinding@CAsyncMonikerFile@@MAEXXZ 5f5652bd f   oleasmon.obj
 0001:000642c8       ?OnStopBinding@CAsyncMonikerFile@@MAEXJPBD@Z 5f5652c8 f   oleasmon.obj
 0001:000642d5       ?OnProgress@CAsyncMonikerFile@@MAEXKKKPBD@Z 5f5652d5 f   oleasmon.obj
 0001:000642e2       ?AssertValid@CAsyncMonikerFile@@UBEXXZ 5f5652e2 f   oleasmon.obj
 0001:000643b8       ?Dump@CAsyncMonikerFile@@UBEXAAVCDumpContext@@@Z 5f5653b8 f   oleasmon.obj
 0001:00064510       ??_GCAsyncMonikerFile@@UAEPAXI@Z 5f565510 f i oleasmon.obj
 0001:00064540       ?Orphan@_AfxBindStatusCallback@@QAEXXZ 5f565540 f i oleasmon.obj
 0001:00064560       ?GetInnerUnknown@_AfxBindStatusCallback@@QAEPAUIUnknown@@XZ 5f565560 f i oleasmon.obj
 0001:00064580       ??1?$CIP@UIUnknown@@$1?IID_IUnknown@@3U_GUID@@B@@QAE@XZ 5f565580 f i oleasmon.obj
 0001:000645a0       ??0_AfxBindStatusCallback@@QAE@PAVCAsyncMonikerFile@@PAUIUnknown@@@Z 5f5655a0 f i oleasmon.obj
 0001:00064670       ??0CInnerUnknown@_AfxBindStatusCallback@@QAE@XZ 5f565670 f i oleasmon.obj
 0001:00064690       ?SetpThis@CInnerUnknown@_AfxBindStatusCallback@@QAEXPAV2@@Z 5f565690 f i oleasmon.obj
 0001:000646d0       ?AddRef@CInnerUnknown@_AfxBindStatusCallback@@UAGKXZ 5f5656d0 f i oleasmon.obj
 0001:000646f0       ?Release@CInnerUnknown@_AfxBindStatusCallback@@UAGKXZ 5f5656f0 f i oleasmon.obj
 0001:00064750       ?QueryInterface@CInnerUnknown@_AfxBindStatusCallback@@UAGJABU_GUID@@PAPAX@Z 5f565750 f i oleasmon.obj
 0001:000647d0       ?AddRef@_AfxBindStatusCallback@@UAGKXZ 5f5657d0 f i oleasmon.obj
 0001:000647f0       ?Release@_AfxBindStatusCallback@@UAGKXZ 5f5657f0 f i oleasmon.obj
 0001:00064810       ?QueryInterface@_AfxBindStatusCallback@@UAGJABU_GUID@@PAPAX@Z 5f565810 f i oleasmon.obj
 0001:00064830       ?GetBindInfo@_AfxBindStatusCallback@@EAGJPAKPAU_tagBINDINFO@@@Z 5f565830 f i oleasmon.obj
 0001:00064990       ?OnStartBinding@_AfxBindStatusCallback@@EAGJKPAUIBinding@@@Z 5f565990 f i oleasmon.obj
 0001:00064ad0       ?GetPriority@_AfxBindStatusCallback@@EAGJPAJ@Z 5f565ad0 f i oleasmon.obj
 0001:00064c10       ?OnProgress@_AfxBindStatusCallback@@EAGJKKKPBG@Z 5f565c10 f i oleasmon.obj
 0001:00064db0       ?OnDataAvailable@_AfxBindStatusCallback@@EAGJKKPAUtagFORMATETC@@PAUtagSTGMEDIUM@@@Z 5f565db0 f i oleasmon.obj
 0001:00064fc0       ?OnLowResource@_AfxBindStatusCallback@@EAGJK@Z 5f565fc0 f i oleasmon.obj
 0001:000650f0       ?OnStopBinding@_AfxBindStatusCallback@@EAGJJPBG@Z 5f5660f0 f i oleasmon.obj
 0001:000652e0       ?OnObjectAvailable@_AfxBindStatusCallback@@EAGJABU_GUID@@PAUIUnknown@@@Z 5f5662e0 f i oleasmon.obj
 0001:00065370       ??_G_AfxBindStatusCallback@@QAEPAXI@Z 5f566370 f i oleasmon.obj
 0001:000653a0       ??1_AfxBindStatusCallback@@QAE@XZ 5f5663a0 f i oleasmon.obj
 0001:00065400       ??0IBindStatusCallback@@QAE@XZ 5f566400 f i oleasmon.obj
 0001:00065420       ?GetOwner@_AfxBindStatusCallback@@QBEPBVCAsyncMonikerFile@@XZ 5f566420 f i oleasmon.obj
 0001:00065440       ?GetRefcount@_AfxBindStatusCallback@@QBEKXZ 5f566440 f i oleasmon.obj
 0001:00065460       ?GetpThisOfInnerUnknown@_AfxBindStatusCallback@@QBEPBV1@XZ 5f566460 f i oleasmon.obj
 0001:00065480       ?GetModuleState@_AfxBindStatusCallback@@QBEPBVAFX_MODULE_STATE@@XZ 5f566480 f i oleasmon.obj
 0001:000654a0       ?GetControllingUnknown@_AfxBindStatusCallback@@QAEPAUIUnknown@@XZ 5f5664a0 f i oleasmon.obj
 0001:000654c0       ??0COleFrameHook@@QAE@PAVCFrameWnd@@PAVCOleClientItem@@@Z 5f5664c0 f   olecli2.obj
 0001:000655bc       ??1COleFrameHook@@UAE@XZ   5f5665bc f   olecli2.obj
 0001:0006565b       ?OnRecalcLayout@COleFrameHook@@UAEXXZ 5f56665b f   olecli2.obj
 0001:000656cc       ?OnDocActivate@COleFrameHook@@UAEHH@Z 5f5666cc f   olecli2.obj
 0001:000657d8       ?OnContextHelp@COleFrameHook@@UAEHH@Z 5f5667d8 f   olecli2.obj
 0001:00065824       ?OnMenuSelect@COleFrameHook@@UAEHIIPAUHMENU__@@@Z 5f566824 f   olecli2.obj
 0001:00065911       ?OnInitMenu@COleFrameHook@@UAEXPAVCMenu@@@Z 5f566911 f   olecli2.obj
 0001:0006594a       ?OnInitMenuPopup@COleFrameHook@@UAEHPAVCMenu@@HH@Z 5f56694a f   olecli2.obj
 0001:000659d5       ?OnPreTranslateMessage@COleFrameHook@@UAEHPAUtagMSG@@@Z 5f5669d5 f   olecli2.obj
 0001:00065abc       ?OnActivate@COleFrameHook@@UAEXH@Z 5f566abc f   olecli2.obj
 0001:00065b1a       ?OnEnableModeless@COleFrameHook@@UAEXH@Z 5f566b1a f   olecli2.obj
 0001:00065b64       ?OnUpdateFrameTitle@COleFrameHook@@UAEHXZ 5f566b64 f   olecli2.obj
 0001:00065bc7       ?OnPaletteChanged@COleFrameHook@@UAEXPAVCWnd@@@Z 5f566bc7 f   olecli2.obj
 0001:00065c02       ?OnQueryNewPalette@COleFrameHook@@UAEHXZ 5f566c02 f   olecli2.obj
 0001:00065c38       ?NotifyAllInPlace@COleFrameHook@@QAEHHP81@AEHH@Z@Z 5f566c38 f   olecli2.obj
 0001:00065dde       ?DoContextSensitiveHelp@COleFrameHook@@QAEHH@Z 5f566dde f   olecli2.obj
 0001:00065e46       ?DoEnableModeless@COleFrameHook@@QAEHH@Z 5f566e46 f   olecli2.obj
 0001:00065efe       ?CanActivate@COleClientItem@@MAEHXZ 5f566efe f   olecli2.obj
 0001:00066000       ?OnActivate@COleClientItem@@UAEXXZ 5f567000 f   olecli2.obj
 0001:00066064       ?OnActivateUI@COleClientItem@@UAEXXZ 5f567064 f   olecli2.obj
 0001:000661b3       ?OnShowControlBars@COleClientItem@@UAEHPAVCFrameWnd@@H@Z 5f5671b3 f   olecli2.obj
 0001:00066304       ?OnGetWindowContext@COleClientItem@@MAEHPAPAVCFrameWnd@@0PAUtagOIFI@@@Z 5f567304 f   olecli2.obj
 0001:0006651b       ?OnScrollBy@COleClientItem@@MAEHVCSize@@@Z 5f56751b f   olecli2.obj
 0001:000665b2       ?OnDeactivateUI@COleClientItem@@UAEXH@Z 5f5675b2 f   olecli2.obj
 0001:0006680d       ?OnDeactivate@COleClientItem@@UAEXXZ 5f56780d f   olecli2.obj
 0001:00066927       ?OnDiscardUndoState@COleClientItem@@MAEXXZ 5f567927 f   olecli2.obj
 0001:00066945       ?OnDeactivateAndUndo@COleClientItem@@MAEXXZ 5f567945 f   olecli2.obj
 0001:0006696b       ?OnChangeItemPosition@COleClientItem@@MAEHABVCRect@@@Z 5f56796b f   olecli2.obj
 0001:00066a43       ?OnInsertMenus@COleClientItem@@UAEXPAVCMenu@@PAUtagOleMenuGroupWidths@@@Z 5f567a43 f   olecli2.obj
 0001:00066b03       ?OnSetMenu@COleClientItem@@UAEXPAVCMenu@@PAXPAUHWND__@@@Z 5f567b03 f   olecli2.obj
 0001:00066c28       ?OnRemoveMenus@COleClientItem@@UAEXPAVCMenu@@@Z 5f567c28 f   olecli2.obj
 0001:00066c94       ?OnUpdateFrameTitle@COleClientItem@@UAEHXZ 5f567c94 f   olecli2.obj
 0001:00066cb4       ?Deactivate@COleClientItem@@QAEXXZ 5f567cb4 f   olecli2.obj
 0001:00066d86       ?DeactivateUI@COleClientItem@@QAEXXZ 5f567d86 f   olecli2.obj
 0001:00066e62       ?SetItemRects@COleClientItem@@QAEHPBUtagRECT@@0@Z 5f567e62 f   olecli2.obj
 0001:00067031       ?ReactivateAndUndo@COleClientItem@@QAEHXZ 5f568031 f   olecli2.obj
 0001:00067102       ?GetInPlaceWindow@COleClientItem@@QAEPAVCWnd@@XZ 5f568102 f   olecli2.obj
 0001:000671c2       ?_GetBaseInterfaceMap@COleFrameHook@@KGPBUAFX_INTERFACEMAP@@XZ 5f5681c2 f   olecli2.obj
 0001:000671cc       ?GetInterfaceMap@COleFrameHook@@MBEPBUAFX_INTERFACEMAP@@XZ 5f5681cc f   olecli2.obj
 0001:000671dc       ?GetInterfaceHook@COleFrameHook@@UAEPAUIUnknown@@PBX@Z 5f5681dc f   olecli2.obj
 0001:00067243       ?AddRef@XOleCommandTarget@COleFrameHook@@UAGKXZ 5f568243 f   olecli2.obj
 0001:0006725e       ?Release@XOleCommandTarget@COleFrameHook@@UAGKXZ 5f56825e f   olecli2.obj
 0001:00067279       ?QueryInterface@XOleCommandTarget@COleFrameHook@@UAGJABU_GUID@@PAPAX@Z 5f568279 f   olecli2.obj
 0001:0006729c       ?Exec@XOleCommandTarget@COleFrameHook@@UAGJPBU_GUID@@KKPAUtagVARIANT@@1@Z 5f56829c f   olecli2.obj
 0001:000672f8       ?QueryStatus@XOleCommandTarget@COleFrameHook@@UAGJPBU_GUID@@KQAU_tagOLECMD@@PAU_tagOLECMDTEXT@@@Z 5f5682f8 f   olecli2.obj
 0001:00067350       ?AddRef@XOleInPlaceFrame@COleFrameHook@@UAGKXZ 5f568350 f   olecli2.obj
 0001:0006736b       ?Release@XOleInPlaceFrame@COleFrameHook@@UAGKXZ 5f56836b f   olecli2.obj
 0001:00067386       ?QueryInterface@XOleInPlaceFrame@COleFrameHook@@UAGJABU_GUID@@PAPAX@Z 5f568386 f   olecli2.obj
 0001:000673a9       ?GetWindow@XOleInPlaceFrame@COleFrameHook@@UAGJPAPAUHWND__@@@Z 5f5683a9 f   olecli2.obj
 0001:000673da       ?ContextSensitiveHelp@XOleInPlaceFrame@COleFrameHook@@UAGJH@Z 5f5683da f   olecli2.obj
 0001:000674fb       ?GetBorder@XOleInPlaceFrame@COleFrameHook@@UAGJPAUtagRECT@@@Z 5f5684fb f   olecli2.obj
 0001:00067631       ?RequestBorderSpace@XOleInPlaceFrame@COleFrameHook@@UAGJPBUtagRECT@@@Z 5f568631 f   olecli2.obj
 0001:000676f6       ?SetBorderSpace@XOleInPlaceFrame@COleFrameHook@@UAGJPBUtagRECT@@@Z 5f5686f6 f   olecli2.obj
 0001:000677ca       ?SetActiveObject@XOleInPlaceFrame@COleFrameHook@@UAGJPAUIOleInPlaceActiveObject@@PBG@Z 5f5687ca f   olecli2.obj
 0001:0006791e       ?InsertMenus@XOleInPlaceFrame@COleFrameHook@@UAGJPAUHMENU__@@PAUtagOleMenuGroupWidths@@@Z 5f56891e f   olecli2.obj
 0001:00067a31       ?SetMenu@XOleInPlaceFrame@COleFrameHook@@UAGJPAUHMENU__@@PAXPAUHWND__@@@Z 5f568a31 f   olecli2.obj
 0001:00067b48       ?RemoveMenus@XOleInPlaceFrame@COleFrameHook@@UAGJPAUHMENU__@@@Z 5f568b48 f   olecli2.obj
 0001:00067c56       ?SetStatusText@XOleInPlaceFrame@COleFrameHook@@UAGJPBG@Z 5f568c56 f   olecli2.obj
 0001:00067cec       ?EnableModeless@XOleInPlaceFrame@COleFrameHook@@UAGJH@Z 5f568cec f   olecli2.obj
 0001:00067e06       ?TranslateAcceleratorA@XOleInPlaceFrame@COleFrameHook@@UAGJPAUtagMSG@@G@Z 5f568e06 f   olecli2.obj
 0001:00067f5b       ?AddRef@XOleIPSite@COleClientItem@@UAGKXZ 5f568f5b f   olecli2.obj
 0001:00067f76       ?Release@XOleIPSite@COleClientItem@@UAGKXZ 5f568f76 f   olecli2.obj
 0001:00067f91       ?QueryInterface@XOleIPSite@COleClientItem@@UAGJABU_GUID@@PAPAX@Z 5f568f91 f   olecli2.obj
 0001:00067fb4       ?GetWindow@XOleIPSite@COleClientItem@@UAGJPAPAUHWND__@@@Z 5f568fb4 f   olecli2.obj
 0001:00067fea       ?ContextSensitiveHelp@XOleIPSite@COleClientItem@@UAGJH@Z 5f568fea f   olecli2.obj
 0001:00068027       ?CanInPlaceActivate@XOleIPSite@COleClientItem@@UAGJXZ 5f569027 f   olecli2.obj
 0001:00068099       ?OnInPlaceActivate@XOleIPSite@COleClientItem@@UAGJXZ 5f569099 f   olecli2.obj
 0001:0006817c       ?OnUIActivate@XOleIPSite@COleClientItem@@UAGJXZ 5f56917c f   olecli2.obj
 0001:0006825f       ?GetWindowContext@XOleIPSite@COleClientItem@@UAGJPAPAUIOleInPlaceFrame@@PAPAUIOleInPlaceUIWindow@@PAUtagRECT@@2PAUtagOIFI@@@Z 5f56925f f   olecli2.obj
 0001:00068525       ?Scroll@XOleIPSite@COleClientItem@@UAGJUtagSIZE@@@Z 5f569525 f   olecli2.obj
 0001:00068633       ?OnUIDeactivate@XOleIPSite@COleClientItem@@UAGJH@Z 5f569633 f   olecli2.obj
 0001:0006871a       ?OnInPlaceDeactivate@XOleIPSite@COleClientItem@@UAGJXZ 5f56971a f   olecli2.obj
 0001:000687fd       ?DiscardUndoState@XOleIPSite@COleClientItem@@UAGJXZ 5f5697fd f   olecli2.obj
 0001:000688e0       ?DeactivateAndUndo@XOleIPSite@COleClientItem@@UAGJXZ 5f5698e0 f   olecli2.obj
 0001:000689c3       ?OnPosRectChange@XOleIPSite@COleClientItem@@UAGJPBUtagRECT@@@Z 5f5699c3 f   olecli2.obj
 0001:00068ac0       ??_ECOleFrameHook@@UAEPAXI@Z 5f569ac0 f i olecli2.obj
 0001:00068ac0       ??_GCOleFrameHook@@UAEPAXI@Z 5f569ac0 f i olecli2.obj
 0001:00068af0       ??0XOleInPlaceFrame@COleFrameHook@@QAE@XZ 5f569af0 f i olecli2.obj
 0001:00068b10       ??0XOleCommandTarget@COleFrameHook@@QAE@XZ 5f569b10 f i olecli2.obj
 0001:00068b30       ??0IOleInPlaceFrame@@QAE@XZ 5f569b30 f i olecli2.obj
 0001:00068b50       ??0IOleCommandTarget@@QAE@XZ 5f569b50 f i olecli2.obj
 0001:00068b70       ??0IOleInPlaceUIWindow@@QAE@XZ 5f569b70 f i olecli2.obj
 0001:00068b90       ??B?$CProcessLocal@V_AFX_OLE_STATE@@@@QAEPAV_AFX_OLE_STATE@@XZ 5f569b90 f i olecli2.obj
 0001:00068bb0       ?GetData@?$CProcessLocal@V_AFX_OLE_STATE@@@@QAEPAV_AFX_OLE_STATE@@XZ 5f569bb0 f i olecli2.obj
 0001:00068c00       ?CreateObject@?$CProcessLocal@V_AFX_OLE_STATE@@@@SGPAVCNoTrackObject@@XZ 5f569c00 f i olecli2.obj
 0001:00068c70       ?_AfxOlePropertiesEnabled@@YGHXZ 5f569c70 f   oledlgs1.obj
 0001:00068ccb       ?_AfxParseDisplayName@@YAJPAUIMoniker@@PAUIBindCtx@@PADPAKPAPAU1@@Z 5f569ccb f   oledlgs1.obj
 0001:00068fff       ??0COleUILinkInfo@@QAE@PAVCOleDocument@@@Z 5f569fff f   oledlgs1.obj
 0001:00069085       ?AddRef@COleUILinkInfo@@UAGKXZ 5f56a085 f   oledlgs1.obj
 0001:0006908e       ?Release@COleUILinkInfo@@UAGKXZ 5f56a08e f   oledlgs1.obj
 0001:00069097       ?QueryInterface@COleUILinkInfo@@UAGJABU_GUID@@PAPAX@Z 5f56a097 f   oledlgs1.obj
 0001:000690a3       ?GetNextLink@COleUILinkInfo@@UAGKK@Z 5f56a0a3 f   oledlgs1.obj
 0001:0006914a       ?SetLinkUpdateOptions@COleUILinkInfo@@UAGJKK@Z 5f56a14a f   oledlgs1.obj
 0001:0006925d       ?GetLinkUpdateOptions@COleUILinkInfo@@UAGJKPAK@Z 5f56a25d f   oledlgs1.obj
 0001:0006936b       ?SetLinkSource@COleUILinkInfo@@UAGJKPADKPAKH@Z 5f56a36b f   oledlgs1.obj
 0001:000698b1       ?GetLinkSource@COleUILinkInfo@@UAGJKPAPADPAK00PAH2@Z 5f56a8b1 f   oledlgs1.obj
 0001:00069b6e       ?OpenLinkSource@COleUILinkInfo@@UAGJK@Z 5f56ab6e f   oledlgs1.obj
 0001:00069c86       ?UpdateLink@COleUILinkInfo@@UAGJKHH@Z 5f56ac86 f   oledlgs1.obj
 0001:00069dab       ?CancelLink@COleUILinkInfo@@UAGJK@Z 5f56adab f   oledlgs1.obj
 0001:00069ee7       ?GetLastUpdate@COleUILinkInfo@@UAGJKPAU_FILETIME@@@Z 5f56aee7 f   oledlgs1.obj
 0001:00069f0c       ??0COleInsertDialog@@QAE@KPAVCWnd@@@Z 5f56af0c f   oledlgs1.obj
 0001:00069ffb       ??1COleInsertDialog@@UAE@XZ 5f56affb f   oledlgs1.obj
 0001:0006a053       ?AddClassIDToList@COleInsertDialog@@IAEXAAPAU_GUID@@AAH1PAU2@@Z 5f56b053 f   oledlgs1.obj
 0001:0006a14b       ?DoModal@COleInsertDialog@@QAEHK@Z 5f56b14b f   oledlgs1.obj
 0001:0006a666       ?DoModal@COleInsertDialog@@UAEHXZ 5f56b666 f   oledlgs1.obj
 0001:0006a6e0       ?GetSelectionType@COleInsertDialog@@QBEIXZ 5f56b6e0 f   oledlgs1.obj
 0001:0006a755       ?CreateItem@COleInsertDialog@@QAEHPAVCOleClientItem@@@Z 5f56b755 f   oledlgs1.obj
 0001:0006a8bd       ?Dump@COleInsertDialog@@UBEXAAVCDumpContext@@@Z 5f56b8bd f   oledlgs1.obj
 0001:0006aa25       ??0COleConvertDialog@@QAE@PAVCOleClientItem@@KPAU_GUID@@PAVCWnd@@@Z 5f56ba25 f   oledlgs1.obj
 0001:0006acc3       ??1COleConvertDialog@@UAE@XZ 5f56bcc3 f   oledlgs1.obj
 0001:0006ad1b       ?DoModal@COleConvertDialog@@UAEHXZ 5f56bd1b f   oledlgs1.obj
 0001:0006ad95       ?DoConvert@COleConvertDialog@@QAEHPAVCOleClientItem@@@Z 5f56bd95 f   oledlgs1.obj
 0001:0006af56       ?GetSelectionType@COleConvertDialog@@QBEIXZ 5f56bf56 f   oledlgs1.obj
 0001:0006afbe       ?Dump@COleConvertDialog@@UBEXAAVCDumpContext@@@Z 5f56bfbe f   oledlgs1.obj
 0001:0006b1a1       ??0COleChangeIconDialog@@QAE@PAVCOleClientItem@@KPAVCWnd@@@Z 5f56c1a1 f   oledlgs1.obj
 0001:0006b295       ??1COleChangeIconDialog@@UAE@XZ 5f56c295 f   oledlgs1.obj
 0001:0006b2ed       ?DoModal@COleChangeIconDialog@@UAEHXZ 5f56c2ed f   oledlgs1.obj
 0001:0006b367       ?DoChangeIcon@COleChangeIconDialog@@QAEHPAVCOleClientItem@@@Z 5f56c367 f   oledlgs1.obj
 0001:0006b3d4       ?Dump@COleChangeIconDialog@@UBEXAAVCDumpContext@@@Z 5f56c3d4 f   oledlgs1.obj
 0001:0006b51e       ??0COleLinksDialog@@QAE@PAVCOleDocument@@PAVCView@@KPAVCWnd@@@Z 5f56c51e f   oledlgs1.obj
 0001:0006b64c       ??1COleLinksDialog@@UAE@XZ 5f56c64c f   oledlgs1.obj
 0001:0006b668       ?DoModal@COleLinksDialog@@UAEHXZ 5f56c668 f   oledlgs1.obj
 0001:0006b6ef       ?Dump@COleLinksDialog@@UBEXAAVCDumpContext@@@Z 5f56c6ef f   oledlgs1.obj
 0001:0006b81b       ?AssertValid@COleLinksDialog@@UBEXXZ 5f56c81b f   oledlgs1.obj
 0001:0006b82e       ??0COleUpdateDialog@@QAE@PAVCOleDocument@@HHPAVCWnd@@@Z 5f56c82e f   oledlgs1.obj
 0001:0006b904       ??1COleUpdateDialog@@UAE@XZ 5f56c904 f   oledlgs1.obj
 0001:0006b95b       ?DoModal@COleUpdateDialog@@UAEHXZ 5f56c95b f   oledlgs1.obj
 0001:0006ba0f       ?Dump@COleUpdateDialog@@UBEXAAVCDumpContext@@@Z 5f56ca0f f   oledlgs1.obj
 0001:0006ba52       ??0COlePasteSpecialDialog@@QAE@KPAVCOleDataObject@@PAVCWnd@@@Z 5f56ca52 f   oledlgs1.obj
 0001:0006bbda       ??1COlePasteSpecialDialog@@UAE@XZ 5f56cbda f   oledlgs1.obj
 0001:0006bcda       ?DoModal@COlePasteSpecialDialog@@UAEHXZ 5f56ccda f   oledlgs1.obj
 0001:0006bd65       ?GetSelectionType@COlePasteSpecialDialog@@QBEIXZ 5f56cd65 f   oledlgs1.obj
 0001:0006be33       ?Dump@COlePasteSpecialDialog@@UBEXAAVCDumpContext@@@Z 5f56ce33 f   oledlgs1.obj
 0001:0006bff5       ?AssertValid@COlePasteSpecialDialog@@UBEXXZ 5f56cff5 f   oledlgs1.obj
 0001:0006c08c       ?AddLinkEntry@COlePasteSpecialDialog@@QAE?AW4tagOLEUIPASTEFLAG@@I@Z 5f56d08c f   oledlgs1.obj
 0001:0006c15b       ?AddFormat@COlePasteSpecialDialog@@QAEXIKIHH@Z 5f56d15b f   oledlgs1.obj
 0001:0006c345       ?AddFormat@COlePasteSpecialDialog@@QAEXABUtagFORMATETC@@PAD1K@Z 5f56d345 f   oledlgs1.obj
 0001:0006c40c       ?AddStandardFormats@COlePasteSpecialDialog@@QAEXH@Z 5f56d40c f   oledlgs1.obj
 0001:0006c4dd       ?CreateItem@COlePasteSpecialDialog@@QAEHPAVCOleClientItem@@@Z 5f56d4dd f   oledlgs1.obj
 0001:0006c6e8       ?GetLastError@COleDialog@@QBEIXZ 5f56d6e8 f   oledlgs1.obj
 0001:0006c6f9       ?GetPathName@COleInsertDialog@@QBE?AVCString@@XZ 5f56d6f9 f   oledlgs1.obj
 0001:0006c76b       ?GetClassID@COleInsertDialog@@QBEABU_GUID@@XZ 5f56d76b f   oledlgs1.obj
 0001:0006c791       ?GetIconicMetafile@COleInsertDialog@@QBEPAXXZ 5f56d791 f   oledlgs1.obj
 0001:0006c7b8       ?GetDrawAspect@COleInsertDialog@@QBE?AW4tagDVASPECT@@XZ 5f56d7b8 f   oledlgs1.obj
 0001:0006c7e9       ?GetIconicMetafile@COleConvertDialog@@QBEPAXXZ 5f56d7e9 f   oledlgs1.obj
 0001:0006c810       ?GetDrawAspect@COleConvertDialog@@QBE?AW4tagDVASPECT@@XZ 5f56d810 f   oledlgs1.obj
 0001:0006c837       ?GetClassID@COleConvertDialog@@QBEABU_GUID@@XZ 5f56d837 f   oledlgs1.obj
 0001:0006c85d       ?GetIconicMetafile@COleChangeIconDialog@@QBEPAXXZ 5f56d85d f   oledlgs1.obj
 0001:0006c884       ?GetPasteIndex@COlePasteSpecialDialog@@QBEHXZ 5f56d884 f   oledlgs1.obj
 0001:0006c8ab       ?GetDrawAspect@COlePasteSpecialDialog@@QBE?AW4tagDVASPECT@@XZ 5f56d8ab f   oledlgs1.obj
 0001:0006c8dc       ?GetIconicMetafile@COlePasteSpecialDialog@@QBEPAXXZ 5f56d8dc f   oledlgs1.obj
 0001:0006c903       ?GetSelectionType@COleBusyDialog@@QBEIXZ 5f56d903 f   oledlgs1.obj
 0001:0006c92a       ?IsValidSource@COleChangeSourceDialog@@QAEHXZ 5f56d92a f   oledlgs1.obj
 0001:0006c93e       ?GetDisplayName@COleChangeSourceDialog@@QAE?AVCString@@XZ 5f56d93e f   oledlgs1.obj
 0001:0006c972       ?GetFileName@COleChangeSourceDialog@@QAE?AVCString@@XZ 5f56d972 f   oledlgs1.obj
 0001:0006c9b0       ?GetItemName@COleChangeSourceDialog@@QAE?AVCString@@XZ 5f56d9b0 f   oledlgs1.obj
 0001:0006c9ec       ?GetFromPrefix@COleChangeSourceDialog@@QAE?AVCString@@XZ 5f56d9ec f   oledlgs1.obj
 0001:0006ca20       ?GetToPrefix@COleChangeSourceDialog@@QAE?AVCString@@XZ 5f56da20 f   oledlgs1.obj
 0001:0006ca60       ??0IOleUILinkInfoA@@QAE@XZ 5f56da60 f i oledlgs1.obj
 0001:0006ca80       ??0IOleUILinkContainerA@@QAE@XZ 5f56da80 f i oledlgs1.obj
 0001:0006caa0       ??_GCOleInsertDialog@@UAEPAXI@Z 5f56daa0 f i oledlgs1.obj
 0001:0006caa0       ??_ECOleInsertDialog@@UAEPAXI@Z 5f56daa0 f i oledlgs1.obj
 0001:0006cad0       ??1COleDialog@@UAE@XZ      5f56dad0 f i oledlgs1.obj
 0001:0006caf0       ??1CCommonDialog@@UAE@XZ   5f56daf0 f i oledlgs1.obj
 0001:0006cb10       ??_ECOleConvertDialog@@UAEPAXI@Z 5f56db10 f i oledlgs1.obj
 0001:0006cb10       ??_GCOleConvertDialog@@UAEPAXI@Z 5f56db10 f i oledlgs1.obj
 0001:0006cb40       ??_GCOleChangeIconDialog@@UAEPAXI@Z 5f56db40 f i oledlgs1.obj
 0001:0006cb40       ??_ECOleChangeIconDialog@@UAEPAXI@Z 5f56db40 f i oledlgs1.obj
 0001:0006cb70       ??_GCOleLinksDialog@@UAEPAXI@Z 5f56db70 f i oledlgs1.obj
 0001:0006cb70       ??_ECOleLinksDialog@@UAEPAXI@Z 5f56db70 f i oledlgs1.obj
 0001:0006cba0       ??_ECOleUpdateDialog@@UAEPAXI@Z 5f56dba0 f i oledlgs1.obj
 0001:0006cba0       ??_GCOleUpdateDialog@@UAEPAXI@Z 5f56dba0 f i oledlgs1.obj
 0001:0006cbd0       ??_GCOlePasteSpecialDialog@@UAEPAXI@Z 5f56dbd0 f i oledlgs1.obj
 0001:0006cbd0       ??_ECOlePasteSpecialDialog@@UAEPAXI@Z 5f56dbd0 f i oledlgs1.obj
 0001:0006cc00       ?AfxOleHookProc@@YGIPAUHWND__@@IIJ@Z 5f56dc00 f   oledlgs2.obj
 0001:0006cc5d       ??0COleDialog@@QAE@PAVCWnd@@@Z 5f56dc5d f   oledlgs2.obj
 0001:0006cc8c       ?MapResult@COleDialog@@QAEHI@Z 5f56dc8c f   oledlgs2.obj
 0001:0006ccbf       ?Dump@COleDialog@@UBEXAAVCDumpContext@@@Z 5f56dcbf f   oledlgs2.obj
 0001:0006cd00       ??0COleBusyDialog@@QAE@PAUHTASK__@@HKPAVCWnd@@@Z 5f56dd00 f   oledlgs2.obj
 0001:0006cdb3       ??1COleBusyDialog@@UAE@XZ  5f56ddb3 f   oledlgs2.obj
 0001:0006cdcf       ?DoModal@COleBusyDialog@@UAEHXZ 5f56ddcf f   oledlgs2.obj
 0001:0006ce9a       ?Dump@COleBusyDialog@@UBEXAAVCDumpContext@@@Z 5f56de9a f   oledlgs2.obj
 0001:0006cff0       ??_GCOleDialog@@UAEPAXI@Z  5f56dff0 f i oledlgs2.obj
 0001:0006cff0       ??_ECOleDialog@@UAEPAXI@Z  5f56dff0 f i oledlgs2.obj
 0001:0006d020       ??_ECOleBusyDialog@@UAEPAXI@Z 5f56e020 f i oledlgs2.obj
 0001:0006d020       ??_GCOleBusyDialog@@UAEPAXI@Z 5f56e020 f i oledlgs2.obj
 0001:0006d050       ??0COlePropertiesDialog@@QAE@PAVCOleClientItem@@IIPAVCWnd@@@Z 5f56e050 f   oledlgs3.obj
 0001:0006d299       ?DoModal@COlePropertiesDialog@@UAEHXZ 5f56e299 f   oledlgs3.obj
 0001:0006d38c       ?OnInitDialog@COlePropertiesDialog@@UAEHXZ 5f56e38c f   oledlgs3.obj
 0001:0006d3c2       ?AddRef@XOleUIObjInfo@COlePropertiesDialog@@UAGKXZ 5f56e3c2 f   oledlgs3.obj
 0001:0006d3cb       ?Release@XOleUIObjInfo@COlePropertiesDialog@@UAGKXZ 5f56e3cb f   oledlgs3.obj
 0001:0006d3d4       ?QueryInterface@XOleUIObjInfo@COlePropertiesDialog@@UAGJABU_GUID@@PAPAX@Z 5f56e3d4 f   oledlgs3.obj
 0001:0006d3e0       ?GetObjectInfo@XOleUIObjInfo@COlePropertiesDialog@@UAGJKPAKPAPAD111@Z 5f56e3e0 f   oledlgs3.obj
 0001:0006d75a       ?GetConvertInfo@XOleUIObjInfo@COlePropertiesDialog@@UAGJKPAU_GUID@@PAG0PAPAU3@PAI@Z 5f56e75a f   oledlgs3.obj
 0001:0006d7e4       ?ConvertObject@XOleUIObjInfo@COlePropertiesDialog@@UAGJKABU_GUID@@@Z 5f56e7e4 f   oledlgs3.obj
 0001:0006d831       ?GetViewInfo@XOleUIObjInfo@COlePropertiesDialog@@UAGJKPAPAXPAKPAH@Z 5f56e831 f   oledlgs3.obj
 0001:0006d88b       ?SetViewInfo@XOleUIObjInfo@COlePropertiesDialog@@UAGJKPAXKHH@Z 5f56e88b f   oledlgs3.obj
 0001:0006d95b       ?OnApplyScale@COlePropertiesDialog@@UAEHPAVCOleClientItem@@HH@Z 5f56e95b f   oledlgs3.obj
 0001:0006d96a       ?Dump@COlePropertiesDialog@@UBEXAAVCDumpContext@@@Z 5f56e96a f   oledlgs3.obj
 0001:0006d983       ?AssertValid@COlePropertiesDialog@@UBEXXZ 5f56e983 f   oledlgs3.obj
 0001:0006da31       ??0COleChangeSourceDialog@@QAE@PAVCOleClientItem@@PAVCWnd@@@Z 5f56ea31 f   oledlgs3.obj
 0001:0006db17       ?DoModal@COleChangeSourceDialog@@UAEHXZ 5f56eb17 f   oledlgs3.obj
 0001:0006db91       ?PreInitDialog@COleChangeSourceDialog@@UAEXXZ 5f56eb91 f   oledlgs3.obj
 0001:0006dbb7       ??1COleChangeSourceDialog@@UAE@XZ 5f56ebb7 f   oledlgs3.obj
 0001:0006dc03       ?Dump@COleChangeSourceDialog@@UBEXAAVCDumpContext@@@Z 5f56ec03 f   oledlgs3.obj
 0001:0006dd2f       ?AssertValid@COleChangeSourceDialog@@UBEXXZ 5f56ed2f f   oledlgs3.obj
 0001:0006dd90       ??_ECOlePropertiesDialog@@UAEPAXI@Z 5f56ed90 f i oledlgs3.obj
 0001:0006dd90       ??_GCOlePropertiesDialog@@UAEPAXI@Z 5f56ed90 f i oledlgs3.obj
 0001:0006ddc0       ??0XOleUIObjInfo@COlePropertiesDialog@@QAE@XZ 5f56edc0 f i oledlgs3.obj
 0001:0006dde0       ??1COlePropertiesDialog@@UAE@XZ 5f56ede0 f i oledlgs3.obj
 0001:0006de00       ??0IOleUIObjInfoA@@QAE@XZ  5f56ee00 f i oledlgs3.obj
 0001:0006de20       ??_ECOleChangeSourceDialog@@UAEPAXI@Z 5f56ee20 f i oledlgs3.obj
 0001:0006de20       ??_GCOleChangeSourceDialog@@UAEPAXI@Z 5f56ee20 f i oledlgs3.obj
 0001:0006de50       ?ReportError@COleClientItem@@UBEHJ@Z 5f56ee50 f   oleui1.obj
 0001:0006df0a       ?DoVerb@COleClientItem@@UAEHJPAVCView@@PAUtagMSG@@@Z 5f56ef0a f   oleui1.obj
 0001:0006e089       ?OnCmdMsg@COleDocument@@UAEHIHPAXPAUAFX_CMDHANDLERINFO@@@Z 5f56f089 f   oleui1.obj
 0001:0006e17c       ?GetPrimarySelectedItem@COleDocument@@UAEPAVCOleClientItem@@PAVCView@@@Z 5f56f17c f   oleui1.obj
 0001:0006e226       ?GetInPlaceActiveItem@COleDocument@@UAEPAVCOleClientItem@@PAVCWnd@@@Z 5f56f226 f   oleui1.obj
 0001:0006e310       ?AfxOleSetEditMenu@@YGXPAVCOleClientItem@@PAVCMenu@@IIII@Z 5f56f310 f   oleui2.obj
 0001:0006e3e6       ?OnUpdatePasteMenu@COleDocument@@IAEXPAVCCmdUI@@@Z 5f56f3e6 f   oleui2.obj
 0001:0006e403       ?OnUpdatePasteLinkMenu@COleDocument@@IAEXPAVCCmdUI@@@Z 5f56f403 f   oleui2.obj
 0001:0006e420       ?OnUpdateEditLinksMenu@COleDocument@@IAEXPAVCCmdUI@@@Z 5f56f420 f   oleui2.obj
 0001:0006e47e       ?OnEditLinks@COleDocument@@IAEXXZ 5f56f47e f   oleui2.obj
 0001:0006e503       ?OnEditConvert@COleDocument@@IAEXXZ 5f56f503 f   oleui2.obj
 0001:0006e5ba       ?OnUpdateEditChangeIcon@COleDocument@@IAEXPAVCCmdUI@@@Z 5f56f5ba f   oleui2.obj
 0001:0006e5fc       ?OnEditChangeIcon@COleDocument@@IAEXXZ 5f56f5fc f   oleui2.obj
 0001:0006e6b1       ?OnUpdateObjectVerbMenu@COleDocument@@IAEXPAVCCmdUI@@@Z 5f56f6b1 f   oleui2.obj
 0001:0006e780       ??0COleDataObject@@QAE@XZ  5f56f780 f   oledobj1.obj
 0001:0006e7b5       ?Attach@COleDataObject@@QAEXPAUIDataObject@@H@Z 5f56f7b5 f   oledobj1.obj
 0001:0006e7fe       ?Release@COleDataObject@@QAEXXZ 5f56f7fe f   oledobj1.obj
 0001:0006e868       ?Detach@COleDataObject@@QAEPAUIDataObject@@XZ 5f56f868 f   oledobj1.obj
 0001:0006e89b       ?GetIDataObject@COleDataObject@@QAEPAUIDataObject@@H@Z 5f56f89b f   oledobj1.obj
 0001:0006e8d5       ?BeginEnumFormats@COleDataObject@@QAEXXZ 5f56f8d5 f   oledobj1.obj
 0001:0006e98f       ?GetNextFormat@COleDataObject@@QAEHPAUtagFORMATETC@@@Z 5f56f98f f   oledobj1.obj
 0001:0006ea58       ?GetFileData@COleDataObject@@QAEPAVCFile@@GPAUtagFORMATETC@@@Z 5f56fa58 f   oledobj1.obj
 0001:0006ee96       ?GetGlobalData@COleDataObject@@QAEPAXGPAUtagFORMATETC@@@Z 5f56fe96 f   oledobj1.obj
 0001:0006f009       ?GetData@COleDataObject@@QAEHGPAUtagSTGMEDIUM@@PAUtagFORMATETC@@@Z 5f570009 f   oledobj1.obj
 0001:0006f0c7       ?IsDataAvailable@COleDataObject@@QAEHGPAUtagFORMATETC@@@Z 5f5700c7 f   oledobj1.obj
 0001:0006f17b       ?AttachClipboard@COleDataObject@@QAEHXZ 5f57017b f   oledobj1.obj
 0001:0006f20b       ?EnsureClipboardObject@COleDataObject@@QAEXXZ 5f57020b f   oledobj1.obj
 0001:0006f280       ??0COleDataSource@@QAE@XZ  5f570280 f   oledobj2.obj
 0001:0006f2ff       ??1COleDataSource@@UAE@XZ  5f5702ff f   oledobj2.obj
 0001:0006f374       ?Empty@COleDataSource@@QAEXXZ 5f570374 f   oledobj2.obj
 0001:0006f4b4       ?SetClipboard@COleDataSource@@QAEXXZ 5f5704b4 f   oledobj2.obj
 0001:0006f540       ?FlushClipboard@COleDataSource@@SGXXZ 5f570540 f   oledobj2.obj
 0001:0006f57a       ?GetClipboardOwner@COleDataSource@@SGPAV1@XZ 5f57057a f   oledobj2.obj
 0001:0006f5e6       ?GetCacheEntry@COleDataSource@@IAEPAUAFX_DATACACHE_ENTRY@@PAUtagFORMATETC@@W4tagDATADIR@@@Z 5f5705e6 f   oledobj2.obj
 0001:0006f774       ?CacheGlobalData@COleDataSource@@QAEXGPAXPAUtagFORMATETC@@@Z 5f570774 f   oledobj2.obj
 0001:0006f827       ?CacheData@COleDataSource@@QAEXGPAUtagSTGMEDIUM@@PAUtagFORMATETC@@@Z 5f570827 f   oledobj2.obj
 0001:0006f953       ?DelayRenderFileData@COleDataSource@@QAEXGPAUtagFORMATETC@@@Z 5f570953 f   oledobj2.obj
 0001:0006f9eb       ?DelayRenderData@COleDataSource@@QAEXGPAUtagFORMATETC@@@Z 5f5709eb f   oledobj2.obj
 0001:0006fa90       ?DelaySetData@COleDataSource@@QAEXGPAUtagFORMATETC@@@Z 5f570a90 f   oledobj2.obj
 0001:0006fb1a       ?Lookup@COleDataSource@@IBEPAUAFX_DATACACHE_ENTRY@@PAUtagFORMATETC@@W4tagDATADIR@@@Z 5f570b1a f   oledobj2.obj
 0001:0006fc26       ?OnRenderGlobalData@COleDataSource@@UAEHPAUtagFORMATETC@@PAPAX@Z 5f570c26 f   oledobj2.obj
 0001:0006fc35       ?OnRenderFileData@COleDataSource@@UAEHPAUtagFORMATETC@@PAVCFile@@@Z 5f570c35 f   oledobj2.obj
 0001:0006fc44       ?OnRenderData@COleDataSource@@UAEHPAUtagFORMATETC@@PAUtagSTGMEDIUM@@@Z 5f570c44 f   oledobj2.obj
 0001:0006fed0       ?OnSetData@COleDataSource@@UAEHPAUtagFORMATETC@@PAUtagSTGMEDIUM@@H@Z 5f570ed0 f   oledobj2.obj
 0001:0006fedf       ?_GetBaseInterfaceMap@CEnumFormatEtc@@KGPBUAFX_INTERFACEMAP@@XZ 5f570edf f   oledobj2.obj
 0001:0006fee9       ?GetInterfaceMap@CEnumFormatEtc@@MBEPBUAFX_INTERFACEMAP@@XZ 5f570ee9 f   oledobj2.obj
 0001:0006fef9       ??0CEnumFormatEtc@@QAE@XZ  5f570ef9 f   oledobj2.obj
 0001:0006ff2a       ??1CEnumFormatEtc@@UAE@XZ  5f570f2a f   oledobj2.obj
 0001:0006ff8d       ?OnNext@CEnumFormatEtc@@MAEHPAX@Z 5f570f8d f   oledobj2.obj
 0001:0006ffe4       ?AddFormat@CEnumFormatEtc@@QAEXPBUtagFORMATETC@@@Z 5f570fe4 f   oledobj2.obj
 0001:00070128       ?_GetBaseInterfaceMap@COleDataSource@@KGPBUAFX_INTERFACEMAP@@XZ 5f571128 f   oledobj2.obj
 0001:00070132       ?GetInterfaceMap@COleDataSource@@MBEPBUAFX_INTERFACEMAP@@XZ 5f571132 f   oledobj2.obj
 0001:00070142       ?AddRef@XDataObject@COleDataSource@@UAGKXZ 5f571142 f   oledobj2.obj
 0001:0007015d       ?Release@XDataObject@COleDataSource@@UAGKXZ 5f57115d f   oledobj2.obj
 0001:00070178       ?QueryInterface@XDataObject@COleDataSource@@UAGJABU_GUID@@PAPAX@Z 5f571178 f   oledobj2.obj
 0001:0007019b       ?GetData@XDataObject@COleDataSource@@UAGJPAUtagFORMATETC@@PAUtagSTGMEDIUM@@@Z 5f57119b f   oledobj2.obj
 0001:00070343       ?GetDataHere@XDataObject@COleDataSource@@UAGJPAUtagFORMATETC@@PAUtagSTGMEDIUM@@@Z 5f571343 f   oledobj2.obj
 0001:00070534       ?QueryGetData@XDataObject@COleDataSource@@UAGJPAUtagFORMATETC@@@Z 5f571534 f   oledobj2.obj
 0001:00070569       ?GetCanonicalFormatEtc@XDataObject@COleDataSource@@UAGJPAUtagFORMATETC@@0@Z 5f571569 f   oledobj2.obj
 0001:00070575       ?SetData@XDataObject@COleDataSource@@UAGJPAUtagFORMATETC@@PAUtagSTGMEDIUM@@H@Z 5f571575 f   oledobj2.obj
 0001:000706fb       ?EnumFormatEtc@XDataObject@COleDataSource@@UAGJKPAPAUIEnumFORMATETC@@@Z 5f5716fb f   oledobj2.obj
 0001:00070854       ?DAdvise@XDataObject@COleDataSource@@UAGJPAUtagFORMATETC@@KPAUIAdviseSink@@PAK@Z 5f571854 f   oledobj2.obj
 0001:00070869       ?DUnadvise@XDataObject@COleDataSource@@UAGJK@Z 5f571869 f   oledobj2.obj
 0001:00070875       ?EnumDAdvise@XDataObject@COleDataSource@@UAGJPAPAUIEnumSTATDATA@@@Z 5f571875 f   oledobj2.obj
 0001:0007088a       ?AssertValid@COleDataSource@@UBEXXZ 5f57188a f   oledobj2.obj
 0001:000708f7       ?Dump@COleDataSource@@UBEXAAVCDumpContext@@@Z 5f5718f7 f   oledobj2.obj
 0001:00070aa0       ??_GCOleDataSource@@UAEPAXI@Z 5f571aa0 f i oledobj2.obj
 0001:00070ad0       ??0XDataObject@COleDataSource@@QAE@XZ 5f571ad0 f i oledobj2.obj
 0001:00070af0       ??_GCEnumFormatEtc@@UAEPAXI@Z 5f571af0 f i oledobj2.obj
 0001:00070af0       ??_ECEnumFormatEtc@@UAEPAXI@Z 5f571af0 f i oledobj2.obj
 0001:00070b20       ??C?$CProcessLocal@V_AFX_OLE_STATE@@@@QAEPAV_AFX_OLE_STATE@@XZ 5f571b20 f i oledobj2.obj
 0001:00070b40       ??0CEnumArray@@QAE@IPBXIH@Z 5f571b40 f   oleenum.obj
 0001:00070be1       ??1CEnumArray@@UAE@XZ      5f571be1 f   oleenum.obj
 0001:00070cb4       ?OnNext@CEnumArray@@MAEHPAX@Z 5f571cb4 f   oleenum.obj
 0001:00070d20       ?OnSkip@CEnumArray@@MAEHXZ 5f571d20 f   oleenum.obj
 0001:00070d6c       ?OnReset@CEnumArray@@MAEXXZ 5f571d6c f   oleenum.obj
 0001:00070d91       ?OnClone@CEnumArray@@MAEPAV1@XZ 5f571d91 f   oleenum.obj
 0001:00070e8b       ?AddRef@XEnumVOID@CEnumArray@@UAGKXZ 5f571e8b f   oleenum.obj
 0001:00070ea6       ?Release@XEnumVOID@CEnumArray@@UAGKXZ 5f571ea6 f   oleenum.obj
 0001:00070ec1       ?QueryInterface@XEnumVOID@CEnumArray@@UAGJABU_GUID@@PAPAX@Z 5f571ec1 f   oleenum.obj
 0001:00070ee4       ?Next@XEnumVOID@CEnumArray@@UAGJKPAXPAK@Z 5f571ee4 f   oleenum.obj
 0001:00071065       ?Skip@XEnumVOID@CEnumArray@@UAGJK@Z 5f572065 f   oleenum.obj
 0001:0007116f       ?Reset@XEnumVOID@CEnumArray@@UAGJXZ 5f57216f f   oleenum.obj
 0001:000711f0       ?Clone@XEnumVOID@CEnumArray@@UAGJPAPAUIEnumVOID@@@Z 5f5721f0 f   oleenum.obj
 0001:00071330       ??_GCEnumArray@@UAEPAXI@Z  5f572330 f i oleenum.obj
 0001:00071330       ??_ECEnumArray@@UAEPAXI@Z  5f572330 f i oleenum.obj
 0001:00071360       ??0XEnumVOID@CEnumArray@@QAE@XZ 5f572360 f i oleenum.obj
 0001:00071380       ??0IEnumVOID@@QAE@XZ       5f572380 f i oleenum.obj
 0001:000713a0       ?_GetBaseInterfaceMap@COleObjectFactory@@KGPBUAFX_INTERFACEMAP@@XZ 5f5723a0 f   olefact.obj
 0001:000713aa       ?GetInterfaceMap@COleObjectFactory@@MBEPBUAFX_INTERFACEMAP@@XZ 5f5723aa f   olefact.obj
 0001:000713ba       ?UpdateRegistry@COleObjectFactory@@QAEXPBD@Z 5f5723ba f   olefact.obj
 0001:00071448       ?UpdateRegistryAll@COleObjectFactory@@SGHH@Z 5f572448 f   olefact.obj
 0001:0007151f       ?OnCreateObject@COleObjectFactory@@MAEPAVCCmdTarget@@XZ 5f57251f f   olefact.obj
 0001:000715cf       ?IsLicenseValid@COleObjectFactory@@QAEHXZ 5f5725cf f   olefact.obj
 0001:00071608       ?UpdateRegistry@COleObjectFactory@@MAEHH@Z 5f572608 f   olefact.obj
 0001:0007162a       ?VerifyUserLicense@COleObjectFactory@@MAEHXZ 5f57262a f   olefact.obj
 0001:0007163a       ?GetLicenseKey@COleObjectFactory@@MAEHKPAPAG@Z 5f57263a f   olefact.obj
 0001:00071649       ?VerifyLicenseKey@COleObjectFactory@@MAEHPAG@Z 5f572649 f   olefact.obj
 0001:000716ef       ?AddRef@XClassFactory@COleObjectFactory@@UAGKXZ 5f5726ef f   olefact.obj
 0001:0007170a       ?Release@XClassFactory@COleObjectFactory@@UAGKXZ 5f57270a f   olefact.obj
 0001:00071725       ?QueryInterface@XClassFactory@COleObjectFactory@@UAGJABU_GUID@@PAPAX@Z 5f572725 f   olefact.obj
 0001:00071748       ?CreateInstance@XClassFactory@COleObjectFactory@@UAGJPAUIUnknown@@ABU_GUID@@PAPAX@Z 5f572748 f   olefact.obj
 0001:0007176b       ?LockServer@XClassFactory@COleObjectFactory@@UAGJH@Z 5f57276b f   olefact.obj
 0001:00071852       ?GetLicInfo@XClassFactory@COleObjectFactory@@UAGJPAUtagLICINFO@@@Z 5f572852 f   olefact.obj
 0001:00071904       ?RequestLicKey@XClassFactory@COleObjectFactory@@UAGJKPAPAG@Z 5f572904 f   olefact.obj
 0001:00071a02       ?CreateInstanceLic@XClassFactory@COleObjectFactory@@UAGJPAUIUnknown@@0ABU_GUID@@PAGPAPAX@Z 5f572a02 f   olefact.obj
 0001:00071c89       ?AssertValid@COleObjectFactory@@UBEXXZ 5f572c89 f   olefact.obj
 0001:00071d45       ?Dump@COleObjectFactory@@UBEXAAVCDumpContext@@@Z 5f572d45 f   olefact.obj
 0001:00071ef0       ??0COleCntrFrameWnd@@QAE@PAVCOleIPFrameWnd@@@Z 5f572ef0 f   oleipfrm.obj
 0001:00071f52       ??1COleCntrFrameWnd@@UAE@XZ 5f572f52 f   oleipfrm.obj
 0001:00071fab       ?RecalcLayout@COleCntrFrameWnd@@UAEXH@Z 5f572fab f   oleipfrm.obj
 0001:000720f6       ?OnIdleUpdateCmdUI@COleCntrFrameWnd@@QAEXXZ 5f5730f6 f   oleipfrm.obj
 0001:000721a4       ?OnCmdMsg@COleCntrFrameWnd@@UAEHIHPAXPAUAFX_CMDHANDLERINFO@@@Z 5f5731a4 f   oleipfrm.obj
 0001:00072237       ?PostNcDestroy@COleCntrFrameWnd@@MAEXXZ 5f573237 f   oleipfrm.obj
 0001:00072242       ?AssertValid@COleCntrFrameWnd@@UBEXXZ 5f573242 f   oleipfrm.obj
 0001:00072284       ?_GetBaseMessageMap@COleIPFrameWnd@@KGPBUAFX_MSGMAP@@XZ 5f573284 f   oleipfrm.obj
 0001:0007228e       ?GetMessageMap@COleIPFrameWnd@@MBEPBUAFX_MSGMAP@@XZ 5f57328e f   oleipfrm.obj
 0001:0007229e       ??0COleIPFrameWnd@@QAE@XZ  5f57329e f   oleipfrm.obj
 0001:000723c0       ??1COleIPFrameWnd@@UAE@XZ  5f5733c0 f   oleipfrm.obj
 0001:0007250a       ?OnCreate@COleIPFrameWnd@@IAEHPAUtagCREATESTRUCTA@@@Z 5f57350a f   oleipfrm.obj
 0001:00072584       ?OnDestroy@COleIPFrameWnd@@IAEXXZ 5f573584 f   oleipfrm.obj
 0001:0007262b       ?OnCreateControlBars@COleIPFrameWnd@@UAEHPAVCWnd@@0@Z 5f57362b f   oleipfrm.obj
 0001:00072663       ?OnCreateControlBars@COleIPFrameWnd@@UAEHPAVCFrameWnd@@0@Z 5f573663 f   oleipfrm.obj
 0001:00072686       ?OnIdleUpdateCmdUI@COleIPFrameWnd@@IAEXXZ 5f573686 f   oleipfrm.obj
 0001:000726c5       ?OnWindowPosChanging@COleIPFrameWnd@@IAEXPAUtagWINDOWPOS@@@Z 5f5736c5 f   oleipfrm.obj
 0001:00072712       ?OnSetMessageString@COleIPFrameWnd@@UAEJIJ@Z 5f573712 f   oleipfrm.obj
 0001:0007288a       ?LoadFrame@COleIPFrameWnd@@UAEHIKPAVCWnd@@PAUCCreateContext@@@Z 5f57388a f   oleipfrm.obj
 0001:00072970       ?OnSize@COleIPFrameWnd@@IAEXIHH@Z 5f573970 f   oleipfrm.obj
 0001:0007297d       ?OnResizeChild@COleIPFrameWnd@@IAEJIJ@Z 5f57397d f   oleipfrm.obj
 0001:00072aee       ?OnRequestPositionChange@COleIPFrameWnd@@MAEXPBUtagRECT@@@Z 5f573aee f   oleipfrm.obj
 0001:00072b6c       ?OnRecalcParent@COleIPFrameWnd@@IAEJIJ@Z 5f573b6c f   oleipfrm.obj
 0001:00072bc7       ?RecalcLayout@COleIPFrameWnd@@UAEXH@Z 5f573bc7 f   oleipfrm.obj
 0001:00072dee       ?RepositionFrame@COleIPFrameWnd@@UAEXPBUtagRECT@@0@Z 5f573dee f   oleipfrm.obj
 0001:00072eb3       ?PreTranslateMessage@COleIPFrameWnd@@UAEHPAUtagMSG@@@Z 5f573eb3 f   oleipfrm.obj
 0001:00072f75       ?OnUpdateControlBarMenu@COleIPFrameWnd@@IAEXPAVCCmdUI@@@Z 5f573f75 f   oleipfrm.obj
 0001:0007301d       ?OnBarCheck@COleIPFrameWnd@@IAEHI@Z 5f57401d f   oleipfrm.obj
 0001:000730b6       ?OnContextHelp@COleIPFrameWnd@@IAEXXZ 5f5740b6 f   oleipfrm.obj
 0001:000731fe       ?GetInPlaceMenu@COleIPFrameWnd@@MAEPAUHMENU__@@XZ 5f5741fe f   oleipfrm.obj
 0001:00073253       ?BuildSharedMenu@COleIPFrameWnd@@MAEHXZ 5f574253 f   oleipfrm.obj
 0001:000733fa       ?DestroySharedMenu@COleIPFrameWnd@@MAEXXZ 5f5743fa f   oleipfrm.obj
 0001:0007353f       ?AssertValid@COleIPFrameWnd@@UBEXXZ 5f57453f f   oleipfrm.obj
 0001:00073592       ?Dump@COleIPFrameWnd@@UBEXAAVCDumpContext@@@Z 5f574592 f   oleipfrm.obj
 0001:00073690       ??_ECOleCntrFrameWnd@@UAEPAXI@Z 5f574690 f i oleipfrm.obj
 0001:00073690       ??_GCOleCntrFrameWnd@@UAEPAXI@Z 5f574690 f i oleipfrm.obj
 0001:000736c0       ??_GCOleIPFrameWnd@@UAEPAXI@Z 5f5746c0 f i oleipfrm.obj
 0001:000736f0       ??0COleLinkingDoc@@QAE@XZ  5f5746f0 f   olelink.obj
 0001:000737c8       ??1COleLinkingDoc@@UAE@XZ  5f5747c8 f   olelink.obj
 0001:0007389a       ?GetMoniker@COleLinkingDoc@@UAEPAUIMoniker@@W4tagOLEGETMONIKER@@@Z 5f57489a f   olelink.obj
 0001:0007395f       ?Register@COleLinkingDoc@@QAEHPAVCOleObjectFactory@@PBD@Z 5f57495f f   olelink.obj
 0001:00073cb0       ?Revoke@COleLinkingDoc@@QAEXXZ 5f574cb0 f   olelink.obj
 0001:00073d6e       ?OnNewDocument@COleLinkingDoc@@UAEHXZ 5f574d6e f   olelink.obj
 0001:00073dc2       ?OnOpenDocument@COleLinkingDoc@@UAEHPBD@Z 5f574dc2 f   olelink.obj
 0001:00073e95       ?OnSaveDocument@COleLinkingDoc@@UAEHPBD@Z 5f574e95 f   olelink.obj
 0001:00073f1a       ?OnCloseDocument@COleLinkingDoc@@UAEXXZ 5f574f1a f   olelink.obj
 0001:00073fd4       ?UpdateVisibleLock@COleLinkingDoc@@IAEXHH@Z 5f574fd4 f   olelink.obj
 0001:0007402e       ?OnShowViews@COleLinkingDoc@@MAEXH@Z 5f57502e f   olelink.obj
 0001:0007404f       ?SaveToStorage@COleLinkingDoc@@MAEXPAVCObject@@@Z 5f57504f f   olelink.obj
 0001:000740e5       ?RegisterIfServerAttached@COleLinkingDoc@@MAEHPBDH@Z 5f5750e5 f   olelink.obj
 0001:000741de       ?GetContainer@COleLinkingDoc@@UAEPAUIOleItemContainer@@XZ 5f5751de f   olelink.obj
 0001:00074212       ?OnGetLinkedItem@COleLinkingDoc@@MAEPAVCOleServerItem@@PBD@Z 5f575212 f   olelink.obj
 0001:00074234       ?OnFindEmbeddedItem@COleLinkingDoc@@MAEPAVCOleClientItem@@PBD@Z 5f575234 f   olelink.obj
 0001:00074304       ?LockExternal@COleLinkingDoc@@IAEXHH@Z 5f575304 f   olelink.obj
 0001:00074366       ?ReportSaveLoadException@COleLinkingDoc@@UAEXPBDPAVCException@@HI@Z 5f575366 f   olelink.obj
 0001:000743b4       ?EndDeferErrors@COleLinkingDoc@@QAEJJ@Z 5f5753b4 f   olelink.obj
 0001:00074478       ?_GetBaseInterfaceMap@COleLinkingDoc@@KGPBUAFX_INTERFACEMAP@@XZ 5f575478 f   olelink.obj
 0001:00074482       ?GetInterfaceMap@COleLinkingDoc@@MBEPBUAFX_INTERFACEMAP@@XZ 5f575482 f   olelink.obj
 0001:00074492       ?AddRef@XPersistFile@COleLinkingDoc@@UAGKXZ 5f575492 f   olelink.obj
 0001:000744af       ?Release@XPersistFile@COleLinkingDoc@@UAGKXZ 5f5754af f   olelink.obj
 0001:000744cc       ?QueryInterface@XPersistFile@COleLinkingDoc@@UAGJABU_GUID@@PAPAX@Z 5f5754cc f   olelink.obj
 0001:000744f1       ?GetClassID@XPersistFile@COleLinkingDoc@@UAGJPAU_GUID@@@Z 5f5754f1 f   olelink.obj
 0001:0007457f       ?IsDirty@XPersistFile@COleLinkingDoc@@UAGJXZ 5f57557f f   olelink.obj
 0001:000745f0       ?Load@XPersistFile@COleLinkingDoc@@UAGJPBGK@Z 5f5755f0 f   olelink.obj
 0001:000747f2       ?Save@XPersistFile@COleLinkingDoc@@UAGJPBGH@Z 5f5757f2 f   olelink.obj
 0001:000749c3       ?SaveCompleted@XPersistFile@COleLinkingDoc@@UAGJPBG@Z 5f5759c3 f   olelink.obj
 0001:00074b1f       ?GetCurFile@XPersistFile@COleLinkingDoc@@UAGJPAPAG@Z 5f575b1f f   olelink.obj
 0001:00074bc4       ?AddRef@XOleItemContainer@COleLinkingDoc@@UAGKXZ 5f575bc4 f   olelink.obj
 0001:00074be1       ?Release@XOleItemContainer@COleLinkingDoc@@UAGKXZ 5f575be1 f   olelink.obj
 0001:00074bfe       ?QueryInterface@XOleItemContainer@COleLinkingDoc@@UAGJABU_GUID@@PAPAX@Z 5f575bfe f   olelink.obj
 0001:00074c23       ?EnumObjects@XOleItemContainer@COleLinkingDoc@@UAGJKPAPAUIEnumUnknown@@@Z 5f575c23 f   olelink.obj
 0001:00074c38       ?ParseDisplayName@XOleItemContainer@COleLinkingDoc@@UAGJPAUIBindCtx@@PAGPAKPAPAUIMoniker@@@Z 5f575c38 f   olelink.obj
 0001:00074fa2       ?LockContainer@XOleItemContainer@COleLinkingDoc@@UAGJH@Z 5f575fa2 f   olelink.obj
 0001:00074fc7       ?GetObjectA@XOleItemContainer@COleLinkingDoc@@UAGJPAGKPAUIBindCtx@@ABU_GUID@@PAPAX@Z 5f575fc7 f   olelink.obj
 0001:00075203       ?GetObjectStorage@XOleItemContainer@COleLinkingDoc@@UAGJPAGPAUIBindCtx@@ABU_GUID@@PAPAX@Z 5f576203 f   olelink.obj
 0001:0007538f       ?IsRunning@XOleItemContainer@COleLinkingDoc@@UAGJPAG@Z 5f57638f f   olelink.obj
 0001:00075571       ?AssertValid@COleLinkingDoc@@UBEXXZ 5f576571 f   olelink.obj
 0001:000755a7       ?Dump@COleLinkingDoc@@UBEXAAVCDumpContext@@@Z 5f5765a7 f   olelink.obj
 0001:00075650       ??_GCOleLinkingDoc@@UAEPAXI@Z 5f576650 f i olelink.obj
 0001:00075650       ??_ECOleLinkingDoc@@UAEPAXI@Z 5f576650 f i olelink.obj
 0001:00075680       ??0XPersistFile@COleLinkingDoc@@QAE@XZ 5f576680 f i olelink.obj
 0001:000756a0       ??0XOleItemContainer@COleLinkingDoc@@QAE@XZ 5f5766a0 f i olelink.obj
 0001:000756c0       ??0IOleItemContainer@@QAE@XZ 5f5766c0 f i olelink.obj
 0001:000756e0       ??0IPersistFile@@QAE@XZ    5f5766e0 f i olelink.obj
 0001:000756e0       ??0IOleContainer@@QAE@XZ   5f5766e0 f i olelink.obj
 0001:00075700       ??0IParseDisplayName@@QAE@XZ 5f576700 f i olelink.obj
 0001:00075700       ??0IPersist@@QAE@XZ        5f576700 f i olelink.obj
 0001:00075700       ??0IDataObject@@QAE@XZ     5f576700 f i olelink.obj
 0001:00075720       ??0COleTemplateServer@@QAE@XZ 5f576720 f   oletsvr.obj
 0001:00075754       ?Register@COleTemplateServer@@UAEHXZ 5f576754 f   oletsvr.obj
 0001:00075767       ?OnCmdMsg@COleTemplateServer@@MAEHIHPAXPAUAFX_CMDHANDLERINFO@@@Z 5f576767 f   oletsvr.obj
 0001:000757a7       ?Unregister@COleTemplateServer@@QAEHXZ 5f5767a7 f   oletsvr.obj
 0001:0007596a       ?ConnectTemplate@COleTemplateServer@@QAEXABU_GUID@@PAVCDocTemplate@@H@Z 5f57696a f   oletsvr.obj
 0001:00075a1a       ?UpdateRegistry@COleTemplateServer@@QAEXW4OLE_APPTYPE@@PAPBD1@Z 5f576a1a f   oletsvr.obj
 0001:00075d3b       ?OnCreateObject@COleTemplateServer@@MAEPAVCCmdTarget@@XZ 5f576d3b f   oletsvr.obj
 0001:00075e00       ??_GCOleTemplateServer@@UAEPAXI@Z 5f576e00 f i oletsvr.obj
 0001:00075e30       ?AfxDllGetClassObject@@YGJABU_GUID@@0PAPAX@Z 5f576e30 f   oledll.obj
 0001:00075fa6       ?AfxDllCanUnloadNow@@YGJXZ 5f576fa6 f   oledll.obj
 0001:000760a0       ??0COleDropSource@@QAE@XZ  5f5770a0 f   oledrop1.obj
 0001:00076182       ?QueryContinueDrag@COleDropSource@@UAEJHK@Z 5f577182 f   oledrop1.obj
 0001:000761e3       ?GiveFeedback@COleDropSource@@UAEJK@Z 5f5771e3 f   oledrop1.obj
 0001:0007620f       ?OnBeginDrag@COleDropSource@@UAEHPAVCWnd@@@Z 5f57720f f   oledrop1.obj
 0001:0007638c       ?_GetBaseInterfaceMap@COleDropSource@@KGPBUAFX_INTERFACEMAP@@XZ 5f57738c f   oledrop1.obj
 0001:00076396       ?GetInterfaceMap@COleDropSource@@MBEPBUAFX_INTERFACEMAP@@XZ 5f577396 f   oledrop1.obj
 0001:000763a6       ?AddRef@XDropSource@COleDropSource@@UAGKXZ 5f5773a6 f   oledrop1.obj
 0001:000763c1       ?Release@XDropSource@COleDropSource@@UAGKXZ 5f5773c1 f   oledrop1.obj
 0001:000763dc       ?QueryInterface@XDropSource@COleDropSource@@UAGJABU_GUID@@PAPAX@Z 5f5773dc f   oledrop1.obj
 0001:000763ff       ?QueryContinueDrag@XDropSource@COleDropSource@@UAGJHK@Z 5f5773ff f   oledrop1.obj
 0001:00076425       ?GiveFeedback@XDropSource@COleDropSource@@UAGJK@Z 5f577425 f   oledrop1.obj
 0001:000764a6       ?DoDragDrop@COleDataSource@@QAEKKPBUtagRECT@@PAVCOleDropSource@@@Z 5f5774a6 f   oledrop1.obj
 0001:00076690       ?Dump@COleDropSource@@UBEXAAVCDumpContext@@@Z 5f577690 f   oledrop1.obj
 0001:00076740       ??_GCOleDropSource@@UAEPAXI@Z 5f577740 f i oledrop1.obj
 0001:00076770       ??0XDropSource@COleDropSource@@QAE@XZ 5f577770 f i oledrop1.obj
 0001:00076790       ??0COleDropTarget@@QAE@XZ  5f577790 f   oledrop2.obj
 0001:0007687b       ??1COleDropTarget@@UAE@XZ  5f57787b f   oledrop2.obj
 0001:00076909       ?Register@COleDropTarget@@QAEHPAVCWnd@@@Z 5f577909 f   oledrop2.obj
 0001:00076a0c       ?Revoke@COleDropTarget@@UAEXXZ 5f577a0c f   oledrop2.obj
 0001:00076abd       ?OnDragScroll@COleDropTarget@@UAEKPAVCWnd@@KVCPoint@@@Z 5f577abd f   oledrop2.obj
 0001:00076e79       ?OnDragEnter@COleDropTarget@@UAEKPAVCWnd@@PAVCOleDataObject@@KVCPoint@@@Z 5f577e79 f   oledrop2.obj
 0001:00076ee9       ?OnDragOver@COleDropTarget@@UAEKPAVCWnd@@PAVCOleDataObject@@KVCPoint@@@Z 5f577ee9 f   oledrop2.obj
 0001:00076f59       ?OnDrop@COleDropTarget@@UAEHPAVCWnd@@PAVCOleDataObject@@KVCPoint@@@Z 5f577f59 f   oledrop2.obj
 0001:00076fc9       ?OnDropEx@COleDropTarget@@UAEKPAVCWnd@@PAVCOleDataObject@@KKVCPoint@@@Z 5f577fc9 f   oledrop2.obj
 0001:0007703e       ?OnDragLeave@COleDropTarget@@UAEXPAVCWnd@@@Z 5f57803e f   oledrop2.obj
 0001:0007709c       ?_GetBaseInterfaceMap@COleDropTarget@@KGPBUAFX_INTERFACEMAP@@XZ 5f57809c f   oledrop2.obj
 0001:000770a6       ?GetInterfaceMap@COleDropTarget@@MBEPBUAFX_INTERFACEMAP@@XZ 5f5780a6 f   oledrop2.obj
 0001:000770b6       ?AddRef@XDropTarget@COleDropTarget@@UAGKXZ 5f5780b6 f   oledrop2.obj
 0001:000770d1       ?Release@XDropTarget@COleDropTarget@@UAGKXZ 5f5780d1 f   oledrop2.obj
 0001:000770ec       ?QueryInterface@XDropTarget@COleDropTarget@@UAGJABU_GUID@@PAPAX@Z 5f5780ec f   oledrop2.obj
 0001:0007710f       ?_AfxFilterDropEffect@@YGKKK@Z 5f57810f f   oledrop2.obj
 0001:00077184       ?DragEnter@XDropTarget@COleDropTarget@@UAGJPAUIDataObject@@KU_POINTL@@PAK@Z 5f578184 f   oledrop2.obj
 0001:000773b9       ?DragOver@XDropTarget@COleDropTarget@@UAGJKU_POINTL@@PAK@Z 5f5783b9 f   oledrop2.obj
 0001:000775b3       ?DragLeave@XDropTarget@COleDropTarget@@UAGJXZ 5f5785b3 f   oledrop2.obj
 0001:000776b8       ?Drop@XDropTarget@COleDropTarget@@UAGJPAUIDataObject@@KU_POINTL@@PAK@Z 5f5786b8 f   oledrop2.obj
 0001:00077933       ?AssertValid@COleDropTarget@@UBEXXZ 5f578933 f   oledrop2.obj
 0001:0007796b       ?Dump@COleDropTarget@@UBEXAAVCDumpContext@@@Z 5f57896b f   oledrop2.obj
 0001:00077a00       ??_GCOleDropTarget@@UAEPAXI@Z 5f578a00 f i oledrop2.obj
 0001:00077a30       ??0XDropTarget@COleDropTarget@@QAE@XZ 5f578a30 f i oledrop2.obj
 0001:00077a50       ?BeginBusyState@COleMessageFilter@@UAEXXZ 5f578a50 f   olemsgf.obj
 0001:00077a7a       ?EndBusyState@COleMessageFilter@@UAEXXZ 5f578a7a f   olemsgf.obj
 0001:00077aad       ?OnMessagePending@COleMessageFilter@@UAEHPBUtagMSG@@@Z 5f578aad f   olemsgf.obj
 0001:00077aef       ?IsSignificantMessage@COleMessageFilter@@UAEHPAUtagMSG@@@Z 5f578aef f   olemsgf.obj
 0001:00077b76       ?OnBusyDialog@COleMessageFilter@@UAEHPAUHTASK__@@@Z 5f578b76 f   olemsgf.obj
 0001:00077c7a       ?OnNotRespondingDialog@COleMessageFilter@@UAEHPAUHTASK__@@@Z 5f578c7a f   olemsgf.obj
 0001:00077d7e       ?_GetBaseInterfaceMap@COleMessageFilter@@KGPBUAFX_INTERFACEMAP@@XZ 5f578d7e f   olemsgf.obj
 0001:00077d88       ?GetInterfaceMap@COleMessageFilter@@MBEPBUAFX_INTERFACEMAP@@XZ 5f578d88 f   olemsgf.obj
 0001:00077d98       ?AddRef@XMessageFilter@COleMessageFilter@@UAGKXZ 5f578d98 f   olemsgf.obj
 0001:00077db3       ?Release@XMessageFilter@COleMessageFilter@@UAGKXZ 5f578db3 f   olemsgf.obj
 0001:00077dce       ?QueryInterface@XMessageFilter@COleMessageFilter@@UAGJABU_GUID@@PAPAX@Z 5f578dce f   olemsgf.obj
 0001:00077df1       ?HandleInComingCall@XMessageFilter@COleMessageFilter@@UAGKKPAUHTASK__@@KPAUtagINTERFACEINFO@@@Z 5f578df1 f   olemsgf.obj
 0001:00077e67       ?RetryRejectedCall@XMessageFilter@COleMessageFilter@@UAGKPAUHTASK__@@KK@Z 5f578e67 f   olemsgf.obj
 0001:00077f91       ?MessagePending@XMessageFilter@COleMessageFilter@@UAGKPAUHTASK__@@KK@Z 5f578f91 f   olemsgf.obj
 0001:00078106       ?AssertValid@COleMessageFilter@@UBEXXZ 5f579106 f   olemsgf.obj
 0001:00078119       ?Dump@COleMessageFilter@@UBEXAAVCDumpContext@@@Z 5f579119 f   olemsgf.obj
 0001:00078220       ??0COleServerDoc@@QAE@XZ   5f579220 f   olesvr1.obj
 0001:00078339       ??1COleServerDoc@@UAE@XZ   5f579339 f   olesvr1.obj
 0001:000784c8       ?DeleteContents@COleServerDoc@@UAEXXZ 5f5794c8 f   olesvr1.obj
 0001:00078599       ?GetEmbeddedItem@COleServerDoc@@QAEPAVCOleServerItem@@XZ 5f579599 f   olesvr1.obj
 0001:000785f4       ?GetDocObjectServer@COleServerDoc@@MAEPAVCDocObjectServer@@PAUIOleDocumentSite@@@Z 5f5795f4 f   olesvr1.obj
 0001:00078603       ?OnExecOleCmd@COleServerDoc@@MAEJPBU_GUID@@KKPAUtagVARIANT@@1@Z 5f579603 f   olesvr1.obj
 0001:00078615       ?GetInterfaceHook@COleServerDoc@@MAEPAUIUnknown@@PBX@Z 5f579615 f   olesvr1.obj
 0001:000786c0       ?ActivateDocObject@COleServerDoc@@QAEXXZ 5f5796c0 f   olesvr1.obj
 0001:000786e5       ?NotifyRename@COleServerDoc@@QAEXPBD@Z 5f5796e5 f   olesvr1.obj
 0001:000787c6       ?NotifyAllItems@COleServerDoc@@IAEXW4OLE_NOTIFICATION@@K@Z 5f5797c6 f   olesvr1.obj
 0001:00078820       ?UpdateAllItems@COleServerDoc@@QAEXPAVCOleServerItem@@JPAVCObject@@W4tagDVASPECT@@@Z 5f579820 f   olesvr1.obj
 0001:0007888d       ?OnUpdate@COleServerItem@@UAEXPAV1@JPAVCObject@@W4tagDVASPECT@@@Z 5f57988d f   olesvr1.obj
 0001:000788a6       ?GetZoomFactor@COleServerDoc@@QBEHPAUtagSIZE@@0PBUtagRECT@@@Z 5f5798a6 f   olesvr1.obj
 0001:00078b3c       ?GetItemPosition@COleServerDoc@@QBEXPAUtagRECT@@@Z 5f579b3c f   olesvr1.obj
 0001:00078bf4       ?GetItemClipRect@COleServerDoc@@QBEXPAUtagRECT@@@Z 5f579bf4 f   olesvr1.obj
 0001:00078cac       ?OnGetLinkedItem@COleServerDoc@@UAEPAVCOleServerItem@@PBD@Z 5f579cac f   olesvr1.obj
 0001:00078d7c       ?OnClose@COleServerDoc@@MAEXW4tagOLECLOSE@@@Z 5f579d7c f   olesvr1.obj
 0001:00078efe       ?SaveModifiedPrompt@COleServerDoc@@IAEHXZ 5f579efe f   olesvr1.obj
 0001:0007902a       ?CanCloseFrame@COleServerDoc@@UAEHPAVCFrameWnd@@@Z 5f57a02a f   olesvr1.obj
 0001:0007906a       ?GetFileTypeString@COleServerDoc@@MAEHAAVCString@@@Z 5f57a06a f   olesvr1.obj
 0001:000790bf       ?OnSetHostNames@COleServerDoc@@MAEXPBD0@Z 5f57a0bf f   olesvr1.obj
 0001:00079238       ?SaveEmbedding@COleServerDoc@@QAEXXZ 5f57a238 f   olesvr1.obj
 0001:000792ab       ?OnUpdateDocument@COleServerDoc@@UAEHXZ 5f57a2ab f   olesvr1.obj
 0001:00079382       ?GetMoniker@COleServerDoc@@UAEPAUIMoniker@@W4tagOLEGETMONIKER@@@Z 5f57a382 f   olesvr1.obj
 0001:000793ea       ?SaveModified@COleServerDoc@@MAEHXZ 5f57a3ea f   olesvr1.obj
 0001:0007944b       ?GetDefaultMenu@COleServerDoc@@MAEPAUHMENU__@@XZ 5f57a44b f   olesvr1.obj
 0001:000794bd       ?GetDefaultAccelerator@COleServerDoc@@MAEPAUHACCEL__@@XZ 5f57a4bd f   olesvr1.obj
 0001:0007952f       ?_GetBaseMessageMap@COleServerDoc@@KGPBUAFX_MSGMAP@@XZ 5f57a52f f   olesvr1.obj
 0001:00079539       ?GetMessageMap@COleServerDoc@@MBEPBUAFX_MSGMAP@@XZ 5f57a539 f   olesvr1.obj
 0001:00079549       ?OnFileUpdate@COleServerDoc@@IAEXXZ 5f57a549 f   olesvr1.obj
 0001:000795af       ?OnFileSaveCopyAs@COleServerDoc@@IAEXXZ 5f57a5af f   olesvr1.obj
 0001:000796d6       ?UpdateUsingHostObj@COleServerDoc@@IAEXIPAVCCmdUI@@@Z 5f57a6d6 f   olesvr1.obj
 0001:000797a5       ?OnUpdateFileExit@COleServerDoc@@IAEXPAVCCmdUI@@@Z 5f57a7a5 f   olesvr1.obj
 0001:000797fc       ?OnUpdateFileUpdate@COleServerDoc@@IAEXPAVCCmdUI@@@Z 5f57a7fc f   olesvr1.obj
 0001:00079853       ?OnSaveDocument@COleServerDoc@@UAEHPBD@Z 5f57a853 f   olesvr1.obj
 0001:00079923       ?OnCloseDocument@COleServerDoc@@UAEXXZ 5f57a923 f   olesvr1.obj
 0001:00079ab0       ?OnShowDocument@COleServerDoc@@MAEXH@Z 5f57aab0 f   olesvr1.obj
 0001:00079f11       ?OnNewEmbedding@COleServerDoc@@MAEXPAUIStorage@@@Z 5f57af11 f   olesvr1.obj
 0001:0007a069       ?OnOpenEmbedding@COleServerDoc@@MAEXPAUIStorage@@@Z 5f57b069 f   olesvr1.obj
 0001:0007a1c4       ?OnSaveEmbedding@COleServerDoc@@MAEXPAUIStorage@@@Z 5f57b1c4 f   olesvr1.obj
 0001:0007a2fd       ?_AfxGetWindow32@@YGPAUHWND__@@PAU1@@Z 5f57b2fd f   olesvr1.obj
 0001:0007a364       ?ActivateInPlace@COleServerDoc@@QAEHXZ 5f57b364 f   olesvr1.obj
 0001:0007acd1       ?CreateInPlaceFrame@COleServerDoc@@MAEPAVCOleIPFrameWnd@@PAVCWnd@@@Z 5f57bcd1 f   olesvr1.obj
 0001:0007ae73       ?DestroyInPlaceFrame@COleServerDoc@@MAEXPAVCOleIPFrameWnd@@@Z 5f57be73 f   olesvr1.obj
 0001:0007afe7       ?ConnectView@COleServerDoc@@IAEXPAVCWnd@@PAVCView@@@Z 5f57bfe7 f   olesvr1.obj
 0001:0007b084       ?OnFrameWindowActivate@COleServerDoc@@MAEXH@Z 5f57c084 f   olesvr1.obj
 0001:0007b154       ?OnDocWindowActivate@COleServerDoc@@MAEXH@Z 5f57c154 f   olesvr1.obj
 0001:0007b335       ?OnShowControlBars@COleServerDoc@@MAEXPAVCFrameWnd@@H@Z 5f57c335 f   olesvr1.obj
 0001:0007b46a       ?OnResizeBorder@COleServerDoc@@UAEXPBUtagRECT@@PAUIOleInPlaceUIWindow@@H@Z 5f57c46a f   olesvr1.obj
 0001:0007b6ff       ?OnDeactivate@COleServerDoc@@UAEXXZ 5f57c6ff f   olesvr1.obj
 0001:0007b908       ?OnDeactivateUI@COleServerDoc@@UAEXH@Z 5f57c908 f   olesvr1.obj
 0001:0007bb2c       ?OnSetItemRects@COleServerDoc@@MAEXPBUtagRECT@@0@Z 5f57cb2c f   olesvr1.obj
 0001:0007bbf1       ?OnReactivateAndUndo@COleServerDoc@@MAEHXZ 5f57cbf1 f   olesvr1.obj
 0001:0007bbfe       ?RequestPositionChange@COleServerDoc@@QAEXPBUtagRECT@@@Z 5f57cbfe f   olesvr1.obj
 0001:0007bcb0       ?ScrollContainerBy@COleServerDoc@@QAEHVCSize@@@Z 5f57ccb0 f   olesvr1.obj
 0001:0007bd56       ?DeactivateAndUndo@COleServerDoc@@QAEHXZ 5f57cd56 f   olesvr1.obj
 0001:0007bde6       ?DiscardUndoState@COleServerDoc@@QAEHXZ 5f57cde6 f   olesvr1.obj
 0001:0007be76       ?_GetBaseInterfaceMap@COleServerDoc@@KGPBUAFX_INTERFACEMAP@@XZ 5f57ce76 f   olesvr1.obj
 0001:0007be80       ?GetInterfaceMap@COleServerDoc@@MBEPBUAFX_INTERFACEMAP@@XZ 5f57ce80 f   olesvr1.obj
 0001:0007be90       ?AddRef@XPersistStorage@COleServerDoc@@UAGKXZ 5f57ce90 f   olesvr1.obj
 0001:0007bead       ?Release@XPersistStorage@COleServerDoc@@UAGKXZ 5f57cead f   olesvr1.obj
 0001:0007beca       ?QueryInterface@XPersistStorage@COleServerDoc@@UAGJABU_GUID@@PAPAX@Z 5f57ceca f   olesvr1.obj
 0001:0007beef       ?GetClassID@XPersistStorage@COleServerDoc@@UAGJPAU_GUID@@@Z 5f57ceef f   olesvr1.obj
 0001:0007bf26       ?IsDirty@XPersistStorage@COleServerDoc@@UAGJXZ 5f57cf26 f   olesvr1.obj
 0001:0007bf59       ?InitNew@XPersistStorage@COleServerDoc@@UAGJPAUIStorage@@@Z 5f57cf59 f   olesvr1.obj
 0001:0007c060       ?Load@XPersistStorage@COleServerDoc@@UAGJPAUIStorage@@@Z 5f57d060 f   olesvr1.obj
 0001:0007c17e       ?Save@XPersistStorage@COleServerDoc@@UAGJPAUIStorage@@H@Z 5f57d17e f   olesvr1.obj
 0001:0007c33b       ?SaveCompleted@XPersistStorage@COleServerDoc@@UAGJPAUIStorage@@@Z 5f57d33b f   olesvr1.obj
 0001:0007c448       ?HandsOffStorage@XPersistStorage@COleServerDoc@@UAGJXZ 5f57d448 f   olesvr1.obj
 0001:0007c54c       ?AddRef@XOleObject@COleServerDoc@@UAGKXZ 5f57d54c f   olesvr1.obj
 0001:0007c569       ?Release@XOleObject@COleServerDoc@@UAGKXZ 5f57d569 f   olesvr1.obj
 0001:0007c586       ?QueryInterface@XOleObject@COleServerDoc@@UAGJABU_GUID@@PAPAX@Z 5f57d586 f   olesvr1.obj
 0001:0007c5ab       ?SetClientSite@XOleObject@COleServerDoc@@UAGJPAUIOleClientSite@@@Z 5f57d5ab f   olesvr1.obj
 0001:0007c68c       ?GetClientSite@XOleObject@COleServerDoc@@UAGJPAPAUIOleClientSite@@@Z 5f57d68c f   olesvr1.obj
 0001:0007c6e5       ?SetHostNames@XOleObject@COleServerDoc@@UAGJPBG0@Z 5f57d6e5 f   olesvr1.obj
 0001:0007c884       ?Close@XOleObject@COleServerDoc@@UAGJK@Z 5f57d884 f   olesvr1.obj
 0001:0007c988       ?SetMoniker@XOleObject@COleServerDoc@@UAGJKPAUIMoniker@@@Z 5f57d988 f   olesvr1.obj
 0001:0007ca62       ?GetMoniker@XOleObject@COleServerDoc@@UAGJKKPAPAUIMoniker@@@Z 5f57da62 f   olesvr1.obj
 0001:0007caa1       ?InitFromData@XOleObject@COleServerDoc@@UAGJPAUIDataObject@@HK@Z 5f57daa1 f   olesvr1.obj
 0001:0007cc23       ?GetClipboardData@XOleObject@COleServerDoc@@UAGJKPAPAUIDataObject@@@Z 5f57dc23 f   olesvr1.obj
 0001:0007cde5       ?DoVerb@XOleObject@COleServerDoc@@UAGJJPAUtagMSG@@PAUIOleClientSite@@JPAUHWND__@@PBUtagRECT@@@Z 5f57dde5 f   olesvr1.obj
 0001:0007cf3f       ?EnumVerbs@XOleObject@COleServerDoc@@UAGJPAPAUIEnumOLEVERB@@@Z 5f57df3f f   olesvr1.obj
 0001:0007cfb3       ?Update@XOleObject@COleServerDoc@@UAGJXZ 5f57dfb3 f   olesvr1.obj
 0001:0007d0fc       ?IsUpToDate@XOleObject@COleServerDoc@@UAGJXZ 5f57e0fc f   olesvr1.obj
 0001:0007d24a       ?GetUserClassID@XOleObject@COleServerDoc@@UAGJPAU_GUID@@@Z 5f57e24a f   olesvr1.obj
 0001:0007d281       ?GetUserType@XOleObject@COleServerDoc@@UAGJKPAPAG@Z 5f57e281 f   olesvr1.obj
 0001:0007d2f9       ?SetExtent@XOleObject@COleServerDoc@@UAGJKPAUtagSIZE@@@Z 5f57e2f9 f   olesvr1.obj
 0001:0007d46c       ?GetExtent@XOleObject@COleServerDoc@@UAGJKPAUtagSIZE@@@Z 5f57e46c f   olesvr1.obj
 0001:0007d5f1       ?Advise@XOleObject@COleServerDoc@@UAGJPAUIAdviseSink@@PAK@Z 5f57e5f1 f   olesvr1.obj
 0001:0007d750       ?Unadvise@XOleObject@COleServerDoc@@UAGJK@Z 5f57e750 f   olesvr1.obj
 0001:0007d8ab       ?EnumAdvise@XOleObject@COleServerDoc@@UAGJPAPAUIEnumSTATDATA@@@Z 5f57e8ab f   olesvr1.obj
 0001:0007da06       ?GetMiscStatus@XOleObject@COleServerDoc@@UAGJKPAK@Z 5f57ea06 f   olesvr1.obj
 0001:0007da7e       ?SetColorScheme@XOleObject@COleServerDoc@@UAGJPAUtagLOGPALETTE@@@Z 5f57ea7e f   olesvr1.obj
 0001:0007dbc6       ?AddRef@XDataObject@COleServerDoc@@UAGKXZ 5f57ebc6 f   olesvr1.obj
 0001:0007dbe3       ?Release@XDataObject@COleServerDoc@@UAGKXZ 5f57ebe3 f   olesvr1.obj
 0001:0007dc00       ?QueryInterface@XDataObject@COleServerDoc@@UAGJABU_GUID@@PAPAX@Z 5f57ec00 f   olesvr1.obj
 0001:0007dc25       ?GetData@XDataObject@COleServerDoc@@UAGJPAUtagFORMATETC@@PAUtagSTGMEDIUM@@@Z 5f57ec25 f   olesvr1.obj
 0001:0007dd84       ?GetDataHere@XDataObject@COleServerDoc@@UAGJPAUtagFORMATETC@@PAUtagSTGMEDIUM@@@Z 5f57ed84 f   olesvr1.obj
 0001:0007dee3       ?QueryGetData@XDataObject@COleServerDoc@@UAGJPAUtagFORMATETC@@@Z 5f57eee3 f   olesvr1.obj
 0001:0007e03e       ?GetCanonicalFormatEtc@XDataObject@COleServerDoc@@UAGJPAUtagFORMATETC@@0@Z 5f57f03e f   olesvr1.obj
 0001:0007e04a       ?SetData@XDataObject@COleServerDoc@@UAGJPAUtagFORMATETC@@PAUtagSTGMEDIUM@@H@Z 5f57f04a f   olesvr1.obj
 0001:0007e1ad       ?EnumFormatEtc@XDataObject@COleServerDoc@@UAGJKPAPAUIEnumFORMATETC@@@Z 5f57f1ad f   olesvr1.obj
 0001:0007e30c       ?DAdvise@XDataObject@COleServerDoc@@UAGJPAUtagFORMATETC@@KPAUIAdviseSink@@PAK@Z 5f57f30c f   olesvr1.obj
 0001:0007e473       ?DUnadvise@XDataObject@COleServerDoc@@UAGJK@Z 5f57f473 f   olesvr1.obj
 0001:0007e5ce       ?EnumDAdvise@XDataObject@COleServerDoc@@UAGJPAPAUIEnumSTATDATA@@@Z 5f57f5ce f   olesvr1.obj
 0001:0007e729       ?AddRef@XOleInPlaceObject@COleServerDoc@@UAGKXZ 5f57f729 f   olesvr1.obj
 0001:0007e746       ?Release@XOleInPlaceObject@COleServerDoc@@UAGKXZ 5f57f746 f   olesvr1.obj
 0001:0007e763       ?QueryInterface@XOleInPlaceObject@COleServerDoc@@UAGJABU_GUID@@PAPAX@Z 5f57f763 f   olesvr1.obj
 0001:0007e788       ?GetWindow@XOleInPlaceObject@COleServerDoc@@UAGJPAPAUHWND__@@@Z 5f57f788 f   olesvr1.obj
 0001:0007e7bf       ?ContextSensitiveHelp@XOleInPlaceObject@COleServerDoc@@UAGJH@Z 5f57f7bf f   olesvr1.obj
 0001:0007e7f6       ?InPlaceDeactivate@XOleInPlaceObject@COleServerDoc@@UAGJXZ 5f57f7f6 f   olesvr1.obj
 0001:0007e921       ?UIDeactivate@XOleInPlaceObject@COleServerDoc@@UAGJXZ 5f57f921 f   olesvr1.obj
 0001:0007ea73       ?SetObjectRects@XOleInPlaceObject@COleServerDoc@@UAGJPBUtagRECT@@0@Z 5f57fa73 f   olesvr1.obj
 0001:0007eb5f       ?ReactivateAndUndo@XOleInPlaceObject@COleServerDoc@@UAGJXZ 5f57fb5f f   olesvr1.obj
 0001:0007ec56       ?AddRef@XOleInPlaceActiveObject@COleServerDoc@@UAGKXZ 5f57fc56 f   olesvr1.obj
 0001:0007ec73       ?Release@XOleInPlaceActiveObject@COleServerDoc@@UAGKXZ 5f57fc73 f   olesvr1.obj
 0001:0007ec90       ?QueryInterface@XOleInPlaceActiveObject@COleServerDoc@@UAGJABU_GUID@@PAPAX@Z 5f57fc90 f   olesvr1.obj
 0001:0007ecb5       ?GetWindow@XOleInPlaceActiveObject@COleServerDoc@@UAGJPAPAUHWND__@@@Z 5f57fcb5 f   olesvr1.obj
 0001:0007ecf0       ?ContextSensitiveHelp@XOleInPlaceActiveObject@COleServerDoc@@UAGJH@Z 5f57fcf0 f   olesvr1.obj
 0001:0007edff       ?TranslateAcceleratorA@XOleInPlaceActiveObject@COleServerDoc@@UAGJPAUtagMSG@@@Z 5f57fdff f   olesvr1.obj
 0001:0007ef39       ?OnFrameWindowActivate@XOleInPlaceActiveObject@COleServerDoc@@UAGJH@Z 5f57ff39 f   olesvr1.obj
 0001:0007f022       ?OnDocWindowActivate@XOleInPlaceActiveObject@COleServerDoc@@UAGJH@Z 5f580022 f   olesvr1.obj
 0001:0007f10b       ?ResizeBorder@XOleInPlaceActiveObject@COleServerDoc@@UAGJPBUtagRECT@@PAUIOleInPlaceUIWindow@@H@Z 5f58010b f   olesvr1.obj
 0001:0007f1fc       ?EnableModeless@XOleInPlaceActiveObject@COleServerDoc@@UAGJH@Z 5f5801fc f   olesvr1.obj
 0001:0007f370       ?AssertValid@COleServerDoc@@UBEXXZ 5f580370 f   olesvr1.obj
 0001:0007f3c9       ?Dump@COleServerDoc@@UBEXAAVCDumpContext@@@Z 5f5803c9 f   olesvr1.obj
 0001:0007f4e3       ?GetDocument@COleServerItem@@QBEPAVCOleServerDoc@@XZ 5f5804e3 f   olesvr1.obj
 0001:0007f507       ?NotifyChanged@COleServerItem@@QAEXW4tagDVASPECT@@@Z 5f580507 f   olesvr1.obj
 0001:0007f535       ?GetItemName@COleServerItem@@QBEABVCString@@XZ 5f580535 f   olesvr1.obj
 0001:0007f559       ?SetItemName@COleServerItem@@QAEXPBD@Z 5f580559 f   olesvr1.obj
 0001:0007f5d7       ?IsLinkedItem@COleServerItem@@QBEHXZ 5f5805d7 f   olesvr1.obj
 0001:0007f60b       ?GetDataSource@COleServerItem@@IAEPAVCOleDataSource@@XZ 5f58060b f   olesvr1.obj
 0001:0007f62f       ?NotifyChanged@COleServerDoc@@QAEXXZ 5f58062f f   olesvr1.obj
 0001:0007f659       ?NotifyClosed@COleServerDoc@@QAEXXZ 5f580659 f   olesvr1.obj
 0001:0007f683       ?NotifySaved@COleServerDoc@@QAEXXZ 5f580683 f   olesvr1.obj
 0001:0007f6ad       ?IsEmbedded@COleServerDoc@@QBEHXZ 5f5806ad f   olesvr1.obj
 0001:0007f6d1       ?IsDocObject@COleServerDoc@@QBEHXZ 5f5806d1 f   olesvr1.obj
 0001:0007f6fe       ?IsInPlaceActive@COleServerDoc@@QBEHXZ 5f5806fe f   olesvr1.obj
 0001:0007f730       ??_ECOleServerDoc@@UAEPAXI@Z 5f580730 f i olesvr1.obj
 0001:0007f730       ??_GCOleServerDoc@@UAEPAXI@Z 5f580730 f i olesvr1.obj
 0001:0007f760       ??0XPersistStorage@COleServerDoc@@QAE@XZ 5f580760 f i olesvr1.obj
 0001:0007f780       ??0XOleObject@COleServerDoc@@QAE@XZ 5f580780 f i olesvr1.obj
 0001:0007f7a0       ??0XDataObject@COleServerDoc@@QAE@XZ 5f5807a0 f i olesvr1.obj
 0001:0007f7c0       ??0XOleInPlaceObject@COleServerDoc@@QAE@XZ 5f5807c0 f i olesvr1.obj
 0001:0007f7e0       ??0XOleInPlaceActiveObject@COleServerDoc@@QAE@XZ 5f5807e0 f i olesvr1.obj
 0001:0007f800       ??0IPersistStorage@@QAE@XZ 5f580800 f i olesvr1.obj
 0001:0007f820       ??0IDropTarget@@QAE@XZ     5f580820 f i olesvr1.obj
 0001:0007f820       ??0IOleObject@@QAE@XZ      5f580820 f i olesvr1.obj
 0001:0007f820       ??0IDropSource@@QAE@XZ     5f580820 f i olesvr1.obj
 0001:0007f840       ??0IOleInPlaceActiveObject@@QAE@XZ 5f580840 f i olesvr1.obj
 0001:0007f840       ??0IOleInPlaceObject@@QAE@XZ 5f580840 f i olesvr1.obj
 0001:0007f860       ??0COleServerItem@@IAE@PAVCOleServerDoc@@H@Z 5f580860 f   olesvr2.obj
 0001:0007f9d6       ??1COleServerItem@@UAE@XZ  5f5809d6 f   olesvr2.obj
 0001:0007fb09       ?IsBlank@COleServerItem@@MBEHXZ 5f580b09 f   olesvr2.obj
 0001:0007fb19       ?IsConnected@COleServerItem@@QBEHXZ 5f580b19 f   olesvr2.obj
 0001:0007fb5a       ?NotifyClient@COleServerItem@@QAEXW4OLE_NOTIFICATION@@K@Z 5f580b5a f   olesvr2.obj
 0001:0007fc4c       ?GetDataObject@COleServerItem@@QAEPAUIDataObject@@XZ 5f580c4c f   olesvr2.obj
 0001:0007fc92       ?GetOleObject@COleServerItem@@QAEPAUIOleObject@@XZ 5f580c92 f   olesvr2.obj
 0001:0007fcd8       ?OnQueryUpdateItems@COleServerItem@@UAEHXZ 5f580cd8 f   olesvr2.obj
 0001:0007fd4a       ?OnUpdateItems@COleServerItem@@UAEXXZ 5f580d4a f   olesvr2.obj
 0001:0007fdc5       ?OnSetExtent@COleServerItem@@UAEHW4tagDVASPECT@@ABVCSize@@@Z 5f580dc5 f   olesvr2.obj
 0001:0007fe05       ?OnGetExtent@COleServerItem@@UAEHW4tagDVASPECT@@AAVCSize@@@Z 5f580e05 f   olesvr2.obj
 0001:0007fe6b       ?OnDoVerb@COleServerItem@@UAEXJ@Z 5f580e6b f   olesvr2.obj
 0001:0007ff08       ?OnDrawEx@COleServerItem@@UAEHPAVCDC@@W4tagDVASPECT@@AAVCSize@@@Z 5f580f08 f   olesvr2.obj
 0001:0007ff76       ?OnShow@COleServerItem@@MAEXXZ 5f580f76 f   olesvr2.obj
 0001:0007ffbb       ?OnOpen@COleServerItem@@MAEXXZ 5f580fbb f   olesvr2.obj
 0001:0008001c       ?OnHide@COleServerItem@@MAEXXZ 5f58101c f   olesvr2.obj
 0001:0008006a       ?GetMetafileData@COleServerItem@@MAEHPAUtagFORMATETC@@PAUtagSTGMEDIUM@@@Z 5f58106a f   olesvr2.obj
 0001:00080419       ?OnSetColorScheme@COleServerItem@@UAEHPBUtagLOGPALETTE@@@Z 5f581419 f   olesvr2.obj
 0001:0008043b       ?OnInitFromData@COleServerItem@@UAEHPAVCOleDataObject@@H@Z 5f58143b f   olesvr2.obj
 0001:00080467       ?CopyToClipboard@COleServerItem@@QAEXH@Z 5f581467 f   olesvr2.obj
 0001:000804a7       ?OnGetClipboardData@COleServerItem@@UAEPAVCOleDataSource@@HPAUtagPOINT@@PAUtagSIZE@@@Z 5f5814a7 f   olesvr2.obj
 0001:000805d9       ?DoDragDrop@COleServerItem@@QAEKPBUtagRECT@@VCPoint@@HK0@Z 5f5815d9 f   olesvr2.obj
 0001:000807e4       ?GetClipboardData@COleServerItem@@QAEXPAVCOleDataSource@@HPAUtagPOINT@@PAUtagSIZE@@@Z 5f5817e4 f   olesvr2.obj
 0001:000808fc       ?GetEmbedSourceData@COleServerItem@@QAEXPAUtagSTGMEDIUM@@@Z 5f5818fc f   olesvr2.obj
 0001:00080b5d       ?AddOtherClipboardData@COleServerItem@@QAEXPAVCOleDataSource@@@Z 5f581b5d f   olesvr2.obj
 0001:00080c56       ?GetMoniker@COleServerItem@@QAEPAUIMoniker@@W4tagOLEGETMONIKER@@@Z 5f581c56 f   olesvr2.obj
 0001:00080cb6       ?GetLinkSourceData@COleServerItem@@QAEHPAUtagSTGMEDIUM@@@Z 5f581cb6 f   olesvr2.obj
 0001:00080e8e       ?GetObjectDescriptorData@COleServerItem@@QAEXPAUtagPOINT@@PAUtagSIZE@@PAUtagSTGMEDIUM@@@Z 5f581e8e f   olesvr2.obj
 0001:0008100c       ?OnSaveEmbedding@COleServerItem@@MAEXPAUIStorage@@@Z 5f58200c f   olesvr2.obj
 0001:00081113       ?OnRenderGlobalData@COleServerItem@@UAEHPAUtagFORMATETC@@PAPAX@Z 5f582113 f   olesvr2.obj
 0001:00081135       ?OnRenderFileData@COleServerItem@@UAEHPAUtagFORMATETC@@PAVCFile@@@Z 5f582135 f   olesvr2.obj
 0001:00081157       ?OnRenderData@COleServerItem@@UAEHPAUtagFORMATETC@@PAUtagSTGMEDIUM@@@Z 5f582157 f   olesvr2.obj
 0001:00081207       ?OnSetData@COleServerItem@@UAEHPAUtagFORMATETC@@PAUtagSTGMEDIUM@@H@Z 5f582207 f   olesvr2.obj
 0001:00081229       ?_GetBaseInterfaceMap@COleServerItem@@KGPBUAFX_INTERFACEMAP@@XZ 5f582229 f   olesvr2.obj
 0001:00081233       ?GetInterfaceMap@COleServerItem@@MBEPBUAFX_INTERFACEMAP@@XZ 5f582233 f   olesvr2.obj
 0001:00081243       ?AddRef@XOleObject@COleServerItem@@UAGKXZ 5f582243 f   olesvr2.obj
 0001:0008125e       ?Release@XOleObject@COleServerItem@@UAGKXZ 5f58225e f   olesvr2.obj
 0001:00081279       ?QueryInterface@XOleObject@COleServerItem@@UAGJABU_GUID@@PAPAX@Z 5f582279 f   olesvr2.obj
 0001:0008129c       ?OnFinalRelease@COleServerItem@@UAEXXZ 5f58229c f   olesvr2.obj
 0001:0008133d       ?SetClientSite@XOleObject@COleServerItem@@UAGJPAUIOleClientSite@@@Z 5f58233d f   olesvr2.obj
 0001:00081349       ?GetClientSite@XOleObject@COleServerItem@@UAGJPAPAUIOleClientSite@@@Z 5f582349 f   olesvr2.obj
 0001:0008135e       ?SetHostNames@XOleObject@COleServerItem@@UAGJPBG0@Z 5f58235e f   olesvr2.obj
 0001:0008136a       ?Close@XOleObject@COleServerItem@@UAGJK@Z 5f58236a f   olesvr2.obj
 0001:00081376       ?SetMoniker@XOleObject@COleServerItem@@UAGJKPAUIMoniker@@@Z 5f582376 f   olesvr2.obj
 0001:00081382       ?GetMoniker@XOleObject@COleServerItem@@UAGJKKPAPAUIMoniker@@@Z 5f582382 f   olesvr2.obj
 0001:0008167f       ?InitFromData@XOleObject@COleServerItem@@UAGJPAUIDataObject@@HK@Z 5f58267f f   olesvr2.obj
 0001:0008168b       ?GetClipboardData@XOleObject@COleServerItem@@UAGJKPAPAUIDataObject@@@Z 5f58268b f   olesvr2.obj
 0001:000817f2       ?DoVerb@XOleObject@COleServerItem@@UAGJJPAUtagMSG@@PAUIOleClientSite@@JPAUHWND__@@PBUtagRECT@@@Z 5f5827f2 f   olesvr2.obj
 0001:000818f1       ?EnumVerbs@XOleObject@COleServerItem@@UAGJPAPAUIEnumOLEVERB@@@Z 5f5828f1 f   olesvr2.obj
 0001:00081938       ?Update@XOleObject@COleServerItem@@UAGJXZ 5f582938 f   olesvr2.obj
 0001:00081a26       ?IsUpToDate@XOleObject@COleServerItem@@UAGJXZ 5f582a26 f   olesvr2.obj
 0001:00081b19       ?GetUserClassID@XOleObject@COleServerItem@@UAGJPAU_GUID@@@Z 5f582b19 f   olesvr2.obj
 0001:00081b53       ?GetUserType@XOleObject@COleServerItem@@UAGJKPAPAG@Z 5f582b53 f   olesvr2.obj
 0001:00081b9e       ?SetExtent@XOleObject@COleServerItem@@UAGJKPAUtagSIZE@@@Z 5f582b9e f   olesvr2.obj
 0001:00081baa       ?GetExtent@XOleObject@COleServerItem@@UAGJKPAUtagSIZE@@@Z 5f582baa f   olesvr2.obj
 0001:00081cd4       ?Advise@XOleObject@COleServerItem@@UAGJPAUIAdviseSink@@PAK@Z 5f582cd4 f   olesvr2.obj
 0001:00081d54       ?Unadvise@XOleObject@COleServerItem@@UAGJK@Z 5f582d54 f   olesvr2.obj
 0001:00081db6       ?EnumAdvise@XOleObject@COleServerItem@@UAGJPAPAUIEnumSTATDATA@@@Z 5f582db6 f   olesvr2.obj
 0001:00081e21       ?GetMiscStatus@XOleObject@COleServerItem@@UAGJKPAK@Z 5f582e21 f   olesvr2.obj
 0001:00081e6c       ?SetColorScheme@XOleObject@COleServerItem@@UAGJPAUtagLOGPALETTE@@@Z 5f582e6c f   olesvr2.obj
 0001:00081f59       ?AddRef@XDataObject@COleServerItem@@UAGKXZ 5f582f59 f   olesvr2.obj
 0001:00081f74       ?Release@XDataObject@COleServerItem@@UAGKXZ 5f582f74 f   olesvr2.obj
 0001:00081f8f       ?QueryInterface@XDataObject@COleServerItem@@UAGJABU_GUID@@PAPAX@Z 5f582f8f f   olesvr2.obj
 0001:00081fb2       ?GetData@XDataObject@COleServerItem@@UAGJPAUtagFORMATETC@@PAUtagSTGMEDIUM@@@Z 5f582fb2 f   olesvr2.obj
 0001:00081fdd       ?GetDataHere@XDataObject@COleServerItem@@UAGJPAUtagFORMATETC@@PAUtagSTGMEDIUM@@@Z 5f582fdd f   olesvr2.obj
 0001:00082008       ?QueryGetData@XDataObject@COleServerItem@@UAGJPAUtagFORMATETC@@@Z 5f583008 f   olesvr2.obj
 0001:0008202f       ?GetCanonicalFormatEtc@XDataObject@COleServerItem@@UAGJPAUtagFORMATETC@@0@Z 5f58302f f   olesvr2.obj
 0001:0008203b       ?SetData@XDataObject@COleServerItem@@UAGJPAUtagFORMATETC@@PAUtagSTGMEDIUM@@H@Z 5f58303b f   olesvr2.obj
 0001:0008206a       ?EnumFormatEtc@XDataObject@COleServerItem@@UAGJKPAPAUIEnumFORMATETC@@@Z 5f58306a f   olesvr2.obj
 0001:00082095       ?DAdvise@XDataObject@COleServerItem@@UAGJPAUtagFORMATETC@@KPAUIAdviseSink@@PAK@Z 5f583095 f   olesvr2.obj
 0001:000821a1       ?DUnadvise@XDataObject@COleServerItem@@UAGJK@Z 5f5831a1 f   olesvr2.obj
 0001:00082203       ?EnumDAdvise@XDataObject@COleServerItem@@UAGJPAPAUIEnumSTATDATA@@@Z 5f583203 f   olesvr2.obj
 0001:0008226e       ?OnRenderGlobalData@CItemDataSource@COleServerItem@@MAEHPAUtagFORMATETC@@PAPAX@Z 5f58326e f   olesvr2.obj
 0001:000822af       ?OnRenderFileData@CItemDataSource@COleServerItem@@MAEHPAUtagFORMATETC@@PAVCFile@@@Z 5f5832af f   olesvr2.obj
 0001:000822f0       ?OnRenderData@CItemDataSource@COleServerItem@@MAEHPAUtagFORMATETC@@PAUtagSTGMEDIUM@@@Z 5f5832f0 f   olesvr2.obj
 0001:0008234c       ?OnSetData@CItemDataSource@COleServerItem@@MAEHPAUtagFORMATETC@@PAUtagSTGMEDIUM@@H@Z 5f58334c f   olesvr2.obj
 0001:00082391       ?AssertValid@COleServerItem@@UBEXXZ 5f583391 f   olesvr2.obj
 0001:000823dc       ?Dump@COleServerItem@@UBEXAAVCDumpContext@@@Z 5f5833dc f   olesvr2.obj
 0001:000824a0       ??_GCOleServerItem@@UAEPAXI@Z 5f5834a0 f i olesvr2.obj
 0001:000824a0       ??_ECOleServerItem@@UAEPAXI@Z 5f5834a0 f i olesvr2.obj
 0001:000824d0       ??0CItemDataSource@COleServerItem@@QAE@XZ 5f5834d0 f i olesvr2.obj
 0001:000824f0       ??1CItemDataSource@COleServerItem@@UAE@XZ 5f5834f0 f i olesvr2.obj
 0001:00082510       ??0XOleObject@COleServerItem@@QAE@XZ 5f583510 f i olesvr2.obj
 0001:00082530       ??0XDataObject@COleServerItem@@QAE@XZ 5f583530 f i olesvr2.obj
 0001:00082550       ??_GCItemDataSource@COleServerItem@@UAEPAXI@Z 5f583550 f i olesvr2.obj
 0001:00082550       ??_ECItemDataSource@COleServerItem@@UAEPAXI@Z 5f583550 f i olesvr2.obj
 0001:00082580       ??0CAfxOleSymbolTable@@QAE@H@Z 5f583580 f   olereg.obj
 0001:000825d3       ??1CAfxOleSymbolTable@@QAE@XZ 5f5835d3 f   olereg.obj
 0001:00082628       ?SetAt@CAfxOleSymbolTable@@QAEXHPBD@Z 5f583628 f   olereg.obj
 0001:000826a7       ?GetAt@CAfxOleSymbolTable@@QBEPBDH@Z 5f5836a7 f   olereg.obj
 0001:000826d4       ?AfxOleRegisterServerClassCompat@@YGHABU_GUID@@PBD11W4OLE_APPTYPE@@PAPBD3@Z 5f5836d4 f   olereg.obj
 0001:00082700       ?_AfxOleMakeSymbolTable@@YGHAAVCAfxOleSymbolTable@@ABU_GUID@@PBD22H22@Z 5f583700 f   olereg.obj
 0001:00082a18       ?AfxOleRegisterServerClass@@YGHABU_GUID@@PBD11W4OLE_APPTYPE@@PAPBD3H1@Z 5f583a18 f   olereg.obj
 0001:00082a4a       ?AfxOleRegisterServerClass@@YGHABU_GUID@@PBD11W4OLE_APPTYPE@@PAPBD3H11@Z 5f583a4a f   olereg.obj
 0001:00082ce6       ?AfxOleUnregisterServerClass@@YGHABU_GUID@@PBD11W4OLE_APPTYPE@@PAPBD3@Z 5f583ce6 f   olereg.obj
 0001:00082dff       ?AfxOleUnregisterHelper@@YGHPBQBD0HPAUHKEY__@@@Z 5f583dff f   olereg.obj
 0001:00082f6b       ?AfxOleRegisterHelper@@YGHPBQBD0HHPAUHKEY__@@@Z 5f583f6b f   olereg.obj
 0001:000831e0       ?GetArray@CAfxOleSymbolTable@@QAEPAPBDXZ 5f5841e0 f i olereg.obj
 0001:000831f0       ??0COleResizeBar@@QAE@XZ   5f5841f0 f   olebar.obj
 0001:00083254       ??1COleResizeBar@@UAE@XZ   5f584254 f   olebar.obj
 0001:000832a8       ?Create@COleResizeBar@@QAEHPAVCWnd@@KI@Z 5f5842a8 f   olebar.obj
 0001:00083342       ?_GetBaseMessageMap@COleResizeBar@@KGPBUAFX_MSGMAP@@XZ 5f584342 f   olebar.obj
 0001:0008334c       ?GetMessageMap@COleResizeBar@@MBEPBUAFX_MSGMAP@@XZ 5f58434c f   olebar.obj
 0001:0008335c       ?OnEraseBkgnd@COleResizeBar@@IAEHPAVCDC@@@Z 5f58435c f   olebar.obj
 0001:0008336e       ?OnPaint@COleResizeBar@@IAEXXZ 5f58436e f   olebar.obj
 0001:000833f9       ?OnSize@COleResizeBar@@IAEXIHH@Z 5f5843f9 f   olebar.obj
 0001:0008343f       ?OnSetCursor@COleResizeBar@@IAEHPAVCWnd@@II@Z 5f58443f f   olebar.obj
 0001:000834b1       ?OnLButtonDown@COleResizeBar@@IAEXIVCPoint@@@Z 5f5844b1 f   olebar.obj
 0001:0008360e       ?OnSizeParent@COleResizeBar@@IAEJIJ@Z 5f58460e f   olebar.obj
 0001:00083669       ?OnUpdateCmdUI@COleResizeBar@@UAEXPAVCFrameWnd@@H@Z 5f584669 f   olebar.obj
 0001:00083680       ??_GCOleResizeBar@@UAEPAXI@Z 5f584680 f i olebar.obj
 0001:000836b0       ?GetStandardProp@CCmdTarget@@IAEXPBUAFX_DISPMAP_ENTRY@@PAUtagVARIANT@@PAI@Z 5f5846b0 f   oledisp1.obj
 0001:00083894       ?SetStandardProp@CCmdTarget@@IAEJPBUAFX_DISPMAP_ENTRY@@PAUtagDISPPARAMS@@PAI@Z 5f584894 f   oledisp1.obj
 0001:00083b8a       ?GetEntryCount@CCmdTarget@@KGIPBUAFX_DISPMAP@@@Z 5f584b8a f   oledisp1.obj
 0001:00083c26       ?MemberIDFromName@CCmdTarget@@KGJPBUAFX_DISPMAP@@PBD@Z 5f584c26 f   oledisp1.obj
 0001:00083d2b       ?GetDispEntry@CCmdTarget@@IAGPBUAFX_DISPMAP_ENTRY@@J@Z 5f584d2b f   oledisp1.obj
 0001:00083ea6       ?GetNotSupported@CCmdTarget@@QAEXXZ 5f584ea6 f   oledisp1.obj
 0001:00083ec2       ?SetNotSupported@CCmdTarget@@QAEXXZ 5f584ec2 f   oledisp1.obj
 0001:00083ede       ?EnableAutomation@CCmdTarget@@QAEXXZ 5f584ede f   oledisp1.obj
 0001:00083f75       ?GetIDispatch@CCmdTarget@@QAEPAUIDispatch@@H@Z 5f584f75 f   oledisp1.obj
 0001:00083fd9       ?FromIDispatch@CCmdTarget@@SGPAV1@PAUIDispatch@@@Z 5f584fd9 f   oledisp1.obj
 0001:00084040       ?IsResultExpected@CCmdTarget@@QAEHXZ 5f585040 f   oledisp1.obj
 0001:00084063       ?Disconnect@COleDispatchImpl@@UAEXXZ 5f585063 f   oledisp1.obj
 0001:00084081       ?AllocSysString@CString@@QBEPAGXZ 5f585081 f   oledisp1.obj
 0001:000840f2       ?SetSysString@CString@@QBEPAGPAPAG@Z 5f5850f2 f   oledisp1.obj
 0001:000841bb       ?GetStackSize@CCmdTarget@@KGIPBEG@Z 5f5851bb f   oledisp1.obj
 0001:000842b4       ?PushStackArgs@CCmdTarget@@IAEJPAEPBEPAXGPAUtagDISPPARAMS@@PAIPAUtagVARIANT@@@Z 5f5852b4 f   oledisp1.obj
 0001:000849e2       ?CallMemberFunc@CCmdTarget@@IAEJPBUAFX_DISPMAP_ENTRY@@GPAUtagVARIANT@@PAUtagDISPPARAMS@@PAI@Z 5f5859e2 f   oledisp1.obj
 0001:0008506b       ?AddRef@COleDispatchImpl@@UAGKXZ 5f58606b f   oledisp1.obj
 0001:00085086       ?Release@COleDispatchImpl@@UAGKXZ 5f586086 f   oledisp1.obj
 0001:000850a1       ?QueryInterface@COleDispatchImpl@@UAGJABU_GUID@@PAPAX@Z 5f5860a1 f   oledisp1.obj
 0001:000850c4       ?GetTypeInfoCount@COleDispatchImpl@@UAGJPAI@Z 5f5860c4 f   oledisp1.obj
 0001:000850e9       ?GetTypeInfo@COleDispatchImpl@@UAGJIKPAPAUITypeInfo@@@Z 5f5860e9 f   oledisp1.obj
 0001:00085170       ?GetIDsOfNames@COleDispatchImpl@@UAGJABU_GUID@@PAPAGIKPAJ@Z 5f586170 f   oledisp1.obj
 0001:00085363       ?Invoke@COleDispatchImpl@@UAGJJABU_GUID@@KGPAUtagDISPPARAMS@@PAUtagVARIANT@@PAUtagEXCEPINFO@@PAI@Z 5f586363 f   oledisp1.obj
 0001:00085c98       ??1COleDispatchException@@UAE@XZ 5f586c98 f   oledisp1.obj
 0001:00085d0a       ?Process@COleDispatchException@@SGXPAUtagEXCEPINFO@@PBVCException@@@Z 5f586d0a f   oledisp1.obj
 0001:0008613b       ??0COleDispatchException@@QAE@PBDIG@Z 5f58713b f   oledisp1.obj
 0001:0008621b       ?GetErrorMessage@COleDispatchException@@UAEHPADIPAI@Z 5f58721b f   oledisp1.obj
 0001:0008628d       ?AfxThrowOleDispatchException@@YGXGPBDI@Z 5f58728d f   oledisp1.obj
 0001:0008634a       ?AfxThrowOleDispatchException@@YGXGII@Z 5f58734a f   oledisp1.obj
 0001:00086450       ??0COleDispatchImpl@@QAE@XZ 5f587450 f i oledisp1.obj
 0001:00086470       ??4COleDispatchImpl@@QAEAAV0@ABV0@@Z 5f587470 f i oledisp1.obj
 0001:00086490       ??0IDispatch@@QAE@XZ       5f587490 f i oledisp1.obj
 0001:000864b0       ??4IDispatch@@QAEAAU0@ABU0@@Z 5f5874b0 f i oledisp1.obj
 0001:000864d0       ??4IUnknown@@QAEAAU0@ABU0@@Z 5f5874d0 f i oledisp1.obj
 0001:000864e0       ??_GCOleDispatchException@@UAEPAXI@Z 5f5874e0 f i oledisp1.obj
 0001:000864e0       ??_ECOleDispatchException@@UAEPAXI@Z 5f5874e0 f i oledisp1.obj
 0001:00086510       ?AfxGetClassIDFromString@@YGJPBDPAU_GUID@@@Z 5f587510 f   oledisp2.obj
 0001:00086603       ??0COleDispatchDriver@@QAE@XZ 5f587603 f   oledisp2.obj
 0001:00086624       ??0COleDispatchDriver@@QAE@PAUIDispatch@@H@Z 5f587624 f   oledisp2.obj
 0001:00086645       ??0COleDispatchDriver@@QAE@ABV0@@Z 5f587645 f   oledisp2.obj
 0001:000866a6       ??4COleDispatchDriver@@QAEABV0@ABV0@@Z 5f5876a6 f   oledisp2.obj
 0001:0008670f       ?CreateDispatch@COleDispatchDriver@@QAEHABU_GUID@@PAVCOleException@@@Z 5f58770f f   oledisp2.obj
 0001:00086852       ?CreateDispatch@COleDispatchDriver@@QAEHPBDPAVCOleException@@@Z 5f587852 f   oledisp2.obj
 0001:000868bf       ?AttachDispatch@COleDispatchDriver@@QAEXPAUIDispatch@@H@Z 5f5878bf f   oledisp2.obj
 0001:0008690b       ?ReleaseDispatch@COleDispatchDriver@@QAEXXZ 5f58790b f   oledisp2.obj
 0001:00086940       ?DetachDispatch@COleDispatchDriver@@QAEPAUIDispatch@@XZ 5f587940 f   oledisp2.obj
 0001:00086961       ?InvokeHelperV@COleDispatchDriver@@QAEXJGGPAXPBEPAD@Z 5f587961 f   oledisp2.obj
 0001:000874a6       ?InvokeHelper@COleDispatchDriver@@QAAXJGGPAXPBEZZ 5f5884a6 f   oledisp2.obj
 0001:000874dd       ?GetProperty@COleDispatchDriver@@QBEXJGPAX@Z 5f5884dd f   oledisp2.obj
 0001:00087507       ?SetProperty@COleDispatchDriver@@QAAXJGZZ 5f588507 f   oledisp2.obj
 0001:000875a0       __AfxDispatchCall@12       5f5885a0 f   olecall.obj
 0001:000875c0       ??1COleMessageFilter@@UAE@XZ 5f5885c0 f   olemsgf.obj
 0001:00087621       ?Revoke@COleMessageFilter@@QAEXXZ 5f588621 f   olemsgf.obj
 0001:00087660       ??1COleObjectFactory@@UAE@XZ 5f588660 f   olefact.obj
 0001:00087750       ?Revoke@COleObjectFactory@@QAEXXZ 5f588750 f   olefact.obj
 0001:000877a1       ?RevokeAll@COleObjectFactory@@SGXXZ 5f5887a1 f   olefact.obj
 0001:00087fc0       ??_ECOleDataSource@@UAEPAXI@Z 5f588fc0 f i dllole.obj
 0001:00088030       ??_ECOleDispatchDriver@@QAEPAXI@Z 5f589030 f i dllole.obj
 0001:000880a0       ??_ECOleDropSource@@UAEPAXI@Z 5f5890a0 f i dllole.obj
 0001:00088110       ??1COleDropSource@@UAE@XZ  5f589110 f i dllole.obj
 0001:00088130       ??_ECOleResizeBar@@UAEPAXI@Z 5f589130 f i dllole.obj
 0001:000881a0       ??_ECOleStreamFile@@UAEPAXI@Z 5f5891a0 f i dllole.obj
 0001:00088210       ??_FCOleStreamFile@@QAEXXZ 5f589210 f i dllole.obj
 0001:00088230       ??_ECMonikerFile@@UAEPAXI@Z 5f589230 f i dllole.obj
 0001:000882a0       ??_ECOleTemplateServer@@UAEPAXI@Z 5f5892a0 f i dllole.obj
 0001:00088310       ??1COleTemplateServer@@UAE@XZ 5f589310 f i dllole.obj
 0001:00088330       ??_ECOleDataObject@@QAEPAXI@Z 5f589330 f i dllole.obj
 0001:000883a0       ??_ECOleDropTarget@@UAEPAXI@Z 5f5893a0 f i dllole.obj
 0001:00088410       ??_ECOleIPFrameWnd@@UAEPAXI@Z 5f589410 f i dllole.obj
 0001:00088480       ??_ECOleDocIPFrameWnd@@UAEPAXI@Z 5f589480 f i dllole.obj
 0001:000884f0       ??_ECAsyncMonikerFile@@UAEPAXI@Z 5f5894f0 f i dllole.obj
 0001:00088560       ??_ECCachedDataPathProperty@@UAEPAXI@Z 5f589560 f i dllole.obj
 0001:000885d0       ??_FCCachedDataPathProperty@@QAEXXZ 5f5895d0 f i dllole.obj
 0001:000885f0       ??1CCachedDataPathProperty@@UAE@XZ 5f5895f0 f i dllole.obj
 0001:00088640       ??_ECDataPathProperty@@UAEPAXI@Z 5f589640 f i dllole.obj
 0001:000886b0       ??_FCDataPathProperty@@QAEXXZ 5f5896b0 f i dllole.obj
 0001:000886d0       ??1CDataPathProperty@@UAE@XZ 5f5896d0 f i dllole.obj
 0001:00088720       ??_ECOleVariant@@QAEPAXI@Z 5f589720 f i dllole.obj
 0001:00088790       ??_ECRichEditView@@UAEPAXI@Z 5f589790 f i dllole.obj
 0001:00088800       ??1CRichEditView@@UAE@XZ   5f589800 f i dllole.obj
 0001:00088860       ??_ECRichEditCntrItem@@UAEPAXI@Z 5f589860 f i dllole.obj
 0001:000888d0       ??_FCRichEditCntrItem@@QAEXXZ 5f5898d0 f i dllole.obj
 0001:000888f0       ??1CCtrlView@@UAE@XZ       5f5898f0 f i dllole.obj
 0001:00088940       ??B?$CTypedSimpleList@PAUCRuntimeClass@@@@QAEPAUCRuntimeClass@@XZ 5f589940 f i dllole.obj
 0001:00088940       ??B?$CTypedSimpleList@PAVCOleObjectFactory@@@@QAEPAVCOleObjectFactory@@XZ 5f589940 f i dllole.obj
 0001:00088940       ?GetHead@?$CTypedSimpleList@PAVCOleObjectFactory@@@@QAEPAVCOleObjectFactory@@XZ 5f589940 f i dllole.obj
 0001:00088940       ?GetHead@?$CTypedSimpleList@PAUCRuntimeClass@@@@QAEPAUCRuntimeClass@@XZ 5f589940 f i dllole.obj
 0002:00000000       __imp__DPtoLP@12           5f58e000     gdi32:GDI32.dll
 0002:00000004       __imp__CopyMetaFileA@8     5f58e004     gdi32:GDI32.dll
 0002:00000008       __imp__CreateDCA@16        5f58e008     gdi32:GDI32.dll
 0002:0000000c       __imp__GetDeviceCaps@8     5f58e00c     gdi32:GDI32.dll
 0002:00000010       __imp__DeleteMetaFile@4    5f58e010     gdi32:GDI32.dll
 0002:00000014       __imp__DeleteDC@4          5f58e014     gdi32:GDI32.dll
 0002:00000018       __imp__ScaleWindowExtEx@24 5f58e018     gdi32:GDI32.dll
 0002:0000001c       __imp__LPtoDP@12           5f58e01c     gdi32:GDI32.dll
 0002:00000020       __imp__SetMapMode@8        5f58e020     gdi32:GDI32.dll
 0002:00000024       __imp__SelectObject@8      5f58e024     gdi32:GDI32.dll
 0002:00000028       __imp__GetPaletteEntries@16 5f58e028     gdi32:GDI32.dll
 0002:0000002c       __imp__CreatePalette@4     5f58e02c     gdi32:GDI32.dll
 0002:00000030       __imp__EnumFontFamiliesA@16 5f58e030     gdi32:GDI32.dll
 0002:00000034       \177GDI32_NULL_THUNK_DATA  5f58e034     gdi32:GDI32.dll
 0002:00000038       __imp__WideCharToMultiByte@32 5f58e038     kernel32:KERNEL32.dll
 0002:0000003c       __imp__lstrlenA@4          5f58e03c     kernel32:KERNEL32.dll
 0002:00000040       __imp__GetTickCount@0      5f58e040     kernel32:KERNEL32.dll
 0002:00000044       __imp__lstrlenW@4          5f58e044     kernel32:KERNEL32.dll
 0002:00000048       __imp__LocalAlloc@8        5f58e048     kernel32:KERNEL32.dll
 0002:0000004c       __imp__LocalFree@4         5f58e04c     kernel32:KERNEL32.dll
 0002:00000050       __imp__LoadLibraryA@4      5f58e050     kernel32:KERNEL32.dll
 0002:00000054       __imp__FreeLibrary@4       5f58e054     kernel32:KERNEL32.dll
 0002:00000058       __imp__GlobalFree@4        5f58e058     kernel32:KERNEL32.dll
 0002:0000005c       __imp__GetModuleHandleA@4  5f58e05c     kernel32:KERNEL32.dll
 0002:00000060       __imp__GlobalLock@4        5f58e060     kernel32:KERNEL32.dll
 0002:00000064       __imp__GlobalAlloc@8       5f58e064     kernel32:KERNEL32.dll
 0002:00000068       __imp__GlobalUnlock@4      5f58e068     kernel32:KERNEL32.dll
 0002:0000006c       __imp__InterlockedIncrement@4 5f58e06c     kernel32:KERNEL32.dll
 0002:00000070       __imp__lstrcmpiA@8         5f58e070     kernel32:KERNEL32.dll
 0002:00000074       __imp__InterlockedDecrement@4 5f58e074     kernel32:KERNEL32.dll
 0002:00000078       __imp__FileTimeToSystemTime@8 5f58e078     kernel32:KERNEL32.dll
 0002:0000007c       __imp__GetLastError@0      5f58e07c     kernel32:KERNEL32.dll
 0002:00000080       __imp__lstrcpynA@12        5f58e080     kernel32:KERNEL32.dll
 0002:00000084       __imp__GetProfileIntA@12   5f58e084     kernel32:KERNEL32.dll
 0002:00000088       __imp__GetCurrentThreadId@0 5f58e088     kernel32:KERNEL32.dll
 0002:0000008c       __imp__FileTimeToLocalFileTime@8 5f58e08c     kernel32:KERNEL32.dll
 0002:00000090       __imp__FormatMessageA@28   5f58e090     kernel32:KERNEL32.dll
 0002:00000094       __imp__GlobalSize@4        5f58e094     kernel32:KERNEL32.dll
 0002:00000098       __imp__lstrcmpA@8          5f58e098     kernel32:KERNEL32.dll
 0002:0000009c       __imp__MulDiv@12           5f58e09c     kernel32:KERNEL32.dll
 0002:000000a0       __imp__lstrcatA@8          5f58e0a0     kernel32:KERNEL32.dll
 0002:000000a4       __imp__CopyFileA@12        5f58e0a4     kernel32:KERNEL32.dll
 0002:000000a8       __imp__FreeResource@4      5f58e0a8     kernel32:KERNEL32.dll
 0002:000000ac       __imp__LockResource@4      5f58e0ac     kernel32:KERNEL32.dll
 0002:000000b0       __imp__GetModuleFileNameA@12 5f58e0b0     kernel32:KERNEL32.dll
 0002:000000b4       __imp__FindResourceA@12    5f58e0b4     kernel32:KERNEL32.dll
 0002:000000b8       __imp__GetThreadLocale@0   5f58e0b8     kernel32:KERNEL32.dll
 0002:000000bc       __imp__LoadResource@8      5f58e0bc     kernel32:KERNEL32.dll
 0002:000000c0       __imp__lstrcpyW@8          5f58e0c0     kernel32:KERNEL32.dll
 0002:000000c4       __imp__GetUserDefaultLCID@0 5f58e0c4     kernel32:KERNEL32.dll
 0002:000000c8       __imp__OutputDebugStringA@4 5f58e0c8     kernel32:KERNEL32.dll
 0002:000000cc       __imp__lstrcpyA@8          5f58e0cc     kernel32:KERNEL32.dll
 0002:000000d0       __imp__GetVersion@0        5f58e0d0     kernel32:KERNEL32.dll
 0002:000000d4       __imp__IsDBCSLeadByte@4    5f58e0d4     kernel32:KERNEL32.dll
 0002:000000d8       __imp__GetProcAddress@8    5f58e0d8     kernel32:KERNEL32.dll
 0002:000000dc       __imp__InterlockedExchange@8 5f58e0dc     kernel32:KERNEL32.dll
 0002:000000e0       __imp__MultiByteToWideChar@24 5f58e0e0     kernel32:KERNEL32.dll
 0002:000000e4       __imp__RaiseException@16   5f58e0e4     kernel32:KERNEL32.dll
 0002:000000e8       \177KERNEL32_NULL_THUNK_DATA 5f58e0e8     kernel32:KERNEL32.dll
 0002:000000ec       __imp_??6CDumpContext@@QAEAAV0@K@Z 5f58e0ec     MFC42D:MFC42D.DLL
 0002:000000f0       __imp_?AfxIsValidAddress@@YGHPBXIH@Z 5f58e0f0     MFC42D:MFC42D.DLL
 0002:000000f4       __imp_?AfxThrowArchiveException@@YGXHPBD@Z 5f58e0f4     MFC42D:MFC42D.DLL
 0002:000000f8       __imp_?Read@CArchive@@QAEIPAXI@Z 5f58e0f8     MFC42D:MFC42D.DLL
 0002:000000fc       __imp_?AfxThrowMemoryException@@YGXXZ 5f58e0fc     MFC42D:MFC42D.DLL
 0002:00000100       __imp_??5CArchive@@QAEAAV0@AAK@Z 5f58e100     MFC42D:MFC42D.DLL
 0002:00000104       __imp_?Write@CArchive@@QAEXPBXI@Z 5f58e104     MFC42D:MFC42D.DLL
 0002:00000108       __imp_??6CArchive@@QAEAAV0@K@Z 5f58e108     MFC42D:MFC42D.DLL
 0002:0000010c       __imp_??5CArchive@@QAEAAV0@AAG@Z 5f58e10c     MFC42D:MFC42D.DLL
 0002:00000110       __imp_??6CArchive@@QAEAAV0@G@Z 5f58e110     MFC42D:MFC42D.DLL
 0002:00000114       __imp_?IsStoring@CArchive@@QBEHXZ 5f58e114     MFC42D:MFC42D.DLL
 0002:00000118       __imp_?GetClientRect@CWnd@@QBEXPAUtagRECT@@@Z 5f58e118     MFC42D:MFC42D.DLL
 0002:0000011c       __imp_?IsEmpty@CString@@QBEHXZ 5f58e11c     MFC42D:MFC42D.DLL
 0002:00000120       __imp_?GetPathName@CDocument@@QBEABVCString@@XZ 5f58e120     MFC42D:MFC42D.DLL
 0002:00000124       __imp_?classCFrameWnd@CFrameWnd@@2UCRuntimeClass@@B 5f58e124     MFC42D:MFC42D.DLL
 0002:00000128       __imp_?GetParentFrame@CWnd@@QBEPAVCFrameWnd@@XZ 5f58e128     MFC42D:MFC42D.DLL
 0002:0000012c       __imp_?AfxGetFileTitle@@YGIPBDPADI@Z 5f58e12c     MFC42D:MFC42D.DLL
 0002:00000130       __imp_?IsPrinting@CDC@@QBEHXZ 5f58e130     MFC42D:MFC42D.DLL
 0002:00000134       __imp_?GetWindowExt@CDC@@QBE?AVCSize@@XZ 5f58e134     MFC42D:MFC42D.DLL
 0002:00000138       __imp_?GetWindowOrg@CDC@@QBE?AVCPoint@@XZ 5f58e138     MFC42D:MFC42D.DLL
 0002:0000013c       __imp_?DPtoHIMETRIC@CDC@@QBEXPAUtagSIZE@@@Z 5f58e13c     MFC42D:MFC42D.DLL
 0002:00000140       __imp_?AfxIsValidString@@YGHPBDH@Z 5f58e140     MFC42D:MFC42D.DLL
 0002:00000144       __imp_?interfaceMap@CCmdTarget@@1UAFX_INTERFACEMAP@@B 5f58e144     MFC42D:MFC42D.DLL
 0002:00000148       __imp_??6CDumpContext@@QAEAAV0@E@Z 5f58e148     MFC42D:MFC42D.DLL
 0002:0000014c       __imp_??6CDumpContext@@QAEAAV0@J@Z 5f58e14c     MFC42D:MFC42D.DLL
 0002:00000150       __imp_??BCString@@QBEPBDXZ 5f58e150     MFC42D:MFC42D.DLL
 0002:00000154       __imp_?GetTitle@CDocument@@QBEABVCString@@XZ 5f58e154     MFC42D:MFC42D.DLL
 0002:00000158       __imp_??6CDumpContext@@QAEAAV0@PBX@Z 5f58e158     MFC42D:MFC42D.DLL
 0002:0000015c       __imp_??6CDumpContext@@QAEAAV0@PBD@Z 5f58e15c     MFC42D:MFC42D.DLL
 0002:00000160       __imp_?Dump@CCmdTarget@@UBEXAAVCDumpContext@@@Z 5f58e160     MFC42D:MFC42D.DLL
 0002:00000164       __imp_?AssertValid@CCmdTarget@@UBEXXZ 5f58e164     MFC42D:MFC42D.DLL
 0002:00000168       __imp_?Serialize@CObject@@UAEXAAVCArchive@@@Z 5f58e168     MFC42D:MFC42D.DLL
 0002:0000016c       __imp_?GetRuntimeClass@CCmdTarget@@UBEPAUCRuntimeClass@@XZ 5f58e16c     MFC42D:MFC42D.DLL
 0002:00000170       __imp_??0CString@@QAE@XZ   5f58e170     MFC42D:MFC42D.DLL
 0002:00000174       __imp_??0CCmdTarget@@QAE@XZ 5f58e174     MFC42D:MFC42D.DLL
 0002:00000178       __imp_?DelayUpdateFrameTitle@CFrameWnd@@QAEXXZ 5f58e178     MFC42D:MFC42D.DLL
 0002:0000017c       __imp_?SendMessageA@CWnd@@QAEJIIJ@Z 5f58e17c     MFC42D:MFC42D.DLL
 0002:00000180       __imp_?GetSafeHmenu@CMenu@@QBEPAUHMENU__@@XZ 5f58e180     MFC42D:MFC42D.DLL
 0002:00000184       __imp_?AfxDynamicDownCast@@YAPAVCObject@@PAUCRuntimeClass@@PAV1@@Z 5f58e184     MFC42D:MFC42D.DLL
 0002:00000188       __imp_?IsWindowEnabled@CWnd@@QBEHXZ 5f58e188     MFC42D:MFC42D.DLL
 0002:0000018c       __imp_?GetSafeHwnd@CWnd@@QBEPAUHWND__@@XZ 5f58e18c     MFC42D:MFC42D.DLL
 0002:00000190       __imp_?AfxIsDescendant@@YGHPAUHWND__@@0@Z 5f58e190     MFC42D:MFC42D.DLL
 0002:00000194       __imp_?classCDocTemplate@CDocTemplate@@2UCRuntimeClass@@B 5f58e194     MFC42D:MFC42D.DLL
 0002:00000198       __imp_?AfxStaticDownCast@@YAPAVCObject@@PAUCRuntimeClass@@PAV1@@Z 5f58e198     MFC42D:MFC42D.DLL
 0002:0000019c       __imp_?GetParent@CWnd@@QBEPAV1@XZ 5f58e19c     MFC42D:MFC42D.DLL
 0002:000001a0       __imp_?classCView@CView@@2UCRuntimeClass@@B 5f58e1a0     MFC42D:MFC42D.DLL
 0002:000001a4       __imp_?GetFocus@CWnd@@SGPAV1@XZ 5f58e1a4     MFC42D:MFC42D.DLL
 0002:000001a8       __imp_?GetDocument@CView@@QBEPAVCDocument@@XZ 5f58e1a8     MFC42D:MFC42D.DLL
 0002:000001ac       __imp_?ModifyStyle@CWnd@@QAEHKKI@Z 5f58e1ac     MFC42D:MFC42D.DLL
 0002:000001b0       __imp_?GetStyle@CWnd@@QBEKXZ 5f58e1b0     MFC42D:MFC42D.DLL
 0002:000001b4       __imp_?ShowControlBar@CFrameWnd@@QAEXPAVCControlBar@@HH@Z 5f58e1b4     MFC42D:MFC42D.DLL
 0002:000001b8       __imp_?GetBarStyle@CControlBar@@QAEKXZ 5f58e1b8     MFC42D:MFC42D.DLL
 0002:000001bc       __imp_??6CDumpContext@@QAEAAV0@H@Z 5f58e1bc     MFC42D:MFC42D.DLL
 0002:000001c0       __imp_?GetNext@CPtrList@@QAEAAPAXAAPAU__POSITION@@@Z 5f58e1c0     MFC42D:MFC42D.DLL
 0002:000001c4       __imp_?GetDocTemplate@CDocument@@QBEPAVCDocTemplate@@XZ 5f58e1c4     MFC42D:MFC42D.DLL
 0002:000001c8       __imp_?GetTopLevelFrame@CWnd@@QBEPAVCFrameWnd@@XZ 5f58e1c8     MFC42D:MFC42D.DLL
 0002:000001cc       __imp_?GetParentSplitter@CView@@SGPAVCSplitterWnd@@PBVCWnd@@H@Z 5f58e1cc     MFC42D:MFC42D.DLL
 0002:000001d0       __imp_?SetFocus@CWnd@@QAEPAV1@XZ 5f58e1d0     MFC42D:MFC42D.DLL
 0002:000001d4       __imp_?GetTopLevelParent@CWnd@@QBEPAV1@XZ 5f58e1d4     MFC42D:MFC42D.DLL
 0002:000001d8       __imp_?AfxGetMainWnd@@YGPAVCWnd@@XZ 5f58e1d8     MFC42D:MFC42D.DLL
 0002:000001dc       __imp_?DelayRecalcLayout@CFrameWnd@@QAEXH@Z 5f58e1dc     MFC42D:MFC42D.DLL
 0002:000001e0       __imp_?IsRectEmpty@CRect@@QBEHXZ 5f58e1e0     MFC42D:MFC42D.DLL
 0002:000001e4       __imp_?IntersectRect@CRect@@QAEHPBUtagRECT@@0@Z 5f58e1e4     MFC42D:MFC42D.DLL
 0002:000001e8       __imp_??BCRect@@QAEPAUtagRECT@@XZ 5f58e1e8     MFC42D:MFC42D.DLL
 0002:000001ec       __imp_??BCRect@@QBEPBUtagRECT@@XZ 5f58e1ec     MFC42D:MFC42D.DLL
 0002:000001f0       __imp_??0CRect@@QAE@XZ     5f58e1f0     MFC42D:MFC42D.DLL
 0002:000001f4       __imp_?FromHandle@CWnd@@SGPAV1@PAUHWND__@@@Z 5f58e1f4     MFC42D:MFC42D.DLL
 0002:000001f8       __imp_?PostMessageA@CWnd@@QAEHIIJ@Z 5f58e1f8     MFC42D:MFC42D.DLL
 0002:000001fc       __imp_?CanEnterHelpMode@CFrameWnd@@QAEHXZ 5f58e1fc     MFC42D:MFC42D.DLL
 0002:00000200       __imp_??4CString@@QAEABV0@PBG@Z 5f58e200     MFC42D:MFC42D.DLL
 0002:00000204       __imp_?Empty@CString@@QAEXXZ 5f58e204     MFC42D:MFC42D.DLL
 0002:00000208       __imp_?FromHandle@CMenu@@SGPAV1@PAUHMENU__@@@Z 5f58e208     MFC42D:MFC42D.DLL
 0002:0000020c       __imp_??0CSize@@QAE@UtagSIZE@@@Z 5f58e20c     MFC42D:MFC42D.DLL
 0002:00000210       __imp_?CopyRect@CRect@@QAEXPBUtagRECT@@@Z 5f58e210     MFC42D:MFC42D.DLL
 0002:00000214       __imp_?GetData@CProcessLocalObject@@QAEPAVCNoTrackObject@@P6GPAV2@XZ@Z 5f58e214     MFC42D:MFC42D.DLL
 0002:00000218       __imp_??3CNoTrackObject@@SGXPAX@Z 5f58e218     MFC42D:MFC42D.DLL
 0002:0000021c       __imp_??2CNoTrackObject@@SGPAXI@Z 5f58e21c     MFC42D:MFC42D.DLL
 0002:00000220       __imp_?SetRectEmpty@CRect@@QAEXXZ 5f58e220     MFC42D:MFC42D.DLL
 0002:00000224       __imp_?SetRect@CRect@@QAEXHHHH@Z 5f58e224     MFC42D:MFC42D.DLL
 0002:00000228       __imp_??0CSize@@QAE@HH@Z   5f58e228     MFC42D:MFC42D.DLL
 0002:0000022c       __imp_?AfxIsValidString@@YGHPBGH@Z 5f58e22c     MFC42D:MFC42D.DLL
 0002:00000230       __imp_?GetBufferSetLength@CString@@QAEPADH@Z 5f58e230     MFC42D:MFC42D.DLL
 0002:00000234       __imp_?AfxA2WHelper@@YGPAGPAGPBDH@Z 5f58e234     MFC42D:MFC42D.DLL
 0002:00000238       __imp_?AfxW2AHelper@@YGPADPADPBGH@Z 5f58e238     MFC42D:MFC42D.DLL
 0002:0000023c       __imp_?SetHandle@CSharedFile@@QAEXPAXH@Z 5f58e23c     MFC42D:MFC42D.DLL
 0002:00000240       __imp_??0CSharedFile@@QAE@II@Z 5f58e240     MFC42D:MFC42D.DLL
 0002:00000244       __imp_??0CFile@@QAE@XZ     5f58e244     MFC42D:MFC42D.DLL
 0002:00000248       __imp_??2@YAPAXIPBDH@Z     5f58e248     MFC42D:MFC42D.DLL
 0002:0000024c       __imp_??1CSharedFile@@UAE@XZ 5f58e24c     MFC42D:MFC42D.DLL
 0002:00000250       __imp_?Detach@CSharedFile@@QAEPAXXZ 5f58e250     MFC42D:MFC42D.DLL
 0002:00000254       __imp_??6CDumpContext@@QAEAAV0@G@Z 5f58e254     MFC42D:MFC42D.DLL
 0002:00000258       __imp_??6CDumpContext@@QAEAAV0@I@Z 5f58e258     MFC42D:MFC42D.DLL
 0002:0000025c       __imp_?GetData@CString@@IBEPAUCStringData@@XZ 5f58e25c     MFC42D:MFC42D.DLL
 0002:00000260       __imp_?ReportError@CException@@UAEHII@Z 5f58e260     MFC42D:MFC42D.DLL
 0002:00000264       __imp_?Dump@CObject@@UBEXAAVCDumpContext@@@Z 5f58e264     MFC42D:MFC42D.DLL
 0002:00000268       __imp_?AssertValid@CObject@@UBEXXZ 5f58e268     MFC42D:MFC42D.DLL
 0002:0000026c       __imp_??1CException@@UAE@XZ 5f58e26c     MFC42D:MFC42D.DLL
 0002:00000270       __imp_??3CException@@SGXPAX@Z 5f58e270     MFC42D:MFC42D.DLL
 0002:00000274       __imp_?AfxLoadString@@YGHIPADI@Z 5f58e274     MFC42D:MFC42D.DLL
 0002:00000278       __imp_?classCMemoryException@CMemoryException@@2UCRuntimeClass@@B 5f58e278     MFC42D:MFC42D.DLL
 0002:0000027c       __imp_??4CString@@QAEABV0@PBD@Z 5f58e27c     MFC42D:MFC42D.DLL
 0002:00000280       __imp_??0CException@@QAE@XZ 5f58e280     MFC42D:MFC42D.DLL
 0002:00000284       __imp_??3CException@@SGXPAXPBDH@Z 5f58e284     MFC42D:MFC42D.DLL
 0002:00000288       __imp_?PreInitDialog@CDialog@@MAEXXZ 5f58e288     MFC42D:MFC42D.DLL
 0002:0000028c       __imp_?OnCancel@CCommonDialog@@MAEXXZ 5f58e28c     MFC42D:MFC42D.DLL
 0002:00000290       __imp_?OnOK@CCommonDialog@@MAEXXZ 5f58e290     MFC42D:MFC42D.DLL
 0002:00000294       __imp_?OnSetFont@CDialog@@UAEXPAVCFont@@@Z 5f58e294     MFC42D:MFC42D.DLL
 0002:00000298       __imp_?GetHeadPosition@CPtrList@@QBEPAU__POSITION@@XZ 5f58e298     MFC42D:MFC42D.DLL
 0002:0000029c       __imp_?OnInitDialog@CDialog@@UAEHXZ 5f58e29c     MFC42D:MFC42D.DLL
 0002:000002a0       __imp_?IsFrameWnd@CWnd@@UBEHXZ 5f58e2a0     MFC42D:MFC42D.DLL
 0002:000002a4       __imp_?CheckAutoCenter@CDialog@@UAEHXZ 5f58e2a4     MFC42D:MFC42D.DLL
 0002:000002a8       __imp_?OnChildNotify@CWnd@@MAEHIIJPAJ@Z 5f58e2a8     MFC42D:MFC42D.DLL
 0002:000002ac       __imp_?PostNcDestroy@CWnd@@MAEXXZ 5f58e2ac     MFC42D:MFC42D.DLL
 0002:000002b0       __imp_?DefWindowProcA@CWnd@@MAEJIIJ@Z 5f58e2b0     MFC42D:MFC42D.DLL
 0002:000002b4       __imp_?OnWndMsg@CWnd@@MAEHIIJPAJ@Z 5f58e2b4     MFC42D:MFC42D.DLL
 0002:000002b8       __imp_?WindowProc@CWnd@@MAEJIIJ@Z 5f58e2b8     MFC42D:MFC42D.DLL
 0002:000002bc       __imp_?OnAmbientProperty@CWnd@@UAEHPAVCOleControlSite@@JPAUtagVARIANT@@@Z 5f58e2bc     MFC42D:MFC42D.DLL
 0002:000002c0       __imp_?PreTranslateMessage@CDialog@@UAEHPAUtagMSG@@@Z 5f58e2c0     MFC42D:MFC42D.DLL
 0002:000002c4       __imp_?EndModalState@CWnd@@UAEXXZ 5f58e2c4     MFC42D:MFC42D.DLL
 0002:000002c8       __imp_?BeginModalState@CWnd@@UAEXXZ 5f58e2c8     MFC42D:MFC42D.DLL
 0002:000002cc       __imp_?DoDataExchange@CWnd@@MAEXPAVCDataExchange@@@Z 5f58e2cc     MFC42D:MFC42D.DLL
 0002:000002d0       __imp_?GetSuperWndProcAddr@CWnd@@MAEPAP6GJPAUHWND__@@IIJ@ZXZ 5f58e2d0     MFC42D:MFC42D.DLL
 0002:000002d4       __imp_?OnNotify@CWnd@@MAEHIJPAJ@Z 5f58e2d4     MFC42D:MFC42D.DLL
 0002:000002d8       __imp_?OnCommand@CWnd@@MAEHIJ@Z 5f58e2d8     MFC42D:MFC42D.DLL
 0002:000002dc       __imp_?EndModalLoop@CWnd@@UAEXH@Z 5f58e2dc     MFC42D:MFC42D.DLL
 0002:000002e0       __imp_?ContinueModal@CWnd@@UAEHXZ 5f58e2e0     MFC42D:MFC42D.DLL
 0002:000002e4       __imp_?WinHelpA@CWnd@@UAEXKI@Z 5f58e2e4     MFC42D:MFC42D.DLL
 0002:000002e8       __imp_?GetScrollBarCtrl@CWnd@@UBEPAVCScrollBar@@H@Z 5f58e2e8     MFC42D:MFC42D.DLL
 0002:000002ec       __imp_?OnToolHitTest@CWnd@@UBEHVCPoint@@PAUtagTOOLINFOA@@@Z 5f58e2ec     MFC42D:MFC42D.DLL
 0002:000002f0       __imp_?CalcWindowRect@CWnd@@UAEXPAUtagRECT@@I@Z 5f58e2f0     MFC42D:MFC42D.DLL
 0002:000002f4       __imp_?PreCreateWindow@CWnd@@UAEHAAUtagCREATESTRUCTA@@@Z 5f58e2f4     MFC42D:MFC42D.DLL
 0002:000002f8       __imp_?DestroyWindow@CWnd@@UAEHXZ 5f58e2f8     MFC42D:MFC42D.DLL
 0002:000002fc       __imp_?Create@CWnd@@UAEHPBD0KABUtagRECT@@PAV1@IPAUCCreateContext@@@Z 5f58e2fc     MFC42D:MFC42D.DLL
 0002:00000300       __imp_?PreSubclassWindow@CWnd@@UAEXXZ 5f58e300     MFC42D:MFC42D.DLL
 0002:00000304       __imp_?GetInterfaceMap@CCmdTarget@@MBEPBUAFX_INTERFACEMAP@@XZ 5f58e304     MFC42D:MFC42D.DLL
 0002:00000308       __imp_?GetMessageMap@CCommonDialog@@MBEPBUAFX_MSGMAP@@XZ 5f58e308     MFC42D:MFC42D.DLL
 0002:0000030c       __imp_?OnFinalRelease@CWnd@@UAEXXZ 5f58e30c     MFC42D:MFC42D.DLL
 0002:00000310       __imp_?OnCmdMsg@CDialog@@UAEHIHPAXPAUAFX_CMDHANDLERINFO@@@Z 5f58e310     MFC42D:MFC42D.DLL
 0002:00000314       __imp_?AssertValid@CDialog@@UBEXXZ 5f58e314     MFC42D:MFC42D.DLL
 0002:00000318       __imp_?AfxHelpEnabled@@YGHXZ 5f58e318     MFC42D:MFC42D.DLL
 0002:0000031c       __imp_?afxData@@3UAUX_DATA@@A 5f58e31c     MFC42D:MFC42D.DLL
 0002:00000320       __imp_??1CDialog@@UAE@XZ   5f58e320     MFC42D:MFC42D.DLL
 0002:00000324       __imp_?AfxMessageBox@@YGHIII@Z 5f58e324     MFC42D:MFC42D.DLL
 0002:00000328       __imp_?Format@CString@@QAAXPBDZZ 5f58e328     MFC42D:MFC42D.DLL
 0002:0000032c       __imp_?AfxStringFromCLSID@@YG?AVCString@@ABU_GUID@@@Z 5f58e32c     MFC42D:MFC42D.DLL
 0002:00000330       __imp_?PostModal@CDialog@@IAEXXZ 5f58e330     MFC42D:MFC42D.DLL
 0002:00000334       __imp_?PreModal@CDialog@@IAEPAUHWND__@@XZ 5f58e334     MFC42D:MFC42D.DLL
 0002:00000338       __imp_??1CWaitCursor@@QAE@XZ 5f58e338     MFC42D:MFC42D.DLL
 0002:0000033c       __imp_??0CWaitCursor@@QAE@XZ 5f58e33c     MFC42D:MFC42D.DLL
 0002:00000340       __imp_?LoadStringA@CString@@QAEHI@Z 5f58e340     MFC42D:MFC42D.DLL
 0002:00000344       __imp_??6@YGAAVCDumpContext@@AAV0@ABVCString@@@Z 5f58e344     MFC42D:MFC42D.DLL
 0002:00000348       __imp_?AfxThrowResourceException@@YGXXZ 5f58e348     MFC42D:MFC42D.DLL
 0002:0000034c       __imp_??0CString@@QAE@PBD@Z 5f58e34c     MFC42D:MFC42D.DLL
 0002:00000350       __imp_??0CString@@QAE@PBDH@Z 5f58e350     MFC42D:MFC42D.DLL
 0002:00000354       __imp_?AfxDlgProc@@YGHPAUHWND__@@IIJ@Z 5f58e354     MFC42D:MFC42D.DLL
 0002:00000358       __imp_?DoModal@CDialog@@UAEHXZ 5f58e358     MFC42D:MFC42D.DLL
 0002:0000035c       __imp_??0CCommonDialog@@QAE@PAVCWnd@@@Z 5f58e35c     MFC42D:MFC42D.DLL
 0002:00000360       __imp_?Dump@CDialog@@UBEXAAVCDumpContext@@@Z 5f58e360     MFC42D:MFC42D.DLL
 0002:00000364       __imp_?Detach@CWnd@@QAEPAUHWND__@@XZ 5f58e364     MFC42D:MFC42D.DLL
 0002:00000368       __imp_?AfxUnhookWindowCreate@@YGHXZ 5f58e368     MFC42D:MFC42D.DLL
 0002:0000036c       __imp_?AfxHookWindowCreate@@YGXPAVCWnd@@@Z 5f58e36c     MFC42D:MFC42D.DLL
 0002:00000370       __imp_?GetSafeOwner_@CWnd@@SGPAUHWND__@@PAU2@PAPAU2@@Z 5f58e370     MFC42D:MFC42D.DLL
 0002:00000374       __imp_?classCDialog@CDialog@@2UCRuntimeClass@@B 5f58e374     MFC42D:MFC42D.DLL
 0002:00000378       __imp_?CenterWindow@CWnd@@QAEXPAV1@@Z 5f58e378     MFC42D:MFC42D.DLL
 0002:0000037c       __imp_??4CString@@QAEABV0@ABV0@@Z 5f58e37c     MFC42D:MFC42D.DLL
 0002:00000380       __imp_??0CString@@QAE@ABV0@@Z 5f58e380     MFC42D:MFC42D.DLL
 0002:00000384       __imp_??1CProcessLocalObject@@QAE@XZ 5f58e384     MFC42D:MFC42D.DLL
 0002:00000388       __imp_?GetData@CByteArray@@QBEPBEXZ 5f58e388     MFC42D:MFC42D.DLL
 0002:0000038c       __imp_?GetSize@CByteArray@@QBEHXZ 5f58e38c     MFC42D:MFC42D.DLL
 0002:00000390       __imp_??6CDumpContext@@QAEAAV0@N@Z 5f58e390     MFC42D:MFC42D.DLL
 0002:00000394       __imp_??6CDumpContext@@QAEAAV0@M@Z 5f58e394     MFC42D:MFC42D.DLL
 0002:00000398       __imp_??6CDumpContext@@QAEAAV0@PBG@Z 5f58e398     MFC42D:MFC42D.DLL
 0002:0000039c       __imp_??0CArchiveStream@@QAE@PAVCArchive@@@Z 5f58e39c     MFC42D:MFC42D.DLL
 0002:000003a0       __imp_??6CArchive@@QAEAAV0@N@Z 5f58e3a0     MFC42D:MFC42D.DLL
 0002:000003a4       __imp_??6CArchive@@QAEAAV0@M@Z 5f58e3a4     MFC42D:MFC42D.DLL
 0002:000003a8       __imp_??6CArchive@@QAEAAV0@J@Z 5f58e3a8     MFC42D:MFC42D.DLL
 0002:000003ac       __imp_??6CArchive@@QAEAAV0@E@Z 5f58e3ac     MFC42D:MFC42D.DLL
 0002:000003b0       __imp_??5CArchive@@QAEAAV0@AAN@Z 5f58e3b0     MFC42D:MFC42D.DLL
 0002:000003b4       __imp_??5CArchive@@QAEAAV0@AAM@Z 5f58e3b4     MFC42D:MFC42D.DLL
 0002:000003b8       __imp_??5CArchive@@QAEAAV0@AAJ@Z 5f58e3b8     MFC42D:MFC42D.DLL
 0002:000003bc       __imp_??5CArchive@@QAEAAV0@AAE@Z 5f58e3bc     MFC42D:MFC42D.DLL
 0002:000003c0       __imp_?HashKey@@YGIPBG@Z   5f58e3c0     MFC42D:MFC42D.DLL
 0002:000003c4       __imp_?ReleaseBuffer@CString@@QAEXH@Z 5f58e3c4     MFC42D:MFC42D.DLL
 0002:000003c8       __imp_?GetLength@CString@@QBEHXZ 5f58e3c8     MFC42D:MFC42D.DLL
 0002:000003cc       __imp_??YCString@@QAEABV0@PBD@Z 5f58e3cc     MFC42D:MFC42D.DLL
 0002:000003d0       __imp_?GetBuffer@CString@@QAEPADH@Z 5f58e3d0     MFC42D:MFC42D.DLL
 0002:000003d4       __imp_?GetDepth@CDumpContext@@QBEHXZ 5f58e3d4     MFC42D:MFC42D.DLL
 0002:000003d8       __imp_?AfxSetWindowText@@YGXPAUHWND__@@PBD@Z 5f58e3d8     MFC42D:MFC42D.DLL
 0002:000003dc       __imp_?Fail@CDataExchange@@QAEXXZ 5f58e3dc     MFC42D:MFC42D.DLL
 0002:000003e0       __imp_?PrepareEditCtrl@CDataExchange@@QAEPAUHWND__@@H@Z 5f58e3e0     MFC42D:MFC42D.DLL
 0002:000003e4       __imp_?GetDefaultAccelerator@CDocument@@UAEPAUHACCEL__@@XZ 5f58e3e4     MFC42D:MFC42D.DLL
 0002:000003e8       __imp_?GetDefaultMenu@CDocument@@UAEPAUHMENU__@@XZ 5f58e3e8     MFC42D:MFC42D.DLL
 0002:000003ec       __imp_?UpdateFrameCounts@CDocument@@UAEXXZ 5f58e3ec     MFC42D:MFC42D.DLL
 0002:000003f0       __imp_?DoFileSave@CDocument@@UAEHXZ 5f58e3f0     MFC42D:MFC42D.DLL
 0002:000003f4       __imp_?DoSave@CDocument@@UAEHPBDH@Z 5f58e3f4     MFC42D:MFC42D.DLL
 0002:000003f8       __imp_?CanCloseFrame@CDocument@@UAEHPAVCFrameWnd@@@Z 5f58e3f8     MFC42D:MFC42D.DLL
 0002:000003fc       __imp_?ReleaseFile@CDocument@@UAEXPAVCFile@@H@Z 5f58e3fc     MFC42D:MFC42D.DLL
 0002:00000400       __imp_?GetFile@CDocument@@UAEPAVCFile@@PBDIPAVCFileException@@@Z 5f58e400     MFC42D:MFC42D.DLL
 0002:00000404       __imp_?ReportSaveLoadException@CDocument@@UAEXPBDPAVCException@@HI@Z 5f58e404     MFC42D:MFC42D.DLL
 0002:00000408       __imp_?OnChangedViewList@CDocument@@UAEXXZ 5f58e408     MFC42D:MFC42D.DLL
 0002:0000040c       __imp_?GetNextView@CDocument@@UBEPAVCView@@AAPAU__POSITION@@@Z 5f58e40c     MFC42D:MFC42D.DLL
 0002:00000410       __imp_?GetFirstViewPosition@CDocument@@UBEPAU__POSITION@@XZ 5f58e410     MFC42D:MFC42D.DLL
 0002:00000414       __imp_?SetModifiedFlag@CDocument@@UAEXH@Z 5f58e414     MFC42D:MFC42D.DLL
 0002:00000418       __imp_?IsModified@CDocument@@UAEHXZ 5f58e418     MFC42D:MFC42D.DLL
 0002:0000041c       __imp_?SetTitle@CDocument@@UAEXPBD@Z 5f58e41c     MFC42D:MFC42D.DLL
 0002:00000420       __imp_?GetMessageMap@CDocument@@MBEPBUAFX_MSGMAP@@XZ 5f58e420     MFC42D:MFC42D.DLL
 0002:00000424       __imp_?OnFinalRelease@CDocument@@UAEXXZ 5f58e424     MFC42D:MFC42D.DLL
 0002:00000428       __imp_??1CObList@@UAE@XZ   5f58e428     MFC42D:MFC42D.DLL
 0002:0000042c       __imp_??1CDocument@@UAE@XZ 5f58e42c     MFC42D:MFC42D.DLL
 0002:00000430       __imp_?IsEmpty@CObList@@QBEHXZ 5f58e430     MFC42D:MFC42D.DLL
 0002:00000434       __imp_?IsEmpty@CPtrList@@QBEHXZ 5f58e434     MFC42D:MFC42D.DLL
 0002:00000438       __imp_??0CObList@@QAE@H@Z  5f58e438     MFC42D:MFC42D.DLL
 0002:0000043c       __imp_??0CDocument@@QAE@XZ 5f58e43c     MFC42D:MFC42D.DLL
 0002:00000440       __imp_?GetCount@CObList@@QBEHXZ 5f58e440     MFC42D:MFC42D.DLL
 0002:00000444       __imp_?AddTail@CObList@@QAEPAU__POSITION@@PAVCObject@@@Z 5f58e444     MFC42D:MFC42D.DLL
 0002:00000448       __imp_?RemoveAt@CObList@@QAEXPAU__POSITION@@@Z 5f58e448     MFC42D:MFC42D.DLL
 0002:0000044c       __imp_?SetOccDialogInfo@CDialog@@MAEHPAU_AFX_OCC_DIALOG_INFO@@@Z 5f58e44c     MFC42D:MFC42D.DLL
 0002:00000450       __imp_?GetHeadPosition@CObList@@QBEPAU__POSITION@@XZ 5f58e450     MFC42D:MFC42D.DLL
 0002:00000454       __imp_?GetNext@CObList@@QBEPAVCObject@@AAPAU__POSITION@@@Z 5f58e454     MFC42D:MFC42D.DLL
 0002:00000458       __imp_?Find@CObList@@QBEPAU__POSITION@@PAVCObject@@PAU2@@Z 5f58e458     MFC42D:MFC42D.DLL
 0002:0000045c       __imp_??6@YGAAVCArchive@@AAV0@PBVCObject@@@Z 5f58e45c     MFC42D:MFC42D.DLL
 0002:00000460       __imp_?SaveModified@CDocument@@UAEHXZ 5f58e460     MFC42D:MFC42D.DLL
 0002:00000464       __imp_?AfxMessageBox@@YGHPBDII@Z 5f58e464     MFC42D:MFC42D.DLL
 0002:00000468       __imp_?AfxFormatString1@@YGXAAVCString@@IPBD@Z 5f58e468     MFC42D:MFC42D.DLL
 0002:0000046c       __imp_?OnNewDocument@CDocument@@UAEHXZ 5f58e46c     MFC42D:MFC42D.DLL
 0002:00000470       __imp_?OnOpenDocument@CDocument@@UAEHPBD@Z 5f58e470     MFC42D:MFC42D.DLL
 0002:00000474       __imp_?AfxComparePath@@YGHPBD0@Z 5f58e474     MFC42D:MFC42D.DLL
 0002:00000478       __imp_?OnSaveDocument@CDocument@@UAEHPBD@Z 5f58e478     MFC42D:MFC42D.DLL
 0002:0000047c       __imp_?OnCloseDocument@CDocument@@UAEXXZ 5f58e47c     MFC42D:MFC42D.DLL
 0002:00000480       __imp_??1CFileException@@UAE@XZ 5f58e480     MFC42D:MFC42D.DLL
 0002:00000484       __imp_??1CArchive@@QAE@XZ  5f58e484     MFC42D:MFC42D.DLL
 0002:00000488       __imp_?Close@CArchive@@QAEXXZ 5f58e488     MFC42D:MFC42D.DLL
 0002:0000048c       __imp_??0CArchive@@QAE@PAVCFile@@IHPAX@Z 5f58e48c     MFC42D:MFC42D.DLL
 0002:00000490       __imp_?AfxThrowFileException@@YGXHJPBD@Z 5f58e490     MFC42D:MFC42D.DLL
 0002:00000494       __imp_??0CFileException@@QAE@HJPBD@Z 5f58e494     MFC42D:MFC42D.DLL
 0002:00000498       __imp_?AssertValid@CDocument@@UBEXXZ 5f58e498     MFC42D:MFC42D.DLL
 0002:0000049c       __imp_?Dump@CDocument@@UBEXAAVCDumpContext@@@Z 5f58e49c     MFC42D:MFC42D.DLL
 0002:000004a0       __imp_?classCCmdTarget@CCmdTarget@@2UCRuntimeClass@@B 5f58e4a0     MFC42D:MFC42D.DLL
 0002:000004a4       __imp_?AfxClassInit@@YGXPAUCRuntimeClass@@@Z 5f58e4a4     MFC42D:MFC42D.DLL
 0002:000004a8       __imp_?ReadObject@CArchive@@QAEPAVCObject@@PBUCRuntimeClass@@@Z 5f58e4a8     MFC42D:MFC42D.DLL
 0002:000004ac       __imp_?classCDocument@CDocument@@2UCRuntimeClass@@B 5f58e4ac     MFC42D:MFC42D.DLL
 0002:000004b0       __imp_?AfxUnlockGlobals@@YGXH@Z 5f58e4b0     MFC42D:MFC42D.DLL
 0002:000004b4       __imp_?AfxLockGlobals@@YGXH@Z 5f58e4b4     MFC42D:MFC42D.DLL
 0002:000004b8       __imp_?PtInRect@CRect@@QBEHUtagPOINT@@@Z 5f58e4b8     MFC42D:MFC42D.DLL
 0002:000004bc       __imp_?GetCapture@CWnd@@SGPAV1@XZ 5f58e4bc     MFC42D:MFC42D.DLL
 0002:000004c0       __imp_?SetCapture@CWnd@@QAEPAV1@XZ 5f58e4c0     MFC42D:MFC42D.DLL
 0002:000004c4       __imp_?InflateRect@CRect@@QAEXHH@Z 5f58e4c4     MFC42D:MFC42D.DLL
 0002:000004c8       __imp_?IsRectNull@CRect@@QBEHXZ 5f58e4c8     MFC42D:MFC42D.DLL
 0002:000004cc       __imp_??0CPoint@@QAE@XZ    5f58e4cc     MFC42D:MFC42D.DLL
 0002:000004d0       __imp_?ScreenToClient@CWnd@@QBEXPAUtagPOINT@@@Z 5f58e4d0     MFC42D:MFC42D.DLL
 0002:000004d4       __imp_??0CPoint@@QAE@HH@Z  5f58e4d4     MFC42D:MFC42D.DLL
 0002:000004d8       __imp_?IsDerivedFrom@CRuntimeClass@@QBEHPBU1@@Z 5f58e4d8     MFC42D:MFC42D.DLL
 0002:000004dc       __imp_?CreateObject@CRuntimeClass@@QAEPAVCObject@@XZ 5f58e4dc     MFC42D:MFC42D.DLL
 0002:000004e0       __imp_?AddHead@CSimpleList@@QAEXPAX@Z 5f58e4e0     MFC42D:MFC42D.DLL
 0002:000004e4       __imp_?Remove@CSimpleList@@QAEHPAX@Z 5f58e4e4     MFC42D:MFC42D.DLL
 0002:000004e8       __imp_?ExitHelpMode@CFrameWnd@@UAEXXZ 5f58e4e8     MFC42D:MFC42D.DLL
 0002:000004ec       __imp_?DelayUpdateFrameMenu@CFrameWnd@@UAEXPAUHMENU__@@@Z 5f58e4ec     MFC42D:MFC42D.DLL
 0002:000004f0       __imp_?GetDefaultAccelerator@CFrameWnd@@UAEPAUHACCEL__@@XZ 5f58e4f0     MFC42D:MFC42D.DLL
 0002:000004f4       __imp_?OnUpdateFrameMenu@CFrameWnd@@UAEXPAUHMENU__@@@Z 5f58e4f4     MFC42D:MFC42D.DLL
 0002:000004f8       __imp_?OnUpdateFrameTitle@CFrameWnd@@UAEXH@Z 5f58e4f8     MFC42D:MFC42D.DLL
 0002:000004fc       __imp_?OnCreateClient@CFrameWnd@@MAEHPAUtagCREATESTRUCTA@@PAUCCreateContext@@@Z 5f58e4fc     MFC42D:MFC42D.DLL
 0002:00000500       __imp_?NegotiateBorderSpace@CFrameWnd@@UAEHIPAUtagRECT@@@Z 5f58e500     MFC42D:MFC42D.DLL
 0002:00000504       __imp_?GetMessageBar@CFrameWnd@@UAEPAVCWnd@@XZ 5f58e504     MFC42D:MFC42D.DLL
 0002:00000508       __imp_?OnSetPreviewMode@CFrameWnd@@UAEXHPAUCPrintPreviewState@@@Z 5f58e508     MFC42D:MFC42D.DLL
 0002:0000050c       __imp_?ActivateFrame@CFrameWnd@@UAEXH@Z 5f58e50c     MFC42D:MFC42D.DLL
 0002:00000510       __imp_?GetMessageString@CFrameWnd@@UBEXIAAVCString@@@Z 5f58e510     MFC42D:MFC42D.DLL
 0002:00000514       __imp_?GetActiveFrame@CFrameWnd@@UAEPAV1@XZ 5f58e514     MFC42D:MFC42D.DLL
 0002:00000518       __imp_?GetActiveDocument@CFrameWnd@@UAEPAVCDocument@@XZ 5f58e518     MFC42D:MFC42D.DLL
 0002:0000051c       __imp_?LoadFrame@CFrameWnd@@UAEHIKPAVCWnd@@PAUCCreateContext@@@Z 5f58e51c     MFC42D:MFC42D.DLL
 0002:00000520       __imp_?SetOccDialogInfo@CWnd@@MAEHPAU_AFX_OCC_DIALOG_INFO@@@Z 5f58e520     MFC42D:MFC42D.DLL
 0002:00000524       __imp_?IsFrameWnd@CFrameWnd@@UBEHXZ 5f58e524     MFC42D:MFC42D.DLL
 0002:00000528       __imp_?CheckAutoCenter@CWnd@@UAEHXZ 5f58e528     MFC42D:MFC42D.DLL
 0002:0000052c       __imp_?PreTranslateMessage@CFrameWnd@@UAEHPAUtagMSG@@@Z 5f58e52c     MFC42D:MFC42D.DLL
 0002:00000530       __imp_?EndModalState@CFrameWnd@@UAEXXZ 5f58e530     MFC42D:MFC42D.DLL
 0002:00000534       __imp_?BeginModalState@CFrameWnd@@UAEXXZ 5f58e534     MFC42D:MFC42D.DLL
 0002:00000538       __imp_?OnCommand@CFrameWnd@@MAEHIJ@Z 5f58e538     MFC42D:MFC42D.DLL
 0002:0000053c       __imp_?PreCreateWindow@CFrameWnd@@MAEHAAUtagCREATESTRUCTA@@@Z 5f58e53c     MFC42D:MFC42D.DLL
 0002:00000540       __imp_?GetMessageMap@CFrameWnd@@MBEPBUAFX_MSGMAP@@XZ 5f58e540     MFC42D:MFC42D.DLL
 0002:00000544       __imp_?Dump@CFrameWnd@@UBEXAAVCDumpContext@@@Z 5f58e544     MFC42D:MFC42D.DLL
 0002:00000548       __imp_?GetRuntimeClass@CFrameWnd@@UBEPAUCRuntimeClass@@XZ 5f58e548     MFC42D:MFC42D.DLL
 0002:0000054c       __imp_??1CFrameWnd@@UAE@XZ 5f58e54c     MFC42D:MFC42D.DLL
 0002:00000550       __imp_?RemoveFrameWnd@CFrameWnd@@IAEXXZ 5f58e550     MFC42D:MFC42D.DLL
 0002:00000554       __imp_??0CFrameWnd@@QAE@XZ 5f58e554     MFC42D:MFC42D.DLL
 0002:00000558       __imp_?AddFrameWnd@CFrameWnd@@IAEXXZ 5f58e558     MFC42D:MFC42D.DLL
 0002:0000055c       __imp_?AfxCallWndProc@@YGJPAVCWnd@@PAUHWND__@@IIJ@Z 5f58e55c     MFC42D:MFC42D.DLL
 0002:00000560       __imp_?messageMap@CFrameWnd@@1UAFX_MSGMAP@@B 5f58e560     MFC42D:MFC42D.DLL
 0002:00000564       __imp_?PostNcDestroy@CFrameWnd@@MAEXXZ 5f58e564     MFC42D:MFC42D.DLL
 0002:00000568       __imp_?OnCmdMsg@CFrameWnd@@UAEHIHPAXPAUAFX_CMDHANDLERINFO@@@Z 5f58e568     MFC42D:MFC42D.DLL
 0002:0000056c       __imp_?ModifyStyleEx@CWnd@@QAEHKKI@Z 5f58e56c     MFC42D:MFC42D.DLL
 0002:00000570       __imp_?OnCreate@CFrameWnd@@IAEHPAUtagCREATESTRUCTA@@@Z 5f58e570     MFC42D:MFC42D.DLL
 0002:00000574       __imp_?OnDestroy@CFrameWnd@@IAEXXZ 5f58e574     MFC42D:MFC42D.DLL
 0002:00000578       __imp_?DestroyDockBars@CFrameWnd@@QAEXXZ 5f58e578     MFC42D:MFC42D.DLL
 0002:0000057c       __imp_?DisconnectViews@CDocument@@QAEXXZ 5f58e57c     MFC42D:MFC42D.DLL
 0002:00000580       __imp_?OnWindowPosChanging@CWnd@@IAEXPAUtagWINDOWPOS@@@Z 5f58e580     MFC42D:MFC42D.DLL
 0002:00000584       __imp_?LoadAccelTable@CFrameWnd@@QAEHPBD@Z 5f58e584     MFC42D:MFC42D.DLL
 0002:00000588       __imp_??0CRect@@QAE@HHHH@Z 5f58e588     MFC42D:MFC42D.DLL
 0002:0000058c       __imp_?GetDlgItem@CWnd@@QBEPAV1@H@Z 5f58e58c     MFC42D:MFC42D.DLL
 0002:00000590       __imp_?ScreenToClient@CWnd@@QBEXPAUtagRECT@@@Z 5f58e590     MFC42D:MFC42D.DLL
 0002:00000594       __imp_?ClientToScreen@CWnd@@QBEXPAUtagRECT@@@Z 5f58e594     MFC42D:MFC42D.DLL
 0002:00000598       __imp_?AfxRepositionWindow@@YGXPAUAFX_SIZEPARENTPARAMS@@PAUHWND__@@PBUtagRECT@@@Z 5f58e598     MFC42D:MFC42D.DLL
 0002:0000059c       __imp_?RepositionBars@CWnd@@QAEXIIIIPAUtagRECT@@PBU2@H@Z 5f58e59c     MFC42D:MFC42D.DLL
 0002:000005a0       __imp_?ContinueRouting@CCmdUI@@QAEXXZ 5f58e5a0     MFC42D:MFC42D.DLL
 0002:000005a4       __imp_?OnUpdateControlBarMenu@CFrameWnd@@QAEXPAVCCmdUI@@@Z 5f58e5a4     MFC42D:MFC42D.DLL
 0002:000005a8       __imp_?GetControlBar@CFrameWnd@@QAEPAVCControlBar@@I@Z 5f58e5a8     MFC42D:MFC42D.DLL
 0002:000005ac       __imp_?OnBarCheck@CFrameWnd@@QAEHI@Z 5f58e5ac     MFC42D:MFC42D.DLL
 0002:000005b0       __imp_?OnContextHelp@CFrameWnd@@QAEXXZ 5f58e5b0     MFC42D:MFC42D.DLL
 0002:000005b4       __imp_?AssertValid@CFrameWnd@@UBEXXZ 5f58e5b4     MFC42D:MFC42D.DLL
 0002:000005b8       __imp_??6@YGAAVCDumpContext@@AAV0@ABUtagRECT@@@Z 5f58e5b8     MFC42D:MFC42D.DLL
 0002:000005bc       __imp_??9@YG_NABVCString@@PBD@Z 5f58e5bc     MFC42D:MFC42D.DLL
 0002:000005c0       __imp_?afxTraceFlags@@3IA  5f58e5c0     MFC42D:MFC42D.DLL
 0002:000005c4       __imp_?SendInitialUpdate@CDocument@@QAEXXZ 5f58e5c4     MFC42D:MFC42D.DLL
 0002:000005c8       __imp_?AfxOleGetUserCtrl@@YGHXZ 5f58e5c8     MFC42D:MFC42D.DLL
 0002:000005cc       __imp_??6CDumpContext@@QAEAAV0@PBVCObject@@@Z 5f58e5cc     MFC42D:MFC42D.DLL
 0002:000005d0       __imp_?classCNotSupportedException@CNotSupportedException@@2UCRuntimeClass@@B 5f58e5d0     MFC42D:MFC42D.DLL
 0002:000005d4       __imp_??YCString@@QAEABV0@D@Z 5f58e5d4     MFC42D:MFC42D.DLL
 0002:000005d8       __imp_?GetBufferPtr@CFile@@UAEIIIPAPAX0@Z 5f58e5d8     MFC42D:MFC42D.DLL
 0002:000005dc       __imp_?Open@CFile@@UAEHPBDIPAVCFileException@@@Z 5f58e5dc     MFC42D:MFC42D.DLL
 0002:000005e0       __imp_?SetFilePath@CFile@@UAEXPBD@Z 5f58e5e0     MFC42D:MFC42D.DLL
 0002:000005e4       __imp_?GetFilePath@CFile@@UBE?AVCString@@XZ 5f58e5e4     MFC42D:MFC42D.DLL
 0002:000005e8       __imp_?GetFileTitle@CFile@@UBE?AVCString@@XZ 5f58e5e8     MFC42D:MFC42D.DLL
 0002:000005ec       __imp_?GetFileName@CFile@@UBE?AVCString@@XZ 5f58e5ec     MFC42D:MFC42D.DLL
 0002:000005f0       __imp_??1CFile@@UAE@XZ     5f58e5f0     MFC42D:MFC42D.DLL
 0002:000005f4       __imp_?AfxFullPath@@YGHPADPBD@Z 5f58e5f4     MFC42D:MFC42D.DLL
 0002:000005f8       __imp_?OsErrorToException@CFileException@@SGHJ@Z 5f58e5f8     MFC42D:MFC42D.DLL
 0002:000005fc       __imp_??4CTime@@QAEABV0@ABV0@@Z 5f58e5fc     MFC42D:MFC42D.DLL
 0002:00000600       __imp_??0CTime@@QAE@ABU_FILETIME@@H@Z 5f58e600     MFC42D:MFC42D.DLL
 0002:00000604       __imp_?AssertValid@CFile@@UBEXXZ 5f58e604     MFC42D:MFC42D.DLL
 0002:00000608       __imp_?Dump@CFile@@UBEXAAVCDumpContext@@@Z 5f58e608     MFC42D:MFC42D.DLL
 0002:0000060c       __imp_?classCFile@CFile@@2UCRuntimeClass@@B 5f58e60c     MFC42D:MFC42D.DLL
 0002:00000610       __imp_??9CSize@@QBEHUtagSIZE@@@Z 5f58e610     MFC42D:MFC42D.DLL
 0002:00000614       __imp_?HIMETRICtoDP@CDC@@QBEXPAUtagSIZE@@@Z 5f58e614     MFC42D:MFC42D.DLL
 0002:00000618       __imp_?Size@CRect@@QBE?AVCSize@@XZ 5f58e618     MFC42D:MFC42D.DLL
 0002:0000061c       __imp_??0CSize@@QAE@XZ     5f58e61c     MFC42D:MFC42D.DLL
 0002:00000620       __imp_?IsWindowVisible@CWnd@@QBEHXZ 5f58e620     MFC42D:MFC42D.DLL
 0002:00000624       __imp_?AfxFormatString2@@YGXAAVCString@@IPBD1@Z 5f58e624     MFC42D:MFC42D.DLL
 0002:00000628       __imp_?messageMap@CDocument@@1UAFX_MSGMAP@@B 5f58e628     MFC42D:MFC42D.DLL
 0002:0000062c       __imp_?HideApplication@CWinApp@@QAEXXZ 5f58e62c     MFC42D:MFC42D.DLL
 0002:00000630       __imp_?SetActiveWindow@CWnd@@QAEPAV1@XZ 5f58e630     MFC42D:MFC42D.DLL
 0002:00000634       __imp_?ShowWindow@CWnd@@QAEHH@Z 5f58e634     MFC42D:MFC42D.DLL
 0002:00000638       __imp_?SetForegroundWindow@CWnd@@QAEHXZ 5f58e638     MFC42D:MFC42D.DLL
 0002:0000063c       __imp_?GetLastActivePopup@CWnd@@QBEPAV1@XZ 5f58e63c     MFC42D:MFC42D.DLL
 0002:00000640       __imp_?UpdateWindow@CWnd@@QAEXXZ 5f58e640     MFC42D:MFC42D.DLL
 0002:00000644       __imp_?ShowOwnedWindows@CFrameWnd@@QAEXH@Z 5f58e644     MFC42D:MFC42D.DLL
 0002:00000648       __imp_?Attach@CWnd@@QAEHPAUHWND__@@@Z 5f58e648     MFC42D:MFC42D.DLL
 0002:0000064c       __imp_?CreateOleFrame@CDocTemplate@@QAEPAVCFrameWnd@@PAVCWnd@@PAVCDocument@@H@Z 5f58e64c     MFC42D:MFC42D.DLL
 0002:00000650       __imp_?GetExStyle@CWnd@@QBEKXZ 5f58e650     MFC42D:MFC42D.DLL
 0002:00000654       __imp_?GetDescendantWindow@CWnd@@QBEPAV1@HH@Z 5f58e654     MFC42D:MFC42D.DLL
 0002:00000658       __imp_?SetActiveView@CFrameWnd@@QAEXPAVCView@@H@Z 5f58e658     MFC42D:MFC42D.DLL
 0002:0000065c       __imp_?SetParent@CWnd@@QAEPAV1@PAV1@@Z 5f58e65c     MFC42D:MFC42D.DLL
 0002:00000660       __imp_?GetActiveView@CFrameWnd@@QBEPAVCView@@XZ 5f58e660     MFC42D:MFC42D.DLL
 0002:00000664       __imp_?IsFloating@CControlBar@@QBEHXZ 5f58e664     MFC42D:MFC42D.DLL
 0002:00000668       __imp_?EnableWindow@CWnd@@QAEHH@Z 5f58e668     MFC42D:MFC42D.DLL
 0002:0000066c       __imp_?InModalState@CFrameWnd@@QBEHXZ 5f58e66c     MFC42D:MFC42D.DLL
 0002:00000670       __imp_?Close@CMetaFileDC@@QAEPAUHMETAFILE__@@XZ 5f58e670     MFC42D:MFC42D.DLL
 0002:00000674       __imp_?SetAttribDC@CMetaFileDC@@UAEXPAUHDC__@@@Z 5f58e674     MFC42D:MFC42D.DLL
 0002:00000678       __imp_??1CMetaFileDC@@UAE@XZ 5f58e678     MFC42D:MFC42D.DLL
 0002:0000067c       __imp_?Create@CMetaFileDC@@QAEHPBD@Z 5f58e67c     MFC42D:MFC42D.DLL
 0002:00000680       __imp_??0CMetaFileDC@@QAE@XZ 5f58e680     MFC42D:MFC42D.DLL
 0002:00000684       __imp_?Left@CString@@QBE?AV1@H@Z 5f58e684     MFC42D:MFC42D.DLL
 0002:00000688       __imp_?Mid@CString@@QBE?AV1@H@Z 5f58e688     MFC42D:MFC42D.DLL
 0002:0000068c       __imp_?Find@CString@@QBEHD@Z 5f58e68c     MFC42D:MFC42D.DLL
 0002:00000690       __imp_?AfxGetModuleShortFileName@@YGXPAUHINSTANCE__@@AAVCString@@@Z 5f58e690     MFC42D:MFC42D.DLL
 0002:00000694       __imp_?AfxGetInstanceHandle@@YGPAUHINSTANCE__@@XZ 5f58e694     MFC42D:MFC42D.DLL
 0002:00000698       __imp_?_AfxDeleteRegKey@@YGHPBD@Z 5f58e698     MFC42D:MFC42D.DLL
 0002:0000069c       __imp_?AfxFormatStrings@@YGXAAVCString@@PBDPBQBDH@Z 5f58e69c     MFC42D:MFC42D.DLL
 0002:000006a0       __imp_?GetNextDocTemplate@CWinApp@@QBEPAVCDocTemplate@@AAPAU__POSITION@@@Z 5f58e6a0     MFC42D:MFC42D.DLL
 0002:000006a4       __imp_?GetFirstDocTemplatePosition@CWinApp@@QBEPAU__POSITION@@XZ 5f58e6a4     MFC42D:MFC42D.DLL
 0002:000006a8       __imp_?OnCmdMsg@CDocument@@UAEHIHPAXPAUAFX_CMDHANDLERINFO@@@Z 5f58e6a8     MFC42D:MFC42D.DLL
 0002:000006ac       __imp_?GetRoutingView_@CCmdTarget@@KGPAVCView@@XZ 5f58e6ac     MFC42D:MFC42D.DLL
 0002:000006b0       __imp_?InsertMenuA@CMenu@@QAEHIIIPBD@Z 5f58e6b0     MFC42D:MFC42D.DLL
 0002:000006b4       __imp_?DeleteMenu@CMenu@@QAEHII@Z 5f58e6b4     MFC42D:MFC42D.DLL
 0002:000006b8       __imp_?GetMenuStringA@CMenu@@QBEHIPADHI@Z 5f58e6b8     MFC42D:MFC42D.DLL
 0002:000006bc       __imp_?AfxFindMessageEntry@@YGPBUAFX_MSGMAP_ENTRY@@PBU1@III@Z 5f58e6bc     MFC42D:MFC42D.DLL
 0002:000006c0       __imp_?OnSize@CWnd@@IAEXIHH@Z 5f58e6c0     MFC42D:MFC42D.DLL
 0002:000006c4       __imp_?messageMap@CCtrlView@@1UAFX_MSGMAP@@B 5f58e6c4     MFC42D:MFC42D.DLL
 0002:000006c8       __imp_?OnEndPrintPreview@CView@@MAEXPAVCDC@@PAUCPrintInfo@@UtagPOINT@@PAVCPreviewView@@@Z 5f58e6c8     MFC42D:MFC42D.DLL
 0002:000006cc       __imp_?OnPreparePrinting@CView@@MAEHPAUCPrintInfo@@@Z 5f58e6cc     MFC42D:MFC42D.DLL
 0002:000006d0       __imp_?OnDraw@CCtrlView@@MAEXPAVCDC@@@Z 5f58e6d0     MFC42D:MFC42D.DLL
 0002:000006d4       __imp_?OnUpdate@CView@@MAEXPAV1@JPAVCObject@@@Z 5f58e6d4     MFC42D:MFC42D.DLL
 0002:000006d8       __imp_?OnActivateFrame@CView@@MAEXIPAVCFrameWnd@@@Z 5f58e6d8     MFC42D:MFC42D.DLL
 0002:000006dc       __imp_?OnActivateView@CView@@MAEXHPAV1@0@Z 5f58e6dc     MFC42D:MFC42D.DLL
 0002:000006e0       __imp_?OnDragScroll@CView@@UAEKKVCPoint@@@Z 5f58e6e0     MFC42D:MFC42D.DLL
 0002:000006e4       __imp_?OnDropEx@CView@@UAEKPAVCOleDataObject@@KKVCPoint@@@Z 5f58e6e4     MFC42D:MFC42D.DLL
 0002:000006e8       __imp_?OnDrop@CView@@UAEHPAVCOleDataObject@@KVCPoint@@@Z 5f58e6e8     MFC42D:MFC42D.DLL
 0002:000006ec       __imp_?OnDragLeave@CView@@UAEXXZ 5f58e6ec     MFC42D:MFC42D.DLL
 0002:000006f0       __imp_?OnDragOver@CView@@UAEKPAVCOleDataObject@@KVCPoint@@@Z 5f58e6f0     MFC42D:MFC42D.DLL
 0002:000006f4       __imp_?OnDragEnter@CView@@UAEKPAVCOleDataObject@@KVCPoint@@@Z 5f58e6f4     MFC42D:MFC42D.DLL
 0002:000006f8       __imp_?OnScrollBy@CView@@UAEHVCSize@@H@Z 5f58e6f8     MFC42D:MFC42D.DLL
 0002:000006fc       __imp_?OnScroll@CView@@UAEHIIH@Z 5f58e6fc     MFC42D:MFC42D.DLL
 0002:00000700       __imp_?PostNcDestroy@CView@@MAEXXZ 5f58e700     MFC42D:MFC42D.DLL
 0002:00000704       __imp_?PreTranslateMessage@CWnd@@UAEHPAUtagMSG@@@Z 5f58e704     MFC42D:MFC42D.DLL
 0002:00000708       __imp_?GetScrollBarCtrl@CView@@UBEPAVCScrollBar@@H@Z 5f58e708     MFC42D:MFC42D.DLL
 0002:0000070c       __imp_?CalcWindowRect@CView@@UAEXPAUtagRECT@@I@Z 5f58e70c     MFC42D:MFC42D.DLL
 0002:00000710       __imp_?OnCmdMsg@CView@@UAEHIHPAXPAUAFX_CMDHANDLERINFO@@@Z 5f58e710     MFC42D:MFC42D.DLL
 0002:00000714       __imp_??0CDWordArray@@QAE@XZ 5f58e714     MFC42D:MFC42D.DLL
 0002:00000718       __imp_??0CDC@@QAE@XZ       5f58e718     MFC42D:MFC42D.DLL
 0002:0000071c       __imp_??0CCtrlView@@QAE@PBDK@Z 5f58e71c     MFC42D:MFC42D.DLL
 0002:00000720       __imp_?PreCreateWindow@CCtrlView@@MAEHAAUtagCREATESTRUCTA@@@Z 5f58e720     MFC42D:MFC42D.DLL
 0002:00000724       __imp_?AfxInitRichEdit@@YGHXZ 5f58e724     MFC42D:MFC42D.DLL
 0002:00000728       __imp_?SetOptions@CRichEditCtrl@@QAEXGK@Z 5f58e728     MFC42D:MFC42D.DLL
 0002:0000072c       __imp_?DragAcceptFiles@CWnd@@QAEXH@Z 5f58e72c     MFC42D:MFC42D.DLL
 0002:00000730       __imp_?GetIRichEditOle@CRichEditCtrl@@QBEPAUIRichEditOle@@XZ 5f58e730     MFC42D:MFC42D.DLL
 0002:00000734       __imp_?SetOLECallback@CRichEditCtrl@@QAEHPAUIRichEditOleCallback@@@Z 5f58e734     MFC42D:MFC42D.DLL
 0002:00000738       __imp_?SetEventMask@CRichEditCtrl@@QAEKK@Z 5f58e738     MFC42D:MFC42D.DLL
 0002:0000073c       __imp_?LimitText@CRichEditCtrl@@QAEXJ@Z 5f58e73c     MFC42D:MFC42D.DLL
 0002:00000740       __imp_?OnCreate@CView@@IAEHPAUtagCREATESTRUCTA@@@Z 5f58e740     MFC42D:MFC42D.DLL
 0002:00000744       __imp_?OnInitialUpdate@CView@@UAEXXZ 5f58e744     MFC42D:MFC42D.DLL
 0002:00000748       __imp_?EmptyUndoBuffer@CRichEditCtrl@@QAEXXZ 5f58e748     MFC42D:MFC42D.DLL
 0002:0000074c       __imp_?SetWindowTextA@CWnd@@QAEXPBD@Z 5f58e74c     MFC42D:MFC42D.DLL
 0002:00000750       __imp_?SetTargetDevice@CRichEditCtrl@@QAEHAAVCDC@@J@Z 5f58e750     MFC42D:MFC42D.DLL
 0002:00000754       __imp_?CreateDCA@CDC@@QAEHPBD00PBX@Z 5f58e754     MFC42D:MFC42D.DLL
 0002:00000758       __imp_?CreatePrinterDC@CWinApp@@QAEHAAVCDC@@@Z 5f58e758     MFC42D:MFC42D.DLL
 0002:0000075c       __imp_?SetTargetDevice@CRichEditCtrl@@QAEHPAUHDC__@@J@Z 5f58e75c     MFC42D:MFC42D.DLL
 0002:00000760       __imp_?Invalidate@CWnd@@QAEXH@Z 5f58e760     MFC42D:MFC42D.DLL
 0002:00000764       __imp_?StreamIn@CRichEditCtrl@@QAEJHAAU_editstream@@@Z 5f58e764     MFC42D:MFC42D.DLL
 0002:00000768       __imp_?StreamOut@CRichEditCtrl@@QAEJHAAU_editstream@@@Z 5f58e768     MFC42D:MFC42D.DLL
 0002:0000076c       __imp_?classCFileException@CFileException@@2UCRuntimeClass@@B 5f58e76c     MFC42D:MFC42D.DLL
 0002:00000770       __imp_?ReadHuge@CFile@@QAEKPAXK@Z 5f58e770     MFC42D:MFC42D.DLL
 0002:00000774       __imp_?WriteHuge@CFile@@QAEXPBXK@Z 5f58e774     MFC42D:MFC42D.DLL
 0002:00000778       __imp_?GetFile@CArchive@@QBEPAVCFile@@XZ 5f58e778     MFC42D:MFC42D.DLL
 0002:0000077c       __imp_?Flush@CArchive@@QAEXXZ 5f58e77c     MFC42D:MFC42D.DLL
 0002:00000780       __imp_?FormatRange@CRichEditCtrl@@QAEJPAU_formatrange@@H@Z 5f58e780     MFC42D:MFC42D.DLL
 0002:00000784       __imp_?Add@CDWordArray@@QAEHK@Z 5f58e784     MFC42D:MFC42D.DLL
 0002:00000788       __imp_?GetSize@CDWordArray@@QBEHXZ 5f58e788     MFC42D:MFC42D.DLL
 0002:0000078c       __imp_?DPtoLP@CDC@@QBEXPAUtagRECT@@@Z 5f58e78c     MFC42D:MFC42D.DLL
 0002:00000790       __imp_?GetDeviceCaps@CDC@@QBEHH@Z 5f58e790     MFC42D:MFC42D.DLL
 0002:00000794       __imp_?IntersectClipRect@CDC@@QAEHHHHH@Z 5f58e794     MFC42D:MFC42D.DLL
 0002:00000798       __imp_?SetMaxPage@CPrintInfo@@QAEXI@Z 5f58e798     MFC42D:MFC42D.DLL
 0002:0000079c       __imp_??ACDWordArray@@QAEAAKH@Z 5f58e79c     MFC42D:MFC42D.DLL
 0002:000007a0       __imp_?RemoveAll@CDWordArray@@QAEXXZ 5f58e7a0     MFC42D:MFC42D.DLL
 0002:000007a4       __imp_?GetSel@CRichEditCtrl@@QBEXAAJ0@Z 5f58e7a4     MFC42D:MFC42D.DLL
 0002:000007a8       __imp_?_afxRichEditState@@3V?$CProcessLocal@V_AFX_RICHEDIT_STATE@@@@A 5f58e7a8     MFC42D:MFC42D.DLL
 0002:000007ac       __imp_?CanUndo@CRichEditCtrl@@QBEHXZ 5f58e7ac     MFC42D:MFC42D.DLL
 0002:000007b0       __imp_?IsKindOf@CObject@@QBEHPBUCRuntimeClass@@@Z 5f58e7b0     MFC42D:MFC42D.DLL
 0002:000007b4       __imp_?SetPathName@CDocument@@UAEXPBDH@Z 5f58e7b4     MFC42D:MFC42D.DLL
 0002:000007b8       __imp_?Paste@CRichEditCtrl@@QAEXXZ 5f58e7b8     MFC42D:MFC42D.DLL
 0002:000007bc       __imp_?Clear@CRichEditCtrl@@QAEXXZ 5f58e7bc     MFC42D:MFC42D.DLL
 0002:000007c0       __imp_?Undo@CRichEditCtrl@@QAEHXZ 5f58e7c0     MFC42D:MFC42D.DLL
 0002:000007c4       __imp_?SetSel@CRichEditCtrl@@QAEXJJ@Z 5f58e7c4     MFC42D:MFC42D.DLL
 0002:000007c8       __imp_?OnDestroy@CView@@IAEXXZ 5f58e7c8     MFC42D:MFC42D.DLL
 0002:000007cc       __imp_?AfxOleUnlockApp@@YGXXZ 5f58e7cc     MFC42D:MFC42D.DLL
 0002:000007d0       __imp_?AfxGetAppName@@YGPBDXZ 5f58e7d0     MFC42D:MFC42D.DLL
 0002:000007d4       __imp_??0CFontDialog@@QAE@ABU_charformat@@KPAVCDC@@PAVCWnd@@@Z 5f58e7d4     MFC42D:MFC42D.DLL
 0002:000007d8       __imp_?PasteSpecial@CRichEditCtrl@@QAEXIKPAUHMETAFILE__@@@Z 5f58e7d8     MFC42D:MFC42D.DLL
 0002:000007dc       __imp_?OnKeyDown@CWnd@@IAEXIII@Z 5f58e7dc     MFC42D:MFC42D.DLL
 0002:000007e0       __imp_?CenterPoint@CRect@@QBE?AVCPoint@@XZ 5f58e7e0     MFC42D:MFC42D.DLL
 0002:000007e4       __imp_?SetSel@CRichEditCtrl@@QAEXAAU_charrange@@@Z 5f58e7e4     MFC42D:MFC42D.DLL
 0002:000007e8       __imp_?GetSel@CRichEditCtrl@@QBEXAAU_charrange@@@Z 5f58e7e8     MFC42D:MFC42D.DLL
 0002:000007ec       __imp_?CanPaste@CRichEditCtrl@@QBEHI@Z 5f58e7ec     MFC42D:MFC42D.DLL
 0002:000007f0       __imp_?GetSelectionCharFormat@CRichEditCtrl@@QBEKAAU_charformat@@@Z 5f58e7f0     MFC42D:MFC42D.DLL
 0002:000007f4       __imp_?GetParaFormat@CRichEditCtrl@@QBEKAAU_paraformat@@@Z 5f58e7f4     MFC42D:MFC42D.DLL
 0002:000007f8       __imp_?SetSelectionCharFormat@CRichEditCtrl@@QAEHAAU_charformat@@@Z 5f58e7f8     MFC42D:MFC42D.DLL
 0002:000007fc       __imp_?SetParaFormat@CRichEditCtrl@@QAEHAAU_paraformat@@@Z 5f58e7fc     MFC42D:MFC42D.DLL
 0002:00000800       __imp_?MoveWindow@CWnd@@QAEXPBUtagRECT@@H@Z 5f58e800     MFC42D:MFC42D.DLL
 0002:00000804       __imp_?OffsetRect@CRect@@QAEXHH@Z 5f58e804     MFC42D:MFC42D.DLL
 0002:00000808       __imp_?Height@CRect@@QBEHXZ 5f58e808     MFC42D:MFC42D.DLL
 0002:0000080c       __imp_?GetWindowRect@CWnd@@QBEXPAUtagRECT@@@Z 5f58e80c     MFC42D:MFC42D.DLL
 0002:00000810       __imp_?ClientToScreen@CWnd@@QBEXPAUtagPOINT@@@Z 5f58e810     MFC42D:MFC42D.DLL
 0002:00000814       __imp_?GetCharPos@CRichEditCtrl@@QBE?AVCPoint@@J@Z 5f58e814     MFC42D:MFC42D.DLL
 0002:00000818       __imp_?Create@CFindReplaceDialog@@QAEHHPBD0KPAVCWnd@@@Z 5f58e818     MFC42D:MFC42D.DLL
 0002:0000081c       __imp_??0CFindReplaceDialog@@QAE@XZ 5f58e81c     MFC42D:MFC42D.DLL
 0002:00000820       __imp_?FindOneOf@CString@@QBEHPBD@Z 5f58e820     MFC42D:MFC42D.DLL
 0002:00000824       __imp_?GetSelText@CRichEditCtrl@@QBE?AVCString@@XZ 5f58e824     MFC42D:MFC42D.DLL
 0002:00000828       __imp_?ReplaceSel@CRichEditCtrl@@QAEXPBDH@Z 5f58e828     MFC42D:MFC42D.DLL
 0002:0000082c       __imp_?HideSelection@CRichEditCtrl@@QAEXHH@Z 5f58e82c     MFC42D:MFC42D.DLL
 0002:00000830       __imp_?ReplaceAll@CFindReplaceDialog@@QBEHXZ 5f58e830     MFC42D:MFC42D.DLL
 0002:00000834       __imp_?GetReplaceString@CFindReplaceDialog@@QBE?AVCString@@XZ 5f58e834     MFC42D:MFC42D.DLL
 0002:00000838       __imp_?ReplaceCurrent@CFindReplaceDialog@@QBEHXZ 5f58e838     MFC42D:MFC42D.DLL
 0002:0000083c       __imp_?GetFindString@CFindReplaceDialog@@QBE?AVCString@@XZ 5f58e83c     MFC42D:MFC42D.DLL
 0002:00000840       __imp_?SearchDown@CFindReplaceDialog@@QBEHXZ 5f58e840     MFC42D:MFC42D.DLL
 0002:00000844       __imp_?MatchCase@CFindReplaceDialog@@QBEHXZ 5f58e844     MFC42D:MFC42D.DLL
 0002:00000848       __imp_?MatchWholeWord@CFindReplaceDialog@@QBEHXZ 5f58e848     MFC42D:MFC42D.DLL
 0002:0000084c       __imp_?FindNext@CFindReplaceDialog@@QBEHXZ 5f58e84c     MFC42D:MFC42D.DLL
 0002:00000850       __imp_?IsTerminating@CFindReplaceDialog@@QBEHXZ 5f58e850     MFC42D:MFC42D.DLL
 0002:00000854       __imp_?GetNotifier@CFindReplaceDialog@@SGPAV1@J@Z 5f58e854     MFC42D:MFC42D.DLL
 0002:00000858       __imp_?FindTextA@CRichEditCtrl@@QBEJKPAU_findtextexa@@@Z 5f58e858     MFC42D:MFC42D.DLL
 0002:0000085c       __imp_?AssertValid@CCtrlView@@UBEXXZ 5f58e85c     MFC42D:MFC42D.DLL
 0002:00000860       __imp_?Dump@CCtrlView@@UBEXAAVCDumpContext@@@Z 5f58e860     MFC42D:MFC42D.DLL
 0002:00000864       __imp_?GetModify@CRichEditCtrl@@QBEHXZ 5f58e864     MFC42D:MFC42D.DLL
 0002:00000868       __imp_?SetModify@CRichEditCtrl@@QAEXH@Z 5f58e868     MFC42D:MFC42D.DLL
 0002:0000086c       __imp_??0CRect@@QAE@UtagPOINT@@UtagSIZE@@@Z 5f58e86c     MFC42D:MFC42D.DLL
 0002:00000870       __imp_?GetTextLength@CRichEditCtrl@@QBEJXZ 5f58e870     MFC42D:MFC42D.DLL
 0002:00000874       __imp_?classCCtrlView@CCtrlView@@2UCRuntimeClass@@B 5f58e874     MFC42D:MFC42D.DLL
 0002:00000878       __imp_??0_AFX_EDIT_STATE@@QAE@XZ 5f58e878     MFC42D:MFC42D.DLL
 0002:0000087c       __imp_??1_AFX_RICHEDIT_STATE@@UAE@XZ 5f58e87c     MFC42D:MFC42D.DLL
 0002:00000880       __imp_?AfxOleCanExitApp@@YGHXZ 5f58e880     MFC42D:MFC42D.DLL
 0002:00000884       __imp_??3@YAXPAXPBDH@Z     5f58e884     MFC42D:MFC42D.DLL
 0002:00000888       __imp_?Lookup@CMapPtrToPtr@@QBEHPAXAAPAX@Z 5f58e888     MFC42D:MFC42D.DLL
 0002:0000088c       __imp_?SetAt@CMapPtrToPtr@@QAEXPAX0@Z 5f58e88c     MFC42D:MFC42D.DLL
 0002:00000890       __imp_?RemoveAll@CTypeLibCacheMap@@UAEXPAX@Z 5f58e890     MFC42D:MFC42D.DLL
 0002:00000894       __imp_?Dump@CMapPtrToPtr@@UBEXAAVCDumpContext@@@Z 5f58e894     MFC42D:MFC42D.DLL
 0002:00000898       __imp_?AssertValid@CMapPtrToPtr@@UBEXXZ 5f58e898     MFC42D:MFC42D.DLL
 0002:0000089c       __imp_?GetRuntimeClass@CMapPtrToPtr@@UBEPAUCRuntimeClass@@XZ 5f58e89c     MFC42D:MFC42D.DLL
 0002:000008a0       __imp_??0CMapPtrToPtr@@QAE@H@Z 5f58e8a0     MFC42D:MFC42D.DLL
 0002:000008a4       __imp_??1CMapPtrToPtr@@UAE@XZ 5f58e8a4     MFC42D:MFC42D.DLL
 0002:000008a8       __imp_?AfxEndDeferRegisterClass@@YGHJ@Z 5f58e8a8     MFC42D:MFC42D.DLL
 0002:000008ac       __imp_??0CTime@@QAE@ABU_SYSTEMTIME@@H@Z 5f58e8ac     MFC42D:MFC42D.DLL
 0002:000008b0       __imp_?GetAsSystemTime@CTime@@QBEHAAU_SYSTEMTIME@@@Z 5f58e8b0     MFC42D:MFC42D.DLL
 0002:000008b4       __imp_?GetMessageMap@CWnd@@MBEPBUAFX_MSGMAP@@XZ 5f58e8b4     MFC42D:MFC42D.DLL
 0002:000008b8       __imp_?Dump@CWnd@@UBEXAAVCDumpContext@@@Z 5f58e8b8     MFC42D:MFC42D.DLL
 0002:000008bc       __imp_?AfxAssertFailedLine@@YGHPBDH@Z 5f58e8bc     MFC42D:MFC42D.DLL
 0002:000008c0       __imp_??1CWnd@@UAE@XZ      5f58e8c0     MFC42D:MFC42D.DLL
 0002:000008c4       __imp_?SetWindowPos@CWnd@@QAEHPBV1@HHHHI@Z 5f58e8c4     MFC42D:MFC42D.DLL
 0002:000008c8       __imp_?Width@CRect@@QBEHXZ 5f58e8c8     MFC42D:MFC42D.DLL
 0002:000008cc       __imp_?PrepareCtrl@CDataExchange@@QAEPAUHWND__@@H@Z 5f58e8cc     MFC42D:MFC42D.DLL
 0002:000008d0       __imp_??MCTime@@QBEHV0@@Z  5f58e8d0     MFC42D:MFC42D.DLL
 0002:000008d4       __imp_??OCTime@@QBEHV0@@Z  5f58e8d4     MFC42D:MFC42D.DLL
 0002:000008d8       __imp_??NCTime@@QBEHV0@@Z  5f58e8d8     MFC42D:MFC42D.DLL
 0002:000008dc       __imp_??0CTime@@QAE@ABV0@@Z 5f58e8dc     MFC42D:MFC42D.DLL
 0002:000008e0       __imp_??0CWnd@@QAE@XZ      5f58e8e0     MFC42D:MFC42D.DLL
 0002:000008e4       __imp_?FromHandle@CFont@@SGPAV1@PAUHFONT__@@@Z 5f58e8e4     MFC42D:MFC42D.DLL
 0002:000008e8       __imp_?classCWnd@CWnd@@2UCRuntimeClass@@B 5f58e8e8     MFC42D:MFC42D.DLL
 0002:000008ec       __imp_?messageMap@CFormView@@1UAFX_MSGMAP@@B 5f58e8ec     MFC42D:MFC42D.DLL
 0002:000008f0       __imp_?eventsinkMap@CCmdTarget@@1UAFX_EVENTSINKMAP@@B 5f58e8f0     MFC42D:MFC42D.DLL
 0002:000008f4       __imp_?OnEndPrinting@CView@@MAEXPAVCDC@@PAUCPrintInfo@@@Z 5f58e8f4     MFC42D:MFC42D.DLL
 0002:000008f8       __imp_?OnPrint@CView@@MAEXPAVCDC@@PAUCPrintInfo@@@Z 5f58e8f8     MFC42D:MFC42D.DLL
 0002:000008fc       __imp_?OnBeginPrinting@CView@@MAEXPAVCDC@@PAUCPrintInfo@@@Z 5f58e8fc     MFC42D:MFC42D.DLL
 0002:00000900       __imp_?OnActivateFrame@CFormView@@MAEXIPAVCFrameWnd@@@Z 5f58e900     MFC42D:MFC42D.DLL
 0002:00000904       __imp_?OnActivateView@CFormView@@MAEXHPAVCView@@0@Z 5f58e904     MFC42D:MFC42D.DLL
 0002:00000908       __imp_?OnInitialUpdate@CFormView@@UAEXXZ 5f58e908     MFC42D:MFC42D.DLL
 0002:0000090c       __imp_?OnPrepareDC@CScrollView@@UAEXPAVCDC@@PAUCPrintInfo@@@Z 5f58e90c     MFC42D:MFC42D.DLL
 0002:00000910       __imp_?OnScrollBy@CScrollView@@UAEHVCSize@@H@Z 5f58e910     MFC42D:MFC42D.DLL
 0002:00000914       __imp_?OnScroll@CScrollView@@UAEHIIH@Z 5f58e914     MFC42D:MFC42D.DLL
 0002:00000918       __imp_?IsSelected@CView@@UBEHPBVCObject@@@Z 5f58e918     MFC42D:MFC42D.DLL
 0002:0000091c       __imp_?SetOccDialogInfo@CFormView@@MAEHPAU_AFX_OCC_DIALOG_INFO@@@Z 5f58e91c     MFC42D:MFC42D.DLL
 0002:00000920       __imp_?PreTranslateMessage@CFormView@@MAEHPAUtagMSG@@@Z 5f58e920     MFC42D:MFC42D.DLL
 0002:00000924       __imp_?CalcWindowRect@CScrollView@@UAEXPAUtagRECT@@I@Z 5f58e924     MFC42D:MFC42D.DLL
 0002:00000928       __imp_?PreCreateWindow@CView@@MAEHAAUtagCREATESTRUCTA@@@Z 5f58e928     MFC42D:MFC42D.DLL
 0002:0000092c       __imp_??0CFormView@@IAE@PBD@Z 5f58e92c     MFC42D:MFC42D.DLL
 0002:00000930       __imp_??1CScrollView@@UAE@XZ 5f58e930     MFC42D:MFC42D.DLL
 0002:00000934       __imp_?AssertValid@CFormView@@UBEXXZ 5f58e934     MFC42D:MFC42D.DLL
 0002:00000938       __imp_?Dump@CFormView@@UBEXAAVCDumpContext@@@Z 5f58e938     MFC42D:MFC42D.DLL
 0002:0000093c       __imp_?OnSize@CScrollView@@QAEXIHH@Z 5f58e93c     MFC42D:MFC42D.DLL
 0002:00000940       __imp_?Default@CWnd@@IAEJXZ 5f58e940     MFC42D:MFC42D.DLL
 0002:00000944       __imp_?GetControlUnknown@CWnd@@QAEPAUIUnknown@@XZ 5f58e944     MFC42D:MFC42D.DLL
 0002:00000948       __imp_??0CString@@QAE@PBG@Z 5f58e948     MFC42D:MFC42D.DLL
 0002:0000094c       __imp_?AfxGetResourceHandle@@YGPAUHINSTANCE__@@XZ 5f58e94c     MFC42D:MFC42D.DLL
 0002:00000950       __imp_?InvokeHelper@CWnd@@QAAXJGGPAXPBEZZ 5f58e950     MFC42D:MFC42D.DLL
 0002:00000954       __imp_??1CByteArray@@UAE@XZ 5f58e954     MFC42D:MFC42D.DLL
 0002:00000958       __imp_?GetData@CByteArray@@QAEPAEXZ 5f58e958     MFC42D:MFC42D.DLL
 0002:0000095c       __imp_?SetSize@CByteArray@@QAEXHH@Z 5f58e95c     MFC42D:MFC42D.DLL
 0002:00000960       __imp_??0CByteArray@@QAE@XZ 5f58e960     MFC42D:MFC42D.DLL
 0002:00000964       __imp_?SetMessageText@CFrameWnd@@QAEXPBD@Z 5f58e964     MFC42D:MFC42D.DLL
 0002:00000968       __imp_?classCFormView@CFormView@@2UCRuntimeClass@@B 5f58e968     MFC42D:MFC42D.DLL
 0002:0000096c       __imp_?AfxFindResourceHandle@@YGPAUHINSTANCE__@@PBD0@Z 5f58e96c     MFC42D:MFC42D.DLL
 0002:00000970       __imp_?GetNextAssoc@CMapPtrToPtr@@QBEXAAPAU__POSITION@@AAPAX1@Z 5f58e970     MFC42D:MFC42D.DLL
 0002:00000974       __imp_?GetStartPosition@CMapPtrToPtr@@QBEPAU__POSITION@@XZ 5f58e974     MFC42D:MFC42D.DLL
 0002:00000978       __imp_??0CMemFile@@QAE@PAEII@Z 5f58e978     MFC42D:MFC42D.DLL
 0002:0000097c       __imp_?AfxThrowNotSupportedException@@YGXXZ 5f58e97c     MFC42D:MFC42D.DLL
 0002:00000980       __imp_?TopLeft@CRect@@QAEAAVCPoint@@XZ 5f58e980     MFC42D:MFC42D.DLL
 0002:00000984       __imp_??0CRect@@QAE@ABUtagRECT@@@Z 5f58e984     MFC42D:MFC42D.DLL
 0002:00000988       __imp_?dispatchMap@CCmdTarget@@1UAFX_DISPMAP@@B 5f58e988     MFC42D:MFC42D.DLL
 0002:0000098c       __imp_?RemoveAll@CMapPtrToPtr@@QAEXXZ 5f58e98c     MFC42D:MFC42D.DLL
 0002:00000990       __imp_?RemoveKey@CMapPtrToPtr@@QAEHPAX@Z 5f58e990     MFC42D:MFC42D.DLL
 0002:00000994       __imp_?GetFont@CWnd@@QBEPAVCFont@@XZ 5f58e994     MFC42D:MFC42D.DLL
 0002:00000998       __imp_??1CWindowDC@@UAE@XZ 5f58e998     MFC42D:MFC42D.DLL
 0002:0000099c       __imp_?GetTextColor@CDC@@QBEKXZ 5f58e99c     MFC42D:MFC42D.DLL
 0002:000009a0       __imp_?GetBkColor@CDC@@QBEKXZ 5f58e9a0     MFC42D:MFC42D.DLL
 0002:000009a4       __imp_??0CWindowDC@@QAE@PAVCWnd@@@Z 5f58e9a4     MFC42D:MFC42D.DLL
 0002:000009a8       __imp_?AfxGetCtl3dState@@YGPAV_AFX_CTL3D_STATE@@XZ 5f58e9a8     MFC42D:MFC42D.DLL
 0002:000009ac       __imp_?GetLogFont@CFont@@QAEHPAUtagLOGFONTA@@@Z 5f58e9ac     MFC42D:MFC42D.DLL
 0002:000009b0       __imp_??1CFont@@UAE@XZ     5f58e9b0     MFC42D:MFC42D.DLL
 0002:000009b4       __imp_?CreateStockObject@CGdiObject@@QAEHH@Z 5f58e9b4     MFC42D:MFC42D.DLL
 0002:000009b8       __imp_??0CFont@@QAE@XZ     5f58e9b8     MFC42D:MFC42D.DLL
 0002:000009bc       __imp_?GetWindowTextA@CWnd@@QBEHPADH@Z 5f58e9bc     MFC42D:MFC42D.DLL
 0002:000009c0       __imp_?GetProperty@CWnd@@QBEXJGPAX@Z 5f58e9c0     MFC42D:MFC42D.DLL
 0002:000009c4       __imp_?GetCount@CMapPtrToPtr@@QBEHXZ 5f58e9c4     MFC42D:MFC42D.DLL
 0002:000009c8       __imp_??1CClientDC@@UAE@XZ 5f58e9c8     MFC42D:MFC42D.DLL
 0002:000009cc       __imp_??0CClientDC@@QAE@PAVCWnd@@@Z 5f58e9cc     MFC42D:MFC42D.DLL
 0002:000009d0       __imp_?UnsubclassWindow@CWnd@@QAEPAUHWND__@@XZ 5f58e9d0     MFC42D:MFC42D.DLL
 0002:000009d4       __imp_?ModifyStyle@CWnd@@SGHPAUHWND__@@KKI@Z 5f58e9d4     MFC42D:MFC42D.DLL
 0002:000009d8       __imp_?ModifyStyleEx@CWnd@@SGHPAUHWND__@@KKI@Z 5f58e9d8     MFC42D:MFC42D.DLL
 0002:000009dc       __imp_??0CRect@@QAE@PBUtagRECT@@@Z 5f58e9dc     MFC42D:MFC42D.DLL
 0002:000009e0       __imp_??1CPtrList@@UAE@XZ  5f58e9e0     MFC42D:MFC42D.DLL
 0002:000009e4       __imp_??0CPtrList@@QAE@H@Z 5f58e9e4     MFC42D:MFC42D.DLL
 0002:000009e8       __imp_?RemoveAll@CPtrList@@QAEXXZ 5f58e9e8     MFC42D:MFC42D.DLL
 0002:000009ec       __imp_?GetHead@CPtrList@@QAEAAPAXXZ 5f58e9ec     MFC42D:MFC42D.DLL
 0002:000009f0       __imp_?MoveWindow@CWnd@@QAEXHHHHH@Z 5f58e9f0     MFC42D:MFC42D.DLL
 0002:000009f4       __imp_?GetDesktopWindow@CWnd@@SGPAV1@XZ 5f58e9f4     MFC42D:MFC42D.DLL
 0002:000009f8       __imp_?RemoveAt@CPtrList@@QAEXPAU__POSITION@@@Z 5f58e9f8     MFC42D:MFC42D.DLL
 0002:000009fc       __imp_??8@YG_NABVCString@@PBD@Z 5f58e9fc     MFC42D:MFC42D.DLL
 0002:00000a00       __imp_?AddTail@CPtrList@@QAEPAU__POSITION@@PAX@Z 5f58ea00     MFC42D:MFC42D.DLL
 0002:00000a04       __imp_??8@YG_NABVCString@@0@Z 5f58ea04     MFC42D:MFC42D.DLL
 0002:00000a08       __imp_?Find@CPtrList@@QBEPAU__POSITION@@PAXPAU2@@Z 5f58ea08     MFC42D:MFC42D.DLL
 0002:00000a0c       __imp_?GetCount@CPtrList@@QBEHXZ 5f58ea0c     MFC42D:MFC42D.DLL
 0002:00000a10       __imp_?SetProperty@CWnd@@QAAXJGZZ 5f58ea10     MFC42D:MFC42D.DLL
 0002:00000a14       __imp_?GetNextWindow@CWnd@@QBEPAV1@I@Z 5f58ea14     MFC42D:MFC42D.DLL
 0002:00000a18       __imp_?GetTopWindow@CWnd@@QBEPAV1@XZ 5f58ea18     MFC42D:MFC42D.DLL
 0002:00000a1c       __imp_?GetNextDlgGroupItem@CWnd@@QBEPAV1@PAV1@H@Z 5f58ea1c     MFC42D:MFC42D.DLL
 0002:00000a20       __imp_?GetNextDlgTabItem@CWnd@@QBEPAV1@PAV1@H@Z 5f58ea20     MFC42D:MFC42D.DLL
 0002:00000a24       __imp_?IsChild@CWnd@@QBEHPBV1@@Z 5f58ea24     MFC42D:MFC42D.DLL
 0002:00000a28       __imp_?GetDlgCtrlID@CWnd@@QBEHXZ 5f58ea28     MFC42D:MFC42D.DLL
 0002:00000a2c       __imp_?messageMap@CCmdTarget@@1UAFX_MSGMAP@@B 5f58ea2c     MFC42D:MFC42D.DLL
 0002:00000a30       __imp_?GetFromPage@CPrintInfo@@QBEIXZ 5f58ea30     MFC42D:MFC42D.DLL
 0002:00000a34       __imp_?GetToPage@CPrintInfo@@QBEIXZ 5f58ea34     MFC42D:MFC42D.DLL
 0002:00000a38       __imp_?GetMinPage@CPrintInfo@@QBEIXZ 5f58ea38     MFC42D:MFC42D.DLL
 0002:00000a3c       __imp_??1CPrintInfo@@QAE@XZ 5f58ea3c     MFC42D:MFC42D.DLL
 0002:00000a40       __imp_??0CPrintInfo@@QAE@XZ 5f58ea40     MFC42D:MFC42D.DLL
 0002:00000a44       __imp_?AbortDoc@CDC@@QAEHXZ 5f58ea44     MFC42D:MFC42D.DLL
 0002:00000a48       __imp_?EndDoc@CDC@@QAEHXZ  5f58ea48     MFC42D:MFC42D.DLL
 0002:00000a4c       __imp_?EndPage@CDC@@QAEHXZ 5f58ea4c     MFC42D:MFC42D.DLL
 0002:00000a50       __imp_?StartPage@CDC@@QAEHXZ 5f58ea50     MFC42D:MFC42D.DLL
 0002:00000a54       __imp_?GetMaxPage@CPrintInfo@@QBEIXZ 5f58ea54     MFC42D:MFC42D.DLL
 0002:00000a58       __imp_?Detach@CDC@@QAEPAUHDC__@@XZ 5f58ea58     MFC42D:MFC42D.DLL
 0002:00000a5c       __imp_?StartDocA@CDC@@QAEHPAU_DOCINFOA@@@Z 5f58ea5c     MFC42D:MFC42D.DLL
 0002:00000a60       __imp_?SetAbortProc@CDC@@QAEHP6GHPAUHDC__@@H@Z@Z 5f58ea60     MFC42D:MFC42D.DLL
 0002:00000a64       __imp_?_AfxAbortProc@@YGHPAUHDC__@@H@Z 5f58ea64     MFC42D:MFC42D.DLL
 0002:00000a68       __imp_?Attach@CDC@@QAEHPAUHDC__@@@Z 5f58ea68     MFC42D:MFC42D.DLL
 0002:00000a6c       __imp_?GetWindowTextA@CWnd@@QBEXAAVCString@@@Z 5f58ea6c     MFC42D:MFC42D.DLL
 0002:00000a70       __imp_?SetRadio@CCmdUI@@UAEXH@Z 5f58ea70     MFC42D:MFC42D.DLL
 0002:00000a74       __imp_??0CCmdUI@@QAE@XZ    5f58ea74     MFC42D:MFC42D.DLL
 0002:00000a78       __imp_?Right@CString@@QBE?AV1@H@Z 5f58ea78     MFC42D:MFC42D.DLL
 0002:00000a7c       __imp_?RemoveMenu@CMenu@@QAEHII@Z 5f58ea7c     MFC42D:MFC42D.DLL
 0002:00000a80       __imp_?GetMenuItemCount@CMenu@@QBEIXZ 5f58ea80     MFC42D:MFC42D.DLL
 0002:00000a84       __imp_?CreateMenu@CMenu@@QAEHXZ 5f58ea84     MFC42D:MFC42D.DLL
 0002:00000a88       __imp_??0CMenu@@QAE@XZ     5f58ea88     MFC42D:MFC42D.DLL
 0002:00000a8c       __imp_?Remove@CString@@QAEHD@Z 5f58ea8c     MFC42D:MFC42D.DLL
 0002:00000a90       __imp_?GetMenuStringA@CMenu@@QBEHIAAVCString@@I@Z 5f58ea90     MFC42D:MFC42D.DLL
 0002:00000a94       __imp_?GetSubMenu@CMenu@@QBEPAV1@H@Z 5f58ea94     MFC42D:MFC42D.DLL
 0002:00000a98       __imp_?SetStatusText@CControlBar@@UAEHH@Z 5f58ea98     MFC42D:MFC42D.DLL
 0002:00000a9c       __imp_?DoPaint@CControlBar@@UAEXPAVCDC@@@Z 5f58ea9c     MFC42D:MFC42D.DLL
 0002:00000aa0       __imp_?OnBarStyleChange@CControlBar@@UAEXKK@Z 5f58eaa0     MFC42D:MFC42D.DLL
 0002:00000aa4       __imp_?IsDockBar@CControlBar@@UBEHXZ 5f58eaa4     MFC42D:MFC42D.DLL
 0002:00000aa8       __imp_?RecalcDelayShow@CControlBar@@UAEKPAUAFX_SIZEPARENTPARAMS@@@Z 5f58eaa8     MFC42D:MFC42D.DLL
 0002:00000aac       __imp_?IsVisible@CControlBar@@UBEHXZ 5f58eaac     MFC42D:MFC42D.DLL
 0002:00000ab0       __imp_?DelayShow@CControlBar@@UAEXH@Z 5f58eab0     MFC42D:MFC42D.DLL
 0002:00000ab4       __imp_?CalcDynamicLayout@CControlBar@@UAE?AVCSize@@HK@Z 5f58eab4     MFC42D:MFC42D.DLL
 0002:00000ab8       __imp_?CalcFixedLayout@CControlBar@@UAE?AVCSize@@HH@Z 5f58eab8     MFC42D:MFC42D.DLL
 0002:00000abc       __imp_?PostNcDestroy@CControlBar@@UAEXXZ 5f58eabc     MFC42D:MFC42D.DLL
 0002:00000ac0       __imp_?WindowProc@CControlBar@@UAEJIIJ@Z 5f58eac0     MFC42D:MFC42D.DLL
 0002:00000ac4       __imp_?PreTranslateMessage@CControlBar@@UAEHPAUtagMSG@@@Z 5f58eac4     MFC42D:MFC42D.DLL
 0002:00000ac8       __imp_?PreCreateWindow@CControlBar@@UAEHAAUtagCREATESTRUCTA@@@Z 5f58eac8     MFC42D:MFC42D.DLL
 0002:00000acc       __imp_?DestroyWindow@CControlBar@@UAEHXZ 5f58eacc     MFC42D:MFC42D.DLL
 0002:00000ad0       __imp_?Dump@CControlBar@@UBEXAAVCDumpContext@@@Z 5f58ead0     MFC42D:MFC42D.DLL
 0002:00000ad4       __imp_?AssertValid@CControlBar@@UBEXXZ 5f58ead4     MFC42D:MFC42D.DLL
 0002:00000ad8       __imp_??1CControlBar@@UAE@XZ 5f58ead8     MFC42D:MFC42D.DLL
 0002:00000adc       __imp_??0CRectTracker@@QAE@XZ 5f58eadc     MFC42D:MFC42D.DLL
 0002:00000ae0       __imp_??0CControlBar@@IAE@XZ 5f58eae0     MFC42D:MFC42D.DLL
 0002:00000ae4       __imp_??1CRectTracker@@UAE@XZ 5f58eae4     MFC42D:MFC42D.DLL
 0002:00000ae8       __imp_?messageMap@CControlBar@@1UAFX_MSGMAP@@B 5f58eae8     MFC42D:MFC42D.DLL
 0002:00000aec       __imp_??1CPaintDC@@UAE@XZ  5f58eaec     MFC42D:MFC42D.DLL
 0002:00000af0       __imp_?Draw@CRectTracker@@QBEXPAVCDC@@@Z 5f58eaf0     MFC42D:MFC42D.DLL
 0002:00000af4       __imp_?SetBrushOrg@CDC@@QAE?AVCPoint@@HH@Z 5f58eaf4     MFC42D:MFC42D.DLL
 0002:00000af8       __imp_??0CPaintDC@@QAE@PAVCWnd@@@Z 5f58eaf8     MFC42D:MFC42D.DLL
 0002:00000afc       __imp_?SetCursor@CRectTracker@@QBEHPAVCWnd@@I@Z 5f58eafc     MFC42D:MFC42D.DLL
 0002:00000b00       __imp_?OnSetCursor@CWnd@@IAEHPAV1@II@Z 5f58eb00     MFC42D:MFC42D.DLL
 0002:00000b04       __imp_?HitTest@CRectTracker@@QBEHVCPoint@@@Z 5f58eb04     MFC42D:MFC42D.DLL
 0002:00000b08       __imp_?GetOwner@CWnd@@QBEPAV1@XZ 5f58eb08     MFC42D:MFC42D.DLL
 0002:00000b0c       __imp_?Track@CRectTracker@@QAEHPAVCWnd@@VCPoint@@H0@Z 5f58eb0c     MFC42D:MFC42D.DLL
 0002:00000b10       __imp_?classCControlBar@CControlBar@@2UCRuntimeClass@@B 5f58eb10     MFC42D:MFC42D.DLL
 0002:00000b14       __imp_?messageMap@CWnd@@1UAFX_MSGMAP@@B 5f58eb14     MFC42D:MFC42D.DLL
 0002:00000b18       __imp_?SetWindowOrg@CDC@@QAE?AVCPoint@@HH@Z 5f58eb18     MFC42D:MFC42D.DLL
 0002:00000b1c       __imp_?SetViewportExt@CDC@@QAE?AVCSize@@UtagSIZE@@@Z 5f58eb1c     MFC42D:MFC42D.DLL
 0002:00000b20       __imp_?CreateEx@CWnd@@QAEHKPBD0KHHHHPAUHWND__@@PAUHMENU__@@PAX@Z 5f58eb20     MFC42D:MFC42D.DLL
 0002:00000b24       __imp_?LPtoDP@CDC@@QBEXPAUtagRECT@@@Z 5f58eb24     MFC42D:MFC42D.DLL
 0002:00000b28       __imp_?SetWindowExt@CDC@@UAE?AVCSize@@HH@Z 5f58eb28     MFC42D:MFC42D.DLL
 0002:00000b2c       __imp_?SetMapMode@CDC@@UAEHH@Z 5f58eb2c     MFC42D:MFC42D.DLL
 0002:00000b30       __imp_?InvalidateRect@CWnd@@QAEXPBUtagRECT@@H@Z 5f58eb30     MFC42D:MFC42D.DLL
 0002:00000b34       __imp_?OffsetRect@CRect@@QAEXUtagPOINT@@@Z 5f58eb34     MFC42D:MFC42D.DLL
 0002:00000b38       __imp_?AfxUnlockTempMaps@@YGHH@Z 5f58eb38     MFC42D:MFC42D.DLL
 0002:00000b3c       __imp_?AfxLockTempMaps@@YGXXZ 5f58eb3c     MFC42D:MFC42D.DLL
 0002:00000b40       __imp_?ValidateRect@CWnd@@QAEXPBUtagRECT@@@Z 5f58eb40     MFC42D:MFC42D.DLL
 0002:00000b44       __imp_?OnEraseBkgnd@CWnd@@IAEHPAVCDC@@@Z 5f58eb44     MFC42D:MFC42D.DLL
 0002:00000b48       __imp_?IsLoading@CArchive@@QBEHXZ 5f58eb48     MFC42D:MFC42D.DLL
 0002:00000b4c       __imp_?OnNcCreate@CWnd@@IAEHPAUtagCREATESTRUCTA@@@Z 5f58eb4c     MFC42D:MFC42D.DLL
 0002:00000b50       __imp_?OnMouseActivate@CWnd@@IAEHPAV1@II@Z 5f58eb50     MFC42D:MFC42D.DLL
 0002:00000b54       __imp_?ReflectChildNotify@CWnd@@IAEHIIJPAJ@Z 5f58eb54     MFC42D:MFC42D.DLL
 0002:00000b58       __imp_?OnCreate@CWnd@@IAEHPAUtagCREATESTRUCTA@@@Z 5f58eb58     MFC42D:MFC42D.DLL
 0002:00000b5c       __imp_?OnMove@CWnd@@IAEXHH@Z 5f58eb5c     MFC42D:MFC42D.DLL
 0002:00000b60       __imp_?OnShowWindow@CWnd@@IAEXHI@Z 5f58eb60     MFC42D:MFC42D.DLL
 0002:00000b64       __imp_?DoUpdate@CCmdUI@@QAEHPAVCCmdTarget@@H@Z 5f58eb64     MFC42D:MFC42D.DLL
 0002:00000b68       __imp_?GetMenuItemID@CMenu@@QBEIH@Z 5f58eb68     MFC42D:MFC42D.DLL
 0002:00000b6c       __imp_?AfxCancelModes@@YGXPAUHWND__@@@Z 5f58eb6c     MFC42D:MFC42D.DLL
 0002:00000b70       __imp_?OnDestroy@CWnd@@IAEXXZ 5f58eb70     MFC42D:MFC42D.DLL
 0002:00000b74       __imp_?OnKillFocus@CWnd@@IAEXPAV1@@Z 5f58eb74     MFC42D:MFC42D.DLL
 0002:00000b78       __imp_?OnSetFocus@CWnd@@IAEXPAV1@@Z 5f58eb78     MFC42D:MFC42D.DLL
 0002:00000b7c       __imp_?GetData@CThreadLocalObject@@QAEPAVCNoTrackObject@@P6GPAV2@XZ@Z 5f58eb7c     MFC42D:MFC42D.DLL
 0002:00000b80       __imp_?GetRuntimeClass@CWnd@@UBEPAUCRuntimeClass@@XZ 5f58eb80     MFC42D:MFC42D.DLL
 0002:00000b84       __imp_?connectionMap@CCmdTarget@@1UAFX_CONNECTIONMAP@@B 5f58eb84     MFC42D:MFC42D.DLL
 0002:00000b88       __imp_?Add@CPtrArray@@QAEHPAX@Z 5f58eb88     MFC42D:MFC42D.DLL
 0002:00000b8c       __imp_?OnGetDlgCode@CWnd@@IAEIXZ 5f58eb8c     MFC42D:MFC42D.DLL
 0002:00000b90       __imp_?OnCancelMode@CWnd@@IAEXXZ 5f58eb90     MFC42D:MFC42D.DLL
 0002:00000b94       __imp_?MessageBoxA@CWnd@@QAEHPBD0I@Z 5f58eb94     MFC42D:MFC42D.DLL
 0002:00000b98       __imp_?classCWinApp@CWinApp@@2UCRuntimeClass@@B 5f58eb98     MFC42D:MFC42D.DLL
 0002:00000b9c       __imp_?ExitInstance@CWinApp@@UAEHXZ 5f58eb9c     MFC42D:MFC42D.DLL
 0002:00000ba0       __imp_?OnActivate@CWnd@@IAEXIPAV1@H@Z 5f58eba0     MFC42D:MFC42D.DLL
 0002:00000ba4       __imp_??4CRect@@QAEXABUtagRECT@@@Z 5f58eba4     MFC42D:MFC42D.DLL
 0002:00000ba8       __imp_?Read@CFile@@UAEIPAXI@Z 5f58eba8     MFC42D:MFC42D.DLL
 0002:00000bac       __imp_?_wcstombsz@@YAHPADPBGI@Z 5f58ebac     MFC42D:MFC42D.DLL
 0002:00000bb0       __imp_??0CFile@@QAE@PBDI@Z 5f58ebb0     MFC42D:MFC42D.DLL
 0002:00000bb4       __imp_?GetSize@CPtrArray@@QBEHXZ 5f58ebb4     MFC42D:MFC42D.DLL
 0002:00000bb8       __imp_?GetAt@CPtrArray@@QBEPAXH@Z 5f58ebb8     MFC42D:MFC42D.DLL
 0002:00000bbc       __imp_??0CPtrArray@@QAE@XZ 5f58ebbc     MFC42D:MFC42D.DLL
 0002:00000bc0       __imp_?RemoveAt@CPtrArray@@QAEXHH@Z 5f58ebc0     MFC42D:MFC42D.DLL
 0002:00000bc4       __imp_??1CPtrArray@@UAE@XZ 5f58ebc4     MFC42D:MFC42D.DLL
 0002:00000bc8       __imp_??1CBitmap@@UAE@XZ   5f58ebc8     MFC42D:MFC42D.DLL
 0002:00000bcc       __imp_?Detach@CGdiObject@@QAEPAXXZ 5f58ebcc     MFC42D:MFC42D.DLL
 0002:00000bd0       __imp_?LoadBitmapA@CBitmap@@QAEHI@Z 5f58ebd0     MFC42D:MFC42D.DLL
 0002:00000bd4       __imp_??0CBitmap@@QAE@XZ   5f58ebd4     MFC42D:MFC42D.DLL
 0002:00000bd8       __imp_?GetSafeHandle@CGdiObject@@QBEPAXXZ 5f58ebd8     MFC42D:MFC42D.DLL
 0002:00000bdc       __imp_?LoadIconA@CWinApp@@QBEPAUHICON__@@I@Z 5f58ebdc     MFC42D:MFC42D.DLL
 0002:00000be0       __imp_??6@YGAAVCArchive@@AAV0@ABVCString@@@Z 5f58ebe0     MFC42D:MFC42D.DLL
 0002:00000be4       __imp_??5@YGAAVCArchive@@AAV0@AAVCString@@@Z 5f58ebe4     MFC42D:MFC42D.DLL
 0002:00000be8       __imp_?OnQuery3dControls@CWnd@@IAEJIJ@Z 5f58ebe8     MFC42D:MFC42D.DLL
 0002:00000bec       __imp_?messageMap@CDialog@@1UAFX_MSGMAP@@B 5f58ebec     MFC42D:MFC42D.DLL
 0002:00000bf0       __imp_?GetRuntimeClass@CObject@@UBEPAUCRuntimeClass@@XZ 5f58ebf0     MFC42D:MFC42D.DLL
 0002:00000bf4       __imp_??0CObject@@IAE@XZ   5f58ebf4     MFC42D:MFC42D.DLL
 0002:00000bf8       __imp_??1CObject@@UAE@XZ   5f58ebf8     MFC42D:MFC42D.DLL
 0002:00000bfc       __imp_?RemoveAll@CPtrArray@@QAEXXZ 5f58ebfc     MFC42D:MFC42D.DLL
 0002:00000c00       __imp_??ACPtrArray@@QAEAAPAXH@Z 5f58ec00     MFC42D:MFC42D.DLL
 0002:00000c04       __imp_?GetFont@CDialogTemplate@@QBEHAAVCString@@AAG@Z 5f58ec04     MFC42D:MFC42D.DLL
 0002:00000c08       __imp_?GetSizeInDialogUnits@CDialogTemplate@@QBEXPAUtagSIZE@@@Z 5f58ec08     MFC42D:MFC42D.DLL
 0002:00000c0c       __imp_?AddHead@CPtrList@@QAEPAU__POSITION@@PAX@Z 5f58ec0c     MFC42D:MFC42D.DLL
 0002:00000c10       __imp_?AfxEnableMemoryTracking@@YGHH@Z 5f58ec10     MFC42D:MFC42D.DLL
 0002:00000c14       __imp_?OnCancel@CDialog@@MAEXXZ 5f58ec14     MFC42D:MFC42D.DLL
 0002:00000c18       __imp_?OnOK@CDialog@@MAEXXZ 5f58ec18     MFC42D:MFC42D.DLL
 0002:00000c1c       __imp_??0CDialog@@QAE@XZ   5f58ec1c     MFC42D:MFC42D.DLL
 0002:00000c20       __imp_??1CDialogTemplate@@QAE@XZ 5f58ec20     MFC42D:MFC42D.DLL
 0002:00000c24       __imp_?Detach@CDialogTemplate@@QAEPAXXZ 5f58ec24     MFC42D:MFC42D.DLL
 0002:00000c28       __imp_?GetSizeInPixels@CDialogTemplate@@QBEXPAUtagSIZE@@@Z 5f58ec28     MFC42D:MFC42D.DLL
 0002:00000c2c       __imp_?SetFont@CDialogTemplate@@QAEHPBDG@Z 5f58ec2c     MFC42D:MFC42D.DLL
 0002:00000c30       __imp_?AfxGetPropSheetFont@@YGHAAVCString@@AAGH@Z 5f58ec30     MFC42D:MFC42D.DLL
 0002:00000c34       __imp_?HasFont@CDialogTemplate@@QBEHXZ 5f58ec34     MFC42D:MFC42D.DLL
 0002:00000c38       __imp_?Load@CDialogTemplate@@QAEHPBD@Z 5f58ec38     MFC42D:MFC42D.DLL
 0002:00000c3c       __imp_??0CDialogTemplate@@QAE@PBUDLGTEMPLATE@@@Z 5f58ec3c     MFC42D:MFC42D.DLL
 0002:00000c40       __imp_?GetCurrentMessage@CWnd@@KGPBUtagMSG@@XZ 5f58ec40     MFC42D:MFC42D.DLL
 0002:00000c44       __imp_?SendChildNotifyLastMsg@CWnd@@QAEHPAJ@Z 5f58ec44     MFC42D:MFC42D.DLL
 0002:00000c48       __imp_??0CDialogTemplate@@QAE@PAX@Z 5f58ec48     MFC42D:MFC42D.DLL
 0002:00000c4c       __imp_?UpdateData@CWnd@@QAEHH@Z 5f58ec4c     MFC42D:MFC42D.DLL
 0002:00000c50       __imp_?Create@CDialog@@QAEHIPAVCWnd@@@Z 5f58ec50     MFC42D:MFC42D.DLL
 0002:00000c54       __imp_?CreateIndirect@CDialog@@QAEHPAXPAVCWnd@@@Z 5f58ec54     MFC42D:MFC42D.DLL
 0002:00000c58       __imp_?GetWindow@CWnd@@QBEPAV1@I@Z 5f58ec58     MFC42D:MFC42D.DLL
 0002:00000c5c       __imp_?GotoDlgCtrl@CDialog@@QAEXPAVCWnd@@@Z 5f58ec5c     MFC42D:MFC42D.DLL
 0002:00000c60       __imp_?GetDefID@CDialog@@QBEKXZ 5f58ec60     MFC42D:MFC42D.DLL
 0002:00000c64       __imp_?GetAt@CDWordArray@@QBEKH@Z 5f58ec64     MFC42D:MFC42D.DLL
 0002:00000c68       __imp_??9@YG_NABVCString@@0@Z 5f58ec68     MFC42D:MFC42D.DLL
 0002:00000c6c       __imp_??6CArchive@@QAEAAV0@H@Z 5f58ec6c     MFC42D:MFC42D.DLL
 0002:00000c70       __imp_??6CArchive@@QAEAAV0@F@Z 5f58ec70     MFC42D:MFC42D.DLL
 0002:00000c74       __imp_??5CArchive@@QAEAAV0@AAH@Z 5f58ec74     MFC42D:MFC42D.DLL
 0002:00000c78       __imp_??5CArchive@@QAEAAV0@AAF@Z 5f58ec78     MFC42D:MFC42D.DLL
 0002:00000c7c       __imp_?GetAt@CStringArray@@QBE?AVCString@@H@Z 5f58ec7c     MFC42D:MFC42D.DLL
 0002:00000c80       __imp_??1CStringArray@@UAE@XZ 5f58ec80     MFC42D:MFC42D.DLL
 0002:00000c84       __imp_?GetSize@CStringArray@@QBEHXZ 5f58ec84     MFC42D:MFC42D.DLL
 0002:00000c88       __imp_??0CStringArray@@QAE@XZ 5f58ec88     MFC42D:MFC42D.DLL
 0002:00000c8c       __imp_?RemoveAll@CStringArray@@QAEXXZ 5f58ec8c     MFC42D:MFC42D.DLL
 0002:00000c90       __imp_?Add@CStringArray@@QAEHABVCString@@@Z 5f58ec90     MFC42D:MFC42D.DLL
 0002:00000c94       __imp_?SeekToEnd@CFile@@QAEKXZ 5f58ec94     MFC42D:MFC42D.DLL
 0002:00000c98       __imp_?Compare@CString@@QBEHPBD@Z 5f58ec98     MFC42D:MFC42D.DLL
 0002:00000c9c       __imp_?AfxDelRegTreeHelper@@YGJPAUHKEY__@@ABVCString@@@Z 5f58ec9c     MFC42D:MFC42D.DLL
 0002:00000ca0       __imp_?ReverseFind@CString@@QBEHD@Z 5f58eca0     MFC42D:MFC42D.DLL
 0002:00000ca4       __imp_??1CBrush@@UAE@XZ    5f58eca4     MFC42D:MFC42D.DLL
 0002:00000ca8       __imp_?FillRect@CDC@@QAEXPBUtagRECT@@PAVCBrush@@@Z 5f58eca8     MFC42D:MFC42D.DLL
 0002:00000cac       __imp_??0CBrush@@QAE@K@Z   5f58ecac     MFC42D:MFC42D.DLL
 0002:00000cb0       __imp_??9CRect@@QBEHABUtagRECT@@@Z 5f58ecb0     MFC42D:MFC42D.DLL
 0002:00000cb4       __imp_?GetHandleSize@CRectTracker@@MBEHPBUtagRECT@@@Z 5f58ecb4     MFC42D:MFC42D.DLL
 0002:00000cb8       __imp_?GetHandleMask@CRectTracker@@UBEIXZ 5f58ecb8     MFC42D:MFC42D.DLL
 0002:00000cbc       __imp_?OnChangedRect@CRectTracker@@UAEXABVCRect@@@Z 5f58ecbc     MFC42D:MFC42D.DLL
 0002:00000cc0       __imp_?AdjustRect@CRectTracker@@UAEXHPAUtagRECT@@@Z 5f58ecc0     MFC42D:MFC42D.DLL
 0002:00000cc4       __imp_?DrawTrackerRect@CRectTracker@@UAEXPBUtagRECT@@PAVCWnd@@PAVCDC@@1@Z 5f58ecc4     MFC42D:MFC42D.DLL
 0002:00000cc8       __imp_??0CRectTracker@@QAE@PBUtagRECT@@I@Z 5f58ecc8     MFC42D:MFC42D.DLL
 0002:00000ccc       __imp_?FromHandle@CDC@@SGPAV1@PAUHDC__@@@Z 5f58eccc     MFC42D:MFC42D.DLL
 0002:00000cd0       __imp_??1CMapStringToPtr@@UAE@XZ 5f58ecd0     MFC42D:MFC42D.DLL
 0002:00000cd4       __imp_??0CMapStringToPtr@@QAE@H@Z 5f58ecd4     MFC42D:MFC42D.DLL
 0002:00000cd8       __imp_?Lookup@CMapStringToPtr@@QBEHPBDAAPAX@Z 5f58ecd8     MFC42D:MFC42D.DLL
 0002:00000cdc       __imp_?MakeLower@CString@@QAEXXZ 5f58ecdc     MFC42D:MFC42D.DLL
 0002:00000ce0       __imp_?SetAt@CMapStringToPtr@@QAEXPBDPAX@Z 5f58ece0     MFC42D:MFC42D.DLL
 0002:00000ce4       __imp_?GetNextAssoc@CMapStringToPtr@@QBEXAAPAU__POSITION@@AAVCString@@AAPAX@Z 5f58ece4     MFC42D:MFC42D.DLL
 0002:00000ce8       __imp_?GetStartPosition@CMapStringToPtr@@QBEPAU__POSITION@@XZ 5f58ece8     MFC42D:MFC42D.DLL
 0002:00000cec       __imp_?GetCount@CMapStringToPtr@@QBEHXZ 5f58ecec     MFC42D:MFC42D.DLL
 0002:00000cf0       __imp_??1CThreadLocalObject@@QAE@XZ 5f58ecf0     MFC42D:MFC42D.DLL
 0002:00000cf4       __imp_?classCDC@CDC@@2UCRuntimeClass@@B 5f58ecf4     MFC42D:MFC42D.DLL
 0002:00000cf8       __imp_?Escape@CDC@@UAEHHHPBDPAX@Z 5f58ecf8     MFC42D:MFC42D.DLL
 0002:00000cfc       __imp_?GrayStringA@CDC@@UAEHPAVCBrush@@P6GHPAUHDC__@@JH@ZJHHHHH@Z 5f58ecfc     MFC42D:MFC42D.DLL
 0002:00000d00       __imp_?DrawTextA@CDC@@UAEHPBDHPAUtagRECT@@I@Z 5f58ed00     MFC42D:MFC42D.DLL
 0002:00000d04       __imp_?TabbedTextOutA@CDC@@UAE?AVCSize@@HHPBDHHPAHH@Z 5f58ed04     MFC42D:MFC42D.DLL
 0002:00000d08       __imp_?ExtTextOutA@CDC@@UAEHHHIPBUtagRECT@@PBDIPAH@Z 5f58ed08     MFC42D:MFC42D.DLL
 0002:00000d0c       __imp_?TextOutA@CDC@@UAEHHHPBDH@Z 5f58ed0c     MFC42D:MFC42D.DLL
 0002:00000d10       __imp_?RectVisible@CDC@@UBEHPBUtagRECT@@@Z 5f58ed10     MFC42D:MFC42D.DLL
 0002:00000d14       __imp_?PtVisible@CDC@@UBEHHH@Z 5f58ed14     MFC42D:MFC42D.DLL
 0002:00000d18       __imp_?GetClipBox@CDC@@UBEHPAUtagRECT@@@Z 5f58ed18     MFC42D:MFC42D.DLL
 0002:00000d1c       __imp_?ScaleWindowExt@CDC@@UAE?AVCSize@@HHHH@Z 5f58ed1c     MFC42D:MFC42D.DLL
 0002:00000d20       __imp_?ScaleViewportExt@CDC@@UAE?AVCSize@@HHHH@Z 5f58ed20     MFC42D:MFC42D.DLL
 0002:00000d24       __imp_?SetViewportExt@CDC@@UAE?AVCSize@@HH@Z 5f58ed24     MFC42D:MFC42D.DLL
 0002:00000d28       __imp_?OffsetViewportOrg@CDC@@UAE?AVCPoint@@HH@Z 5f58ed28     MFC42D:MFC42D.DLL
 0002:00000d2c       __imp_?SetViewportOrg@CDC@@UAE?AVCPoint@@HH@Z 5f58ed2c     MFC42D:MFC42D.DLL
 0002:00000d30       __imp_?SetTextColor@CDC@@UAEKK@Z 5f58ed30     MFC42D:MFC42D.DLL
 0002:00000d34       __imp_?SetBkColor@CDC@@UAEKK@Z 5f58ed34     MFC42D:MFC42D.DLL
 0002:00000d38       __imp_?SelectObject@CDC@@UAEPAVCFont@@PAV2@@Z 5f58ed38     MFC42D:MFC42D.DLL
 0002:00000d3c       __imp_?SelectStockObject@CDC@@UAEPAVCGdiObject@@H@Z 5f58ed3c     MFC42D:MFC42D.DLL
 0002:00000d40       __imp_?RestoreDC@CDC@@UAEHH@Z 5f58ed40     MFC42D:MFC42D.DLL
 0002:00000d44       __imp_?SaveDC@CDC@@UAEHXZ  5f58ed44     MFC42D:MFC42D.DLL
 0002:00000d48       __imp_?ReleaseOutputDC@CDC@@UAEXXZ 5f58ed48     MFC42D:MFC42D.DLL
 0002:00000d4c       __imp_?ReleaseAttribDC@CDC@@UAEXXZ 5f58ed4c     MFC42D:MFC42D.DLL
 0002:00000d50       __imp_?SetOutputDC@CDC@@UAEXPAUHDC__@@@Z 5f58ed50     MFC42D:MFC42D.DLL
 0002:00000d54       __imp_?SetAttribDC@CDC@@UAEXPAUHDC__@@@Z 5f58ed54     MFC42D:MFC42D.DLL
 0002:00000d58       __imp_?Dump@CDC@@UBEXAAVCDumpContext@@@Z 5f58ed58     MFC42D:MFC42D.DLL
 0002:00000d5c       __imp_?AssertValid@CDC@@UBEXXZ 5f58ed5c     MFC42D:MFC42D.DLL
 0002:00000d60       __imp_?SetViewportOrg@CDC@@QAE?AVCPoint@@UtagPOINT@@@Z 5f58ed60     MFC42D:MFC42D.DLL
 0002:00000d64       __imp_??HCPoint@@QBE?AV0@UtagPOINT@@@Z 5f58ed64     MFC42D:MFC42D.DLL
 0002:00000d68       __imp_?GetViewportOrg@CDC@@QBE?AVCPoint@@XZ 5f58ed68     MFC42D:MFC42D.DLL
 0002:00000d6c       __imp_?GetDC@CWnd@@QAEPAVCDC@@XZ 5f58ed6c     MFC42D:MFC42D.DLL
 0002:00000d70       __imp_?ReleaseDC@CWnd@@QAEHPAVCDC@@@Z 5f58ed70     MFC42D:MFC42D.DLL
 0002:00000d74       __imp_?InvalidateRgn@CWnd@@QAEXPAVCRgn@@H@Z 5f58ed74     MFC42D:MFC42D.DLL
 0002:00000d78       __imp_??1CRgn@@UAE@XZ      5f58ed78     MFC42D:MFC42D.DLL
 0002:00000d7c       __imp_??BCRgn@@QBEPAUHRGN__@@XZ 5f58ed7c     MFC42D:MFC42D.DLL
 0002:00000d80       __imp_?OffsetRgn@CRgn@@QAEHUtagPOINT@@@Z 5f58ed80     MFC42D:MFC42D.DLL
 0002:00000d84       __imp_?CopyRgn@CRgn@@QAEHPAV1@@Z 5f58ed84     MFC42D:MFC42D.DLL
 0002:00000d88       __imp_??0CRgn@@QAE@XZ      5f58ed88     MFC42D:MFC42D.DLL
 0002:00000d8c       __imp_?ScrollWindow@CWnd@@QAEXHHPBUtagRECT@@0@Z 5f58ed8c     MFC42D:MFC42D.DLL
 0002:00000d90       __imp_?OnChildNotify@CButton@@MAEHIIJPAJ@Z 5f58ed90     MFC42D:MFC42D.DLL
 0002:00000d94       __imp_?GetRuntimeClass@CButton@@UBEPAUCRuntimeClass@@XZ 5f58ed94     MFC42D:MFC42D.DLL
 0002:00000d98       __imp_??0CButton@@QAE@XZ   5f58ed98     MFC42D:MFC42D.DLL
 0002:00000d9c       __imp_??1CButton@@UAE@XZ   5f58ed9c     MFC42D:MFC42D.DLL
 0002:00000da0       __imp_?GetNearestColor@CDC@@QBEKK@Z 5f58eda0     MFC42D:MFC42D.DLL
 0002:00000da4       __imp_?GetState@CButton@@QBEIXZ 5f58eda4     MFC42D:MFC42D.DLL
 0002:00000da8       __imp_?RealizePalette@CDC@@QAEIXZ 5f58eda8     MFC42D:MFC42D.DLL
 0002:00000dac       __imp_?SelectPalette@CDC@@QAEPAVCPalette@@PAV2@H@Z 5f58edac     MFC42D:MFC42D.DLL
 0002:00000db0       __imp_?FromHandle@CPalette@@SGPAV1@PAUHPALETTE__@@@Z 5f58edb0     MFC42D:MFC42D.DLL
 0002:00000db4       __imp_??1CComboBox@@UAE@XZ 5f58edb4     MFC42D:MFC42D.DLL
 0002:00000db8       __imp_??0CComboBox@@QAE@XZ 5f58edb8     MFC42D:MFC42D.DLL
 0002:00000dbc       __imp_?SubclassDlgItem@CWnd@@QAEHIPAV1@@Z 5f58edbc     MFC42D:MFC42D.DLL
 0002:00000dc0       __imp_?SetCurSel@CComboBox@@QAEHH@Z 5f58edc0     MFC42D:MFC42D.DLL
 0002:00000dc4       __imp_?SetItemData@CComboBox@@QAEHHK@Z 5f58edc4     MFC42D:MFC42D.DLL
 0002:00000dc8       __imp_?AddString@CComboBox@@QAEHPBD@Z 5f58edc8     MFC42D:MFC42D.DLL
 0002:00000dcc       __imp_?GetCount@CComboBox@@QBEHXZ 5f58edcc     MFC42D:MFC42D.DLL
 0002:00000dd0       __imp_?GetItemData@CComboBox@@QBEKH@Z 5f58edd0     MFC42D:MFC42D.DLL
 0002:00000dd4       __imp_?GetCurSel@CComboBox@@QBEHXZ 5f58edd4     MFC42D:MFC42D.DLL
 0002:00000dd8       __imp_?DDX_Control@@YGXPAVCDataExchange@@HAAVCWnd@@@Z 5f58edd8     MFC42D:MFC42D.DLL
 0002:00000ddc       __imp_?LineTo@CDC@@QAEHHH@Z 5f58eddc     MFC42D:MFC42D.DLL
 0002:00000de0       __imp_?MoveTo@CDC@@QAE?AVCPoint@@HH@Z 5f58ede0     MFC42D:MFC42D.DLL
 0002:00000de4       __imp_?SelectObject@CDC@@QAEPAVCPen@@PAV2@@Z 5f58ede4     MFC42D:MFC42D.DLL
 0002:00000de8       __imp_??0CPen@@QAE@HHK@Z   5f58ede8     MFC42D:MFC42D.DLL
 0002:00000dec       __imp_?FrameRect@CDC@@QAEXPBUtagRECT@@PAVCBrush@@@Z 5f58edec     MFC42D:MFC42D.DLL
 0002:00000df0       __imp_??1CStatic@@UAE@XZ   5f58edf0     MFC42D:MFC42D.DLL
 0002:00000df4       __imp_??0CStatic@@QAE@XZ   5f58edf4     MFC42D:MFC42D.DLL
 0002:00000df8       __imp_?DeleteItem@CComboBox@@UAEXPAUtagDELETEITEMSTRUCT@@@Z 5f58edf8     MFC42D:MFC42D.DLL
 0002:00000dfc       __imp_?CompareItem@CComboBox@@UAEHPAUtagCOMPAREITEMSTRUCT@@@Z 5f58edfc     MFC42D:MFC42D.DLL
 0002:00000e00       __imp_?MeasureItem@CComboBox@@UAEXPAUtagMEASUREITEMSTRUCT@@@Z 5f58ee00     MFC42D:MFC42D.DLL
 0002:00000e04       __imp_?DrawItem@CComboBox@@UAEXPAUtagDRAWITEMSTRUCT@@@Z 5f58ee04     MFC42D:MFC42D.DLL
 0002:00000e08       __imp_?OnChildNotify@CComboBox@@MAEHIIJPAJ@Z 5f58ee08     MFC42D:MFC42D.DLL
 0002:00000e0c       __imp_?GetRuntimeClass@CComboBox@@UBEPAUCRuntimeClass@@XZ 5f58ee0c     MFC42D:MFC42D.DLL
 0002:00000e10       __imp_?BitBlt@CDC@@QAEHHHHHPAV1@HHK@Z 5f58ee10     MFC42D:MFC42D.DLL
 0002:00000e14       __imp_?SelectObject@CDC@@QAEPAVCBitmap@@PAV2@@Z 5f58ee14     MFC42D:MFC42D.DLL
 0002:00000e18       __imp_?CreateCompatibleDC@CDC@@QAEHPAV1@@Z 5f58ee18     MFC42D:MFC42D.DLL
 0002:00000e1c       __imp_?GetPixel@CDC@@QBEKHH@Z 5f58ee1c     MFC42D:MFC42D.DLL
 0002:00000e20       __imp_?CreateBitmap@CBitmap@@QAEHHHIIPBX@Z 5f58ee20     MFC42D:MFC42D.DLL
 0002:00000e24       __imp_?GetObjectA@CGdiObject@@QBEHHPAX@Z 5f58ee24     MFC42D:MFC42D.DLL
 0002:00000e28       __imp_?GetSafeHdc@CDC@@QBEPAUHDC__@@XZ 5f58ee28     MFC42D:MFC42D.DLL
 0002:00000e2c       __imp_?ResetContent@CComboBox@@QAEXXZ 5f58ee2c     MFC42D:MFC42D.DLL
 0002:00000e30       __imp_?SelectString@CComboBox@@QAEHHPBD@Z 5f58ee30     MFC42D:MFC42D.DLL
 0002:00000e34       __imp_?FindString@CComboBox@@QBEHHPBD@Z 5f58ee34     MFC42D:MFC42D.DLL
 0002:00000e38       __imp_?GetLBText@CComboBox@@QBEXHAAVCString@@@Z 5f58ee38     MFC42D:MFC42D.DLL
 0002:00000e3c       __imp_?DrawFocusRect@CDC@@QAEXPBUtagRECT@@@Z 5f58ee3c     MFC42D:MFC42D.DLL
 0002:00000e40       __imp_?GetTextMetricsA@CDC@@QBEHPAUtagTEXTMETRICA@@@Z 5f58ee40     MFC42D:MFC42D.DLL
 0002:00000e44       __imp_?InsertString@CComboBox@@QAEHHPBD@Z 5f58ee44     MFC42D:MFC42D.DLL
 0002:00000e48       __imp_?SetEditSel@CComboBox@@QAEHHH@Z 5f58ee48     MFC42D:MFC42D.DLL
 0002:00000e4c       __imp_?FindStringExact@CComboBox@@QBEHHPBD@Z 5f58ee4c     MFC42D:MFC42D.DLL
 0002:00000e50       __imp_?CreateFontIndirectA@CFont@@QAEHPBUtagLOGFONTA@@@Z 5f58ee50     MFC42D:MFC42D.DLL
 0002:00000e54       __imp_?DeleteObject@CGdiObject@@QAEHXZ 5f58ee54     MFC42D:MFC42D.DLL
 0002:00000e58       __imp_?GetTextExtent@CDC@@QBE?AVCSize@@PBDH@Z 5f58ee58     MFC42D:MFC42D.DLL
 0002:00000e5c       __imp_?SetBkMode@CDC@@QAEHH@Z 5f58ee5c     MFC42D:MFC42D.DLL
 0002:00000e60       __imp_?SetCheck@CButton@@QAEXH@Z 5f58ee60     MFC42D:MFC42D.DLL
 0002:00000e64       __imp_?GetCheck@CButton@@QBEHXZ 5f58ee64     MFC42D:MFC42D.DLL
 0002:00000e68       __imp_?GetStatus@CFile@@SGHPBDAAUCFileStatus@@@Z 5f58ee68     MFC42D:MFC42D.DLL
 0002:00000e6c       __imp_??0CTime@@QAE@XZ     5f58ee6c     MFC42D:MFC42D.DLL
 0002:00000e70       __imp_?GetPathName@CFileDialog@@QBE?AVCString@@XZ 5f58ee70     MFC42D:MFC42D.DLL
 0002:00000e74       __imp_?DoModal@CFileDialog@@UAEHXZ 5f58ee74     MFC42D:MFC42D.DLL
 0002:00000e78       __imp_??0CFileDialog@@QAE@HPBD0K0PAVCWnd@@@Z 5f58ee78     MFC42D:MFC42D.DLL
 0002:00000e7c       __imp_??0CMemFile@@QAE@I@Z 5f58ee7c     MFC42D:MFC42D.DLL
 0002:00000e80       __imp_?classCException@CException@@2UCRuntimeClass@@B 5f58ee80     MFC42D:MFC42D.DLL
 0002:00000e84       __imp_?Cut@CRichEditCtrl@@QAEXXZ 5f58ee84     MFC42D:MFC42D.DLL
 0002:00000e88       __imp_?Delete@CException@@QAEXXZ 5f58ee88     MFC42D:MFC42D.DLL
 0002:00000e8c       __imp_??0AFX_MAINTAIN_STATE2@@QAE@PAVAFX_MODULE_STATE@@@Z 5f58ee8c     MFC42D:MFC42D.DLL
 0002:00000e90       __imp_??1AFX_MAINTAIN_STATE2@@QAE@XZ 5f58ee90     MFC42D:MFC42D.DLL
 0002:00000e94       __imp_?AfxGetAppModuleState@@YGPAVAFX_MODULE_STATE@@XZ 5f58ee94     MFC42D:MFC42D.DLL
 0002:00000e98       __imp_??3CObject@@SGXPAX@Z 5f58ee98     MFC42D:MFC42D.DLL
 0002:00000e9c       __imp_?AfxInitExtensionModule@@YGHAAUAFX_EXTENSION_MODULE@@PAUHINSTANCE__@@@Z 5f58ee9c     MFC42D:MFC42D.DLL
 0002:00000ea0       __imp_?AfxCoreInitModule@@YGXXZ 5f58eea0     MFC42D:MFC42D.DLL
 0002:00000ea4       __imp_?AfxWinInit@@YGHPAUHINSTANCE__@@0PADH@Z 5f58eea4     MFC42D:MFC42D.DLL
 0002:00000ea8       __imp_??2CObject@@SGPAXI@Z 5f58eea8     MFC42D:MFC42D.DLL
 0002:00000eac       __imp_??0CDynLinkLibrary@@QAE@AAUAFX_EXTENSION_MODULE@@H@Z 5f58eeac     MFC42D:MFC42D.DLL
 0002:00000eb0       __imp_?AfxTermExtensionModule@@YGXAAUAFX_EXTENSION_MODULE@@H@Z 5f58eeb0     MFC42D:MFC42D.DLL
 0002:00000eb4       __imp_?AfxTermThread@@YGXPAUHINSTANCE__@@@Z 5f58eeb4     MFC42D:MFC42D.DLL
 0002:00000eb8       __imp_?AfxGetModuleState@@YGPAVAFX_MODULE_STATE@@XZ 5f58eeb8     MFC42D:MFC42D.DLL
 0002:00000ebc       __imp_?AfxGetThreadState@@YGPAV_AFX_THREAD_STATE@@XZ 5f58eebc     MFC42D:MFC42D.DLL
 0002:00000ec0       __imp_?AfxSetModuleState@@YGPAVAFX_MODULE_STATE@@PAV1@@Z 5f58eec0     MFC42D:MFC42D.DLL
 0002:00000ec4       __imp_?AfxGetApp@@YGPAVCWinApp@@XZ 5f58eec4     MFC42D:MFC42D.DLL
 0002:00000ec8       __imp_?OnCmdMsg@CCmdTarget@@UAEHIHPAXPAUAFX_CMDHANDLERINFO@@@Z 5f58eec8     MFC42D:MFC42D.DLL
 0002:00000ecc       __imp_?AfxAssertValidObject@@YGXPBVCObject@@PBDH@Z 5f58eecc     MFC42D:MFC42D.DLL
 0002:00000ed0       __imp_?AfxOleLockApp@@YGXXZ 5f58eed0     MFC42D:MFC42D.DLL
 0002:00000ed4       __imp_?GetDispatchIID@CCmdTarget@@UAEHPAU_GUID@@@Z 5f58eed4     MFC42D:MFC42D.DLL
 0002:00000ed8       __imp_?OnFinalRelease@CCmdTarget@@UAEXXZ 5f58eed8     MFC42D:MFC42D.DLL
 0002:00000edc       __imp_?IsInvokeAllowed@CCmdTarget@@UAEHJ@Z 5f58eedc     MFC42D:MFC42D.DLL
 0002:00000ee0       __imp_?GetTypeLib@CCmdTarget@@UAEJKPAPAUITypeLib@@@Z 5f58eee0     MFC42D:MFC42D.DLL
 0002:00000ee4       __imp_?GetTypeInfoCount@CCmdTarget@@UAEIXZ 5f58eee4     MFC42D:MFC42D.DLL
 0002:00000ee8       __imp_?GetTypeLibCache@CCmdTarget@@UAEPAVCTypeLibCache@@XZ 5f58eee8     MFC42D:MFC42D.DLL
 0002:00000eec       __imp_?GetDispatchMap@CCmdTarget@@MBEPBUAFX_DISPMAP@@XZ 5f58eeec     MFC42D:MFC42D.DLL
 0002:00000ef0       __imp_?GetMessageMap@CCmdTarget@@MBEPBUAFX_MSGMAP@@XZ 5f58eef0     MFC42D:MFC42D.DLL
 0002:00000ef4       __imp_?GetCommandMap@CCmdTarget@@MBEPBUAFX_OLECMDMAP@@XZ 5f58eef4     MFC42D:MFC42D.DLL
 0002:00000ef8       __imp_?OnCreateAggregates@CCmdTarget@@UAEHXZ 5f58eef8     MFC42D:MFC42D.DLL
 0002:00000efc       __imp_?GetConnectionMap@CCmdTarget@@MBEPBUAFX_CONNECTIONMAP@@XZ 5f58eefc     MFC42D:MFC42D.DLL
 0002:00000f00       __imp_?GetEventSinkMap@CCmdTarget@@MBEPBUAFX_EVENTSINKMAP@@XZ 5f58ef00     MFC42D:MFC42D.DLL
 0002:00000f04       __imp_?GetConnectionHook@CCmdTarget@@MAEPAUIConnectionPoint@@ABU_GUID@@@Z 5f58ef04     MFC42D:MFC42D.DLL
 0002:00000f08       __imp_?GetInterfaceHook@CCmdTarget@@UAEPAUIUnknown@@PBX@Z 5f58ef08     MFC42D:MFC42D.DLL
 0002:00000f0c       __imp_?GetExtraConnectionPoints@CCmdTarget@@MAEHPAVCPtrArray@@@Z 5f58ef0c     MFC42D:MFC42D.DLL
 0002:00000f10       __imp_?AfxGetThread@@YGPAVCWinThread@@XZ 5f58ef10     MFC42D:MFC42D.DLL
 0002:00000f14       __imp_?AfxOleSetUserCtrl@@YGXH@Z 5f58ef14     MFC42D:MFC42D.DLL
 0002:00000f18       __imp_?AfxTrace@@YAXPBDZZ  5f58ef18     MFC42D:MFC42D.DLL
 0002:00000f1c       __imp_??3CObject@@SGXPAXPBDH@Z 5f58ef1c     MFC42D:MFC42D.DLL
 0002:00000f20       __imp_??2CObject@@SGPAXIPBDH@Z 5f58ef20     MFC42D:MFC42D.DLL
 0002:00000f24       __imp_?AfxOleGetMessageFilter@@YGPAVCOleMessageFilter@@XZ 5f58ef24     MFC42D:MFC42D.DLL
 0002:00000f28       __imp_??1CDC@@UAE@XZ       5f58ef28     MFC42D:MFC42D.DLL
 0002:00000f2c       __imp_??1CView@@UAE@XZ     5f58ef2c     MFC42D:MFC42D.DLL
 0002:00000f30       __imp_??1CDWordArray@@UAE@XZ 5f58ef30     MFC42D:MFC42D.DLL
 0002:00000f34       __imp_??1CCmdTarget@@UAE@XZ 5f58ef34     MFC42D:MFC42D.DLL
 0002:00000f38       __imp_??1CString@@QAE@XZ   5f58ef38     MFC42D:MFC42D.DLL
 0002:00000f3c       __imp_??1CMemFile@@UAE@XZ  5f58ef3c     MFC42D:MFC42D.DLL
 0002:00000f40       __imp_??1AFX_MODULE_STATE@@UAE@XZ 5f58ef40     MFC42D:MFC42D.DLL
 0002:00000f44       __imp_??2@YAPAXI@Z         5f58ef44     MFC42D:MFC42D.DLL
 0002:00000f48       __imp_??3@YAXPAX@Z         5f58ef48     MFC42D:MFC42D.DLL
 0002:00000f4c       __imp_??1CWinApp@@UAE@XZ   5f58ef4c     MFC42D:MFC42D.DLL
 0002:00000f50       __imp_??0AFX_MODULE_STATE@@QAE@HP6GJPAUHWND__@@IIJ@ZKH@Z 5f58ef50     MFC42D:MFC42D.DLL
 0002:00000f54       __imp_?AfxWndProc@@YGJPAUHWND__@@IIJ@Z 5f58ef54     MFC42D:MFC42D.DLL
 0002:00000f58       __imp_?GetCharFormat@CFontDialog@@QBEXAAU_charformat@@@Z 5f58ef58     MFC42D:MFC42D.DLL
 0002:00000f5c       __imp_??0CWinApp@@QAE@PBD@Z 5f58ef5c     MFC42D:MFC42D.DLL
 0002:00000f60       __imp_?DoModal@CFontDialog@@UAEHXZ 5f58ef60     MFC42D:MFC42D.DLL
 0002:00000f64       __imp_?Copy@CRichEditCtrl@@QAEXXZ 5f58ef64     MFC42D:MFC42D.DLL
 0002:00000f68       __imp_?AssertValid@CWnd@@UBEXXZ 5f58ef68     MFC42D:MFC42D.DLL
 0002:00000f6c       \177MFC42D_NULL_THUNK_DATA 5f58ef6c     MFC42D:MFC42D.DLL
 0002:00000f70       __imp____CxxFrameHandler   5f58ef70     msvcrtd:MSVCRTD.dll
 0002:00000f74       __imp___adjust_fdiv        5f58ef74     msvcrtd:MSVCRTD.dll
 0002:00000f78       __imp___malloc_dbg         5f58ef78     msvcrtd:MSVCRTD.dll
 0002:00000f7c       __imp___initterm           5f58ef7c     msvcrtd:MSVCRTD.dll
 0002:00000f80       __imp___free_dbg           5f58ef80     msvcrtd:MSVCRTD.dll
 0002:00000f84       __imp_??1type_info@@UAE@XZ 5f58ef84     msvcrtd:MSVCRTD.dll
 0002:00000f88       __imp_?terminate@@YAXXZ    5f58ef88     msvcrtd:MSVCRTD.dll
 0002:00000f8c       __imp___except_handler3    5f58ef8c     msvcrtd:MSVCRTD.dll
 0002:00000f90       __imp___onexit             5f58ef90     msvcrtd:MSVCRTD.dll
 0002:00000f94       __imp____dllonexit         5f58ef94     msvcrtd:MSVCRTD.dll
 0002:00000f98       __imp___mbsrchr            5f58ef98     msvcrtd:MSVCRTD.dll
 0002:00000f9c       __imp__wcsncpy             5f58ef9c     msvcrtd:MSVCRTD.dll
 0002:00000fa0       __imp__wcscpy              5f58efa0     msvcrtd:MSVCRTD.dll
 0002:00000fa4       __imp___vsnprintf          5f58efa4     msvcrtd:MSVCRTD.dll
 0002:00000fa8       __imp___ltoa               5f58efa8     msvcrtd:MSVCRTD.dll
 0002:00000fac       __imp___ultoa              5f58efac     msvcrtd:MSVCRTD.dll
 0002:00000fb0       __imp___ismbcspace         5f58efb0     msvcrtd:MSVCRTD.dll
 0002:00000fb4       __imp___ismbcdigit         5f58efb4     msvcrtd:MSVCRTD.dll
 0002:00000fb8       __imp__strtol              5f58efb8     msvcrtd:MSVCRTD.dll
 0002:00000fbc       __imp__strtoul             5f58efbc     msvcrtd:MSVCRTD.dll
 0002:00000fc0       __imp__malloc              5f58efc0     msvcrtd:MSVCRTD.dll
 0002:00000fc4       __imp__swprintf            5f58efc4     msvcrtd:MSVCRTD.dll
 0002:00000fc8       __imp___itoa               5f58efc8     msvcrtd:MSVCRTD.dll
 0002:00000fcc       __imp__modf                5f58efcc     msvcrtd:MSVCRTD.dll
 0002:00000fd0       __imp__strftime            5f58efd0     msvcrtd:MSVCRTD.dll
 0002:00000fd4       __imp__localtime           5f58efd4     msvcrtd:MSVCRTD.dll
 0002:00000fd8       __imp__time                5f58efd8     msvcrtd:MSVCRTD.dll
 0002:00000fdc       __imp__ceil                5f58efdc     msvcrtd:MSVCRTD.dll
 0002:00000fe0       __imp__fabs                5f58efe0     msvcrtd:MSVCRTD.dll
 0002:00000fe4       __imp__floor               5f58efe4     msvcrtd:MSVCRTD.dll
 0002:00000fe8       __imp__labs                5f58efe8     msvcrtd:MSVCRTD.dll
 0002:00000fec       __imp___ftol               5f58efec     msvcrtd:MSVCRTD.dll
 0002:00000ff0       __imp___mbschr             5f58eff0     msvcrtd:MSVCRTD.dll
 0002:00000ff4       __imp__realloc             5f58eff4     msvcrtd:MSVCRTD.dll
 0002:00000ff8       __imp___strdup             5f58eff8     msvcrtd:MSVCRTD.dll
 0002:00000ffc       __imp__free                5f58effc     msvcrtd:MSVCRTD.dll
 0002:00001000       __imp___purecall           5f58f000     msvcrtd:MSVCRTD.dll
 0002:00001004       __imp___mbctype            5f58f004     msvcrtd:MSVCRTD.dll
 0002:00001008       __imp__memset              5f58f008     msvcrtd:MSVCRTD.dll
 0002:0000100c       __imp__wcslen              5f58f00c     msvcrtd:MSVCRTD.dll
 0002:00001010       __imp__memcpy              5f58f010     msvcrtd:MSVCRTD.dll
 0002:00001014       __imp___CxxThrowException@8 5f58f014     msvcrtd:MSVCRTD.dll
 0002:00001018       __imp___CrtDbgReport       5f58f018     msvcrtd:MSVCRTD.dll
 0002:0000101c       __imp__memcmp              5f58f01c     msvcrtd:MSVCRTD.dll
 0002:00001020       __imp___mbsinc             5f58f020     msvcrtd:MSVCRTD.dll
 0002:00001024       __imp__atol                5f58f024     msvcrtd:MSVCRTD.dll
 0002:00001028       __imp__memmove             5f58f028     msvcrtd:MSVCRTD.dll
 0002:0000102c       __imp___mbsnbcmp           5f58f02c     msvcrtd:MSVCRTD.dll
 0002:00001030       \177MSVCRTD_NULL_THUNK_DATA 5f58f030     msvcrtd:MSVCRTD.dll
 0002:00001034       __imp__CopyAcceleratorTableA@12 5f58f034     user32:USER32.dll
 0002:00001038       __imp__IsWindow@4          5f58f038     user32:USER32.dll
 0002:0000103c       __imp__CopyRect@8          5f58f03c     user32:USER32.dll
 0002:00001040       __imp__IsClipboardFormatAvailable@4 5f58f040     user32:USER32.dll
 0002:00001044       __imp__SendMessageA@16     5f58f044     user32:USER32.dll
 0002:00001048       __imp__EnableWindow@8      5f58f048     user32:USER32.dll
 0002:0000104c       __imp__wsprintfA           5f58f04c     user32:USER32.dll
 0002:00001050       __imp__GetActiveWindow@0   5f58f050     user32:USER32.dll
 0002:00001054       __imp__InSendMessage@0     5f58f054     user32:USER32.dll
 0002:00001058       __imp__ReleaseCapture@0    5f58f058     user32:USER32.dll
 0002:0000105c       __imp__PeekMessageA@20     5f58f05c     user32:USER32.dll
 0002:00001060       __imp__GetKeyState@4       5f58f060     user32:USER32.dll
 0002:00001064       __imp__GetCursorPos@4      5f58f064     user32:USER32.dll
 0002:00001068       __imp__DispatchMessageA@4  5f58f068     user32:USER32.dll
 0002:0000106c       __imp__PostThreadMessageA@16 5f58f06c     user32:USER32.dll
 0002:00001070       __imp__GetWindowTextA@12   5f58f070     user32:USER32.dll
 0002:00001074       __imp__GetWindowTextLengthA@4 5f58f074     user32:USER32.dll
 0002:00001078       __imp__IsMenu@4            5f58f078     user32:USER32.dll
 0002:0000107c       __imp__GetMenuItemID@8     5f58f07c     user32:USER32.dll
 0002:00001080       __imp__InsertMenuA@20      5f58f080     user32:USER32.dll
 0002:00001084       __imp__AppendMenuA@16      5f58f084     user32:USER32.dll
 0002:00001088       __imp__GetMenuStringA@20   5f58f088     user32:USER32.dll
 0002:0000108c       __imp__GetMenuState@12     5f58f08c     user32:USER32.dll
 0002:00001090       __imp__GetSubMenu@8        5f58f090     user32:USER32.dll
 0002:00001094       __imp__GetMenuItemCount@4  5f58f094     user32:USER32.dll
 0002:00001098       __imp__RemoveMenu@12       5f58f098     user32:USER32.dll
 0002:0000109c       __imp__ReleaseDC@8         5f58f09c     user32:USER32.dll
 0002:000010a0       __imp__WindowFromDC@4      5f58f0a0     user32:USER32.dll
 0002:000010a4       __imp__GetDC@4             5f58f0a4     user32:USER32.dll
 0002:000010a8       __imp__IsRectEmpty@4       5f58f0a8     user32:USER32.dll
 0002:000010ac       __imp__SetScrollRange@20   5f58f0ac     user32:USER32.dll
 0002:000010b0       __imp__SetFocus@4          5f58f0b0     user32:USER32.dll
 0002:000010b4       __imp__GetParent@4         5f58f0b4     user32:USER32.dll
 0002:000010b8       __imp__GetFocus@0          5f58f0b8     user32:USER32.dll
 0002:000010bc       __imp__DestroyIcon@4       5f58f0bc     user32:USER32.dll
 0002:000010c0       __imp__RegisterWindowMessageA@4 5f58f0c0     user32:USER32.dll
 0002:000010c4       __imp__CountClipboardFormats@0 5f58f0c4     user32:USER32.dll
 0002:000010c8       __imp__GetSystemMetrics@4  5f58f0c8     user32:USER32.dll
 0002:000010cc       __imp__RegisterClipboardFormatA@4 5f58f0cc     user32:USER32.dll
 0002:000010d0       __imp__GetWindowLongA@8    5f58f0d0     user32:USER32.dll
 0002:000010d4       __imp__AdjustWindowRectEx@16 5f58f0d4     user32:USER32.dll
 0002:000010d8       __imp__SetWindowContextHelpId@8 5f58f0d8     user32:USER32.dll
 0002:000010dc       __imp__GetWindow@8         5f58f0dc     user32:USER32.dll
 0002:000010e0       __imp__SetWindowPos@28     5f58f0e0     user32:USER32.dll
 0002:000010e4       __imp__MapDialogRect@8     5f58f0e4     user32:USER32.dll
 0002:000010e8       __imp__GetDlgItem@8        5f58f0e8     user32:USER32.dll
 0002:000010ec       __imp__CharNextA@4         5f58f0ec     user32:USER32.dll
 0002:000010f0       __imp__IsWindowVisible@4   5f58f0f0     user32:USER32.dll
 0002:000010f4       __imp__IsDialogMessageA@8  5f58f0f4     user32:USER32.dll
 0002:000010f8       __imp__GetDlgCtrlID@4      5f58f0f8     user32:USER32.dll
 0002:000010fc       __imp__ClipCursor@4        5f58f0fc     user32:USER32.dll
 0002:00001100       __imp__InflateRect@12      5f58f100     user32:USER32.dll
 0002:00001104       __imp__DestroyWindow@4     5f58f104     user32:USER32.dll
 0002:00001108       __imp__SetWindowLongA@12   5f58f108     user32:USER32.dll
 0002:0000110c       __imp__DefWindowProcA@16   5f58f10c     user32:USER32.dll
 0002:00001110       __imp__CallWindowProcA@20  5f58f110     user32:USER32.dll
 0002:00001114       __imp__SetParent@8         5f58f114     user32:USER32.dll
 0002:00001118       __imp__DrawEdge@16         5f58f118     user32:USER32.dll
 0002:0000111c       __imp__ShowWindow@8        5f58f11c     user32:USER32.dll
 0002:00001120       __imp__GetWindowRect@8     5f58f120     user32:USER32.dll
 0002:00001124       __imp__GetMenu@4           5f58f124     user32:USER32.dll
 0002:00001128       __imp__GetDesktopWindow@0  5f58f128     user32:USER32.dll
 0002:0000112c       __imp__PostMessageA@16     5f58f12c     user32:USER32.dll
 0002:00001130       __imp__GetClassNameA@12    5f58f130     user32:USER32.dll
 0002:00001134       __imp__IsChild@8           5f58f134     user32:USER32.dll
 0002:00001138       __imp__IntersectRect@12    5f58f138     user32:USER32.dll
 0002:0000113c       __imp__ScreenToClient@8    5f58f13c     user32:USER32.dll
 0002:00001140       __imp__MessageBoxA@16      5f58f140     user32:USER32.dll
 0002:00001144       __imp__EnumChildWindows@12 5f58f144     user32:USER32.dll
 0002:00001148       __imp__LockWindowUpdate@4  5f58f148     user32:USER32.dll
 0002:0000114c       __imp__GetSysColor@4       5f58f14c     user32:USER32.dll
 0002:00001150       __imp__SetCursor@4         5f58f150     user32:USER32.dll
 0002:00001154       __imp__LoadCursorA@8       5f58f154     user32:USER32.dll
 0002:00001158       __imp__PtInRect@12         5f58f158     user32:USER32.dll
 0002:0000115c       __imp__SetRectEmpty@4      5f58f15c     user32:USER32.dll
 0002:00001160       __imp__OffsetRect@12       5f58f160     user32:USER32.dll
 0002:00001164       __imp__GetDialogBaseUnits@0 5f58f164     user32:USER32.dll
 0002:00001168       __imp__MessageBeep@4       5f58f168     user32:USER32.dll
 0002:0000116c       __imp__DestroyMenu@4       5f58f16c     user32:USER32.dll
 0002:00001170       __imp__CreateMenu@0        5f58f170     user32:USER32.dll
 0002:00001174       \177USER32_NULL_THUNK_DATA 5f58f174     user32:USER32.dll
 0002:000011a0       _IID_IDocHostUIHandlerDispatch 5f58f1a0     dllole.obj
 0002:000011b0       _IID_IInternalConnection   5f58f1b0     dllole.obj
 0002:000011c0       _IID_IAxWinAmbientDispatch 5f58f1c0     dllole.obj
 0002:000011d0       _IID_IAxWinHostWindow      5f58f1d0     dllole.obj
 0002:000011e0       _IID_IRegistrar            5f58f1e0     dllole.obj
 0002:000011f0       _CLSID_Registrar           5f58f1f0     dllole.obj
 0002:00001200       _LIBID_ATLLib              5f58f200     dllole.obj
 0002:00001210       ??_C@_0L@LDKI@MFC42D?4DLL?$AA@ 5f58f210     dllole.obj
 0002:0000121c       ??_C@_00A@?$AA@            5f58f21c     dllole.obj
 0002:00001220       ??_C@_0BK@CHHF@RichEdit?5Text?5and?5Objects?$AA@ 5f58f220     oleinit.obj
 0002:0000123c       ??_C@_0BB@HIML@Rich?5Text?5Format?$AA@ 5f58f23c     oleinit.obj
 0002:00001250       ??_C@_09IKIM@FileNameW?$AA@ 5f58f250     oleinit.obj
 0002:0000125c       ??_C@_08NJLM@FileName?$AA@ 5f58f25c     oleinit.obj
 0002:00001268       ??_C@_0BH@FOOO@Link?5Source?5Descriptor?$AA@ 5f58f268     oleinit.obj
 0002:00001280       ??_C@_0BC@GMEI@Object?5Descriptor?$AA@ 5f58f280     oleinit.obj
 0002:00001294       ??_C@_0M@KPGD@Link?5Source?$AA@ 5f58f294     oleinit.obj
 0002:000012a0       ??_C@_0N@LHIH@Embed?5Source?$AA@ 5f58f2a0     oleinit.obj
 0002:000012b0       ??_C@_0BA@IEJA@Embedded?5Object?$AA@ 5f58f2b0     oleinit.obj
 0002:000012c0       ??_C@_0L@KADP@ObjectLink?$AA@ 5f58f2c0     oleinit.obj
 0002:000012cc       ??_C@_09NJ@OwnerLink?$AA@  5f58f2cc     oleinit.obj
 0002:000012d8       ??_C@_06LLCL@Native?$AA@   5f58f2d8     oleinit.obj
 0002:000012e0       ??_C@_0CN@JJKE@Warning?3?5OleInitialize?5returned?5@ 5f58f2e0     oleinit.obj
 0002:00001310       ??_C@_09LHIP@Embedding?$AA@ 5f58f310     oleinit.obj
 0002:0000131c       ??_C@_0L@POJA@Automation?$AA@ 5f58f31c     oleinit.obj
 0002:00001328       ?classCOleLinkingDoc@COleLinkingDoc@@2UCRuntimeClass@@B 5f58f328     olecli1.obj
 0002:00001340       ??_C@_0P@EIOM@COleLinkingDoc?$AA@ 5f58f340     olecli1.obj
 0002:00001350       ?interfaceMap@COleClientItem@@1UAFX_INTERFACEMAP@@B 5f58f350     olecli1.obj
 0002:00001358       ?_interfaceEntries@COleClientItem@@0QBUAFX_INTERFACEMAP_ENTRY@@B 5f58f358     olecli1.obj
 0002:00001384       ??_7COleClientItem@@6B@    5f58f384     olecli1.obj
 0002:00001470       ??_7XOleClientSite@COleClientItem@@6B@ 5f58f470     olecli1.obj
 0002:00001498       ??_7XAdviseSink@COleClientItem@@6B@ 5f58f498     olecli1.obj
 0002:000014bc       ??_7XOleIPSite@COleClientItem@@6B@ 5f58f4bc     olecli1.obj
 0002:000014f8       ??_C@_0O@COMH@Embedding?5?$CFlu?$AA@ 5f58f4f8     olecli1.obj
 0002:00001508       ??_C@_0M@GLOE@DocShortcut?$AA@ 5f58f508     olecli1.obj
 0002:00001514       ??_C@_0M@JONA@DefaultIcon?$AA@ 5f58f514     olecli1.obj
 0002:00001520       ??_C@_05DNNF@clsid?$AA@    5f58f520     olecli1.obj
 0002:00001528       ??_C@_08NDGO@lpw?5?$CB?$DN?50?$AA@ 5f58f528     olecli1.obj
 0002:00001534       ??_C@_0CH@IIKL@E?3?28168?2vc98?2mfc?2atl?2include?2atl@ 5f58f534     olecli1.obj
 0002:0000155c       ??_C@_08PEKM@lpa?5?$CB?$DN?50?$AA@ 5f58f55c     olecli1.obj
 0002:00001568       ??_C@_0CN@MKCO@Warning?3?5unable?5to?5create?5child?5@ 5f58f568     olecli1.obj
 0002:00001598       ??_C@_02DILL@?$CFs?$AA@    5f58f598     olecli1.obj
 0002:0000159c       ??_C@_0EA@BHCI@Warning?5OnNewDocument?5failed?5dur@ 5f58f59c     olecli1.obj
 0002:000015dc       ??_C@_0CL@NAHC@Warning?3?5unable?5to?5open?5child?5st@ 5f58f5dc     olecli1.obj
 0002:00001608       ??_C@_0DH@LDBM@Warning?3?5object?5does?5not?5support@ 5f58f608     olecli1.obj
 0002:00001640       ??_C@_0DC@MPHG@Warning?3?5unable?5to?5get?5moniker?5f@ 5f58f640     olecli1.obj
 0002:00001674       ??_C@_0DC@DPDJ@Warning?3?5unable?5to?5get?5moniker?5f@ 5f58f674     olecli1.obj
 0002:000016a8       ??_C@_13HMCP@?$AA?2?$AA?$AA@ 5f58f6a8     olecli1.obj
 0002:000016ac       ??_C@_0BB@JMCJ@?6m_hWndServer?5?$DN?5?$AA@ 5f58f6ac     olecli1.obj
 0002:000016c0       ??_C@_0BE@DEMF@?6m_pInPlaceFrame?5?$DN?5?$AA@ 5f58f6c0     olecli1.obj
 0002:000016d4       ??_C@_0BH@JIDM@?6m_dwContainerStyle?5?$DN?5?$AA@ 5f58f6d4     olecli1.obj
 0002:000016ec       ??_C@_0M@EFKC@?6m_pView?5?$DN?5?$AA@ 5f58f6ec     olecli1.obj
 0002:000016f8       ??_C@_0BB@JNMD@?6m_nItemState?5?$DN?5?$AA@ 5f58f6f8     olecli1.obj
 0002:0000170c       ??_C@_0BC@CJ@?6m_bNeedCommit?5?$DN?5?$AA@ 5f58f70c     olecli1.obj
 0002:00001720       ??_C@_0BD@DFML@?6m_lpNewStorage?5?$DN?5?$AA@ 5f58f720     olecli1.obj
 0002:00001734       ??_C@_0P@HJAA@?6m_bMoniker?5?$DN?5?$AA@ 5f58f734     olecli1.obj
 0002:00001744       ??_C@_0BD@CALL@?6m_bLinkUnavail?5?$DN?5?$AA@ 5f58f744     olecli1.obj
 0002:00001758       ??_C@_0BD@DPMG@?6m_dwConnection?5?$DN?5?$AA@ 5f58f758     olecli1.obj
 0002:0000176c       ??_C@_0BC@DIDM@?6m_lpLockBytes?5?$DN?5?$AA@ 5f58f76c     olecli1.obj
 0002:00001780       ??_C@_0BA@LKEM@?6m_lpStorage?5?$DN?5?$AA@ 5f58f780     olecli1.obj
 0002:00001790       ??_C@_0N@EFDC@?6m_scLast?5?$DN?5?$AA@ 5f58f790     olecli1.obj
 0002:000017a0       ??_C@_0BC@DBNB@?6m_nDrawAspect?5?$DN?5?$AA@ 5f58f7a0     olecli1.obj
 0002:000017b4       ??_C@_0BD@MOJB@?6m_dwItemNumber?5?$DN?5?$AA@ 5f58f7b4     olecli1.obj
 0002:000017c8       ??_C@_0O@EOEE@m_lpObject?5?$DN?5?$AA@ 5f58f7c8     olecli1.obj
 0002:000017d8       ?interfaceMap@COleFrameHook@@1UAFX_INTERFACEMAP@@B 5f58f7d8     olecli2.obj
 0002:000017e0       ?_interfaceEntries@COleFrameHook@@0QBUAFX_INTERFACEMAP_ENTRY@@B 5f58f7e0     olecli2.obj
 0002:00001804       ??_7COleFrameHook@@6B@     5f58f804     olecli2.obj
 0002:00001890       ??_7XOleInPlaceFrame@COleFrameHook@@6B@ 5f58f890     olecli2.obj
 0002:000018d0       ??_7XOleCommandTarget@COleFrameHook@@6B@ 5f58f8d0     olecli2.obj
 0002:000018e4       ??_C@_0CH@KFAI@E?3?28168?2vc98?2mfc?2mfc?2include?2afx@ 5f58f8e4     olecli2.obj
 0002:0000190c       ??_C@_0CJ@LLBM@Warning?3?5operation?5returned?5scod@ 5f58f90c     olecli3.obj
 0002:00001938       ?interfaceMap@COleDataSource@@1UAFX_INTERFACEMAP@@B 5f58f938     oledobj2.obj
 0002:00001940       ?_interfaceEntries@COleDataSource@@0QBUAFX_INTERFACEMAP_ENTRY@@B 5f58f940     oledobj2.obj
 0002:00001950       ?interfaceMap@CEnumFormatEtc@@1UAFX_INTERFACEMAP@@B 5f58f950     oledobj2.obj
 0002:00001958       ?_interfaceEntries@CEnumFormatEtc@@0QBUAFX_INTERFACEMAP_ENTRY@@B 5f58f958     oledobj2.obj
 0002:0000196c       ??_7COleDataSource@@6B@    5f58f96c     oledobj2.obj
 0002:000019d8       ??_7XDataObject@COleDataSource@@6B@ 5f58f9d8     oledobj2.obj
 0002:00001a0c       ??_7CEnumFormatEtc@@6B@    5f58fa0c     oledobj2.obj
 0002:00001a74       ??_C@_01BJG@?6?$AA@        5f58fa74     oledobj2.obj
 0002:00001a78       ??_C@_03JNEF@?6?7?$HN?$AA@ 5f58fa78     oledobj2.obj
 0002:00001a7c       ??_C@_0BB@GMOB@?6?7?5m_nDataDir?5?$DN?5?$AA@ 5f58fa7c     oledobj2.obj
 0002:00001a90       ??_C@_0BI@PNP@?6?7?5m_stgMedium?4tymed?5?$DN?5?$AA@ 5f58fa90     oledobj2.obj
 0002:00001aa8       ??_C@_0BI@EFAF@?6?7?5m_formatEtc?4tymed?5?$DN?5?$AA@ 5f58faa8     oledobj2.obj
 0002:00001ac0       ??_C@_0BJ@LPOO@?6?7?5m_formatEtc?4lindex?5?$DN?5?$AA@ 5f58fac0     oledobj2.obj
 0002:00001adc       ??_C@_0BL@HFLA@?6?7?5m_formatEtc?4dwAspect?5?$DN?5?$AA@ 5f58fadc     oledobj2.obj
 0002:00001af8       ??_C@_0BG@LHAO@?6?7?5m_formatEtc?4pdt?5?$DN?5?$AA@ 5f58faf8     oledobj2.obj
 0002:00001b10       ??_C@_0BL@IPEG@?6?7?5m_formatEtc?4cfFormat?5?$DN?5?$AA@ 5f58fb10     oledobj2.obj
 0002:00001b2c       ??_C@_09EIHB@?6?7entry?5?$FL?$AA@ 5f58fb2c     oledobj2.obj
 0002:00001b38       ??_C@_05EJJM@?$FN?5?$DN?5?$HL?$AA@ 5f58fb38     oledobj2.obj
 0002:00001b40       ??_C@_0BB@IFBL@?6m_pDataCache?5?$DN?5?$AA@ 5f58fb40     oledobj2.obj
 0002:00001b54       ??_C@_0M@NOBL@?6m_nSize?5?$DN?5?$AA@ 5f58fb54     oledobj2.obj
 0002:00001b60       ??_C@_0O@JNKF@m_nMaxSize?5?$DN?5?$AA@ 5f58fb60     oledobj2.obj
 0002:00001b70       ?classCOleDispatchException@COleDispatchException@@2UCRuntimeClass@@B 5f58fb70     oledisp1.obj
 0002:00001b88       ??_C@_0BG@OGI@COleDispatchException?$AA@ 5f58fb88     oledisp1.obj
 0002:00001ba0       ?_afxRetVal@@3QBIB         5f58fba0     oledisp1.obj
 0002:00001bdc       ?_afxByRef@@3QBIB          5f58fbdc     oledisp1.obj
 0002:00001c18       ?_afxByValue@@3QBIB        5f58fc18     oledisp1.obj
 0002:00001c54       ??_C@_0CP@MIP@Warning?3?5automation?5property?5coe@ 5f58fc54     oledisp1.obj
 0002:00001c88       ??_7COleDispatchImpl@@6B@  5f58fc88     oledisp1.obj
 0002:00001ca8       ??_C@_0CP@OPOA@Warning?3?5automation?5argument?5coe@ 5f58fca8     oledisp1.obj
 0002:00001cd8       ??_C@_0CN@BHMH@Error?3?5stack?5overflow?5in?5IDispat@ 5f58fcd8     oledisp1.obj
 0002:00001d0c       ??_7COleDispatchException@@6B@ 5f58fd0c     oledisp1.obj
 0002:00001d28       ??_C@_0CP@DOIF@Warning?3?5CreateDispatch?5returnin@ 5f58fd28     oledisp2.obj
 0002:00001d58       ??_C@_0DD@MKKH@Warning?3?5automation?5return?5value@ 5f58fd58     oledisp2.obj
 0002:00001d8c       ??_C@_0DJ@LJMD@Warning?3?5attempt?5to?5call?5Invoke?5@ 5f58fd8c     oledisp2.obj
 0002:00001dc8       ?classCOlePasteSpecialDialog@COlePasteSpecialDialog@@2UCRuntimeClass@@B 5f58fdc8     oledlgs1.obj
 0002:00001de0       ??_C@_0BH@NAFF@COlePasteSpecialDialog?$AA@ 5f58fde0     oledlgs1.obj
 0002:00001df8       ?classCOleUpdateDialog@COleUpdateDialog@@2UCRuntimeClass@@B 5f58fdf8     oledlgs1.obj
 0002:00001e10       ??_C@_0BB@HGD@COleUpdateDialog?$AA@ 5f58fe10     oledlgs1.obj
 0002:00001e28       ?classCOleLinksDialog@COleLinksDialog@@2UCRuntimeClass@@B 5f58fe28     oledlgs1.obj
 0002:00001e40       ??_C@_0BA@PIHM@COleLinksDialog?$AA@ 5f58fe40     oledlgs1.obj
 0002:00001e50       ?classCOleChangeIconDialog@COleChangeIconDialog@@2UCRuntimeClass@@B 5f58fe50     oledlgs1.obj
 0002:00001e68       ??_C@_0BF@JMPM@COleChangeIconDialog?$AA@ 5f58fe68     oledlgs1.obj
 0002:00001e80       ?classCOleConvertDialog@COleConvertDialog@@2UCRuntimeClass@@B 5f58fe80     oledlgs1.obj
 0002:00001e98       ??_C@_0BC@CIPN@COleConvertDialog?$AA@ 5f58fe98     oledlgs1.obj
 0002:00001eb0       ?classCOleInsertDialog@COleInsertDialog@@2UCRuntimeClass@@B 5f58feb0     oledlgs1.obj
 0002:00001ec8       ??_C@_0BB@KPPE@COleInsertDialog?$AA@ 5f58fec8     oledlgs1.obj
 0002:00001ee0       ??_7COleUILinkInfo@@6B@    5f58fee0     oledlgs1.obj
 0002:00001f14       ??_7IOleUILinkInfoA@@6B@   5f58ff14     oledlgs1.obj
 0002:00001f48       ??_7IOleUILinkContainerA@@6B@ 5f58ff48     oledlgs1.obj
 0002:00001f78       ??_7COleInsertDialog@@6B@  5f58ff78     oledlgs1.obj
 0002:00002050       ??_C@_0BD@KJLP@CLSID?2?$CFs?2DocObject?$AA@ 5f590050     oledlgs1.obj
 0002:00002064       ??_C@_09LLJL@DocObject?$AA@ 5f590064     oledlgs1.obj
 0002:00002070       ??_C@_09IKLH@Ole1Class?$AA@ 5f590070     oledlgs1.obj
 0002:0000207c       ??_C@_0L@PBL@Insertable?$AA@ 5f59007c     oledlgs1.obj
 0002:00002088       ??_C@_05FGFK@CLSID?$AA@    5f590088     oledlgs1.obj
 0002:00002090       ??_C@_0DF@IHKK@Warning?3?5failed?5to?5set?5iconic?5as@ 5f590090     oledlgs1.obj
 0002:000020c8       ??_C@_0BD@CHHM@?6m_io?4hMetaPict?5?$DN?5?$AA@ 5f5900c8     oledlgs1.obj
 0002:000020dc       ??_C@_0DB@BLDH@?6hook?5function?5set?5to?5non?9standa@ 5f5900dc     oledlgs1.obj
 0002:00002110       ??_C@_0DB@MAOJ@?6hook?5function?5set?5to?5standard?5M@ 5f590110     oledlgs1.obj
 0002:00002144       ??_C@_0BD@IPNN@?6m_io?4hResource?5?$DN?5?$AA@ 5f590144     oledlgs1.obj
 0002:00002158       ??_C@_0BG@EDJJ@?6m_io?4lpszTemplate?5?$DN?5?$AA@ 5f590158     oledlgs1.obj
 0002:00002170       ??_C@_0BD@ELPK@?6m_io?4hInstance?5?$DN?5?$AA@ 5f590170     oledlgs1.obj
 0002:00002184       ??_C@_0BD@JLLA@?6m_io?4lCustData?5?$DN?5?$AA@ 5f590184     oledlgs1.obj
 0002:00002198       ??_C@_0BF@PECB@?6m_io?4lpszCaption?5?$DN?5?$AA@ 5f590198     oledlgs1.obj
 0002:000021b0       ??_C@_0BD@NMHJ@?6m_io?4hWndOwner?5?$DN?5?$AA@ 5f5901b0     oledlgs1.obj
 0002:000021c4       ??_C@_0BB@FCGN@?6m_io?4dwFlags?5?$DN?5?$AA@ 5f5901c4     oledlgs1.obj
 0002:000021d8       ??_C@_0BC@LPPE@?6m_io?4cbStruct?5?$DN?5?$AA@ 5f5901d8     oledlgs1.obj
 0002:000021ec       ??_C@_0BA@KFFI@m_szFileName?5?$DN?5?$AA@ 5f5901ec     oledlgs1.obj
 0002:00002200       ??_7COleConvertDialog@@6B@ 5f590200     oledlgs1.obj
 0002:000022d8       ??_C@_0BN@NCPK@?6m_cv?4fObjectsIconChanged?5?$DN?5?$AA@ 5f5902d8     oledlgs1.obj
 0002:000022f8       ??_C@_0BG@FMAM@?6m_cv?4lpszUserType?5?$DN?5?$AA@ 5f5902f8     oledlgs1.obj
 0002:00002310       ??_C@_0BD@BAPC@?6m_cv?4hMetaPict?5?$DN?5?$AA@ 5f590310     oledlgs1.obj
 0002:00002324       ??_C@_0BJ@PDJL@?6m_cv?4fIsLinkedObject?5?$DN?5?$AA@ 5f590324     oledlgs1.obj
 0002:00002340       ??_C@_0BB@NDIA@?6m_cv?4wFormat?5?$DN?5?$AA@ 5f590340     oledlgs1.obj
 0002:00002354       ??_C@_0BC@DIHB@?6m_cv?4dvAspect?5?$DN?5?$AA@ 5f590354     oledlgs1.obj
 0002:00002368       ??_C@_0BD@LIFD@?6m_cv?4hResource?5?$DN?5?$AA@ 5f590368     oledlgs1.obj
 0002:0000237c       ??_C@_0BG@NAOD@?6m_cv?4lpszTemplate?5?$DN?5?$AA@ 5f59037c     oledlgs1.obj
 0002:00002394       ??_C@_0BD@HMHE@?6m_cv?4hInstance?5?$DN?5?$AA@ 5f590394     oledlgs1.obj
 0002:000023a8       ??_C@_0BD@KMDO@?6m_cv?4lCustData?5?$DN?5?$AA@ 5f5903a8     oledlgs1.obj
 0002:000023bc       ??_C@_0BF@IOJB@?6m_cv?4lpszCaption?5?$DN?5?$AA@ 5f5903bc     oledlgs1.obj
 0002:000023d4       ??_C@_0BD@OLPH@?6m_cv?4hWndOwner?5?$DN?5?$AA@ 5f5903d4     oledlgs1.obj
 0002:000023e8       ??_C@_0BB@KHMP@?6m_cv?4dwFlags?5?$DN?5?$AA@ 5f5903e8     oledlgs1.obj
 0002:000023fc       ??_C@_0BB@HIEM@m_cv?4cbStruct?5?$DN?5?$AA@ 5f5903fc     oledlgs1.obj
 0002:00002414       ??_7COleChangeIconDialog@@6B@ 5f590414     oledlgs1.obj
 0002:000024ec       ??_C@_0BD@HGNJ@?6m_ci?4hMetaPict?5?$DN?5?$AA@ 5f5904ec     oledlgs1.obj
 0002:00002500       ??_C@_0BD@NOHI@?6m_ci?4hResource?5?$DN?5?$AA@ 5f590500     oledlgs1.obj
 0002:00002514       ??_C@_0BG@PPBE@?6m_ci?4lpszTemplate?5?$DN?5?$AA@ 5f590514     oledlgs1.obj
 0002:0000252c       ??_C@_0BD@BKFP@?6m_ci?4hInstance?5?$DN?5?$AA@ 5f59052c     oledlgs1.obj
 0002:00002540       ??_C@_0BD@MKBF@?6m_ci?4lCustData?5?$DN?5?$AA@ 5f590540     oledlgs1.obj
 0002:00002554       ??_C@_0BF@HJOD@?6m_ci?4lpszCaption?5?$DN?5?$AA@ 5f590554     oledlgs1.obj
 0002:0000256c       ??_C@_0BD@INNM@?6m_ci?4hWndOwner?5?$DN?5?$AA@ 5f59056c     oledlgs1.obj
 0002:00002580       ??_C@_0BB@BHKG@?6m_ci?4dwFlags?5?$DN?5?$AA@ 5f590580     oledlgs1.obj
 0002:00002594       ??_C@_0BB@FDPM@m_ci?4cbStruct?5?$DN?5?$AA@ 5f590594     oledlgs1.obj
 0002:000025ac       ??_7COleLinksDialog@@6B@   5f5905ac     oledlgs1.obj
 0002:00002684       ??_C@_0BD@HAKN@?6m_el?4hResource?5?$DN?5?$AA@ 5f590684     oledlgs1.obj
 0002:00002698       ??_C@_0BG@KHIK@?6m_el?4lpszTemplate?5?$DN?5?$AA@ 5f590698     oledlgs1.obj
 0002:000026b0       ??_C@_0BD@LEIK@?6m_el?4hInstance?5?$DN?5?$AA@ 5f5906b0     oledlgs1.obj
 0002:000026c4       ??_C@_0BD@GEMA@?6m_el?4lCustData?5?$DN?5?$AA@ 5f5906c4     oledlgs1.obj
 0002:000026d8       ??_C@_0BF@OHOP@?6m_el?4lpszCaption?5?$DN?5?$AA@ 5f5906d8     oledlgs1.obj
 0002:000026f0       ??_C@_0BD@CDAJ@?6m_el?4hWndOwner?5?$DN?5?$AA@ 5f5906f0     oledlgs1.obj
 0002:00002704       ??_C@_0BB@CKIK@?6m_el?4dwFlags?5?$DN?5?$AA@ 5f590704     oledlgs1.obj
 0002:00002718       ??_C@_0BC@MPIM@?6m_el?4cbStruct?5?$DN?5?$AA@ 5f590718     oledlgs1.obj
 0002:00002730       ??_7COleUpdateDialog@@6B@  5f590730     oledlgs1.obj
 0002:00002808       ??_C@_0BA@OFIG@m_strCaption?5?$DN?5?$AA@ 5f590808     oledlgs1.obj
 0002:0000281c       ??_7COlePasteSpecialDialog@@6B@ 5f59081c     oledlgs1.obj
 0002:000028f4       ??_C@_0P@JJLH@?6m_ps?4fLink?5?$DN?5?$AA@ 5f5908f4     oledlgs1.obj
 0002:00002904       ??_C@_0BI@PHBO@?6m_ps?4nSelectedIndex?5?$DN?5?$AA@ 5f590904     oledlgs1.obj
 0002:0000291c       ??_C@_0BE@OPOD@?6m_ps?4cLinkTypes?5?$DN?5?$AA@ 5f59091c     oledlgs1.obj
 0002:00002930       ??_C@_0BH@IOIO@?6m_ps?4cPasteEntries?5?$DN?5?$AA@ 5f590930     oledlgs1.obj
 0002:00002948       ??_C@_0BG@GBAG@?6m_ps?4lpSrcDataObj?5?$DN?5?$AA@ 5f590948     oledlgs1.obj
 0002:00002960       ??_C@_0BD@PEKC@?6m_ps?4hResource?5?$DN?5?$AA@ 5f590960     oledlgs1.obj
 0002:00002974       ??_C@_0BG@JFBL@?6m_ps?4lpszTemplate?5?$DN?5?$AA@ 5f590974     oledlgs1.obj
 0002:0000298c       ??_C@_0BD@DAIF@?6m_ps?4hInstance?5?$DN?5?$AA@ 5f59098c     oledlgs1.obj
 0002:000029a0       ??_C@_0BD@OAMP@?6m_ps?4lCustData?5?$DN?5?$AA@ 5f5909a0     oledlgs1.obj
 0002:000029b4       ??_C@_0BF@HGCH@?6m_ps?4lpszCaption?5?$DN?5?$AA@ 5f5909b4     oledlgs1.obj
 0002:000029cc       ??_C@_0BD@KHAG@?6m_ps?4hWndOwner?5?$DN?5?$AA@ 5f5909cc     oledlgs1.obj
 0002:000029e0       ??_C@_0BB@JIOH@?6m_ps?4dwFlags?5?$DN?5?$AA@ 5f5909e0     oledlgs1.obj
 0002:000029f4       ??_C@_0BB@IJHD@m_ps?4cbStruct?5?$DN?5?$AA@ 5f5909f4     oledlgs1.obj
 0002:00002a08       ??_C@_0CH@ICMM@Warning?3?5failed?5to?5set?5iconic?5as@ 5f590a08     oledlgs1.obj
 0002:00002a30       ??_C@_0CB@CMHB@Warning?3?5CreateFromData?5failed?4?6@ 5f590a30     oledlgs1.obj
 0002:00002a54       ??_C@_0CH@BNEA@Warning?3?5CreateStaticFromData?5fa@ 5f590a54     oledlgs1.obj
 0002:00002a7c       ??_C@_0CF@PLKL@Warning?3?5CreateLinkFromData?5fail@ 5f590a7c     oledlgs1.obj
 0002:00002aa8       ?classCOleBusyDialog@COleBusyDialog@@2UCRuntimeClass@@B 5f590aa8     oledlgs2.obj
 0002:00002ac0       ??_C@_0P@CLOH@COleBusyDialog?$AA@ 5f590ac0     oledlgs2.obj
 0002:00002ad0       ?classCOleDialog@COleDialog@@2UCRuntimeClass@@B 5f590ad0     oledlgs2.obj
 0002:00002ae8       ??_C@_0L@HMIO@COleDialog?$AA@ 5f590ae8     oledlgs2.obj
 0002:00002af8       ??_7COleDialog@@6B@        5f590af8     oledlgs2.obj
 0002:00002bd0       ??_C@_0BA@LHGD@m_nLastError?5?$DN?5?$AA@ 5f590bd0     oledlgs2.obj
 0002:00002be4       ??_7COleBusyDialog@@6B@    5f590be4     oledlgs2.obj
 0002:00002cbc       ??_C@_0P@PHCO@?6m_bz?4hTask?5?$DN?5?$AA@ 5f590cbc     oledlgs2.obj
 0002:00002ccc       ??_C@_0BD@PJDN@?6m_bz?4hResource?5?$DN?5?$AA@ 5f590ccc     oledlgs2.obj
 0002:00002ce0       ??_C@_0BG@LEJO@?6m_bz?4lpszTemplate?5?$DN?5?$AA@ 5f590ce0     oledlgs2.obj
 0002:00002cf8       ??_C@_0BD@DNBK@?6m_bz?4hInstance?5?$DN?5?$AA@ 5f590cf8     oledlgs2.obj
 0002:00002d0c       ??_C@_0BD@ONFA@?6m_bz?4lCustData?5?$DN?5?$AA@ 5f590d0c     oledlgs2.obj
 0002:00002d20       ??_C@_0BF@PDKP@?6m_bz?4lpszCaption?5?$DN?5?$AA@ 5f590d20     oledlgs2.obj
 0002:00002d38       ??_C@_0BD@KKJJ@?6m_bz?4hWndOwner?5?$DN?5?$AA@ 5f590d38     oledlgs2.obj
 0002:00002d4c       ??_C@_0BB@COFM@?6m_bz?4dwFlags?5?$DN?5?$AA@ 5f590d4c     oledlgs2.obj
 0002:00002d60       ??_C@_0BB@BGMF@m_bz?4cbStruct?5?$DN?5?$AA@ 5f590d60     oledlgs2.obj
 0002:00002d78       ?classCOleChangeSourceDialog@COleChangeSourceDialog@@2UCRuntimeClass@@B 5f590d78     oledlgs3.obj
 0002:00002d90       ??_C@_0BH@HBLJ@COleChangeSourceDialog?$AA@ 5f590d90     oledlgs3.obj
 0002:00002da8       ?classCOlePropertiesDialog@COlePropertiesDialog@@2UCRuntimeClass@@B 5f590da8     oledlgs3.obj
 0002:00002dc0       ??_C@_0BF@IDJJ@COlePropertiesDialog?$AA@ 5f590dc0     oledlgs3.obj
 0002:00002ddc       ??_7COlePropertiesDialog@@6B@ 5f590ddc     oledlgs3.obj
 0002:00002ebc       ??_7XOleUIObjInfo@COlePropertiesDialog@@6B@ 5f590ebc     oledlgs3.obj
 0002:00002ee0       ??_7IOleUIObjInfoA@@6B@    5f590ee0     oledlgs3.obj
 0002:00002f04       ??_7COleChangeSourceDialog@@6B@ 5f590f04     oledlgs3.obj
 0002:00002fdc       ??_C@_0BD@JJEH@?6m_cs?4hResource?5?$DN?5?$AA@ 5f590fdc     oledlgs3.obj
 0002:00002ff0       ??_C@_0BG@PEEF@?6m_cs?4lpszTemplate?5?$DN?5?$AA@ 5f590ff0     oledlgs3.obj
 0002:00003008       ??_C@_0BD@FNGA@?6m_cs?4hInstance?5?$DN?5?$AA@ 5f591008     oledlgs3.obj
 0002:0000301c       ??_C@_0BD@INCK@?6m_cs?4lCustData?5?$DN?5?$AA@ 5f59101c     oledlgs3.obj
 0002:00003030       ??_C@_0BF@CIFJ@?6m_cs?4lpszCaption?5?$DN?5?$AA@ 5f591030     oledlgs3.obj
 0002:00003048       ??_C@_0BD@MKOD@?6m_cs?4hWndOwner?5?$DN?5?$AA@ 5f591048     oledlgs3.obj
 0002:0000305c       ??_C@_0BB@HNIP@?6m_cs?4dwFlags?5?$DN?5?$AA@ 5f59105c     oledlgs3.obj
 0002:00003070       ??_C@_0BB@GMJG@m_cs?4cbStruct?5?$DN?5?$AA@ 5f591070     oledlgs3.obj
 0002:00003088       ??_7_AFX_OLE_STATE@@6B@    5f591088     oledata.obj
 0002:00003090       ??_7CNoTrackObject@@6B@    5f591090     oledata.obj
 0002:00003094       ??_C@_0O@MAFH@?6?7?5punkVal?5?$DN?5?$AA@ 5f591094     olevar.obj
 0002:000030a4       ??_C@_0M@GFHL@?6?7?5scode?5?$DN?5?$AA@ 5f5910a4     olevar.obj
 0002:000030b0       ??_C@_0O@EOOF@?6?7?5bstrVal?5?$DN?5?$AA@ 5f5910b0     olevar.obj
 0002:000030c0       ??_C@_0L@KHBD@?6?7?5date?5?$DN?5?$AA@ 5f5910c0     olevar.obj
 0002:000030cc       ??_C@_0N@PCIP@?6?7?5dblVal?5?$DN?5?$AA@ 5f5910cc     olevar.obj
 0002:000030dc       ??_C@_0N@BKHL@?6?7?5fltVal?5?$DN?5?$AA@ 5f5910dc     olevar.obj
 0002:000030ec       ??_C@_0M@NOJL@?6?7?5cyVal?5?$DN?5?$AA@ 5f5910ec     olevar.obj
 0002:000030f8       ??_C@_0L@PIPP@?6?7?5lVal?5?$DN?5?$AA@ 5f5910f8     olevar.obj
 0002:00003104       ??_C@_0L@GMDM@?6?7?5iVal?5?$DN?5?$AA@ 5f591104     olevar.obj
 0002:00003110       ??_C@_0L@GLCP@?6?7?5bVal?5?$DN?5?$AA@ 5f591110     olevar.obj
 0002:0000311c       ??_C@_0O@NJPJ@?6?7?5VT_BOOL?5?$DN?5?$AA@ 5f59111c     olevar.obj
 0002:0000312c       ??_C@_08JIFF@?6?7?5vt?5?$DN?5?$AA@ 5f59112c     olevar.obj
 0002:00003138       ??_C@_0BF@NHIO@?6COleVariant?5Object?3?$AA@ 5f591138     olevar.obj
 0002:00003150       __real@8@40038000000000000000 5f591150     olevar.obj
 0002:00003158       __real@4@40038000000000000000 5f591158     olevar.obj
 0002:0000315c       ??_C@_0CK@JMOE@?6COleCurrency?5VarCyFromStr?5call?5@ 5f59115c     olevar.obj
 0002:00003188       ??_C@_0O@GEHN@?6?7Currency?5?$DN?5?$AA@ 5f591188     olevar.obj
 0002:00003198       ??_C@_0O@DBAA@?6?7m_status?5?$DN?5?$AA@ 5f591198     olevar.obj
 0002:000031a8       ??_C@_0BG@PNJ@?6COleCurrency?5Object?3?$AA@ 5f5911a8     olevar.obj
 0002:000031c0       __real@8@400fa8c0000000000000 5f5911c0     olevar.obj
 0002:000031c8       __real@8@00000000000000000000 5f5911c8     olevar.obj
 0002:000031d0       __real@8@c012a081a00000000000 5f5911d0     olevar.obj
 0002:000031d8       __real@8@4014b492040000000000 5f5911d8     olevar.obj
 0002:000031e0       ??_C@_0DA@FCDK@?6FileTimeToLocalFileTime?5failed?4@ 5f5911e0     olevar.obj
 0002:00003210       ??_C@_0CM@PAKN@?6COleDateTime?5VarDateFromStr?5cal@ 5f591210     olevar.obj
 0002:0000323c       ??_C@_09IMNF@?6?7date?5?$DN?5?$AA@ 5f59123c     olevar.obj
 0002:00003248       ??_C@_0BG@FBOI@?6COleDateTime?5Object?3?$AA@ 5f591248     olevar.obj
 0002:00003260       __real@8@4003c000000000000000 5f591260     olevar.obj
 0002:00003268       __real@8@3fedc22e450672894800 5f591268     olevar.obj
 0002:00003270       __real@8@4004f000000000000000 5f591270     olevar.obj
 0002:00003278       __real@8@4009b400000000000000 5f591278     olevar.obj
 0002:00003280       __real@8@4014dcb2640000000000 5f591280     olevar.obj
 0002:00003288       __real@8@c014dcb2640000000000 5f591288     olevar.obj
 0002:00003290       ??_C@_0O@CNBC@?6?7dateSpan?5?$DN?5?$AA@ 5f591290     olevar.obj
 0002:000032a0       ??_C@_0BK@NGPI@?6COleDateTimeSpan?5Object?3?$AA@ 5f5912a0     olevar.obj
 0002:000032bc       ??_C@_03FGJK@?5?$DN?5?$AA@ 5f5912bc     olevar.obj
 0002:000032c0       ??_C@_01KHLB@?$FL?$AA@     5f5912c0     olevar.obj
 0002:000032c4       ??_C@_01FIMD@?$FN?$AA@     5f5912c4     olevar.obj
 0002:000032c8       ??_C@_02GGCO@?6?7?$AA@     5f5912c8     olevar.obj
 0002:000032cc       ??_C@_03JBDO@?6?7?$CI?$AA@ 5f5912cc     olevar.obj
 0002:000032d0       ??_C@_02GIEM@?0?5?$AA@     5f5912d0     olevar.obj
 0002:000032d4       ??_C@_01KMMP@?$CJ?$AA@     5f5912d4     olevar.obj
 0002:000032d8       ??_C@_09FDDC@?6?7bounds?3?$AA@ 5f5912d8     olevar.obj
 0002:000032e4       ??_C@_07LGGH@?6?7vt?5?$DN?5?$AA@ 5f5912e4     olevar.obj
 0002:000032ec       ??_C@_0BH@NEKA@?6COleSafeArray?5Object?3?$AA@ 5f5912ec     olevar.obj
 0002:00003308       ?classCOleServerItem@COleServerItem@@2UCRuntimeClass@@B 5f591308     oledoc1.obj
 0002:00003320       ??_C@_0P@ODMG@COleServerItem?$AA@ 5f591320     oledoc1.obj
 0002:00003330       ?classCOleClientItem@COleClientItem@@2UCRuntimeClass@@B 5f591330     oledoc1.obj
 0002:00003348       ??_C@_0P@JNNP@COleClientItem?$AA@ 5f591348     oledoc1.obj
 0002:00003358       ?classCOleDocument@COleDocument@@2UCRuntimeClass@@B 5f591358     oledoc1.obj
 0002:00003370       ??_C@_0N@KLEF@COleDocument?$AA@ 5f591370     oledoc1.obj
 0002:00003380       ??_C@_08NNLJ@CDocItem?$AA@ 5f591380     oledoc1.obj
 0002:0000338c       ??_C@_0CM@MMBL@?7perhaps?5AfxOleInit?$CI?$CJ?5has?5not?5be@ 5f59138c     oledoc1.obj
 0002:000033b8       ??_C@_0DC@OHFM@Warning?3?5CoGetMalloc?$CIMEMCTX_TASK@ 5f5913b8     oledoc1.obj
 0002:000033f0       ??_7COleDocument@@6B@      5f5913f0     oledoc1.obj
 0002:000034d8       ??_C@_0DF@GLPN@Warning?3?5destroying?5COleDocument@ 5f5914d8     oledoc1.obj
 0002:00003510       ??_C@_0DH@OIJJ@Warning?3?5OnOpenDocument?5replaces@ 5f591510     oledoc1.obj
 0002:00003548       ??_C@_08IBMA@Contents?$AA@ 5f591548     oledoc1.obj
 0002:00003554       ??_C@_09HEBF@?6m_ptd?5?$DN?5?$AA@ 5f591554     oledoc1.obj
 0002:00003560       ??_C@_0BA@DJOI@?6m_bRemember?5?$DN?5?$AA@ 5f591560     oledoc1.obj
 0002:00003570       ??_C@_0BC@BIJ@?6m_bSameAsLoad?5?$DN?5?$AA@ 5f591570     oledoc1.obj
 0002:00003584       ??_C@_0BA@MPDA@?6m_lpRootStg?5?$DN?5?$AA@ 5f591584     oledoc1.obj
 0002:00003594       ??_C@_0BA@IKCF@?6m_bEmbedded?5?$DN?5?$AA@ 5f591594     oledoc1.obj
 0002:000035a4       ??_C@_0BD@KBMC@?6m_bLastVisible?5?$DN?5?$AA@ 5f5915a4     oledoc1.obj
 0002:000035b8       ??_C@_0BH@BKJA@?6m_dwNextItemNumber?5?$DN?5?$AA@ 5f5915b8     oledoc1.obj
 0002:000035d0       ??_C@_05KIFI@with?5?$AA@   5f5915d0     oledoc1.obj
 0002:000035d8       ??_C@_0L@EFON@?5doc?5items?$AA@ 5f5915d8     oledoc1.obj
 0002:000035e8       ??_7CDocItem@@6B@          5f5915e8     oledoc1.obj
 0002:00003644       ??_C@_0P@NBEM@m_pDocument?5?$DN?5?$AA@ 5f591644     oledoc1.obj
 0002:00003658       ?interfaceMap@COleDropSource@@1UAFX_INTERFACEMAP@@B 5f591658     oledrop1.obj
 0002:00003660       ?_interfaceEntries@COleDropSource@@0QBUAFX_INTERFACEMAP_ENTRY@@B 5f591660     oledrop1.obj
 0002:00003694       ??_7COleDropSource@@6B@    5f591694     oledrop1.obj
 0002:000036fc       ??_7XDropSource@COleDropSource@@6B@ 5f5916fc     oledrop1.obj
 0002:00003710       ??_C@_0BL@ICEB@?6m_rectStartDrag?4bottom?5?$DN?5?$AA@ 5f591710     oledrop1.obj
 0002:0000372c       ??_C@_0BK@NCCF@?6m_rectStartDrag?4right?5?$DN?5?$AA@ 5f59172c     oledrop1.obj
 0002:00003748       ??_C@_0BI@LLBJ@?6m_rectStartDrag?4top?5?$DN?5?$AA@ 5f591748     oledrop1.obj
 0002:00003760       ??_C@_0BJ@IMOF@?6m_rectStartDrag?4left?5?$DN?5?$AA@ 5f591760     oledrop1.obj
 0002:0000377c       ??_C@_0BC@ECHL@m_bDragStarted?5?$DN?5?$AA@ 5f59177c     oledrop1.obj
 0002:00003790       ?interfaceMap@COleDropTarget@@1UAFX_INTERFACEMAP@@B 5f591790     oledrop2.obj
 0002:00003798       ?_interfaceEntries@COleDropTarget@@0QBUAFX_INTERFACEMAP_ENTRY@@B 5f591798     oledrop2.obj
 0002:000037e8       ??_7COleDropTarget@@6B@    5f5917e8     oledrop2.obj
 0002:00003860       ??_7XDropTarget@COleDropTarget@@6B@ 5f591860     oledrop2.obj
 0002:0000387c       ??_C@_0CG@HKAA@?7may?5cause?5RIPs?5under?5debug?5Wind@ 5f59187c     oledrop2.obj
 0002:000038a4       ??_C@_0DI@PFLH@COleDropTarget?3?3Revoke?5not?5calle@ 5f5918a4     oledrop2.obj
 0002:000038dc       ??_C@_0BB@OINI@?6m_dwLastTick?5?$DN?5?$AA@ 5f5918dc     oledrop2.obj
 0002:000038f0       ??_C@_0P@NGLE@?6m_nTimerID?5?$DN?5?$AA@ 5f5918f0     oledrop2.obj
 0002:00003900       ??_C@_0BD@KEMD@?6m_lpDataObject?5?$DN?5?$AA@ 5f591900     oledrop2.obj
 0002:00003914       ??_C@_09BKNC@m_hWnd?5?$DN?5?$AA@ 5f591914     oledrop2.obj
 0002:00003920       ?interfaceMap@COleMessageFilter@@1UAFX_INTERFACEMAP@@B 5f591920     olemsgf.obj
 0002:00003928       ?_interfaceEntries@COleMessageFilter@@0QBUAFX_INTERFACEMAP_ENTRY@@B 5f591928     olemsgf.obj
 0002:00003938       ?_afxSignificantMsgs@@3QBIB 5f591938     olemsgf.obj
 0002:00003978       ??_7COleMessageFilter@@6B@ 5f591978     olemsgf.obj
 0002:000039ec       ??_7XMessageFilter@COleMessageFilter@@6B@ 5f5919ec     olemsgf.obj
 0002:00003a04       ??_C@_0P@JKLE@?6m_nTimeout?5?$DN?5?$AA@ 5f591a04     olemsgf.obj
 0002:00003a14       ??_C@_0BB@PGOJ@?6m_nBusyReply?5?$DN?5?$AA@ 5f591a14     olemsgf.obj
 0002:00003a28       ??_C@_0BC@GKAC@?6m_nRetryReply?5?$DN?5?$AA@ 5f591a28     olemsgf.obj
 0002:00003a3c       ??_C@_0BC@IEIC@?6m_bUnblocking?5?$DN?5?$AA@ 5f591a3c     olemsgf.obj
 0002:00003a50       ??_C@_0BL@KMOL@?6m_bEnableNotResponding?5?$DN?5?$AA@ 5f591a50     olemsgf.obj
 0002:00003a6c       ??_C@_0BC@KPPB@?6m_bEnableBusy?5?$DN?5?$AA@ 5f591a6c     olemsgf.obj
 0002:00003a80       ??_C@_0BB@MEI@?6m_nBusyCount?5?$DN?5?$AA@ 5f591a80     olemsgf.obj
 0002:00003a94       ??_C@_0BB@EDJN@m_bRegistered?5?$DN?5?$AA@ 5f591a94     olemsgf.obj
 0002:00003aac       ??_7CEnumArray@@6B@        5f591aac     oleenum.obj
 0002:00003b18       ??_7XEnumVOID@CEnumArray@@6B@ 5f591b18     oleenum.obj
 0002:00003b38       ??_7IEnumVOID@@6B@         5f591b38     oleenum.obj
 0002:00003b58       ?classCOleObjectFactory@COleObjectFactory@@2UCRuntimeClass@@B 5f591b58     olefact.obj
 0002:00003b70       ??_C@_0BC@HKPN@COleObjectFactory?$AA@ 5f591b70     olefact.obj
 0002:00003b88       ?interfaceMap@COleObjectFactory@@1UAFX_INTERFACEMAP@@B 5f591b88     olefact.obj
 0002:00003b90       ?_interfaceEntries@COleObjectFactory@@0QBUAFX_INTERFACEMAP_ENTRY@@B 5f591b90     olefact.obj
 0002:00003bac       ??_7COleObjectFactory@@6B@ 5f591bac     olefact.obj
 0002:00003c24       ??_7XClassFactory@COleObjectFactory@@6B@ 5f591c24     olefact.obj
 0002:00003c44       ??_C@_0DD@FLGE@Warning?3?5CoRegisterClassObject?5f@ 5f591c44     olefact.obj
 0002:00003c78       ??_C@_0CP@CCDB@Warning?3?5object?5created?5with?5ref@ 5f591c78     olefact.obj
 0002:00003ca8       ??_C@_0BE@OGII@?6m_bLicenseValid?5?$DN?5?$AA@ 5f591ca8     olefact.obj
 0002:00003cbc       ??_C@_0BG@HOFD@?6m_bLicenseChecked?5?$DN?5?$AA@ 5f591cbc     olefact.obj
 0002:00003cd4       ??_C@_0BB@CECH@?6m_lpszProgID?5?$DN?5?$AA@ 5f591cd4     olefact.obj
 0002:00003ce8       ??_C@_0BF@OMHN@?6m_bMultiInstance?5?$DN?5?$AA@ 5f591ce8     olefact.obj
 0002:00003d00       ??_C@_0BE@BMEC@?6m_pRuntimeClass?5?$DN?5?$AA@ 5f591d00     olefact.obj
 0002:00003d14       ??_C@_0M@GKHL@?6m_clsid?5?$DN?5?$AA@ 5f591d14     olefact.obj
 0002:00003d20       ??_C@_0BC@KNA@?6m_bRegistered?5?$DN?5?$AA@ 5f591d20     olefact.obj
 0002:00003d34       ??_C@_0BB@GHJL@?6m_dwRegister?5?$DN?5?$AA@ 5f591d34     olefact.obj
 0002:00003d48       ??_C@_0BC@HEHA@m_pNextFactory?5?$DN?5?$AA@ 5f591d48     olefact.obj
 0002:00003d60       ?classCOleIPFrameWnd@COleIPFrameWnd@@2UCRuntimeClass@@B 5f591d60     oleipfrm.obj
 0002:00003d78       ??_C@_0P@CBLJ@COleIPFrameWnd?$AA@ 5f591d78     oleipfrm.obj
 0002:00003d88       ?messageMap@COleIPFrameWnd@@1UAFX_MSGMAP@@B 5f591d88     oleipfrm.obj
 0002:00003d90       ?_messageEntries@COleIPFrameWnd@@0QBUAFX_MSGMAP_ENTRY@@B 5f591d90     oleipfrm.obj
 0002:00003ecc       ??_7COleCntrFrameWnd@@6B@  5f591ecc     oleipfrm.obj
 0002:00003fcc       ??_7COleIPFrameWnd@@6B@    5f591fcc     oleipfrm.obj
 0002:000040e8       ??_C@_0BC@GPEG@?6m_hSharedMenu?5?$DN?5?$AA@ 5f5920e8     oleipfrm.obj
 0002:000040fc       ??_C@_0BE@EIME@?6m_bInsideRecalc?5?$DN?5?$AA@ 5f5920fc     oleipfrm.obj
 0002:00004110       ??_C@_0P@MHEP@?6m_rectClip?5?$DN?5?$AA@ 5f592110     oleipfrm.obj
 0002:00004120       ??_C@_0O@FEOJ@?6m_rectPos?5?$DN?5?$AA@ 5f592120     oleipfrm.obj
 0002:00004130       ??_C@_0P@JLOC@?6m_hOleMenu?5?$DN?5?$AA@ 5f592130     oleipfrm.obj
 0002:00004140       ??_C@_0BB@PHGG@?6m_lpDocFrame?5?$DN?5?$AA@ 5f592140     oleipfrm.obj
 0002:00004154       ??_C@_0N@LBG@m_lpFrame?5?$DN?5?$AA@ 5f592154     oleipfrm.obj
 0002:00004168       ?interfaceMap@COleLinkingDoc@@1UAFX_INTERFACEMAP@@B 5f592168     olelink.obj
 0002:00004170       ?_interfaceEntries@COleLinkingDoc@@0QBUAFX_INTERFACEMAP_ENTRY@@B 5f592170     olelink.obj
 0002:000041a4       ??_7COleLinkingDoc@@6B@    5f5921a4     olelink.obj
 0002:0000429c       ??_7XPersistFile@COleLinkingDoc@@6B@ 5f59229c     olelink.obj
 0002:000042c4       ??_7XOleItemContainer@COleLinkingDoc@@6B@ 5f5922c4     olelink.obj
 0002:000042e8       ??_C@_0DF@OLP@Warning?3?5Unable?5to?5register?5moni@ 5f5922e8     olelink.obj
 0002:00004320       ??_C@_0CL@JGGO@?7implementation?5failed?5to?5find?5i@ 5f592320     olelink.obj
 0002:0000434c       ??_C@_0DF@JBIB@Warning?3?5default?5COleLinkingDoc?3@ 5f59234c     olelink.obj
 0002:00004384       ??_C@_0BB@BIHL@?6with?5no?5factory?$AA@ 5f592384     olelink.obj
 0002:00004398       ??_C@_0BA@KOFE@?6with?5factory?3?5?$AA@ 5f592398     olelink.obj
 0002:000043a8       ??_C@_0BD@KPFI@?6m_bVisibleLock?5?$DN?5?$AA@ 5f5923a8     olelink.obj
 0002:000043c0       ?classCOleException@COleException@@2UCRuntimeClass@@B 5f5923c0     olemisc.obj
 0002:000043d8       ??_C@_0O@EEPE@COleException?$AA@ 5f5923d8     olemisc.obj
 0002:000043e8       ??_C@_0BB@FEOB@FACILITY_WINDOWS?$AA@ 5f5923e8     olemisc.obj
 0002:000043fc       ??_C@_0P@NGEF@FACILITY_WIN32?$AA@ 5f5923fc     olemisc.obj
 0002:0000440c       ??_C@_0O@BJCN@FACILITY_0x06?$AA@ 5f59240c     olemisc.obj
 0002:0000441c       ??_C@_0O@OGJE@FACILITY_0x05?$AA@ 5f59241c     olemisc.obj
 0002:0000442c       ??_C@_0N@HAFM@FACILITY_ITF?$AA@ 5f59242c     olemisc.obj
 0002:0000443c       ??_C@_0BB@LABF@FACILITY_STORAGE?$AA@ 5f59243c     olemisc.obj
 0002:00004450       ??_C@_0BC@MMLL@FACILITY_DISPATCH?$AA@ 5f592450     olemisc.obj
 0002:00004464       ??_C@_0N@GNNJ@FACILITY_RPC?$AA@ 5f592464     olemisc.obj
 0002:00004474       ??_C@_0O@CKPN@FACILITY_NULL?$AA@ 5f592474     olemisc.obj
 0002:00004484       ??_C@_0P@EJLP@SEVERITY_ERROR?$AA@ 5f592484     olemisc.obj
 0002:00004494       ??_C@_0BB@HNBI@SEVERITY_SUCCESS?$AA@ 5f592494     olemisc.obj
 0002:00004dc0       ??_C@_0BL@BBDA@VIEW_S_FIRST?4?4?4VIEW_S_LAST?$AA@ 5f592dc0     olemisc.obj
 0002:00004ddc       ??_C@_0BL@FDEF@VIEW_E_FIRST?4?4?4VIEW_E_LAST?$AA@ 5f592ddc     olemisc.obj
 0002:00004df8       ??_C@_0BN@OJHK@REGDB_S_FIRST?4?4?4REGDB_S_LAST?$AA@ 5f592df8     olemisc.obj
 0002:00004e18       ??_C@_0BN@LINN@REGDB_E_FIRST?4?4?4REGDB_E_LAST?$AA@ 5f592e18     olemisc.obj
 0002:00004e38       ??_C@_0BJ@LDNK@OLE_S_FIRST?4?4?4OLE_S_LAST?$AA@ 5f592e38     olemisc.obj
 0002:00004e54       ??_C@_0BJ@CDPN@OLE_E_FIRST?4?4?4OLE_E_LAST?$AA@ 5f592e54     olemisc.obj
 0002:00004e70       ??_C@_0BP@LNJ@OLEOBJ_S_FIRST?4?4?4OLEOBJ_S_LAST?$AA@ 5f592e70     olemisc.obj
 0002:00004e90       ??_C@_0BP@FJGN@OLEOBJ_E_FIRST?4?4?4OLEOBJ_E_LAST?$AA@ 5f592e90     olemisc.obj
 0002:00004eb0       ??_C@_0BH@CIDM@MK_S_FIRST?4?4?4MK_S_LAST?$AA@ 5f592eb0     olemisc.obj
 0002:00004ec8       ??_C@_0BH@OKNN@MK_E_FIRST?4?4?4MK_E_LAST?$AA@ 5f592ec8     olemisc.obj
 0002:00004ee0       ??_C@_0CB@PFHE@MARSHAL_S_FIRST?4?4?4MARSHAL_S_LAST@ 5f592ee0     olemisc.obj
 0002:00004f04       ??_C@_0CB@JCMD@MARSHAL_E_FIRST?4?4?4MARSHAL_E_LAST@ 5f592f04     olemisc.obj
 0002:00004f28       ??_C@_0CB@OBKF@INPLACE_S_FIRST?4?4?4INPLACE_S_LAST@ 5f592f28     olemisc.obj
 0002:00004f4c       ??_C@_0CB@IGBC@INPLACE_E_FIRST?4?4?4INPLACE_E_LAST@ 5f592f4c     olemisc.obj
 0002:00004f70       ??_C@_0BL@BPFC@ENUM_S_FIRST?4?4?4ENUM_S_LAST?$AA@ 5f592f70     olemisc.obj
 0002:00004f8c       ??_C@_0BL@FNCH@ENUM_E_FIRST?4?4?4ENUM_E_LAST?$AA@ 5f592f8c     olemisc.obj
 0002:00004fa8       ??_C@_0CD@MDEB@DRAGDROP_S_FIRST?4?4?4DRAGDROP_S_LA@ 5f592fa8     olemisc.obj
 0002:00004fcc       ??_C@_0CD@MKMD@DRAGDROP_E_FIRST?4?4?4DRAGDROP_E_LA@ 5f592fcc     olemisc.obj
 0002:00004ff0       ??_C@_0BL@FEGO@DATA_S_FIRST?4?4?4DATA_S_LAST?$AA@ 5f592ff0     olemisc.obj
 0002:0000500c       ??_C@_0BL@BGBL@DATA_E_FIRST?4?4?4DATA_E_LAST?$AA@ 5f59300c     olemisc.obj
 0002:00005028       ??_C@_0BH@NNJL@CO_S_FIRST?4?4?4CO_S_LAST?$AA@ 5f593028     olemisc.obj
 0002:00005040       ??_C@_0BH@BPHK@CO_E_FIRST?4?4?4CO_E_LAST?$AA@ 5f593040     olemisc.obj
 0002:00005058       ??_C@_0CF@FBAG@CONVERT10_S_FIRST?4?4?4CONVERT10_S_@ 5f593058     olemisc.obj
 0002:00005080       ??_C@_0CF@CMOK@CONVERT10_E_FIRST?4?4?4CONVERT10_E_@ 5f593080     olemisc.obj
 0002:000050a8       ??_C@_0CB@HENF@CLIPBRD_S_FIRST?4?4?4CLIPBRD_S_LAST@ 5f5930a8     olemisc.obj
 0002:000050cc       ??_C@_0CB@BDGC@CLIPBRD_E_FIRST?4?4?4CLIPBRD_E_LAST@ 5f5930cc     olemisc.obj
 0002:000050f0       ??_C@_0CH@MFPB@CLIENTSITE_S_FIRST?4?4?4CLIENTSITE_@ 5f5930f0     olemisc.obj
 0002:00005118       ??_C@_0CH@MGGJ@CLIENTSITE_E_FIRST?4?4?4CLIENTSITE_@ 5f593118     olemisc.obj
 0002:00005140       ??_C@_0CL@DCFF@CLASSFACTORY_S_FIRST?4?4?4CLASSFACT@ 5f593140     olemisc.obj
 0002:0000516c       ??_C@_0CL@FKOP@CLASSFACTORY_E_FIRST?4?4?4CLASSFACT@ 5f59316c     olemisc.obj
 0002:00005198       ??_C@_0BN@BFHH@CACHE_S_FIRST?4?4?4CACHE_S_LAST?$AA@ 5f593198     olemisc.obj
 0002:000051b8       ??_C@_0BN@EENA@CACHE_E_FIRST?4?4?4CACHE_E_LAST?$AA@ 5f5931b8     olemisc.obj
 0002:000051d8       ??_C@_0M@EJHN@VIEW_E_DRAW?$AA@ 5f5931d8     olemisc.obj
 0002:000051e4       ??_C@_0BF@DOMI@TYPE_E_WRONGTYPEKIND?$AA@ 5f5931e4     olemisc.obj
 0002:000051fc       ??_C@_0BD@KID@TYPE_E_UNSUPFORMAT?$AA@ 5f5931fc     olemisc.obj
 0002:00005210       ??_C@_0BD@NMIN@TYPE_E_UNKNOWNLCID?$AA@ 5f593210     olemisc.obj
 0002:00005224       ??_C@_0BF@MJPL@TYPE_E_UNDEFINEDTYPE?$AA@ 5f593224     olemisc.obj
 0002:0000523c       ??_C@_0BE@HAEH@TYPE_E_TYPEMISMATCH?$AA@ 5f59323c     olemisc.obj
 0002:00005250       ??_C@_0BC@JDHF@TYPE_E_SIZETOOBIG?$AA@ 5f593250     olemisc.obj
 0002:00005264       ??_C@_0BG@FFPJ@TYPE_E_REGISTRYACCESS?$AA@ 5f593264     olemisc.obj
 0002:0000527c       ??_C@_0BP@GAEP@TYPE_E_QUALIFIEDNAMEDISALLOWED?$AA@ 5f59327c     olemisc.obj
 0002:0000529c       ??_C@_0BD@GAJB@TYPE_E_OUTOFBOUNDS?$AA@ 5f59329c     olemisc.obj
 0002:000052b0       ??_C@_0BE@HBBE@TYPE_E_NAMECONFLICT?$AA@ 5f5932b0     olemisc.obj
 0002:000052c4       ??_C@_0BI@IKOE@TYPE_E_LIBNOTREGISTERED?$AA@ 5f5932c4     olemisc.obj
 0002:000052dc       ??_C@_0P@GDJH@TYPE_E_IOERROR?$AA@ 5f5932dc     olemisc.obj
 0002:000052ec       ??_C@_0BD@BDCM@TYPE_E_INVDATAREAD?$AA@ 5f5932ec     olemisc.obj
 0002:00005300       ??_C@_0BE@LHHL@TYPE_E_INVALIDSTATE?$AA@ 5f593300     olemisc.obj
 0002:00005314       ??_C@_0BN@IIKI@TYPE_E_INCONSISTENTPROPFUNCS?$AA@ 5f593314     olemisc.obj
 0002:00005334       ??_C@_0BH@PKEE@TYPE_E_ELEMENTNOTFOUND?$AA@ 5f593334     olemisc.obj
 0002:0000534c       ??_C@_0BD@HFCB@TYPE_E_DUPLICATEID?$AA@ 5f59334c     olemisc.obj
 0002:00005360       ??_C@_0BL@KFLM@TYPE_E_DLLFUNCTIONNOTFOUND?$AA@ 5f593360     olemisc.obj
 0002:0000537c       ??_C@_0BE@LKMM@TYPE_E_CIRCULARTYPE?$AA@ 5f59337c     olemisc.obj
 0002:00005390       ??_C@_0BH@OEOC@TYPE_E_CANTLOADLIBRARY?$AA@ 5f593390     olemisc.obj
 0002:000053a8       ??_C@_0BJ@PDNG@TYPE_E_CANTCREATETMPFILE?$AA@ 5f5933a8     olemisc.obj
 0002:000053c4       ??_C@_0BG@HMOE@TYPE_E_BUFFERTOOSMALL?$AA@ 5f5933c4     olemisc.obj
 0002:000053dc       ??_C@_0BF@FACD@TYPE_E_BADMODULEKIND?$AA@ 5f5933dc     olemisc.obj
 0002:000053f4       ??_C@_0BF@DCPG@TYPE_E_AMBIGUOUSNAME?$AA@ 5f5933f4     olemisc.obj
 0002:0000540c       ??_C@_0BB@MCHJ@STG_E_WRITEFAULT?$AA@ 5f59340c     olemisc.obj
 0002:00005420       ??_C@_0O@CGJ@STG_E_UNKNOWN?$AA@ 5f593420     olemisc.obj
 0002:00005430       ??_C@_0BM@PNME@STG_E_UNIMPLEMENTEDFUNCTION?$AA@ 5f593430     olemisc.obj
 0002:0000544c       ??_C@_0BH@KKDE@STG_E_TOOMANYOPENFILES?$AA@ 5f59344c     olemisc.obj
 0002:00005464       ??_C@_0BF@LHLD@STG_E_SHAREVIOLATION?$AA@ 5f593464     olemisc.obj
 0002:0000547c       ??_C@_0BE@PMHE@STG_E_SHAREREQUIRED?$AA@ 5f59347c     olemisc.obj
 0002:00005490       ??_C@_0BA@NAPD@STG_E_SEEKERROR?$AA@ 5f593490     olemisc.obj
 0002:000054a0       ??_C@_0P@ODBJ@STG_E_REVERTED?$AA@ 5f5934a0     olemisc.obj
 0002:000054b0       ??_C@_0BA@ENNI@STG_E_READFAULT?$AA@ 5f5934b0     olemisc.obj
 0002:000054c0       ??_C@_0BD@MAIA@STG_E_PATHNOTFOUND?$AA@ 5f5934c0     olemisc.obj
 0002:000054d4       ??_C@_0BA@NFPJ@STG_E_OLDFORMAT?$AA@ 5f5934d4     olemisc.obj
 0002:000054e4       ??_C@_0N@CCGN@STG_E_OLDDLL?$AA@ 5f5934e4     olemisc.obj
 0002:000054f4       ??_C@_0BK@KDLL@STG_E_NOTFILEBASEDSTORAGE?$AA@ 5f5934f4     olemisc.obj
 0002:00005510       ??_C@_0BB@FHLH@STG_E_NOTCURRENT?$AA@ 5f593510     olemisc.obj
 0002:00005524       ??_C@_0BC@JPKH@STG_E_NOMOREFILES?$AA@ 5f593524     olemisc.obj
 0002:00005538       ??_C@_0BB@KIFE@STG_E_MEDIUMFULL?$AA@ 5f593538     olemisc.obj
 0002:0000554c       ??_C@_0BE@PJLD@STG_E_LOCKVIOLATION?$AA@ 5f59354c     olemisc.obj
 0002:00005560       ??_C@_0BF@EEHM@STG_E_INVALIDPOINTER?$AA@ 5f593560     olemisc.obj
 0002:00005578       ??_C@_0BH@DEML@STG_E_INVALIDPARAMETER?$AA@ 5f593578     olemisc.obj
 0002:00005590       ??_C@_0BC@FGBC@STG_E_INVALIDNAME?$AA@ 5f593590     olemisc.obj
 0002:000055a4       ??_C@_0BE@MKFL@STG_E_INVALIDHEADER?$AA@ 5f5935a4     olemisc.obj
 0002:000055b8       ??_C@_0BE@MFIL@STG_E_INVALIDHANDLE?$AA@ 5f5935b8     olemisc.obj
 0002:000055cc       ??_C@_0BG@BIHE@STG_E_INVALIDFUNCTION?$AA@ 5f5935cc     olemisc.obj
 0002:000055e4       ??_C@_0BC@EMKL@STG_E_INVALIDFLAG?$AA@ 5f5935e4     olemisc.obj
 0002:000055f8       ??_C@_0M@EFDG@STG_E_INUSE?$AA@ 5f5935f8     olemisc.obj
 0002:00005604       ??_C@_0BJ@OANH@STG_E_INSUFFICIENTMEMORY?$AA@ 5f593604     olemisc.obj
 0002:00005620       ??_C@_0BD@HNDG@STG_E_FILENOTFOUND?$AA@ 5f593620     olemisc.obj
 0002:00005634       ??_C@_0BI@GNCB@STG_E_FILEALREADYEXISTS?$AA@ 5f593634     olemisc.obj
 0002:0000564c       ??_C@_0BJ@NBHO@STG_E_EXTANTMARSHALLINGS?$AA@ 5f59364c     olemisc.obj
 0002:00005668       ??_C@_0BL@LBKA@STG_E_DISKISWRITEPROTECTED?$AA@ 5f593668     olemisc.obj
 0002:00005684       ??_C@_0P@CDEO@STG_E_CANTSAVE?$AA@ 5f593684     olemisc.obj
 0002:00005694       ??_C@_0BD@EICG@STG_E_ACCESSDENIED?$AA@ 5f593694     olemisc.obj
 0002:000056a8       ??_C@_0BG@PCHB@STG_E_ABNORMALAPIEXIT?$AA@ 5f5936a8     olemisc.obj
 0002:000056c0       ??_C@_0BD@JAPF@RPC_E_WRONG_THREAD?$AA@ 5f5936c0     olemisc.obj
 0002:000056d4       ??_C@_0BB@IMFM@RPC_E_UNEXPECTED?$AA@ 5f5936d4     olemisc.obj
 0002:000056e8       ??_C@_0BG@GBJK@RPC_E_THREAD_NOT_INIT?$AA@ 5f5936e8     olemisc.obj
 0002:00005700       ??_C@_0BG@JMDA@RPC_E_SYS_CALL_FAILED?$AA@ 5f593700     olemisc.obj
 0002:00005718       ??_C@_0BC@GELD@RPC_E_SERVERFAULT?$AA@ 5f593718     olemisc.obj
 0002:0000572c       ??_C@_0BM@NJMP@RPC_E_SERVERCALL_RETRYLATER?$AA@ 5f59372c     olemisc.obj
 0002:00005748       ??_C@_0BK@LGIK@RPC_E_SERVERCALL_REJECTED?$AA@ 5f593748     olemisc.obj
 0002:00005764       ??_C@_0BG@NHGE@RPC_E_SERVER_DIED_DNE?$AA@ 5f593764     olemisc.obj
 0002:0000577c       ??_C@_0BC@IEPI@RPC_E_SERVER_DIED?$AA@ 5f59377c     olemisc.obj
 0002:00005790       ??_C@_0CA@NNPK@RPC_E_SERVER_CANTUNMARSHAL_DATA?$AA@ 5f593790     olemisc.obj
 0002:000057b0       ??_C@_0BO@PBDM@RPC_E_SERVER_CANTMARSHAL_DATA?$AA@ 5f5937b0     olemisc.obj
 0002:000057d0       ??_C@_0M@CMMO@RPC_E_RETRY?$AA@ 5f5937d0     olemisc.obj
 0002:000057dc       ??_C@_0BH@IACH@RPC_E_OUT_OF_RESOURCES?$AA@ 5f5937dc     olemisc.obj
 0002:000057f4       ??_C@_0BF@GPDN@RPC_E_NOT_REGISTERED?$AA@ 5f5937f4     olemisc.obj
 0002:0000580c       ??_C@_0BE@IDOO@RPC_E_INVALIDMETHOD?$AA@ 5f59380c     olemisc.obj
 0002:00005820       ??_C@_0BI@DDIP@RPC_E_INVALID_PARAMETER?$AA@ 5f593820     olemisc.obj
 0002:00005838       ??_C@_0BJ@DCAC@RPC_E_INVALID_DATAPACKET?$AA@ 5f593838     olemisc.obj
 0002:00005854       ??_C@_0BD@PO@RPC_E_INVALID_DATA?$AA@ 5f593854     olemisc.obj
 0002:00005868       ??_C@_0BH@NBG@RPC_E_INVALID_CALLDATA?$AA@ 5f593868     olemisc.obj
 0002:00005880       ??_C@_0M@JFCB@RPC_E_FAULT?$AA@ 5f593880     olemisc.obj
 0002:0000588c       ??_C@_0BD@HNKB@RPC_E_DISCONNECTED?$AA@ 5f59388c     olemisc.obj
 0002:000058a0       ??_C@_0BM@KEOD@RPC_E_CONNECTION_TERMINATED?$AA@ 5f5938a0     olemisc.obj
 0002:000058bc       ??_C@_0BC@INIG@RPC_E_CLIENT_DIED?$AA@ 5f5938bc     olemisc.obj
 0002:000058d0       ??_C@_0CA@EKFA@RPC_E_CLIENT_CANTUNMARSHAL_DATA?$AA@ 5f5938d0     olemisc.obj
 0002:000058f0       ??_C@_0BO@IBCJ@RPC_E_CLIENT_CANTMARSHAL_DATA?$AA@ 5f5938f0     olemisc.obj
 0002:00005910       ??_C@_0BD@CBIE@RPC_E_CHANGED_MODE?$AA@ 5f593910     olemisc.obj
 0002:00005924       ??_C@_0BI@HEFH@RPC_E_CANTTRANSMIT_CALL?$AA@ 5f593924     olemisc.obj
 0002:0000593c       ??_C@_0BK@BFAI@RPC_E_CANTPOST_INSENDCALL?$AA@ 5f59393c     olemisc.obj
 0002:00005958       ??_C@_0CC@KEOJ@RPC_E_CANTCALLOUT_ININPUTSYNCCAL@ 5f593958     olemisc.obj
 0002:0000597c       ??_C@_0CB@IKHF@RPC_E_CANTCALLOUT_INEXTERNALCALL@ 5f59397c     olemisc.obj
 0002:000059a0       ??_C@_0BO@FIAD@RPC_E_CANTCALLOUT_INASYNCCALL?$AA@ 5f5939a0     olemisc.obj
 0002:000059c0       ??_C@_0BI@BODI@RPC_E_CANTCALLOUT_AGAIN?$AA@ 5f5939c0     olemisc.obj
 0002:000059d8       ??_C@_0BE@FCIF@RPC_E_CALL_REJECTED?$AA@ 5f5939d8     olemisc.obj
 0002:000059ec       ??_C@_0BE@NKHI@RPC_E_CALL_CANCELED?$AA@ 5f5939ec     olemisc.obj
 0002:00005a00       ??_C@_0BM@EEED@RPC_E_ATTEMPTED_MULTITHREAD?$AA@ 5f593a00     olemisc.obj
 0002:00005a1c       ??_C@_0BD@GKF@REGDB_E_WRITEREGDB?$AA@ 5f593a1c     olemisc.obj
 0002:00005a30       ??_C@_0BC@HJEG@REGDB_E_READREGDB?$AA@ 5f593a30     olemisc.obj
 0002:00005a44       ??_C@_0BD@NEAK@REGDB_E_KEYMISSING?$AA@ 5f593a44     olemisc.obj
 0002:00005a58       ??_C@_0BF@ENHM@REGDB_E_INVALIDVALUE?$AA@ 5f593a58     olemisc.obj
 0002:00005a70       ??_C@_0BC@EOK@REGDB_E_IIDNOTREG?$AA@ 5f593a70     olemisc.obj
 0002:00005a84       ??_C@_0BE@PII@REGDB_E_CLASSNOTREG?$AA@ 5f593a84     olemisc.obj
 0002:00005a98       ??_C@_0BB@ICH@OLEOBJ_E_NOVERBS?$AA@ 5f593a98     olemisc.obj
 0002:00005aac       ??_C@_0BF@CFIB@OLEOBJ_E_INVALIDVERB?$AA@ 5f593aac     olemisc.obj
 0002:00005ac4       ??_C@_0BD@HFND@OLE_E_WRONGCOMPOBJ?$AA@ 5f593ac4     olemisc.obj
 0002:00005ad8       ??_C@_0N@LJOM@OLE_E_STATIC?$AA@ 5f593ad8     olemisc.obj
 0002:00005ae8       ??_C@_0BK@GAIP@OLE_E_PROMPTSAVECANCELLED?$AA@ 5f593ae8     olemisc.obj
 0002:00005b04       ??_C@_0O@GNCI@OLE_E_OLEVERB?$AA@ 5f593b04     olemisc.obj
 0002:00005b14       ??_C@_0BB@JNNN@OLE_E_NOTRUNNING?$AA@ 5f593b14     olemisc.obj
 0002:00005b28       ??_C@_0BI@DOAN@OLE_E_NOT_INPLACEACTIVE?$AA@ 5f593b28     olemisc.obj
 0002:00005b40       ??_C@_0BA@KCAF@OLE_E_NOSTORAGE?$AA@ 5f593b40     olemisc.obj
 0002:00005b50       ??_C@_0BD@BCBD@OLE_E_NOCONNECTION?$AA@ 5f593b50     olemisc.obj
 0002:00005b64       ??_C@_0O@NJCH@OLE_E_NOCACHE?$AA@ 5f593b64     olemisc.obj
 0002:00005b74       ??_C@_0BC@JBBH@OLE_E_INVALIDRECT?$AA@ 5f593b74     olemisc.obj
 0002:00005b88       ??_C@_0BC@HBGB@OLE_E_INVALIDHWND?$AA@ 5f593b88     olemisc.obj
 0002:00005b9c       ??_C@_0BC@BFPC@OLE_E_ENUM_NOMORE?$AA@ 5f593b9c     olemisc.obj
 0002:00005bb0       ??_C@_0BA@IPMP@OLE_E_CLASSDIFF?$AA@ 5f593bb0     olemisc.obj
 0002:00005bc0       ??_C@_0BC@HFDL@OLE_E_CANTCONVERT?$AA@ 5f593bc0     olemisc.obj
 0002:00005bd4       ??_C@_0BG@PNJG@OLE_E_CANT_GETMONIKER?$AA@ 5f593bd4     olemisc.obj
 0002:00005bec       ??_C@_0BI@CFOJ@OLE_E_CANT_BINDTOSOURCE?$AA@ 5f593bec     olemisc.obj
 0002:00005c04       ??_C@_0M@OPML@OLE_E_BLANK?$AA@ 5f593c04     olemisc.obj
 0002:00005c10       ??_C@_0BJ@KCME@OLE_E_ADVISENOTSUPPORTED?$AA@ 5f593c10     olemisc.obj
 0002:00005c2c       ??_C@_0L@KKHN@OLE_E_ADVF?$AA@ 5f593c2c     olemisc.obj
 0002:00005c38       ??_C@_0BB@LKHO@MK_E_UNAVAILABLE?$AA@ 5f593c38     olemisc.obj
 0002:00005c4c       ??_C@_0M@FPAP@MK_E_SYNTAX?$AA@ 5f593c4c     olemisc.obj
 0002:00005c58       ??_C@_0O@JEII@MK_E_NOTBOUND?$AA@ 5f593c58     olemisc.obj
 0002:00005c68       ??_C@_0BB@CGPA@MK_E_NOTBINDABLE?$AA@ 5f593c68     olemisc.obj
 0002:00005c7c       ??_C@_0P@JOCA@MK_E_NOSTORAGE?$AA@ 5f593c7c     olemisc.obj
 0002:00005c8c       ??_C@_0O@EBPJ@MK_E_NOPREFIX?$AA@ 5f593c8c     olemisc.obj
 0002:00005c9c       ??_C@_0O@BMDP@MK_E_NOOBJECT?$AA@ 5f593c9c     olemisc.obj
 0002:00005cac       ??_C@_0P@GJCI@MK_E_NOINVERSE?$AA@ 5f593cac     olemisc.obj
 0002:00005cbc       ??_C@_0BD@DDAE@MK_E_NO_NORMALIZED?$AA@ 5f593cbc     olemisc.obj
 0002:00005cd0       ??_C@_0BB@NHEK@MK_E_NEEDGENERIC?$AA@ 5f593cd0     olemisc.obj
 0002:00005ce4       ??_C@_0BE@INIG@MK_E_MUSTBOTHERUSER?$AA@ 5f593ce4     olemisc.obj
 0002:00005cf8       ??_C@_0BG@ILAE@MK_E_INVALIDEXTENSION?$AA@ 5f593cf8     olemisc.obj
 0002:00005d10       ??_C@_0CH@PHBE@MK_E_INTERMEDIATEINTERFACENOTSUP@ 5f593d10     olemisc.obj
 0002:00005d38       ??_C@_0BG@JGDM@MK_E_EXCEEDEDDEADLINE?$AA@ 5f593d38     olemisc.obj
 0002:00005d50       ??_C@_0BI@MKAC@MK_E_ENUMERATION_FAILED?$AA@ 5f593d50     olemisc.obj
 0002:00005d68       ??_C@_0BF@NPHN@MK_E_CONNECTMANUALLY?$AA@ 5f593d68     olemisc.obj
 0002:00005d80       ??_C@_0BC@CLAA@MK_E_CANTOPENFILE?$AA@ 5f593d80     olemisc.obj
 0002:00005d94       ??_C@_0BD@GCCM@MEM_E_INVALID_SIZE?$AA@ 5f593d94     olemisc.obj
 0002:00005da8       ??_C@_0BD@IOEH@MEM_E_INVALID_ROOT?$AA@ 5f593da8     olemisc.obj
 0002:00005dbc       ??_C@_0BD@HMOK@MEM_E_INVALID_LINK?$AA@ 5f593dbc     olemisc.obj
 0002:00005dd0       ??_C@_0BG@NFLN@INPLACE_E_NOTUNDOABLE?$AA@ 5f593dd0     olemisc.obj
 0002:00005de8       ??_C@_0BG@NEEK@INPLACE_E_NOTOOLSPACE?$AA@ 5f593de8     olemisc.obj
 0002:00005e00       ??_C@_0L@OBAK@DV_E_TYMED?$AA@ 5f593e00     olemisc.obj
 0002:00005e0c       ??_C@_0P@CKCH@DV_E_STGMEDIUM?$AA@ 5f593e0c     olemisc.obj
 0002:00005e1c       ??_C@_0O@OFOL@DV_E_STATDATA?$AA@ 5f593e1c     olemisc.obj
 0002:00005e2c       ??_C@_0BD@IDLA@DV_E_NOIVIEWOBJECT?$AA@ 5f593e2c     olemisc.obj
 0002:00005e40       ??_C@_0M@LFPF@DV_E_LINDEX?$AA@ 5f593e40     olemisc.obj
 0002:00005e4c       ??_C@_0P@BDIB@DV_E_FORMATETC?$AA@ 5f593e4c     olemisc.obj
 0002:00005e5c       ??_C@_0BJ@MFG@DV_E_DVTARGETDEVICE_SIZE?$AA@ 5f593e5c     olemisc.obj
 0002:00005e78       ??_C@_0BE@IMCM@DV_E_DVTARGETDEVICE?$AA@ 5f593e78     olemisc.obj
 0002:00005e8c       ??_C@_0O@IIGO@DV_E_DVASPECT?$AA@ 5f593e8c     olemisc.obj
 0002:00005e9c       ??_C@_0BA@OMEF@DV_E_CLIPFORMAT?$AA@ 5f593e9c     olemisc.obj
 0002:00005eac       ??_C@_0BJ@KCOG@DRAGDROP_E_NOTREGISTERED?$AA@ 5f593eac     olemisc.obj
 0002:00005ec8       ??_C@_0BH@CFBH@DRAGDROP_E_INVALIDHWND?$AA@ 5f593ec8     olemisc.obj
 0002:00005ee0       ??_C@_0BN@GCLF@DRAGDROP_E_ALREADYREGISTERED?$AA@ 5f593ee0     olemisc.obj
 0002:00005f00       ??_C@_0BD@FPAE@DISP_E_UNKNOWNNAME?$AA@ 5f593f00     olemisc.obj
 0002:00005f14       ??_C@_0BD@EBLA@DISP_E_UNKNOWNLCID?$AA@ 5f593f14     olemisc.obj
 0002:00005f28       ??_C@_0BI@BKFO@DISP_E_UNKNOWNINTERFACE?$AA@ 5f593f28     olemisc.obj
 0002:00005f40       ??_C@_0BE@GINK@DISP_E_TYPEMISMATCH?$AA@ 5f593f40     olemisc.obj
 0002:00005f54       ??_C@_0BI@ONEA@DISP_E_PARAMNOTOPTIONAL?$AA@ 5f593f54     olemisc.obj
 0002:00005f6c       ??_C@_0BF@BKDN@DISP_E_PARAMNOTFOUND?$AA@ 5f593f6c     olemisc.obj
 0002:00005f84       ??_C@_0BA@GHFB@DISP_E_OVERFLOW?$AA@ 5f593f84     olemisc.obj
 0002:00005f94       ??_C@_0BG@DJIC@DISP_E_NOTACOLLECTION?$AA@ 5f593f94     olemisc.obj
 0002:00005fac       ??_C@_0BD@MFHE@DISP_E_NONAMEDARGS?$AA@ 5f593fac     olemisc.obj
 0002:00005fc0       ??_C@_0BG@DMGK@DISP_E_MEMBERNOTFOUND?$AA@ 5f593fc0     olemisc.obj
 0002:00005fd8       ??_C@_0BB@IEIB@DISP_E_EXCEPTION?$AA@ 5f593fd8     olemisc.obj
 0002:00005fec       ??_C@_0BC@FHKP@DISP_E_BADVARTYPE?$AA@ 5f593fec     olemisc.obj
 0002:00006000       ??_C@_0BF@IKPH@DISP_E_BADPARAMCOUNT?$AA@ 5f594000     olemisc.obj
 0002:00006018       ??_C@_0BA@DLMK@DISP_E_BADINDEX?$AA@ 5f594018     olemisc.obj
 0002:00006028       ??_C@_0BB@GP@DISP_E_BADCALLEE?$AA@ 5f594028     olemisc.obj
 0002:0000603c       ??_C@_0BF@PNAE@DISP_E_ARRAYISLOCKED?$AA@ 5f59403c     olemisc.obj
 0002:00006054       ??_C@_0BO@LMOC@CONVERT10_E_STG_NO_STD_STREAM?$AA@ 5f594054     olemisc.obj
 0002:00006074       ??_C@_0BE@NF@CONVERT10_E_STG_FMT?$AA@ 5f594074     olemisc.obj
 0002:00006088       ??_C@_0BO@MDDA@CONVERT10_E_STG_DIB_TO_BITMAP?$AA@ 5f594088     olemisc.obj
 0002:000060a8       ??_C@_0BK@PNGG@CONVERT10_E_OLESTREAM_PUT?$AA@ 5f5940a8     olemisc.obj
 0002:000060c4       ??_C@_0BK@IME@CONVERT10_E_OLESTREAM_GET?$AA@ 5f5940c4     olemisc.obj
 0002:000060e0       ??_C@_0BK@OPIG@CONVERT10_E_OLESTREAM_FMT?$AA@ 5f5940e0     olemisc.obj
 0002:000060fc       ??_C@_0CE@NBMK@CONVERT10_E_OLESTREAM_BITMAP_TO_@ 5f5940fc     olemisc.obj
 0002:00006120       ??_C@_0BD@IGGN@CO_E_WRONGOSFORAPP?$AA@ 5f594120     olemisc.obj
 0002:00006134       ??_C@_0BF@GIFE@CO_E_SERVER_STOPPING?$AA@ 5f594134     olemisc.obj
 0002:0000614c       ??_C@_0BJ@GJB@CO_E_SERVER_EXEC_FAILURE?$AA@ 5f59414c     olemisc.obj
 0002:00006168       ??_C@_0BF@PIKI@CO_E_SCM_RPC_FAILURE?$AA@ 5f594168     olemisc.obj
 0002:00006180       ??_C@_0P@DCAF@CO_E_SCM_ERROR?$AA@ 5f594180     olemisc.obj
 0002:00006190       ??_C@_0BI@LDEK@CO_E_OBJSRV_RPC_FAILURE?$AA@ 5f594190     olemisc.obj
 0002:000061a8       ??_C@_0P@OMLE@CO_E_OBJNOTREG?$AA@ 5f5941a8     olemisc.obj
 0002:000061b8       ??_C@_0BF@PKMO@CO_E_OBJNOTCONNECTED?$AA@ 5f5941b8     olemisc.obj
 0002:000061d0       ??_C@_0O@KJGN@CO_E_OBJISREG?$AA@ 5f5941d0     olemisc.obj
 0002:000061e0       ??_C@_0BE@EFPN@CO_E_NOTINITIALIZED?$AA@ 5f5941e0     olemisc.obj
 0002:000061f4       ??_C@_0P@KKED@CO_E_IIDSTRING?$AA@ 5f5941f4     olemisc.obj
 0002:00006204       ??_C@_0BA@DCHM@CO_E_ERRORINDLL?$AA@ 5f594204     olemisc.obj
 0002:00006214       ??_C@_0BA@PKPD@CO_E_ERRORINAPP?$AA@ 5f594214     olemisc.obj
 0002:00006224       ??_C@_0BB@DGAA@CO_E_DLLNOTFOUND?$AA@ 5f594224     olemisc.obj
 0002:00006238       ??_C@_0BB@JFMG@CO_E_CLASSSTRING?$AA@ 5f594238     olemisc.obj
 0002:0000624c       ??_C@_0BJ@DHFM@CO_E_CLASS_CREATE_FAILED?$AA@ 5f59424c     olemisc.obj
 0002:00006268       ??_C@_0BI@KADN@CO_E_CANTDETERMINECLASS?$AA@ 5f594268     olemisc.obj
 0002:00006280       ??_C@_0O@CEIB@CO_E_BAD_PATH?$AA@ 5f594280     olemisc.obj
 0002:00006290       ??_C@_0BC@MIJJ@CO_E_APPSINGLEUSE?$AA@ 5f594290     olemisc.obj
 0002:000062a4       ??_C@_0BB@PEGM@CO_E_APPNOTFOUND?$AA@ 5f5942a4     olemisc.obj
 0002:000062b8       ??_C@_0BB@EGCE@CO_E_APPDIDNTREG?$AA@ 5f5942b8     olemisc.obj
 0002:000062cc       ??_C@_0BI@LPFC@CO_E_ALREADYINITIALIZED?$AA@ 5f5942cc     olemisc.obj
 0002:000062e4       ??_C@_0BD@FIPH@CLIPBRD_E_CANT_SET?$AA@ 5f5942e4     olemisc.obj
 0002:000062f8       ??_C@_0BE@MCIO@CLIPBRD_E_CANT_OPEN?$AA@ 5f5942f8     olemisc.obj
 0002:0000630c       ??_C@_0BF@OABI@CLIPBRD_E_CANT_EMPTY?$AA@ 5f59430c     olemisc.obj
 0002:00006324       ??_C@_0BF@DMOK@CLIPBRD_E_CANT_CLOSE?$AA@ 5f594324     olemisc.obj
 0002:0000633c       ??_C@_0BD@DHGF@CLIPBRD_E_BAD_DATA?$AA@ 5f59433c     olemisc.obj
 0002:00006350       ??_C@_0BG@KBLK@CLASS_E_NOAGGREGATION?$AA@ 5f594350     olemisc.obj
 0002:00006368       ??_C@_0BK@OJDN@CLASS_E_CLASSNOTAVAILABLE?$AA@ 5f594368     olemisc.obj
 0002:00006384       ??_C@_0BI@LGBI@CACHE_E_NOCACHE_UPDATED?$AA@ 5f594384     olemisc.obj
 0002:0000639c       ??_C@_0P@IBAM@E_ACCESSDENIED?$AA@ 5f59439c     olemisc.obj
 0002:000063ac       ??_C@_06MPFC@E_FAIL?$AA@   5f5943ac     olemisc.obj
 0002:000063b4       ??_C@_07BBFK@E_ABORT?$AA@  5f5943b4     olemisc.obj
 0002:000063bc       ??_C@_08HCGG@E_HANDLE?$AA@ 5f5943bc     olemisc.obj
 0002:000063c8       ??_C@_09FCML@E_POINTER?$AA@ 5f5943c8     olemisc.obj
 0002:000063d4       ??_C@_0O@OKLN@E_NOINTERFACE?$AA@ 5f5943d4     olemisc.obj
 0002:000063e4       ??_C@_0N@OEAO@E_INVALIDARG?$AA@ 5f5943e4     olemisc.obj
 0002:000063f4       ??_C@_0O@EBOJ@E_OUTOFMEMORY?$AA@ 5f5943f4     olemisc.obj
 0002:00006404       ??_C@_09DGOK@E_NOTIMPL?$AA@ 5f594404     olemisc.obj
 0002:00006410       ??_C@_0N@KFCI@E_UNEXPECTED?$AA@ 5f594410     olemisc.obj
 0002:00006420       ??_C@_0BG@GHLI@VIEW_S_ALREADY_FROZEN?$AA@ 5f594420     olemisc.obj
 0002:00006438       ??_C@_0BA@ODMA@STG_S_CONVERTED?$AA@ 5f594438     olemisc.obj
 0002:00006448       ??_C@_0O@LMGC@OLEOBJ_S_LAST?$AA@ 5f594448     olemisc.obj
 0002:00006458       ??_C@_0BF@NEDD@OLEOBJ_S_INVALIDVERB?$AA@ 5f594458     olemisc.obj
 0002:00006470       ??_C@_0BF@ILAM@OLEOBJ_S_INVALIDHWND?$AA@ 5f594470     olemisc.obj
 0002:00006488       ??_C@_0BL@PKNP@OLEOBJ_S_CANNOT_DOVERB_NOW?$AA@ 5f594488     olemisc.obj
 0002:000064a4       ??_C@_0N@KKEF@OLE_S_USEREG?$AA@ 5f5944a4     olemisc.obj
 0002:000064b4       ??_C@_0N@ILOC@OLE_S_STATIC?$AA@ 5f5944b4     olemisc.obj
 0002:000064c4       ??_C@_0BF@NFAK@OLE_S_MAC_CLIPFORMAT?$AA@ 5f5944c4     olemisc.obj
 0002:000064dc       ??_C@_07MPHM@MK_S_US?$AA@  5f5944dc     olemisc.obj
 0002:000064e4       ??_C@_0BF@JEJH@MK_S_REDUCED_TO_SELF?$AA@ 5f5944e4     olemisc.obj
 0002:000064fc       ??_C@_0BO@JADJ@MK_S_MONIKERALREADYREGISTERED?$AA@ 5f5944fc     olemisc.obj
 0002:0000651c       ??_C@_07EGID@MK_S_ME?$AA@  5f59451c     olemisc.obj
 0002:00006524       ??_C@_08CAEH@MK_S_HIM?$AA@ 5f594524     olemisc.obj
 0002:00006530       ??_C@_0BE@DPEC@INPLACE_S_TRUNCATED?$AA@ 5f594530     olemisc.obj
 0002:00006544       ??_C@_0BN@CANI@DRAGDROP_S_USEDEFAULTCURSORS?$AA@ 5f594544     olemisc.obj
 0002:00006564       ??_C@_0BA@HKCB@DRAGDROP_S_DROP?$AA@ 5f594564     olemisc.obj
 0002:00006574       ??_C@_0BC@LMCE@DRAGDROP_S_CANCEL?$AA@ 5f594574     olemisc.obj
 0002:00006588       ??_C@_0BF@LEIP@DATA_S_SAMEFORMATETC?$AA@ 5f594588     olemisc.obj
 0002:000065a0       ??_C@_0BM@OOOI@CONVERT10_S_NO_PRESENTATION?$AA@ 5f5945a0     olemisc.obj
 0002:000065bc       ??_C@_0BO@HNEP@CACHE_S_SOMECACHES_NOTUPDATED?$AA@ 5f5945bc     olemisc.obj
 0002:000065dc       ??_C@_0BC@NMDD@CACHE_S_SAMECACHE?$AA@ 5f5945dc     olemisc.obj
 0002:000065f0       ??_C@_0BP@BLBM@CACHE_S_FORMATETC_NOTSUPPORTED?$AA@ 5f5945f0     olemisc.obj
 0002:00006610       ??_C@_07PDAH@S_FALSE?$AA@  5f594610     olemisc.obj
 0002:00006618       ??_C@_04JECD@S_OK?$AA@     5f594618     olemisc.obj
 0002:00006620       ??_C@_0BD@HIFJ@?$DMUnknown?5Facility?$DO?$AA@ 5f594620     olemisc.obj
 0002:00006634       ??_C@_0CE@IEAA@severity?3?5?$CFs?0?5facility?3?5?$CFs?5?$CI$?$CF08@ 5f594634     olemisc.obj
 0002:00006658       ??_C@_0BD@BOCN@range?3?5?$CFs?5?$CI$?$CF08lX?$CJ?$AA@ 5f594658     olemisc.obj
 0002:0000666c       ??_C@_0M@HCJP@?$CFs?5?$CI$?$CF08lX?$CJ?$AA@ 5f59466c     olemisc.obj
 0002:00006678       ??_C@_0DC@MCGB@Warning?3?5constructing?5COleExcept@ 5f594678     olemisc.obj
 0002:000066ac       ??_C@_0BA@DNCN@lpDevModeW?5?$CB?$DN?50?$AA@ 5f5946ac     olemisc.obj
 0002:000066bc       ??_C@_07LGIJ@DISPLAY?$AA@  5f5946bc     olemisc.obj
 0002:000066c4       ??_C@_0BA@BKOP@lpDevModeA?5?$CB?$DN?50?$AA@ 5f5946c4     olemisc.obj
 0002:000066d8       ?classCOleStreamFile@COleStreamFile@@2UCRuntimeClass@@B 5f5946d8     olestrm.obj
 0002:000066f0       ??_C@_0P@CGBG@COleStreamFile?$AA@ 5f5946f0     olestrm.obj
 0002:00006704       ??_7COleStreamFile@@6B@    5f594704     olestrm.obj
 0002:00006764       ??_C@_02PJJB@?$CC?6?$AA@   5f594764     olestrm.obj
 0002:00006768       ??_C@_0BF@MCAF@m_strStorageName?5?$DN?5?$CC?$AA@ 5f594768     olestrm.obj
 0002:00006780       ??_C@_0O@MEPH@m_lpStream?5?$DN?5?$AA@ 5f594780     olestrm.obj
 0002:00006790       ?classCOleServerDoc@COleServerDoc@@2UCRuntimeClass@@B 5f594790     olesvr1.obj
 0002:000067a8       ??_C@_0O@ELE@COleServerDoc?$AA@ 5f5947a8     olesvr1.obj
 0002:000067b8       ?interfaceMap@COleServerDoc@@1UAFX_INTERFACEMAP@@B 5f5947b8     olesvr1.obj
 0002:000067c0       ?_interfaceEntries@COleServerDoc@@0QBUAFX_INTERFACEMAP_ENTRY@@B 5f5947c0     olesvr1.obj
 0002:000067f8       ?messageMap@COleServerDoc@@1UAFX_MSGMAP@@B 5f5947f8     olesvr1.obj
 0002:00006800       ?_messageEntries@COleServerDoc@@0QBUAFX_MSGMAP_ENTRY@@B 5f594800     olesvr1.obj
 0002:0000687c       ??_7COleServerDoc@@6B@     5f59487c     olesvr1.obj
 0002:000069c8       ??_7XPersistStorage@COleServerDoc@@6B@ 5f5949c8     olesvr1.obj
 0002:000069f4       ??_7XOleObject@COleServerDoc@@6B@ 5f5949f4     olesvr1.obj
 0002:00006a58       ??_7XDataObject@COleServerDoc@@6B@ 5f594a58     olesvr1.obj
 0002:00006a8c       ??_7XOleInPlaceObject@COleServerDoc@@6B@ 5f594a8c     olesvr1.obj
 0002:00006ab4       ??_7XOleInPlaceActiveObject@COleServerDoc@@6B@ 5f594ab4     olesvr1.obj
 0002:00006adc       ??_C@_0DN@OECB@Warning?3?5zero?5?8zoom?5denominator?8@ 5f594adc     olesvr1.obj
 0002:00006b1c       ??_C@_0BM@MODF@?7failed?5to?5find?5item?5?8?$CFs?8?4?6?$AA@ 5f594b1c     olesvr1.obj
 0002:00006b38       ??_C@_0EA@NLBA@Warning?3?5default?5COleServerDoc?3?3@ 5f594b38     olesvr1.obj
 0002:00006b78       ??_C@_0CN@CBGM@Warning?3?5OnUpdateDocument?5failed@ 5f594b78     olesvr1.obj
 0002:00006ba8       ??_C@_0BC@JDAG@?6m_dwOrigStyle?5?$DN?5?$AA@ 5f594ba8     olesvr1.obj
 0002:00006bbc       ??_C@_0BD@IBCE@?6m_bCntrVisible?5?$DN?5?$AA@ 5f594bbc     olesvr1.obj
 0002:00006bd0       ??_C@_0BB@HMNG@?6m_strHostObj?5?$DN?5?$AA@ 5f594bd0     olesvr1.obj
 0002:00006be4       ??_C@_0BC@JBGM@m_lpClientSite?5?$DN?5?$AA@ 5f594be4     olesvr1.obj
 0002:00006bf8       ??_C@_0BJ@FFMJ@with?5no?5original?5parent?6?$AA@ 5f594bf8     olesvr1.obj
 0002:00006c14       ??_C@_0BI@GHAM@?6with?5original?5parent?3?5?$AA@ 5f594c14     olesvr1.obj
 0002:00006c2c       ??_C@_0BJ@CNKJ@?6with?5no?5in?9place?5frame?6?$AA@ 5f594c2c     olesvr1.obj
 0002:00006c48       ??_C@_0BH@HIOP@?6with?5in?9place?5frame?3?5?$AA@ 5f594c48     olesvr1.obj
 0002:00006c60       ?interfaceMap@COleServerItem@@1UAFX_INTERFACEMAP@@B 5f594c60     olesvr2.obj
 0002:00006c68       ?_interfaceEntries@COleServerItem@@0QBUAFX_INTERFACEMAP_ENTRY@@B 5f594c68     olesvr2.obj
 0002:00006c84       ??_7COleServerItem@@6B@    5f594c84     olesvr2.obj
 0002:00006d34       ??_7CItemDataSource@COleServerItem@@6B@ 5f594d34     olesvr2.obj
 0002:00006da0       ??_7XOleObject@COleServerItem@@6B@ 5f594da0     olesvr2.obj
 0002:00006e04       ??_7XDataObject@COleServerItem@@6B@ 5f594e04     olesvr2.obj
 0002:00006e34       ??_C@_0CO@KIPM@?7will?5not?5work?5with?5some?5apps?5li@ 5f594e34     olesvr2.obj
 0002:00006e64       ??_C@_0DA@CODI@Warning?3?5COleServerItem?5has?5no?5n@ 5f594e64     olesvr2.obj
 0002:00006e94       ??_C@_0CN@ELPE@Warning?3?5HIMETRIC?5natural?5size?5i@ 5f594e94     olesvr2.obj
 0002:00006ec4       ??_C@_0CN@HMAH@?7presentation?5metafile?5may?5be?5ba@ 5f594ec4     olesvr2.obj
 0002:00006ef4       ??_C@_0DA@GLHD@Warning?3?5OnGetExtent?5failed?5duri@ 5f594ef4     olesvr2.obj
 0002:00006f24       ??_C@_0CL@FNJD@calling?5COleServerItem?3?3OnDrawEx@ 5f594f24     olesvr2.obj
 0002:00006f50       ??_C@_0CM@KOCB@Warning?3?5unable?5to?5get?5moniker?5f@ 5f594f50     olesvr2.obj
 0002:00006f7c       ??_C@_0BF@OOCM@?6with?5m_dataSource?3?5?$AA@ 5f594f7c     olesvr2.obj
 0002:00006f94       ??_C@_0BJ@NNND@?6m_lpDataAdviseHolder?5?$DN?5?$AA@ 5f594f94     olesvr2.obj
 0002:00006fb0       ??_C@_0BI@EGAL@?6m_lpOleAdviseHolder?5?$DN?5?$AA@ 5f594fb0     olesvr2.obj
 0002:00006fc8       ??_C@_0BC@MFJM@?6m_strItemName?5?$DN?5?$AA@ 5f594fc8     olesvr2.obj
 0002:00006fdc       ??_C@_0BC@BDB@?6m_bAutoDelete?5?$DN?5?$AA@ 5f594fdc     olesvr2.obj
 0002:00006ff0       ??_C@_0BB@GJMC@m_bNeedUnlock?5?$DN?5?$AA@ 5f594ff0     olesvr2.obj
 0002:00007398       ??_C@_02MECO@?$CFd?$AA@    5f595398     olereg.obj
 0002:0000739c       ??_C@_0EA@JDBP@Warning?3?5StringFromCLSID?5failed?5@ 5f59539c     olereg.obj
 0002:000073dc       ??_C@_02EEIP@?4?$CK?$AA@   5f5953dc     olereg.obj
 0002:000073e0       ??_C@_0CD@JLBC@Warning?3?5skipping?5empty?5key?5?8?$CFs?8@ 5f5953e0     olereg.obj
 0002:00007404       ??_C@_0CP@ECBG@Error?3?5failed?5setting?5key?5?8?$CFs?8?5t@ 5f595404     olereg.obj
 0002:00007434       ??_C@_0BL@FDON@?7intended?5value?5was?5?8?$CFs?8?4?6?$AA@ 5f595434     olereg.obj
 0002:00007450       ??_C@_0DG@LPNG@Warning?3?5Leaving?5value?5?8?$CFs?8?5for?5@ 5f595450     olereg.obj
 0002:0000748c       ??_7COleTemplateServer@@6B@ 5f59548c     oletsvr.obj
 0002:00007500       ??_C@_0EI@FPDN@Error?3?5not?5enough?5information?5in@ 5f595500     oletsvr.obj
 0002:00007548       ??_C@_0EG@GJJP@Error?3?5not?5enough?5information?5in@ 5f595548     oletsvr.obj
 0002:000077f0       ??_C@_08KIPN@IID_NULL?$AA@ 5f5957f0     oleunk.obj
 0002:000077fc       ??_C@_0BB@GJDL@IID_IViewObject2?$AA@ 5f5957fc     oleunk.obj
 0002:00007810       ??_C@_0BA@IFJI@IID_IViewObject?$AA@ 5f595810     oleunk.obj
 0002:00007820       ??_C@_0N@LBDP@IID_IUnknown?$AA@ 5f595820     oleunk.obj
 0002:00007830       ??_C@_0BB@LCAG@IID_IStubManager?$AA@ 5f595830     oleunk.obj
 0002:00007844       ??_C@_0M@LNGD@IID_IStream?$AA@ 5f595844     oleunk.obj
 0002:00007850       ??_C@_0N@FNAH@IID_IStorage?$AA@ 5f595850     oleunk.obj
 0002:00007860       ??_C@_0BE@PIN@IID_IStdMarshalInfo?$AA@ 5f595860     oleunk.obj
 0002:00007874       ??_C@_0BI@NGAL@IID_IRunningObjectTable?$AA@ 5f595874     oleunk.obj
 0002:0000788c       ??_C@_0BE@JDJL@IID_IRunnableObject?$AA@ 5f59588c     oleunk.obj
 0002:000078a0       ??_C@_0N@CIC@IID_IRpcStub?$AA@ 5f5958a0     oleunk.obj
 0002:000078b0       ??_C@_0O@IJKE@IID_IRpcProxy?$AA@ 5f5958b0     oleunk.obj
 0002:000078c0       ??_C@_0BA@LKLP@IID_IRpcChannel?$AA@ 5f5958c0     oleunk.obj
 0002:000078d0       ??_C@_0BB@IOEJ@IID_IRootStorage?$AA@ 5f5958d0     oleunk.obj
 0002:000078e4       ??_C@_0BC@JDHA@IID_IProxyManager?$AA@ 5f5958e4     oleunk.obj
 0002:000078f8       ??_C@_0BD@DEIH@IID_IPersistStream?$AA@ 5f5958f8     oleunk.obj
 0002:0000790c       ??_C@_0BE@EKIO@IID_IPersistStorage?$AA@ 5f59590c     oleunk.obj
 0002:00007920       ??_C@_0BB@FCIP@IID_IPersistFile?$AA@ 5f595920     oleunk.obj
 0002:00007934       ??_C@_0N@EENH@IID_IPersist?$AA@ 5f595934     oleunk.obj
 0002:00007944       ??_C@_0BG@DMGB@IID_IParseDisplayName?$AA@ 5f595944     oleunk.obj
 0002:0000795c       ??_C@_0P@HPIB@IID_IPSFactory?$AA@ 5f59595c     oleunk.obj
 0002:0000796c       ??_C@_0P@CADM@IID_IOleWindow?$AA@ 5f59596c     oleunk.obj
 0002:0000797c       ??_C@_0BA@IADL@IID_IOlePresObj?$AA@ 5f59597c     oleunk.obj
 0002:0000798c       ??_C@_0P@OBGD@IID_IOleObject?$AA@ 5f59598c     oleunk.obj
 0002:0000799c       ??_C@_0BA@NNNA@IID_IOleManager?$AA@ 5f59599c     oleunk.obj
 0002:000079ac       ??_C@_0N@FOFL@IID_IOleLink?$AA@ 5f5959ac     oleunk.obj
 0002:000079bc       ??_C@_0BG@PBDH@IID_IOleItemContainer?$AA@ 5f5959bc     oleunk.obj
 0002:000079d4       ??_C@_0BI@OLNG@IID_IOleInPlaceUIWindow?$AA@ 5f5959d4     oleunk.obj
 0002:000079ec       ??_C@_0BE@OJME@IID_IOleInPlaceSite?$AA@ 5f5959ec     oleunk.obj
 0002:00007a00       ??_C@_0BG@JKFN@IID_IOleInPlaceObject?$AA@ 5f595a00     oleunk.obj
 0002:00007a18       ??_C@_0BF@IJNC@IID_IOleInPlaceFrame?$AA@ 5f595a18     oleunk.obj
 0002:00007a30       ??_C@_0BM@BGLO@IID_IOleInPlaceActiveObject?$AA@ 5f595a30     oleunk.obj
 0002:00007a4c       ??_C@_0BC@HLPG@IID_IOleContainer?$AA@ 5f595a4c     oleunk.obj
 0002:00007a60       ??_C@_0BD@NOBJ@IID_IOleClientSite?$AA@ 5f595a60     oleunk.obj
 0002:00007a74       ??_C@_0BF@MLIB@IID_IOleCacheControl?$AA@ 5f595a74     oleunk.obj
 0002:00007a8c       ??_C@_0P@FCPL@IID_IOleCache2?$AA@ 5f595a8c     oleunk.obj
 0002:00007a9c       ??_C@_0O@EFPD@IID_IOleCache?$AA@ 5f595a9c     oleunk.obj
 0002:00007aac       ??_C@_0BF@NNC@IID_IOleAdviseHolder?$AA@ 5f595aac     oleunk.obj
 0002:00007ac4       ??_C@_0N@DLFE@IID_IMoniker?$AA@ 5f595ac4     oleunk.obj
 0002:00007ad4       ??_C@_0BD@LLPF@IID_IMessageFilter?$AA@ 5f595ad4     oleunk.obj
 0002:00007ae8       ??_C@_0N@PDEB@IID_IMarshal?$AA@ 5f595ae8     oleunk.obj
 0002:00007af8       ??_C@_0M@BONK@IID_IMalloc?$AA@ 5f595af8     oleunk.obj
 0002:00007b04       ??_C@_0P@BFCK@IID_ILockBytes?$AA@ 5f595b04     oleunk.obj
 0002:00007b14       ??_C@_0BF@DHJA@IID_IInternalMoniker?$AA@ 5f595b14     oleunk.obj
 0002:00007b2c       ??_C@_0BB@EEMD@IID_IEnumVARIANT?$AA@ 5f595b2c     oleunk.obj
 0002:00007b40       ??_C@_0BB@OJAA@IID_IEnumUnknown?$AA@ 5f595b40     oleunk.obj
 0002:00007b54       ??_C@_0BA@IPPN@IID_IEnumString?$AA@ 5f595b54     oleunk.obj
 0002:00007b64       ??_C@_0BB@EFJF@IID_IEnumSTATSTG?$AA@ 5f595b64     oleunk.obj
 0002:00007b78       ??_C@_0BC@DOPN@IID_IEnumSTATDATA?$AA@ 5f595b78     oleunk.obj
 0002:00007b8c       ??_C@_0BB@OFCP@IID_IEnumOLEVERB?$AA@ 5f595b8c     oleunk.obj
 0002:00007ba0       ??_C@_0BB@GDGL@IID_IEnumMoniker?$AA@ 5f595ba0     oleunk.obj
 0002:00007bb4       ??_C@_0BA@CILK@IID_IEnumHolder?$AA@ 5f595bb4     oleunk.obj
 0002:00007bc4       ??_C@_0BB@HMKE@IID_IEnumGeneric?$AA@ 5f595bc4     oleunk.obj
 0002:00007bd8       ??_C@_0BD@IOFK@IID_IEnumFORMATETC?$AA@ 5f595bd8     oleunk.obj
 0002:00007bec       ??_C@_0BC@HEGK@IID_IEnumCallback?$AA@ 5f595bec     oleunk.obj
 0002:00007c00       ??_C@_0BA@LAN@IID_IDropTarget?$AA@ 5f595c00     oleunk.obj
 0002:00007c10       ??_C@_0BA@JHBI@IID_IDropSource?$AA@ 5f595c10     oleunk.obj
 0002:00007c20       ??_C@_0O@MMLG@IID_IDispatch?$AA@ 5f595c20     oleunk.obj
 0002:00007c30       ??_C@_0BB@PNNK@IID_IDfReserved3?$AA@ 5f595c30     oleunk.obj
 0002:00007c44       ??_C@_0BB@FHEN@IID_IDfReserved2?$AA@ 5f595c44     oleunk.obj
 0002:00007c58       ??_C@_0BB@KIPE@IID_IDfReserved1?$AA@ 5f595c58     oleunk.obj
 0002:00007c6c       ??_C@_0BB@PMNF@IID_IDebugStream?$AA@ 5f595c6c     oleunk.obj
 0002:00007c80       ??_C@_0L@JGFF@IID_IDebug?$AA@ 5f595c80     oleunk.obj
 0002:00007c8c       ??_C@_0BA@LAJJ@IID_IDataObject?$AA@ 5f595c8c     oleunk.obj
 0002:00007c9c       ??_C@_0BG@GJIF@IID_IDataAdviseHolder?$AA@ 5f595c9c     oleunk.obj
 0002:00007cb4       ??_C@_0L@GPEP@IID_IPrint?$AA@ 5f595cb4     oleunk.obj
 0002:00007cc0       ??_C@_0BF@IDLL@IID_IOleDocumentView?$AA@ 5f595cc0     oleunk.obj
 0002:00007cd8       ??_C@_0BF@LDPM@IID_IOleDocumentSite?$AA@ 5f595cd8     oleunk.obj
 0002:00007cf0       ??_C@_0BB@NKNJ@IID_IOleDocument?$AA@ 5f595cf0     oleunk.obj
 0002:00007d04       ??_C@_0BG@LOJB@IID_IOleCommandTarget?$AA@ 5f595d04     oleunk.obj
 0002:00007d1c       ??_C@_0BK@NIDF@IID_IEnumOleDocumentViews?$AA@ 5f595d1c     oleunk.obj
 0002:00007d38       ??_C@_0BG@HLGF@IID_IContinueCallback?$AA@ 5f595d38     oleunk.obj
 0002:00007d50       ??_C@_0BC@FAJA@IID_IClassFactory?$AA@ 5f595d50     oleunk.obj
 0002:00007d64       ??_C@_0N@MOKO@IID_IBindCtx?$AA@ 5f595d64     oleunk.obj
 0002:00007d74       ??_C@_0BB@LKJN@IID_IAdviseSink2?$AA@ 5f595d74     oleunk.obj
 0002:00007d88       ??_C@_0BA@CDIA@IID_IAdviseSink?$AA@ 5f595d88     oleunk.obj
 0002:00007d98       ??_C@_05GFGM@?$CF2?42X?$AA@ 5f595d98     oleunk.obj
 0002:00007da0       ??_C@_0BD@FJGA@?$CF8?48X?9?$CF4?44X?9?$CF4?44X?9?$AA@ 5f595da0     oleunk.obj
 0002:00007db8       ??_7CInnerUnknown@@6B@     5f595db8     oleunk.obj
 0002:00007dc8       ??_7COleException@@6B@     5f595dc8     oleunk.obj
 0002:00007de8       ?interfaceMap@CEnumOleVerb@@1UAFX_INTERFACEMAP@@B 5f595de8     oleverb.obj
 0002:00007df0       ?_interfaceEntries@CEnumOleVerb@@0QBUAFX_INTERFACEMAP_ENTRY@@B 5f595df0     oleverb.obj
 0002:00007e04       ??_7CEnumOleVerb@@6B@      5f595e04     oleverb.obj
 0002:00007e6c       ??_C@_0P@JAMM@?$DMunknown?5verb?$DO?$AA@ 5f595e6c     oleverb.obj
 0002:00007e80       ?classCRichEditView@CRichEditView@@2UCRuntimeClass@@B 5f595e80     viewrich.obj
 0002:00007e98       ??_C@_0O@OMMG@CRichEditView?$AA@ 5f595e98     viewrich.obj
 0002:00007ea8       ?classCRichEditDoc@CRichEditDoc@@2UCRuntimeClass@@B 5f595ea8     viewrich.obj
 0002:00007ec0       ??_C@_0N@HOLH@CRichEditDoc?$AA@ 5f595ec0     viewrich.obj
 0002:00007ed0       ??_C@_0BC@CJOP@CRichEditCntrItem?$AA@ 5f595ed0     viewrich.obj
 0002:00007ef0       ?interfaceMap@CRichEditView@@1UAFX_INTERFACEMAP@@B 5f595ef0     viewrich.obj
 0002:00007ef8       ?_interfaceEntries@CRichEditView@@0QBUAFX_INTERFACEMAP_ENTRY@@B 5f595ef8     viewrich.obj
 0002:00007f08       ?messageMap@CRichEditView@@1UAFX_MSGMAP@@B 5f595f08     viewrich.obj
 0002:00007f10       ?_messageEntries@CRichEditView@@0QBUAFX_MSGMAP_ENTRY@@B 5f595f10     viewrich.obj
 0002:000081e0       ??_C@_0BE@OBBF@commdlg_FindReplace?$AA@ 5f5961e0     viewrich.obj
 0002:000081f8       ??_7CRichEditView@@6B@     5f5961f8     viewrich.obj
 0002:00008334       ??_C@_08LOAO@RICHEDIT?$AA@ 5f596334     viewrich.obj
 0002:00008344       ??_7XRichEditOleCallback@CRichEditView@@6B@ 5f596344     viewrich.obj
 0002:0000837c       ??_7IRichEditOleCallback@@6B@ 5f59637c     viewrich.obj
 0002:000083b0       ??_C@_0BB@CEKL@End?5of?5Document?6?$AA@ 5f5963b0     viewrich.obj
 0002:000083c4       ??_C@_02MMHC@?6?$AN?$AA@   5f5963c4     viewrich.obj
 0002:000083c8       ??_C@_09EHNL@?6bNext?5?$DN?5?$AA@ 5f5963c8     viewrich.obj
 0002:000083d4       ??_C@_09GGLJ@?6bWord?5?$DN?5?$AA@ 5f5963d4     viewrich.obj
 0002:000083e0       ??_C@_09GAAD@?6bCase?5?$DN?5?$AA@ 5f5963e0     viewrich.obj
 0002:000083ec       ??_C@_0P@HKAL@?6strReplace?5?$DN?5?$AA@ 5f5963ec     viewrich.obj
 0002:000083fc       ??_C@_0M@FIBA@?6strFind?5?$DN?5?$AA@ 5f5963fc     viewrich.obj
 0002:00008408       ??_C@_0O@BAGE@?6bFindOnly?5?$DN?5?$AA@ 5f596408     viewrich.obj
 0002:00008418       ??_C@_0BE@BDLE@?6pFindReplaceDlg?5?$DN?5?$AA@ 5f596418     viewrich.obj
 0002:0000842c       ??_C@_0BG@LJPA@?6?5Static?5Member?5Data?3?$AA@ 5f59642c     viewrich.obj
 0002:00008444       ??_C@_0P@POCL@?6m_aPageStart?5?$AA@ 5f596444     viewrich.obj
 0002:00008458       ??_7CRichEditDoc@@6B@      5f596458     viewrich.obj
 0002:000085ac       ??_7CRichEditCntrItem@@6B@ 5f5965ac     viewrich.obj
 0002:00008698       ??_7_AFX_RICHEDIT_STATE@@6B@ 5f596698     viewrich.obj
 0002:0000869c       ??_C@_0CJ@KOGB@Info?3?5AfxDllCanUnloadNow?5returni@ 5f59669c     oledll.obj
 0002:000086cc       ??_7CTypeLibCacheMap@@6B@  5f5966cc     oletyplb.obj
 0002:000086e8       ?classCMonikerFile@CMonikerFile@@2UCRuntimeClass@@B 5f5966e8     olemon.obj
 0002:00008700       ??_C@_0N@CIKC@CMonikerFile?$AA@ 5f596700     olemon.obj
 0002:00008714       ??_7CMonikerFile@@6B@      5f596714     olemon.obj
 0002:0000878c       ??_7_AfxBindHost@@6B@      5f59678c     olemon.obj
 0002:000087a8       ??_7IBindHost@@6B@         5f5967a8     olemon.obj
 0002:000087c0       ??_C@_0O@KOAJ@?6m_Moniker?5?$DN?5?$AA@ 5f5967c0     olemon.obj
 0002:000087d0       ??_C@_0CH@FHFI@E?3?28168?2vc98?2mfc?2mfc?2include?2afx@ 5f5967d0     olemon.obj
 0002:000087f8       ?classCMonthCalCtrl@CMonthCalCtrl@@2UCRuntimeClass@@B 5f5967f8     winctrl5.obj
 0002:00008810       ??_C@_0O@MIA@CMonthCalCtrl?$AA@ 5f596810     winctrl5.obj
 0002:00008820       ?classCDateTimeCtrl@CDateTimeCtrl@@2UCRuntimeClass@@B 5f596820     winctrl5.obj
 0002:00008838       ??_C@_0O@BJFB@CDateTimeCtrl?$AA@ 5f596838     winctrl5.obj
 0002:00008858       ??_C@_0BC@GKLI@SysDateTimePick32?$AA@ 5f596858     winctrl5.obj
 0002:00008870       ??_7CDateTimeCtrl@@6B@     5f596870     winctrl5.obj
 0002:00008930       ??_C@_0O@NFNC@SysMonthCal32?$AA@ 5f596930     winctrl5.obj
 0002:00008944       ??_7CMonthCalCtrl@@6B@     5f596944     winctrl5.obj
 0002:00008a04       ??_C@_0EA@ILLA@Warning?3?5initial?5dialog?5data?5is?5@ 5f596a04     winctrl5.obj
 0002:00008a48       ?classCHtmlView@CHtmlView@@2UCRuntimeClass@@B 5f596a48     viewhtml.obj
 0002:00008a60       ??_C@_09GHGJ@CHtmlView?$AA@ 5f596a60     viewhtml.obj
 0002:00008a70       ?eventsinkMap@CHtmlView@@1UAFX_EVENTSINKMAP@@B 5f596a70     viewhtml.obj
 0002:00008a80       ?_eventsinkEntries@CHtmlView@@0QBUAFX_EVENTSINKMAP_ENTRY@@B 5f596a80     viewhtml.obj
 0002:00008d78       ??_C@_01KLAB@?$AL?$AA@     5f596d78     viewhtml.obj
 0002:00008d7c       ??_C@_02HJK@IK?$AA@        5f596d7c     viewhtml.obj
 0002:00008d80       ??_C@_07LMNJ@?7LLLLLK?$AA@ 5f596d80     viewhtml.obj
 0002:00008d88       ??_C@_02PINK@?7L?$AA@      5f596d88     viewhtml.obj
 0002:00008d8c       ??_C@_02JAPO@?$AD?$AL?$AA@ 5f596d8c     viewhtml.obj
 0002:00008d90       ??_C@_02MEEG@?$AD?$AD?$AA@ 5f596d90     viewhtml.obj
 0002:00008d94       ??_C@_01KLMK@?$AO?$AA@     5f596d94     viewhtml.obj
 0002:00008d98       ?messageMap@CHtmlView@@1UAFX_MSGMAP@@B 5f596d98     viewhtml.obj
 0002:00008da0       ?_messageEntries@CHtmlView@@0QBUAFX_MSGMAP_ENTRY@@B 5f596da0     viewhtml.obj
 0002:00008e1c       ??_7CHtmlView@@6B@         5f596e1c     viewhtml.obj
 0002:00008f80       ??_C@_0M@PCJJ@res?3?1?1?$CFs?1?$CFs?$AA@ 5f596f80     viewhtml.obj
 0002:00008f8c       ??_C@_0M@OAM@res?3?1?1?$CFs?1?$CFd?$AA@ 5f596f8c     viewhtml.obj
 0002:00008f98       ??_C@_0DM@FLMO@Dialog?5has?5OLE?5controls?0?5but?5no?5@ 5f596f98     occmgr.obj
 0002:00008fd4       ??_C@_0DG@GNMC@DLGINIT?5resource?5was?5found?0?5but?5@ 5f596fd4     occmgr.obj
 0002:0000900c       ??_C@_0CJ@GM@?$DO?$DO?$DO?5Is?5the?5control?5properly?5regi@ 5f59700c     occmgr.obj
 0002:00009038       ??_C@_0BK@BFDM@?$DO?$DO?$DO?5Result?5code?3?50x?$CF08lx?6?$AA@ 5f597038     occmgr.obj
 0002:00009054       ??_C@_0CI@LMIH@Unable?5to?5convert?5?$CC?$CFls?$CC?5to?5a?5cla@ 5f597054     occmgr.obj
 0002:0000907c       ??_C@_0DA@GCFP@Error?3?5no?5data?5exchange?5control?5@ 5f59707c     occmgr.obj
 0002:000090b0       ??_7COccManager@@6B@       5f5970b0     occmgr.obj
 0002:000090d8       ?interfaceMap@CEnumUnknown@@1UAFX_INTERFACEMAP@@B 5f5970d8     occcont.obj
 0002:000090e0       ?_interfaceEntries@CEnumUnknown@@0QBUAFX_INTERFACEMAP_ENTRY@@B 5f5970e0     occcont.obj
 0002:000090f0       ?dispatchMap@COleControlContainer@@1UAFX_DISPMAP@@B 5f5970f0     occcont.obj
 0002:00009100       ?_dispatchEntries@COleControlContainer@@0QBUAFX_DISPMAP_ENTRY@@B 5f597100     occcont.obj
 0002:00009120       ?interfaceMap@COleControlContainer@@1UAFX_INTERFACEMAP@@B 5f597120     occcont.obj
 0002:00009128       ?_interfaceEntries@COleControlContainer@@0QBUAFX_INTERFACEMAP_ENTRY@@B 5f597128     occcont.obj
 0002:00009140       ??_C@_0DN@NDMB@?$DO?$DO?$DO?5You?5should?5call?5it?5in?5your?5a@ 5f597140     occcont.obj
 0002:00009180       ??_C@_0DN@PMFD@Warning?3?5AfxEnableControlContain@ 5f597180     occcont.obj
 0002:000091c4       ??_7COleControlContainer@@6B@ 5f5971c4     occcont.obj
 0002:0000925c       ??_7XOleIPFrame@COleControlContainer@@6B@ 5f59725c     occcont.obj
 0002:0000929c       ??_7XOleContainer@COleControlContainer@@6B@ 5f59729c     occcont.obj
 0002:000092b8       ??_7CEnumUnknown@@6B@      5f5972b8     occcont.obj
 0002:00009320       _IID_IDataSourceListener   5f597320     occsite.obj
 0002:00009330       _IID_IDataSource           5f597330     occsite.obj
 0002:00009350       ?_afxAmbients@@3QBU__unnamed@@B 5f597350     occsite.obj
 0002:00009390       ?interfaceMap@COleControlSite@@1UAFX_INTERFACEMAP@@B 5f597390     occsite.obj
 0002:00009398       ?_interfaceEntries@COleControlSite@@0QBUAFX_INTERFACEMAP_ENTRY@@B 5f597398     occsite.obj
 0002:000093d8       _IID_IDCInfo               5f5973d8     occsite.obj
 0002:000093e8       _IID_IDataConvert          5f5973e8     occsite.obj
 0002:000093fc       ??_7COleControlSite@@6B@   5f5973fc     occsite.obj
 0002:000094c8       ??_7XOleClientSite@COleControlSite@@6B@ 5f5974c8     occsite.obj
 0002:000094f0       ??_7XOleIPSite@COleControlSite@@6B@ 5f5974f0     occsite.obj
 0002:00009530       ??_7XOleControlSite@COleControlSite@@6B@ 5f597530     occsite.obj
 0002:0000955c       ??_7XAmbientProps@COleControlSite@@6B@ 5f59755c     occsite.obj
 0002:0000957c       ??_7XPropertyNotifySink@COleControlSite@@6B@ 5f59757c     occsite.obj
 0002:00009594       ??_7XEventSink@COleControlSite@@6B@ 5f597594     occsite.obj
 0002:000095b4       ??_7XBoundObjectSite@COleControlSite@@6B@ 5f5975b4     occsite.obj
 0002:000095c8       ??_7XNotifyDBEvents@COleControlSite@@6B@ 5f5975c8     occsite.obj
 0002:000095f4       ??_7XRowsetNotify@COleControlSite@@6B@ 5f5975f4     occsite.obj
 0002:00009610       ??_7IBoundObjectSite@@6B@  5f597610     occsite.obj
 0002:00009624       ??_7INotifyDBEvents@@6B@   5f597624     occsite.obj
 0002:00009650       ??_7IRowsetNotify@@6B@     5f597650     occsite.obj
 0002:00009668       ??_C@_0EA@KGHC@IOleInPlaceObject?5not?5supported?5@ 5f597668     occsite.obj
 0002:000096a8       ??_C@_0CP@DGPI@Persistence?5not?5supported?5on?5OLE@ 5f5976a8     occsite.obj
 0002:000096d8       ??_C@_0CM@LFKC@InitNew?5or?5Load?5on?5OLE?5control?5?$CF@ 5f5976d8     occsite.obj
 0002:00009704       ??_C@_0CK@HBAC@SetClientSite?5on?5OLE?5control?5?$CFls@ 5f597704     occsite.obj
 0002:00009730       ??_C@_0CM@NHNE@?$DO?$DO?$DO?5Is?5the?5control?5is?5properly?5r@ 5f597730     occsite.obj
 0002:0000975c       ??_C@_0CN@DPNB@CoCreateInstance?5of?5OLE?5control?5@ 5f59775c     occsite.obj
 0002:0000978c       ??_C@_0CN@PLJA@Warning?3?5control?5has?5no?5IDispatc@ 5f59778c     occsite.obj
 0002:000097c0       ??_7CDataSourceControl@@6B@ 5f5977c0     occsite.obj
 0002:000097d8       ??_C@_0BF@GPJA@m_pAccessorInfo?5?$CB?$DN?50?$AA@ 5f5977d8     occsite.obj
 0002:000097f0       ??_C@_0L@DJPI@atldbcli?4h?$AA@ 5f5977f0     occsite.obj
 0002:000097fc       ??_C@_09HJIK@pUnk?5?$CB?$DN?50?$AA@ 5f5977fc     occsite.obj
 0002:00009808       ??_C@_0BF@IFGJ@m_pAccessorInfo?5?$DN?$DN?50?$AA@ 5f597808     occsite.obj
 0002:00009820       ??_C@_0BC@CNEL@m_nAccessors?5?$DN?$DN?50?$AA@ 5f597820     occsite.obj
 0002:00009834       ??_C@_0BA@EFBK@m_spRowset?5?$CB?$DN?50?$AA@ 5f597834     occsite.obj
 0002:00009844       ??_C@_0BB@OJDA@m_pAccessor?5?$CB?$DN?50?$AA@ 5f597844     occsite.obj
 0002:00009858       ??_C@_0CB@CEAB@GetData?5failed?5?9?5HRESULT?5?$DN?50x?$CFX?6@ 5f597858     occsite.obj
 0002:0000987c       ??_C@_05BFMC@ATL?3?5?$AA@  5f59787c     occsite.obj
 0002:00009884       ??_C@_09PLJB@atlbase?4h?$AA@ 5f597884     occsite.obj
 0002:00009890       ??_C@_0BI@CIAH@nBuf?5?$DM?5sizeof?$CIszBuffer?$CJ?$AA@ 5f597890     occsite.obj
 0002:000098a8       ??_C@_0BJ@NICA@nAccessor?5?$DM?5m_nAccessors?$AA@ 5f5978a8     occsite.obj
 0002:000098c4       ??_C@_0M@DLL@m_hRow?5?$CB?$DN?50?$AA@ 5f5978c4     occsite.obj
 0002:000098d0       ??_C@_0BH@DLBO@nAccessor?$DMm_nAccessors?$AA@ 5f5978d0     occsite.obj
 0002:000098e8       ??_C@_0CF@OLLL@Binding?5entry?5?$CFd?5failed?4?5Status?3@ 5f5978e8     occsite.obj
 0002:00009910       ??_C@_0P@NDGD@pAccessor?5?$CB?$DN?50?$AA@ 5f597910     occsite.obj
 0002:00009920       ??_C@_0BA@IMI@pHAccessor?5?$CB?$DN?50?$AA@ 5f597920     occsite.obj
 0002:00009930       ??_C@_0P@PHAP@pBindings?5?$CB?$DN?50?$AA@ 5f597930     occsite.obj
 0002:00009940       ??_C@_0O@JCIO@pBinding?5?$CB?$DN?50?$AA@ 5f597940     occsite.obj
 0002:00009950       ??_C@_0BD@PMHF@m_pColumnInfo?5?$CB?$DN?50?$AA@ 5f597950     occsite.obj
 0002:00009964       ??_C@_0CG@FMPB@Unsupported?5DBTYPE?5?$CI?$CFd?$CJ?5in?5colum@ 5f597964     occsite.obj
 0002:00009990       __real@8@4002a000000000000000 5f597990     occsite.obj
 0002:00009998       ??_C@_0N@CNMG@pStatus?5?$CB?$DN?50?$AA@ 5f597998     occsite.obj
 0002:000099a8       ??_C@_0BG@GDJO@m_nEntry?5?$DM?5m_nColumns?$AA@ 5f5979a8     occsite.obj
 0002:000099c0       ??_C@_04PPJP@p?$DN?$DN0?$AA@ 5f5979c0     occsite.obj
 0002:000099c8       ??_C@_04GBK@p?$CB?$DN0?$AA@ 5f5979c8     occsite.obj
 0002:000099d0       ??_C@_0DF@JBBA@m_pColumnInfo?$FLnColumn?$FN?4ulColumnS@ 5f5979d0     occsite.obj
 0002:00009a08       ??_C@_0L@IMO@pData?5?$CB?$DN?50?$AA@ 5f597a08     occsite.obj
 0002:00009a18       ??_7COleControlLock@@6B@   5f597a18     occlock.obj
 0002:00009a20       ?classCDocObjectServerItem@CDocObjectServerItem@@2UCRuntimeClass@@B 5f597a20     oledocob.obj
 0002:00009a38       ??_C@_0BF@FCEC@CDocObjectServerItem?$AA@ 5f597a38     oledocob.obj
 0002:00009a50       ?interfaceMap@CDocObjectServer@@1UAFX_INTERFACEMAP@@B 5f597a50     oledocob.obj
 0002:00009a58       ?_interfaceEntries@CDocObjectServer@@0QBUAFX_INTERFACEMAP_ENTRY@@B 5f597a58     oledocob.obj
 0002:00009a88       ?messageMap@CDocObjectServer@@1UAFX_MSGMAP@@B 5f597a88     oledocob.obj
 0002:00009a90       ?_messageEntries@CDocObjectServer@@0QBUAFX_MSGMAP_ENTRY@@B 5f597a90     oledocob.obj
 0002:00009aa8       ?classCDocObjectServer@CDocObjectServer@@2UCRuntimeClass@@B 5f597aa8     oledocob.obj
 0002:00009ac0       ??_C@_0BB@ICMG@CDocObjectServer?$AA@ 5f597ac0     oledocob.obj
 0002:00009ad8       ??_7CDocObjectServer@@6B@  5f597ad8     oledocob.obj
 0002:00009b44       ??_7XOleObject@CDocObjectServer@@6B@ 5f597b44     oledocob.obj
 0002:00009ba8       ??_7XOleDocument@CDocObjectServer@@6B@ 5f597ba8     oledocob.obj
 0002:00009bc4       ??_7XOleDocumentView@CDocObjectServer@@6B@ 5f597bc4     oledocob.obj
 0002:00009c08       ??_7XOleCommandTarget@CDocObjectServer@@6B@ 5f597c08     oledocob.obj
 0002:00009c20       ??_7XPrint@CDocObjectServer@@6B@ 5f597c20     oledocob.obj
 0002:00009c38       ??_C@_0DL@MFIO@Error?3?5An?5appropriate?5DocObject?5@ 5f597c38     oledocob.obj
 0002:00009c74       ??_C@_0EB@JHJF@CDocObjectServer?3?3XOleDocument?3?3@ 5f597c74     oledocob.obj
 0002:00009cb8       ??_C@_0P@PBDG@m_pViewSite?5?$DN?5?$AA@ 5f597cb8     oledocob.obj
 0002:00009cc8       ??_C@_0O@KKDN@m_pDocSite?5?$DN?5?$AA@ 5f597cc8     oledocob.obj
 0002:00009cdc       ??_7CDocObjectServerItem@@6B@ 5f597cdc     oledocob.obj
 0002:00009d8c       ??_7COleCmdUI@@6B@         5f597d8c     oledoctg.obj
 0002:00009da0       ??_C@_0EH@PLND@Warning?3?5IOleCommandTarget?3?3Exec@ 5f597da0     oledoctg.obj
 0002:00009de8       ?messageMap@COleDocIPFrameWnd@@1UAFX_MSGMAP@@B 5f597de8     oledocip.obj
 0002:00009df0       ?_messageEntries@COleDocIPFrameWnd@@0QBUAFX_MSGMAP_ENTRY@@B 5f597df0     oledocip.obj
 0002:00009e08       ?classCOleDocIPFrameWnd@COleDocIPFrameWnd@@2UCRuntimeClass@@B 5f597e08     oledocip.obj
 0002:00009e20       ??_C@_0BC@DHMK@COleDocIPFrameWnd?$AA@ 5f597e20     oledocip.obj
 0002:00009e38       ??_7COleDocIPFrameWnd@@6B@ 5f597e38     oledocip.obj
 0002:00009f58       ?interfaceMap@COleDocObjectItem@@1UAFX_INTERFACEMAP@@B 5f597f58     oledoccl.obj
 0002:00009f60       ?_interfaceEntries@COleDocObjectItem@@0QBUAFX_INTERFACEMAP_ENTRY@@B 5f597f60     oledoccl.obj
 0002:00009f70       ?classCOleDocObjectItem@COleDocObjectItem@@2UCRuntimeClass@@B 5f597f70     oledoccl.obj
 0002:00009f88       ??_C@_0BC@ODBE@COleDocObjectItem?$AA@ 5f597f88     oledoccl.obj
 0002:00009fa0       ??_7COleDocObjectItem@@6B@ 5f597fa0     oledoccl.obj
 0002:0000a090       ??_7XOleDocumentSite@COleDocObjectItem@@6B@ 5f598090     oledoccl.obj
 0002:0000a0a0       ??_C@_05JKGE@?$CFs?5?$CFs?$AA@ 5f5980a0     oledoccl.obj
 0002:0000a0a8       ??_C@_0DP@FKOC@Error?3?5COleDocObjectItem?3?3OnInse@ 5f5980a8     oledoccl.obj
 0002:0000a0e8       ??_C@_0CK@IGIM@IOleCommandTarget?3?3Exec?$CI?$CJ?5return@ 5f5980e8     oledoccl.obj
 0002:0000a114       ??_C@_0CA@HODD@IPrint?3?3Print?$CI?$CJ?5returned?5?$CF8?48X?6?$AA@ 5f598114     oledoccl.obj
 0002:0000a138       ?classCAsyncMonikerFile@CAsyncMonikerFile@@2UCRuntimeClass@@B 5f598138     oleasmon.obj
 0002:0000a150       ??_C@_0BC@OCAO@CAsyncMonikerFile?$AA@ 5f598150     oleasmon.obj
 0002:0000a168       ??_7CAsyncMonikerFile@@6B@ 5f598168     oleasmon.obj
 0002:0000a218       ??_7_AfxBindStatusCallback@@6B@ 5f598218     oleasmon.obj
 0002:0000a248       ??_7CInnerUnknown@_AfxBindStatusCallback@@6B@ 5f598248     oleasmon.obj
 0002:0000a258       ??_7IBindStatusCallback@@6B@ 5f598258     oleasmon.obj
 0002:0000a284       ??_C@_0CH@MDKP@?6m_pAfxBSCCurrent?9?$DOGetModuleStat@ 5f598284     oleasmon.obj
 0002:0000a2ac       ??_C@_0CP@JLPE@?6m_pAfxBSCCurrent?9?$DOGetpThisOfInn@ 5f5982ac     oleasmon.obj
 0002:0000a2dc       ??_C@_0CI@DKMD@?6m_pAfxBSCCurrent?9?$DOGetInnerUnkno@ 5f5982dc     oleasmon.obj
 0002:0000a304       ??_C@_0CO@OBDK@?6m_pAfxBSCCurrent?9?$DOGetControllin@ 5f598304     oleasmon.obj
 0002:0000a334       ??_C@_0CE@CFCF@?6m_pAfxBSCCurrent?9?$DOGetRefcount?$CI?$CJ@ 5f598334     oleasmon.obj
 0002:0000a358       ??_C@_0CB@HOPK@?6m_pAfxBSCCurrent?9?$DOGetOwner?$CI?$CJ?5?$DN?5@ 5f598358     oleasmon.obj
 0002:0000a37c       ??_C@_0BF@HPLG@?6m_pAfxBSCCurrent?5?$DN?5?$AA@ 5f59837c     oleasmon.obj
 0002:0000a394       ??_C@_0BB@DDKI@?6m_pFormatEtc?5?$DN?5?$AA@ 5f598394     oleasmon.obj
 0002:0000a3a8       ??_C@_0O@DNLE@?6m_Binding?5?$DN?5?$AA@ 5f5983a8     oleasmon.obj
 0002:0000a3b8       ?classCOleResizeBar@COleResizeBar@@2UCRuntimeClass@@B 5f5983b8     olebar.obj
 0002:0000a3d0       ??_C@_0O@BGCL@COleResizeBar?$AA@ 5f5983d0     olebar.obj
 0002:0000a3e0       ?messageMap@COleResizeBar@@1UAFX_MSGMAP@@B 5f5983e0     olebar.obj
 0002:0000a3e8       ?_messageEntries@COleResizeBar@@0QBUAFX_MSGMAP_ENTRY@@B 5f5983e8     olebar.obj
 0002:0000a494       ??_7COleResizeBar@@6B@     5f598494     olebar.obj
 0002:0000a57c       ??_C@_0BB@LGBH@AfxControlBar42d?$AA@ 5f59857c     olebar.obj
 0002:0000a590       ?classCOleControl@COleControl@@2UCRuntimeClass@@B 5f598590     ctlcore.obj
 0002:0000a5a8       ??_C@_0M@EGDG@COleControl?$AA@ 5f5985a8     ctlcore.obj
 0002:0000a5b8       ?messageMap@COleControl@@1UAFX_MSGMAP@@B 5f5985b8     ctlcore.obj
 0002:0000a5c0       ?_messageEntries@COleControl@@0QBUAFX_MSGMAP_ENTRY@@B 5f5985c0     ctlcore.obj
 0002:0000aa10       ?eventMap@COleControl@@1UAFX_EVENTMAP@@B 5f598a10     ctlcore.obj
 0002:0000aa20       ?interfaceMap@COleControl@@1UAFX_INTERFACEMAP@@B 5f598a20     ctlcore.obj
 0002:0000aa28       ?_interfaceEntries@COleControl@@0QBUAFX_INTERFACEMAP_ENTRY@@B 5f598a28     ctlcore.obj
 0002:0000aae4       ??_7COleControl@@6B@       5f598ae4     ctlcore.obj
 0002:0000ace0       ??_7XPersistStorage@COleControl@@6B@ 5f598ce0     ctlcore.obj
 0002:0000ad0c       ??_7XPersistStreamInit@COleControl@@6B@ 5f598d0c     ctlcore.obj
 0002:0000ad34       ??_7XPersistMemory@COleControl@@6B@ 5f598d34     ctlcore.obj
 0002:0000ad5c       ??_7XPersistPropertyBag@COleControl@@6B@ 5f598d5c     ctlcore.obj
 0002:0000ad7c       ??_7XOleObject@COleControl@@6B@ 5f598d7c     ctlcore.obj
 0002:0000ade0       ??_7XViewObject@COleControl@@6B@ 5f598de0     ctlcore.obj
 0002:0000ae20       ??_7XDataObject@COleControl@@6B@ 5f598e20     ctlcore.obj
 0002:0000ae54       ??_7XOleInPlaceObject@COleControl@@6B@ 5f598e54     ctlcore.obj
 0002:0000ae84       ??_7XOleInPlaceActiveObject@COleControl@@6B@ 5f598e84     ctlcore.obj
 0002:0000aeb0       ??_7XOleCache@COleControl@@6B@ 5f598eb0     ctlcore.obj
 0002:0000aed4       ??_7XOleControl@COleControl@@6B@ 5f598ed4     ctlcore.obj
 0002:0000aef4       ??_7XProvideClassInfo@COleControl@@6B@ 5f598ef4     ctlcore.obj
 0002:0000af0c       ??_7XSpecifyPropertyPages@COleControl@@6B@ 5f598f0c     ctlcore.obj
 0002:0000af20       ??_7XPerPropertyBrowsing@COleControl@@6B@ 5f598f20     ctlcore.obj
 0002:0000af40       ??_7XFontNotification@COleControl@@6B@ 5f598f40     ctlcore.obj
 0002:0000af58       ??_7XQuickActivate@COleControl@@6B@ 5f598f58     ctlcore.obj
 0002:0000af74       ??_7XPointerInactive@COleControl@@6B@ 5f598f74     ctlcore.obj
 0002:0000af8c       ??_C@_06NEML@?$CINULL?$CJ?$AA@ 5f598f8c     ctlcore.obj
 0002:0000af94       ??_C@_07KCHC@0x?$CF08lx?$AA@ 5f598f94     ctlcore.obj
 0002:0000af9c       ??_C@_0O@GJBD@?6m_bUIDead?5?$DN?5?$AA@ 5f598f9c     ctlcore.obj
 0002:0000afac       ??_C@_0BD@FKID@?6m_bSimpleFrame?5?$DN?5?$AA@ 5f598fac     ctlcore.obj
 0002:0000afc0       ??_C@_0BC@HCBP@?6m_bConvertVBX?5?$DN?5?$AA@ 5f598fc0     ctlcore.obj
 0002:0000afd4       ??_C@_0BG@DGPF@?6m_bChangingExtent?5?$DN?5?$AA@ 5f598fd4     ctlcore.obj
 0002:0000afec       ??_C@_0M@NMDE@?6m_bOpen?5?$DN?5?$AA@ 5f598fec     ctlcore.obj
 0002:0000aff8       ??_C@_0BL@GHHG@?6m_bPendingUIActivation?5?$DN?5?$AA@ 5f598ff8     ctlcore.obj
 0002:0000b014       ??_C@_0BA@BKLA@?6m_bUIActive?5?$DN?5?$AA@ 5f599014     ctlcore.obj
 0002:0000b024       ??_C@_0BF@HHGG@?6m_bInPlaceActive?5?$DN?5?$AA@ 5f599024     ctlcore.obj
 0002:0000b03c       ??_C@_0BD@IOMN@?6m_iDblClkState?5?$DN?5?$AA@ 5f59903c     ctlcore.obj
 0002:0000b050       ??_C@_0BD@GJIM@?6m_iButtonState?5?$DN?5?$AA@ 5f599050     ctlcore.obj
 0002:0000b064       ??_C@_0BH@KOMC@?6m_bCountOnAmbients?5?$DN?5?$AA@ 5f599064     ctlcore.obj
 0002:0000b07c       ??_C@_0BA@BOKL@?6m_bModified?5?$DN?5?$AA@ 5f59907c     ctlcore.obj
 0002:0000b08c       ??_C@_0BK@GELF@?6m_bFinalReleaseCalled?5?$DN?5?$AA@ 5f59908c     ctlcore.obj
 0002:0000b0a8       ??_C@_0P@KCGN@?6m_cyExtent?5?$DN?5?$AA@ 5f5990a8     ctlcore.obj
 0002:0000b0b8       ??_C@_0P@CNKP@?6m_cxExtent?5?$DN?5?$AA@ 5f5990b8     ctlcore.obj
 0002:0000b0c8       ??_C@_0M@HIFN@?6m_rcPos?5?$DN?5?$AA@ 5f5990c8     ctlcore.obj
 0002:0000b0d4       ??_C@_0BE@BOHF@?6m_cEventsFrozen?5?$DN?5?$AA@ 5f5990d4     ctlcore.obj
 0002:0000b0e8       ??_C@_0BG@IAJB@?6m_dwVersionLoaded?5?$DN?5?$AA@ 5f5990e8     ctlcore.obj
 0002:0000b100       ??_C@_0BC@BCLH@?6m_piidEvents?5?$DN?5?5?$AA@ 5f599100     ctlcore.obj
 0002:0000b114       ??_C@_0BC@EKAH@?6m_piidPrimary?5?$DN?5?$AA@ 5f599114     ctlcore.obj
 0002:0000b128       ??_C@_0BD@DIIE@?6m_pModuleState?5?$DN?5?$AA@ 5f599128     ctlcore.obj
 0002:0000b13c       ??_C@_0BB@KJOA@AfxOleControl42d?$AA@ 5f59913c     ctlcore.obj
 0002:0000b150       ??_C@_0DD@LJNL@Warning?3?5COleControl?3?3fastBeginP@ 5f599150     ctlcore.obj
 0002:0000b184       ??_C@_0DA@FOMA@Warning?3?5no?5message?5line?5prompt?5@ 5f599184     ctlcore.obj
 0002:0000b1b8       ??_7XEventConnPt@COleControl@@6B@ 5f5991b8     ctlcore.obj
 0002:0000b228       ??_7XPropConnPt@COleControl@@6B@ 5f599228     ctlcore.obj
 0002:0000b298       ??_7CReflectorWnd@@6B@     5f599298     ctlcore.obj
 0002:0000b35c       ??_7CParkingWnd@@6B@       5f59935c     ctlcore.obj
 0002:0000b420       ?connectionMap@COleControl@@1UAFX_CONNECTIONMAP@@B 5f599420     ctlconn.obj
 0002:0000b428       ?_connectionEntries@COleControl@@0QBUAFX_CONNECTIONMAP_ENTRY@@B 5f599428     ctlconn.obj
 0002:0000b438       ??_C@_0DE@KHI@?$HL?$CF08lX?9?$CF04X?9?$CF04X?9?$CF02X?$CF02X?9?$CF02X?$CF0@ 5f599438     ctldata.obj
 0002:0000b470       ??_7CControlDataSource@COleControl@@6B@ 5f599470     ctldata.obj
 0002:0000b4d8       ?_afxStockEvents@@3QBKB    5f5994d8     ctlevent.obj
 0002:0000b500       ??_C@_08EIKH@ComboBox?$AA@ 5f599500     ctlevent.obj
 0002:0000b50c       ??_C@_07NOMM@ListBox?$AA@  5f59950c     ctlevent.obj
 0002:0000b514       ??_C@_04EDLP@Edit?$AA@     5f599514     ctlevent.obj
 0002:0000b51c       ??_C@_07GFMD@?$ACH?6?$AO?$AO?$ADK?$AA@ 5f59951c     ctlevent.obj
 0002:0000b528       ?classCOleControlModule@COleControlModule@@2UCRuntimeClass@@B 5f599528     ctlmodul.obj
 0002:0000b540       ??_C@_0BC@KPIB@COleControlModule?$AA@ 5f599540     ctlmodul.obj
 0002:0000b558       ?messageMap@CControlFrameWnd@@1UAFX_MSGMAP@@B 5f599558     ctlframe.obj
 0002:0000b560       ?_messageEntries@CControlFrameWnd@@0QBUAFX_MSGMAP_ENTRY@@B 5f599560     ctlframe.obj
 0002:0000b5ac       ??_7CControlFrameWnd@@6B@  5f5995ac     ctlframe.obj
 0002:0000b670       ??_C@_09JNCA@AfxWnd42d?$AA@ 5f599670     ctlframe.obj
 0002:0000b67c       ??_C@_0CM@COH@Warning?3?5failed?5to?5create?5CContr@ 5f59967c     ctlframe.obj
 0002:0000b6a8       ?_afxFontDescDefault@@3UtagFONTDESC@@B 5f5996a8     ctlfont.obj
 0002:0000b6c8       ??_C@_1BM@LDDO@?$AAM?$AAS?$AA?5?$AAS?$AAa?$AAn?$AAs?$AA?5?$AAS?$AAe?$AAr?$AAi?$AAf?$AA?$AA@ 5f5996c8     ctlfont.obj
 0002:0000b6e8       ?interfaceMap@CEnumConnPoints@@1UAFX_INTERFACEMAP@@B 5f5996e8     oleconn.obj
 0002:0000b6f0       ?_interfaceEntries@CEnumConnPoints@@0QBUAFX_INTERFACEMAP_ENTRY@@B 5f5996f0     oleconn.obj
 0002:0000b700       ?interfaceMap@CEnumConnections@@1UAFX_INTERFACEMAP@@B 5f599700     oleconn.obj
 0002:0000b708       ?_interfaceEntries@CEnumConnections@@0QBUAFX_INTERFACEMAP_ENTRY@@B 5f599708     oleconn.obj
 0002:0000b71c       ??_7CConnectionPoint@@6B@  5f59971c     oleconn.obj
 0002:0000b78c       ??_7XConnPt@CConnectionPoint@@6B@ 5f59978c     oleconn.obj
 0002:0000b7b0       ??_7CEnumConnections@@6B@  5f5997b0     oleconn.obj
 0002:0000b81c       ??_7CEnumConnPoints@@6B@   5f59981c     oleconn.obj
 0002:0000b888       ??_7COleConnPtContainer@@6B@ 5f599888     oleconn.obj
 0002:0000b8a0       ?_afx_CLSID_StdPicture2_V1@@3U_GUID@@B 5f5998a0     ctlpropx.obj
 0002:0000b8b0       ??_C@_08ONGB@_ExtentY?$AA@ 5f5998b0     ctlpropx.obj
 0002:0000b8bc       ??_C@_08EHPG@_ExtentX?$AA@ 5f5998bc     ctlpropx.obj
 0002:0000b8c8       ??_C@_08PNKC@_Version?$AA@ 5f5998c8     ctlpropx.obj
 0002:0000b8d8       ??_7CArchivePropExchange@@6B@ 5f5998d8     ctlpropx.obj
 0002:0000b8f0       ??_7CResetPropExchange@@6B@ 5f5998f0     ctlpropx.obj
 0002:0000b908       ??_7CAsyncPropExchange@@6B@ 5f599908     ctlpropx.obj
 0002:0000b91c       ??_C@_0P@BMCK@FontStrikethru?$AA@ 5f59991c     ctlpropx.obj
 0002:0000b92c       ??_C@_0O@BGLC@FontUnderline?$AA@ 5f59992c     ctlpropx.obj
 0002:0000b93c       ??_C@_0L@ECJP@FontItalic?$AA@ 5f59993c     ctlpropx.obj
 0002:0000b948       ??_C@_08MING@FontBold?$AA@ 5f599948     ctlpropx.obj
 0002:0000b954       ??_C@_08ODBD@FontSize?$AA@ 5f599954     ctlpropx.obj
 0002:0000b960       ??_C@_08LHPB@FontName?$AA@ 5f599960     ctlpropx.obj
 0002:0000b96c       ??_C@_0BP@PMCF@No?5client?5site?5in?5PX_DataPath?$CB?$AA@ 5f59996c     ctlpropx.obj
 0002:0000b98c       ??_C@_0BL@CLJC@No?5control?5in?5PX_DataPath?$CB?$AA@ 5f59998c     ctlpropx.obj
 0002:0000b9a8       ?classCOlePropertyPage@COlePropertyPage@@2UCRuntimeClass@@B 5f5999a8     ctlppg.obj
 0002:0000b9c0       ??_C@_0BB@LGDG@COlePropertyPage?$AA@ 5f5999c0     ctlppg.obj
 0002:0000b9d8       ?_afxUpdateList@@3QBUNotifyInfo@@B 5f5999d8     ctlppg.obj
 0002:0000ba08       ?_afxNotifyList@@3QBUNotifyInfo@@B 5f599a08     ctlppg.obj
 0002:0000ba38       ??_C@_07EOKN@listbox?$AA@  5f599a38     ctlppg.obj
 0002:0000ba40       ??_C@_08PKA@combobox?$AA@  5f599a40     ctlppg.obj
 0002:0000ba4c       ??_C@_06LPKL@button?$AA@   5f599a4c     ctlppg.obj
 0002:0000ba54       ??_C@_04OJPN@edit?$AA@     5f599a54     ctlppg.obj
 0002:0000ba60       ?messageMap@COlePropertyPage@@1UAFX_MSGMAP@@B 5f599a60     ctlppg.obj
 0002:0000ba68       ?_messageEntries@COlePropertyPage@@0QBUAFX_MSGMAP_ENTRY@@B 5f599a68     ctlppg.obj
 0002:0000bab0       ?interfaceMap@COlePropertyPage@@1UAFX_INTERFACEMAP@@B 5f599ab0     ctlppg.obj
 0002:0000bab8       ?_interfaceEntries@COlePropertyPage@@0QBUAFX_INTERFACEMAP_ENTRY@@B 5f599ab8     ctlppg.obj
 0002:0000bad4       ??_7AFX_DDPDATA@@6B@       5f599ad4     ctlppg.obj
 0002:0000bae8       ??_C@_0CB@BHFH@?5Font?5should?5be?5MS?5Sans?5Serif?58?4@ 5f599ae8     ctlppg.obj
 0002:0000bb0c       ??_C@_0CM@IHAN@Property?5page?5?8?$CFs?8?5uses?5a?5nonsta@ 5f599b0c     ctlppg.obj
 0002:0000bb38       ??_C@_0N@KBJM@MS?5Shell?5Dlg?$AA@ 5f599b38     ctlppg.obj
 0002:0000bb48       ??_C@_04JCAN@Helv?$AA@     5f599b48     ctlppg.obj
 0002:0000bb50       ??_C@_0O@JHLN@MS?5Sans?5Serif?$AA@ 5f599b50     ctlppg.obj
 0002:0000bb60       ??_C@_0BG@PJFA@Property?5page?5warning?$AA@ 5f599b60     ctlppg.obj
 0002:0000bb78       ??_C@_0DG@EFMM@?5Dimensions?5should?5be?5250x62?5or?5@ 5f599b78     ctlppg.obj
 0002:0000bbb0       ??_C@_0N@FPKC@Warning?3?5?$CFs?6?$AA@ 5f599bb0     ctlppg.obj
 0002:0000bbc0       ??_C@_0CP@DBCC@Property?5page?5?8?$CFs?8?5has?5nonstanda@ 5f599bc0     ctlppg.obj
 0002:0000bbf4       ??_7COlePropertyPage@@6B@  5f599bf4     ctlppg.obj
 0002:0000bce0       ??_7XPropertyPage@COlePropertyPage@@6B@ 5f599ce0     ctlppg.obj
 0002:0000bd20       ??_7XPropNotifySink@COlePropertyPage@@6B@ 5f599d20     ctlppg.obj
 0002:0000bd34       ??_C@_04IGNI@EDIT?$AA@     5f599d34     ctlppg.obj
 0002:0000bd40       ?classCCachedDataPathProperty@CCachedDataPathProperty@@2UCRuntimeClass@@B 5f599d40     ctlprop.obj
 0002:0000bd58       ??_C@_0BI@EKAI@CCachedDataPathProperty?$AA@ 5f599d58     ctlprop.obj
 0002:0000bd70       ?classCDataPathProperty@CDataPathProperty@@2UCRuntimeClass@@B 5f599d70     ctlprop.obj
 0002:0000bd88       ??_C@_0BC@OBPM@CDataPathProperty?$AA@ 5f599d88     ctlprop.obj
 0002:0000bd9c       ?_afxAmbientFlags@@3QBKB   5f599d9c     ctlprop.obj
 0002:0000bdc4       ?_afxStockProps@@3QBKB     5f599dc4     ctlprop.obj
 0002:0000be14       ??_C@_0L@DKNK@Appearance?$AA@ 5f599e14     ctlprop.obj
 0002:0000be20       ??_C@_07FFME@Enabled?$AA@  5f599e20     ctlprop.obj
 0002:0000be28       ??_C@_0M@CCHM@BorderStyle?$AA@ 5f599e28     ctlprop.obj
 0002:0000be34       ??_C@_04CLJC@Font?$AA@     5f599e34     ctlprop.obj
 0002:0000be3c       ??_C@_09ODIG@BackColor?$AA@ 5f599e3c     ctlprop.obj
 0002:0000be48       ??_C@_09MDL@ForeColor?$AA@ 5f599e48     ctlprop.obj
 0002:0000be54       ??_C@_04BNNJ@Text?$AA@     5f599e54     ctlprop.obj
 0002:0000be5c       ??_C@_07FMLO@Caption?$AA@  5f599e5c     ctlprop.obj
 0002:0000be64       ??_C@_0M@GLJK@_StockProps?$AA@ 5f599e64     ctlprop.obj
 0002:0000be70       ??_C@_0P@CJNJ@?6m_strPath?5?$DN?5?$CC?$AA@ 5f599e70     ctlprop.obj
 0002:0000be80       ??_C@_0P@NANG@?6m_pControl?5?$DN?5?$AA@ 5f599e80     ctlprop.obj
 0002:0000be90       ?_afxFontDescHelv@@3UtagFONTDESC@@B 5f599e90     ctlpset.obj
 0002:0000beb0       ??_C@_19OFHG@?$AAH?$AAe?$AAl?$AAv?$AA?$AA@ 5f599eb0     ctlpset.obj
 0002:0000bec0       ?_afx_CLSID_StdPicture_V1@@3U_GUID@@B 5f599ec0     ctlpset.obj
 0002:0000bed0       ?_afx_CLSID_StdFont_V1@@3U_GUID@@B 5f599ed0     ctlpset.obj
 0002:0000bee0       ??_C@_0CH@PGBF@Failed?5to?5allocate?5memory?5for?5st@ 5f599ee0     ctlpset.obj
 0002:0000bf08       ??_C@_0BP@BOB@CreateStreamOnHGlobal?5failed?4?6?$AA@ 5f599f08     ctlpset.obj
 0002:0000bf28       ??_C@_0CF@PGGM@CPropertySet?3?3WriteToStream?5fail@ 5f599f28     ctlpset.obj
 0002:0000bf50       ??_C@_0BI@FPIA@DoPropExchange?5failed?4?6?$AA@ 5f599f50     ctlpset.obj
 0002:0000bf68       ??_C@_0CC@ONFG@CPropertySet?3?3AddSection?5failed?4@ 5f599f68     ctlpset.obj
 0002:0000bf8c       ??_C@_0CA@IILE@IStorage?3?3CreateStream?5failed?4?6?$AA@ 5f599f8c     ctlpset.obj
 0002:0000bfac       ??_C@_1BC@DBBK@?$AAC?$AAo?$AAn?$AAt?$AAe?$AAn?$AAt?$AAs?$AA?$AA@ 5f599fac     ctlpset.obj
 0002:0000bfc0       ??_C@_0CG@PJBL@StgCreateDocfileOnILockBytes?5fai@ 5f599fc0     ctlpset.obj
 0002:0000bfe8       ??_C@_0CD@ONN@CreateILockBytesOnHGlobal?5failed@ 5f599fe8     ctlpset.obj
 0002:0000c00c       ??_C@_0CP@LJIM@Propset?5only?5supported?5for?5strea@ 5f59a00c     ctlpset.obj
 0002:0000c03c       ??_C@_0DJ@GGJO@CLSID_PersistPropset?5section?5not@ 5f59a03c     ctlpset.obj
 0002:0000c078       ??_C@_0CG@KPJI@CPropertySet?3?3ReadFromStream?5fai@ 5f59a078     ctlpset.obj
 0002:0000c0a0       ??_C@_0CA@OFOL@Failed?5to?5open?5content?5stream?4?6?$AA@ 5f59a0a0     ctlpset.obj
 0002:0000c0c4       ??_7CPropsetPropExchange@@6B@ 5f59a0c4     ctlpset.obj
 0002:0000c0d8       ?_afxPropPageClass@@3QBQBDB 5f59a0d8     ctlreg.obj
 0002:0000c0e4       ??_C@_0BC@IJIG@InprocServer32?$AA?$CF2?$AA@ 5f59a0e4     ctlreg.obj
 0002:0000c0f8       ?_afxCtrlClassID@@3QBQBDB  5f59a0f8     ctlreg.obj
 0002:0000c120       ??_C@_0L@HJLI@Version?$AA?$CF7?$AA@ 5f59a120     ctlreg.obj
 0002:0000c12c       ??_C@_0L@GFBB@TypeLib?$AA?$CF6?$AA@ 5f59a12c     ctlreg.obj
 0002:0000c138       ??_C@_08CFN@Control?$AA?$AA@ 5f59a138     ctlreg.obj
 0002:0000c144       ??_C@_0BA@GBNN@MiscStatus?21?$AA?$CF5?$AA@ 5f59a144     ctlreg.obj
 0002:0000c154       ??_C@_0N@DJBP@MiscStatus?$AA0?$AA@ 5f59a154     ctlreg.obj
 0002:0000c164       ??_C@_0BH@FMOH@ToolboxBitmap32?$AA?$CF3?0?5?$CF4?$AA@ 5f59a164     ctlreg.obj
 0002:0000c17c       ??_C@_0BC@CDBB@InprocServer32?$AA?$CF3?$AA@ 5f59a17c     ctlreg.obj
 0002:0000c190       ??_C@_09KME@ProgID?$AA?$CF2?$AA@ 5f59a190     ctlreg.obj
 0002:0000c19c       ?_afxCtrlProgID@@3QBQBDB   5f59a19c     ctlreg.obj
 0002:0000c1a8       ??_C@_08GKNE@CLSID?$AA?$CF2?$AA@ 5f59a1a8     ctlreg.obj
 0002:0000c1b4       ??_C@_03MIFF@?$AA?$CF1?$AA@ 5f59a1b4     ctlreg.obj
 0002:0000c1b8       ??_C@_0L@EBJK@Interface?2?$AA@ 5f59a1b8     ctlreg.obj
 0002:0000c1c4       ??_C@_0CO@JGLP@Warning?3?5Could?5not?5load?5type?5lib@ 5f59a1c4     ctlreg.obj
 0002:0000c1f4       ??_C@_05PFD@win32?$AA@     5f59a1f4     ctlreg.obj
 0002:0000c1fc       ??_C@_05IIFK@win16?$AA@    5f59a1fc     ctlreg.obj
 0002:0000c204       ??_C@_05MNJD@FLAGS?$AA@    5f59a204     ctlreg.obj
 0002:0000c20c       ??_C@_07GOJG@HELPDIR?$AA@  5f59a20c     ctlreg.obj
 0002:0000c214       ??_C@_0L@IMLO@TYPELIB?2?$CFs?$AA@ 5f59a214     ctlreg.obj
 0002:0000c220       ??_C@_0P@CMNN@ThreadingModel?$AA@ 5f59a220     ctlreg.obj
 0002:0000c230       ??_C@_0P@IIOA@InprocServer32?$AA@ 5f59a230     ctlreg.obj
 0002:0000c240       ??_C@_08BJKM@CLSID?2?$CFs?$AA@ 5f59a240     ctlreg.obj
 0002:0000c24c       ??_C@_05LFKM@?$CFd?4?$CFd?$AA@ 5f59a24c     ctlreg.obj
 0002:0000c254       ??_C@_0BA@OPOP@ToolboxBitmap32?$AA@ 5f59a254     ctlreg.obj
 0002:0000c264       ??_C@_0M@KNGN@CLSID?2?$CFs?2?$CFs?$AA@ 5f59a264     ctlreg.obj
 0002:0000c270       ??_C@_0N@OPAM@InprocServer?$AA@ 5f59a270     ctlreg.obj
 0002:0000c280       ?_afxResizeStyle@@3HB      5f59a280     ctltrack.obj
 0002:0000c288       ??_7CControlRectTracker@@6B@ 5f59a288     ctltrack.obj
 0002:0000c2a0       ??_C@_0BN@FGCC@CProperty?3?3AllocValue?5failed?$AA@ 5f59a2a0     olepset.obj
 0002:0000c2c0       ??_C@_0CF@KMMN@Write?5of?5section?5header?5failed?5?$CI@ 5f59a2c0     olepset.obj
 0002:0000c2e8       ??_C@_0BI@HHCD@Write?5of?5?8pido?8?5failed?6?$AA@ 5f59a2e8     olepset.obj
 0002:0000c300       ??_C@_0CI@DHPP@Warning?3?5Wrote?5empty?5property?5se@ 5f59a300     olepset.obj
 0002:0000c328       ??_C@_0CF@MDDL@Write?5of?5section?5header?5failed?5?$CI@ 5f59a328     olepset.obj
 0002:0000c350       ??_C@_0CE@HOIF@Failed?5to?5add?5entry?5to?5dictionar@ 5f59a350     olepset.obj
 0002:0000c374       ??_C@_0CC@LPMO@Read?5of?5dictionary?5entry?5failed?4@ 5f59a374     olepset.obj
 0002:0000c398       ??_C@_0CD@INEG@Read?5of?5dictionary?5header?5failed@ 5f59a398     olepset.obj
 0002:0000c3bc       ??_C@_0CD@EHMG@Write?5of?5dictionary?5entry?5failed@ 5f59a3bc     olepset.obj
 0002:0000c3e0       ??_C@_0CE@EELO@Write?5of?5dictionary?5header?5faile@ 5f59a3e0     olepset.obj
 0002:0000c404       ??_C@_0BJ@FAOI@Write?5of?5?8fido?8?5failed?4?6?$AA@ 5f59a404     olepset.obj
 0002:0000c420       ??_C@_0CE@HDCK@Warning?3?5Wrote?5empty?5property?5se@ 5f59a420     olepset.obj
 0002:0000c444       ??_C@_0CG@DNK@Write?5of?5Property?5Set?5Header?5fai@ 5f59a444     olepset.obj
 0002:0000c470       ?_afx_CLSID_BlobProperty@@3U_GUID@@B 5f59a470     ctlpbag.obj
 0002:0000c484       ??_7CBlobProperty@@6B@     5f59a484     ctlpbag.obj
 0002:0000c4a8       ??_7CPropbagPropExchange@@6B@ 5f59a4a8     ctlpbag.obj
 0002:0000c4c0       ??_7_AFXCTL_AMBIENT_CACHE@@6B@ 5f59a4c0     ctlquick.obj
 0002:0000c4c8       ?classCWindowlessDC@CWindowlessDC@@2UCRuntimeClass@@B 5f59a4c8     ctlnownd.obj
 0002:0000c4e0       ??_C@_0O@FBOP@CWindowlessDC?$AA@ 5f59a4e0     ctlnownd.obj
 0002:0000c4f4       ??_7CWindowlessDC@@6B@     5f59a4f4     ctlnownd.obj
 0002:0000c570       ?classCColorPropPage@CColorPropPage@@2UCRuntimeClass@@B 5f59a570     ppgcolor.obj
 0002:0000c588       ??_C@_0P@PKCG@CColorPropPage?$AA@ 5f59a588     ppgcolor.obj
 0002:0000c5b0       ?guid@CColorPropPage@@2U_GUID@@B 5f59a5b0     ppgcolor.obj
 0002:0000c5c0       ?messageMap@CColorPropPage@@1UAFX_MSGMAP@@B 5f59a5c0     ppgcolor.obj
 0002:0000c5c8       ?_messageEntries@CColorPropPage@@0QBUAFX_MSGMAP_ENTRY@@B 5f59a5c8     ppgcolor.obj
 0002:0000c790       ?_afxSysColorsList@@3QBUSysColorsInfo@@B 5f59a790     ppgcolor.obj
 0002:0000c844       ??_7CColorButton@@6B@      5f59a844     ppgcolor.obj
 0002:0000c90c       ??_7CColorPropPage@@6B@    5f59a90c     ppgcolor.obj
 0002:0000c9fc       ??_7CColorPropPageFactory@CColorPropPage@@6B@ 5f59a9fc     ppgcolor.obj
 0002:0000ca70       ?classCFontPropPage@CFontPropPage@@2UCRuntimeClass@@B 5f59aa70     ppgfont.obj
 0002:0000ca88       ??_C@_0O@IMID@CFontPropPage?$AA@ 5f59aa88     ppgfont.obj
 0002:0000cab0       ?guid@CFontPropPage@@2U_GUID@@B 5f59aab0     ppgfont.obj
 0002:0000cac0       ?messageMap@CFontPropPage@@1UAFX_MSGMAP@@B 5f59aac0     ppgfont.obj
 0002:0000cac8       ?_messageEntries@CFontPropPage@@0QBUAFX_MSGMAP_ENTRY@@B 5f59aac8     ppgfont.obj
 0002:0000cbd4       ??_7CFontPropPage@@6B@     5f59abd4     ppgfont.obj
 0002:0000ccc8       ??_7CSizeComboBox@@6B@     5f59acc8     ppgfont.obj
 0002:0000cd9c       ??_7CFontComboBox@@6B@     5f59ad9c     ppgfont.obj
 0002:0000ce70       ??_7CFontPropPageFactory@CFontPropPage@@6B@ 5f59ae70     ppgfont.obj
 0002:0000cee8       ?classCPicturePropPage@CPicturePropPage@@2UCRuntimeClass@@B 5f59aee8     ppgpict.obj
 0002:0000cf00       ??_C@_0BB@EHCI@CPicturePropPage?$AA@ 5f59af00     ppgpict.obj
 0002:0000cf30       ?guid@CPicturePropPage@@2U_GUID@@B 5f59af30     ppgpict.obj
 0002:0000cf40       ?messageMap@CPicturePropPage@@1UAFX_MSGMAP@@B 5f59af40     ppgpict.obj
 0002:0000cf48       ?_messageEntries@CPicturePropPage@@0QBUAFX_MSGMAP_ENTRY@@B 5f59af48     ppgpict.obj
 0002:0000cfc4       ??_7CPicturePropPage@@6B@  5f59afc4     ppgpict.obj
 0002:0000d0b4       ??_7CPicturePropPageFactory@CPicturePropPage@@6B@ 5f59b0b4     ppgpict.obj
 0002:0000d128       ?classCStockPropPage@CStockPropPage@@2UCRuntimeClass@@B 5f59b128     ppgstock.obj
 0002:0000d140       ??_C@_0P@GBDL@CStockPropPage?$AA@ 5f59b140     ppgstock.obj
 0002:0000d150       ?messageMap@CStockPropPage@@1UAFX_MSGMAP@@B 5f59b150     ppgstock.obj
 0002:0000d158       ?_messageEntries@CStockPropPage@@0QBUAFX_MSGMAP_ENTRY@@B 5f59b158     ppgstock.obj
 0002:0000d174       ??_7CStockPropPage@@6B@    5f59b174     ppgstock.obj
 0002:0000d25c       ??_C@_02NCNO@B?$AC?$AA@    5f59b25c     ctlinl.obj
 0002:0000d260       ??_C@_01PAOO@B?$AA@        5f59b260     ctlinl.obj
 0002:0000d264       ??_C@_04CKMP@?$AC?$AC?$AD?$AD?$AA@ 5f59b264     ctlinl.obj
 0002:0000d26c       ??_C@_01PPLJ@?$AD?$AA@     5f59b26c     ctlinl.obj
 0002:0000d274       ??_7CPropExchange@@6B@     5f59b274     ctlinl.obj
 0002:0000d28c       ??_7CDataPathProperty@@6B@ 5f59b28c     ctlinl.obj
 0002:0000d34c       ??_7CCachedDataPathProperty@@6B@ 5f59b34c     ctlinl.obj
 0002:0000d438       ??_7type_info@@6B@         5f59b438     msvcrtd:ti_inst.obj
 0002:0000d43c       ??_C@_08JKC@crtdll?4c?$AA@ 5f59b43c     msvcrtd:crtdll.obj
 0002:0000d448       _IID_IOleInPlaceSite       5f59b448     uuid:oleidl_i_guid15.obj
 0002:0000d458       _IID_IOleWindow            5f59b458     uuid:oleidl_i_guid8.obj
 0002:0000d468       _IID_IAdviseSink           5f59b468     uuid:objidl_i_guid27.obj
 0002:0000d478       _IID_IOleClientSite        5f59b478     uuid:oleidl_i_guid6.obj
 0002:0000d488       _GUID_NULL                 5f59b488     uuid:cguid_i_guid0.obj
 0002:0000d498       _IID_IOleLink              5f59b498     uuid:oleidl_i_guid9.obj
 0002:0000d4a8       _IID_IViewObject2          5f59b4a8     uuid:oleidl_i_guid18.obj
 0002:0000d4b8       _IID_IOleObject            5f59b4b8     uuid:oleidl_i_guid7.obj
 0002:0000d4c8       _IID_IUnknown              5f59b4c8     uuid:unknwn_i_guid0.obj
 0002:0000d4d8       _IID_IPersistStorage       5f59b4d8     uuid:objidl_i_guid22.obj
 0002:0000d4e8       _IID_IPersistStream        5f59b4e8     uuid:objidl_i_guid13.obj
 0002:0000d4f8       _IID_IPersistStreamInit    5f59b4f8     uuid:ocidl_i_guid16.obj
 0002:0000d508       _IID_IOleCache             5f59b508     uuid:oleidl_i_guid1.obj
 0002:0000d518       _IID_IDataObject           5f59b518     uuid:objidl_i_guid31.obj
 0002:0000d528       _IID_IOleInPlaceFrame      5f59b528     uuid:oleidl_i_guid13.obj
 0002:0000d538       _IID_IOleInPlaceUIWindow   5f59b538     uuid:oleidl_i_guid11.obj
 0002:0000d548       _IID_IOleInPlaceObject     5f59b548     uuid:oleidl_i_guid14.obj
 0002:0000d558       _IID_IOleCommandTarget     5f59b558     uuid:docobj_i_guid6.obj
 0002:0000d568       _IID_IEnumFORMATETC        5f59b568     uuid:objidl_i_guid24.obj
 0002:0000d578       _IID_IDispatch             5f59b578     uuid:oaidl_i_guid4.obj
 0002:0000d588       _IID_IDropSource           5f59b588     uuid:oleidl_i_guid19.obj
 0002:0000d598       _IID_IDropTarget           5f59b598     uuid:oleidl_i_guid20.obj
 0002:0000d5a8       _IID_IMessageFilter        5f59b5a8     uuid:objidl_i_guid33.obj
 0002:0000d5b8       _IID_IClassFactory2        5f59b5b8     uuid:ocidl_i_guid4.obj
 0002:0000d5c8       _IID_IClassFactory         5f59b5c8     uuid:unknwn_i_guid1.obj
 0002:0000d5d8       _IID_IOleItemContainer     5f59b5d8     uuid:oleidl_i_guid10.obj
 0002:0000d5e8       _IID_IOleContainer         5f59b5e8     uuid:oleidl_i_guid5.obj
 0002:0000d5f8       _IID_IParseDisplayName     5f59b5f8     uuid:oleidl_i_guid4.obj
 0002:0000d608       _IID_IPersistFile          5f59b608     uuid:objidl_i_guid21.obj
 0002:0000d618       _IID_IPersist              5f59b618     uuid:objidl_i_guid12.obj
 0002:0000d628       _IID_IStorage              5f59b628     uuid:objidl_i_guid20.obj
 0002:0000d638       _IID_IOleInPlaceActiveObject 5f59b638     uuid:oleidl_i_guid12.obj
 0002:0000d648       _IID_IOleDocumentSite      5f59b648     uuid:docobj_i_guid1.obj
 0002:0000d658       _IID_IViewObject           5f59b658     uuid:oleidl_i_guid17.obj
 0002:0000d668       _IID_IStubManager          5f59b668     uuid:cguid_i_guid3.obj
 0002:0000d678       _IID_IStream               5f59b678     uuid:objidl_i_guid18.obj
 0002:0000d688       _IID_IStdMarshalInfo       5f59b688     uuid:objidl_i_guid3.obj
 0002:0000d698       _IID_IRunningObjectTable   5f59b698     uuid:objidl_i_guid11.obj
 0002:0000d6a8       _IID_IRunnableObject       5f59b6a8     uuid:objidl_i_guid10.obj
 0002:0000d6b8       _IID_IRpcStub              5f59b6b8     uuid:cguid_i_guid2.obj
 0002:0000d6c8       _IID_IRpcProxy             5f59b6c8     uuid:cguid_i_guid4.obj
 0002:0000d6d8       _IID_IRpcChannel           5f59b6d8     uuid:cguid_i_guid1.obj
 0002:0000d6e8       _IID_IRootStorage          5f59b6e8     uuid:objidl_i_guid26.obj
 0002:0000d6f8       _IID_IProxyManager         5f59b6f8     uuid:cguid_i_guid5.obj
 0002:0000d708       _IID_IPSFactory            5f59b708     uuid:cguid_i_guid6.obj
 0002:0000d718       _IID_IOlePresObj           5f59b718     uuid:cguid_i_guid18.obj
 0002:0000d728       _IID_IOleManager           5f59b728     uuid:cguid_i_guid17.obj
 0002:0000d738       _IID_IOleCacheControl      5f59b738     uuid:oleidl_i_guid3.obj
 0002:0000d748       _IID_IOleCache2            5f59b748     uuid:oleidl_i_guid2.obj
 0002:0000d758       _IID_IOleAdviseHolder      5f59b758     uuid:oleidl_i_guid0.obj
 0002:0000d768       _IID_IMoniker              5f59b768     uuid:objidl_i_guid14.obj
 0002:0000d778       _IID_IMarshal              5f59b778     uuid:objidl_i_guid0.obj
 0002:0000d788       _IID_IMalloc               5f59b788     uuid:objidl_i_guid1.obj
 0002:0000d798       _IID_ILockBytes            5f59b798     uuid:objidl_i_guid23.obj
 0002:0000d7a8       _IID_IInternalMoniker      5f59b7a8     uuid:cguid_i_guid7.obj
 0002:0000d7b8       _IID_IEnumVARIANT          5f59b7b8     uuid:oaidl_i_guid5.obj
 0002:0000d7c8       _IID_IEnumUnknown          5f59b7c8     uuid:objidl_i_guid7.obj
 0002:0000d7d8       _IID_IEnumString           5f59b7d8     uuid:objidl_i_guid16.obj
 0002:0000d7e8       _IID_IEnumSTATSTG          5f59b7e8     uuid:objidl_i_guid19.obj
 0002:0000d7f8       _IID_IEnumSTATDATA         5f59b7f8     uuid:objidl_i_guid25.obj
 0002:0000d808       _IID_IEnumOLEVERB          5f59b808     uuid:oleidl_i_guid21.obj
 0002:0000d818       _IID_IEnumMoniker          5f59b818     uuid:objidl_i_guid9.obj
 0002:0000d828       _IID_IEnumHolder           5f59b828     uuid:cguid_i_guid15.obj
 0002:0000d838       _IID_IEnumGeneric          5f59b838     uuid:cguid_i_guid14.obj
 0002:0000d848       _IID_IEnumCallback         5f59b848     uuid:cguid_i_guid16.obj
 0002:0000d858       _IID_IDfReserved3          5f59b858     uuid:cguid_i_guid10.obj
 0002:0000d868       _IID_IDfReserved2          5f59b868     uuid:cguid_i_guid9.obj
 0002:0000d878       _IID_IDfReserved1          5f59b878     uuid:cguid_i_guid8.obj
 0002:0000d888       _IID_IDebugStream          5f59b888     uuid:cguid_i_guid20.obj
 0002:0000d898       _IID_IDebug                5f59b898     uuid:cguid_i_guid19.obj
 0002:0000d8a8       _IID_IDataAdviseHolder     5f59b8a8     uuid:objidl_i_guid32.obj
 0002:0000d8b8       _IID_IPrint                5f59b8b8     uuid:docobj_i_guid5.obj
 0002:0000d8c8       _IID_IOleDocumentView      5f59b8c8     uuid:docobj_i_guid2.obj
 0002:0000d8d8       _IID_IOleDocument          5f59b8d8     uuid:docobj_i_guid0.obj
 0002:0000d8e8       _IID_IEnumOleDocumentViews 5f59b8e8     uuid:docobj_i_guid3.obj
 0002:0000d8f8       _IID_IContinueCallback     5f59b8f8     uuid:docobj_i_guid4.obj
 0002:0000d908       _IID_IBindCtx              5f59b908     uuid:objidl_i_guid8.obj
 0002:0000d918       _IID_IAdviseSink2          5f59b918     uuid:objidl_i_guid29.obj
 0002:0000d928       _IID_IBindHost             5f59b928     uuid:urlmon_i_guid11.obj
 0002:0000d938       _IID_IWebBrowser2          5f59b938     uuid:exdisp_i_guid4.obj
 0002:0000d948       _CLSID_WebBrowser          5f59b948     uuid:exdisp_i_guid7.obj
 0002:0000d958       _IID_IFontDisp             5f59b958     uuid:ocidl_i_guid22.obj
 0002:0000d968       _DBPROPSET_PROVIDERCONNATTR 5f59b968     uuid:guids.obj
 0002:0000d978       _DBPROPSET_PROVIDERSTMTATTR 5f59b978     uuid:guids.obj
 0002:0000d988       _DBPROPSET_PROVIDERDBINIT  5f59b988     uuid:guids.obj
 0002:0000d998       _DBPROPSET_PROVIDERROWSET  5f59b998     uuid:guids.obj
 0002:0000d9a8       _DBPROPSET_PROVIDERDATASOURCEINFO 5f59b9a8     uuid:guids.obj
 0002:0000d9b8       _IID_ITransaction          5f59b9b8     uuid:guids.obj
 0002:0000d9c8       _IID_ITransactionDispenser 5f59b9c8     uuid:guids.obj
 0002:0000d9d8       _IID_ITransactionOptions   5f59b9d8     uuid:guids.obj
 0002:0000d9e8       _IID_ITransactionOutcomeEvents 5f59b9e8     uuid:guids.obj
 0002:0000d9f8       _CLSID_MSDASQL             5f59b9f8     uuid:guids.obj
 0002:0000da08       _CLSID_MSDASQL_ENUMERATOR  5f59ba08     uuid:guids.obj
 0002:0000da18       _IID_IRowsetChangeExtInfo  5f59ba18     uuid:guids.obj
 0002:0000da28       _IID_ISQLGetDiagField      5f59ba28     uuid:guids.obj
 0002:0000da38       _IID_ISQLRequestDiagFields 5f59ba38     uuid:guids.obj
 0002:0000da48       _CLSID_OLEDB_ROWPOSITIONLIBRARY 5f59ba48     uuid:guids.obj
 0002:0000da58       _CLSID_OLEDB_CONVERSIONLIBRARY 5f59ba58     uuid:guids.obj
 0002:0000da68       _CLSID_MSDAVTM             5f59ba68     uuid:guids.obj
 0002:0000da78       _CLSID_EXTENDEDERRORINFO   5f59ba78     uuid:guids.obj
 0002:0000da88       _CLSID_OLEDB_ENUMERATOR    5f59ba88     uuid:guids.obj
 0002:0000da98       _IID_ITransactionObject    5f59ba98     uuid:guids.obj
 0002:0000daa8       _IID_ITransactionJoin      5f59baa8     uuid:guids.obj
 0002:0000dab8       _IID_ITransactionLocal     5f59bab8     uuid:guids.obj
 0002:0000dac8       _IID_IGetDataSource        5f59bac8     uuid:guids.obj
 0002:0000dad8       _IID_ISQLErrorInfo         5f59bad8     uuid:guids.obj
 0002:0000dae8       _IID_IErrorLookup          5f59bae8     uuid:guids.obj
 0002:0000daf8       _IID_IErrorRecords         5f59baf8     uuid:guids.obj
 0002:0000db08       _IID_IMDRangeRowset        5f59bb08     uuid:guids.obj
 0002:0000db18       _IID_IMDFind               5f59bb18     uuid:guids.obj
 0002:0000db28       _IID_IMDDataset            5f59bb28     uuid:guids.obj
 0002:0000db38       _IID_IProvideMoniker       5f59bb38     uuid:guids.obj
 0002:0000db48       _IID_IDBSchemaRowset       5f59bb48     uuid:guids.obj
 0002:0000db58       _IID_IDBSecurityInfo       5f59bb58     uuid:guids.obj
 0002:0000db68       _IID_IDBSchemaCommand      5f59bb68     uuid:guids.obj
 0002:0000db78       _IID_ITableRename          5f59bb78     uuid:guids.obj
 0002:0000db88       _IID_IOpenRowset           5f59bb88     uuid:guids.obj
 0002:0000db98       _IID_ITableDefinition      5f59bb98     uuid:guids.obj
 0002:0000dba8       _IID_IIndexDefinition      5f59bba8     uuid:guids.obj
 0002:0000dbb8       _IID_ISessionProperties    5f59bbb8     uuid:guids.obj
 0002:0000dbc8       _IID_IDBAsynchStatus       5f59bbc8     uuid:guids.obj
 0002:0000dbd8       _IID_IDBAsynchNotify       5f59bbd8     uuid:guids.obj
 0002:0000dbe8       _IID_IDBDataSourceAdmin    5f59bbe8     uuid:guids.obj
 0002:0000dbf8       _IID_IDBInfo               5f59bbf8     uuid:guids.obj
 0002:0000dc08       _IID_IDBInitialize         5f59bc08     uuid:guids.obj
 0002:0000dc18       _IID_IDBProperties         5f59bc18     uuid:guids.obj
 0002:0000dc28       _IID_ISourcesRowset        5f59bc28     uuid:guids.obj
 0002:0000dc38       _IID_IDBCreateSession      5f59bc38     uuid:guids.obj
 0002:0000dc48       _IID_IDBCreateCommand      5f59bc48     uuid:guids.obj
 0002:0000dc58       _IID_IColumnsInfo          5f59bc58     uuid:guids.obj
 0002:0000dc68       _IID_IColumnsRowset        5f59bc68     uuid:guids.obj
 0002:0000dc78       _IID_IQuery                5f59bc78     uuid:guids.obj
 0002:0000dc88       _IID_ICommandWithParameters 5f59bc88     uuid:guids.obj
 0002:0000dc98       _IID_ICommandValidate      5f59bc98     uuid:guids.obj
 0002:0000dca8       _IID_ICommandTree          5f59bca8     uuid:guids.obj
 0002:0000dcb8       _IID_ICommandText          5f59bcb8     uuid:guids.obj
 0002:0000dcc8       _IID_ICommandProperties    5f59bcc8     uuid:guids.obj
 0002:0000dcd8       _IID_ICommandPrepare       5f59bcd8     uuid:guids.obj
 0002:0000dce8       _IID_ICommandCost          5f59bce8     uuid:guids.obj
 0002:0000dcf8       _IID_IConvertType          5f59bcf8     uuid:guids.obj
 0002:0000dd08       _IID_IMultipleResults      5f59bd08     uuid:guids.obj
 0002:0000dd18       _IID_ICommand              5f59bd18     uuid:guids.obj
 0002:0000dd28       _IID_IReadData             5f59bd28     uuid:guids.obj
 0002:0000dd38       _IID_IRowsetCopyRows       5f59bd38     uuid:guids.obj
 0002:0000dd48       _IID_IRowsetWatchRegion    5f59bd48     uuid:guids.obj
 0002:0000dd58       _IID_IRowsetWatchNotify    5f59bd58     uuid:guids.obj
 0002:0000dd68       _IID_IRowsetWatchAll       5f59bd68     uuid:guids.obj
 0002:0000dd78       _IID_IRowsetIndex          5f59bd78     uuid:guids.obj
 0002:0000dd88       _IID_IRowsetNotify         5f59bd88     uuid:guids.obj
 0002:0000dd98       _IID_IRowsetKeys           5f59bd98     uuid:guids.obj
 0002:0000dda8       _IID_IRowsetAsynch         5f59bda8     uuid:guids.obj
 0002:0000ddb8       _IID_IRowsetWithParameters 5f59bdb8     uuid:guids.obj
 0002:0000ddc8       _IID_IRowsetNewRowAfter    5f59bdc8     uuid:guids.obj
 0002:0000ddd8       _IID_IRowsetIdentity       5f59bdd8     uuid:guids.obj
 0002:0000dde8       _IID_IRowsetNextRowset     5f59bde8     uuid:guids.obj
 0002:0000ddf8       _IID_IRowsetUpdate         5f59bdf8     uuid:guids.obj
 0002:0000de08       _IID_IRowsetChange         5f59be08     uuid:guids.obj
 0002:0000de18       _IID_IRowsetExactScroll    5f59be18     uuid:guids.obj
 0002:0000de28       _IID_IRowsetView           5f59be28     uuid:guids.obj
 0002:0000de38       _IID_IViewFilter           5f59be38     uuid:guids.obj
 0002:0000de48       _IID_IViewSort             5f59be48     uuid:guids.obj
 0002:0000de58       _IID_IViewChapter          5f59be58     uuid:guids.obj
 0002:0000de68       _IID_IViewRowset           5f59be68     uuid:guids.obj
 0002:0000de78       _IID_IRowPositionChange    5f59be78     uuid:guids.obj
 0002:0000de88       _IID_IRowPosition          5f59be88     uuid:guids.obj
 0002:0000de98       _IID_IRowsetFind           5f59be98     uuid:guids.obj
 0002:0000dea8       _IID_IChapteredRowset      5f59bea8     uuid:guids.obj
 0002:0000deb8       _IID_IRowsetScroll         5f59beb8     uuid:guids.obj
 0002:0000dec8       _IID_IRowsetResynch        5f59bec8     uuid:guids.obj
 0002:0000ded8       _IID_IRowsetLocate         5f59bed8     uuid:guids.obj
 0002:0000dee8       _IID_IRowsetInfo           5f59bee8     uuid:guids.obj
 0002:0000def8       _IID_IRowset               5f59bef8     uuid:guids.obj
 0002:0000df08       _IID_IAccessor             5f59bf08     uuid:guids.obj
 0002:0000df18       _DBGUID_SQL                5f59bf18     uuid:guids.obj
 0002:0000df28       _DBGUID_DEFAULT            5f59bf28     uuid:guids.obj
 0002:0000df38       _DBGUID_DBSQL              5f59bf38     uuid:guids.obj
 0002:0000df48       _DBPROPSET_VIEW            5f59bf48     uuid:guids.obj
 0002:0000df58       _DBPROPSET_PROPERTIESINERROR 5f59bf58     uuid:guids.obj
 0002:0000df68       _DBPROPSET_DBINITALL       5f59bf68     uuid:guids.obj
 0002:0000df78       _DBPROPSET_SESSIONALL      5f59bf78     uuid:guids.obj
 0002:0000df88       _DBPROPSET_SESSION         5f59bf88     uuid:guids.obj
 0002:0000df98       _DBPROPSET_ROWSETALL       5f59bf98     uuid:guids.obj
 0002:0000dfa8       _DBPROPSET_DATASOURCEINFOALL 5f59bfa8     uuid:guids.obj
 0002:0000dfb8       _DBPROPSET_DATASOURCEALL   5f59bfb8     uuid:guids.obj
 0002:0000dfc8       _DBPROPSET_TABLE           5f59bfc8     uuid:guids.obj
 0002:0000dfd8       _DBPROPSET_ROWSET          5f59bfd8     uuid:guids.obj
 0002:0000dfe8       _DBPROPSET_INDEX           5f59bfe8     uuid:guids.obj
 0002:0000dff8       _DBPROPSET_DBINIT          5f59bff8     uuid:guids.obj
 0002:0000e008       _DBPROPSET_DATASOURCEINFO  5f59c008     uuid:guids.obj
 0002:0000e018       _DBPROPSET_DATASOURCE      5f59c018     uuid:guids.obj
 0002:0000e028       _DBPROPSET_COLUMN          5f59c028     uuid:guids.obj
 0002:0000e038       _PSGUID_QUERY              5f59c038     uuid:guids.obj
 0002:0000e048       _DBCOL_SPECIALCOL          5f59c048     uuid:guids.obj
 0002:0000e058       _DBCOL_SELFCOLUMNS         5f59c058     uuid:guids.obj
 0002:0000e068       _DBSCHEMA_PROCEDURE_COLUMNS 5f59c068     uuid:guids.obj
 0002:0000e078       _DBSCHEMA_PRIMARY_KEYS     5f59c078     uuid:guids.obj
 0002:0000e088       _DBSCHEMA_FOREIGN_KEYS     5f59c088     uuid:guids.obj
 0002:0000e098       _DBSCHEMA_PROCEDURE_PARAMETERS 5f59c098     uuid:guids.obj
 0002:0000e0a8       _DBSCHEMA_VIEW_TABLE_USAGE 5f59c0a8     uuid:guids.obj
 0002:0000e0b8       _DBSCHEMA_VIEW_COLUMN_USAGE 5f59c0b8     uuid:guids.obj
 0002:0000e0c8       _DBSCHEMA_VIEWS            5f59c0c8     uuid:guids.obj
 0002:0000e0d8       _DBSCHEMA_PROVIDER_TYPES   5f59c0d8     uuid:guids.obj
 0002:0000e0e8       _DBSCHEMA_TRANSLATIONS     5f59c0e8     uuid:guids.obj
 0002:0000e0f8       _DBSCHEMA_TABLES           5f59c0f8     uuid:guids.obj
 0002:0000e108       _DBSCHEMA_STATISTICS       5f59c108     uuid:guids.obj
 0002:0000e118       _DBSCHEMA_SQL_LANGUAGES    5f59c118     uuid:guids.obj
 0002:0000e128       _DBSCHEMA_SCHEMATA         5f59c128     uuid:guids.obj
 0002:0000e138       _DBSCHEMA_PROCEDURES       5f59c138     uuid:guids.obj
 0002:0000e148       _DBSCHEMA_USAGE_PRIVILEGES 5f59c148     uuid:guids.obj
 0002:0000e158       _DBSCHEMA_TABLE_PRIVILEGES 5f59c158     uuid:guids.obj
 0002:0000e168       _DBSCHEMA_COLUMN_PRIVILEGES 5f59c168     uuid:guids.obj
 0002:0000e178       _DBSCHEMA_INDEXES          5f59c178     uuid:guids.obj
 0002:0000e188       _DBSCHEMA_COLUMN_DOMAIN_USAGE 5f59c188     uuid:guids.obj
 0002:0000e198       _DBSCHEMA_TABLE_CONSTRAINTS 5f59c198     uuid:guids.obj
 0002:0000e1a8       _DBSCHEMA_REFERENTIAL_CONSTRAINTS 5f59c1a8     uuid:guids.obj
 0002:0000e1b8       _DBSCHEMA_KEY_COLUMN_USAGE 5f59c1b8     uuid:guids.obj
 0002:0000e1c8       _DBSCHEMA_CONSTRAINT_TABLE_USAGE 5f59c1c8     uuid:guids.obj
 0002:0000e1d8       _DBSCHEMA_CONSTRAINT_COLUMN_USAGE 5f59c1d8     uuid:guids.obj
 0002:0000e1e8       _DBSCHEMA_CHECK_CONSTRAINTS 5f59c1e8     uuid:guids.obj
 0002:0000e1f8       _DBSCHEMA_COLUMNS          5f59c1f8     uuid:guids.obj
 0002:0000e208       _DBSCHEMA_COLLATIONS       5f59c208     uuid:guids.obj
 0002:0000e218       _DBSCHEMA_CHARACTER_SETS   5f59c218     uuid:guids.obj
 0002:0000e228       _DBSCHEMA_CATALOGS         5f59c228     uuid:guids.obj
 0002:0000e238       _DBSCHEMA_ASSERTIONS       5f59c238     uuid:guids.obj
 0002:0000e248       _DBCOLUMN_KEYCOLUMN        5f59c248     uuid:guids.obj
 0002:0000e260       _DBCOLUMN_BASETABLEVERSION 5f59c260     uuid:guids.obj
 0002:0000e278       _MDSCHEMA_MEMBERS          5f59c278     uuid:guids.obj
 0002:0000e288       _MDSCHEMA_PROPERTIES       5f59c288     uuid:guids.obj
 0002:0000e298       _MDSCHEMA_MEASURES         5f59c298     uuid:guids.obj
 0002:0000e2a8       _MDSCHEMA_LEVELS           5f59c2a8     uuid:guids.obj
 0002:0000e2b8       _MDSCHEMA_HIERARCHIES      5f59c2b8     uuid:guids.obj
 0002:0000e2c8       _MDSCHEMA_DIMENSIONS       5f59c2c8     uuid:guids.obj
 0002:0000e2d8       _MDSCHEMA_CUBES            5f59c2d8     uuid:guids.obj
 0002:0000e2e8       _DBGUID_MDX                5f59c2e8     uuid:guids.obj
 0002:0000e2f8       _MDGUID_MDX                5f59c2f8     uuid:guids.obj
 0002:0000e308       _DBSCHEMA_TABLES_INFO      5f59c308     uuid:guids.obj
 0002:0000e318       _DBCOLUMN_MAYSORT          5f59c318     uuid:guids.obj
 0002:0000e330       _DBCOLUMN_CLSID            5f59c330     uuid:guids.obj
 0002:0000e348       _DBCOLUMN_COLUMNSIZE       5f59c348     uuid:guids.obj
 0002:0000e360       _DBCOLUMN_OCTETLENGTH      5f59c360     uuid:guids.obj
 0002:0000e378       _DBCOLUMN_NUMERICPRECISIONRADIX 5f59c378     uuid:guids.obj
 0002:0000e390       _DBCOLUMN_DATETIMEPRECISION 5f59c390     uuid:guids.obj
 0002:0000e3a8       _DBCOLUMN_DOMAINSCHEMA     5f59c3a8     uuid:guids.obj
 0002:0000e3c0       _DBCOLUMN_DOMAINCATALOG    5f59c3c0     uuid:guids.obj
 0002:0000e3d8       _DBCOLUMN_TYPEINFO         5f59c3d8     uuid:guids.obj
 0002:0000e3f0       _DBCOLUMN_PROPID           5f59c3f0     uuid:guids.obj
 0002:0000e408       _DBCOLUMN_GUID             5f59c408     uuid:guids.obj
 0002:0000e420       _DBCOLUMN_BASESCHEMANAME   5f59c420     uuid:guids.obj
 0002:0000e438       _DBCOLUMN_BASECATALOGNAME  5f59c438     uuid:guids.obj
 0002:0000e450       _DBCOLUMN_ISUNIQUE         5f59c450     uuid:guids.obj
 0002:0000e468       _DBCOLUMN_ISSEARCHABLE     5f59c468     uuid:guids.obj
 0002:0000e480       _DBCOLUMN_ISCASESENSITIVE  5f59c480     uuid:guids.obj
 0002:0000e498       _DBCOLUMN_ISAUTOINCREMENT  5f59c498     uuid:guids.obj
 0002:0000e4b0       _DBCOLUMN_HASDEFAULT       5f59c4b0     uuid:guids.obj
 0002:0000e4c8       _DBCOLUMN_DOMAINNAME       5f59c4c8     uuid:guids.obj
 0002:0000e4e0       _DBCOLUMN_DEFAULTVALUE     5f59c4e0     uuid:guids.obj
 0002:0000e4f8       _DBCOLUMN_COMPUTEMODE      5f59c4f8     uuid:guids.obj
 0002:0000e510       _DBCOLUMN_COLLATINGSEQUENCE 5f59c510     uuid:guids.obj
 0002:0000e528       _DBCOLUMN_BASETABLENAME    5f59c528     uuid:guids.obj
 0002:0000e540       _DBCOLUMN_BASECOLUMNNAME   5f59c540     uuid:guids.obj
 0002:0000e558       _DBCOLUMN_FLAGS            5f59c558     uuid:guids.obj
 0002:0000e570       _DBCOLUMN_SCALE            5f59c570     uuid:guids.obj
 0002:0000e588       _DBCOLUMN_PRECISION        5f59c588     uuid:guids.obj
 0002:0000e5a0       _DBCOLUMN_TYPE             5f59c5a0     uuid:guids.obj
 0002:0000e5b8       _DBCOLUMN_NUMBER           5f59c5b8     uuid:guids.obj
 0002:0000e5d0       _DBCOLUMN_NAME             5f59c5d0     uuid:guids.obj
 0002:0000e5e8       _DBCOLUMN_IDNAME           5f59c5e8     uuid:guids.obj
 0002:0000e600       _DB_NULLID                 5f59c600     uuid:guids.obj
 0002:0000e618       _CLSID_DataConvert         5f59c618     uuid:guids.obj
 0002:0000e628       _CLSID_MRCM                5f59c628     uuid:guids.obj
 0002:0000e638       _CLSID_RCM                 5f59c638     uuid:guids.obj
 0002:0000e648       _CLSID_CCM                 5f59c648     uuid:guids.obj
 0002:0000e658       _CLSID_SCM                 5f59c658     uuid:guids.obj
 0002:0000e668       _CLSID_DCM                 5f59c668     uuid:guids.obj
 0002:0000e678       _CLSID_MSDADCM             5f59c678     uuid:guids.obj
 0002:0000e688       _CLSID_MSDAINITIALIZE      5f59c688     uuid:guids.obj
 0002:0000e698       _CLSID_DataLinks           5f59c698     uuid:guids.obj
 0002:0000e6a8       _IID_IDataSourceLocator    5f59c6a8     uuid:guids.obj
 0002:0000e6b8       _LIBID_MSDASC              5f59c6b8     uuid:guids.obj
 0002:0000e6c8       _IID_IDBPromptCustomize    5f59c6c8     uuid:guids.obj
 0002:0000e6d8       _IID_IDataInitialize       5f59c6d8     uuid:guids.obj
 0002:0000e6e8       _IID_IDBPromptInitialize   5f59c6e8     uuid:guids.obj
 0002:0000e6f8       _IID_IJoinSessionPool      5f59c6f8     uuid:guids.obj
 0002:0000e708       _IID_IPoolSession          5f59c708     uuid:guids.obj
 0002:0000e718       _IID_IOuterUnknown         5f59c718     uuid:guids.obj
 0002:0000e728       _IID_IService              5f59c728     uuid:guids.obj
 0002:0000e738       _IID_INotifyDBEvents       5f59c738     uuid:cguid_i_guid84.obj
 0002:0000e748       _IID_IBoundObjectSite      5f59c748     uuid:cguid_i_guid91.obj
 0002:0000e758       _IID_IOleControlSite       5f59c758     uuid:ocidl_i_guid9.obj
 0002:0000e768       _IID_IPropertyNotifySink   5f59c768     uuid:ocidl_i_guid13.obj
 0002:0000e778       _IID_IFont                 5f59c778     uuid:ocidl_i_guid19.obj
 0002:0000e788       _IID_IQuickActivate        5f59c788     uuid:ocidl_i_guid40.obj
 0002:0000e798       _IID_IPersistMemory        5f59c798     uuid:ocidl_i_guid15.obj
 0002:0000e7a8       _IID_IOleControl           5f59c7a8     uuid:ocidl_i_guid8.obj
 0002:0000e7b8       _IID_IConnectionPointContainer 5f59c7b8     uuid:ocidl_i_guid3.obj
 0002:0000e7c8       _IID_IProvideClassInfo     5f59c7c8     uuid:ocidl_i_guid5.obj
 0002:0000e7d8       _IID_IProvideClassInfo2    5f59c7d8     uuid:ocidl_i_guid6.obj
 0002:0000e7e8       _IID_ICursorUpdateARow     5f59c7e8     uuid:cguid_i_guid83.obj
 0002:0000e7f8       _IID_ICursorMove           5f59c7f8     uuid:cguid_i_guid81.obj
 0002:0000e808       _IID_ICursor               5f59c808     uuid:cguid_i_guid80.obj
 0002:0000e818       _COLUMNID_INVALID          5f59c818     uuid:vcguids.obj
 0002:0000e830       _COLUMN_AUTOINCREMENT      5f59c830     uuid:vcguids.obj
 0002:0000e848       _COLUMN_BASECOLUMNNAME     5f59c848     uuid:vcguids.obj
 0002:0000e860       _COLUMN_BASENAME           5f59c860     uuid:vcguids.obj
 0002:0000e878       _COLUMN_BINARYCOMPARABLE   5f59c878     uuid:vcguids.obj
 0002:0000e890       _COLUMN_BINDTYPE           5f59c890     uuid:vcguids.obj
 0002:0000e8a8       _COLUMN_CASESENSITIVE      5f59c8a8     uuid:vcguids.obj
 0002:0000e8c0       _COLUMN_COLLATINGORDER     5f59c8c0     uuid:vcguids.obj
 0002:0000e8d8       _COLUMN_COLUMNID           5f59c8d8     uuid:vcguids.obj
 0002:0000e8f0       _COLUMN_CURSORCOLUMN       5f59c8f0     uuid:vcguids.obj
 0002:0000e908       _COLUMN_DATACOLUMN         5f59c908     uuid:vcguids.obj
 0002:0000e920       _COLUMN_DEFAULTVALUE       5f59c920     uuid:vcguids.obj
 0002:0000e938       _COLUMN_ENTRYIDMAXLENGTH   5f59c938     uuid:vcguids.obj
 0002:0000e950       _COLUMN_FIXED              5f59c950     uuid:vcguids.obj
 0002:0000e968       _COLUMN_HASDEFAULT         5f59c968     uuid:vcguids.obj
 0002:0000e980       _COLUMN_MAXLENGTH          5f59c980     uuid:vcguids.obj
 0002:0000e998       _COLUMN_MULTIVALUED        5f59c998     uuid:vcguids.obj
 0002:0000e9b0       _COLUMN_NAME               5f59c9b0     uuid:vcguids.obj
 0002:0000e9c8       _COLUMN_NULLABLE           5f59c9c8     uuid:vcguids.obj
 0002:0000e9e0       _COLUMN_PHYSICALSORT       5f59c9e0     uuid:vcguids.obj
 0002:0000e9f8       _COLUMN_NUMBER             5f59c9f8     uuid:vcguids.obj
 0002:0000ea10       _COLUMN_ROWENTRYID         5f59ca10     uuid:vcguids.obj
 0002:0000ea28       _COLUMN_SCALE              5f59ca28     uuid:vcguids.obj
 0002:0000ea40       _COLUMN_SEARCHABLE         5f59ca40     uuid:vcguids.obj
 0002:0000ea58       _COLUMN_TYPE               5f59ca58     uuid:vcguids.obj
 0002:0000ea70       _COLUMN_UNIQUE             5f59ca70     uuid:vcguids.obj
 0002:0000ea88       _COLUMN_UPDATABLE          5f59ca88     uuid:vcguids.obj
 0002:0000eaa0       _COLUMN_VERSION            5f59caa0     uuid:vcguids.obj
 0002:0000eab8       _COLUMN_STATUS             5f59cab8     uuid:vcguids.obj
 0002:0000ead0       _COLUMN_BMKTEMPORARY       5f59cad0     uuid:vcguids.obj
 0002:0000eae8       _COLUMN_BMKTEMPORARYREL    5f59cae8     uuid:vcguids.obj
 0002:0000eb00       _COLUMN_BMKCURSOR          5f59cb00     uuid:vcguids.obj
 0002:0000eb18       _COLUMN_BMKCURSORREL       5f59cb18     uuid:vcguids.obj
 0002:0000eb30       _COLUMN_BMKSESSION         5f59cb30     uuid:vcguids.obj
 0002:0000eb48       _COLUMN_BMKSESSIONREL      5f59cb48     uuid:vcguids.obj
 0002:0000eb60       _COLUMN_BMKPERSIST         5f59cb60     uuid:vcguids.obj
 0002:0000eb78       _COLUMN_BMKPERSISTREL      5f59cb78     uuid:vcguids.obj
 0002:0000eb90       _DBBMK_INVALID             5f59cb90     uuid:vcguids.obj
 0002:0000eb94       _DBBMK_CURRENT             5f59cb94     uuid:vcguids.obj
 0002:0000eb98       _DBBMK_BEGINNING           5f59cb98     uuid:vcguids.obj
 0002:0000eb9c       _DBBMK_END                 5f59cb9c     uuid:vcguids.obj
 0002:0000eba0       _IID_ISequentialStream     5f59cba0     uuid:objidl_i_guid17.obj
 0002:0000ebb0       _IID_IBoundObject          5f59cbb0     uuid:cguid_i_guid90.obj
 0002:0000ebc0       _IID_IBindStatusCallback   5f59cbc0     uuid:urlmon_i_guid3.obj
 0002:0000ebd0       _IID_IServiceProvider      5f59cbd0     uuid:servprov_i_guid0.obj
 0002:0000ebe0       _IID_IPerPropertyBrowsing  5f59cbe0     uuid:ocidl_i_guid36.obj
 0002:0000ebf0       _IID_ISpecifyPropertyPages 5f59cbf0     uuid:ocidl_i_guid14.obj
 0002:0000ec00       _IID_IPersistPropertyBag   5f59cc00     uuid:ocidl_i_guid17.obj
 0002:0000ec10       _IID_IOleInPlaceObjectWindowless 5f59cc10     uuid:ocidl_i_guid24.obj
 0002:0000ec20       _IID_IViewObjectEx         5f59cc20     uuid:ocidl_i_guid27.obj
 0002:0000ec30       _IID_IPointerInactive      5f59cc30     uuid:ocidl_i_guid32.obj
 0002:0000ec40       _CLSID_ConvertVBX          5f59cc40     uuid:cguid_i_guid56.obj
 0002:0000ec50       _CLSID_PersistPropset      5f59cc50     uuid:cguid_i_guid55.obj
 0002:0000ec60       _IID_IOleInPlaceSiteEx     5f59cc60     uuid:ocidl_i_guid25.obj
 0002:0000ec70       _IID_IOleInPlaceSiteWindowless 5f59cc70     uuid:ocidl_i_guid26.obj
 0002:0000ec80       _IID_IEnumConnectionPoints 5f59cc80     uuid:ocidl_i_guid2.obj
 0002:0000ec90       _IID_IEnumConnections      5f59cc90     uuid:ocidl_i_guid0.obj
 0002:0000eca0       _IID_IConnectionPoint      5f59cca0     uuid:ocidl_i_guid1.obj
 0002:0000ecb0       _IID_ISimpleFrameSite      5f59ccb0     uuid:ocidl_i_guid18.obj
 0002:0000ecc0       _IID_IPicture              5f59ccc0     uuid:ocidl_i_guid20.obj
 0002:0000ecd0       _IID_IPictureDisp          5f59ccd0     uuid:ocidl_i_guid23.obj
 0002:0000ece0       _CLSID_StdPicture          5f59cce0     uuid:cguid_i_guid58.obj
 0002:0000ecf0       _IID_IPropertyPage         5f59ccf0     uuid:ocidl_i_guid10.obj
 0002:0000ed00       _IID_IPropertyPage2        5f59cd00     uuid:ocidl_i_guid11.obj
 0002:0000ed10       _CLSID_CColorPropPage      5f59cd10     uuid:cguid_i_guid50.obj
 0002:0000ed20       _CLSID_CFontPropPage       5f59cd20     uuid:cguid_i_guid49.obj
 0002:0000ed30       _CLSID_StdFont             5f59cd30     uuid:cguid_i_guid57.obj
 0002:0000ed40       _GUID_COLOR                5f59cd40     uuid:cguid_i_guid60.obj
 0002:0000ed50       __sz_OLEPRO32              5f59cd50     olepro32:OLEPRO32.DLL
 0002:0000ed60       __sz_ADVAPI32              5f59cd60     advapi32:ADVAPI32.dll
 0002:0000ed70       __sz_ole32                 5f59cd70     ole32:ole32.dll
 0002:0000ed80       __sz_OLEAUT32              5f59cd80     oleaut32:OLEAUT32.dll
 0002:0000ed90       __sz_oledlg                5f59cd90     oledlg:oledlg.dll
 0002:0000eda0       __sz_urlmon                5f59cda0     urlmon:urlmon.dll
 0002:0000edb0       __sz_SHELL32               5f59cdb0     shell32:SHELL32.dll
 0002:0000edc0       ??_R1A@?0A@A@CObject@@8    5f59cdc0     olecli1.obj
 0002:0000edd8       ??_R1A@?0A@A@CCmdTarget@@8 5f59cdd8     olecli1.obj
 0002:0000edf0       ??_R1A@?0A@A@CDocItem@@8   5f59cdf0     olecli1.obj
 0002:0000ee08       ??_R1A@?0A@A@COleClientItem@@8 5f59ce08     olecli1.obj
 0002:0000ee20       ??_R2COleClientItem@@8     5f59ce20     olecli1.obj
 0002:0000ee38       ??_R3COleClientItem@@8     5f59ce38     olecli1.obj
 0002:0000ee48       ??_R4COleClientItem@@6B@   5f59ce48     olecli1.obj
 0002:0000ee60       ??_R1A@?0A@A@IUnknown@@8   5f59ce60     olecli1.obj
 0002:0000ee78       ??_R1A@?0A@A@IOleClientSite@@8 5f59ce78     olecli1.obj
 0002:0000ee90       ??_R1A@?0A@A@XOleClientSite@COleClientItem@@8 5f59ce90     olecli1.obj
 0002:0000eea8       ??_R2XOleClientSite@COleClientItem@@8 5f59cea8     olecli1.obj
 0002:0000eeb8       ??_R3XOleClientSite@COleClientItem@@8 5f59ceb8     olecli1.obj
 0002:0000eec8       ??_R4XOleClientSite@COleClientItem@@6B@ 5f59cec8     olecli1.obj
 0002:0000eee0       ??_R1A@?0A@A@IAdviseSink@@8 5f59cee0     olecli1.obj
 0002:0000eef8       ??_R1A@?0A@A@XAdviseSink@COleClientItem@@8 5f59cef8     olecli1.obj
 0002:0000ef10       ??_R2XAdviseSink@COleClientItem@@8 5f59cf10     olecli1.obj
 0002:0000ef20       ??_R3XAdviseSink@COleClientItem@@8 5f59cf20     olecli1.obj
 0002:0000ef30       ??_R4XAdviseSink@COleClientItem@@6B@ 5f59cf30     olecli1.obj
 0002:0000ef48       ??_R1A@?0A@A@IOleWindow@@8 5f59cf48     olecli1.obj
 0002:0000ef60       ??_R1A@?0A@A@IOleInPlaceSite@@8 5f59cf60     olecli1.obj
 0002:0000ef78       ??_R1A@?0A@A@XOleIPSite@COleClientItem@@8 5f59cf78     olecli1.obj
 0002:0000ef90       ??_R2XOleIPSite@COleClientItem@@8 5f59cf90     olecli1.obj
 0002:0000efa8       ??_R3XOleIPSite@COleClientItem@@8 5f59cfa8     olecli1.obj
 0002:0000efb8       ??_R4XOleIPSite@COleClientItem@@6B@ 5f59cfb8     olecli1.obj
 0002:0000efd0       ??_R1A@?0A@A@COleFrameHook@@8 5f59cfd0     olecli2.obj
 0002:0000efe8       ??_R2COleFrameHook@@8      5f59cfe8     olecli2.obj
 0002:0000eff8       ??_R3COleFrameHook@@8      5f59cff8     olecli2.obj
 0002:0000f008       ??_R4COleFrameHook@@6B@    5f59d008     olecli2.obj
 0002:0000f020       ??_R1A@?0A@A@IOleInPlaceUIWindow@@8 5f59d020     olecli2.obj
 0002:0000f038       ??_R1A@?0A@A@IOleInPlaceFrame@@8 5f59d038     olecli2.obj
 0002:0000f050       ??_R1A@?0A@A@XOleInPlaceFrame@COleFrameHook@@8 5f59d050     olecli2.obj
 0002:0000f068       ??_R2XOleInPlaceFrame@COleFrameHook@@8 5f59d068     olecli2.obj
 0002:0000f080       ??_R3XOleInPlaceFrame@COleFrameHook@@8 5f59d080     olecli2.obj
 0002:0000f090       ??_R4XOleInPlaceFrame@COleFrameHook@@6B@ 5f59d090     olecli2.obj
 0002:0000f0a8       ??_R1A@?0A@A@IOleCommandTarget@@8 5f59d0a8     olecli2.obj
 0002:0000f0c0       ??_R1A@?0A@A@XOleCommandTarget@COleFrameHook@@8 5f59d0c0     olecli2.obj
 0002:0000f0d8       ??_R2XOleCommandTarget@COleFrameHook@@8 5f59d0d8     olecli2.obj
 0002:0000f0e8       ??_R3XOleCommandTarget@COleFrameHook@@8 5f59d0e8     olecli2.obj
 0002:0000f0f8       ??_R4XOleCommandTarget@COleFrameHook@@6B@ 5f59d0f8     olecli2.obj
 0002:0000f110       ??_R1A@?0A@A@COleDataSource@@8 5f59d110     oledobj2.obj
 0002:0000f128       ??_R2COleDataSource@@8     5f59d128     oledobj2.obj
 0002:0000f138       ??_R3COleDataSource@@8     5f59d138     oledobj2.obj
 0002:0000f148       ??_R4COleDataSource@@6B@   5f59d148     oledobj2.obj
 0002:0000f160       ??_R1A@?0A@A@IDataObject@@8 5f59d160     oledobj2.obj
 0002:0000f178       ??_R1A@?0A@A@XDataObject@COleDataSource@@8 5f59d178     oledobj2.obj
 0002:0000f190       ??_R2XDataObject@COleDataSource@@8 5f59d190     oledobj2.obj
 0002:0000f1a0       ??_R3XDataObject@COleDataSource@@8 5f59d1a0     oledobj2.obj
 0002:0000f1b0       ??_R4XDataObject@COleDataSource@@6B@ 5f59d1b0     oledobj2.obj
 0002:0000f1c8       ??_R1A@?0A@A@CEnumArray@@8 5f59d1c8     oledobj2.obj
 0002:0000f1e0       ??_R1A@?0A@A@CEnumFormatEtc@@8 5f59d1e0     oledobj2.obj
 0002:0000f1f8       ??_R2CEnumFormatEtc@@8     5f59d1f8     oledobj2.obj
 0002:0000f210       ??_R3CEnumFormatEtc@@8     5f59d210     oledobj2.obj
 0002:0000f220       ??_R4CEnumFormatEtc@@6B@   5f59d220     oledobj2.obj
 0002:0000f238       ??_R1A@?0A@A@IDispatch@@8  5f59d238     oledisp1.obj
 0002:0000f250       ??_R1A@?0A@A@COleDispatchImpl@@8 5f59d250     oledisp1.obj
 0002:0000f268       ??_R2COleDispatchImpl@@8   5f59d268     oledisp1.obj
 0002:0000f278       ??_R3COleDispatchImpl@@8   5f59d278     oledisp1.obj
 0002:0000f288       ??_R4COleDispatchImpl@@6B@ 5f59d288     oledisp1.obj
 0002:0000f2a0       ??_R1A@?0A@A@CException@@8 5f59d2a0     oledisp1.obj
 0002:0000f2b8       ??_R1A@?0A@A@COleDispatchException@@8 5f59d2b8     oledisp1.obj
 0002:0000f2d0       ??_R2COleDispatchException@@8 5f59d2d0     oledisp1.obj
 0002:0000f2e0       ??_R3COleDispatchException@@8 5f59d2e0     oledisp1.obj
 0002:0000f2f0       ??_R4COleDispatchException@@6B@ 5f59d2f0     oledisp1.obj
 0002:0000f308       ??_R1A@?0A@A@IOleUILinkContainerA@@8 5f59d308     oledlgs1.obj
 0002:0000f320       ??_R1A@?0A@A@IOleUILinkInfoA@@8 5f59d320     oledlgs1.obj
 0002:0000f338       ??_R1A@?0A@A@COleUILinkInfo@@8 5f59d338     oledlgs1.obj
 0002:0000f350       ??_R2COleUILinkInfo@@8     5f59d350     oledlgs1.obj
 0002:0000f368       ??_R3COleUILinkInfo@@8     5f59d368     oledlgs1.obj
 0002:0000f378       ??_R4COleUILinkInfo@@6B@   5f59d378     oledlgs1.obj
 0002:0000f390       ??_R2IOleUILinkInfoA@@8    5f59d390     oledlgs1.obj
 0002:0000f3a0       ??_R3IOleUILinkInfoA@@8    5f59d3a0     oledlgs1.obj
 0002:0000f3b0       ??_R4IOleUILinkInfoA@@6B@  5f59d3b0     oledlgs1.obj
 0002:0000f3c8       ??_R2IOleUILinkContainerA@@8 5f59d3c8     oledlgs1.obj
 0002:0000f3d8       ??_R3IOleUILinkContainerA@@8 5f59d3d8     oledlgs1.obj
 0002:0000f3e8       ??_R4IOleUILinkContainerA@@6B@ 5f59d3e8     oledlgs1.obj
 0002:0000f400       ??_R1A@?0A@A@CWnd@@8       5f59d400     oledlgs1.obj
 0002:0000f418       ??_R1A@?0A@A@CDialog@@8    5f59d418     oledlgs1.obj
 0002:0000f430       ??_R1A@?0A@A@CCommonDialog@@8 5f59d430     oledlgs1.obj
 0002:0000f448       ??_R1A@?0A@A@COleDialog@@8 5f59d448     oledlgs1.obj
 0002:0000f460       ??_R1A@?0A@A@COleInsertDialog@@8 5f59d460     oledlgs1.obj
 0002:0000f478       ??_R2COleInsertDialog@@8   5f59d478     oledlgs1.obj
 0002:0000f498       ??_R3COleInsertDialog@@8   5f59d498     oledlgs1.obj
 0002:0000f4a8       ??_R4COleInsertDialog@@6B@ 5f59d4a8     oledlgs1.obj
 0002:0000f4c0       ??_R1A@?0A@A@COleConvertDialog@@8 5f59d4c0     oledlgs1.obj
 0002:0000f4d8       ??_R2COleConvertDialog@@8  5f59d4d8     oledlgs1.obj
 0002:0000f4f8       ??_R3COleConvertDialog@@8  5f59d4f8     oledlgs1.obj
 0002:0000f508       ??_R4COleConvertDialog@@6B@ 5f59d508     oledlgs1.obj
 0002:0000f520       ??_R1A@?0A@A@COleChangeIconDialog@@8 5f59d520     oledlgs1.obj
 0002:0000f538       ??_R2COleChangeIconDialog@@8 5f59d538     oledlgs1.obj
 0002:0000f558       ??_R3COleChangeIconDialog@@8 5f59d558     oledlgs1.obj
 0002:0000f568       ??_R4COleChangeIconDialog@@6B@ 5f59d568     oledlgs1.obj
 0002:0000f580       ??_R1A@?0A@A@COleLinksDialog@@8 5f59d580     oledlgs1.obj
 0002:0000f598       ??_R2COleLinksDialog@@8    5f59d598     oledlgs1.obj
 0002:0000f5b8       ??_R3COleLinksDialog@@8    5f59d5b8     oledlgs1.obj
 0002:0000f5c8       ??_R4COleLinksDialog@@6B@  5f59d5c8     oledlgs1.obj
 0002:0000f5e0       ??_R1A@?0A@A@COleUpdateDialog@@8 5f59d5e0     oledlgs1.obj
 0002:0000f5f8       ??_R2COleUpdateDialog@@8   5f59d5f8     oledlgs1.obj
 0002:0000f620       ??_R3COleUpdateDialog@@8   5f59d620     oledlgs1.obj
 0002:0000f630       ??_R4COleUpdateDialog@@6B@ 5f59d630     oledlgs1.obj
 0002:0000f648       ??_R1A@?0A@A@COlePasteSpecialDialog@@8 5f59d648     oledlgs1.obj
 0002:0000f660       ??_R2COlePasteSpecialDialog@@8 5f59d660     oledlgs1.obj
 0002:0000f680       ??_R3COlePasteSpecialDialog@@8 5f59d680     oledlgs1.obj
 0002:0000f690       ??_R4COlePasteSpecialDialog@@6B@ 5f59d690     oledlgs1.obj
 0002:0000f6a8       ??_R2COleDialog@@8         5f59d6a8     oledlgs2.obj
 0002:0000f6c8       ??_R3COleDialog@@8         5f59d6c8     oledlgs2.obj
 0002:0000f6d8       ??_R4COleDialog@@6B@       5f59d6d8     oledlgs2.obj
 0002:0000f6f0       ??_R1A@?0A@A@COleBusyDialog@@8 5f59d6f0     oledlgs2.obj
 0002:0000f708       ??_R2COleBusyDialog@@8     5f59d708     oledlgs2.obj
 0002:0000f728       ??_R3COleBusyDialog@@8     5f59d728     oledlgs2.obj
 0002:0000f738       ??_R4COleBusyDialog@@6B@   5f59d738     oledlgs2.obj
 0002:0000f750       ??_R1A@?0A@A@COlePropertiesDialog@@8 5f59d750     oledlgs3.obj
 0002:0000f768       ??_R2COlePropertiesDialog@@8 5f59d768     oledlgs3.obj
 0002:0000f788       ??_R3COlePropertiesDialog@@8 5f59d788     oledlgs3.obj
 0002:0000f798       ??_R4COlePropertiesDialog@@6B@ 5f59d798     oledlgs3.obj
 0002:0000f7b0       ??_R1A@?0A@A@IOleUIObjInfoA@@8 5f59d7b0     oledlgs3.obj
 0002:0000f7c8       ??_R1A@?0A@A@XOleUIObjInfo@COlePropertiesDialog@@8 5f59d7c8     oledlgs3.obj
 0002:0000f7e0       ??_R2XOleUIObjInfo@COlePropertiesDialog@@8 5f59d7e0     oledlgs3.obj
 0002:0000f7f0       ??_R3XOleUIObjInfo@COlePropertiesDialog@@8 5f59d7f0     oledlgs3.obj
 0002:0000f800       ??_R4XOleUIObjInfo@COlePropertiesDialog@@6B@ 5f59d800     oledlgs3.obj
 0002:0000f818       ??_R2IOleUIObjInfoA@@8     5f59d818     oledlgs3.obj
 0002:0000f828       ??_R3IOleUIObjInfoA@@8     5f59d828     oledlgs3.obj
 0002:0000f838       ??_R4IOleUIObjInfoA@@6B@   5f59d838     oledlgs3.obj
 0002:0000f850       ??_R1A@?0A@A@COleChangeSourceDialog@@8 5f59d850     oledlgs3.obj
 0002:0000f868       ??_R2COleChangeSourceDialog@@8 5f59d868     oledlgs3.obj
 0002:0000f888       ??_R3COleChangeSourceDialog@@8 5f59d888     oledlgs3.obj
 0002:0000f898       ??_R4COleChangeSourceDialog@@6B@ 5f59d898     oledlgs3.obj
 0002:0000f8b0       ??_R1A@?0A@A@CNoTrackObject@@8 5f59d8b0     oledata.obj
 0002:0000f8c8       ??_R1A@?0A@A@_AFX_OLE_STATE@@8 5f59d8c8     oledata.obj
 0002:0000f8e0       ??_R2_AFX_OLE_STATE@@8     5f59d8e0     oledata.obj
 0002:0000f8f0       ??_R3_AFX_OLE_STATE@@8     5f59d8f0     oledata.obj
 0002:0000f900       ??_R4_AFX_OLE_STATE@@6B@   5f59d900     oledata.obj
 0002:0000f914       ??_R2CNoTrackObject@@8     5f59d914     oledata.obj
 0002:0000f920       ??_R3CNoTrackObject@@8     5f59d920     oledata.obj
 0002:0000f930       ??_R4CNoTrackObject@@6B@   5f59d930     oledata.obj
 0002:0000f948       ??_R1A@?0A@A@CDocument@@8  5f59d948     oledoc1.obj
 0002:0000f960       ??_R1A@?0A@A@COleDocument@@8 5f59d960     oledoc1.obj
 0002:0000f978       ??_R2COleDocument@@8       5f59d978     oledoc1.obj
 0002:0000f990       ??_R3COleDocument@@8       5f59d990     oledoc1.obj
 0002:0000f9a0       ??_R4COleDocument@@6B@     5f59d9a0     oledoc1.obj
 0002:0000f9b8       ??_R2CDocItem@@8           5f59d9b8     oledoc1.obj
 0002:0000f9c8       ??_R3CDocItem@@8           5f59d9c8     oledoc1.obj
 0002:0000f9d8       ??_R4CDocItem@@6B@         5f59d9d8     oledoc1.obj
 0002:0000f9f0       ??_R1A@?0A@A@COleDropSource@@8 5f59d9f0     oledrop1.obj
 0002:0000fa08       ??_R2COleDropSource@@8     5f59da08     oledrop1.obj
 0002:0000fa18       ??_R3COleDropSource@@8     5f59da18     oledrop1.obj
 0002:0000fa28       ??_R4COleDropSource@@6B@   5f59da28     oledrop1.obj
 0002:0000fa40       ??_R1A@?0A@A@IDropSource@@8 5f59da40     oledrop1.obj
 0002:0000fa58       ??_R1A@?0A@A@XDropSource@COleDropSource@@8 5f59da58     oledrop1.obj
 0002:0000fa70       ??_R2XDropSource@COleDropSource@@8 5f59da70     oledrop1.obj
 0002:0000fa80       ??_R3XDropSource@COleDropSource@@8 5f59da80     oledrop1.obj
 0002:0000fa90       ??_R4XDropSource@COleDropSource@@6B@ 5f59da90     oledrop1.obj
 0002:0000faa8       ??_R1A@?0A@A@COleDropTarget@@8 5f59daa8     oledrop2.obj
 0002:0000fac0       ??_R2COleDropTarget@@8     5f59dac0     oledrop2.obj
 0002:0000fad0       ??_R3COleDropTarget@@8     5f59dad0     oledrop2.obj
 0002:0000fae0       ??_R4COleDropTarget@@6B@   5f59dae0     oledrop2.obj
 0002:0000faf8       ??_R1A@?0A@A@IDropTarget@@8 5f59daf8     oledrop2.obj
 0002:0000fb10       ??_R1A@?0A@A@XDropTarget@COleDropTarget@@8 5f59db10     oledrop2.obj
 0002:0000fb28       ??_R2XDropTarget@COleDropTarget@@8 5f59db28     oledrop2.obj
 0002:0000fb38       ??_R3XDropTarget@COleDropTarget@@8 5f59db38     oledrop2.obj
 0002:0000fb48       ??_R4XDropTarget@COleDropTarget@@6B@ 5f59db48     oledrop2.obj
 0002:0000fb60       ??_R1A@?0A@A@COleMessageFilter@@8 5f59db60     olemsgf.obj
 0002:0000fb78       ??_R2COleMessageFilter@@8  5f59db78     olemsgf.obj
 0002:0000fb88       ??_R3COleMessageFilter@@8  5f59db88     olemsgf.obj
 0002:0000fb98       ??_R4COleMessageFilter@@6B@ 5f59db98     olemsgf.obj
 0002:0000fbb0       ??_R1A@?0A@A@IMessageFilter@@8 5f59dbb0     olemsgf.obj
 0002:0000fbc8       ??_R1A@?0A@A@XMessageFilter@COleMessageFilter@@8 5f59dbc8     olemsgf.obj
 0002:0000fbe0       ??_R2XMessageFilter@COleMessageFilter@@8 5f59dbe0     olemsgf.obj
 0002:0000fbf0       ??_R3XMessageFilter@COleMessageFilter@@8 5f59dbf0     olemsgf.obj
 0002:0000fc00       ??_R4XMessageFilter@COleMessageFilter@@6B@ 5f59dc00     olemsgf.obj
 0002:0000fc18       ??_R2CEnumArray@@8         5f59dc18     oleenum.obj
 0002:0000fc28       ??_R3CEnumArray@@8         5f59dc28     oleenum.obj
 0002:0000fc38       ??_R4CEnumArray@@6B@       5f59dc38     oleenum.obj
 0002:0000fc50       ??_R1A@?0A@A@IEnumVOID@@8  5f59dc50     oleenum.obj
 0002:0000fc68       ??_R1A@?0A@A@XEnumVOID@CEnumArray@@8 5f59dc68     oleenum.obj
 0002:0000fc80       ??_R2XEnumVOID@CEnumArray@@8 5f59dc80     oleenum.obj
 0002:0000fc90       ??_R3XEnumVOID@CEnumArray@@8 5f59dc90     oleenum.obj
 0002:0000fca0       ??_R4XEnumVOID@CEnumArray@@6B@ 5f59dca0     oleenum.obj
 0002:0000fcb8       ??_R2IEnumVOID@@8          5f59dcb8     oleenum.obj
 0002:0000fcc8       ??_R3IEnumVOID@@8          5f59dcc8     oleenum.obj
 0002:0000fcd8       ??_R4IEnumVOID@@6B@        5f59dcd8     oleenum.obj
 0002:0000fcf0       ??_R1A@?0A@A@COleObjectFactory@@8 5f59dcf0     olefact.obj
 0002:0000fd08       ??_R2COleObjectFactory@@8  5f59dd08     olefact.obj
 0002:0000fd18       ??_R3COleObjectFactory@@8  5f59dd18     olefact.obj
 0002:0000fd28       ??_R4COleObjectFactory@@6B@ 5f59dd28     olefact.obj
 0002:0000fd40       ??_R1A@?0A@A@IClassFactory@@8 5f59dd40     olefact.obj
 0002:0000fd58       ??_R1A@?0A@A@IClassFactory2@@8 5f59dd58     olefact.obj
 0002:0000fd70       ??_R1A@?0A@A@XClassFactory@COleObjectFactory@@8 5f59dd70     olefact.obj
 0002:0000fd88       ??_R2XClassFactory@COleObjectFactory@@8 5f59dd88     olefact.obj
 0002:0000fda0       ??_R3XClassFactory@COleObjectFactory@@8 5f59dda0     olefact.obj
 0002:0000fdb0       ??_R4XClassFactory@COleObjectFactory@@6B@ 5f59ddb0     olefact.obj
 0002:0000fdc8       ??_R1A@?0A@A@CFrameWnd@@8  5f59ddc8     oleipfrm.obj
 0002:0000fde0       ??_R1A@?0A@A@COleCntrFrameWnd@@8 5f59dde0     oleipfrm.obj
 0002:0000fdf8       ??_R2COleCntrFrameWnd@@8   5f59ddf8     oleipfrm.obj
 0002:0000fe10       ??_R3COleCntrFrameWnd@@8   5f59de10     oleipfrm.obj
 0002:0000fe20       ??_R4COleCntrFrameWnd@@6B@ 5f59de20     oleipfrm.obj
 0002:0000fe38       ??_R1A@?0A@A@COleIPFrameWnd@@8 5f59de38     oleipfrm.obj
 0002:0000fe50       ??_R2COleIPFrameWnd@@8     5f59de50     oleipfrm.obj
 0002:0000fe68       ??_R3COleIPFrameWnd@@8     5f59de68     oleipfrm.obj
 0002:0000fe78       ??_R4COleIPFrameWnd@@6B@   5f59de78     oleipfrm.obj
 0002:0000fe90       ??_R1A@?0A@A@COleLinkingDoc@@8 5f59de90     olelink.obj
 0002:0000fea8       ??_R2COleLinkingDoc@@8     5f59dea8     olelink.obj
 0002:0000fec0       ??_R3COleLinkingDoc@@8     5f59dec0     olelink.obj
 0002:0000fed0       ??_R4COleLinkingDoc@@6B@   5f59ded0     olelink.obj
 0002:0000fee8       ??_R1A@?0A@A@IPersist@@8   5f59dee8     olelink.obj
 0002:0000ff00       ??_R1A@?0A@A@IPersistFile@@8 5f59df00     olelink.obj
 0002:0000ff18       ??_R1A@?0A@A@XPersistFile@COleLinkingDoc@@8 5f59df18     olelink.obj
 0002:0000ff30       ??_R2XPersistFile@COleLinkingDoc@@8 5f59df30     olelink.obj
 0002:0000ff48       ??_R3XPersistFile@COleLinkingDoc@@8 5f59df48     olelink.obj
 0002:0000ff58       ??_R4XPersistFile@COleLinkingDoc@@6B@ 5f59df58     olelink.obj
 0002:0000ff70       ??_R1A@?0A@A@IParseDisplayName@@8 5f59df70     olelink.obj
 0002:0000ff88       ??_R1A@?0A@A@IOleContainer@@8 5f59df88     olelink.obj
 0002:0000ffa0       ??_R1A@?0A@A@IOleItemContainer@@8 5f59dfa0     olelink.obj
 0002:0000ffb8       ??_R1A@?0A@A@XOleItemContainer@COleLinkingDoc@@8 5f59dfb8     olelink.obj
 0002:0000ffd0       ??_R2XOleItemContainer@COleLinkingDoc@@8 5f59dfd0     olelink.obj
 0002:0000ffe8       ??_R3XOleItemContainer@COleLinkingDoc@@8 5f59dfe8     olelink.obj
 0002:0000fff8       ??_R4XOleItemContainer@COleLinkingDoc@@6B@ 5f59dff8     olelink.obj
 0002:00010010       ??_R1A@?0A@A@CFile@@8      5f59e010     olestrm.obj
 0002:00010028       ??_R1A@?0A@A@COleStreamFile@@8 5f59e028     olestrm.obj
 0002:00010040       ??_R2COleStreamFile@@8     5f59e040     olestrm.obj
 0002:00010050       ??_R3COleStreamFile@@8     5f59e050     olestrm.obj
 0002:00010060       ??_R4COleStreamFile@@6B@   5f59e060     olestrm.obj
 0002:00010078       ??_R1A@?0A@A@COleServerDoc@@8 5f59e078     olesvr1.obj
 0002:00010090       ??_R2COleServerDoc@@8      5f59e090     olesvr1.obj
 0002:000100b0       ??_R3COleServerDoc@@8      5f59e0b0     olesvr1.obj
 0002:000100c0       ??_R4COleServerDoc@@6B@    5f59e0c0     olesvr1.obj
 0002:000100d8       ??_R1A@?0A@A@IPersistStorage@@8 5f59e0d8     olesvr1.obj
 0002:000100f0       ??_R1A@?0A@A@XPersistStorage@COleServerDoc@@8 5f59e0f0     olesvr1.obj
 0002:00010108       ??_R2XPersistStorage@COleServerDoc@@8 5f59e108     olesvr1.obj
 0002:00010120       ??_R3XPersistStorage@COleServerDoc@@8 5f59e120     olesvr1.obj
 0002:00010130       ??_R4XPersistStorage@COleServerDoc@@6B@ 5f59e130     olesvr1.obj
 0002:00010148       ??_R1A@?0A@A@IOleObject@@8 5f59e148     olesvr1.obj
 0002:00010160       ??_R1A@?0A@A@XOleObject@COleServerDoc@@8 5f59e160     olesvr1.obj
 0002:00010178       ??_R2XOleObject@COleServerDoc@@8 5f59e178     olesvr1.obj
 0002:00010188       ??_R3XOleObject@COleServerDoc@@8 5f59e188     olesvr1.obj
 0002:00010198       ??_R4XOleObject@COleServerDoc@@6B@ 5f59e198     olesvr1.obj
 0002:000101b0       ??_R1A@?0A@A@XDataObject@COleServerDoc@@8 5f59e1b0     olesvr1.obj
 0002:000101c8       ??_R2XDataObject@COleServerDoc@@8 5f59e1c8     olesvr1.obj
 0002:000101d8       ??_R3XDataObject@COleServerDoc@@8 5f59e1d8     olesvr1.obj
 0002:000101e8       ??_R4XDataObject@COleServerDoc@@6B@ 5f59e1e8     olesvr1.obj
 0002:00010200       ??_R1A@?0A@A@IOleInPlaceObject@@8 5f59e200     olesvr1.obj
 0002:00010218       ??_R1A@?0A@A@XOleInPlaceObject@COleServerDoc@@8 5f59e218     olesvr1.obj
 0002:00010230       ??_R2XOleInPlaceObject@COleServerDoc@@8 5f59e230     olesvr1.obj
 0002:00010248       ??_R3XOleInPlaceObject@COleServerDoc@@8 5f59e248     olesvr1.obj
 0002:00010258       ??_R4XOleInPlaceObject@COleServerDoc@@6B@ 5f59e258     olesvr1.obj
 0002:00010270       ??_R1A@?0A@A@IOleInPlaceActiveObject@@8 5f59e270     olesvr1.obj
 0002:00010288       ??_R1A@?0A@A@XOleInPlaceActiveObject@COleServerDoc@@8 5f59e288     olesvr1.obj
 0002:000102a0       ??_R2XOleInPlaceActiveObject@COleServerDoc@@8 5f59e2a0     olesvr1.obj
 0002:000102b8       ??_R3XOleInPlaceActiveObject@COleServerDoc@@8 5f59e2b8     olesvr1.obj
 0002:000102c8       ??_R4XOleInPlaceActiveObject@COleServerDoc@@6B@ 5f59e2c8     olesvr1.obj
 0002:000102e0       ??_R1A@?0A@A@COleServerItem@@8 5f59e2e0     olesvr2.obj
 0002:000102f8       ??_R2COleServerItem@@8     5f59e2f8     olesvr2.obj
 0002:00010310       ??_R3COleServerItem@@8     5f59e310     olesvr2.obj
 0002:00010320       ??_R4COleServerItem@@6B@   5f59e320     olesvr2.obj
 0002:00010338       ??_R1A@?0A@A@CItemDataSource@COleServerItem@@8 5f59e338     olesvr2.obj
 0002:00010350       ??_R2CItemDataSource@COleServerItem@@8 5f59e350     olesvr2.obj
 0002:00010368       ??_R3CItemDataSource@COleServerItem@@8 5f59e368     olesvr2.obj
 0002:00010378       ??_R4CItemDataSource@COleServerItem@@6B@ 5f59e378     olesvr2.obj
 0002:00010390       ??_R1A@?0A@A@XOleObject@COleServerItem@@8 5f59e390     olesvr2.obj
 0002:000103a8       ??_R2XOleObject@COleServerItem@@8 5f59e3a8     olesvr2.obj
 0002:000103b8       ??_R3XOleObject@COleServerItem@@8 5f59e3b8     olesvr2.obj
 0002:000103c8       ??_R4XOleObject@COleServerItem@@6B@ 5f59e3c8     olesvr2.obj
 0002:000103e0       ??_R1A@?0A@A@XDataObject@COleServerItem@@8 5f59e3e0     olesvr2.obj
 0002:000103f8       ??_R2XDataObject@COleServerItem@@8 5f59e3f8     olesvr2.obj
 0002:00010408       ??_R3XDataObject@COleServerItem@@8 5f59e408     olesvr2.obj
 0002:00010418       ??_R4XDataObject@COleServerItem@@6B@ 5f59e418     olesvr2.obj
 0002:00010430       ??_R1A@?0A@A@COleTemplateServer@@8 5f59e430     oletsvr.obj
 0002:00010448       ??_R2COleTemplateServer@@8 5f59e448     oletsvr.obj
 0002:00010460       ??_R3COleTemplateServer@@8 5f59e460     oletsvr.obj
 0002:00010470       ??_R4COleTemplateServer@@6B@ 5f59e470     oletsvr.obj
 0002:00010488       ??_R1A@?0A@A@CInnerUnknown@@8 5f59e488     oleunk.obj
 0002:000104a0       ??_R2CInnerUnknown@@8      5f59e4a0     oleunk.obj
 0002:000104b0       ??_R3CInnerUnknown@@8      5f59e4b0     oleunk.obj
 0002:000104c0       ??_R4CInnerUnknown@@6B@    5f59e4c0     oleunk.obj
 0002:000104d8       ??_R1A@?0A@A@COleException@@8 5f59e4d8     oleunk.obj
 0002:000104f0       ??_R2COleException@@8      5f59e4f0     oleunk.obj
 0002:00010500       ??_R3COleException@@8      5f59e500     oleunk.obj
 0002:00010510       ??_R4COleException@@6B@    5f59e510     oleunk.obj
 0002:00010528       ??_R1A@?0A@A@CEnumOleVerb@@8 5f59e528     oleverb.obj
 0002:00010540       ??_R2CEnumOleVerb@@8       5f59e540     oleverb.obj
 0002:00010558       ??_R3CEnumOleVerb@@8       5f59e558     oleverb.obj
 0002:00010568       ??_R4CEnumOleVerb@@6B@     5f59e568     oleverb.obj
 0002:00010580       ??_R1A@?0A@A@CView@@8      5f59e580     viewrich.obj
 0002:00010598       ??_R1A@?0A@A@CCtrlView@@8  5f59e598     viewrich.obj
 0002:000105b0       ??_R1A@?0A@A@CRichEditView@@8 5f59e5b0     viewrich.obj
 0002:000105c8       ??_R2CRichEditView@@8      5f59e5c8     viewrich.obj
 0002:000105e8       ??_R3CRichEditView@@8      5f59e5e8     viewrich.obj
 0002:000105f8       ??_R4CRichEditView@@6B@    5f59e5f8     viewrich.obj
 0002:00010610       ??_R1A@?0A@A@IRichEditOleCallback@@8 5f59e610     viewrich.obj
 0002:00010628       ??_R1A@?0A@A@XRichEditOleCallback@CRichEditView@@8 5f59e628     viewrich.obj
 0002:00010640       ??_R2XRichEditOleCallback@CRichEditView@@8 5f59e640     viewrich.obj
 0002:00010650       ??_R3XRichEditOleCallback@CRichEditView@@8 5f59e650     viewrich.obj
 0002:00010660       ??_R4XRichEditOleCallback@CRichEditView@@6B@ 5f59e660     viewrich.obj
 0002:00010678       ??_R2IRichEditOleCallback@@8 5f59e678     viewrich.obj
 0002:00010688       ??_R3IRichEditOleCallback@@8 5f59e688     viewrich.obj
 0002:00010698       ??_R4IRichEditOleCallback@@6B@ 5f59e698     viewrich.obj
 0002:000106b0       ??_R1A@?0A@A@CRichEditDoc@@8 5f59e6b0     viewrich.obj
 0002:000106c8       ??_R2CRichEditDoc@@8       5f59e6c8     viewrich.obj
 0002:000106e8       ??_R3CRichEditDoc@@8       5f59e6e8     viewrich.obj
 0002:000106f8       ??_R4CRichEditDoc@@6B@     5f59e6f8     viewrich.obj
 0002:00010710       ??_R1A@?0A@A@CRichEditCntrItem@@8 5f59e710     viewrich.obj
 0002:00010728       ??_R2CRichEditCntrItem@@8  5f59e728     viewrich.obj
 0002:00010740       ??_R3CRichEditCntrItem@@8  5f59e740     viewrich.obj
 0002:00010750       ??_R4CRichEditCntrItem@@6B@ 5f59e750     viewrich.obj
 0002:00010768       ??_R1A@?0A@A@_AFX_EDIT_STATE@@8 5f59e768     viewrich.obj
 0002:00010780       ??_R1A@?0A@A@_AFX_RICHEDIT_STATE@@8 5f59e780     viewrich.obj
 0002:00010798       ??_R2_AFX_RICHEDIT_STATE@@8 5f59e798     viewrich.obj
 0002:000107a8       ??_R3_AFX_RICHEDIT_STATE@@8 5f59e7a8     viewrich.obj
 0002:000107b8       ??_R4_AFX_RICHEDIT_STATE@@6B@ 5f59e7b8     viewrich.obj
 0002:000107d0       ??_R1A@?0A@A@CMapPtrToPtr@@8 5f59e7d0     oletyplb.obj
 0002:000107e8       ??_R1A@?0A@A@CTypeLibCacheMap@@8 5f59e7e8     oletyplb.obj
 0002:00010800       ??_R2CTypeLibCacheMap@@8   5f59e800     oletyplb.obj
 0002:00010810       ??_R3CTypeLibCacheMap@@8   5f59e810     oletyplb.obj
 0002:00010820       ??_R4CTypeLibCacheMap@@6B@ 5f59e820     oletyplb.obj
 0002:00010838       ??_R1A@?0A@A@CMonikerFile@@8 5f59e838     olemon.obj
 0002:00010850       ??_R2CMonikerFile@@8       5f59e850     olemon.obj
 0002:00010868       ??_R3CMonikerFile@@8       5f59e868     olemon.obj
 0002:00010878       ??_R4CMonikerFile@@6B@     5f59e878     olemon.obj
 0002:00010890       ??_R1A@?0A@A@IBindHost@@8  5f59e890     olemon.obj
 0002:000108a8       ??_R1A@?0A@A@_AfxBindHost@@8 5f59e8a8     olemon.obj
 0002:000108c0       ??_R2_AfxBindHost@@8       5f59e8c0     olemon.obj
 0002:000108d0       ??_R3_AfxBindHost@@8       5f59e8d0     olemon.obj
 0002:000108e0       ??_R4_AfxBindHost@@6B@     5f59e8e0     olemon.obj
 0002:000108f8       ??_R2IBindHost@@8          5f59e8f8     olemon.obj
 0002:00010908       ??_R3IBindHost@@8          5f59e908     olemon.obj
 0002:00010918       ??_R4IBindHost@@6B@        5f59e918     olemon.obj
 0002:00010930       ??_R1A@?0A@A@CDateTimeCtrl@@8 5f59e930     winctrl5.obj
 0002:00010948       ??_R2CDateTimeCtrl@@8      5f59e948     winctrl5.obj
 0002:00010960       ??_R3CDateTimeCtrl@@8      5f59e960     winctrl5.obj
 0002:00010970       ??_R4CDateTimeCtrl@@6B@    5f59e970     winctrl5.obj
 0002:00010988       ??_R1A@?0A@A@CMonthCalCtrl@@8 5f59e988     winctrl5.obj
 0002:000109a0       ??_R2CMonthCalCtrl@@8      5f59e9a0     winctrl5.obj
 0002:000109b8       ??_R3CMonthCalCtrl@@8      5f59e9b8     winctrl5.obj
 0002:000109c8       ??_R4CMonthCalCtrl@@6B@    5f59e9c8     winctrl5.obj
 0002:000109e0       ??_R1A@?0A@A@CScrollView@@8 5f59e9e0     viewhtml.obj
 0002:000109f8       ??_R1A@?0A@A@CFormView@@8  5f59e9f8     viewhtml.obj
 0002:00010a10       ??_R1A@?0A@A@CHtmlView@@8  5f59ea10     viewhtml.obj
 0002:00010a28       ??_R2CHtmlView@@8          5f59ea28     viewhtml.obj
 0002:00010a48       ??_R3CHtmlView@@8          5f59ea48     viewhtml.obj
 0002:00010a58       ??_R4CHtmlView@@6B@        5f59ea58     viewhtml.obj
 0002:00010a70       ??_R1A@?0A@A@COccManager@@8 5f59ea70     occmgr.obj
 0002:00010a88       ??_R2COccManager@@8        5f59ea88     occmgr.obj
 0002:00010a98       ??_R3COccManager@@8        5f59ea98     occmgr.obj
 0002:00010aa8       ??_R4COccManager@@6B@      5f59eaa8     occmgr.obj
 0002:00010ac0       ??_R1A@?0A@A@COleControlContainer@@8 5f59eac0     occcont.obj
 0002:00010ad8       ??_R2COleControlContainer@@8 5f59ead8     occcont.obj
 0002:00010ae8       ??_R3COleControlContainer@@8 5f59eae8     occcont.obj
 0002:00010af8       ??_R4COleControlContainer@@6B@ 5f59eaf8     occcont.obj
 0002:00010b10       ??_R1A@?0A@A@XOleIPFrame@COleControlContainer@@8 5f59eb10     occcont.obj
 0002:00010b28       ??_R2XOleIPFrame@COleControlContainer@@8 5f59eb28     occcont.obj
 0002:00010b40       ??_R3XOleIPFrame@COleControlContainer@@8 5f59eb40     occcont.obj
 0002:00010b50       ??_R4XOleIPFrame@COleControlContainer@@6B@ 5f59eb50     occcont.obj
 0002:00010b68       ??_R1A@?0A@A@XOleContainer@COleControlContainer@@8 5f59eb68     occcont.obj
 0002:00010b80       ??_R2XOleContainer@COleControlContainer@@8 5f59eb80     occcont.obj
 0002:00010b98       ??_R3XOleContainer@COleControlContainer@@8 5f59eb98     occcont.obj
 0002:00010ba8       ??_R4XOleContainer@COleControlContainer@@6B@ 5f59eba8     occcont.obj
 0002:00010bc0       ??_R1A@?0A@A@CEnumUnknown@@8 5f59ebc0     occcont.obj
 0002:00010bd8       ??_R2CEnumUnknown@@8       5f59ebd8     occcont.obj
 0002:00010bf0       ??_R3CEnumUnknown@@8       5f59ebf0     occcont.obj
 0002:00010c00       ??_R4CEnumUnknown@@6B@     5f59ec00     occcont.obj
 0002:00010c18       ??_R1A@?0A@A@COleControlSite@@8 5f59ec18     occsite.obj
 0002:00010c30       ??_R2COleControlSite@@8    5f59ec30     occsite.obj
 0002:00010c40       ??_R3COleControlSite@@8    5f59ec40     occsite.obj
 0002:00010c50       ??_R4COleControlSite@@6B@  5f59ec50     occsite.obj
 0002:00010c68       ??_R1A@?0A@A@XOleClientSite@COleControlSite@@8 5f59ec68     occsite.obj
 0002:00010c80       ??_R2XOleClientSite@COleControlSite@@8 5f59ec80     occsite.obj
 0002:00010c90       ??_R3XOleClientSite@COleControlSite@@8 5f59ec90     occsite.obj
 0002:00010ca0       ??_R4XOleClientSite@COleControlSite@@6B@ 5f59eca0     occsite.obj
 0002:00010cb8       ??_R1A@?0A@A@XOleIPSite@COleControlSite@@8 5f59ecb8     occsite.obj
 0002:00010cd0       ??_R2XOleIPSite@COleControlSite@@8 5f59ecd0     occsite.obj
 0002:00010ce8       ??_R3XOleIPSite@COleControlSite@@8 5f59ece8     occsite.obj
 0002:00010cf8       ??_R4XOleIPSite@COleControlSite@@6B@ 5f59ecf8     occsite.obj
 0002:00010d10       ??_R1A@?0A@A@IOleControlSite@@8 5f59ed10     occsite.obj
 0002:00010d28       ??_R1A@?0A@A@XOleControlSite@COleControlSite@@8 5f59ed28     occsite.obj
 0002:00010d40       ??_R2XOleControlSite@COleControlSite@@8 5f59ed40     occsite.obj
 0002:00010d50       ??_R3XOleControlSite@COleControlSite@@8 5f59ed50     occsite.obj
 0002:00010d60       ??_R4XOleControlSite@COleControlSite@@6B@ 5f59ed60     occsite.obj
 0002:00010d78       ??_R1A@?0A@A@XAmbientProps@COleControlSite@@8 5f59ed78     occsite.obj
 0002:00010d90       ??_R2XAmbientProps@COleControlSite@@8 5f59ed90     occsite.obj
 0002:00010da0       ??_R3XAmbientProps@COleControlSite@@8 5f59eda0     occsite.obj
 0002:00010db0       ??_R4XAmbientProps@COleControlSite@@6B@ 5f59edb0     occsite.obj
 0002:00010dc8       ??_R1A@?0A@A@IPropertyNotifySink@@8 5f59edc8     occsite.obj
 0002:00010de0       ??_R1A@?0A@A@XPropertyNotifySink@COleControlSite@@8 5f59ede0     occsite.obj
 0002:00010df8       ??_R2XPropertyNotifySink@COleControlSite@@8 5f59edf8     occsite.obj
 0002:00010e08       ??_R3XPropertyNotifySink@COleControlSite@@8 5f59ee08     occsite.obj
 0002:00010e18       ??_R4XPropertyNotifySink@COleControlSite@@6B@ 5f59ee18     occsite.obj
 0002:00010e30       ??_R1A@?0A@A@XEventSink@COleControlSite@@8 5f59ee30     occsite.obj
 0002:00010e48       ??_R2XEventSink@COleControlSite@@8 5f59ee48     occsite.obj
 0002:00010e58       ??_R3XEventSink@COleControlSite@@8 5f59ee58     occsite.obj
 0002:00010e68       ??_R4XEventSink@COleControlSite@@6B@ 5f59ee68     occsite.obj
 0002:00010e80       ??_R1A@?0A@A@IBoundObjectSite@@8 5f59ee80     occsite.obj
 0002:00010e98       ??_R1A@?0A@A@XBoundObjectSite@COleControlSite@@8 5f59ee98     occsite.obj
 0002:00010eb0       ??_R2XBoundObjectSite@COleControlSite@@8 5f59eeb0     occsite.obj
 0002:00010ec0       ??_R3XBoundObjectSite@COleControlSite@@8 5f59eec0     occsite.obj
 0002:00010ed0       ??_R4XBoundObjectSite@COleControlSite@@6B@ 5f59eed0     occsite.obj
 0002:00010ee8       ??_R1A@?0A@A@INotifyDBEvents@@8 5f59eee8     occsite.obj
 0002:00010f00       ??_R1A@?0A@A@XNotifyDBEvents@COleControlSite@@8 5f59ef00     occsite.obj
 0002:00010f18       ??_R2XNotifyDBEvents@COleControlSite@@8 5f59ef18     occsite.obj
 0002:00010f28       ??_R3XNotifyDBEvents@COleControlSite@@8 5f59ef28     occsite.obj
 0002:00010f38       ??_R4XNotifyDBEvents@COleControlSite@@6B@ 5f59ef38     occsite.obj
 0002:00010f50       ??_R1A@?0A@A@IRowsetNotify@@8 5f59ef50     occsite.obj
 0002:00010f68       ??_R1A@?0A@A@XRowsetNotify@COleControlSite@@8 5f59ef68     occsite.obj
 0002:00010f80       ??_R2XRowsetNotify@COleControlSite@@8 5f59ef80     occsite.obj
 0002:00010f90       ??_R3XRowsetNotify@COleControlSite@@8 5f59ef90     occsite.obj
 0002:00010fa0       ??_R4XRowsetNotify@COleControlSite@@6B@ 5f59efa0     occsite.obj
 0002:00010fb8       ??_R2IBoundObjectSite@@8   5f59efb8     occsite.obj
 0002:00010fc8       ??_R3IBoundObjectSite@@8   5f59efc8     occsite.obj
 0002:00010fd8       ??_R4IBoundObjectSite@@6B@ 5f59efd8     occsite.obj
 0002:00010ff0       ??_R2INotifyDBEvents@@8    5f59eff0     occsite.obj
 0002:00011000       ??_R3INotifyDBEvents@@8    5f59f000     occsite.obj
 0002:00011010       ??_R4INotifyDBEvents@@6B@  5f59f010     occsite.obj
 0002:00011028       ??_R2IRowsetNotify@@8      5f59f028     occsite.obj
 0002:00011038       ??_R3IRowsetNotify@@8      5f59f038     occsite.obj
 0002:00011048       ??_R4IRowsetNotify@@6B@    5f59f048     occsite.obj
 0002:00011060       ??_R1A@?0A@A@CDataSourceControl@@8 5f59f060     occsite.obj
 0002:00011078       ??_R2CDataSourceControl@@8 5f59f078     occsite.obj
 0002:00011080       ??_R3CDataSourceControl@@8 5f59f080     occsite.obj
 0002:00011090       ??_R4CDataSourceControl@@6B@ 5f59f090     occsite.obj
 0002:000110a8       ??_R1A@?0A@A@COleControlLock@@8 5f59f0a8     occlock.obj
 0002:000110c0       ??_R2COleControlLock@@8    5f59f0c0     occlock.obj
 0002:000110c8       ??_R3COleControlLock@@8    5f59f0c8     occlock.obj
 0002:000110d8       ??_R4COleControlLock@@6B@  5f59f0d8     occlock.obj
 0002:000110f0       ??_R1A@?0A@A@CDocObjectServer@@8 5f59f0f0     oledocob.obj
 0002:00011108       ??_R2CDocObjectServer@@8   5f59f108     oledocob.obj
 0002:00011118       ??_R3CDocObjectServer@@8   5f59f118     oledocob.obj
 0002:00011128       ??_R4CDocObjectServer@@6B@ 5f59f128     oledocob.obj
 0002:00011140       ??_R1A@?0A@A@XOleObject@CDocObjectServer@@8 5f59f140     oledocob.obj
 0002:00011158       ??_R2XOleObject@CDocObjectServer@@8 5f59f158     oledocob.obj
 0002:00011168       ??_R3XOleObject@CDocObjectServer@@8 5f59f168     oledocob.obj
 0002:00011178       ??_R4XOleObject@CDocObjectServer@@6B@ 5f59f178     oledocob.obj
 0002:00011190       ??_R1A@?0A@A@IOleDocument@@8 5f59f190     oledocob.obj
 0002:000111a8       ??_R1A@?0A@A@XOleDocument@CDocObjectServer@@8 5f59f1a8     oledocob.obj
 0002:000111c0       ??_R2XOleDocument@CDocObjectServer@@8 5f59f1c0     oledocob.obj
 0002:000111d0       ??_R3XOleDocument@CDocObjectServer@@8 5f59f1d0     oledocob.obj
 0002:000111e0       ??_R4XOleDocument@CDocObjectServer@@6B@ 5f59f1e0     oledocob.obj
 0002:000111f8       ??_R1A@?0A@A@IOleDocumentView@@8 5f59f1f8     oledocob.obj
 0002:00011210       ??_R1A@?0A@A@XOleDocumentView@CDocObjectServer@@8 5f59f210     oledocob.obj
 0002:00011228       ??_R2XOleDocumentView@CDocObjectServer@@8 5f59f228     oledocob.obj
 0002:00011238       ??_R3XOleDocumentView@CDocObjectServer@@8 5f59f238     oledocob.obj
 0002:00011248       ??_R4XOleDocumentView@CDocObjectServer@@6B@ 5f59f248     oledocob.obj
 0002:00011260       ??_R1A@?0A@A@XOleCommandTarget@CDocObjectServer@@8 5f59f260     oledocob.obj
 0002:00011278       ??_R2XOleCommandTarget@CDocObjectServer@@8 5f59f278     oledocob.obj
 0002:00011288       ??_R3XOleCommandTarget@CDocObjectServer@@8 5f59f288     oledocob.obj
 0002:00011298       ??_R4XOleCommandTarget@CDocObjectServer@@6B@ 5f59f298     oledocob.obj
 0002:000112b0       ??_R1A@?0A@A@IPrint@@8     5f59f2b0     oledocob.obj
 0002:000112c8       ??_R1A@?0A@A@XPrint@CDocObjectServer@@8 5f59f2c8     oledocob.obj
 0002:000112e0       ??_R2XPrint@CDocObjectServer@@8 5f59f2e0     oledocob.obj
 0002:000112f0       ??_R3XPrint@CDocObjectServer@@8 5f59f2f0     oledocob.obj
 0002:00011300       ??_R4XPrint@CDocObjectServer@@6B@ 5f59f300     oledocob.obj
 0002:00011318       ??_R1A@?0A@A@CDocObjectServerItem@@8 5f59f318     oledocob.obj
 0002:00011330       ??_R2CDocObjectServerItem@@8 5f59f330     oledocob.obj
 0002:00011348       ??_R3CDocObjectServerItem@@8 5f59f348     oledocob.obj
 0002:00011358       ??_R4CDocObjectServerItem@@6B@ 5f59f358     oledocob.obj
 0002:00011370       ??_R1A@?0A@A@CCmdUI@@8     5f59f370     oledoctg.obj
 0002:00011388       ??_R1A@?0A@A@COleCmdUI@@8  5f59f388     oledoctg.obj
 0002:000113a0       ??_R2COleCmdUI@@8          5f59f3a0     oledoctg.obj
 0002:000113b0       ??_R3COleCmdUI@@8          5f59f3b0     oledoctg.obj
 0002:000113c0       ??_R4COleCmdUI@@6B@        5f59f3c0     oledoctg.obj
 0002:000113d8       ??_R1A@?0A@A@COleDocIPFrameWnd@@8 5f59f3d8     oledocip.obj
 0002:000113f0       ??_R2COleDocIPFrameWnd@@8  5f59f3f0     oledocip.obj
 0002:00011410       ??_R3COleDocIPFrameWnd@@8  5f59f410     oledocip.obj
 0002:00011420       ??_R4COleDocIPFrameWnd@@6B@ 5f59f420     oledocip.obj
 0002:00011438       ??_R1A@?0A@A@COleDocObjectItem@@8 5f59f438     oledoccl.obj
 0002:00011450       ??_R2COleDocObjectItem@@8  5f59f450     oledoccl.obj
 0002:00011468       ??_R3COleDocObjectItem@@8  5f59f468     oledoccl.obj
 0002:00011478       ??_R4COleDocObjectItem@@6B@ 5f59f478     oledoccl.obj
 0002:00011490       ??_R1A@?0A@A@IOleDocumentSite@@8 5f59f490     oledoccl.obj
 0002:000114a8       ??_R1A@?0A@A@XOleDocumentSite@COleDocObjectItem@@8 5f59f4a8     oledoccl.obj
 0002:000114c0       ??_R2XOleDocumentSite@COleDocObjectItem@@8 5f59f4c0     oledoccl.obj
 0002:000114d0       ??_R3XOleDocumentSite@COleDocObjectItem@@8 5f59f4d0     oledoccl.obj
 0002:000114e0       ??_R4XOleDocumentSite@COleDocObjectItem@@6B@ 5f59f4e0     oledoccl.obj
 0002:000114f8       ??_R1A@?0A@A@CAsyncMonikerFile@@8 5f59f4f8     oleasmon.obj
 0002:00011510       ??_R2CAsyncMonikerFile@@8  5f59f510     oleasmon.obj
 0002:00011528       ??_R3CAsyncMonikerFile@@8  5f59f528     oleasmon.obj
 0002:00011538       ??_R4CAsyncMonikerFile@@6B@ 5f59f538     oleasmon.obj
 0002:00011550       ??_R1A@?0A@A@IBindStatusCallback@@8 5f59f550     oleasmon.obj
 0002:00011568       ??_R1A@?0A@A@_AfxBindStatusCallback@@8 5f59f568     oleasmon.obj
 0002:00011580       ??_R2_AfxBindStatusCallback@@8 5f59f580     oleasmon.obj
 0002:00011590       ??_R3_AfxBindStatusCallback@@8 5f59f590     oleasmon.obj
 0002:000115a0       ??_R4_AfxBindStatusCallback@@6B@ 5f59f5a0     oleasmon.obj
 0002:000115b8       ??_R1A@?0A@A@CInnerUnknown@_AfxBindStatusCallback@@8 5f59f5b8     oleasmon.obj
 0002:000115d0       ??_R2CInnerUnknown@_AfxBindStatusCallback@@8 5f59f5d0     oleasmon.obj
 0002:000115e0       ??_R3CInnerUnknown@_AfxBindStatusCallback@@8 5f59f5e0     oleasmon.obj
 0002:000115f0       ??_R4CInnerUnknown@_AfxBindStatusCallback@@6B@ 5f59f5f0     oleasmon.obj
 0002:00011608       ??_R2IBindStatusCallback@@8 5f59f608     oleasmon.obj
 0002:00011618       ??_R3IBindStatusCallback@@8 5f59f618     oleasmon.obj
 0002:00011628       ??_R4IBindStatusCallback@@6B@ 5f59f628     oleasmon.obj
 0002:00011640       ??_R1A@?0A@A@CControlBar@@8 5f59f640     olebar.obj
 0002:00011658       ??_R1A@?0A@A@COleResizeBar@@8 5f59f658     olebar.obj
 0002:00011670       ??_R2COleResizeBar@@8      5f59f670     olebar.obj
 0002:00011688       ??_R3COleResizeBar@@8      5f59f688     olebar.obj
 0002:00011698       ??_R4COleResizeBar@@6B@    5f59f698     olebar.obj
 0002:000116b0       ??_R1A@?0A@A@COleControl@@8 5f59f6b0     ctlcore.obj
 0002:000116c8       ??_R2COleControl@@8        5f59f6c8     ctlcore.obj
 0002:000116e0       ??_R3COleControl@@8        5f59f6e0     ctlcore.obj
 0002:000116f0       ??_R4COleControl@@6B@      5f59f6f0     ctlcore.obj
 0002:00011708       ??_R1A@?0A@A@XPersistStorage@COleControl@@8 5f59f708     ctlcore.obj
 0002:00011720       ??_R2XPersistStorage@COleControl@@8 5f59f720     ctlcore.obj
 0002:00011738       ??_R3XPersistStorage@COleControl@@8 5f59f738     ctlcore.obj
 0002:00011748       ??_R4XPersistStorage@COleControl@@6B@ 5f59f748     ctlcore.obj
 0002:00011760       ??_R1A@?0A@A@IPersistStreamInit@@8 5f59f760     ctlcore.obj
 0002:00011778       ??_R1A@?0A@A@XPersistStreamInit@COleControl@@8 5f59f778     ctlcore.obj
 0002:00011790       ??_R2XPersistStreamInit@COleControl@@8 5f59f790     ctlcore.obj
 0002:000117a8       ??_R3XPersistStreamInit@COleControl@@8 5f59f7a8     ctlcore.obj
 0002:000117b8       ??_R4XPersistStreamInit@COleControl@@6B@ 5f59f7b8     ctlcore.obj
 0002:000117d0       ??_R1A@?0A@A@IPersistMemory@@8 5f59f7d0     ctlcore.obj
 0002:000117e8       ??_R1A@?0A@A@XPersistMemory@COleControl@@8 5f59f7e8     ctlcore.obj
 0002:00011800       ??_R2XPersistMemory@COleControl@@8 5f59f800     ctlcore.obj
 0002:00011818       ??_R3XPersistMemory@COleControl@@8 5f59f818     ctlcore.obj
 0002:00011828       ??_R4XPersistMemory@COleControl@@6B@ 5f59f828     ctlcore.obj
 0002:00011840       ??_R1A@?0A@A@IPersistPropertyBag@@8 5f59f840     ctlcore.obj
 0002:00011858       ??_R1A@?0A@A@XPersistPropertyBag@COleControl@@8 5f59f858     ctlcore.obj
 0002:00011870       ??_R2XPersistPropertyBag@COleControl@@8 5f59f870     ctlcore.obj
 0002:00011888       ??_R3XPersistPropertyBag@COleControl@@8 5f59f888     ctlcore.obj
 0002:00011898       ??_R4XPersistPropertyBag@COleControl@@6B@ 5f59f898     ctlcore.obj
 0002:000118b0       ??_R1A@?0A@A@XOleObject@COleControl@@8 5f59f8b0     ctlcore.obj
 0002:000118c8       ??_R2XOleObject@COleControl@@8 5f59f8c8     ctlcore.obj
 0002:000118d8       ??_R3XOleObject@COleControl@@8 5f59f8d8     ctlcore.obj
 0002:000118e8       ??_R4XOleObject@COleControl@@6B@ 5f59f8e8     ctlcore.obj
 0002:00011900       ??_R1A@?0A@A@IViewObject@@8 5f59f900     ctlcore.obj
 0002:00011918       ??_R1A@?0A@A@IViewObject2@@8 5f59f918     ctlcore.obj
 0002:00011930       ??_R1A@?0A@A@IViewObjectEx@@8 5f59f930     ctlcore.obj
 0002:00011948       ??_R1A@?0A@A@XViewObject@COleControl@@8 5f59f948     ctlcore.obj
 0002:00011960       ??_R2XViewObject@COleControl@@8 5f59f960     ctlcore.obj
 0002:00011978       ??_R3XViewObject@COleControl@@8 5f59f978     ctlcore.obj
 0002:00011988       ??_R4XViewObject@COleControl@@6B@ 5f59f988     ctlcore.obj
 0002:000119a0       ??_R1A@?0A@A@XDataObject@COleControl@@8 5f59f9a0     ctlcore.obj
 0002:000119b8       ??_R2XDataObject@COleControl@@8 5f59f9b8     ctlcore.obj
 0002:000119c8       ??_R3XDataObject@COleControl@@8 5f59f9c8     ctlcore.obj
 0002:000119d8       ??_R4XDataObject@COleControl@@6B@ 5f59f9d8     ctlcore.obj
 0002:000119f0       ??_R1A@?0A@A@IOleInPlaceObjectWindowless@@8 5f59f9f0     ctlcore.obj
 0002:00011a08       ??_R1A@?0A@A@XOleInPlaceObject@COleControl@@8 5f59fa08     ctlcore.obj
 0002:00011a20       ??_R2XOleInPlaceObject@COleControl@@8 5f59fa20     ctlcore.obj
 0002:00011a38       ??_R3XOleInPlaceObject@COleControl@@8 5f59fa38     ctlcore.obj
 0002:00011a48       ??_R4XOleInPlaceObject@COleControl@@6B@ 5f59fa48     ctlcore.obj
 0002:00011a60       ??_R1A@?0A@A@XOleInPlaceActiveObject@COleControl@@8 5f59fa60     ctlcore.obj
 0002:00011a78       ??_R2XOleInPlaceActiveObject@COleControl@@8 5f59fa78     ctlcore.obj
 0002:00011a90       ??_R3XOleInPlaceActiveObject@COleControl@@8 5f59fa90     ctlcore.obj
 0002:00011aa0       ??_R4XOleInPlaceActiveObject@COleControl@@6B@ 5f59faa0     ctlcore.obj
 0002:00011ab8       ??_R1A@?0A@A@IOleCache@@8  5f59fab8     ctlcore.obj
 0002:00011ad0       ??_R1A@?0A@A@XOleCache@COleControl@@8 5f59fad0     ctlcore.obj
 0002:00011ae8       ??_R2XOleCache@COleControl@@8 5f59fae8     ctlcore.obj
 0002:00011af8       ??_R3XOleCache@COleControl@@8 5f59faf8     ctlcore.obj
 0002:00011b08       ??_R4XOleCache@COleControl@@6B@ 5f59fb08     ctlcore.obj
 0002:00011b20       ??_R1A@?0A@A@IOleControl@@8 5f59fb20     ctlcore.obj
 0002:00011b38       ??_R1A@?0A@A@XOleControl@COleControl@@8 5f59fb38     ctlcore.obj
 0002:00011b50       ??_R2XOleControl@COleControl@@8 5f59fb50     ctlcore.obj
 0002:00011b60       ??_R3XOleControl@COleControl@@8 5f59fb60     ctlcore.obj
 0002:00011b70       ??_R4XOleControl@COleControl@@6B@ 5f59fb70     ctlcore.obj
 0002:00011b88       ??_R1A@?0A@A@IProvideClassInfo@@8 5f59fb88     ctlcore.obj
 0002:00011ba0       ??_R1A@?0A@A@IProvideClassInfo2@@8 5f59fba0     ctlcore.obj
 0002:00011bb8       ??_R1A@?0A@A@XProvideClassInfo@COleControl@@8 5f59fbb8     ctlcore.obj
 0002:00011bd0       ??_R2XProvideClassInfo@COleControl@@8 5f59fbd0     ctlcore.obj
 0002:00011be8       ??_R3XProvideClassInfo@COleControl@@8 5f59fbe8     ctlcore.obj
 0002:00011bf8       ??_R4XProvideClassInfo@COleControl@@6B@ 5f59fbf8     ctlcore.obj
 0002:00011c10       ??_R1A@?0A@A@ISpecifyPropertyPages@@8 5f59fc10     ctlcore.obj
 0002:00011c28       ??_R1A@?0A@A@XSpecifyPropertyPages@COleControl@@8 5f59fc28     ctlcore.obj
 0002:00011c40       ??_R2XSpecifyPropertyPages@COleControl@@8 5f59fc40     ctlcore.obj
 0002:00011c50       ??_R3XSpecifyPropertyPages@COleControl@@8 5f59fc50     ctlcore.obj
 0002:00011c60       ??_R4XSpecifyPropertyPages@COleControl@@6B@ 5f59fc60     ctlcore.obj
 0002:00011c78       ??_R1A@?0A@A@IPerPropertyBrowsing@@8 5f59fc78     ctlcore.obj
 0002:00011c90       ??_R1A@?0A@A@XPerPropertyBrowsing@COleControl@@8 5f59fc90     ctlcore.obj
 0002:00011ca8       ??_R2XPerPropertyBrowsing@COleControl@@8 5f59fca8     ctlcore.obj
 0002:00011cb8       ??_R3XPerPropertyBrowsing@COleControl@@8 5f59fcb8     ctlcore.obj
 0002:00011cc8       ??_R4XPerPropertyBrowsing@COleControl@@6B@ 5f59fcc8     ctlcore.obj
 0002:00011ce0       ??_R1A@?0A@A@XFontNotification@COleControl@@8 5f59fce0     ctlcore.obj
 0002:00011cf8       ??_R2XFontNotification@COleControl@@8 5f59fcf8     ctlcore.obj
 0002:00011d08       ??_R3XFontNotification@COleControl@@8 5f59fd08     ctlcore.obj
 0002:00011d18       ??_R4XFontNotification@COleControl@@6B@ 5f59fd18     ctlcore.obj
 0002:00011d30       ??_R1A@?0A@A@IQuickActivate@@8 5f59fd30     ctlcore.obj
 0002:00011d48       ??_R1A@?0A@A@XQuickActivate@COleControl@@8 5f59fd48     ctlcore.obj
 0002:00011d60       ??_R2XQuickActivate@COleControl@@8 5f59fd60     ctlcore.obj
 0002:00011d70       ??_R3XQuickActivate@COleControl@@8 5f59fd70     ctlcore.obj
 0002:00011d80       ??_R4XQuickActivate@COleControl@@6B@ 5f59fd80     ctlcore.obj
 0002:00011d98       ??_R1A@?0A@A@IPointerInactive@@8 5f59fd98     ctlcore.obj
 0002:00011db0       ??_R1A@?0A@A@XPointerInactive@COleControl@@8 5f59fdb0     ctlcore.obj
 0002:00011dc8       ??_R2XPointerInactive@COleControl@@8 5f59fdc8     ctlcore.obj
 0002:00011dd8       ??_R3XPointerInactive@COleControl@@8 5f59fdd8     ctlcore.obj
 0002:00011de8       ??_R4XPointerInactive@COleControl@@6B@ 5f59fde8     ctlcore.obj
 0002:00011e00       ??_R1A@?0A@A@CConnectionPoint@@8 5f59fe00     ctlcore.obj
 0002:00011e18       ??_R1A@?0A@A@XEventConnPt@COleControl@@8 5f59fe18     ctlcore.obj
 0002:00011e30       ??_R2XEventConnPt@COleControl@@8 5f59fe30     ctlcore.obj
 0002:00011e48       ??_R3XEventConnPt@COleControl@@8 5f59fe48     ctlcore.obj
 0002:00011e58       ??_R4XEventConnPt@COleControl@@6B@ 5f59fe58     ctlcore.obj
 0002:00011e70       ??_R1A@?0A@A@XPropConnPt@COleControl@@8 5f59fe70     ctlcore.obj
 0002:00011e88       ??_R2XPropConnPt@COleControl@@8 5f59fe88     ctlcore.obj
 0002:00011ea0       ??_R3XPropConnPt@COleControl@@8 5f59fea0     ctlcore.obj
 0002:00011eb0       ??_R4XPropConnPt@COleControl@@6B@ 5f59feb0     ctlcore.obj
 0002:00011ec8       ??_R1A@?0A@A@CReflectorWnd@@8 5f59fec8     ctlcore.obj
 0002:00011ee0       ??_R2CReflectorWnd@@8      5f59fee0     ctlcore.obj
 0002:00011ef8       ??_R3CReflectorWnd@@8      5f59fef8     ctlcore.obj
 0002:00011f08       ??_R4CReflectorWnd@@6B@    5f59ff08     ctlcore.obj
 0002:00011f20       ??_R1A@?0A@A@CParkingWnd@@8 5f59ff20     ctlcore.obj
 0002:00011f38       ??_R2CParkingWnd@@8        5f59ff38     ctlcore.obj
 0002:00011f50       ??_R3CParkingWnd@@8        5f59ff50     ctlcore.obj
 0002:00011f60       ??_R4CParkingWnd@@6B@      5f59ff60     ctlcore.obj
 0002:00011f78       ??_R1A@?0A@A@CControlDataSource@COleControl@@8 5f59ff78     ctldata.obj
 0002:00011f90       ??_R2CControlDataSource@COleControl@@8 5f59ff90     ctldata.obj
 0002:00011fa8       ??_R3CControlDataSource@COleControl@@8 5f59ffa8     ctldata.obj
 0002:00011fb8       ??_R4CControlDataSource@COleControl@@6B@ 5f59ffb8     ctldata.obj
 0002:00011fd0       ??_R1A@?0A@A@CControlFrameWnd@@8 5f59ffd0     ctlframe.obj
 0002:00011fe8       ??_R2CControlFrameWnd@@8   5f59ffe8     ctlframe.obj
 0002:00012000       ??_R3CControlFrameWnd@@8   5f5a0000     ctlframe.obj
 0002:00012010       ??_R4CControlFrameWnd@@6B@ 5f5a0010     ctlframe.obj
 0002:00012028       ??_R2CConnectionPoint@@8   5f5a0028     oleconn.obj
 0002:00012038       ??_R3CConnectionPoint@@8   5f5a0038     oleconn.obj
 0002:00012048       ??_R4CConnectionPoint@@6B@ 5f5a0048     oleconn.obj
 0002:00012060       ??_R1A@?0A@A@IConnectionPoint@@8 5f5a0060     oleconn.obj
 0002:00012078       ??_R1A@?0A@A@XConnPt@CConnectionPoint@@8 5f5a0078     oleconn.obj
 0002:00012090       ??_R2XConnPt@CConnectionPoint@@8 5f5a0090     oleconn.obj
 0002:000120a0       ??_R3XConnPt@CConnectionPoint@@8 5f5a00a0     oleconn.obj
 0002:000120b0       ??_R4XConnPt@CConnectionPoint@@6B@ 5f5a00b0     oleconn.obj
 0002:000120c8       ??_R1A@?0A@A@CEnumConnections@@8 5f5a00c8     oleconn.obj
 0002:000120e0       ??_R2CEnumConnections@@8   5f5a00e0     oleconn.obj
 0002:000120f8       ??_R3CEnumConnections@@8   5f5a00f8     oleconn.obj
 0002:00012108       ??_R4CEnumConnections@@6B@ 5f5a0108     oleconn.obj
 0002:00012120       ??_R1A@?0A@A@CEnumConnPoints@@8 5f5a0120     oleconn.obj
 0002:00012138       ??_R2CEnumConnPoints@@8    5f5a0138     oleconn.obj
 0002:00012150       ??_R3CEnumConnPoints@@8    5f5a0150     oleconn.obj
 0002:00012160       ??_R4CEnumConnPoints@@6B@  5f5a0160     oleconn.obj
 0002:00012178       ??_R1A@?0A@A@IConnectionPointContainer@@8 5f5a0178     oleconn.obj
 0002:00012190       ??_R1A@?0A@A@COleConnPtContainer@@8 5f5a0190     oleconn.obj
 0002:000121a8       ??_R2COleConnPtContainer@@8 5f5a01a8     oleconn.obj
 0002:000121b8       ??_R3COleConnPtContainer@@8 5f5a01b8     oleconn.obj
 0002:000121c8       ??_R4COleConnPtContainer@@6B@ 5f5a01c8     oleconn.obj
 0002:000121e0       ??_R1A@?0A@A@CPropExchange@@8 5f5a01e0     ctlpropx.obj
 0002:000121f8       ??_R1A@?0A@A@CArchivePropExchange@@8 5f5a01f8     ctlpropx.obj
 0002:00012210       ??_R2CArchivePropExchange@@8 5f5a0210     ctlpropx.obj
 0002:00012220       ??_R3CArchivePropExchange@@8 5f5a0220     ctlpropx.obj
 0002:00012230       ??_R4CArchivePropExchange@@6B@ 5f5a0230     ctlpropx.obj
 0002:00012248       ??_R1A@?0A@A@CResetPropExchange@@8 5f5a0248     ctlpropx.obj
 0002:00012260       ??_R2CResetPropExchange@@8 5f5a0260     ctlpropx.obj
 0002:00012270       ??_R3CResetPropExchange@@8 5f5a0270     ctlpropx.obj
 0002:00012280       ??_R4CResetPropExchange@@6B@ 5f5a0280     ctlpropx.obj
 0002:00012298       ??_R1A@?0A@A@CAsyncPropExchange@@8 5f5a0298     ctlpropx.obj
 0002:000122b0       ??_R2CAsyncPropExchange@@8 5f5a02b0     ctlpropx.obj
 0002:000122c0       ??_R3CAsyncPropExchange@@8 5f5a02c0     ctlpropx.obj
 0002:000122d0       ??_R4CAsyncPropExchange@@6B@ 5f5a02d0     ctlpropx.obj
 0002:000122e8       ??_R1A@?0A@A@AFX_DDPDATA@@8 5f5a02e8     ctlppg.obj
 0002:00012300       ??_R2AFX_DDPDATA@@8        5f5a0300     ctlppg.obj
 0002:00012310       ??_R3AFX_DDPDATA@@8        5f5a0310     ctlppg.obj
 0002:00012320       ??_R4AFX_DDPDATA@@6B@      5f5a0320     ctlppg.obj
 0002:00012338       ??_R1A@?0A@A@COlePropertyPage@@8 5f5a0338     ctlppg.obj
 0002:00012350       ??_R2COlePropertyPage@@8   5f5a0350     ctlppg.obj
 0002:00012368       ??_R3COlePropertyPage@@8   5f5a0368     ctlppg.obj
 0002:00012378       ??_R4COlePropertyPage@@6B@ 5f5a0378     ctlppg.obj
 0002:00012390       ??_R1A@?0A@A@IPropertyPage@@8 5f5a0390     ctlppg.obj
 0002:000123a8       ??_R1A@?0A@A@IPropertyPage2@@8 5f5a03a8     ctlppg.obj
 0002:000123c0       ??_R1A@?0A@A@XPropertyPage@COlePropertyPage@@8 5f5a03c0     ctlppg.obj
 0002:000123d8       ??_R2XPropertyPage@COlePropertyPage@@8 5f5a03d8     ctlppg.obj
 0002:000123f0       ??_R3XPropertyPage@COlePropertyPage@@8 5f5a03f0     ctlppg.obj
 0002:00012400       ??_R4XPropertyPage@COlePropertyPage@@6B@ 5f5a0400     ctlppg.obj
 0002:00012418       ??_R1A@?0A@A@XPropNotifySink@COlePropertyPage@@8 5f5a0418     ctlppg.obj
 0002:00012430       ??_R2XPropNotifySink@COlePropertyPage@@8 5f5a0430     ctlppg.obj
 0002:00012440       ??_R3XPropNotifySink@COlePropertyPage@@8 5f5a0440     ctlppg.obj
 0002:00012450       ??_R4XPropNotifySink@COlePropertyPage@@6B@ 5f5a0450     ctlppg.obj
 0002:00012468       ??_R1A@?0A@A@CPropsetPropExchange@@8 5f5a0468     ctlpset.obj
 0002:00012480       ??_R2CPropsetPropExchange@@8 5f5a0480     ctlpset.obj
 0002:00012490       ??_R3CPropsetPropExchange@@8 5f5a0490     ctlpset.obj
 0002:000124a0       ??_R4CPropsetPropExchange@@6B@ 5f5a04a0     ctlpset.obj
 0002:000124b8       ??_R1A@?0A@A@CRectTracker@@8 5f5a04b8     ctltrack.obj
 0002:000124d0       ??_R1A@?0A@A@CControlRectTracker@@8 5f5a04d0     ctltrack.obj
 0002:000124e8       ??_R2CControlRectTracker@@8 5f5a04e8     ctltrack.obj
 0002:000124f8       ??_R3CControlRectTracker@@8 5f5a04f8     ctltrack.obj
 0002:00012508       ??_R4CControlRectTracker@@6B@ 5f5a0508     ctltrack.obj
 0002:00012520       ??_R1A@?0A@A@IPersistStream@@8 5f5a0520     ctlpbag.obj
 0002:00012538       ??_R1A@?0A@A@CBlobProperty@@8 5f5a0538     ctlpbag.obj
 0002:00012550       ??_R2CBlobProperty@@8      5f5a0550     ctlpbag.obj
 0002:00012568       ??_R3CBlobProperty@@8      5f5a0568     ctlpbag.obj
 0002:00012578       ??_R4CBlobProperty@@6B@    5f5a0578     ctlpbag.obj
 0002:00012590       ??_R1A@?0A@A@CPropbagPropExchange@@8 5f5a0590     ctlpbag.obj
 0002:000125a8       ??_R2CPropbagPropExchange@@8 5f5a05a8     ctlpbag.obj
 0002:000125b8       ??_R3CPropbagPropExchange@@8 5f5a05b8     ctlpbag.obj
 0002:000125c8       ??_R4CPropbagPropExchange@@6B@ 5f5a05c8     ctlpbag.obj
 0002:000125e0       ??_R1A@?0A@A@_AFXCTL_AMBIENT_CACHE@@8 5f5a05e0     ctlquick.obj
 0002:000125f8       ??_R2_AFXCTL_AMBIENT_CACHE@@8 5f5a05f8     ctlquick.obj
 0002:00012608       ??_R3_AFXCTL_AMBIENT_CACHE@@8 5f5a0608     ctlquick.obj
 0002:00012618       ??_R4_AFXCTL_AMBIENT_CACHE@@6B@ 5f5a0618     ctlquick.obj
 0002:00012630       ??_R1A@?0A@A@CDC@@8        5f5a0630     ctlnownd.obj
 0002:00012648       ??_R1A@?0A@A@CWindowlessDC@@8 5f5a0648     ctlnownd.obj
 0002:00012660       ??_R2CWindowlessDC@@8      5f5a0660     ctlnownd.obj
 0002:00012670       ??_R3CWindowlessDC@@8      5f5a0670     ctlnownd.obj
 0002:00012680       ??_R4CWindowlessDC@@6B@    5f5a0680     ctlnownd.obj
 0002:00012698       ??_R1A@?0A@A@CButton@@8    5f5a0698     ppgcolor.obj
 0002:000126b0       ??_R1A@?0A@A@CColorButton@@8 5f5a06b0     ppgcolor.obj
 0002:000126c8       ??_R2CColorButton@@8       5f5a06c8     ppgcolor.obj
 0002:000126e0       ??_R3CColorButton@@8       5f5a06e0     ppgcolor.obj
 0002:000126f0       ??_R4CColorButton@@6B@     5f5a06f0     ppgcolor.obj
 0002:00012708       ??_R1A@?0A@A@CStockPropPage@@8 5f5a0708     ppgcolor.obj
 0002:00012720       ??_R1A@?0A@A@CColorPropPage@@8 5f5a0720     ppgcolor.obj
 0002:00012738       ??_R2CColorPropPage@@8     5f5a0738     ppgcolor.obj
 0002:00012758       ??_R3CColorPropPage@@8     5f5a0758     ppgcolor.obj
 0002:00012768       ??_R4CColorPropPage@@6B@   5f5a0768     ppgcolor.obj
 0002:00012780       ??_R1A@?0A@A@CColorPropPageFactory@CColorPropPage@@8 5f5a0780     ppgcolor.obj
 0002:00012798       ??_R2CColorPropPageFactory@CColorPropPage@@8 5f5a0798     ppgcolor.obj
 0002:000127b0       ??_R3CColorPropPageFactory@CColorPropPage@@8 5f5a07b0     ppgcolor.obj
 0002:000127c0       ??_R4CColorPropPageFactory@CColorPropPage@@6B@ 5f5a07c0     ppgcolor.obj
 0002:000127d8       ??_R1A@?0A@A@CFontPropPage@@8 5f5a07d8     ppgfont.obj
 0002:000127f0       ??_R2CFontPropPage@@8      5f5a07f0     ppgfont.obj
 0002:00012810       ??_R3CFontPropPage@@8      5f5a0810     ppgfont.obj
 0002:00012820       ??_R4CFontPropPage@@6B@    5f5a0820     ppgfont.obj
 0002:00012838       ??_R1A@?0A@A@CComboBox@@8  5f5a0838     ppgfont.obj
 0002:00012850       ??_R1A@?0A@A@CSizeComboBox@@8 5f5a0850     ppgfont.obj
 0002:00012868       ??_R2CSizeComboBox@@8      5f5a0868     ppgfont.obj
 0002:00012880       ??_R3CSizeComboBox@@8      5f5a0880     ppgfont.obj
 0002:00012890       ??_R4CSizeComboBox@@6B@    5f5a0890     ppgfont.obj
 0002:000128a8       ??_R1A@?0A@A@CFontComboBox@@8 5f5a08a8     ppgfont.obj
 0002:000128c0       ??_R2CFontComboBox@@8      5f5a08c0     ppgfont.obj
 0002:000128d8       ??_R3CFontComboBox@@8      5f5a08d8     ppgfont.obj
 0002:000128e8       ??_R4CFontComboBox@@6B@    5f5a08e8     ppgfont.obj
 0002:00012900       ??_R1A@?0A@A@CFontPropPageFactory@CFontPropPage@@8 5f5a0900     ppgfont.obj
 0002:00012918       ??_R2CFontPropPageFactory@CFontPropPage@@8 5f5a0918     ppgfont.obj
 0002:00012930       ??_R3CFontPropPageFactory@CFontPropPage@@8 5f5a0930     ppgfont.obj
 0002:00012940       ??_R4CFontPropPageFactory@CFontPropPage@@6B@ 5f5a0940     ppgfont.obj
 0002:00012958       ??_R1A@?0A@A@CPicturePropPage@@8 5f5a0958     ppgpict.obj
 0002:00012970       ??_R2CPicturePropPage@@8   5f5a0970     ppgpict.obj
 0002:00012990       ??_R3CPicturePropPage@@8   5f5a0990     ppgpict.obj
 0002:000129a0       ??_R4CPicturePropPage@@6B@ 5f5a09a0     ppgpict.obj
 0002:000129b8       ??_R1A@?0A@A@CPicturePropPageFactory@CPicturePropPage@@8 5f5a09b8     ppgpict.obj
 0002:000129d0       ??_R2CPicturePropPageFactory@CPicturePropPage@@8 5f5a09d0     ppgpict.obj
 0002:000129e8       ??_R3CPicturePropPageFactory@CPicturePropPage@@8 5f5a09e8     ppgpict.obj
 0002:000129f8       ??_R4CPicturePropPageFactory@CPicturePropPage@@6B@ 5f5a09f8     ppgpict.obj
 0002:00012a10       ??_R2CStockPropPage@@8     5f5a0a10     ppgstock.obj
 0002:00012a30       ??_R3CStockPropPage@@8     5f5a0a30     ppgstock.obj
 0002:00012a40       ??_R4CStockPropPage@@6B@   5f5a0a40     ppgstock.obj
 0002:00012a54       ??_R2CPropExchange@@8      5f5a0a54     ctlinl.obj
 0002:00012a60       ??_R3CPropExchange@@8      5f5a0a60     ctlinl.obj
 0002:00012a70       ??_R4CPropExchange@@6B@    5f5a0a70     ctlinl.obj
 0002:00012a88       ??_R1A@?0A@A@CDataPathProperty@@8 5f5a0a88     ctlinl.obj
 0002:00012aa0       ??_R2CDataPathProperty@@8  5f5a0aa0     ctlinl.obj
 0002:00012ac0       ??_R3CDataPathProperty@@8  5f5a0ac0     ctlinl.obj
 0002:00012ad0       ??_R4CDataPathProperty@@6B@ 5f5a0ad0     ctlinl.obj
 0002:00012ae8       ??_R1A@?0A@A@CCachedDataPathProperty@@8 5f5a0ae8     ctlinl.obj
 0002:00012b00       ??_R2CCachedDataPathProperty@@8 5f5a0b00     ctlinl.obj
 0002:00012b20       ??_R3CCachedDataPathProperty@@8 5f5a0b20     ctlinl.obj
 0002:00012b30       ??_R4CCachedDataPathProperty@@6B@ 5f5a0b30     ctlinl.obj
 0002:00012b48       ??_R1A@?0A@A@type_info@@8  5f5a0b48     msvcrtd:ti_inst.obj
 0002:00012b60       ??_R2type_info@@8          5f5a0b60     msvcrtd:ti_inst.obj
 0002:00012b68       ??_R3type_info@@8          5f5a0b68     msvcrtd:ti_inst.obj
 0002:00012b78       ??_R4type_info@@6B@        5f5a0b78     msvcrtd:ti_inst.obj
 0002:00013cc0       __CT??_R0PAX@84            5f5a1cc0     oledisp1.obj
 0002:00013ce0       __CT??_R0PAVCObject@@@84   5f5a1ce0     oledisp1.obj
 0002:00013d00       __CT??_R0PAVCException@@@84 5f5a1d00     oledisp1.obj
 0002:00013d20       __CT??_R0PAVCOleDispatchException@@@84 5f5a1d20     oledisp1.obj
 0002:00013d40       __CTA4PAVCOleDispatchException@@ 5f5a1d40     oledisp1.obj
 0002:00013d58       __TI4PAVCOleDispatchException@@ 5f5a1d58     oledisp1.obj
 0002:000154c8       __CT??_R0PAVCOleException@@@84 5f5a34c8     olemisc.obj
 0002:000154e8       __CTA4PAVCOleException@@   5f5a34e8     olemisc.obj
 0002:00015500       __TI4PAVCOleException@@    5f5a3500     olemisc.obj
 0002:00016dc8       __CTA3PAVCException@@      5f5a4dc8     oleverb.obj
 0002:00016dd8       __TI3PAVCException@@       5f5a4dd8     oleverb.obj
 0002:0001c798       __DELAY_IMPORT_DESCRIPTOR_OLEPRO32 5f5aa798     olepro32:OLEPRO32.DLL
 0002:0001c7b8       __DELAY_IMPORT_DESCRIPTOR_ADVAPI32 5f5aa7b8     advapi32:ADVAPI32.dll
 0002:0001c7d8       __DELAY_IMPORT_DESCRIPTOR_ole32 5f5aa7d8     ole32:ole32.dll
 0002:0001c7f8       __DELAY_IMPORT_DESCRIPTOR_OLEAUT32 5f5aa7f8     oleaut32:OLEAUT32.dll
 0002:0001c818       __DELAY_IMPORT_DESCRIPTOR_oledlg 5f5aa818     oledlg:oledlg.dll
 0002:0001c838       __DELAY_IMPORT_DESCRIPTOR_urlmon 5f5aa838     urlmon:urlmon.dll
 0002:0001c858       __DELAY_IMPORT_DESCRIPTOR_SHELL32 5f5aa858     shell32:SHELL32.dll
 0002:0001c878       __NULL_DELAY_IMPORT_DESCRIPTOR 5f5aa878     olepro32:OLEPRO32.DLL
 0002:0001c8c0       \177ADVAPI32_NULL_THUNK_DATA_DLN 5f5aa8c0     advapi32:ADVAPI32.dll
 0002:0001c960       \177OLEAUT32_NULL_THUNK_DATA_DLN 5f5aa960     oleaut32:OLEAUT32.dll
 0002:0001c978       \177OLEPRO32_NULL_THUNK_DATA_DLN 5f5aa978     olepro32:OLEPRO32.DLL
 0002:0001c988       \177SHELL32_NULL_THUNK_DATA_DLN 5f5aa988     shell32:SHELL32.dll
 0002:0001cac0       \177ole32_NULL_THUNK_DATA_DLN 5f5aaac0     ole32:ole32.dll
 0002:0001caec       \177oledlg_NULL_THUNK_DATA_DLN 5f5aaaec     oledlg:oledlg.dll
 0002:0001cb00       \177urlmon_NULL_THUNK_DATA_DLN 5f5aab00     urlmon:urlmon.dll
 0002:0001d254       \177OLEPRO32_NULL_THUNK_DATA_DLB 5f5ab254     olepro32:OLEPRO32.DLL
 0002:0001d26c       \177ADVAPI32_NULL_THUNK_DATA_DLB 5f5ab26c     advapi32:ADVAPI32.dll
 0002:0001d298       \177ole32_NULL_THUNK_DATA_DLB 5f5ab298     ole32:ole32.dll
 0002:0001d3d0       \177OLEAUT32_NULL_THUNK_DATA_DLB 5f5ab3d0     oleaut32:OLEAUT32.dll
 0002:0001d470       \177oledlg_NULL_THUNK_DATA_DLB 5f5ab470     oledlg:oledlg.dll
 0002:0001d49c       \177urlmon_NULL_THUNK_DATA_DLB 5f5ab49c     urlmon:urlmon.dll
 0002:0001d4b0       \177SHELL32_NULL_THUNK_DATA_DLB 5f5ab4b0     shell32:SHELL32.dll
 0002:0001d4bc       __IMPORT_DESCRIPTOR_MFC42D 5f5ab4bc     MFC42D:MFC42D.DLL
 0002:0001d4d0       __IMPORT_DESCRIPTOR_MSVCRTD 5f5ab4d0     msvcrtd:MSVCRTD.dll
 0002:0001d4e4       __IMPORT_DESCRIPTOR_KERNEL32 5f5ab4e4     kernel32:KERNEL32.dll
 0002:0001d4f8       __IMPORT_DESCRIPTOR_GDI32  5f5ab4f8     gdi32:GDI32.dll
 0002:0001d50c       __IMPORT_DESCRIPTOR_USER32 5f5ab50c     user32:USER32.dll
 0002:0001d520       __NULL_IMPORT_DESCRIPTOR   5f5ab520     MFC42D:MFC42D.DLL
 0003:00000000       ___xc_a                    5f5b1000     msvcrtd:cinitexe.obj
 0003:00000038       ___xc_z                    5f5b1038     msvcrtd:cinitexe.obj
 0003:0000003c       ___xi_a                    5f5b103c     msvcrtd:cinitexe.obj
 0003:00000040       ___xi_z                    5f5b1040     msvcrtd:cinitexe.obj
 0003:0000005c       __pRawDllMain              5f5b105c     dllole.obj
 0003:00000060       ?_afxForceVectorDelete_mfco@@3P6AXXZA 5f5b1060     dllole.obj
 0003:00000068       ?GUID_ATLVer30@ATL@@3U_GUID@@A 5f5b1068     dllole.obj
 0003:00000078       ?_afxTickCount@@3KA        5f5b1078     oleinit.obj
 0003:000000a0       ??_R0?AVCObject@@@8        5f5b10a0     olecli1.obj
 0003:000000b8       ??_R0?AVCCmdTarget@@@8     5f5b10b8     olecli1.obj
 0003:000000d8       ??_R0?AVCDocItem@@@8       5f5b10d8     olecli1.obj
 0003:000000f0       ??_R0?AVCOleClientItem@@@8 5f5b10f0     olecli1.obj
 0003:00000110       ??_R0?AUIUnknown@@@8       5f5b1110     olecli1.obj
 0003:00000128       ??_R0?AUIOleClientSite@@@8 5f5b1128     olecli1.obj
 0003:00000148       ??_R0?AVXOleClientSite@COleClientItem@@@8 5f5b1148     olecli1.obj
 0003:00000178       ??_R0?AUIAdviseSink@@@8    5f5b1178     olecli1.obj
 0003:00000198       ??_R0?AVXAdviseSink@COleClientItem@@@8 5f5b1198     olecli1.obj
 0003:000001c8       ??_R0?AUIOleWindow@@@8     5f5b11c8     olecli1.obj
 0003:000001e8       ??_R0?AUIOleInPlaceSite@@@8 5f5b11e8     olecli1.obj
 0003:00000208       ??_R0?AVXOleIPSite@COleClientItem@@@8 5f5b1208     olecli1.obj
 0003:00000230       ??_R0PAVCException@@@8     5f5b1230     olecli1.obj
 0003:00000258       ??_R0?AVCOleFrameHook@@@8  5f5b1258     olecli2.obj
 0003:00000278       ??_R0?AUIOleInPlaceUIWindow@@@8 5f5b1278     olecli2.obj
 0003:000002a0       ??_R0?AUIOleInPlaceFrame@@@8 5f5b12a0     olecli2.obj
 0003:000002c0       ??_R0?AVXOleInPlaceFrame@COleFrameHook@@@8 5f5b12c0     olecli2.obj
 0003:000002f0       ??_R0?AUIOleCommandTarget@@@8 5f5b12f0     olecli2.obj
 0003:00000310       ??_R0?AVXOleCommandTarget@COleFrameHook@@@8 5f5b1310     olecli2.obj
 0003:00000380       ??_R0?AVCOleDataSource@@@8 5f5b1380     oledobj2.obj
 0003:000003a0       ??_R0?AUIDataObject@@@8    5f5b13a0     oledobj2.obj
 0003:000003c0       ??_R0?AVXDataObject@COleDataSource@@@8 5f5b13c0     oledobj2.obj
 0003:000003f0       ??_R0?AVCEnumArray@@@8     5f5b13f0     oledobj2.obj
 0003:00000410       ??_R0?AVCEnumFormatEtc@@@8 5f5b1410     oledobj2.obj
 0003:00000440       ??_R0?AUIDispatch@@@8      5f5b1440     oledisp1.obj
 0003:00000458       ??_R0?AVCOleDispatchImpl@@@8 5f5b1458     oledisp1.obj
 0003:00000478       ??_R0PAVCOleException@@@8  5f5b1478     oledisp1.obj
 0003:00000498       ??_R0?AVCException@@@8     5f5b1498     oledisp1.obj
 0003:000004b8       ??_R0?AVCOleDispatchException@@@8 5f5b14b8     oledisp1.obj
 0003:000004e0       ??_R0PAX@8                 5f5b14e0     oledisp1.obj
 0003:000004f0       ??_R0PAVCObject@@@8        5f5b14f0     oledisp1.obj
 0003:00000508       ??_R0PAVCOleDispatchException@@@8 5f5b1508     oledisp1.obj
 0003:00000558       ??_R0?AUIOleUILinkContainerA@@@8 5f5b1558     oledlgs1.obj
 0003:00000580       ??_R0?AUIOleUILinkInfoA@@@8 5f5b1580     oledlgs1.obj
 0003:000005a0       ??_R0?AVCOleUILinkInfo@@@8 5f5b15a0     oledlgs1.obj
 0003:000005c0       ??_R0?AVCWnd@@@8           5f5b15c0     oledlgs1.obj
 0003:000005d8       ??_R0?AVCDialog@@@8        5f5b15d8     oledlgs1.obj
 0003:000005f0       ??_R0?AVCCommonDialog@@@8  5f5b15f0     oledlgs1.obj
 0003:00000610       ??_R0?AVCOleDialog@@@8     5f5b1610     oledlgs1.obj
 0003:00000630       ??_R0?AVCOleInsertDialog@@@8 5f5b1630     oledlgs1.obj
 0003:00000650       ??_R0?AVCOleConvertDialog@@@8 5f5b1650     oledlgs1.obj
 0003:00000670       ??_R0?AVCOleChangeIconDialog@@@8 5f5b1670     oledlgs1.obj
 0003:00000698       ??_R0?AVCOleLinksDialog@@@8 5f5b1698     oledlgs1.obj
 0003:000006b8       ??_R0?AVCOleUpdateDialog@@@8 5f5b16b8     oledlgs1.obj
 0003:000006d8       ??_R0?AVCOlePasteSpecialDialog@@@8 5f5b16d8     oledlgs1.obj
 0003:00000710       ??_R0?AVCOleBusyDialog@@@8 5f5b1710     oledlgs2.obj
 0003:00000740       ??_R0?AVCOlePropertiesDialog@@@8 5f5b1740     oledlgs3.obj
 0003:00000768       ??_R0?AUIOleUIObjInfoA@@@8 5f5b1768     oledlgs3.obj
 0003:00000788       ??_R0?AVXOleUIObjInfo@COlePropertiesDialog@@@8 5f5b1788     oledlgs3.obj
 0003:000007c0       ??_R0?AVCOleChangeSourceDialog@@@8 5f5b17c0     oledlgs3.obj
 0003:000007e8       ??_R0?AVCNoTrackObject@@@8 5f5b17e8     oledata.obj
 0003:00000808       ??_R0?AV_AFX_OLE_STATE@@@8 5f5b1808     oledata.obj
 0003:00000828       ?_afxMonthDays@@3PAHA      5f5b1828     olevar.obj
 0003:00000880       ?classCDocItem@CDocItem@@2UCRuntimeClass@@A 5f5b1880     oledoc1.obj
 0003:000008b0       ??_R0?AVCDocument@@@8      5f5b18b0     oledoc1.obj
 0003:000008c8       ??_R0?AVCOleDocument@@@8   5f5b18c8     oledoc1.obj
 0003:00000900       ??_R0?AVCOleDropSource@@@8 5f5b1900     oledrop1.obj
 0003:00000920       ??_R0?AUIDropSource@@@8    5f5b1920     oledrop1.obj
 0003:00000940       ??_R0?AVXDropSource@COleDropSource@@@8 5f5b1940     oledrop1.obj
 0003:00000980       ??_R0?AVCOleDropTarget@@@8 5f5b1980     oledrop2.obj
 0003:000009a0       ??_R0?AUIDropTarget@@@8    5f5b19a0     oledrop2.obj
 0003:000009c0       ??_R0?AVXDropTarget@COleDropTarget@@@8 5f5b19c0     oledrop2.obj
 0003:000009f8       ??_R0?AVCOleMessageFilter@@@8 5f5b19f8     olemsgf.obj
 0003:00000a18       ??_R0?AUIMessageFilter@@@8 5f5b1a18     olemsgf.obj
 0003:00000a38       ??_R0?AVXMessageFilter@COleMessageFilter@@@8 5f5b1a38     olemsgf.obj
 0003:00000a78       ??_R0?AUIEnumVOID@@@8      5f5b1a78     oleenum.obj
 0003:00000a90       ??_R0?AVXEnumVOID@CEnumArray@@@8 5f5b1a90     oleenum.obj
 0003:00000ac0       ??_R0?AVCOleObjectFactory@@@8 5f5b1ac0     olefact.obj
 0003:00000ae0       ??_R0?AUIClassFactory@@@8  5f5b1ae0     olefact.obj
 0003:00000b00       ??_R0?AUIClassFactory2@@@8 5f5b1b00     olefact.obj
 0003:00000b20       ??_R0?AVXClassFactory@COleObjectFactory@@@8 5f5b1b20     olefact.obj
 0003:00000b60       ??_R0?AVCFrameWnd@@@8      5f5b1b60     oleipfrm.obj
 0003:00000b78       ??_R0?AVCOleCntrFrameWnd@@@8 5f5b1b78     oleipfrm.obj
 0003:00000b98       ??_R0?AVCOleIPFrameWnd@@@8 5f5b1b98     oleipfrm.obj
 0003:00000bc8       ??_R0?AVCOleLinkingDoc@@@8 5f5b1bc8     olelink.obj
 0003:00000be8       ??_R0?AUIPersist@@@8       5f5b1be8     olelink.obj
 0003:00000c00       ??_R0?AUIPersistFile@@@8   5f5b1c00     olelink.obj
 0003:00000c20       ??_R0?AVXPersistFile@COleLinkingDoc@@@8 5f5b1c20     olelink.obj
 0003:00000c50       ??_R0?AUIParseDisplayName@@@8 5f5b1c50     olelink.obj
 0003:00000c70       ??_R0?AUIOleContainer@@@8  5f5b1c70     olelink.obj
 0003:00000c90       ??_R0?AUIOleItemContainer@@@8 5f5b1c90     olelink.obj
 0003:00000cb0       ??_R0?AVXOleItemContainer@COleLinkingDoc@@@8 5f5b1cb0     olelink.obj
 0003:00000d28       ??_R0?AVCFile@@@8          5f5b1d28     olestrm.obj
 0003:00000d40       ??_R0?AVCOleStreamFile@@@8 5f5b1d40     olestrm.obj
 0003:00000d78       ??_R0?AVCOleServerDoc@@@8  5f5b1d78     olesvr1.obj
 0003:00000d98       ??_R0?AUIPersistStorage@@@8 5f5b1d98     olesvr1.obj
 0003:00000db8       ??_R0?AVXPersistStorage@COleServerDoc@@@8 5f5b1db8     olesvr1.obj
 0003:00000de8       ??_R0?AUIOleObject@@@8     5f5b1de8     olesvr1.obj
 0003:00000e08       ??_R0?AVXOleObject@COleServerDoc@@@8 5f5b1e08     olesvr1.obj
 0003:00000e30       ??_R0?AVXDataObject@COleServerDoc@@@8 5f5b1e30     olesvr1.obj
 0003:00000e58       ??_R0?AUIOleInPlaceObject@@@8 5f5b1e58     olesvr1.obj
 0003:00000e78       ??_R0?AVXOleInPlaceObject@COleServerDoc@@@8 5f5b1e78     olesvr1.obj
 0003:00000ea8       ??_R0?AUIOleInPlaceActiveObject@@@8 5f5b1ea8     olesvr1.obj
 0003:00000ed0       ??_R0?AVXOleInPlaceActiveObject@COleServerDoc@@@8 5f5b1ed0     olesvr1.obj
 0003:00000f10       ??_R0?AVCOleServerItem@@@8 5f5b1f10     olesvr2.obj
 0003:00000f30       ??_R0?AVCItemDataSource@COleServerItem@@@8 5f5b1f30     olesvr2.obj
 0003:00000f60       ??_R0?AVXOleObject@COleServerItem@@@8 5f5b1f60     olesvr2.obj
 0003:00000f88       ??_R0?AVXDataObject@COleServerItem@@@8 5f5b1f88     olesvr2.obj
 0003:00000fd0       ??_R0?AVCOleTemplateServer@@@8 5f5b1fd0     oletsvr.obj
 0003:00001028       ??_R0?AVCInnerUnknown@@@8  5f5b2028     oleunk.obj
 0003:00001048       ??_R0?AVCOleException@@@8  5f5b2048     oleunk.obj
 0003:00001070       ??_R0?AVCEnumOleVerb@@@8   5f5b2070     oleverb.obj
 0003:00001090       ?classCRichEditCntrItem@CRichEditCntrItem@@2UCRuntimeClass@@A 5f5b2090     viewrich.obj
 0003:000010b8       ?lMaxSize@CRichEditView@@2KA 5f5b20b8     viewrich.obj
 0003:000010c0       ??_R0?AVCView@@@8          5f5b20c0     viewrich.obj
 0003:000010d8       ??_R0?AVCCtrlView@@@8      5f5b20d8     viewrich.obj
 0003:000010f0       ??_R0?AVCRichEditView@@@8  5f5b20f0     viewrich.obj
 0003:00001110       ??_R0?AUIRichEditOleCallback@@@8 5f5b2110     viewrich.obj
 0003:00001138       ??_R0?AVXRichEditOleCallback@CRichEditView@@@8 5f5b2138     viewrich.obj
 0003:00001170       ??_R0PAVCFileException@@@8 5f5b2170     viewrich.obj
 0003:00001190       ??_R0?AVCRichEditDoc@@@8   5f5b2190     viewrich.obj
 0003:000011b0       ??_R0?AVCRichEditCntrItem@@@8 5f5b21b0     viewrich.obj
 0003:000011d0       ??_R0?AV_AFX_EDIT_STATE@@@8 5f5b21d0     viewrich.obj
 0003:000011f0       ??_R0?AV_AFX_RICHEDIT_STATE@@@8 5f5b21f0     viewrich.obj
 0003:00001230       ??_R0?AVCMapPtrToPtr@@@8   5f5b2230     oletyplb.obj
 0003:00001250       ??_R0?AVCTypeLibCacheMap@@@8 5f5b2250     oletyplb.obj
 0003:00001288       ??_R0?AVCMonikerFile@@@8   5f5b2288     olemon.obj
 0003:000012a8       ??_R0?AUIBindHost@@@8      5f5b22a8     olemon.obj
 0003:000012c0       ??_R0?AV_AfxBindHost@@@8   5f5b22c0     olemon.obj
 0003:000012f0       ??_R0?AVCDateTimeCtrl@@@8  5f5b22f0     winctrl5.obj
 0003:00001310       ??_R0?AVCMonthCalCtrl@@@8  5f5b2310     winctrl5.obj
 0003:0000133c       ?_eventsinkEntryCount@CHtmlView@@0IA 5f5b233c     viewhtml.obj
 0003:00001350       ??_R0?AVCScrollView@@@8    5f5b2350     viewhtml.obj
 0003:00001370       ??_R0?AVCFormView@@@8      5f5b2370     viewhtml.obj
 0003:00001388       ??_R0?AVCHtmlView@@@8      5f5b2388     viewhtml.obj
 0003:000013b0       ??_R0?AVCOccManager@@@8    5f5b23b0     occmgr.obj
 0003:000013dc       ?_dwStockPropMask@COleControlContainer@@0KA 5f5b23dc     occcont.obj
 0003:000013e0       ?_dispatchEntryCount@COleControlContainer@@0IA 5f5b23e0     occcont.obj
 0003:000013f0       ??_R0?AVCOleControlContainer@@@8 5f5b23f0     occcont.obj
 0003:00001418       ??_R0?AVXOleIPFrame@COleControlContainer@@@8 5f5b2418     occcont.obj
 0003:00001448       ??_R0?AVXOleContainer@COleControlContainer@@@8 5f5b2448     occcont.obj
 0003:00001480       ??_R0?AVCEnumUnknown@@@8   5f5b2480     occcont.obj
 0003:000014a8       ??_R0?AVCOleControlSite@@@8 5f5b24a8     occsite.obj
 0003:000014c8       ??_R0?AVXOleClientSite@COleControlSite@@@8 5f5b24c8     occsite.obj
 0003:000014f8       ??_R0?AVXOleIPSite@COleControlSite@@@8 5f5b24f8     occsite.obj
 0003:00001528       ??_R0?AUIOleControlSite@@@8 5f5b2528     occsite.obj
 0003:00001548       ??_R0?AVXOleControlSite@COleControlSite@@@8 5f5b2548     occsite.obj
 0003:00001578       ??_R0?AVXAmbientProps@COleControlSite@@@8 5f5b2578     occsite.obj
 0003:000015a8       ??_R0?AUIPropertyNotifySink@@@8 5f5b25a8     occsite.obj
 0003:000015d0       ??_R0?AVXPropertyNotifySink@COleControlSite@@@8 5f5b25d0     occsite.obj
 0003:00001608       ??_R0?AVXEventSink@COleControlSite@@@8 5f5b2608     occsite.obj
 0003:00001638       ??_R0?AUIBoundObjectSite@@@8 5f5b2638     occsite.obj
 0003:00001658       ??_R0?AVXBoundObjectSite@COleControlSite@@@8 5f5b2658     occsite.obj
 0003:00001688       ??_R0?AUINotifyDBEvents@@@8 5f5b2688     occsite.obj
 0003:000016a8       ??_R0?AVXNotifyDBEvents@COleControlSite@@@8 5f5b26a8     occsite.obj
 0003:000016d8       ??_R0?AUIRowsetNotify@@@8  5f5b26d8     occsite.obj
 0003:000016f8       ??_R0?AVXRowsetNotify@COleControlSite@@@8 5f5b26f8     occsite.obj
 0003:00001728       ??_R0?AVCDataSourceControl@@@8 5f5b2728     occsite.obj
 0003:00001750       __GUID_0c733a05_2a1c_11ce_ade5_00aa0044773d 5f5b2750     occsite.obj
 0003:00001760       __GUID_0c733a11_2a1c_11ce_ade5_00aa0044773d 5f5b2760     occsite.obj
 0003:00001770       __GUID_0c733a8c_2a1c_11ce_ade5_00aa0044773d 5f5b2770     occsite.obj
 0003:00001790       ??_R0?AVCOleControlLock@@@8 5f5b2790     occlock.obj
 0003:000017f8       ??_R0?AVCDocObjectServer@@@8 5f5b27f8     oledocob.obj
 0003:00001818       ??_R0?AVXOleObject@CDocObjectServer@@@8 5f5b2818     oledocob.obj
 0003:00001848       ??_R0?AUIOleDocument@@@8   5f5b2848     oledocob.obj
 0003:00001868       ??_R0?AVXOleDocument@CDocObjectServer@@@8 5f5b2868     oledocob.obj
 0003:00001898       ??_R0?AUIOleDocumentView@@@8 5f5b2898     oledocob.obj
 0003:000018b8       ??_R0?AVXOleDocumentView@CDocObjectServer@@@8 5f5b28b8     oledocob.obj
 0003:000018e8       ??_R0?AVXOleCommandTarget@CDocObjectServer@@@8 5f5b28e8     oledocob.obj
 0003:00001920       ??_R0?AUIPrint@@@8         5f5b2920     oledocob.obj
 0003:00001938       ??_R0?AVXPrint@CDocObjectServer@@@8 5f5b2938     oledocob.obj
 0003:00001960       ??_R0?AVCDocObjectServerItem@@@8 5f5b2960     oledocob.obj
 0003:00001998       ??_R0?AVCCmdUI@@@8         5f5b2998     oledoctg.obj
 0003:000019b0       ??_R0?AVCOleCmdUI@@@8      5f5b29b0     oledoctg.obj
 0003:000019d8       ??_R0?AVCOleDocIPFrameWnd@@@8 5f5b29d8     oledocip.obj
 0003:00001a08       ??_R0?AVCOleDocObjectItem@@@8 5f5b2a08     oledoccl.obj
 0003:00001a28       ??_R0?AUIOleDocumentSite@@@8 5f5b2a28     oledoccl.obj
 0003:00001a48       ??_R0?AVXOleDocumentSite@COleDocObjectItem@@@8 5f5b2a48     oledoccl.obj
 0003:00001a90       ??_R0?AVCAsyncMonikerFile@@@8 5f5b2a90     oleasmon.obj
 0003:00001ab0       ??_R0?AUIBindStatusCallback@@@8 5f5b2ab0     oleasmon.obj
 0003:00001ad8       ??_R0?AV_AfxBindStatusCallback@@@8 5f5b2ad8     oleasmon.obj
 0003:00001b00       ??_R0?AVCInnerUnknown@_AfxBindStatusCallback@@@8 5f5b2b00     oleasmon.obj
 0003:00001b40       ??_R0?AVCControlBar@@@8    5f5b2b40     olebar.obj
 0003:00001b60       ??_R0?AVCOleResizeBar@@@8  5f5b2b60     olebar.obj
 0003:00001b98       ??_R0?AVCOleControl@@@8    5f5b2b98     ctlcore.obj
 0003:00001bb8       ??_R0?AVXPersistStorage@COleControl@@@8 5f5b2bb8     ctlcore.obj
 0003:00001be8       ??_R0?AUIPersistStreamInit@@@8 5f5b2be8     ctlcore.obj
 0003:00001c10       ??_R0?AVXPersistStreamInit@COleControl@@@8 5f5b2c10     ctlcore.obj
 0003:00001c40       ??_R0?AUIPersistMemory@@@8 5f5b2c40     ctlcore.obj
 0003:00001c60       ??_R0?AVXPersistMemory@COleControl@@@8 5f5b2c60     ctlcore.obj
 0003:00001c90       ??_R0?AUIPersistPropertyBag@@@8 5f5b2c90     ctlcore.obj
 0003:00001cb8       ??_R0?AVXPersistPropertyBag@COleControl@@@8 5f5b2cb8     ctlcore.obj
 0003:00001ce8       ??_R0?AVXOleObject@COleControl@@@8 5f5b2ce8     ctlcore.obj
 0003:00001d10       ??_R0?AUIViewObject@@@8    5f5b2d10     ctlcore.obj
 0003:00001d30       ??_R0?AUIViewObject2@@@8   5f5b2d30     ctlcore.obj
 0003:00001d50       ??_R0?AUIViewObjectEx@@@8  5f5b2d50     ctlcore.obj
 0003:00001d70       ??_R0?AVXViewObject@COleControl@@@8 5f5b2d70     ctlcore.obj
 0003:00001d98       ??_R0?AVXDataObject@COleControl@@@8 5f5b2d98     ctlcore.obj
 0003:00001dc0       ??_R0?AUIOleInPlaceObjectWindowless@@@8 5f5b2dc0     ctlcore.obj
 0003:00001df0       ??_R0?AVXOleInPlaceObject@COleControl@@@8 5f5b2df0     ctlcore.obj
 0003:00001e20       ??_R0?AVXOleInPlaceActiveObject@COleControl@@@8 5f5b2e20     ctlcore.obj
 0003:00001e58       ??_R0?AUIOleCache@@@8      5f5b2e58     ctlcore.obj
 0003:00001e70       ??_R0?AVXOleCache@COleControl@@@8 5f5b2e70     ctlcore.obj
 0003:00001e98       ??_R0?AUIOleControl@@@8    5f5b2e98     ctlcore.obj
 0003:00001eb8       ??_R0?AVXOleControl@COleControl@@@8 5f5b2eb8     ctlcore.obj
 0003:00001ee0       ??_R0?AUIProvideClassInfo@@@8 5f5b2ee0     ctlcore.obj
 0003:00001f00       ??_R0?AUIProvideClassInfo2@@@8 5f5b2f00     ctlcore.obj
 0003:00001f28       ??_R0?AVXProvideClassInfo@COleControl@@@8 5f5b2f28     ctlcore.obj
 0003:00001f58       ??_R0?AUISpecifyPropertyPages@@@8 5f5b2f58     ctlcore.obj
 0003:00001f80       ??_R0?AVXSpecifyPropertyPages@COleControl@@@8 5f5b2f80     ctlcore.obj
 0003:00001fb0       ??_R0?AUIPerPropertyBrowsing@@@8 5f5b2fb0     ctlcore.obj
 0003:00001fd8       ??_R0?AVXPerPropertyBrowsing@COleControl@@@8 5f5b2fd8     ctlcore.obj
 0003:00002008       ??_R0?AVXFontNotification@COleControl@@@8 5f5b3008     ctlcore.obj
 0003:00002038       ??_R0?AUIQuickActivate@@@8 5f5b3038     ctlcore.obj
 0003:00002058       ??_R0?AVXQuickActivate@COleControl@@@8 5f5b3058     ctlcore.obj
 0003:00002088       ??_R0?AUIPointerInactive@@@8 5f5b3088     ctlcore.obj
 0003:000020a8       ??_R0?AVXPointerInactive@COleControl@@@8 5f5b30a8     ctlcore.obj
 0003:000020d8       ??_R0?AVCConnectionPoint@@@8 5f5b30d8     ctlcore.obj
 0003:000020f8       ??_R0?AVXEventConnPt@COleControl@@@8 5f5b30f8     ctlcore.obj
 0003:00002120       ??_R0?AVXPropConnPt@COleControl@@@8 5f5b3120     ctlcore.obj
 0003:00002148       ??_R0?AVCReflectorWnd@@@8  5f5b3148     ctlcore.obj
 0003:00002168       ??_R0?AVCParkingWnd@@@8    5f5b3168     ctlcore.obj
 0003:000021a0       ??_R0?AVCControlDataSource@COleControl@@@8 5f5b31a0     ctldata.obj
 0003:00002200       ??_R0?AVCControlFrameWnd@@@8 5f5b3200     ctlframe.obj
 0003:00002258       ??_R0?AUIConnectionPoint@@@8 5f5b3258     oleconn.obj
 0003:00002278       ??_R0?AVXConnPt@CConnectionPoint@@@8 5f5b3278     oleconn.obj
 0003:000022a0       ??_R0?AVCEnumConnections@@@8 5f5b32a0     oleconn.obj
 0003:000022c0       ??_R0?AVCEnumConnPoints@@@8 5f5b32c0     oleconn.obj
 0003:000022e0       ??_R0?AUIConnectionPointContainer@@@8 5f5b32e0     oleconn.obj
 0003:00002308       ??_R0?AVCOleConnPtContainer@@@8 5f5b3308     oleconn.obj
 0003:00002358       ??_R0?AVCPropExchange@@@8  5f5b3358     ctlpropx.obj
 0003:00002378       ??_R0?AVCArchivePropExchange@@@8 5f5b3378     ctlpropx.obj
 0003:000023a0       ??_R0?AVCResetPropExchange@@@8 5f5b33a0     ctlpropx.obj
 0003:000023c8       ??_R0?AVCAsyncPropExchange@@@8 5f5b33c8     ctlpropx.obj
 0003:000023f8       ??_R0?AUAFX_DDPDATA@@@8    5f5b33f8     ctlppg.obj
 0003:00002418       ??_R0?AVCOlePropertyPage@@@8 5f5b3418     ctlppg.obj
 0003:00002438       ??_R0?AUIPropertyPage@@@8  5f5b3438     ctlppg.obj
 0003:00002458       ??_R0?AUIPropertyPage2@@@8 5f5b3458     ctlppg.obj
 0003:00002478       ??_R0?AVXPropertyPage@COlePropertyPage@@@8 5f5b3478     ctlppg.obj
 0003:000024a8       ??_R0?AVXPropNotifySink@COlePropertyPage@@@8 5f5b34a8     ctlppg.obj
 0003:000024f0       ??_R0?AVCPropsetPropExchange@@@8 5f5b34f0     ctlpset.obj
 0003:00002570       ??_R0?AVCRectTracker@@@8   5f5b3570     ctltrack.obj
 0003:00002590       ??_R0?AVCControlRectTracker@@@8 5f5b3590     ctltrack.obj
 0003:000025d8       ??_R0?AUIPersistStream@@@8 5f5b35d8     ctlpbag.obj
 0003:000025f8       ??_R0?AVCBlobProperty@@@8  5f5b35f8     ctlpbag.obj
 0003:00002618       ??_R0?AVCPropbagPropExchange@@@8 5f5b3618     ctlpbag.obj
 0003:00002650       ??_R0?AV_AFXCTL_AMBIENT_CACHE@@@8 5f5b3650     ctlquick.obj
 0003:00002688       ??_R0?AVCDC@@@8            5f5b3688     ctlnownd.obj
 0003:000026a0       ??_R0?AVCWindowlessDC@@@8  5f5b36a0     ctlnownd.obj
 0003:000026d0       ??_R0?AVCButton@@@8        5f5b36d0     ppgcolor.obj
 0003:000026e8       ??_R0?AVCColorButton@@@8   5f5b36e8     ppgcolor.obj
 0003:00002708       ??_R0?AVCStockPropPage@@@8 5f5b3708     ppgcolor.obj
 0003:00002728       ??_R0?AVCColorPropPage@@@8 5f5b3728     ppgcolor.obj
 0003:00002748       ??_R0?AVCColorPropPageFactory@CColorPropPage@@@8 5f5b3748     ppgcolor.obj
 0003:0000277c       ?_afxTTDefaults@@3PAHA     5f5b377c     ppgfont.obj
 0003:000027c8       ??_R0?AVCFontPropPage@@@8  5f5b37c8     ppgfont.obj
 0003:000027e8       ??_R0?AVCComboBox@@@8      5f5b37e8     ppgfont.obj
 0003:00002800       ??_R0?AVCSizeComboBox@@@8  5f5b3800     ppgfont.obj
 0003:00002820       ??_R0?AVCFontComboBox@@@8  5f5b3820     ppgfont.obj
 0003:00002840       ??_R0PAVCMemoryException@@@8 5f5b3840     ppgfont.obj
 0003:00002860       ??_R0?AVCFontPropPageFactory@CFontPropPage@@@8 5f5b3860     ppgfont.obj
 0003:00002898       ?_afxPictDescEmpty@@3UtagPICTDESC@@A 5f5b3898     ppgpict.obj
 0003:000028b8       ??_R0?AVCPicturePropPage@@@8 5f5b38b8     ppgpict.obj
 0003:000028d8       ??_R0?AVCPicturePropPageFactory@CPicturePropPage@@@8 5f5b38d8     ppgpict.obj
 0003:00002930       ??_R0?AVCDataPathProperty@@@8 5f5b3930     ctlinl.obj
 0003:00002950       ??_R0?AVCCachedDataPathProperty@@@8 5f5b3950     ctlinl.obj
 0003:00002980       ??_R0?AVtype_info@@@8      5f5b3980     msvcrtd:ti_inst.obj
 0003:000029a0       __imp__RegOpenKeyA@12      5f5b39a0     advapi32:ADVAPI32.dll
 0003:000029a4       __imp__RegDeleteKeyA@8     5f5b39a4     advapi32:ADVAPI32.dll
 0003:000029a8       __imp__RegCreateKeyA@12    5f5b39a8     advapi32:ADVAPI32.dll
 0003:000029ac       __imp__RegSetValueExA@24   5f5b39ac     advapi32:ADVAPI32.dll
 0003:000029b0       __imp__RegQueryValueA@16   5f5b39b0     advapi32:ADVAPI32.dll
 0003:000029b4       __imp__RegSetValueA@20     5f5b39b4     advapi32:ADVAPI32.dll
 0003:000029b8       __imp__RegCloseKey@4       5f5b39b8     advapi32:ADVAPI32.dll
 0003:000029bc       __imp__RegQueryValueExA@24 5f5b39bc     advapi32:ADVAPI32.dll
 0003:000029c0       __imp__RegOpenKeyExA@20    5f5b39c0     advapi32:ADVAPI32.dll
 0003:000029c4       __imp__RegEnumKeyA@16      5f5b39c4     advapi32:ADVAPI32.dll
 0003:000029c8       \177ADVAPI32_NULL_THUNK_DATA_DLA 5f5b39c8     advapi32:ADVAPI32.dll
 0003:000029cc       __imp__SafeArrayPutElement@12 5f5b39cc     oleaut32:OLEAUT32.dll
 0003:000029d0       __imp__VarBstrFromDate@20  5f5b39d0     oleaut32:OLEAUT32.dll
 0003:000029d4       __imp__VarDateFromStr@16   5f5b39d4     oleaut32:OLEAUT32.dll
 0003:000029d8       __imp__SysAllocStringByteLen@8 5f5b39d8     oleaut32:OLEAUT32.dll
 0003:000029dc       __imp__SysStringLen@4      5f5b39dc     oleaut32:OLEAUT32.dll
 0003:000029e0       __imp__LoadRegTypeLib@20   5f5b39e0     oleaut32:OLEAUT32.dll
 0003:000029e4       __imp__RegisterTypeLib@12  5f5b39e4     oleaut32:OLEAUT32.dll
 0003:000029e8       __imp__VariantTimeToSystemTime@12 5f5b39e8     oleaut32:OLEAUT32.dll
 0003:000029ec       __imp__LoadTypeLib@8       5f5b39ec     oleaut32:OLEAUT32.dll
 0003:000029f0       __imp__DosDateTimeToVariantTime@12 5f5b39f0     oleaut32:OLEAUT32.dll
 0003:000029f4       __imp__SafeArrayCreateVector@12 5f5b39f4     oleaut32:OLEAUT32.dll
 0003:000029f8       __imp__SafeArrayDestroyDescriptor@4 5f5b39f8     oleaut32:OLEAUT32.dll
 0003:000029fc       __imp__SafeArrayDestroyData@4 5f5b39fc     oleaut32:OLEAUT32.dll
 0003:00002a00       __imp__SafeArrayDestroy@4  5f5b3a00     oleaut32:OLEAUT32.dll
 0003:00002a04       __imp__SafeArrayUnlock@4   5f5b3a04     oleaut32:OLEAUT32.dll
 0003:00002a08       __imp__SafeArrayLock@4     5f5b3a08     oleaut32:OLEAUT32.dll
 0003:00002a0c       __imp__SafeArrayGetDim@4   5f5b3a0c     oleaut32:OLEAUT32.dll
 0003:00002a10       __imp__SafeArrayPtrOfIndex@12 5f5b3a10     oleaut32:OLEAUT32.dll
 0003:00002a14       __imp__SafeArrayGetElement@12 5f5b3a14     oleaut32:OLEAUT32.dll
 0003:00002a18       __imp__SafeArrayAllocDescriptor@8 5f5b3a18     oleaut32:OLEAUT32.dll
 0003:00002a1c       __imp__SafeArrayAllocData@4 5f5b3a1c     oleaut32:OLEAUT32.dll
 0003:00002a20       __imp__SafeArrayCopy@8     5f5b3a20     oleaut32:OLEAUT32.dll
 0003:00002a24       __imp__SafeArrayGetUBound@12 5f5b3a24     oleaut32:OLEAUT32.dll
 0003:00002a28       __imp__SafeArrayGetLBound@12 5f5b3a28     oleaut32:OLEAUT32.dll
 0003:00002a2c       __imp__VarBstrFromCy@20    5f5b3a2c     oleaut32:OLEAUT32.dll
 0003:00002a30       __imp__VarCyFromStr@16     5f5b3a30     oleaut32:OLEAUT32.dll
 0003:00002a34       __imp__SysStringByteLen@4  5f5b3a34     oleaut32:OLEAUT32.dll
 0003:00002a38       __imp__SafeArrayCreate@12  5f5b3a38     oleaut32:OLEAUT32.dll
 0003:00002a3c       __imp__SafeArrayRedim@8    5f5b3a3c     oleaut32:OLEAUT32.dll
 0003:00002a40       __imp__SafeArrayUnaccessData@4 5f5b3a40     oleaut32:OLEAUT32.dll
 0003:00002a44       __imp__SafeArrayGetElemsize@4 5f5b3a44     oleaut32:OLEAUT32.dll
 0003:00002a48       __imp__VariantClear@4      5f5b3a48     oleaut32:OLEAUT32.dll
 0003:00002a4c       __imp__VariantCopy@8       5f5b3a4c     oleaut32:OLEAUT32.dll
 0003:00002a50       __imp__SafeArrayAccessData@8 5f5b3a50     oleaut32:OLEAUT32.dll
 0003:00002a54       __imp__SysAllocString@4    5f5b3a54     oleaut32:OLEAUT32.dll
 0003:00002a58       __imp__SysFreeString@4     5f5b3a58     oleaut32:OLEAUT32.dll
 0003:00002a5c       __imp__SysReAllocStringLen@12 5f5b3a5c     oleaut32:OLEAUT32.dll
 0003:00002a60       __imp__SysAllocStringLen@8 5f5b3a60     oleaut32:OLEAUT32.dll
 0003:00002a64       __imp__VariantChangeType@16 5f5b3a64     oleaut32:OLEAUT32.dll
 0003:00002a68       \177OLEAUT32_NULL_THUNK_DATA_DLA 5f5b3a68     oleaut32:OLEAUT32.dll
 0003:00002a6c       __imp__OleCreateFontIndirect@12 5f5b3a6c     olepro32:OLEPRO32.DLL
 0003:00002a70       __imp__OleCreatePropertyFrame@44 5f5b3a70     olepro32:OLEPRO32.DLL
 0003:00002a74       __imp__OleLoadPicture@20   5f5b3a74     olepro32:OLEPRO32.DLL
 0003:00002a78       __imp__OleTranslateColor@12 5f5b3a78     olepro32:OLEPRO32.DLL
 0003:00002a7c       __imp__OleCreatePictureIndirect@16 5f5b3a7c     olepro32:OLEPRO32.DLL
 0003:00002a80       \177OLEPRO32_NULL_THUNK_DATA_DLA 5f5b3a80     olepro32:OLEPRO32.DLL
 0003:00002a84       __imp__ExtractIconA@12     5f5b3a84     shell32:SHELL32.dll
 0003:00002a88       __imp__DragFinish@4        5f5b3a88     shell32:SHELL32.dll
 0003:00002a8c       __imp__DragQueryFileA@16   5f5b3a8c     shell32:SHELL32.dll
 0003:00002a90       \177SHELL32_NULL_THUNK_DATA_DLA 5f5b3a90     shell32:SHELL32.dll
 0003:00002a94       __imp__ReadFmtUserTypeStg@12 5f5b3a94     ole32:ole32.dll
 0003:00002a98       __imp__CreateFileMoniker@8 5f5b3a98     ole32:ole32.dll
 0003:00002a9c       __imp__CoGetMalloc@8       5f5b3a9c     ole32:ole32.dll
 0003:00002aa0       __imp__StgCreateDocfile@16 5f5b3aa0     ole32:ole32.dll
 0003:00002aa4       __imp__StgOpenStorage@24   5f5b3aa4     ole32:ole32.dll
 0003:00002aa8       __imp__OleRegGetUserType@12 5f5b3aa8     ole32:ole32.dll
 0003:00002aac       __imp__GetClassFile@8      5f5b3aac     ole32:ole32.dll
 0003:00002ab0       __imp__ReadClassStg@8      5f5b3ab0     ole32:ole32.dll
 0003:00002ab4       __imp__StgIsStorageFile@4  5f5b3ab4     ole32:ole32.dll
 0003:00002ab8       __imp__CoLockObjectExternal@12 5f5b3ab8     ole32:ole32.dll
 0003:00002abc       __imp__RevokeDragDrop@4    5f5b3abc     ole32:ole32.dll
 0003:00002ac0       __imp__CoRegisterMessageFilter@8 5f5b3ac0     ole32:ole32.dll
 0003:00002ac4       __imp__CoRegisterClassObject@20 5f5b3ac4     ole32:ole32.dll
 0003:00002ac8       __imp__CoRevokeClassObject@4 5f5b3ac8     ole32:ole32.dll
 0003:00002acc       __imp__OleTranslateAccelerator@12 5f5b3acc     ole32:ole32.dll
 0003:00002ad0       __imp__IsAccelerator@16    5f5b3ad0     ole32:ole32.dll
 0003:00002ad4       __imp__CoCreateInstance@20 5f5b3ad4     ole32:ole32.dll
 0003:00002ad8       __imp__OleDestroyMenuDescriptor@4 5f5b3ad8     ole32:ole32.dll
 0003:00002adc       __imp__GetRunningObjectTable@8 5f5b3adc     ole32:ole32.dll
 0003:00002ae0       __imp__WriteClassStg@8     5f5b3ae0     ole32:ole32.dll
 0003:00002ae4       __imp__OleDuplicateData@12 5f5b3ae4     ole32:ole32.dll
 0003:00002ae8       __imp__SetConvertStg@8     5f5b3ae8     ole32:ole32.dll
 0003:00002aec       __imp__WriteFmtUserTypeStg@12 5f5b3aec     ole32:ole32.dll
 0003:00002af0       __imp__CoTreatAsClass@8    5f5b3af0     ole32:ole32.dll
 0003:00002af4       __imp__CoDisconnectObject@8 5f5b3af4     ole32:ole32.dll
 0003:00002af8       __imp__OleRegEnumVerbs@8   5f5b3af8     ole32:ole32.dll
 0003:00002afc       __imp__OleRegGetMiscStatus@12 5f5b3afc     ole32:ole32.dll
 0003:00002b00       __imp__CreateOleAdviseHolder@4 5f5b3b00     ole32:ole32.dll
 0003:00002b04       __imp__CreateDataAdviseHolder@4 5f5b3b04     ole32:ole32.dll
 0003:00002b08       __imp__CoGetClassObject@20 5f5b3b08     ole32:ole32.dll
 0003:00002b0c       __imp__StringFromGUID2@12  5f5b3b0c     ole32:ole32.dll
 0003:00002b10       __imp__CreateDataCache@16  5f5b3b10     ole32:ole32.dll
 0003:00002b14       __imp__ReadClassStm@8      5f5b3b14     ole32:ole32.dll
 0003:00002b18       __imp__OleLoadFromStream@12 5f5b3b18     ole32:ole32.dll
 0003:00002b1c       __imp__CLSIDFromString@8   5f5b3b1c     ole32:ole32.dll
 0003:00002b20       __imp__CLSIDFromProgID@8   5f5b3b20     ole32:ole32.dll
 0003:00002b24       __imp__CreateBindCtx@8     5f5b3b24     ole32:ole32.dll
 0003:00002b28       __imp__OleSetClipboard@4   5f5b3b28     ole32:ole32.dll
 0003:00002b2c       __imp__OleIsCurrentClipboard@4 5f5b3b2c     ole32:ole32.dll
 0003:00002b30       __imp__OleGetClipboard@4   5f5b3b30     ole32:ole32.dll
 0003:00002b34       __imp__CoTaskMemAlloc@4    5f5b3b34     ole32:ole32.dll
 0003:00002b38       __imp__OleRun@4            5f5b3b38     ole32:ole32.dll
 0003:00002b3c       __imp__OleQueryLinkFromData@4 5f5b3b3c     ole32:ole32.dll
 0003:00002b40       __imp__OleQueryCreateFromData@4 5f5b3b40     ole32:ole32.dll
 0003:00002b44       __imp__OleSetMenuDescriptor@20 5f5b3b44     ole32:ole32.dll
 0003:00002b48       __imp__OleIsRunning@4      5f5b3b48     ole32:ole32.dll
 0003:00002b4c       __imp__CreateItemMoniker@12 5f5b3b4c     ole32:ole32.dll
 0003:00002b50       __imp__CreateGenericComposite@12 5f5b3b50     ole32:ole32.dll
 0003:00002b54       __imp__CreateStreamOnHGlobal@12 5f5b3b54     ole32:ole32.dll
 0003:00002b58       __imp__OleSaveToStream@8   5f5b3b58     ole32:ole32.dll
 0003:00002b5c       __imp__WriteClassStm@8     5f5b3b5c     ole32:ole32.dll
 0003:00002b60       __imp__OleGetIconOfClass@12 5f5b3b60     ole32:ole32.dll
 0003:00002b64       __imp__ReleaseStgMedium@4  5f5b3b64     ole32:ole32.dll
 0003:00002b68       __imp__GetHGlobalFromILockBytes@8 5f5b3b68     ole32:ole32.dll
 0003:00002b6c       __imp__StgIsStorageILockBytes@4 5f5b3b6c     ole32:ole32.dll
 0003:00002b70       __imp__StgOpenStorageOnILockBytes@24 5f5b3b70     ole32:ole32.dll
 0003:00002b74       __imp__CreateILockBytesOnHGlobal@12 5f5b3b74     ole32:ole32.dll
 0003:00002b78       __imp__StgCreateDocfileOnILockBytes@16 5f5b3b78     ole32:ole32.dll
 0003:00002b7c       __imp__OleSave@12          5f5b3b7c     ole32:ole32.dll
 0003:00002b80       __imp__OleLoad@16          5f5b3b80     ole32:ole32.dll
 0003:00002b84       __imp__OleCreate@28        5f5b3b84     ole32:ole32.dll
 0003:00002b88       __imp__OleCreateLinkToFile@28 5f5b3b88     ole32:ole32.dll
 0003:00002b8c       __imp__OleCreateFromFile@32 5f5b3b8c     ole32:ole32.dll
 0003:00002b90       __imp__OleCreateStaticFromData@28 5f5b3b90     ole32:ole32.dll
 0003:00002b94       __imp__OleCreateLinkFromData@28 5f5b3b94     ole32:ole32.dll
 0003:00002b98       __imp__OleCreateFromData@28 5f5b3b98     ole32:ole32.dll
 0003:00002b9c       __imp__OleSetContainedObject@8 5f5b3b9c     ole32:ole32.dll
 0003:00002ba0       __imp__StringFromCLSID@8   5f5b3ba0     ole32:ole32.dll
 0003:00002ba4       __imp__CoTaskMemFree@4     5f5b3ba4     ole32:ole32.dll
 0003:00002ba8       __imp__OleLockRunning@12   5f5b3ba8     ole32:ole32.dll
 0003:00002bac       __imp__CoFreeUnusedLibraries@0 5f5b3bac     ole32:ole32.dll
 0003:00002bb0       __imp__OleUninitialize@0   5f5b3bb0     ole32:ole32.dll
 0003:00002bb4       __imp__OleInitialize@4     5f5b3bb4     ole32:ole32.dll
 0003:00002bb8       __imp__OleFlushClipboard@0 5f5b3bb8     ole32:ole32.dll
 0003:00002bbc       __imp__DoDragDrop@16       5f5b3bbc     ole32:ole32.dll
 0003:00002bc0       __imp__RegisterDragDrop@8  5f5b3bc0     ole32:ole32.dll
 0003:00002bc4       __imp__OleCreateMenuDescriptor@8 5f5b3bc4     ole32:ole32.dll
 0003:00002bc8       \177ole32_NULL_THUNK_DATA_DLA 5f5b3bc8     ole32:ole32.dll
 0003:00002bcc       __imp__OleUIInsertObjectA@4 5f5b3bcc     oledlg:oledlg.dll
 0003:00002bd0       __imp__OleUIUpdateLinksA@16 5f5b3bd0     oledlg:oledlg.dll
 0003:00002bd4       __imp__OleUIPasteSpecialA@4 5f5b3bd4     oledlg:oledlg.dll
 0003:00002bd8       __imp__OleUIBusyA@4        5f5b3bd8     oledlg:oledlg.dll
 0003:00002bdc       __imp__OleUIObjectPropertiesA@4 5f5b3bdc     oledlg:oledlg.dll
 0003:00002be0       __imp__OleUIChangeSourceA@4 5f5b3be0     oledlg:oledlg.dll
 0003:00002be4       __imp__OleUIAddVerbMenuA@36 5f5b3be4     oledlg:oledlg.dll
 0003:00002be8       __imp__OleUIEditLinksA@4   5f5b3be8     oledlg:oledlg.dll
 0003:00002bec       __imp__OleUIChangeIconA@4  5f5b3bec     oledlg:oledlg.dll
 0003:00002bf0       __imp__OleUIConvertA@4     5f5b3bf0     oledlg:oledlg.dll
 0003:00002bf4       \177oledlg_NULL_THUNK_DATA_DLA 5f5b3bf4     oledlg:oledlg.dll
 0003:00002bf8       __imp__IsAsyncMoniker@4    5f5b3bf8     urlmon:urlmon.dll
 0003:00002bfc       __imp__RegisterBindStatusCallback@16 5f5b3bfc     urlmon:urlmon.dll
 0003:00002c00       __imp__CreateAsyncBindCtx@16 5f5b3c00     urlmon:urlmon.dll
 0003:00002c04       __imp__CreateURLMoniker@12 5f5b3c04     urlmon:urlmon.dll
 0003:00002c08       \177urlmon_NULL_THUNK_DATA_DLA 5f5b3c08     urlmon:urlmon.dll
 0003:00002c10       ?ATL_CREATE_OBJECT@CComApartment@ATL@@2IA 5f5b3c10     dllole.obj
 0003:00002c18       ?m_libid@CComModule@ATL@@2U_GUID@@A 5f5b3c18     dllole.obj
 0003:00002c28       ?_pModule@ATL@@3PAVCComModule@1@A 5f5b3c28     dllole.obj
 0003:00003cd8       ?_afxOleWinApp@@3VCWinApp@@A 5f5b4cd8     dllole.obj
 0003:00003da0       ?_afxInitOleDllState@@3V_AFX_INIT_OLE_DLL_STATE@@A 5f5b4da0     dllole.obj
 0003:00003da4       ?_afxTickInit@@3HA         5f5b4da4     oleinit.obj
 0003:00003da8       ?_oleData@@3UOLE_DATA@@A   5f5b4da8     oleinit.obj
 0003:00003de8       ?_afxOleState@@3V?$CProcessLocal@V_AFX_OLE_STATE@@@@A 5f5b4de8     oledata.obj
 0003:00003dec       ?_init_CDocItem@@3UAFX_CLASSINIT@@A 5f5b4dec     oledoc1.obj
 0003:00003df4       ?nDragDelay@COleDropSource@@1IA 5f5b4df4     oledrop1.obj
 0003:00003df8       ?nDragMinDist@COleDropSource@@1IA 5f5b4df8     oledrop1.obj
 0003:00003e00       ?nScrollInterval@COleDropTarget@@1IA 5f5b4e00     oledrop2.obj
 0003:00003e04       ?nScrollDelay@COleDropTarget@@1IA 5f5b4e04     oledrop2.obj
 0003:00003e08       ?nScrollInset@COleDropTarget@@1HA 5f5b4e08     oledrop2.obj
 0003:00003edc       ?_init_CRichEditCntrItem@@3UAFX_CLASSINIT@@A 5f5b4edc     viewrich.obj
 0003:00003ee0       ?_afxMsgFindReplace2@@3IB  5f5b4ee0     viewrich.obj
 0003:00003ee4       ?_afxOccManager@@3V?$CProcessLocal@VCOccManager@@@@A 5f5b4ee4     occmgr.obj
 0003:00003f38       ?_afxLargeZero@@3T_LARGE_INTEGER@@A 5f5b4f38     ctlpset.obj
 0003:00003f40       ?_afxAmbientCache@@3V?$CThreadLocal@V_AFXCTL_AMBIENT_CACHE@@@@A 5f5b4f40     ctlquick.obj
 0003:00003f50       ?factory@CColorPropPage@@1VCColorPropPageFactory@1@A 5f5b4f50     ppgcolor.obj
 0003:00003f9c       ?hPal@@3PAUHPALETTE__@@A   5f5b4f9c     ppgcolor.obj
 0003:00003fa0       ?idClicked@CColorButton@@2IA 5f5b4fa0     ppgcolor.obj
 0003:00003fb0       ?factory@CFontPropPage@@1VCFontPropPageFactory@1@A 5f5b4fb0     ppgfont.obj
 0003:00004008       ?factory@CPicturePropPage@@1VCPicturePropPageFactory@1@A 5f5b5008     ppgpict.obj
 0003:00004058       __hmod__OLEPRO32           5f5b5058     olepro32:OLEPRO32.DLL
 0003:0000405c       __hmod__ADVAPI32           5f5b505c     advapi32:ADVAPI32.dll
 0003:00004060       __hmod__OLE32              5f5b5060     ole32:ole32.dll
 0003:00004064       __hmod__OLEAUT32           5f5b5064     oleaut32:OLEAUT32.dll
 0003:00004068       __hmod__OLEDLG             5f5b5068     oledlg:oledlg.dll
 0003:0000406c       __hmod__URLMON             5f5b506c     urlmon:urlmon.dll
 0003:00004070       __hmod__SHELL32            5f5b5070     shell32:SHELL32.dll
 0003:00004074       ___puiHead                 5f5b5074     delayimp:delayhlp.obj
 0003:00004078       ___pfnDliFailureHook       5f5b5078     delayimp:delayhk1.obj
 0003:0000407c       ___pfnDliNotifyHook        5f5b507c     delayimp:delayhk2.obj
 0003:00004080       __adjust_fdiv              5f5b5080     <common>
 0003:00004084       ___onexitend               5f5b5084     <common>
 0003:00004088       ___onexitbegin             5f5b5088     <common>

 entry point at        0001:0004ba70

 Static symbols

 0001:0004910b       _$E376                     5f54a10b f   ppgpict.obj
 0001:0004911a       _$E372                     5f54a11a f   ppgpict.obj
 0001:0004913a       _$E375                     5f54a13a f   ppgpict.obj
 0001:0004914c       _$E373                     5f54a14c f   ppgpict.obj
 0001:00047c02       _$E376                     5f548c02 f   ppgfont.obj
 0001:00047c11       _$E372                     5f548c11 f   ppgfont.obj
 0001:00047c31       _$E375                     5f548c31 f   ppgfont.obj
 0001:00047c43       _$E373                     5f548c43 f   ppgfont.obj
 0001:00045161       _$E376                     5f546161 f   ppgcolor.obj
 0001:00045170       _$E372                     5f546170 f   ppgcolor.obj
 0001:00045190       _$E375                     5f546190 f   ppgcolor.obj
 0001:000451a2       _$E373                     5f5461a2 f   ppgcolor.obj
 0001:00042890       _$E375                     5f543890 f   ctlquick.obj
 0001:0004289f       _$E372                     5f54389f f   ctlquick.obj
 0001:000428a4       _$E374                     5f5438a4 f   ctlquick.obj
 0001:000428b6       _$E373                     5f5438b6 f   ctlquick.obj
 0001:0003101b       _$E373                     5f53201b f   ctlppg.obj
 0001:00034bfa       _$E375                     5f535bfa f   ctlppg.obj
 0001:0001aef7       ?HasChildStyle@@YAHPAVCWnd@@@Z 5f51bef7 f   occdlg.obj
 0001:0001af19       ?TestStyle@@YAKPAVCWnd@@K@Z 5f51bf19 f   occdlg.obj
 0001:0001af30       ?IsControlParent@@YAHPAVCWnd@@@Z 5f51bf30 f   occdlg.obj
 0001:0001af46       ?TestExStyle@@YAKPAVCWnd@@K@Z 5f51bf46 f   occdlg.obj
 0001:0001aab1       ?DDX_OCPropertyRO@@YAXPAVCDataExchange@@HJGPAX@Z 5f51bab1 f   occddx.obj
 0001:0000c790       _$E383                     5f50d790 f   occmgr.obj
 0001:0000c79f       _$E380                     5f50d79f f   occmgr.obj
 0001:0000c7a4       _$E382                     5f50d7a4 f   occmgr.obj
 0001:0000c7b6       _$E381                     5f50d7b6 f   occmgr.obj
 0001:0000c8f9       ?IsDialogEx@@YAHPBUDLGTEMPLATE@@@Z 5f50d8f9 f   occmgr.obj
 0001:0000cb73       ?DlgTemplateItemCount@@YAABGPBUDLGTEMPLATE@@@Z 5f50db73 f   occmgr.obj
 0001:0000ce13       ?DlgTemplateItemCount@@YAAAGPAUDLGTEMPLATE@@@Z 5f50de13 f   occmgr.obj
 0001:0004ce51       _$E373                     5f54de51 f   viewrich.obj
 0001:0004ce5b       _$E372                     5f54de5b f   viewrich.obj
 0001:00053ecf       _$E376                     5f554ecf f   viewrich.obj
 0001:00053ed9       _$E375                     5f554ed9 f   viewrich.obj
 0001:00053628       _$E373                     5f554628 f   oledoc1.obj
 0001:00053632       _$E372                     5f554632 f   oledoc1.obj
 0001:000534fb       _$E375                     5f5544fb f   oledata.obj
 0001:0005350a       _$E372                     5f55450a f   oledata.obj
 0001:0005350f       _$E374                     5f55450f f   oledata.obj
 0001:00053521       _$E373                     5f554521 f   oledata.obj
 0001:00055566       ?AfxGetIconInfo@@YAXPBDPADAAI@Z 5f556566 f   olecli1.obj
 0001:00052860       _$E373                     5f553860 f   oleinit.obj
 0001:0005286a       _$E372                     5f55386a f   oleinit.obj
 0001:0005270d       _$E375                     5f55370d f   dllole.obj
 0001:0005271c       _$E372                     5f55371c f   dllole.obj
 0001:0005272d       _$E374                     5f55372d f   dllole.obj
 0001:0005273f       _$E373                     5f55373f f   dllole.obj
 0001:000527d2       _$E380                     5f5537d2 f   dllole.obj
 0001:000527e1       _$E377                     5f5537e1 f   dllole.obj
 0001:000527fe       _$E379                     5f5537fe f   dllole.obj
 0001:00052810       _$E378                     5f553810 f   dllole.obj
 0001:0005281f       _$E385                     5f55381f f   dllole.obj
 0001:0005282e       _$E382                     5f55382e f   dllole.obj
 0001:00052833       _$E384                     5f553833 f   dllole.obj
 0001:00052845       _$E383                     5f553845 f   dllole.obj
 0001:00087850       ?_AfxForceVectorDelete@@YAXXZ 5f588850 f   dllole.obj
 0001:0004b850       _$$$00001                  5f54c850 f   msvcrtd:chkstk.obj
 0001:0004b85c       probepages                 5f54c85c f   msvcrtd:chkstk.obj
 0001:0004b870       lastpage                   5f54c870 f   msvcrtd:chkstk.obj
 0001:0004b7b0       ?ArrayUnwindFilter@@YAHPAU_EXCEPTION_POINTERS@@@Z 5f54c7b0 f   msvcrtd:ehvecdtr.obj
 0001:0004cc05       ?OverlayIAT@@YGXPAU_IMAGE_THUNK_DATA32@@PBU1@@Z 5f54dc05 f   delayimp:delayhlp.obj

 5087 bytes saved through ICF

